 CANTest_slrt

 Timestamp is 64acc4d1 (Tue Jul 11 11:56:17 2023)

 Preferred load address is 10000000

 Start         Length     Name                   Class
 0001:00000000 00001a3aH .text$di                CODE
 0001:00001a40 000f9467H .text$mn                CODE
 0001:000faeb0 00004cc4H .text$x                 CODE
 0001:000ffb80 00001610H .text$yd                CODE
 0002:00000000 00000104H .CRT$XCA                DATA
 0002:00000104 00000121H .CRT$XCC                DATA
 0002:00000228 00000109H .CRT$XCL                DATA
 0002:00000334 00000156H .CRT$XCU                DATA
 0002:0000048c 00000104H .CRT$XCZ                DATA
 0002:00000590 00000104H .CRT$XIA                DATA
 0002:00000694 00000118H .CRT$XIC                DATA
 0002:000007ac 00000104H .CRT$XIZ                DATA
 0002:000008b0 00000104H .CRT$XPA                DATA
 0002:000009b4 00000109H .CRT$XPX                DATA
 0002:00000ac0 00000104H .CRT$XPXA               DATA
 0002:00000bc4 00000104H .CRT$XPZ                DATA
 0002:00000cc8 00000104H .CRT$XTA                DATA
 0002:00000dcc 00000104H .CRT$XTZ                DATA
 0002:00000ed0 00038497H .rdata                  DATA
 0002:00039368 000001b1H .rdata$debug            DATA
 0002:0003951c 000022c4H .rdata$r                DATA
 0002:0003b7e0 000005beH .rdata$sxdata           DATA
 0002:0003bda0 00000104H .rtc$IAA                DATA
 0002:0003bea4 00000104H .rtc$IZZ                DATA
 0002:0003bfa8 00000104H .rtc$TAA                DATA
 0002:0003c0ac 00000104H .rtc$TZZ                DATA
 0002:0003c1b0 000055feH .xdata$x                DATA
 0002:000417b0 000001ffH .edata                  DATA
 0003:00000000 00002623H .data                   DATA
 0003:00002628 000013baH .data$r                 DATA
 0003:00003a00 00015b64H .bss                    DATA
 0004:00000000 000001e8H .idata$5                DATA
 0004:000001e8 00000014H .idata$2                DATA
 0004:000001fc 00000014H .idata$3                DATA
 0004:00000210 000001e8H .idata$4                DATA
 0004:000003f8 00000871H .idata$6                DATA

  Address         Publics by Value              Rva+Base       Lib:Object

 0000:00000000       ___guard_fids_count        00000000     <absolute>
 0000:00000000       __except_list              00000000     <absolute>
 0000:00000000       ___guard_flags             00000000     <absolute>
 0000:00000000       ___guard_fids_table        00000000     <absolute>
 0000:000000fd       ___safe_se_handler_count   000000fd     <absolute>
 0000:00000000       ___ImageBase               10000000     <linker-defined>
 0001:00001a40       _CANTest_ChangeStepSize    10002a40 f   xpctarget.obj
 0001:00001a90       _DllMain@12                10002a90 f   xpctarget.obj
 0001:00001aa0       _SLRTSetErrorStatus        10002aa0 f   xpctarget.obj
 0001:00001ac0       _changeStepSize            10002ac0 f   xpctarget.obj
 0001:00001b10       _getDLMVersion             10002b10 f   xpctarget.obj
 0001:00001b20       _getFullPathToRefMdl       10002b20 f   xpctarget.obj
 0001:00001bd0       _getRefMdlPath             10002bd0 f   xpctarget.obj
 0001:00001c50       _getRefMdlSignalNumber     10002c50 f   xpctarget.obj
 0001:00001d00       _getrlmdlinfo              10002d00 f   xpctarget.obj
 0001:00001e60       _slrtRegisterSignalToLoggingService 10002e60 f   xpctarget.obj
 0001:00001fb0       _updateDiscreteEvents      10002fb0 f   xpctarget.obj
 0001:00001fc0       _getNumRef                 10002fc0 f   appmappingData.obj
 0001:00001fd0       _rt_mxCreateCharMatrixFromStrings 10002fd0 f   rt_matrx.obj
 0001:00002120       _rt_mxCreateDoubleMatrix   10003120 f   rt_matrx.obj
 0001:00002180       _rt_mxCreateNumericArray   10003180 f   rt_matrx.obj
 0001:00002200       _rt_mxCreateString         10003200 f   rt_matrx.obj
 0001:00002290       _rt_mxDuplicateArray       10003290 f   rt_matrx.obj
 0001:000022f0       _rt_mxGetDimensions        100032f0 f   rt_matrx.obj
 0001:00002330       _rt_mxGetEps               10003330 f   rt_matrx.obj
 0001:00002340       _rt_mxGetString            10003340 f   rt_matrx.obj
 0001:000023c0       _rtPrintfNoOp              100033c0 f   rt_printf.obj
 0001:00002ce0       _rt_CreateLogVar           10003ce0 f   rt_logging.obj
 0001:00002d70       _rt_CreateLogVarWithConvert 10003d70 f   rt_logging.obj
 0001:000036f0       _rt_CreateStructLogVar     100046f0 f   rt_logging.obj
 0001:00004460       _rt_GetMxIdFromDTypeId     10005460 f   rt_logging.obj
 0001:00004490       _rt_GetMxIdFromDTypeIdForRSim 10005490 f   rt_logging.obj
 0001:00006de0       _rt_StartDataLogging       10007de0 f   rt_logging.obj
 0001:000072a0       _rt_StartDataLoggingWithStartTime 100082a0 f   rt_logging.obj
 0001:00007c10       _rt_StopDataLogging        10008c10 f   rt_logging.obj
 0001:00007c30       _rt_StopDataLoggingImpl    10008c30 f   rt_logging.obj
 0001:00007f70       _rt_UpdateLogVar           10008f70 f   rt_logging.obj
 0001:000093e0       _rt_UpdateStructLogVar     1000a3e0 f   rt_logging.obj
 0001:00009470       _rt_UpdateTXXFYLogVars     1000a470 f   rt_logging.obj
 0001:00009a50       _rt_UpdateTXYLogVars       1000aa50 f   rt_logging.obj
 0001:00009ca0       _rt_getTempMemory          1000aca0 f   rt_logging.obj
 0001:00009ce0       _CANTest                   1000ace0 f   CANTest.obj
 0001:0000b660       _MdlInitialize             1000c660 f   CANTest.obj
 0001:0000b670       _MdlInitializeSampleTimes  1000c670 f   CANTest.obj
 0001:0000b680       _MdlInitializeSizes        1000c680 f   CANTest.obj
 0001:0000b690       _MdlOutputs                1000c690 f   CANTest.obj
 0001:0000b6a0       _MdlStart                  1000c6a0 f   CANTest.obj
 0001:0000b6b0       _MdlTerminate              1000c6b0 f   CANTest.obj
 0001:0000b700       _MdlUpdate                 1000c700 f   CANTest.obj
 0001:0000b710       _CANTest_GetCAPIStaticMap  1000c710 f   CANTest_capi.obj
 0001:0000b720       _CANTest_InitializeDataMapInfo 1000c720 f   CANTest_capi.obj
 0001:0000b7f0       _mdlXcp_GetMdlXcpInfo      1000c7f0 f   CANTest_xcp.obj
 0001:0000b800       _SLRT_update_TET           1000c800 f   CANTest_xcp_TET.obj
 0001:0000b8d0       _rtGetInf                  1000c8d0 f   rtGetInf.obj
 0001:0000b900       _rtGetInfF                 1000c900 f   rtGetInf.obj
 0001:0000b920       _rtGetMinusInf             1000c920 f   rtGetInf.obj
 0001:0000b950       _rtGetMinusInfF            1000c950 f   rtGetInf.obj
 0001:0000b970       _rtGetNaN                  1000c970 f   rtGetNaN.obj
 0001:0000b9a0       _rtGetNaNF                 1000c9a0 f   rtGetNaN.obj
 0001:0000b9c0       _rtIsInf                   1000c9c0 f   rt_nonfinite.obj
 0001:0000ba00       _rtIsInfF                  1000ca00 f   rt_nonfinite.obj
 0001:0000ba40       _rtIsNaN                   1000ca40 f   rt_nonfinite.obj
 0001:0000ba60       _rtIsNaNF                  1000ca60 f   rt_nonfinite.obj
 0001:0000ba80       _rt_InitInfAndNaN          1000ca80 f   rt_nonfinite.obj
 0001:0000bae0       _rt_CleanUpForStateLogWithMMI 1000cae0 f   rt_logging_mmi.obj
 0001:0000bbf0       _rt_FillStateSigInfoFromMMI 1000cbf0 f   rt_logging_mmi.obj
 0001:0000bfc0       _rtwCAPI_CountSysRan       1000cfc0 f   rtw_modelmap_utils.obj
 0001:0000c060       _rtwCAPI_EncodePath        1000d060 f   rtw_modelmap_utils.obj
 0001:0000c150       _rtwCAPI_FillSysRan        1000d150 f   rtw_modelmap_utils.obj
 0001:0000c240       _rtwCAPI_FreeFullPaths     1000d240 f   rtw_modelmap_utils.obj
 0001:0000c2d0       _rtwCAPI_GetFullStateBlockPath 1000d2d0 f   rtw_modelmap_utils.obj
 0001:0000c480       _rtwCAPI_GetNumContStateRecords 1000d480 f   rtw_modelmap_utils.obj
 0001:0000c540       _rtwCAPI_GetNumSigLogRecords 1000d540 f   rtw_modelmap_utils.obj
 0001:0000c590       _rtwCAPI_GetNumSigLogRecordsForRTWLogging 1000d590 f   rtw_modelmap_utils.obj
 0001:0000c620       _rtwCAPI_GetNumStateRecords 1000d620 f   rtw_modelmap_utils.obj
 0001:0000c670       _rtwCAPI_GetNumStateRecordsForRTWLogging 1000d670 f   rtw_modelmap_utils.obj
 0001:0000c700       _rtwCAPI_GetSigAddrFromMap 1000d700 f   rtw_modelmap_utils.obj
 0001:0000c7c0       _rtwCAPI_GetSigLogRecordInfo 1000d7c0 f   rtw_modelmap_utils.obj
 0001:0000cbf0       _rtwCAPI_GetStateRecordInfo 1000dbf0 f   rtw_modelmap_utils.obj
 0001:0000d0e0       _rtwCAPI_GetStateWidth     1000e0e0 f   rtw_modelmap_utils.obj
 0001:0000d140       _rtwCAPI_HasStates         1000e140 f   rtw_modelmap_utils.obj
 0001:0000d1b0       _rtwCAPI_UpdateFullPaths   1000e1b0 f   rtw_modelmap_utils.obj
 0001:0000d390       _timestamp_x86             1000e390 f   host_timer_x86.obj
 0001:0000d3a0       _taskTimeEnd               1000e3a0 f   xpc_code_profiling_utility_functions.obj
 0001:0000d3b0       _taskTimeEnd_              1000e3b0 f   xpc_code_profiling_utility_functions.obj
 0001:0000d3c0       _taskTimeStart             1000e3c0 f   xpc_code_profiling_utility_functions.obj
 0001:0000d3d0       _taskTimeStart_            1000e3d0 f   xpc_code_profiling_utility_functions.obj
 0001:0000d3e0       _xilProfilingTimerFreeze   1000e3e0 f   xpc_code_profiling_utility_functions.obj
 0001:0000d3f0       _xilProfilingTimerUnFreeze 1000e3f0 f   xpc_code_profiling_utility_functions.obj
 0001:0000d400       _xilUploadProfilingData    1000e400 f   xpc_code_profiling_utility_functions.obj
 0001:0000e0d0       _sg_IO613_setup_s          1000f0d0 f   sg_IO613_setup_s.obj
 0001:0000e120       ?CleanupOnError@@YAXHHPBD@Z 1000f120 f i sg_IO61X_read_s.obj
 0001:0000e8b0       _sg_IO61X_read_s           1000f8b0 f   sg_IO61X_read_s.obj
 0001:0000f200       _sg_IO61X_write_s          10010200 f   sg_IO61X_write_s.obj
 0001:0000f250       _GetPCIDeviceFull          10010250 f   xpcruntime:xpcimports.obj
 0001:0000f290       _GetPCIDeviceFunction      10010290 f   xpcruntime:xpcimports.obj
 0001:0000f2c0       _ShowPCIDevice             100102c0 f   xpcruntime:xpcimports.obj
 0001:0000f7d0       _slrtGetPciConfigAtFunction 100107d0 f   xpcruntime:xpcimports.obj
 0001:0000fab0       _xpcGetPciConfigAtSlot     10010ab0 f   xpcruntime:xpcimports.obj
 0001:0000fad0       _xpcInitProcs              10010ad0 f   xpcruntime:xpcimports.obj
 0001:00010cd0       _xpceuploadevent           10011cd0 f   xpcruntime:xpcimports.obj
 0001:00010ce0       _sg_module_alloc_custom_data 10011ce0 f   libsg_MSVC120_vc:sg_module_registry.obj
 0001:00010d00       _sg_module_get             10011d00 f   libsg_MSVC120_vc:sg_module_registry.obj
 0001:00010d90       _sg_module_register        10011d90 f   libsg_MSVC120_vc:sg_module_registry.obj
 0001:00010e20       _sg_module_unregister      10011e20 f   libsg_MSVC120_vc:sg_module_registry.obj
 0001:00010e90       ??$_Allocate@D@std@@YAPADIPAD@Z 10011e90 f i IO61X_Library_MSVC120_vc:IO61X_iConcurrentExecution.obj
 0001:00010ec0       ??$addressof@D@std@@YAPADAAD@Z 10011ec0 f i IO61X_Library_MSVC120_vc:IO61X_iConcurrentExecution.obj
 0001:00010ed0       ??$construct@PADAAPAD@?$_Wrap_alloc@V?$allocator@D@std@@@std@@QAEXPAPADAAPAD@Z 10011ed0 f i IO61X_Library_MSVC120_vc:IO61X_iConcurrentExecution.obj
 0001:00010ef0       ??$construct@PADAAPAD@?$allocator@D@std@@QAEXPAPADAAPAD@Z 10011ef0 f i IO61X_Library_MSVC120_vc:IO61X_iConcurrentExecution.obj
 0001:00010f10       ??$construct@PADAAPAD@?$allocator_traits@V?$allocator@D@std@@@std@@SAXAAV?$allocator@D@1@PAPADAAPAD@Z 10011f10 f i IO61X_Library_MSVC120_vc:IO61X_iConcurrentExecution.obj
 0001:00010f30       ??$destroy@PAD@?$_Wrap_alloc@V?$allocator@D@std@@@std@@QAEXPAPAD@Z 10011f30 f i IO61X_Library_MSVC120_vc:IO61X_iConcurrentExecution.obj
 0001:00010f40       ??$destroy@PAD@?$allocator@D@std@@QAEXPAPAD@Z 10011f40 f i IO61X_Library_MSVC120_vc:IO61X_iConcurrentExecution.obj
 0001:00010f50       ??$destroy@PAD@?$allocator_traits@V?$allocator@D@std@@@std@@SAXAAV?$allocator@D@1@PAPAD@Z 10011f50 f i IO61X_Library_MSVC120_vc:IO61X_iConcurrentExecution.obj
 0001:00010f60       ??$forward@AAPAD@std@@YAAAPADAAPAD@Z 10011f60 f i IO61X_Library_MSVC120_vc:IO61X_iConcurrentExecution.obj
 0001:00010f70       ??0?$_String_alloc@$0A@U?$_String_base_types@DV?$allocator@D@std@@@std@@@std@@QAE@ABV?$allocator@D@1@@Z 10011f70 f i IO61X_Library_MSVC120_vc:IO61X_iConcurrentExecution.obj
 0001:00010f90       ??0?$_String_val@U?$_Simple_types@D@std@@@std@@QAE@XZ 10011f90 f i IO61X_Library_MSVC120_vc:IO61X_iConcurrentExecution.obj
 0001:00010fb0       ??0?$_Wrap_alloc@V?$allocator@D@std@@@std@@QAE@XZ 10011fb0 f i IO61X_Library_MSVC120_vc:IO61X_iConcurrentExecution.obj
 0001:00010fc0       ??0?$allocator@D@std@@QAE@XZ 10011fc0 f i IO61X_Library_MSVC120_vc:IO61X_iConcurrentExecution.obj
 0001:00010fd0       ??0?$atomic@H@std@@QAE@H@Z 10011fd0 f i IO61X_Library_MSVC120_vc:IO61X_iConcurrentExecution.obj
 0001:00010fe0       ??0?$basic_string@DU?$char_traits@D@std@@V?$allocator@D@2@@std@@QAE@PBD@Z 10011fe0 f i IO61X_Library_MSVC120_vc:IO61X_iConcurrentExecution.obj
 0001:00011040       ??0_Generic_error_category@std@@QAE@XZ 10012040 f i IO61X_Library_MSVC120_vc:IO61X_iConcurrentExecution.obj
 0001:00011050       ??0_Ignore@std@@QAE@XZ     10012050 f i IO61X_Library_MSVC120_vc:IO61X_iConcurrentExecution.obj
 0001:00011060       ??0_Iostream_error_category@std@@QAE@XZ 10012060 f i IO61X_Library_MSVC120_vc:IO61X_iConcurrentExecution.obj
 0001:00011070       ??0_System_error_category@std@@QAE@XZ 10012070 f i IO61X_Library_MSVC120_vc:IO61X_iConcurrentExecution.obj
 0001:00011080       ??0error_category@std@@QAE@XZ 10012080 f i IO61X_Library_MSVC120_vc:IO61X_iConcurrentExecution.obj
 0001:00011090       ??0error_condition@std@@QAE@HABVerror_category@1@@Z 10012090 f i IO61X_Library_MSVC120_vc:IO61X_iConcurrentExecution.obj
 0001:000110b0       ??1?$basic_string@DU?$char_traits@D@std@@V?$allocator@D@2@@std@@QAE@XZ 100120b0 f i IO61X_Library_MSVC120_vc:IO61X_iConcurrentExecution.obj
 0001:000110e0       ??1_Generic_error_category@std@@UAE@XZ 100120e0 f i IO61X_Library_MSVC120_vc:IO61X_iConcurrentExecution.obj
 0001:000110f0       ??1_Iostream_error_category@std@@UAE@XZ 100120f0 f i IO61X_Library_MSVC120_vc:IO61X_iConcurrentExecution.obj
 0001:00011100       ??1_System_error_category@std@@UAE@XZ 10012100 f i IO61X_Library_MSVC120_vc:IO61X_iConcurrentExecution.obj
 0001:00011110       ??1error_category@std@@UAE@XZ 10012110 f i IO61X_Library_MSVC120_vc:IO61X_iConcurrentExecution.obj
 0001:00011120       ??2@YAPAXIPAX@Z            10012120 f i IO61X_Library_MSVC120_vc:IO61X_iConcurrentExecution.obj
 0001:00011130       ??3@YAXPAX0@Z              10012130 f i IO61X_Library_MSVC120_vc:IO61X_iConcurrentExecution.obj
 0001:00011140       ??4atomic_int@std@@QAEHH@Z 10012140 f i IO61X_Library_MSVC120_vc:IO61X_iConcurrentExecution.obj
 0001:00011150       ??8error_category@std@@QBE_NABV01@@Z 10012150 f i IO61X_Library_MSVC120_vc:IO61X_iConcurrentExecution.obj
 0001:00011160       ??8error_condition@std@@QBE_NABV01@@Z 10012160 f i IO61X_Library_MSVC120_vc:IO61X_iConcurrentExecution.obj
 0001:00011180       ??_G_Generic_error_category@std@@UAEPAXI@Z 10012180 f i IO61X_Library_MSVC120_vc:IO61X_iConcurrentExecution.obj
 0001:00011180       ??_E_Generic_error_category@std@@UAEPAXI@Z 10012180 f i IO61X_Library_MSVC120_vc:IO61X_iConcurrentExecution.obj
 0001:000111b0       ??_G_Iostream_error_category@std@@UAEPAXI@Z 100121b0 f i IO61X_Library_MSVC120_vc:IO61X_iConcurrentExecution.obj
 0001:000111b0       ??_E_Iostream_error_category@std@@UAEPAXI@Z 100121b0 f i IO61X_Library_MSVC120_vc:IO61X_iConcurrentExecution.obj
 0001:000111e0       ??_E_System_error_category@std@@UAEPAXI@Z 100121e0 f i IO61X_Library_MSVC120_vc:IO61X_iConcurrentExecution.obj
 0001:000111e0       ??_G_System_error_category@std@@UAEPAXI@Z 100121e0 f i IO61X_Library_MSVC120_vc:IO61X_iConcurrentExecution.obj
 0001:00011210       ??_Gerror_category@std@@UAEPAXI@Z 10012210 f i IO61X_Library_MSVC120_vc:IO61X_iConcurrentExecution.obj
 0001:00011210       ??_Eerror_category@std@@UAEPAXI@Z 10012210 f i IO61X_Library_MSVC120_vc:IO61X_iConcurrentExecution.obj
 0001:00011240       ?CleanupOnError@@YAXHH@Z   10012240 f   IO61X_Library_MSVC120_vc:IO61X_iConcurrentExecution.obj
 0001:00011290       ?IO61X_ActivateBusRecovery@@YAEIEPAD@Z 10012290 f   IO61X_Library_MSVC120_vc:IO61X_iConcurrentExecution.obj
 0001:000112f0       ?IO61X_ActivateBusRecoveryThread@@YAXIEII@Z 100122f0 f   IO61X_Library_MSVC120_vc:IO61X_iConcurrentExecution.obj
 0001:00011360       ?IO61X_ActivateStatusHandling@@YAEIEEPAD@Z 10012360 f   IO61X_Library_MSVC120_vc:IO61X_iConcurrentExecution.obj
 0001:00011420       ?IO61X_CanFdCheckAndGetBaudrate@@YAHIEIPAD@Z 10012420 f   IO61X_Library_MSVC120_vc:IO61X_iConcurrentExecution.obj
 0001:000114d0       ?IO61X_CheckIsDriverInitialized@@YAEIPBDPAD@Z 100124d0 f   IO61X_Library_MSVC120_vc:IO61X_iConcurrentExecution.obj
 0001:00011500       ?IO61X_CheckIsModuleStatusReady@@YAEIPAD@Z 10012500 f   IO61X_Library_MSVC120_vc:IO61X_iConcurrentExecution.obj
 0001:00011530       ?IO61X_CheckLinDlcAndChecksum@@YAEIEEEPAD@Z 10012530 f   IO61X_Library_MSVC120_vc:IO61X_iConcurrentExecution.obj
 0001:000115d0       ?IO61X_ClearPortBuffer@@YAXI@Z 100125d0 f   IO61X_Library_MSVC120_vc:IO61X_iConcurrentExecution.obj
 0001:000116c0       ?IO61X_CreateDriverModuleList@@YAEIPBDPAD@Z 100126c0 f   IO61X_Library_MSVC120_vc:IO61X_iConcurrentExecution.obj
 0001:00011730       ?IO61X_CreatePort@@YAEIEEEEPAD@Z 10012730 f   IO61X_Library_MSVC120_vc:IO61X_iConcurrentExecution.obj
 0001:000118e0       ?IO61X_GetBlockBuffer_spin@@YAEIEEIPAPAXPAD@Z 100128e0 f   IO61X_Library_MSVC120_vc:IO61X_iConcurrentExecution.obj
 0001:00011970       ?IO61X_GetCANFDStatusBaudRatePrescalerByStatusBlock@@YAXIEPAI@Z 10012970 f   IO61X_Library_MSVC120_vc:IO61X_iConcurrentExecution.obj
 0001:000119a0       ?IO61X_GetCANFDStatusBitTimeSegment1ByStatusBlock@@YAXIEPAI@Z 100129a0 f   IO61X_Library_MSVC120_vc:IO61X_iConcurrentExecution.obj
 0001:000119d0       ?IO61X_GetCANFDStatusBitTimeSegment2ByStatusBlock@@YAXIEPAI@Z 100129d0 f   IO61X_Library_MSVC120_vc:IO61X_iConcurrentExecution.obj
 0001:00011a00       ?IO61X_GetCANFDStatusSynchronisationJumpWidthByStatusBlock@@YAXIEPAI@Z 10012a00 f   IO61X_Library_MSVC120_vc:IO61X_iConcurrentExecution.obj
 0001:00011a30       ?IO61X_GetCANFDStatusTimingModeByStatusBlock@@YAXIEPAI@Z 10012a30 f   IO61X_Library_MSVC120_vc:IO61X_iConcurrentExecution.obj
 0001:00011a60       ?IO61X_GetCANStatusBaudRatePrescalerByStatusBlock@@YAXIEPAI@Z 10012a60 f   IO61X_Library_MSVC120_vc:IO61X_iConcurrentExecution.obj
 0001:00011ab0       ?IO61X_GetCANStatusBitTimeSegment1ByStatusBlock@@YAXIEPAI@Z 10012ab0 f   IO61X_Library_MSVC120_vc:IO61X_iConcurrentExecution.obj
 0001:00011ae0       ?IO61X_GetCANStatusBitTimeSegment2ByStatusBlock@@YAXIEPAI@Z 10012ae0 f   IO61X_Library_MSVC120_vc:IO61X_iConcurrentExecution.obj
 0001:00011b10       ?IO61X_GetCANStatusSynchronisationJumpWidthByStatusBlock@@YAXIEPAI@Z 10012b10 f   IO61X_Library_MSVC120_vc:IO61X_iConcurrentExecution.obj
 0001:00011b40       ?IO61X_GetCANStatusTimingModeByStatusBlock@@YAXIEPAI@Z 10012b40 f   IO61X_Library_MSVC120_vc:IO61X_iConcurrentExecution.obj
 0001:00011b90       ?IO61X_GetCANStatusTransceiverDelayOffsetByStatusBlock@@YAXIEPAI@Z 10012b90 f   IO61X_Library_MSVC120_vc:IO61X_iConcurrentExecution.obj
 0001:00011bc0       ?IO61X_GetControllerStatus@@YAEI@Z 10012bc0 f   IO61X_Library_MSVC120_vc:IO61X_iConcurrentExecution.obj
 0001:00011d10       ?IO61X_GetLinMessageById@@YAEIEEPAULINMsg_T@@@Z 10012d10 f   IO61X_Library_MSVC120_vc:IO61X_iConcurrentExecution.obj
 0001:00011de0       ?IO61X_GetLinRawMessageById@@YAEIEEPAI00000PAE@Z 10012de0 f   IO61X_Library_MSVC120_vc:IO61X_iConcurrentExecution.obj
 0001:00011ec0       ?IO61X_GetModuleIndex@@YAEIPBDPAIPAD@Z 10012ec0 f   IO61X_Library_MSVC120_vc:IO61X_iConcurrentExecution.obj
 0001:00011f00       ?IO61X_GetModuleStatusInitialized@@YAHI@Z 10012f00 f   IO61X_Library_MSVC120_vc:IO61X_iConcurrentExecution.obj
 0001:00011f30       ?IO61X_GetReceivedMessageLin@@YAEIIEPAHPAI11PAE@Z 10012f30 f   IO61X_Library_MSVC120_vc:IO61X_iConcurrentExecution.obj
 0001:00011f80       ?IO61X_GetStatusBusCouplingErrorByStatusblock@@YAXIEPAI@Z 10012f80 f   IO61X_Library_MSVC120_vc:IO61X_iConcurrentExecution.obj
 0001:00011fc0       ?IO61X_GetStatusBusLoadByStatusBlock@@YAXIEPAI@Z 10012fc0 f   IO61X_Library_MSVC120_vc:IO61X_iConcurrentExecution.obj
 0001:00011ff0       ?IO61X_GetStatusBusOffByStatusblock@@YAXIEPAI@Z 10012ff0 f   IO61X_Library_MSVC120_vc:IO61X_iConcurrentExecution.obj
 0001:00012030       ?IO61X_GetStatusBusRecoveryCounterByStatusblock@@YAXIEPAI@Z 10013030 f   IO61X_Library_MSVC120_vc:IO61X_iConcurrentExecution.obj
 0001:00012060       ?IO61X_GetStatusDataOverrunByStatusblock@@YAXIEPAI@Z 10013060 f   IO61X_Library_MSVC120_vc:IO61X_iConcurrentExecution.obj
 0001:000120a0       ?IO61X_GetStatusErrorWarningByStatusblock@@YAXIEPAI@Z 100130a0 f   IO61X_Library_MSVC120_vc:IO61X_iConcurrentExecution.obj
 0001:000120e0       ?IO61X_GetStatusExtendedOperatingModeByStatusBlock@@YAXIEPAI@Z 100130e0 f   IO61X_Library_MSVC120_vc:IO61X_iConcurrentExecution.obj
 0001:00012110       ?IO61X_GetStatusInitModeByStatusblock@@YAXIEPAI@Z 10013110 f   IO61X_Library_MSVC120_vc:IO61X_iConcurrentExecution.obj
 0001:00012150       ?IO61X_GetStatusOperatingModeByStatusBlock@@YAXIEPAI@Z 10013150 f   IO61X_Library_MSVC120_vc:IO61X_iConcurrentExecution.obj
 0001:00012180       ?IO61X_GetStatusPrioTransmissionPendingByStatusblock@@YAXIEPAI@Z 10013180 f   IO61X_Library_MSVC120_vc:IO61X_iConcurrentExecution.obj
 0001:000121c0       ?IO61X_GetStatusTransmissionPendingByStatusBlock@@YAXIEPAI@Z 100131c0 f   IO61X_Library_MSVC120_vc:IO61X_iConcurrentExecution.obj
 0001:00012200       ?IO61X_InitializeCanController@@YAEIEEEEGGGGGGGGNGIIIIPAD@Z 10013200 f   IO61X_Library_MSVC120_vc:IO61X_iConcurrentExecution.obj
 0001:000123a0       ?IO61X_InitializeLincotroller@@YAEIEEIEEEPAD@Z 100133a0 f   IO61X_Library_MSVC120_vc:IO61X_iConcurrentExecution.obj
 0001:000124e0       ?IO61X_InitializeModule@@YAEIEPBDFFPAIPAD@Z 100134e0 f   IO61X_Library_MSVC120_vc:IO61X_iConcurrentExecution.obj
 0001:00012550       ?IO61X_LINGetStatusBdr@@YAXIEPAX@Z 10013550 f   IO61X_Library_MSVC120_vc:IO61X_iConcurrentExecution.obj
 0001:00012580       ?IO61X_LINGetStatusBusLoad@@YAXIEPAX@Z 10013580 f   IO61X_Library_MSVC120_vc:IO61X_iConcurrentExecution.obj
 0001:000125b0       ?IO61X_LINGetStatusDataOvrn@@YAXIEPAX@Z 100135b0 f   IO61X_Library_MSVC120_vc:IO61X_iConcurrentExecution.obj
 0001:000125f0       ?IO61X_LINGetStatusInitAct@@YAXIEPAX@Z 100135f0 f   IO61X_Library_MSVC120_vc:IO61X_iConcurrentExecution.obj
 0001:00012630       ?IO61X_LINGetStatusOpMode@@YAXIEPAX@Z 10013630 f   IO61X_Library_MSVC120_vc:IO61X_iConcurrentExecution.obj
 0001:00012660       ?IO61X_LinRecMsg_spin@@YAEIENH@Z 10013660 f   IO61X_Library_MSVC120_vc:IO61X_iConcurrentExecution.obj
 0001:000126f0       ?IO61X_LinUpdateRwwbBuffer@@YAXIEEEEEE@Z 100136f0 f   IO61X_Library_MSVC120_vc:IO61X_iConcurrentExecution.obj
 0001:00012750       ?IO61X_PrintModuleInfo@@YAEIFFPBD@Z 10013750 f   IO61X_Library_MSVC120_vc:IO61X_iConcurrentExecution.obj
 0001:000128d0       ?IO61X_ReceiveCanAndCanRawMessage@@YAEIEEPAUCANMsg_T@@PAI11PANPAX@Z 100138d0 f   IO61X_Library_MSVC120_vc:IO61X_iConcurrentExecution.obj
 0001:00012930       ?IO61X_ReceiveCanFdAndCanFdRawMessage@@YAEIEPAXPAI111PAN0@Z 10013930 f   IO61X_Library_MSVC120_vc:IO61X_iConcurrentExecution.obj
 0001:000129a0       ?IO61X_ReceiveCanFdMessage@@YAEIEPAX@Z 100139a0 f   IO61X_Library_MSVC120_vc:IO61X_iConcurrentExecution.obj
 0001:00012b20       ?IO61X_ReceiveCanFdMessageRaw@@YAEIEPAI000PANPAX@Z 10013b20 f   IO61X_Library_MSVC120_vc:IO61X_iConcurrentExecution.obj
 0001:00012cd0       ?IO61X_ReceiveCanMessage@@YAEIEEPAUCANMsg_T@@@Z 10013cd0 f   IO61X_Library_MSVC120_vc:IO61X_iConcurrentExecution.obj
 0001:00012f50       ?IO61X_ReceiveCanRawMessage@@YAEIEEPAI00PANPAX@Z 10013f50 f   IO61X_Library_MSVC120_vc:IO61X_iConcurrentExecution.obj
 0001:00013000       ?IO61X_ReceiveLinMessage@@YAEIE@Z 10014000 f   IO61X_Library_MSVC120_vc:IO61X_iConcurrentExecution.obj
 0001:00013040       ?IO61X_ReleaseWriteSempahore@@YAXI@Z 10014040 f   IO61X_Library_MSVC120_vc:IO61X_iConcurrentExecution.obj
 0001:00013060       ?IO61X_SendCanFdMessage@@YAEIEPBX@Z 10014060 f   IO61X_Library_MSVC120_vc:IO61X_iConcurrentExecution.obj
 0001:00013170       ?IO61X_SendCanFdRawMessage@@YAEIEPBI000PBE@Z 10014170 f   IO61X_Library_MSVC120_vc:IO61X_iConcurrentExecution.obj
 0001:00013280       ?IO61X_SendCanMessage@@YAEIEEPBUCANMsg_T@@@Z 10014280 f   IO61X_Library_MSVC120_vc:IO61X_iConcurrentExecution.obj
 0001:000133c0       ?IO61X_SendLinMessage@@YAEIEPBULINMsg_T@@@Z 100143c0 f   IO61X_Library_MSVC120_vc:IO61X_iConcurrentExecution.obj
 0001:00013550       ?IO61X_SendLinRawMessage@@YAEIEPBE0000@Z 10014550 f   IO61X_Library_MSVC120_vc:IO61X_iConcurrentExecution.obj
 0001:00013710       ?IO61X_SetLinBuffer@@YAXIEEE@Z 10014710 f   IO61X_Library_MSVC120_vc:IO61X_iConcurrentExecution.obj
 0001:00013780       ?IO61X_SetLinMessageFilter@@YAXIEPBE000@Z 10014780 f   IO61X_Library_MSVC120_vc:IO61X_iConcurrentExecution.obj
 0001:00013930       ?IO61X_SetModuleStatusNotReady@@YAEI@Z 10014930 f   IO61X_Library_MSVC120_vc:IO61X_iConcurrentExecution.obj
 0001:00013970       ?IO61X_SetModuleStatusReady@@YAEIPAD@Z 10014970 f   IO61X_Library_MSVC120_vc:IO61X_iConcurrentExecution.obj
 0001:00013a30       ?IO61X_SetModuleStatusStartPorts@@YAEIPAD@Z 10014a30 f   IO61X_Library_MSVC120_vc:IO61X_iConcurrentExecution.obj
 0001:00013b00       ?IO61X_StartCanController@@YAEIEPAD@Z 10014b00 f   IO61X_Library_MSVC120_vc:IO61X_iConcurrentExecution.obj
 0001:00013bf0       ?IO61X_StartLinController@@YAEIEPAD@Z 10014bf0 f   IO61X_Library_MSVC120_vc:IO61X_iConcurrentExecution.obj
 0001:00013d00       ?IO61X_StopCanController@@YAEIE@Z 10014d00 f   IO61X_Library_MSVC120_vc:IO61X_iConcurrentExecution.obj
 0001:00013e50       ?IO61X_StopLinController@@YAEIE@Z 10014e50 f   IO61X_Library_MSVC120_vc:IO61X_iConcurrentExecution.obj
 0001:00013f40       ?IO61X_TargetDefaults@@YAXXZ 10014f40 f   IO61X_Library_MSVC120_vc:IO61X_iConcurrentExecution.obj
 0001:00013f50       ?IO61X_UpdateBuffer@@YACIEPAX0PAD@Z 10014f50 f   IO61X_Library_MSVC120_vc:IO61X_iConcurrentExecution.obj
 0001:00014050       ?IO6X_SetLinMessageQuantity@@YAXIEI@Z 10015050 f   IO61X_Library_MSVC120_vc:IO61X_iConcurrentExecution.obj
 0001:00014090       ?SendInitTermStructure@@YA_NI_NPBN@Z 10015090 f   IO61X_Library_MSVC120_vc:IO61X_iConcurrentExecution.obj
 0001:000142d0       ?_Atomic_load_8@std@@YA_KPC_KW4memory_order@1@@Z 100152d0 f i IO61X_Library_MSVC120_vc:IO61X_iConcurrentExecution.obj
 0001:00014320       ?_Atomic_store_4@std@@YAXPCKKW4memory_order@1@@Z 10015320 f i IO61X_Library_MSVC120_vc:IO61X_iConcurrentExecution.obj
 0001:00014350       ?_Atomic_store_8@std@@YAXPC_K_KW4memory_order@1@@Z 10015350 f i IO61X_Library_MSVC120_vc:IO61X_iConcurrentExecution.obj
 0001:00014380       ?_Copy@?$basic_string@DU?$char_traits@D@std@@V?$allocator@D@2@@std@@QAEXII@Z 10015380 f i IO61X_Library_MSVC120_vc:IO61X_iConcurrentExecution.obj
 0001:000144d0       ?_Eos@?$basic_string@DU?$char_traits@D@std@@V?$allocator@D@2@@std@@QAEXI@Z 100154d0 f i IO61X_Library_MSVC120_vc:IO61X_iConcurrentExecution.obj
 0001:00014500       ?_Getal@?$_String_alloc@$0A@U?$_String_base_types@DV?$allocator@D@std@@@std@@@std@@QBE?AU?$_Wrap_alloc@V?$allocator@D@std@@@2@XZ 10015500 f i IO61X_Library_MSVC120_vc:IO61X_iConcurrentExecution.obj
 0001:00014510       ?_Grow@?$basic_string@DU?$char_traits@D@std@@V?$allocator@D@2@@std@@QAE_NI_N@Z 10015510 f i IO61X_Library_MSVC120_vc:IO61X_iConcurrentExecution.obj
 0001:000145d0       ?_Inside@?$basic_string@DU?$char_traits@D@std@@V?$allocator@D@2@@std@@QAE_NPBD@Z 100155d0 f i IO61X_Library_MSVC120_vc:IO61X_iConcurrentExecution.obj
 0001:00014610       ?_InterlockedExchange64_ASM@@YA_JPC_J_J@Z 10015610 f i IO61X_Library_MSVC120_vc:IO61X_iConcurrentExecution.obj
 0001:00014640       ?_InterlockedOr64_ASM@@YA_JPC_J_J@Z 10015640 f i IO61X_Library_MSVC120_vc:IO61X_iConcurrentExecution.obj
 0001:00014670       ?_Load@?$_Atomic_impl@$07@std@@QDEXPAXPBXW4memory_order@2@@Z 10015670 f i IO61X_Library_MSVC120_vc:IO61X_iConcurrentExecution.obj
 0001:000146e0       ?_Load_acquire_8@std@@YA_KPC_K@Z 100156e0 f i IO61X_Library_MSVC120_vc:IO61X_iConcurrentExecution.obj
 0001:00014700       ?_Load_relaxed_8@std@@YA_KPC_K@Z 10015700 f i IO61X_Library_MSVC120_vc:IO61X_iConcurrentExecution.obj
 0001:00014720       ?_Load_seq_cst_8@std@@YA_KPC_K@Z 10015720 f i IO61X_Library_MSVC120_vc:IO61X_iConcurrentExecution.obj
 0001:00014740       ?_Myptr@?$_String_val@U?$_Simple_types@D@std@@@std@@QAEPADXZ 10015740 f i IO61X_Library_MSVC120_vc:IO61X_iConcurrentExecution.obj
 0001:00014750       ?_Myptr@?$_String_val@U?$_Simple_types@D@std@@@std@@QBEPBDXZ 10015750 f i IO61X_Library_MSVC120_vc:IO61X_iConcurrentExecution.obj
 0001:00014760       ?_Store@?$_Atomic_impl@$07@std@@QCEXPAXPBXW4memory_order@2@@Z 10015760 f i IO61X_Library_MSVC120_vc:IO61X_iConcurrentExecution.obj
 0001:00014790       ?_Store_relaxed_4@std@@YAXPCKK@Z 10015790 f i IO61X_Library_MSVC120_vc:IO61X_iConcurrentExecution.obj
 0001:000147a0       ?_Store_relaxed_8@std@@YAXPC_K_K@Z 100157a0 f i IO61X_Library_MSVC120_vc:IO61X_iConcurrentExecution.obj
 0001:000147c0       ?_Store_release_4@std@@YAXPCKK@Z 100157c0 f i IO61X_Library_MSVC120_vc:IO61X_iConcurrentExecution.obj
 0001:000147d0       ?_Store_release_8@std@@YAXPC_K_K@Z 100157d0 f i IO61X_Library_MSVC120_vc:IO61X_iConcurrentExecution.obj
 0001:000147f0       ?_Store_seq_cst_4@std@@YAXPCKK@Z 100157f0 f i IO61X_Library_MSVC120_vc:IO61X_iConcurrentExecution.obj
 0001:00014800       ?_Store_seq_cst_8@std@@YAXPC_K_K@Z 10015800 f i IO61X_Library_MSVC120_vc:IO61X_iConcurrentExecution.obj
 0001:00014820       ?_Tidy@?$basic_string@DU?$char_traits@D@std@@V?$allocator@D@2@@std@@QAEX_NI@Z 10015820 f i IO61X_Library_MSVC120_vc:IO61X_iConcurrentExecution.obj
 0001:00014870       ?_Xlen@?$basic_string@DU?$char_traits@D@std@@V?$allocator@D@2@@std@@QBEXXZ 10015870 f i IO61X_Library_MSVC120_vc:IO61X_iConcurrentExecution.obj
 0001:00014880       ?_Xran@?$basic_string@DU?$char_traits@D@std@@V?$allocator@D@2@@std@@QBEXXZ 10015880 f i IO61X_Library_MSVC120_vc:IO61X_iConcurrentExecution.obj
 0001:00014890       ?allocate@?$_Wrap_alloc@V?$allocator@D@std@@@std@@QAEPADI@Z 10015890 f i IO61X_Library_MSVC120_vc:IO61X_iConcurrentExecution.obj
 0001:000148c0       ?allocate@?$allocator@D@std@@QAEPADI@Z 100158c0 f i IO61X_Library_MSVC120_vc:IO61X_iConcurrentExecution.obj
 0001:000148f0       ?assign@?$basic_string@DU?$char_traits@D@std@@V?$allocator@D@2@@std@@QAEAAV12@ABV12@II@Z 100158f0 f i IO61X_Library_MSVC120_vc:IO61X_iConcurrentExecution.obj
 0001:00014a20       ?assign@?$basic_string@DU?$char_traits@D@std@@V?$allocator@D@2@@std@@QAEAAV12@PBD@Z 10015a20 f i IO61X_Library_MSVC120_vc:IO61X_iConcurrentExecution.obj
 0001:00014a60       ?assign@?$basic_string@DU?$char_traits@D@std@@V?$allocator@D@2@@std@@QAEAAV12@PBDI@Z 10015a60 f i IO61X_Library_MSVC120_vc:IO61X_iConcurrentExecution.obj
 0001:00014b60       ?assign@?$char_traits@D@std@@SAXAADABD@Z 10015b60 f i IO61X_Library_MSVC120_vc:IO61X_iConcurrentExecution.obj
 0001:00014b70       ?atomic_store@std@@YAXPAUatomic_int@1@H@Z 10015b70 f i IO61X_Library_MSVC120_vc:IO61X_iConcurrentExecution.obj
 0001:00014b80       ?atomic_store_explicit@std@@YAXPAUatomic_int@1@HW4memory_order@1@@Z 10015b80 f i IO61X_Library_MSVC120_vc:IO61X_iConcurrentExecution.obj
 0001:00014bb0       ?category@error_code@std@@QBEABVerror_category@2@XZ 10015bb0 f i IO61X_Library_MSVC120_vc:IO61X_iConcurrentExecution.obj
 0001:00014bc0       ?category@error_condition@std@@QBEABVerror_category@2@XZ 10015bc0 f i IO61X_Library_MSVC120_vc:IO61X_iConcurrentExecution.obj
 0001:00014bd0       ?copy@?$char_traits@D@std@@SAPADPADPBDI@Z 10015bd0 f i IO61X_Library_MSVC120_vc:IO61X_iConcurrentExecution.obj
 0001:00014bf0       ?deallocate@?$_Wrap_alloc@V?$allocator@D@std@@@std@@QAEXPADI@Z 10015bf0 f i IO61X_Library_MSVC120_vc:IO61X_iConcurrentExecution.obj
 0001:00014c10       ?deallocate@?$allocator@D@std@@QAEXPADI@Z 10015c10 f i IO61X_Library_MSVC120_vc:IO61X_iConcurrentExecution.obj
 0001:00014c30       ?default_error_condition@_System_error_category@std@@UBE?AVerror_condition@2@H@Z 10015c30 f i IO61X_Library_MSVC120_vc:IO61X_iConcurrentExecution.obj
 0001:00014c70       ?default_error_condition@error_category@std@@UBE?AVerror_condition@2@H@Z 10015c70 f i IO61X_Library_MSVC120_vc:IO61X_iConcurrentExecution.obj
 0001:00014c90       ?equivalent@error_category@std@@UBE_NABVerror_code@2@H@Z 10015c90 f i IO61X_Library_MSVC120_vc:IO61X_iConcurrentExecution.obj
 0001:00014cb0       ?equivalent@error_category@std@@UBE_NHABVerror_condition@2@@Z 10015cb0 f i IO61X_Library_MSVC120_vc:IO61X_iConcurrentExecution.obj
 0001:00014cf0       ?erase@?$basic_string@DU?$char_traits@D@std@@V?$allocator@D@2@@std@@QAEAAV12@I@Z 10015cf0 f i IO61X_Library_MSVC120_vc:IO61X_iConcurrentExecution.obj
 0001:00014d30       ?erase@?$basic_string@DU?$char_traits@D@std@@V?$allocator@D@2@@std@@QAEAAV12@II@Z 10015d30 f i IO61X_Library_MSVC120_vc:IO61X_iConcurrentExecution.obj
 0001:00014dd0       ?generic_category@std@@YAABVerror_category@1@XZ 10015dd0 f i IO61X_Library_MSVC120_vc:IO61X_iConcurrentExecution.obj
 0001:00014de0       ?getLastTaskTime@IO61X_Port@@QAENXZ 10015de0 f i IO61X_Library_MSVC120_vc:IO61X_iConcurrentExecution.obj
 0001:00014e10       ?length@?$char_traits@D@std@@SAIPBD@Z 10015e10 f i IO61X_Library_MSVC120_vc:IO61X_iConcurrentExecution.obj
 0001:00014e30       ?load@?$_Atomic@N$07@std@@QBENW4memory_order@2@@Z 10015e30 f i IO61X_Library_MSVC120_vc:IO61X_iConcurrentExecution.obj
 0001:00014ea0       ?max_size@?$_Wrap_alloc@V?$allocator@D@std@@@std@@QBEIXZ 10015ea0 f i IO61X_Library_MSVC120_vc:IO61X_iConcurrentExecution.obj
 0001:00014eb0       ?max_size@?$allocator@D@std@@QBEIXZ 10015eb0 f i IO61X_Library_MSVC120_vc:IO61X_iConcurrentExecution.obj
 0001:00014ec0       ?max_size@?$allocator_traits@V?$allocator@D@std@@@std@@SAIABV?$allocator@D@2@@Z 10015ec0 f i IO61X_Library_MSVC120_vc:IO61X_iConcurrentExecution.obj
 0001:00014ed0       ?max_size@?$basic_string@DU?$char_traits@D@std@@V?$allocator@D@2@@std@@QBEIXZ 10015ed0 f i IO61X_Library_MSVC120_vc:IO61X_iConcurrentExecution.obj
 0001:00014ee0       ?message@_Generic_error_category@std@@UBE?AV?$basic_string@DU?$char_traits@D@std@@V?$allocator@D@2@@2@H@Z 10015ee0 f i IO61X_Library_MSVC120_vc:IO61X_iConcurrentExecution.obj
 0001:00014f50       ?message@_Iostream_error_category@std@@UBE?AV?$basic_string@DU?$char_traits@D@std@@V?$allocator@D@2@@2@H@Z 10015f50 f i IO61X_Library_MSVC120_vc:IO61X_iConcurrentExecution.obj
 0001:00014fa0       ?message@_System_error_category@std@@UBE?AV?$basic_string@DU?$char_traits@D@std@@V?$allocator@D@2@@2@H@Z 10015fa0 f i IO61X_Library_MSVC120_vc:IO61X_iConcurrentExecution.obj
 0001:00015010       ?move@?$char_traits@D@std@@SAPADPADPBDI@Z 10016010 f i IO61X_Library_MSVC120_vc:IO61X_iConcurrentExecution.obj
 0001:00015030       ?name@_Generic_error_category@std@@UBEPBDXZ 10016030 f i IO61X_Library_MSVC120_vc:IO61X_iConcurrentExecution.obj
 0001:00015040       ?name@_Iostream_error_category@std@@UBEPBDXZ 10016040 f i IO61X_Library_MSVC120_vc:IO61X_iConcurrentExecution.obj
 0001:00015050       ?name@_System_error_category@std@@UBEPBDXZ 10016050 f i IO61X_Library_MSVC120_vc:IO61X_iConcurrentExecution.obj
 0001:00015060       ?setLastTaskTime@IO61X_Port@@QAEXN@Z 10016060 f i IO61X_Library_MSVC120_vc:IO61X_iConcurrentExecution.obj
 0001:00015090       ?size@?$basic_string@DU?$char_traits@D@std@@V?$allocator@D@2@@std@@QBEIXZ 10016090 f i IO61X_Library_MSVC120_vc:IO61X_iConcurrentExecution.obj
 0001:000150a0       ?store@?$_Atomic@N$07@std@@QAEXNW4memory_order@2@@Z 100160a0 f i IO61X_Library_MSVC120_vc:IO61X_iConcurrentExecution.obj
 0001:000150d0       ?system_category@std@@YAABVerror_category@1@XZ 100160d0 f i IO61X_Library_MSVC120_vc:IO61X_iConcurrentExecution.obj
 0001:000150e0       ?value@error_code@std@@QBEHXZ 100160e0 f i IO61X_Library_MSVC120_vc:IO61X_iConcurrentExecution.obj
 0001:000150f0       ?value@error_condition@std@@QBEHXZ 100160f0 f i IO61X_Library_MSVC120_vc:IO61X_iConcurrentExecution.obj
 0001:00015100       _hypot                     10016100 f i IO61X_Library_MSVC120_vc:IO61X_iConcurrentExecution.obj
 0001:00015130       ?IO61X_GlbSenderThr@@YAPAXPAX@Z 10016130 f   IO61X_Library_MSVC120_vc:IO61X_GlobalSender.obj
 0001:00015210       ?isActive@IO61X_Port@@QAE_NXZ 10016210 f i IO61X_Library_MSVC120_vc:IO61X_GlobalSender.obj
 0001:00015220       ?setActive@IO61X_GlobalSenderObj@@QAE_NH_NPAD@Z 10016220 f   IO61X_Library_MSVC120_vc:IO61X_GlobalSender.obj
 0001:00015400       ?setActive@IO61X_Port@@QAEX_N@Z 10016400 f i IO61X_Library_MSVC120_vc:IO61X_GlobalSender.obj
 0001:00015410       ??$?6U?$char_traits@D@std@@@std@@YAAAV?$basic_ostream@DU?$char_traits@D@std@@@0@AAV10@PBD@Z 10016410 f i IO61X_Library_MSVC120_vc:IO61X_DriverObject.obj
 0001:00015760       ??$_Fgetc@D@std@@YA_NAADPAU_iobuf@@@Z 10016760 f i IO61X_Library_MSVC120_vc:IO61X_DriverObject.obj
 0001:00015790       ??$_Fputc@D@std@@YA_NDPAU_iobuf@@@Z 10016790 f i IO61X_Library_MSVC120_vc:IO61X_DriverObject.obj
 0001:000157b0       ??$_Ungetc@D@std@@YA_NABDPAU_iobuf@@@Z 100167b0 f i IO61X_Library_MSVC120_vc:IO61X_DriverObject.obj
 0001:000157d0       ??$forward@V?$basic_string@DU?$char_traits@D@std@@V?$allocator@D@2@@std@@@std@@YA$$QAV?$basic_string@DU?$char_traits@D@std@@V?$allocator@D@2@@0@AAV10@@Z 100167d0 f i IO61X_Library_MSVC120_vc:IO61X_DriverObject.obj
 0001:000157e0       ??$use_facet@V?$codecvt@DDH@std@@@std@@YAABV?$codecvt@DDH@0@ABVlocale@0@@Z 100167e0 f i IO61X_Library_MSVC120_vc:IO61X_DriverObject.obj
 0001:00015900       ??$use_facet@V?$ctype@D@std@@@std@@YAABV?$ctype@D@0@ABVlocale@0@@Z 10016900 f i IO61X_Library_MSVC120_vc:IO61X_DriverObject.obj
 0001:00015a20       ??0?$IO61X_LoggerFifo@ULogLine@@@@QAE@I@Z 10016a20 f i IO61X_Library_MSVC120_vc:IO61X_DriverObject.obj
 0001:00015b00       ??0?$_String_const_iterator@V?$_String_val@U?$_Simple_types@D@std@@@std@@@std@@QAE@PBDPBU_Container_base0@1@@Z 10016b00 f i IO61X_Library_MSVC120_vc:IO61X_DriverObject.obj
 0001:00015b10       ??0?$_String_iterator@V?$_String_val@U?$_Simple_types@D@std@@@std@@@std@@QAE@PADPBU_Container_base0@1@@Z 10016b10 f i IO61X_Library_MSVC120_vc:IO61X_DriverObject.obj
 0001:00015b20       ??0?$_Wrap_alloc@V?$allocator@D@std@@@std@@QAE@ABV?$allocator@D@1@@Z 10016b20 f i IO61X_Library_MSVC120_vc:IO61X_DriverObject.obj
 0001:00015b30       ??0?$_Yarn@D@std@@QAE@XZ   10016b30 f i IO61X_Library_MSVC120_vc:IO61X_DriverObject.obj
 0001:00015b40       ??0?$_Yarn@_W@std@@QAE@XZ  10016b40 f i IO61X_Library_MSVC120_vc:IO61X_DriverObject.obj
 0001:00015b50       ??0?$allocator@D@std@@QAE@ABV01@@Z 10016b50 f i IO61X_Library_MSVC120_vc:IO61X_DriverObject.obj
 0001:00015b60       ??0?$atomic@_N@std@@QAE@XZ 10016b60 f i IO61X_Library_MSVC120_vc:IO61X_DriverObject.obj
 0001:00015b70       ??0?$basic_filebuf@DU?$char_traits@D@std@@@std@@QAE@PAU_iobuf@@@Z 10016b70 f i IO61X_Library_MSVC120_vc:IO61X_DriverObject.obj
 0001:00015ba0       ??0?$basic_ios@DU?$char_traits@D@std@@@std@@IAE@XZ 10016ba0 f i IO61X_Library_MSVC120_vc:IO61X_DriverObject.obj
 0001:00015bb0       ??0?$basic_ofstream@DU?$char_traits@D@std@@@std@@QAE@PBDHH@Z 10016bb0 f i IO61X_Library_MSVC120_vc:IO61X_DriverObject.obj
 0001:00015d90       ??0?$basic_ostream@DU?$char_traits@D@std@@@std@@QAE@PAV?$basic_streambuf@DU?$char_traits@D@std@@@1@_N@Z 10016d90 f i IO61X_Library_MSVC120_vc:IO61X_DriverObject.obj
 0001:00015e30       ??0?$basic_streambuf@DU?$char_traits@D@std@@@std@@IAE@XZ 10016e30 f i IO61X_Library_MSVC120_vc:IO61X_DriverObject.obj
 0001:00015ec0       ??0?$basic_string@DU?$char_traits@D@std@@V?$allocator@D@2@@std@@QAE@$$QAV01@@Z 10016ec0 f i IO61X_Library_MSVC120_vc:IO61X_DriverObject.obj
 0001:00015f30       ??0?$basic_string@DU?$char_traits@D@std@@V?$allocator@D@2@@std@@QAE@ABV01@@Z 10016f30 f i IO61X_Library_MSVC120_vc:IO61X_DriverObject.obj
 0001:00015f60       ??0?$basic_string@DU?$char_traits@D@std@@V?$allocator@D@2@@std@@QAE@ID@Z 10016f60 f i IO61X_Library_MSVC120_vc:IO61X_DriverObject.obj
 0001:00015f90       ??0?$basic_string@DU?$char_traits@D@std@@V?$allocator@D@2@@std@@QAE@XZ 10016f90 f i IO61X_Library_MSVC120_vc:IO61X_DriverObject.obj
 0001:00015fb0       ??0?$codecvt@DDH@std@@QAE@ABV_Locinfo@1@I@Z 10016fb0 f i IO61X_Library_MSVC120_vc:IO61X_DriverObject.obj
 0001:00015fd0       ??0?$ctype@D@std@@QAE@ABV_Locinfo@1@I@Z 10016fd0 f i IO61X_Library_MSVC120_vc:IO61X_DriverObject.obj
 0001:00016010       ??0?$fpos@H@std@@QAE@H_J@Z 10017010 f i IO61X_Library_MSVC120_vc:IO61X_DriverObject.obj
 0001:00016040       ??0?$fpos@H@std@@QAE@_J@Z  10017040 f i IO61X_Library_MSVC120_vc:IO61X_DriverObject.obj
 0001:00016070       ??0IO61X_DriverObject@@QAE@XZ 10017070 f   IO61X_Library_MSVC120_vc:IO61X_DriverObject.obj
 0001:000160a0       ??0IO61X_Logger@@QAE@XZ    100170a0 f   IO61X_Library_MSVC120_vc:IO61X_DriverObject.obj
 0001:000160d0       ??0LogLine@@QAE@HPBD@Z     100170d0 f   IO61X_Library_MSVC120_vc:IO61X_DriverObject.obj
 0001:00016110       ??0LogLine@@QAE@XZ         10017110 f i IO61X_Library_MSVC120_vc:IO61X_DriverObject.obj
 0001:00016120       ??0_Facet_base@std@@QAE@XZ 10017120 f i IO61X_Library_MSVC120_vc:IO61X_DriverObject.obj
 0001:00016130       ??0_Locinfo@std@@QAE@PBD@Z 10017130 f i IO61X_Library_MSVC120_vc:IO61X_DriverObject.obj
 0001:000161f0       ??0_Sentry_base@?$basic_ostream@DU?$char_traits@D@std@@@std@@QAE@AAV12@@Z 100171f0 f i IO61X_Library_MSVC120_vc:IO61X_DriverObject.obj
 0001:00016220       ??0_System_error@std@@IAE@Verror_code@1@ABV?$basic_string@DU?$char_traits@D@std@@V?$allocator@D@2@@1@@Z 10017220 f i IO61X_Library_MSVC120_vc:IO61X_DriverObject.obj
 0001:000162f0       ??0_System_error@std@@QAE@ABV01@@Z 100172f0 f i IO61X_Library_MSVC120_vc:IO61X_DriverObject.obj
 0001:00016320       ??0codecvt_base@std@@QAE@I@Z 10017320 f i IO61X_Library_MSVC120_vc:IO61X_DriverObject.obj
 0001:00016340       ??0ctype_base@std@@QAE@I@Z 10017340 f i IO61X_Library_MSVC120_vc:IO61X_DriverObject.obj
 0001:00016360       ??0error_code@std@@QAE@HABVerror_category@1@@Z 10017360 f i IO61X_Library_MSVC120_vc:IO61X_DriverObject.obj
 0001:00016380       ??0facet@locale@std@@IAE@I@Z 10017380 f i IO61X_Library_MSVC120_vc:IO61X_DriverObject.obj
 0001:000163a0       ??0failure@ios_base@std@@QAE@ABV012@@Z 100173a0 f i IO61X_Library_MSVC120_vc:IO61X_DriverObject.obj
 0001:000163d0       ??0failure@ios_base@std@@QAE@PBDABVerror_code@2@@Z 100173d0 f i IO61X_Library_MSVC120_vc:IO61X_DriverObject.obj
 0001:00016400       ??0id@locale@std@@QAE@I@Z  10017400 f i IO61X_Library_MSVC120_vc:IO61X_DriverObject.obj
 0001:00016410       ??0invalid_argument@std@@QAE@ABV01@@Z 10017410 f i IO61X_Library_MSVC120_vc:IO61X_DriverObject.obj
 0001:00016430       ??0invalid_argument@std@@QAE@PBD@Z 10017430 f i IO61X_Library_MSVC120_vc:IO61X_DriverObject.obj
 0001:00016460       ??0ios_base@std@@IAE@XZ    10017460 f i IO61X_Library_MSVC120_vc:IO61X_DriverObject.obj
 0001:00016470       ??0locale@std@@QAE@ABV01@@Z 10017470 f i IO61X_Library_MSVC120_vc:IO61X_DriverObject.obj
 0001:00016490       ??0locale@std@@QAE@XZ      10017490 f i IO61X_Library_MSVC120_vc:IO61X_DriverObject.obj
 0001:000164b0       ??0logic_error@std@@QAE@ABV01@@Z 100174b0 f i IO61X_Library_MSVC120_vc:IO61X_DriverObject.obj
 0001:000164d0       ??0logic_error@std@@QAE@PBD@Z 100174d0 f i IO61X_Library_MSVC120_vc:IO61X_DriverObject.obj
 0001:000164f0       ??0runtime_error@std@@QAE@ABV01@@Z 100174f0 f i IO61X_Library_MSVC120_vc:IO61X_DriverObject.obj
 0001:00016510       ??0runtime_error@std@@QAE@ABV?$basic_string@DU?$char_traits@D@std@@V?$allocator@D@2@@1@@Z 10017510 f i IO61X_Library_MSVC120_vc:IO61X_DriverObject.obj
 0001:00016540       ??0runtime_error@std@@QAE@PBD@Z 10017540 f i IO61X_Library_MSVC120_vc:IO61X_DriverObject.obj
 0001:00016560       ??0sentry@?$basic_ostream@DU?$char_traits@D@std@@@std@@QAE@AAV12@@Z 10017560 f i IO61X_Library_MSVC120_vc:IO61X_DriverObject.obj
 0001:000165f0       ??0system_error@std@@QAE@ABV01@@Z 100175f0 f i IO61X_Library_MSVC120_vc:IO61X_DriverObject.obj
 0001:00016620       ??0system_error@std@@QAE@Verror_code@1@PBD@Z 10017620 f i IO61X_Library_MSVC120_vc:IO61X_DriverObject.obj
 0001:000166e0       ??1?$IO61X_LoggerFifo@ULogLine@@@@QAE@XZ 100176e0 f i IO61X_Library_MSVC120_vc:IO61X_DriverObject.obj
 0001:00016700       ??1?$_Yarn@D@std@@QAE@XZ   10017700 f i IO61X_Library_MSVC120_vc:IO61X_DriverObject.obj
 0001:00016720       ??1?$_Yarn@_W@std@@QAE@XZ  10017720 f i IO61X_Library_MSVC120_vc:IO61X_DriverObject.obj
 0001:00016740       ??1?$basic_filebuf@DU?$char_traits@D@std@@@std@@UAE@XZ 10017740 f i IO61X_Library_MSVC120_vc:IO61X_DriverObject.obj
 0001:000167b0       ??1?$basic_ios@DU?$char_traits@D@std@@@std@@UAE@XZ 100177b0 f i IO61X_Library_MSVC120_vc:IO61X_DriverObject.obj
 0001:000167c0       ??1?$basic_ofstream@DU?$char_traits@D@std@@@std@@UAE@XZ 100177c0 f i IO61X_Library_MSVC120_vc:IO61X_DriverObject.obj
 0001:00016810       ??1?$basic_ostream@DU?$char_traits@D@std@@@std@@UAE@XZ 10017810 f i IO61X_Library_MSVC120_vc:IO61X_DriverObject.obj
 0001:00016830       ??1?$basic_streambuf@DU?$char_traits@D@std@@@std@@UAE@XZ 10017830 f i IO61X_Library_MSVC120_vc:IO61X_DriverObject.obj
 0001:00016860       ??1?$codecvt@DDH@std@@MAE@XZ 10017860 f i IO61X_Library_MSVC120_vc:IO61X_DriverObject.obj
 0001:00016870       ??1?$ctype@D@std@@MAE@XZ   10017870 f i IO61X_Library_MSVC120_vc:IO61X_DriverObject.obj
 0001:000168b0       ??1IO61X_DriverObject@@QAE@XZ 100178b0 f   IO61X_Library_MSVC120_vc:IO61X_DriverObject.obj
 0001:000168e0       ??1IO61X_Logger@@QAE@XZ    100178e0 f   IO61X_Library_MSVC120_vc:IO61X_DriverObject.obj
 0001:00016950       ??1_Facet_base@std@@UAE@XZ 10017950 f i IO61X_Library_MSVC120_vc:IO61X_DriverObject.obj
 0001:00016960       ??1_Locinfo@std@@QAE@XZ    10017960 f i IO61X_Library_MSVC120_vc:IO61X_DriverObject.obj
 0001:00016a00       ??1_Sentry_base@?$basic_ostream@DU?$char_traits@D@std@@@std@@QAE@XZ 10017a00 f i IO61X_Library_MSVC120_vc:IO61X_DriverObject.obj
 0001:00016a20       ??1_System_error@std@@UAE@XZ 10017a20 f i IO61X_Library_MSVC120_vc:IO61X_DriverObject.obj
 0001:00016a30       ??1codecvt_base@std@@UAE@XZ 10017a30 f i IO61X_Library_MSVC120_vc:IO61X_DriverObject.obj
 0001:00016a40       ??1ctype_base@std@@UAE@XZ  10017a40 f i IO61X_Library_MSVC120_vc:IO61X_DriverObject.obj
 0001:00016a50       ??1facet@locale@std@@MAE@XZ 10017a50 f i IO61X_Library_MSVC120_vc:IO61X_DriverObject.obj
 0001:00016a60       ??1failure@ios_base@std@@UAE@XZ 10017a60 f i IO61X_Library_MSVC120_vc:IO61X_DriverObject.obj
 0001:00016a70       ??1invalid_argument@std@@UAE@XZ 10017a70 f i IO61X_Library_MSVC120_vc:IO61X_DriverObject.obj
 0001:00016a80       ??1ios_base@std@@UAE@XZ    10017a80 f i IO61X_Library_MSVC120_vc:IO61X_DriverObject.obj
 0001:00016a90       ??1locale@std@@QAE@XZ      10017a90 f i IO61X_Library_MSVC120_vc:IO61X_DriverObject.obj
 0001:00016ab0       ??1logic_error@std@@UAE@XZ 10017ab0 f i IO61X_Library_MSVC120_vc:IO61X_DriverObject.obj
 0001:00016ac0       ??1runtime_error@std@@UAE@XZ 10017ac0 f i IO61X_Library_MSVC120_vc:IO61X_DriverObject.obj
 0001:00016ad0       ??1sentry@?$basic_ostream@DU?$char_traits@D@std@@@std@@QAE@XZ 10017ad0 f i IO61X_Library_MSVC120_vc:IO61X_DriverObject.obj
 0001:00016b00       ??1system_error@std@@UAE@XZ 10017b00 f i IO61X_Library_MSVC120_vc:IO61X_DriverObject.obj
 0001:00016b10       ??4?$atomic@_N@std@@QAE_N_N@Z 10017b10 f i IO61X_Library_MSVC120_vc:IO61X_DriverObject.obj
 0001:00016b20       ??4atomic_bool@std@@QAE_N_N@Z 10017b20 f i IO61X_Library_MSVC120_vc:IO61X_DriverObject.obj
 0001:00016b30       ??B?$fpos@H@std@@QBE_JXZ   10017b30 f i IO61X_Library_MSVC120_vc:IO61X_DriverObject.obj
 0001:00016b40       ??Batomic_bool@std@@QBE_NXZ 10017b40 f i IO61X_Library_MSVC120_vc:IO61X_DriverObject.obj
 0001:00016b50       ??Bid@locale@std@@QAEIXZ   10017b50 f i IO61X_Library_MSVC120_vc:IO61X_DriverObject.obj
 0001:00016b90       ??Bsentry@?$basic_ostream@DU?$char_traits@D@std@@@std@@QBE_NXZ 10017b90 f i IO61X_Library_MSVC120_vc:IO61X_DriverObject.obj
 0001:00016ba0       ??D?$_String_const_iterator@V?$_String_val@U?$_Simple_types@D@std@@@std@@@std@@QBEABDXZ 10017ba0 f i IO61X_Library_MSVC120_vc:IO61X_DriverObject.obj
 0001:00016bb0       ??D?$_String_iterator@V?$_String_val@U?$_Simple_types@D@std@@@std@@@std@@QBEAADXZ 10017bb0 f i IO61X_Library_MSVC120_vc:IO61X_DriverObject.obj
 0001:00016bc0       ??_D?$basic_ofstream@DU?$char_traits@D@std@@@std@@QAEXXZ 10017bc0 f i IO61X_Library_MSVC120_vc:IO61X_DriverObject.obj
 0001:00016c20       ??_D?$basic_ostream@DU?$char_traits@D@std@@@std@@QAEXXZ 10017c20 f i IO61X_Library_MSVC120_vc:IO61X_DriverObject.obj
 0001:00016c4b       ??_E?$basic_ofstream@DU?$char_traits@D@std@@@std@@$4PPPPPPPM@A@AEPAXI@Z 10017c4b f i IO61X_Library_MSVC120_vc:IO61X_DriverObject.obj
 0001:00016c53       ??_E?$basic_ostream@DU?$char_traits@D@std@@@std@@$4PPPPPPPM@A@AEPAXI@Z 10017c53 f i IO61X_Library_MSVC120_vc:IO61X_DriverObject.obj
 0001:00016c60       ??_G?$IO61X_LoggerFifo@ULogLine@@@@QAEPAXI@Z 10017c60 f i IO61X_Library_MSVC120_vc:IO61X_DriverObject.obj
 0001:00016ca0       ??_E?$basic_filebuf@DU?$char_traits@D@std@@@std@@UAEPAXI@Z 10017ca0 f i IO61X_Library_MSVC120_vc:IO61X_DriverObject.obj
 0001:00016ca0       ??_G?$basic_filebuf@DU?$char_traits@D@std@@@std@@UAEPAXI@Z 10017ca0 f i IO61X_Library_MSVC120_vc:IO61X_DriverObject.obj
 0001:00016cd0       ??_E?$basic_ios@DU?$char_traits@D@std@@@std@@UAEPAXI@Z 10017cd0 f i IO61X_Library_MSVC120_vc:IO61X_DriverObject.obj
 0001:00016cd0       ??_G?$basic_ios@DU?$char_traits@D@std@@@std@@UAEPAXI@Z 10017cd0 f i IO61X_Library_MSVC120_vc:IO61X_DriverObject.obj
 0001:00016d00       ??_G?$basic_ofstream@DU?$char_traits@D@std@@@std@@UAEPAXI@Z 10017d00 f i IO61X_Library_MSVC120_vc:IO61X_DriverObject.obj
 0001:00016d00       ??_E?$basic_ofstream@DU?$char_traits@D@std@@@std@@UAEPAXI@Z 10017d00 f i IO61X_Library_MSVC120_vc:IO61X_DriverObject.obj
 0001:00016d70       ??_E?$basic_ostream@DU?$char_traits@D@std@@@std@@UAEPAXI@Z 10017d70 f i IO61X_Library_MSVC120_vc:IO61X_DriverObject.obj
 0001:00016d70       ??_G?$basic_ostream@DU?$char_traits@D@std@@@std@@UAEPAXI@Z 10017d70 f i IO61X_Library_MSVC120_vc:IO61X_DriverObject.obj
 0001:00016dc0       ??_E?$basic_streambuf@DU?$char_traits@D@std@@@std@@UAEPAXI@Z 10017dc0 f i IO61X_Library_MSVC120_vc:IO61X_DriverObject.obj
 0001:00016dc0       ??_G?$basic_streambuf@DU?$char_traits@D@std@@@std@@UAEPAXI@Z 10017dc0 f i IO61X_Library_MSVC120_vc:IO61X_DriverObject.obj
 0001:00016e10       ??_G?$codecvt@DDH@std@@MAEPAXI@Z 10017e10 f i IO61X_Library_MSVC120_vc:IO61X_DriverObject.obj
 0001:00016e10       ??_E?$codecvt@DDH@std@@MAEPAXI@Z 10017e10 f i IO61X_Library_MSVC120_vc:IO61X_DriverObject.obj
 0001:00016e40       ??_G?$ctype@D@std@@MAEPAXI@Z 10017e40 f i IO61X_Library_MSVC120_vc:IO61X_DriverObject.obj
 0001:00016e40       ??_E?$ctype@D@std@@MAEPAXI@Z 10017e40 f i IO61X_Library_MSVC120_vc:IO61X_DriverObject.obj
 0001:00016ea0       ??_G_Facet_base@std@@UAEPAXI@Z 10017ea0 f i IO61X_Library_MSVC120_vc:IO61X_DriverObject.obj
 0001:00016ea0       ??_E_Facet_base@std@@UAEPAXI@Z 10017ea0 f i IO61X_Library_MSVC120_vc:IO61X_DriverObject.obj
 0001:00016ed0       ??_G_System_error@std@@UAEPAXI@Z 10017ed0 f i IO61X_Library_MSVC120_vc:IO61X_DriverObject.obj
 0001:00016ed0       ??_E_System_error@std@@UAEPAXI@Z 10017ed0 f i IO61X_Library_MSVC120_vc:IO61X_DriverObject.obj
 0001:00016f00       ??_Gcodecvt_base@std@@UAEPAXI@Z 10017f00 f i IO61X_Library_MSVC120_vc:IO61X_DriverObject.obj
 0001:00016f00       ??_Ecodecvt_base@std@@UAEPAXI@Z 10017f00 f i IO61X_Library_MSVC120_vc:IO61X_DriverObject.obj
 0001:00016f30       ??_Gctype_base@std@@UAEPAXI@Z 10017f30 f i IO61X_Library_MSVC120_vc:IO61X_DriverObject.obj
 0001:00016f30       ??_Ectype_base@std@@UAEPAXI@Z 10017f30 f i IO61X_Library_MSVC120_vc:IO61X_DriverObject.obj
 0001:00016f60       ??_Efacet@locale@std@@MAEPAXI@Z 10017f60 f i IO61X_Library_MSVC120_vc:IO61X_DriverObject.obj
 0001:00016f60       ??_Gfacet@locale@std@@MAEPAXI@Z 10017f60 f i IO61X_Library_MSVC120_vc:IO61X_DriverObject.obj
 0001:00016f90       ??_Gfailure@ios_base@std@@UAEPAXI@Z 10017f90 f i IO61X_Library_MSVC120_vc:IO61X_DriverObject.obj
 0001:00016f90       ??_Efailure@ios_base@std@@UAEPAXI@Z 10017f90 f i IO61X_Library_MSVC120_vc:IO61X_DriverObject.obj
 0001:00016fc0       ??_Ginvalid_argument@std@@UAEPAXI@Z 10017fc0 f i IO61X_Library_MSVC120_vc:IO61X_DriverObject.obj
 0001:00016fc0       ??_Einvalid_argument@std@@UAEPAXI@Z 10017fc0 f i IO61X_Library_MSVC120_vc:IO61X_DriverObject.obj
 0001:00016ff0       ??_Gios_base@std@@UAEPAXI@Z 10017ff0 f i IO61X_Library_MSVC120_vc:IO61X_DriverObject.obj
 0001:00016ff0       ??_Eios_base@std@@UAEPAXI@Z 10017ff0 f i IO61X_Library_MSVC120_vc:IO61X_DriverObject.obj
 0001:00017020       ??_Glocale@std@@QAEPAXI@Z  10018020 f i IO61X_Library_MSVC120_vc:IO61X_DriverObject.obj
 0001:00017060       ??_Glogic_error@std@@UAEPAXI@Z 10018060 f i IO61X_Library_MSVC120_vc:IO61X_DriverObject.obj
 0001:00017060       ??_Elogic_error@std@@UAEPAXI@Z 10018060 f i IO61X_Library_MSVC120_vc:IO61X_DriverObject.obj
 0001:00017090       ??_Gruntime_error@std@@UAEPAXI@Z 10018090 f i IO61X_Library_MSVC120_vc:IO61X_DriverObject.obj
 0001:00017090       ??_Eruntime_error@std@@UAEPAXI@Z 10018090 f i IO61X_Library_MSVC120_vc:IO61X_DriverObject.obj
 0001:000170c0       ??_Esystem_error@std@@UAEPAXI@Z 100180c0 f i IO61X_Library_MSVC120_vc:IO61X_DriverObject.obj
 0001:000170c0       ??_Gsystem_error@std@@UAEPAXI@Z 100180c0 f i IO61X_Library_MSVC120_vc:IO61X_DriverObject.obj
 0001:000170f0       ??_H@YGXPAXIHP6EPAX0@Z@Z   100180f0 f i IO61X_Library_MSVC120_vc:IO61X_DriverObject.obj
 0001:00017120       ?AddMessageOverwriting@?$IO61X_LoggerFifo@ULogLine@@@@QAEXPBULogLine@@@Z 10018120 f i IO61X_Library_MSVC120_vc:IO61X_DriverObject.obj
 0001:00017190       ?GetMessageFromBuffer@?$IO61X_LoggerFifo@ULogLine@@@@QAEPAULogLine@@XZ 10018190 f i IO61X_Library_MSVC120_vc:IO61X_DriverObject.obj
 0001:000171c0       ?GetNextFreeModuleIndex@IO61X_DriverObject@@QAEHXZ 100181c0 f   IO61X_Library_MSVC120_vc:IO61X_DriverObject.obj
 0001:000171f0       ?IsDebug@IO61X_Logger@@QAE_NXZ 100181f0 f i IO61X_Library_MSVC120_vc:IO61X_DriverObject.obj
 0001:00017210       ?IsErr@IO61X_Logger@@QAE_NXZ 10018210 f i IO61X_Library_MSVC120_vc:IO61X_DriverObject.obj
 0001:00017220       ?IsInfo@IO61X_Logger@@QAE_NXZ 10018220 f i IO61X_Library_MSVC120_vc:IO61X_DriverObject.obj
 0001:00017240       ?IsWarn@IO61X_Logger@@QAE_NXZ 10018240 f i IO61X_Library_MSVC120_vc:IO61X_DriverObject.obj
 0001:00017250       ?_Adopt@_Iterator_base0@std@@QAEXPBX@Z 10018250 f i IO61X_Library_MSVC120_vc:IO61X_DriverObject.obj
 0001:00017260       ?_Assign_rv@?$basic_string@DU?$char_traits@D@std@@V?$allocator@D@2@@std@@QAEX$$QAV12@@Z 10018260 f i IO61X_Library_MSVC120_vc:IO61X_DriverObject.obj
 0001:000172c0       ?_Atomic_fetch_add_4@std@@YAKPCKKW4memory_order@1@@Z 100182c0 f i IO61X_Library_MSVC120_vc:IO61X_DriverObject.obj
 0001:00017300       ?_Atomic_load_1@std@@YAEPCEW4memory_order@1@@Z 10018300 f i IO61X_Library_MSVC120_vc:IO61X_DriverObject.obj
 0001:00017340       ?_Atomic_load_4@std@@YAKPCKW4memory_order@1@@Z 10018340 f i IO61X_Library_MSVC120_vc:IO61X_DriverObject.obj
 0001:00017380       ?_Atomic_store_1@std@@YAXPCEEW4memory_order@1@@Z 10018380 f i IO61X_Library_MSVC120_vc:IO61X_DriverObject.obj
 0001:000173b0       ?_Chassign@?$basic_string@DU?$char_traits@D@std@@V?$allocator@D@2@@std@@QAEXIID@Z 100183b0 f i IO61X_Library_MSVC120_vc:IO61X_DriverObject.obj
 0001:00017400       ?_Decref@facet@locale@std@@UAEPAV_Facet_base@3@XZ 10018400 f i IO61X_Library_MSVC120_vc:IO61X_DriverObject.obj
 0001:00017420       ?_Endwrite@?$basic_filebuf@DU?$char_traits@D@std@@@std@@IAE_NXZ 10018420 f i IO61X_Library_MSVC120_vc:IO61X_DriverObject.obj
 0001:00017570       ?_Fetch_add_acquire_4@std@@YAKPCKK@Z 10018570 f i IO61X_Library_MSVC120_vc:IO61X_DriverObject.obj
 0001:00017580       ?_Fetch_add_relaxed_4@std@@YAKPCKK@Z 10018580 f i IO61X_Library_MSVC120_vc:IO61X_DriverObject.obj
 0001:00017590       ?_Fetch_add_release_4@std@@YAKPCKK@Z 10018590 f i IO61X_Library_MSVC120_vc:IO61X_DriverObject.obj
 0001:000175a0       ?_Fetch_add_seq_cst_4@std@@YAKPCKK@Z 100185a0 f i IO61X_Library_MSVC120_vc:IO61X_DriverObject.obj
 0001:000175b0       ?_Getcat@?$codecvt@DDH@std@@SAIPAPBVfacet@locale@2@PBV42@@Z 100185b0 f i IO61X_Library_MSVC120_vc:IO61X_DriverObject.obj
 0001:00017660       ?_Getcat@?$ctype@D@std@@SAIPAPBVfacet@locale@2@PBV42@@Z 10018660 f i IO61X_Library_MSVC120_vc:IO61X_DriverObject.obj
 0001:00017730       ?_Getctype@_Locinfo@std@@QBE?AU_Ctypevec@@XZ 10018730 f i IO61X_Library_MSVC120_vc:IO61X_DriverObject.obj
 0001:00017760       ?_Getfacet@locale@std@@QBEPBVfacet@12@I@Z 10018760 f i IO61X_Library_MSVC120_vc:IO61X_DriverObject.obj
 0001:000177a0       ?_Gnavail@?$basic_streambuf@DU?$char_traits@D@std@@@std@@IBE_JXZ 100187a0 f i IO61X_Library_MSVC120_vc:IO61X_DriverObject.obj
 0001:000177c0       ?_Gndec@?$basic_streambuf@DU?$char_traits@D@std@@@std@@IAEPADXZ 100187c0 f i IO61X_Library_MSVC120_vc:IO61X_DriverObject.obj
 0001:000177d0       ?_Gninc@?$basic_streambuf@DU?$char_traits@D@std@@@std@@IAEPADXZ 100187d0 f i IO61X_Library_MSVC120_vc:IO61X_DriverObject.obj
 0001:000177e0       ?_Incref@facet@locale@std@@UAEXXZ 100187e0 f i IO61X_Library_MSVC120_vc:IO61X_DriverObject.obj
 0001:000177f0       ?_Init@?$basic_filebuf@DU?$char_traits@D@std@@@std@@IAEXPAU_iobuf@@W4_Initfl@12@@Z 100187f0 f i IO61X_Library_MSVC120_vc:IO61X_DriverObject.obj
 0001:00017890       ?_Init@?$basic_streambuf@DU?$char_traits@D@std@@@std@@IAEXPAPAD0PAH001@Z 10018890 f i IO61X_Library_MSVC120_vc:IO61X_DriverObject.obj
 0001:000178c0       ?_Init@?$basic_streambuf@DU?$char_traits@D@std@@@std@@IAEXXZ 100188c0 f i IO61X_Library_MSVC120_vc:IO61X_DriverObject.obj
 0001:00017920       ?_Init@?$codecvt@DDH@std@@IAEXABV_Locinfo@2@@Z 10018920 f i IO61X_Library_MSVC120_vc:IO61X_DriverObject.obj
 0001:00017930       ?_Init@?$ctype@D@std@@IAEXABV_Locinfo@2@@Z 10018930 f i IO61X_Library_MSVC120_vc:IO61X_DriverObject.obj
 0001:00017960       ?_Init@ios_base@std@@IAEXXZ 10018960 f i IO61X_Library_MSVC120_vc:IO61X_DriverObject.obj
 0001:000179e0       ?_Init_atomic_counter@std@@YAXAAKK@Z 100189e0 f i IO61X_Library_MSVC120_vc:IO61X_DriverObject.obj
 0001:000179f0       ?_Initcvt@?$basic_filebuf@DU?$char_traits@D@std@@@std@@IAEXPBV?$codecvt@DDH@2@@Z 100189f0 f i IO61X_Library_MSVC120_vc:IO61X_DriverObject.obj
 0001:00017a30       ?_Load_acquire_1@std@@YAEPCE@Z 10018a30 f i IO61X_Library_MSVC120_vc:IO61X_DriverObject.obj
 0001:00017a40       ?_Load_acquire_4@std@@YAKPCK@Z 10018a40 f i IO61X_Library_MSVC120_vc:IO61X_DriverObject.obj
 0001:00017a50       ?_Load_relaxed_1@std@@YAEPCE@Z 10018a50 f i IO61X_Library_MSVC120_vc:IO61X_DriverObject.obj
 0001:00017a60       ?_Load_relaxed_4@std@@YAKPCK@Z 10018a60 f i IO61X_Library_MSVC120_vc:IO61X_DriverObject.obj
 0001:00017a70       ?_Load_seq_cst_1@std@@YAEPCE@Z 10018a70 f i IO61X_Library_MSVC120_vc:IO61X_DriverObject.obj
 0001:00017a80       ?_Load_seq_cst_4@std@@YAKPCK@Z 10018a80 f i IO61X_Library_MSVC120_vc:IO61X_DriverObject.obj
 0001:00017a90       ?_Lock@?$basic_filebuf@DU?$char_traits@D@std@@@std@@UAEXXZ 10018a90 f i IO61X_Library_MSVC120_vc:IO61X_DriverObject.obj
 0001:00017aa0       ?_Lock@?$basic_streambuf@DU?$char_traits@D@std@@@std@@UAEXXZ 10018aa0 f i IO61X_Library_MSVC120_vc:IO61X_DriverObject.obj
 0001:00017ab0       ?_Makestr@_System_error@std@@CA?AV?$basic_string@DU?$char_traits@D@std@@V?$allocator@D@2@@2@Verror_code@2@V32@@Z 10018ab0 f i IO61X_Library_MSVC120_vc:IO61X_DriverObject.obj
 0001:00017b90       ?_Osfx@?$basic_ostream@DU?$char_traits@D@std@@@std@@QAEXXZ 10018b90 f i IO61X_Library_MSVC120_vc:IO61X_DriverObject.obj
 0001:00017cc0       ?_Pnavail@?$basic_streambuf@DU?$char_traits@D@std@@@std@@IBE_JXZ 10018cc0 f i IO61X_Library_MSVC120_vc:IO61X_DriverObject.obj
 0001:00017ce0       ?_Pninc@?$basic_streambuf@DU?$char_traits@D@std@@@std@@IAEPADXZ 10018ce0 f i IO61X_Library_MSVC120_vc:IO61X_DriverObject.obj
 0001:00017cf0       ?_Reset_back@?$basic_filebuf@DU?$char_traits@D@std@@@std@@AAEXXZ 10018cf0 f i IO61X_Library_MSVC120_vc:IO61X_DriverObject.obj
 0001:00017d20       ?_Set_back@?$basic_filebuf@DU?$char_traits@D@std@@@std@@AAEXXZ 10018d20 f i IO61X_Library_MSVC120_vc:IO61X_DriverObject.obj
 0001:00017d60       ?_Store_relaxed_1@std@@YAXPCEE@Z 10018d60 f i IO61X_Library_MSVC120_vc:IO61X_DriverObject.obj
 0001:00017d70       ?_Store_release_1@std@@YAXPCEE@Z 10018d70 f i IO61X_Library_MSVC120_vc:IO61X_DriverObject.obj
 0001:00017d80       ?_Store_seq_cst_1@std@@YAXPCEE@Z 10018d80 f i IO61X_Library_MSVC120_vc:IO61X_DriverObject.obj
 0001:00017d90       ?_Tidy@?$_Yarn@D@std@@AAEXXZ 10018d90 f i IO61X_Library_MSVC120_vc:IO61X_DriverObject.obj
 0001:00017db0       ?_Tidy@?$_Yarn@_W@std@@AAEXXZ 10018db0 f i IO61X_Library_MSVC120_vc:IO61X_DriverObject.obj
 0001:00017dd0       ?_Tidy@?$ctype@D@std@@IAEXXZ 10018dd0 f i IO61X_Library_MSVC120_vc:IO61X_DriverObject.obj
 0001:00017e10       ?_Unlock@?$basic_filebuf@DU?$char_traits@D@std@@@std@@UAEXXZ 10018e10 f i IO61X_Library_MSVC120_vc:IO61X_DriverObject.obj
 0001:00017e20       ?_Unlock@?$basic_streambuf@DU?$char_traits@D@std@@@std@@UAEXXZ 10018e20 f i IO61X_Library_MSVC120_vc:IO61X_DriverObject.obj
 0001:00017e30       ?always_noconv@codecvt_base@std@@QBE_NXZ 10018e30 f i IO61X_Library_MSVC120_vc:IO61X_DriverObject.obj
 0001:00017e40       ?append@?$basic_string@DU?$char_traits@D@std@@V?$allocator@D@2@@std@@QAEAAV12@ABV12@@Z 10018e40 f i IO61X_Library_MSVC120_vc:IO61X_DriverObject.obj
 0001:00017e60       ?append@?$basic_string@DU?$char_traits@D@std@@V?$allocator@D@2@@std@@QAEAAV12@ABV12@II@Z 10018e60 f i IO61X_Library_MSVC120_vc:IO61X_DriverObject.obj
 0001:00017f20       ?append@?$basic_string@DU?$char_traits@D@std@@V?$allocator@D@2@@std@@QAEAAV12@ID@Z 10018f20 f i IO61X_Library_MSVC120_vc:IO61X_DriverObject.obj
 0001:00017fd0       ?append@?$basic_string@DU?$char_traits@D@std@@V?$allocator@D@2@@std@@QAEAAV12@PBD@Z 10018fd0 f i IO61X_Library_MSVC120_vc:IO61X_DriverObject.obj
 0001:00018010       ?append@?$basic_string@DU?$char_traits@D@std@@V?$allocator@D@2@@std@@QAEAAV12@PBDI@Z 10019010 f i IO61X_Library_MSVC120_vc:IO61X_DriverObject.obj
 0001:00018100       ?assign@?$basic_string@DU?$char_traits@D@std@@V?$allocator@D@2@@std@@QAEAAV12@ID@Z 10019100 f i IO61X_Library_MSVC120_vc:IO61X_DriverObject.obj
 0001:000181d0       ?assign@?$char_traits@D@std@@SAPADPADID@Z 100191d0 f i IO61X_Library_MSVC120_vc:IO61X_DriverObject.obj
 0001:000181f0       ?atomic_fetch_add_explicit@std@@YAHPAUatomic_int@1@HW4memory_order@1@@Z 100191f0 f i IO61X_Library_MSVC120_vc:IO61X_DriverObject.obj
 0001:00018230       ?atomic_load@std@@YA_NPBUatomic_bool@1@@Z 10019230 f i IO61X_Library_MSVC120_vc:IO61X_DriverObject.obj
 0001:00018240       ?atomic_load_explicit@std@@YAHPBUatomic_int@1@W4memory_order@1@@Z 10019240 f i IO61X_Library_MSVC120_vc:IO61X_DriverObject.obj
 0001:00018280       ?atomic_load_explicit@std@@YA_NPBUatomic_bool@1@W4memory_order@1@@Z 10019280 f i IO61X_Library_MSVC120_vc:IO61X_DriverObject.obj
 0001:000182d0       ?atomic_store@std@@YAXPAUatomic_bool@1@_N@Z 100192d0 f i IO61X_Library_MSVC120_vc:IO61X_DriverObject.obj
 0001:000182e0       ?atomic_store_explicit@std@@YAXPAUatomic_bool@1@_NW4memory_order@1@@Z 100192e0 f i IO61X_Library_MSVC120_vc:IO61X_DriverObject.obj
 0001:00018310       ?begin@?$basic_string@DU?$char_traits@D@std@@V?$allocator@D@2@@std@@QAE?AV?$_String_iterator@V?$_String_val@U?$_Simple_types@D@std@@@std@@@2@XZ 10019310 f i IO61X_Library_MSVC120_vc:IO61X_DriverObject.obj
 0001:00018330       ?c_str@?$_Yarn@D@std@@QBEPBDXZ 10019330 f i IO61X_Library_MSVC120_vc:IO61X_DriverObject.obj
 0001:00018340       ?c_str@?$basic_string@DU?$char_traits@D@std@@V?$allocator@D@2@@std@@QBEPBDXZ 10019340 f i IO61X_Library_MSVC120_vc:IO61X_DriverObject.obj
 0001:00018350       ?c_str@locale@std@@QBEPBDXZ 10019350 f i IO61X_Library_MSVC120_vc:IO61X_DriverObject.obj
 0001:00018370       ?clear@?$basic_ios@DU?$char_traits@D@std@@@std@@QAEXH_N@Z 10019370 f i IO61X_Library_MSVC120_vc:IO61X_DriverObject.obj
 0001:00018390       ?clear@ios_base@std@@QAEXH@Z 10019390 f i IO61X_Library_MSVC120_vc:IO61X_DriverObject.obj
 0001:00018410       ?clear@ios_base@std@@QAEXH_N@Z 10019410 f i IO61X_Library_MSVC120_vc:IO61X_DriverObject.obj
 0001:000184a0       ?close@?$basic_filebuf@DU?$char_traits@D@std@@@std@@QAEPAV12@XZ 100194a0 f i IO61X_Library_MSVC120_vc:IO61X_DriverObject.obj
 0001:00018550       ?close@?$basic_ofstream@DU?$char_traits@D@std@@@std@@QAEXXZ 10019550 f i IO61X_Library_MSVC120_vc:IO61X_DriverObject.obj
 0001:00018600       ?dbg@IO61X_Logger@@QAAXPBDZZ 10019600 f   IO61X_Library_MSVC120_vc:IO61X_DriverObject.obj
 0001:000186d0       ?deinit@IO61X_DriverObject@@QAEXXZ 100196d0 f   IO61X_Library_MSVC120_vc:IO61X_DriverObject.obj
 0001:00018890       ?disable@IO61X_Logger@@QAEXXZ 10019890 f i IO61X_Library_MSVC120_vc:IO61X_DriverObject.obj
 0001:000188b0       ?do_always_noconv@?$codecvt@DDH@std@@MBE_NXZ 100198b0 f i IO61X_Library_MSVC120_vc:IO61X_DriverObject.obj
 0001:000188c0       ?do_always_noconv@codecvt_base@std@@MBE_NXZ 100198c0 f i IO61X_Library_MSVC120_vc:IO61X_DriverObject.obj
 0001:000188d0       ?do_encoding@codecvt_base@std@@MBEHXZ 100198d0 f i IO61X_Library_MSVC120_vc:IO61X_DriverObject.obj
 0001:000188e0       ?do_in@?$codecvt@DDH@std@@MBEHAAHPBD1AAPBDPAD3AAPAD@Z 100198e0 f i IO61X_Library_MSVC120_vc:IO61X_DriverObject.obj
 0001:00018900       ?do_length@?$codecvt@DDH@std@@MBEHAAHPBD1I@Z 10019900 f i IO61X_Library_MSVC120_vc:IO61X_DriverObject.obj
 0001:00018920       ?do_max_length@codecvt_base@std@@MBEHXZ 10019920 f i IO61X_Library_MSVC120_vc:IO61X_DriverObject.obj
 0001:00018930       ?do_narrow@?$ctype@D@std@@MBEDDD@Z 10019930 f i IO61X_Library_MSVC120_vc:IO61X_DriverObject.obj
 0001:00018940       ?do_narrow@?$ctype@D@std@@MBEPBDPBD0DPAD@Z 10019940 f i IO61X_Library_MSVC120_vc:IO61X_DriverObject.obj
 0001:00018960       ?do_out@?$codecvt@DDH@std@@MBEHAAHPBD1AAPBDPAD3AAPAD@Z 10019960 f i IO61X_Library_MSVC120_vc:IO61X_DriverObject.obj
 0001:00018980       ?do_tolower@?$ctype@D@std@@MBEDD@Z 10019980 f i IO61X_Library_MSVC120_vc:IO61X_DriverObject.obj
 0001:000189a0       ?do_tolower@?$ctype@D@std@@MBEPBDPADPBD@Z 100199a0 f i IO61X_Library_MSVC120_vc:IO61X_DriverObject.obj
 0001:000189f0       ?do_toupper@?$ctype@D@std@@MBEDD@Z 100199f0 f i IO61X_Library_MSVC120_vc:IO61X_DriverObject.obj
 0001:00018a10       ?do_toupper@?$ctype@D@std@@MBEPBDPADPBD@Z 10019a10 f i IO61X_Library_MSVC120_vc:IO61X_DriverObject.obj
 0001:00018a60       ?do_unshift@?$codecvt@DDH@std@@MBEHAAHPAD1AAPAD@Z 10019a60 f i IO61X_Library_MSVC120_vc:IO61X_DriverObject.obj
 0001:00018a80       ?do_widen@?$ctype@D@std@@MBEDD@Z 10019a80 f i IO61X_Library_MSVC120_vc:IO61X_DriverObject.obj
 0001:00018a90       ?do_widen@?$ctype@D@std@@MBEPBDPBD0PAD@Z 10019a90 f i IO61X_Library_MSVC120_vc:IO61X_DriverObject.obj
 0001:00018ab0       ?eback@?$basic_streambuf@DU?$char_traits@D@std@@@std@@IBEPADXZ 10019ab0 f i IO61X_Library_MSVC120_vc:IO61X_DriverObject.obj
 0001:00018ac0       ?egptr@?$basic_streambuf@DU?$char_traits@D@std@@@std@@IBEPADXZ 10019ac0 f i IO61X_Library_MSVC120_vc:IO61X_DriverObject.obj
 0001:00018ad0       ?empty@?$basic_string@DU?$char_traits@D@std@@V?$allocator@D@2@@std@@QBE_NXZ 10019ad0 f i IO61X_Library_MSVC120_vc:IO61X_DriverObject.obj
 0001:00018ae0       ?eof@?$char_traits@D@std@@SAHXZ 10019ae0 f i IO61X_Library_MSVC120_vc:IO61X_DriverObject.obj
 0001:00018af0       ?epptr@?$basic_streambuf@DU?$char_traits@D@std@@@std@@IBEPADXZ 10019af0 f i IO61X_Library_MSVC120_vc:IO61X_DriverObject.obj
 0001:00018b00       ?eq_int_type@?$char_traits@D@std@@SA_NABH0@Z 10019b00 f i IO61X_Library_MSVC120_vc:IO61X_DriverObject.obj
 0001:00018b20       ?err@IO61X_Logger@@QAAXPBDZZ 10019b20 f   IO61X_Library_MSVC120_vc:IO61X_DriverObject.obj
 0001:00018b80       ?fetch_add@atomic_int@std@@QAEHHW4memory_order@2@@Z 10019b80 f i IO61X_Library_MSVC120_vc:IO61X_DriverObject.obj
 0001:00018bc0       ?fill@?$basic_ios@DU?$char_traits@D@std@@@std@@QBEDXZ 10019bc0 f i IO61X_Library_MSVC120_vc:IO61X_DriverObject.obj
 0001:00018bd0       ?flags@ios_base@std@@QBEHXZ 10019bd0 f i IO61X_Library_MSVC120_vc:IO61X_DriverObject.obj
 0001:00018be0       ?flush@?$basic_ostream@DU?$char_traits@D@std@@@std@@QAEAAV12@XZ 10019be0 f i IO61X_Library_MSVC120_vc:IO61X_DriverObject.obj
 0001:00018d40       ?flush@IO61X_Logger@@QAEXXZ 10019d40 f   IO61X_Library_MSVC120_vc:IO61X_DriverObject.obj
 0001:00018fb0       ?gbump@?$basic_streambuf@DU?$char_traits@D@std@@@std@@IAEXH@Z 10019fb0 f i IO61X_Library_MSVC120_vc:IO61X_DriverObject.obj
 0001:00018fd0       ?getReadIdx@?$IO61X_LoggerFifo@ULogLine@@@@QAEHXZ 10019fd0 f i IO61X_Library_MSVC120_vc:IO61X_DriverObject.obj
 0001:00018fe0       ?getloc@?$basic_streambuf@DU?$char_traits@D@std@@@std@@QBE?AVlocale@2@XZ 10019fe0 f i IO61X_Library_MSVC120_vc:IO61X_DriverObject.obj
 0001:00019010       ?getloc@ios_base@std@@QBE?AVlocale@2@XZ 1001a010 f i IO61X_Library_MSVC120_vc:IO61X_DriverObject.obj
 0001:00019040       ?good@ios_base@std@@QBE_NXZ 1001a040 f i IO61X_Library_MSVC120_vc:IO61X_DriverObject.obj
 0001:00019050       ?gptr@?$basic_streambuf@DU?$char_traits@D@std@@@std@@IBEPADXZ 1001a050 f i IO61X_Library_MSVC120_vc:IO61X_DriverObject.obj
 0001:00019060       ?imbue@?$basic_filebuf@DU?$char_traits@D@std@@@std@@MAEXABVlocale@2@@Z 1001a060 f i IO61X_Library_MSVC120_vc:IO61X_DriverObject.obj
 0001:000190a0       ?imbue@?$basic_streambuf@DU?$char_traits@D@std@@@std@@MAEXABVlocale@2@@Z 1001a0a0 f i IO61X_Library_MSVC120_vc:IO61X_DriverObject.obj
 0001:000190b0       ?in@?$codecvt@DDH@std@@QBEHAAHPBD1AAPBDPAD3AAPAD@Z 1001a0b0 f i IO61X_Library_MSVC120_vc:IO61X_DriverObject.obj
 0001:000190c0       ?info@IO61X_Logger@@QAAXPBDZZ 1001a0c0 f   IO61X_Library_MSVC120_vc:IO61X_DriverObject.obj
 0001:00019120       ?init@?$basic_ios@DU?$char_traits@D@std@@@std@@IAEXPAV?$basic_streambuf@DU?$char_traits@D@std@@@2@_N@Z 1001a120 f i IO61X_Library_MSVC120_vc:IO61X_DriverObject.obj
 0001:00019240       ?iostream_category@std@@YAABVerror_category@1@XZ 1001a240 f i IO61X_Library_MSVC120_vc:IO61X_DriverObject.obj
 0001:00019250       ?is_open@?$basic_filebuf@DU?$char_traits@D@std@@@std@@QBE_NXZ 1001a250 f i IO61X_Library_MSVC120_vc:IO61X_DriverObject.obj
 0001:00019260       ?is_open@?$basic_ofstream@DU?$char_traits@D@std@@@std@@QBE_NXZ 1001a260 f i IO61X_Library_MSVC120_vc:IO61X_DriverObject.obj
 0001:00019270       ?load@atomic_int@std@@QBEHW4memory_order@2@@Z 1001a270 f i IO61X_Library_MSVC120_vc:IO61X_DriverObject.obj
 0001:000192b0       ?log@IO61X_Logger@@QAEXHPBD@Z 1001a2b0 f   IO61X_Library_MSVC120_vc:IO61X_DriverObject.obj
 0001:00019410       ?make_error_code@std@@YA?AVerror_code@1@W4io_errc@1@@Z 1001a410 f i IO61X_Library_MSVC120_vc:IO61X_DriverObject.obj
 0001:00019430       ?message@error_code@std@@QBE?AV?$basic_string@DU?$char_traits@D@std@@V?$allocator@D@2@@2@XZ 1001a430 f i IO61X_Library_MSVC120_vc:IO61X_DriverObject.obj
 0001:00019460       ?not_eof@?$char_traits@D@std@@SAHABH@Z 1001a460 f i IO61X_Library_MSVC120_vc:IO61X_DriverObject.obj
 0001:00019480       ?open@?$basic_filebuf@DU?$char_traits@D@std@@@std@@QAEPAV12@PBDHH@Z 1001a480 f i IO61X_Library_MSVC120_vc:IO61X_DriverObject.obj
 0001:00019560       ?out@?$codecvt@DDH@std@@QBEHAAHPBD1AAPBDPAD3AAPAD@Z 1001a560 f i IO61X_Library_MSVC120_vc:IO61X_DriverObject.obj
 0001:00019570       ?overflow@?$basic_filebuf@DU?$char_traits@D@std@@@std@@MAEHH@Z 1001a570 f i IO61X_Library_MSVC120_vc:IO61X_DriverObject.obj
 0001:00019760       ?overflow@?$basic_streambuf@DU?$char_traits@D@std@@@std@@MAEHH@Z 1001a760 f i IO61X_Library_MSVC120_vc:IO61X_DriverObject.obj
 0001:00019770       ?pbackfail@?$basic_filebuf@DU?$char_traits@D@std@@@std@@MAEHH@Z 1001a770 f i IO61X_Library_MSVC120_vc:IO61X_DriverObject.obj
 0001:00019800       ?pbackfail@?$basic_streambuf@DU?$char_traits@D@std@@@std@@MAEHH@Z 1001a800 f i IO61X_Library_MSVC120_vc:IO61X_DriverObject.obj
 0001:00019810       ?pbump@?$basic_streambuf@DU?$char_traits@D@std@@@std@@IAEXH@Z 1001a810 f i IO61X_Library_MSVC120_vc:IO61X_DriverObject.obj
 0001:00019830       ?pptr@?$basic_streambuf@DU?$char_traits@D@std@@@std@@IBEPADXZ 1001a830 f i IO61X_Library_MSVC120_vc:IO61X_DriverObject.obj
 0001:00019840       ?pubsync@?$basic_streambuf@DU?$char_traits@D@std@@@std@@QAEHXZ 1001a840 f i IO61X_Library_MSVC120_vc:IO61X_DriverObject.obj
 0001:00019850       ?rdbuf@?$basic_ios@DU?$char_traits@D@std@@@std@@QBEPAV?$basic_streambuf@DU?$char_traits@D@std@@@2@XZ 1001a850 f i IO61X_Library_MSVC120_vc:IO61X_DriverObject.obj
 0001:00019860       ?rdstate@ios_base@std@@QBEHXZ 1001a860 f i IO61X_Library_MSVC120_vc:IO61X_DriverObject.obj
 0001:00019870       ?seekoff@?$basic_filebuf@DU?$char_traits@D@std@@@std@@MAE?AV?$fpos@H@2@_JHH@Z 1001a870 f i IO61X_Library_MSVC120_vc:IO61X_DriverObject.obj
 0001:00019970       ?seekoff@?$basic_streambuf@DU?$char_traits@D@std@@@std@@MAE?AV?$fpos@H@2@_JHH@Z 1001a970 f i IO61X_Library_MSVC120_vc:IO61X_DriverObject.obj
 0001:000199a0       ?seekpos@?$basic_filebuf@DU?$char_traits@D@std@@@std@@MAE?AV?$fpos@H@2@V32@H@Z 1001a9a0 f i IO61X_Library_MSVC120_vc:IO61X_DriverObject.obj
 0001:00019a80       ?seekpos@?$basic_streambuf@DU?$char_traits@D@std@@@std@@MAE?AV?$fpos@H@2@V32@H@Z 1001aa80 f i IO61X_Library_MSVC120_vc:IO61X_DriverObject.obj
 0001:00019ab0       ?seekpos@?$fpos@H@std@@QBE_JXZ 1001aab0 f i IO61X_Library_MSVC120_vc:IO61X_DriverObject.obj
 0001:00019ac0       ?select_on_container_copy_construction@?$_Wrap_alloc@V?$allocator@D@std@@@std@@QBE?AU12@XZ 1001aac0 f i IO61X_Library_MSVC120_vc:IO61X_DriverObject.obj
 0001:00019ad0       ?select_on_container_copy_construction@?$allocator@D@std@@QBE?AV12@XZ 1001aad0 f i IO61X_Library_MSVC120_vc:IO61X_DriverObject.obj
 0001:00019ae0       ?select_on_container_copy_construction@?$allocator_traits@V?$allocator@D@std@@@std@@SA?AV?$allocator@D@2@ABV32@@Z 1001aae0 f i IO61X_Library_MSVC120_vc:IO61X_DriverObject.obj
 0001:00019af0       ?setBuffered@IO61X_Logger@@QAEXPBDH@Z 1001aaf0 f   IO61X_Library_MSVC120_vc:IO61X_DriverObject.obj
 0001:00019c60       ?setReadIdx@?$IO61X_LoggerFifo@ULogLine@@@@QAEXH@Z 1001ac60 f i IO61X_Library_MSVC120_vc:IO61X_DriverObject.obj
 0001:00019c70       ?setbuf@?$basic_filebuf@DU?$char_traits@D@std@@@std@@MAEPAV?$basic_streambuf@DU?$char_traits@D@std@@@2@PAD_J@Z 1001ac70 f i IO61X_Library_MSVC120_vc:IO61X_DriverObject.obj
 0001:00019cc0       ?setbuf@?$basic_streambuf@DU?$char_traits@D@std@@@std@@MAEPAV12@PAD_J@Z 1001acc0 f i IO61X_Library_MSVC120_vc:IO61X_DriverObject.obj
 0001:00019cd0       ?setg@?$basic_streambuf@DU?$char_traits@D@std@@@std@@IAEXPAD00@Z 1001acd0 f i IO61X_Library_MSVC120_vc:IO61X_DriverObject.obj
 0001:00019d00       ?setp@?$basic_streambuf@DU?$char_traits@D@std@@@std@@IAEXPAD0@Z 1001ad00 f i IO61X_Library_MSVC120_vc:IO61X_DriverObject.obj
 0001:00019d20       ?setstate@?$basic_ios@DU?$char_traits@D@std@@@std@@QAEXH_N@Z 1001ad20 f i IO61X_Library_MSVC120_vc:IO61X_DriverObject.obj
 0001:00019d50       ?showmanyc@?$basic_streambuf@DU?$char_traits@D@std@@@std@@MAE_JXZ 1001ad50 f i IO61X_Library_MSVC120_vc:IO61X_DriverObject.obj
 0001:00019d60       ?sputc@?$basic_streambuf@DU?$char_traits@D@std@@@std@@QAEHD@Z 1001ad60 f i IO61X_Library_MSVC120_vc:IO61X_DriverObject.obj
 0001:00019da0       ?sputn@?$basic_streambuf@DU?$char_traits@D@std@@@std@@QAE_JPBD_J@Z 1001ada0 f i IO61X_Library_MSVC120_vc:IO61X_DriverObject.obj
 0001:00019dc0       ?state@?$fpos@H@std@@QBEHXZ 1001adc0 f i IO61X_Library_MSVC120_vc:IO61X_DriverObject.obj
 0001:00019dd0       ?store@atomic_int@std@@QAEXHW4memory_order@2@@Z 1001add0 f i IO61X_Library_MSVC120_vc:IO61X_DriverObject.obj
 0001:00019e00       ?sync@?$basic_filebuf@DU?$char_traits@D@std@@@std@@MAEHXZ 1001ae00 f i IO61X_Library_MSVC120_vc:IO61X_DriverObject.obj
 0001:00019e30       ?sync@?$basic_streambuf@DU?$char_traits@D@std@@@std@@MAEHXZ 1001ae30 f i IO61X_Library_MSVC120_vc:IO61X_DriverObject.obj
 0001:00019e40       ?tie@?$basic_ios@DU?$char_traits@D@std@@@std@@QBEPAV?$basic_ostream@DU?$char_traits@D@std@@@2@XZ 1001ae40 f i IO61X_Library_MSVC120_vc:IO61X_DriverObject.obj
 0001:00019e50       ?to_char_type@?$char_traits@D@std@@SADABH@Z 1001ae50 f i IO61X_Library_MSVC120_vc:IO61X_DriverObject.obj
 0001:00019e60       ?to_int_type@?$char_traits@D@std@@SAHABD@Z 1001ae60 f i IO61X_Library_MSVC120_vc:IO61X_DriverObject.obj
 0001:00019e70       ?uflow@?$basic_filebuf@DU?$char_traits@D@std@@@std@@MAEHXZ 1001ae70 f i IO61X_Library_MSVC120_vc:IO61X_DriverObject.obj
 0001:0001a060       ?uflow@?$basic_streambuf@DU?$char_traits@D@std@@@std@@MAEHXZ 1001b060 f i IO61X_Library_MSVC120_vc:IO61X_DriverObject.obj
 0001:0001a090       ?underflow@?$basic_filebuf@DU?$char_traits@D@std@@@std@@MAEHXZ 1001b090 f i IO61X_Library_MSVC120_vc:IO61X_DriverObject.obj
 0001:0001a0d0       ?underflow@?$basic_streambuf@DU?$char_traits@D@std@@@std@@MAEHXZ 1001b0d0 f i IO61X_Library_MSVC120_vc:IO61X_DriverObject.obj
 0001:0001a0e0       ?unshift@?$codecvt@DDH@std@@QBEHAAHPAD1AAPAD@Z 1001b0e0 f i IO61X_Library_MSVC120_vc:IO61X_DriverObject.obj
 0001:0001a0f0       ?useTargetDefaults@IO61X_Logger@@QAEXXZ 1001b0f0 f   IO61X_Library_MSVC120_vc:IO61X_DriverObject.obj
 0001:0001a120       ?warn@IO61X_Logger@@QAAXPBDZZ 1001b120 f   IO61X_Library_MSVC120_vc:IO61X_DriverObject.obj
 0001:0001a180       ?widen@?$basic_ios@DU?$char_traits@D@std@@@std@@QBEDD@Z 1001b180 f i IO61X_Library_MSVC120_vc:IO61X_DriverObject.obj
 0001:0001a200       ?widen@?$ctype@D@std@@QBEDD@Z 1001b200 f i IO61X_Library_MSVC120_vc:IO61X_DriverObject.obj
 0001:0001a210       ?width@ios_base@std@@QAE_J_J@Z 1001b210 f i IO61X_Library_MSVC120_vc:IO61X_DriverObject.obj
 0001:0001a230       ?width@ios_base@std@@QBE_JXZ 1001b230 f i IO61X_Library_MSVC120_vc:IO61X_DriverObject.obj
 0001:0001a240       ?xsgetn@?$basic_streambuf@DU?$char_traits@D@std@@@std@@MAE_JPAD_J@Z 1001b240 f i IO61X_Library_MSVC120_vc:IO61X_DriverObject.obj
 0001:0001a330       ?xsputn@?$basic_streambuf@DU?$char_traits@D@std@@@std@@MAE_JPBD_J@Z 1001b330 f i IO61X_Library_MSVC120_vc:IO61X_DriverObject.obj
 0001:0001a420       ??0IO61X_HEXARRAY@@QAE@PBDII@Z 1001b420 f i IO61X_Library_MSVC120_vc:IO61X_ModuleManager.obj
 0001:0001a470       ?IO61X_AddModuleToModuleList@@YA_NIEPAIFFPBDPAD@Z 1001b470 f   IO61X_Library_MSVC120_vc:IO61X_ModuleManager.obj
 0001:0001a600       ?IO61X_CheckFirmwareData@@YA_NABUIO61X_FW_INFO@@ABUIO61X_HEXARRAY@@AAI@Z 1001b600 f   IO61X_Library_MSVC120_vc:IO61X_ModuleManager.obj
 0001:0001a7a0       ?IO61X_CheckIsFwRunning@@YA_NI@Z 1001b7a0 f   IO61X_Library_MSVC120_vc:IO61X_ModuleManager.obj
 0001:0001a8b0       ?IO61X_CheckModuleArryForId@@YA_NIPAIPBD@Z 1001b8b0 f   IO61X_Library_MSVC120_vc:IO61X_ModuleManager.obj
 0001:0001a940       ?IO61X_CheckModuleExpansions@@YA_NIPAD@Z 1001b940 f   IO61X_Library_MSVC120_vc:IO61X_ModuleManager.obj
 0001:0001ab40       ?IO61X_CreateModulePortArray@@YA_NI@Z 1001bb40 f   IO61X_Library_MSVC120_vc:IO61X_ModuleManager.obj
 0001:0001ac80       ?IO61X_DoEstablishDma@@YA_NII@Z 1001bc80 f   IO61X_Library_MSVC120_vc:IO61X_ModuleManager.obj
 0001:0001ad70       ?IO61X_DoModuleInitialization@@YA_NIPAD@Z 1001bd70 f   IO61X_Library_MSVC120_vc:IO61X_ModuleManager.obj
 0001:0001ae00       ?IO61X_DownloadFirmwareToMC@@YA_NPBUIO61X_PciObject_T@@ABUIO61X_FW_INFO@@ABUIO61X_HEXARRAY@@I@Z 1001be00 f   IO61X_Library_MSVC120_vc:IO61X_ModuleManager.obj
 0001:0001af10       ?IO61X_EstablishDma@@YA_NIPAD@Z 1001bf10 f   IO61X_Library_MSVC120_vc:IO61X_ModuleManager.obj
 0001:0001b0f0       ?IO61X_GetDmaInfoFromMC@@YAXPBUIO61X_PciObject_T@@PAIPAG@Z 1001c0f0 f   IO61X_Library_MSVC120_vc:IO61X_ModuleManager.obj
 0001:0001b1b0       ?IO61X_GetFirmware@@YAPAUIO61X_HEXARRAY@@AAUIO61X_FW_INFO@@@Z 1001c1b0 f   IO61X_Library_MSVC120_vc:IO61X_ModuleManager.obj
 0001:0006e4d0       ?IO61X_GetModuleCapabilities@@YA_NIPAD@Z 1006f4d0 f   IO61X_Library_MSVC120_vc:IO61X_ModuleManager.obj
 0001:0006e5f0       ?IO61X_GetPciDeviceData@@YA_NIFFPAD@Z 1006f5f0 f   IO61X_Library_MSVC120_vc:IO61X_ModuleManager.obj
 0001:0006e850       ?IO61X_LoadAndStartFirmware@@YA_NIPAD@Z 1006f850 f   IO61X_Library_MSVC120_vc:IO61X_ModuleManager.obj
 0001:0006e940       ?IO61X_LoadFirmwareToMC@@YA_NI@Z 1006f940 f   IO61X_Library_MSVC120_vc:IO61X_ModuleManager.obj
 0001:0006e9f0       ?IO61X_ModuleGetAndSetPortQuantity@@YA_NIPAD@Z 1006f9f0 f   IO61X_Library_MSVC120_vc:IO61X_ModuleManager.obj
 0001:0006ea50       ?IO61X_RegisterDma@@YA_NPAUIO61X_PciObject_T@@@Z 1006fa50 f   IO61X_Library_MSVC120_vc:IO61X_ModuleManager.obj
 0001:0006eb20       ?IO61X_RequestDmaSizeFromMC@@YA_NIAAI@Z 1006fb20 f   IO61X_Library_MSVC120_vc:IO61X_ModuleManager.obj
 0001:0006ec70       ?IO61X_RequestModuleCapabilities@@YA_NPBUIO61X_PciObject_T@@@Z 1006fc70 f   IO61X_Library_MSVC120_vc:IO61X_ModuleManager.obj
 0001:0006edc0       ?IO61X_ResetMC@@YAXPBUIO61X_PciObject_T@@@Z 1006fdc0 f   IO61X_Library_MSVC120_vc:IO61X_ModuleManager.obj
 0001:0006ee40       ?IO61X_SetLinRwwbMailbox@@YA_NII@Z 1006fe40 f   IO61X_Library_MSVC120_vc:IO61X_ModuleManager.obj
 0001:0006ef70       ?IO61X_SetModulePortMailboxesTxRx@@YA_NIEEI@Z 1006ff70 f   IO61X_Library_MSVC120_vc:IO61X_ModuleManager.obj
 0001:0006f200       ?IO61X_StartCan@@YA_NIEW4IO61X_PtMbxDirecVals_E@@I@Z 10070200 f   IO61X_Library_MSVC120_vc:IO61X_ModuleManager.obj
 0001:0006f360       ?IO61X_StartFirmware@@YA_NI@Z 10070360 f   IO61X_Library_MSVC120_vc:IO61X_ModuleManager.obj
 0001:0006f470       ?IO61X_StopCan@@YA_NIEW4IO61X_PtMbxDirecVals_E@@I@Z 10070470 f   IO61X_Library_MSVC120_vc:IO61X_ModuleManager.obj
 0001:0006f560       ?IO61X_TestBasicInitializationOfModule@@YA_NI@Z 10070560 f   IO61X_Library_MSVC120_vc:IO61X_ModuleManager.obj
 0001:0006f610       ?IO61X_TestDMARdCmd@@YA_NPBUIO61X_PciObject_T@@W4IO61X_PtMbxDirecVals_E@@@Z 10070610 f   IO61X_Library_MSVC120_vc:IO61X_ModuleManager.obj
 0001:0006f7a0       ?IO61X_TestDMAWrtCmd@@YA_NPBUIO61X_PciObject_T@@W4IO61X_PtMbxDirecVals_E@@@Z 100707a0 f   IO61X_Library_MSVC120_vc:IO61X_ModuleManager.obj
 0001:0006f900       ?IO61X_TestModuleCommandMailbox@@YA_NPBUIO61X_PciObject_T@@W4IO61X_PtMbxDirecVals_E@@@Z 10070900 f   IO61X_Library_MSVC120_vc:IO61X_ModuleManager.obj
 0001:0006fa70       ?_Atomic_exchange_4@std@@YAKPCKKW4memory_order@1@@Z 10070a70 f i IO61X_Library_MSVC120_vc:IO61X_ModuleManager.obj
 0001:0006fab0       ?_Atomic_thread_fence@std@@YAXW4memory_order@1@@Z 10070ab0 f i IO61X_Library_MSVC120_vc:IO61X_ModuleManager.obj
 0001:0006fad0       ?_Exchange_acquire_4@std@@YAKPCKK@Z 10070ad0 f i IO61X_Library_MSVC120_vc:IO61X_ModuleManager.obj
 0001:0006fae0       ?_Exchange_relaxed_4@std@@YAKPCKK@Z 10070ae0 f i IO61X_Library_MSVC120_vc:IO61X_ModuleManager.obj
 0001:0006faf0       ?_Exchange_release_4@std@@YAKPCKK@Z 10070af0 f i IO61X_Library_MSVC120_vc:IO61X_ModuleManager.obj
 0001:0006fb00       ?_Exchange_seq_cst_4@std@@YAKPCKK@Z 10070b00 f i IO61X_Library_MSVC120_vc:IO61X_ModuleManager.obj
 0001:0006fb10       ?set@IO61X_HEXARRAY@@QAEXHGIPAE@Z 10070b10 f i IO61X_Library_MSVC120_vc:IO61X_ModuleManager.obj
 0001:0006fb50       _atomic_thread_fence       10070b50 f i IO61X_Library_MSVC120_vc:IO61X_ModuleManager.obj
 0001:0006fb70       ?IO61X_CanAllocatePortMemory@@YA_NIE@Z 10070b70 f   IO61X_Library_MSVC120_vc:IO61X_CanManager.obj
 0001:0006fc60       ?IO61X_CanSendReceivePortStatusInfo@@YA_NIW4IO61X_PtMbxDirecVals_E@@I@Z 10070c60 f   IO61X_Library_MSVC120_vc:IO61X_CanManager.obj
 0001:0006fe90       ?IO61X_InitializeCan@@YA_NIEW4IO61X_PtMbxDirecVals_E@@I@Z 10070e90 f   IO61X_Library_MSVC120_vc:IO61X_CanManager.obj
 0001:00070090       ?IO61X_InitializeCanController@@YA_NIEPAD@Z 10071090 f   IO61X_Library_MSVC120_vc:IO61X_CanManager.obj
 0001:00070130       ?IO61X_ReadCanFdMessageFromReceiveQueue@@YAEPAUIO61X_ComMbxObj_T@@PAUIO61X_CANFDMsgSndRecPkt_T@@@Z 10071130 f   IO61X_Library_MSVC120_vc:IO61X_CanManager.obj
 0001:000701a0       ?IO61X_ReadCanMessageFromReceiveQueue@@YAEPAUIO61X_ComMbxObj_T@@PAUIO61X_CANMsgRecPkt_T@@@Z 100711a0 f   IO61X_Library_MSVC120_vc:IO61X_CanManager.obj
 0001:00070220       ?IO61X_SetCanAcceptanceMaskAndCode@@YA_NIE_NW4IO61X_PtMbxDirecVals_E@@I@Z 10071220 f   IO61X_Library_MSVC120_vc:IO61X_CanManager.obj
 0001:000703b0       ?IO61X_SetCanFdPortValues@@YAXIEGGGGNG@Z 100713b0 f   IO61X_Library_MSVC120_vc:IO61X_CanManager.obj
 0001:000704f0       ?IO61X_SetCanPortValues@@YA_NIEEEGGGGIIII@Z 100714f0 f   IO61X_Library_MSVC120_vc:IO61X_CanManager.obj
 0001:00070650       ?IO61X_WriteCanFdMessageToSendQueue@@YAEPBEPCIPAUIO61X_ComMbxObj_T@@@Z 10071650 f   IO61X_Library_MSVC120_vc:IO61X_CanManager.obj
 0001:000706d0       ?IO61X_WriteCanMessageToSendQueue@@YAEPBEPCIPAUIO61X_ComMbxObj_T@@@Z 100716d0 f   IO61X_Library_MSVC120_vc:IO61X_CanManager.obj
 0001:00070720       ??0?$_Atomic@N$07@std@@QAE@N@Z 10071720 f i IO61X_Library_MSVC120_vc:IO61X_Port.obj
 0001:00070740       ??0?$atomic@N@std@@QAE@N@Z 10071740 f i IO61X_Library_MSVC120_vc:IO61X_Port.obj
 0001:00070760       ??0IO61X_Port@@QAE@II@Z    10071760 f   IO61X_Library_MSVC120_vc:IO61X_Port.obj
 0001:00070790       ??1IO61X_Port@@UAE@XZ      10071790 f   IO61X_Library_MSVC120_vc:IO61X_Port.obj
 0001:000707a0       ??_EIO61X_Port@@UAEPAXI@Z  100717a0 f i IO61X_Library_MSVC120_vc:IO61X_Port.obj
 0001:000707a0       ??_GIO61X_Port@@UAEPAXI@Z  100717a0 f i IO61X_Library_MSVC120_vc:IO61X_Port.obj
 0001:000707d0       ?GetTimeStamp@IO61X_Port@@QAENXZ 100717d0 f   IO61X_Library_MSVC120_vc:IO61X_Port.obj
 0001:000707e0       ?ReleaseLockFlag@IO61X_Port@@QAEXXZ 100717e0 f   IO61X_Library_MSVC120_vc:IO61X_Port.obj
 0001:000707f0       ?SpinLock@IO61X_Port@@QAEHXZ 100717f0 f   IO61X_Library_MSVC120_vc:IO61X_Port.obj
 0001:00070810       ?_Atomic_flag_clear@std@@YAXPCJW4memory_order@1@@Z 10071810 f i IO61X_Library_MSVC120_vc:IO61X_Port.obj
 0001:00070850       ?_Atomic_flag_test_and_set@std@@YAHPCJW4memory_order@1@@Z 10071850 f i IO61X_Library_MSVC120_vc:IO61X_Port.obj
 0001:00070890       ?clear@atomic_flag@std@@QAEXW4memory_order@2@@Z 10071890 f i IO61X_Library_MSVC120_vc:IO61X_Port.obj
 0001:000708d0       ?test_and_set@atomic_flag@std@@QAE_NW4memory_order@2@@Z 100718d0 f i IO61X_Library_MSVC120_vc:IO61X_Port.obj
 0001:00070920       ??$_Allocate@U?$_List_node@V?$IO61X_BufferFifo@UIO61X_CanMessage_T@@@@PAX@std@@@std@@YAPAU?$_List_node@V?$IO61X_BufferFifo@UIO61X_CanMessage_T@@@@PAX@0@IPAU10@@Z 10071920 f i IO61X_Library_MSVC120_vc:IO61X_CanPort.obj
 0001:00070960       ??$_Buynode@V?$IO61X_BufferFifo@UIO61X_CanMessage_T@@@@@?$_List_buy@V?$IO61X_BufferFifo@UIO61X_CanMessage_T@@@@V?$allocator@V?$IO61X_BufferFifo@UIO61X_CanMessage_T@@@@@std@@@std@@QAEPAU?$_List_node@V?$IO61X_BufferFifo@UIO61X_CanMessage_T@@@@PAX@1@PAU21@0$$QAV?$IO61X_BufferFifo@UIO61X_CanMessage_T@@@@@Z 10071960 f i IO61X_Library_MSVC120_vc:IO61X_CanPort.obj
 0001:000709f0       ??$_Insert@V?$IO61X_BufferFifo@UIO61X_CanMessage_T@@@@@?$list@V?$IO61X_BufferFifo@UIO61X_CanMessage_T@@@@V?$allocator@V?$IO61X_BufferFifo@UIO61X_CanMessage_T@@@@@std@@@std@@QAEXV?$_List_unchecked_const_iterator@V?$_List_val@U?$_List_simple_types@V?$IO61X_BufferFifo@UIO61X_CanMessage_T@@@@@std@@@std@@U_Iterator_base0@2@@1@$$QAV?$IO61X_BufferFifo@UIO61X_CanMessage_T@@@@@Z 100719f0 f i IO61X_Library_MSVC120_vc:IO61X_CanPort.obj
 0001:00070a40       ??$addressof@PAU?$_List_node@V?$IO61X_BufferFifo@UIO61X_CanMessage_T@@@@PAX@std@@@std@@YAPAPAU?$_List_node@V?$IO61X_BufferFifo@UIO61X_CanMessage_T@@@@PAX@0@AAPAU10@@Z 10071a40 f i IO61X_Library_MSVC120_vc:IO61X_CanPort.obj
 0001:00070a50       ??$addressof@V?$IO61X_BufferFifo@UIO61X_CanMessage_T@@@@@std@@YAPAV?$IO61X_BufferFifo@UIO61X_CanMessage_T@@@@AAV1@@Z 10071a50 f i IO61X_Library_MSVC120_vc:IO61X_CanPort.obj
 0001:00070a60       ??$construct@PAU?$_List_node@V?$IO61X_BufferFifo@UIO61X_CanMessage_T@@@@PAX@std@@AAPAU12@@?$_Wrap_alloc@V?$allocator@U?$_List_node@V?$IO61X_BufferFifo@UIO61X_CanMessage_T@@@@PAX@std@@@std@@@std@@QAEXPAPAU?$_List_node@V?$IO61X_BufferFifo@UIO61X_CanMessage_T@@@@PAX@1@AAPAU21@@Z 10071a60 f i IO61X_Library_MSVC120_vc:IO61X_CanPort.obj
 0001:00070a80       ??$construct@PAU?$_List_node@V?$IO61X_BufferFifo@UIO61X_CanMessage_T@@@@PAX@std@@AAPAU12@@?$allocator@U?$_List_node@V?$IO61X_BufferFifo@UIO61X_CanMessage_T@@@@PAX@std@@@std@@QAEXPAPAU?$_List_node@V?$IO61X_BufferFifo@UIO61X_CanMessage_T@@@@PAX@1@AAPAU21@@Z 10071a80 f i IO61X_Library_MSVC120_vc:IO61X_CanPort.obj
 0001:00070aa0       ??$construct@PAU?$_List_node@V?$IO61X_BufferFifo@UIO61X_CanMessage_T@@@@PAX@std@@AAPAU12@@?$allocator_traits@V?$allocator@U?$_List_node@V?$IO61X_BufferFifo@UIO61X_CanMessage_T@@@@PAX@std@@@std@@@std@@SAXAAV?$allocator@U?$_List_node@V?$IO61X_BufferFifo@UIO61X_CanMessage_T@@@@PAX@std@@@1@PAPAU?$_List_node@V?$IO61X_BufferFifo@UIO61X_CanMessage_T@@@@PAX@1@AAPAU31@@Z 10071aa0 f i IO61X_Library_MSVC120_vc:IO61X_CanPort.obj
 0001:00070ac0       ??$construct@V?$IO61X_BufferFifo@UIO61X_CanMessage_T@@@@V1@@?$_Wrap_alloc@V?$allocator@U?$_List_node@V?$IO61X_BufferFifo@UIO61X_CanMessage_T@@@@PAX@std@@@std@@@std@@QAEXPAV?$IO61X_BufferFifo@UIO61X_CanMessage_T@@@@$$QAV2@@Z 10071ac0 f i IO61X_Library_MSVC120_vc:IO61X_CanPort.obj
 0001:00070b10       ??$construct@V?$IO61X_BufferFifo@UIO61X_CanMessage_T@@@@V1@@?$allocator@U?$_List_node@V?$IO61X_BufferFifo@UIO61X_CanMessage_T@@@@PAX@std@@@std@@QAEXPAV?$IO61X_BufferFifo@UIO61X_CanMessage_T@@@@$$QAV2@@Z 10071b10 f i IO61X_Library_MSVC120_vc:IO61X_CanPort.obj
 0001:00070b60       ??$construct@V?$IO61X_BufferFifo@UIO61X_CanMessage_T@@@@V1@@?$allocator_traits@V?$allocator@U?$_List_node@V?$IO61X_BufferFifo@UIO61X_CanMessage_T@@@@PAX@std@@@std@@@std@@SAXAAV?$allocator@U?$_List_node@V?$IO61X_BufferFifo@UIO61X_CanMessage_T@@@@PAX@std@@@1@PAV?$IO61X_BufferFifo@UIO61X_CanMessage_T@@@@$$QAV3@@Z 10071b60 f i IO61X_Library_MSVC120_vc:IO61X_CanPort.obj
 0001:00070bb0       ??$destroy@PAU?$_List_node@V?$IO61X_BufferFifo@UIO61X_CanMessage_T@@@@PAX@std@@@?$_Wrap_alloc@V?$allocator@U?$_List_node@V?$IO61X_BufferFifo@UIO61X_CanMessage_T@@@@PAX@std@@@std@@@std@@QAEXPAPAU?$_List_node@V?$IO61X_BufferFifo@UIO61X_CanMessage_T@@@@PAX@1@@Z 10071bb0 f i IO61X_Library_MSVC120_vc:IO61X_CanPort.obj
 0001:00070bc0       ??$destroy@PAU?$_List_node@V?$IO61X_BufferFifo@UIO61X_CanMessage_T@@@@PAX@std@@@?$allocator@U?$_List_node@V?$IO61X_BufferFifo@UIO61X_CanMessage_T@@@@PAX@std@@@std@@QAEXPAPAU?$_List_node@V?$IO61X_BufferFifo@UIO61X_CanMessage_T@@@@PAX@1@@Z 10071bc0 f i IO61X_Library_MSVC120_vc:IO61X_CanPort.obj
 0001:00070bd0       ??$destroy@PAU?$_List_node@V?$IO61X_BufferFifo@UIO61X_CanMessage_T@@@@PAX@std@@@?$allocator_traits@V?$allocator@U?$_List_node@V?$IO61X_BufferFifo@UIO61X_CanMessage_T@@@@PAX@std@@@std@@@std@@SAXAAV?$allocator@U?$_List_node@V?$IO61X_BufferFifo@UIO61X_CanMessage_T@@@@PAX@std@@@1@PAPAU?$_List_node@V?$IO61X_BufferFifo@UIO61X_CanMessage_T@@@@PAX@1@@Z 10071bd0 f i IO61X_Library_MSVC120_vc:IO61X_CanPort.obj
 0001:00070be0       ??$destroy@V?$IO61X_BufferFifo@UIO61X_CanMessage_T@@@@@?$_Wrap_alloc@V?$allocator@U?$_List_node@V?$IO61X_BufferFifo@UIO61X_CanMessage_T@@@@PAX@std@@@std@@@std@@QAEXPAV?$IO61X_BufferFifo@UIO61X_CanMessage_T@@@@@Z 10071be0 f i IO61X_Library_MSVC120_vc:IO61X_CanPort.obj
 0001:00070c00       ??$destroy@V?$IO61X_BufferFifo@UIO61X_CanMessage_T@@@@@?$allocator@U?$_List_node@V?$IO61X_BufferFifo@UIO61X_CanMessage_T@@@@PAX@std@@@std@@QAEXPAV?$IO61X_BufferFifo@UIO61X_CanMessage_T@@@@@Z 10071c00 f i IO61X_Library_MSVC120_vc:IO61X_CanPort.obj
 0001:00070c20       ??$destroy@V?$IO61X_BufferFifo@UIO61X_CanMessage_T@@@@@?$allocator_traits@V?$allocator@U?$_List_node@V?$IO61X_BufferFifo@UIO61X_CanMessage_T@@@@PAX@std@@@std@@@std@@SAXAAV?$allocator@U?$_List_node@V?$IO61X_BufferFifo@UIO61X_CanMessage_T@@@@PAX@std@@@1@PAV?$IO61X_BufferFifo@UIO61X_CanMessage_T@@@@@Z 10071c20 f i IO61X_Library_MSVC120_vc:IO61X_CanPort.obj
 0001:00070c40       ??$forward@AAPAU?$_List_node@V?$IO61X_BufferFifo@UIO61X_CanMessage_T@@@@PAX@std@@@std@@YAAAPAU?$_List_node@V?$IO61X_BufferFifo@UIO61X_CanMessage_T@@@@PAX@0@AAPAU10@@Z 10071c40 f i IO61X_Library_MSVC120_vc:IO61X_CanPort.obj
 0001:00070c50       ??$forward@V?$IO61X_BufferFifo@UIO61X_CanMessage_T@@@@@std@@YA$$QAV?$IO61X_BufferFifo@UIO61X_CanMessage_T@@@@AAV1@@Z 10071c50 f i IO61X_Library_MSVC120_vc:IO61X_CanPort.obj
 0001:00070c60       ??0?$IO61X_BufferFifo@UIO61X_CanMessage_T@@@@QAE@ABV0@@Z 10071c60 f i IO61X_Library_MSVC120_vc:IO61X_CanPort.obj
 0001:00070ce0       ??0?$IO61X_BufferFifo@UIO61X_CanMessage_T@@@@QAE@IPAUIO61X_CanMessage_T@@@Z 10071ce0 f i IO61X_Library_MSVC120_vc:IO61X_CanPort.obj
 0001:00070d50       ??0?$_List_alloc@$0A@U?$_List_base_types@V?$IO61X_BufferFifo@UIO61X_CanMessage_T@@@@V?$allocator@V?$IO61X_BufferFifo@UIO61X_CanMessage_T@@@@@std@@@std@@@std@@QAE@ABV?$allocator@V?$IO61X_BufferFifo@UIO61X_CanMessage_T@@@@@1@@Z 10071d50 f i IO61X_Library_MSVC120_vc:IO61X_CanPort.obj
 0001:00070d80       ??0?$_List_buy@V?$IO61X_BufferFifo@UIO61X_CanMessage_T@@@@V?$allocator@V?$IO61X_BufferFifo@UIO61X_CanMessage_T@@@@@std@@@std@@QAE@ABV?$allocator@V?$IO61X_BufferFifo@UIO61X_CanMessage_T@@@@@1@@Z 10071d80 f i IO61X_Library_MSVC120_vc:IO61X_CanPort.obj
 0001:00070db0       ??0?$_List_const_iterator@V?$_List_val@U?$_List_simple_types@V?$IO61X_BufferFifo@UIO61X_CanMessage_T@@@@@std@@@std@@@std@@QAE@PAU?$_List_node@V?$IO61X_BufferFifo@UIO61X_CanMessage_T@@@@PAX@1@PBV?$_List_val@U?$_List_simple_types@V?$IO61X_BufferFifo@UIO61X_CanMessage_T@@@@@std@@@1@@Z 10071db0 f i IO61X_Library_MSVC120_vc:IO61X_CanPort.obj
 0001:00070dc0       ??0?$_List_iterator@V?$_List_val@U?$_List_simple_types@V?$IO61X_BufferFifo@UIO61X_CanMessage_T@@@@@std@@@std@@@std@@QAE@PAU?$_List_node@V?$IO61X_BufferFifo@UIO61X_CanMessage_T@@@@PAX@1@PBV?$_List_val@U?$_List_simple_types@V?$IO61X_BufferFifo@UIO61X_CanMessage_T@@@@@std@@@1@@Z 10071dc0 f i IO61X_Library_MSVC120_vc:IO61X_CanPort.obj
 0001:00070dd0       ??0?$_List_unchecked_const_iterator@V?$_List_val@U?$_List_simple_types@V?$IO61X_BufferFifo@UIO61X_CanMessage_T@@@@@std@@@std@@U_Iterator_base0@2@@std@@QAE@PAU?$_List_node@V?$IO61X_BufferFifo@UIO61X_CanMessage_T@@@@PAX@1@PBV?$_List_val@U?$_List_simple_types@V?$IO61X_BufferFifo@UIO61X_CanMessage_T@@@@@std@@@1@@Z 10071dd0 f i IO61X_Library_MSVC120_vc:IO61X_CanPort.obj
 0001:00070de0       ??0?$_List_unchecked_iterator@V?$_List_val@U?$_List_simple_types@V?$IO61X_BufferFifo@UIO61X_CanMessage_T@@@@@std@@@std@@@std@@QAE@PAU?$_List_node@V?$IO61X_BufferFifo@UIO61X_CanMessage_T@@@@PAX@1@PBV?$_List_val@U?$_List_simple_types@V?$IO61X_BufferFifo@UIO61X_CanMessage_T@@@@@std@@@1@@Z 10071de0 f i IO61X_Library_MSVC120_vc:IO61X_CanPort.obj
 0001:00070df0       ??0?$_List_val@U?$_List_simple_types@V?$IO61X_BufferFifo@UIO61X_CanMessage_T@@@@@std@@@std@@QAE@XZ 10071df0 f i IO61X_Library_MSVC120_vc:IO61X_CanPort.obj
 0001:00070e00       ??0?$_Wrap_alloc@V?$allocator@U?$_List_node@V?$IO61X_BufferFifo@UIO61X_CanMessage_T@@@@PAX@std@@@std@@@std@@QAE@XZ 10071e00 f i IO61X_Library_MSVC120_vc:IO61X_CanPort.obj
 0001:00070e10       ??0?$allocator@U?$_List_node@V?$IO61X_BufferFifo@UIO61X_CanMessage_T@@@@PAX@std@@@std@@QAE@XZ 10071e10 f i IO61X_Library_MSVC120_vc:IO61X_CanPort.obj
 0001:00070e20       ??0?$allocator@V?$IO61X_BufferFifo@UIO61X_CanMessage_T@@@@@std@@QAE@XZ 10071e20 f i IO61X_Library_MSVC120_vc:IO61X_CanPort.obj
 0001:00070e30       ??0?$atomic@H@std@@QAE@XZ  10071e30 f i IO61X_Library_MSVC120_vc:IO61X_CanPort.obj
 0001:00070e40       ??0?$list@V?$IO61X_BufferFifo@UIO61X_CanMessage_T@@@@V?$allocator@V?$IO61X_BufferFifo@UIO61X_CanMessage_T@@@@@std@@@std@@QAE@XZ 10071e40 f i IO61X_Library_MSVC120_vc:IO61X_CanPort.obj
 0001:00070e60       ??0IO61X_CanPort@@QAE@II@Z 10071e60 f   IO61X_Library_MSVC120_vc:IO61X_CanPort.obj
 0001:00070f20       ??1?$IO61X_BufferFifo@UIO61X_CanMessage_T@@@@QAE@XZ 10071f20 f i IO61X_Library_MSVC120_vc:IO61X_CanPort.obj
 0001:00070f30       ??1?$_List_alloc@$0A@U?$_List_base_types@V?$IO61X_BufferFifo@UIO61X_CanMessage_T@@@@V?$allocator@V?$IO61X_BufferFifo@UIO61X_CanMessage_T@@@@@std@@@std@@@std@@QAE@XZ 10071f30 f i IO61X_Library_MSVC120_vc:IO61X_CanPort.obj
 0001:00070f40       ??1?$_List_buy@V?$IO61X_BufferFifo@UIO61X_CanMessage_T@@@@V?$allocator@V?$IO61X_BufferFifo@UIO61X_CanMessage_T@@@@@std@@@std@@QAE@XZ 10071f40 f i IO61X_Library_MSVC120_vc:IO61X_CanPort.obj
 0001:00070f50       ??1?$list@V?$IO61X_BufferFifo@UIO61X_CanMessage_T@@@@V?$allocator@V?$IO61X_BufferFifo@UIO61X_CanMessage_T@@@@@std@@@std@@QAE@XZ 10071f50 f i IO61X_Library_MSVC120_vc:IO61X_CanPort.obj
 0001:00070f70       ??1IO61X_CanPort@@UAE@XZ   10071f70 f   IO61X_Library_MSVC120_vc:IO61X_CanPort.obj
 0001:00070fa0       ??8?$_List_const_iterator@V?$_List_val@U?$_List_simple_types@V?$IO61X_BufferFifo@UIO61X_CanMessage_T@@@@@std@@@std@@@std@@QBE_NABV01@@Z 10071fa0 f i IO61X_Library_MSVC120_vc:IO61X_CanPort.obj
 0001:00070fc0       ??9?$_List_const_iterator@V?$_List_val@U?$_List_simple_types@V?$IO61X_BufferFifo@UIO61X_CanMessage_T@@@@@std@@@std@@@std@@QBE_NABV01@@Z 10071fc0 f i IO61X_Library_MSVC120_vc:IO61X_CanPort.obj
 0001:00070fe0       ??Batomic_int@std@@QBEHXZ  10071fe0 f i IO61X_Library_MSVC120_vc:IO61X_CanPort.obj
 0001:00070ff0       ??D?$_List_const_iterator@V?$_List_val@U?$_List_simple_types@V?$IO61X_BufferFifo@UIO61X_CanMessage_T@@@@@std@@@std@@@std@@QBEABV?$IO61X_BufferFifo@UIO61X_CanMessage_T@@@@XZ 10071ff0 f i IO61X_Library_MSVC120_vc:IO61X_CanPort.obj
 0001:00071000       ??D?$_List_iterator@V?$_List_val@U?$_List_simple_types@V?$IO61X_BufferFifo@UIO61X_CanMessage_T@@@@@std@@@std@@@std@@QBEAAV?$IO61X_BufferFifo@UIO61X_CanMessage_T@@@@XZ 10072000 f i IO61X_Library_MSVC120_vc:IO61X_CanPort.obj
 0001:00071010       ??E?$_List_const_iterator@V?$_List_val@U?$_List_simple_types@V?$IO61X_BufferFifo@UIO61X_CanMessage_T@@@@@std@@@std@@@std@@QAEAAV01@XZ 10072010 f i IO61X_Library_MSVC120_vc:IO61X_CanPort.obj
 0001:00071020       ??E?$_List_iterator@V?$_List_val@U?$_List_simple_types@V?$IO61X_BufferFifo@UIO61X_CanMessage_T@@@@@std@@@std@@@std@@QAE?AV01@H@Z 10072020 f i IO61X_Library_MSVC120_vc:IO61X_CanPort.obj
 0001:00071040       ??E?$_List_iterator@V?$_List_val@U?$_List_simple_types@V?$IO61X_BufferFifo@UIO61X_CanMessage_T@@@@@std@@@std@@@std@@QAEAAV01@XZ 10072040 f i IO61X_Library_MSVC120_vc:IO61X_CanPort.obj
 0001:00071050       ??F?$_List_const_iterator@V?$_List_val@U?$_List_simple_types@V?$IO61X_BufferFifo@UIO61X_CanMessage_T@@@@@std@@@std@@@std@@QAEAAV01@XZ 10072050 f i IO61X_Library_MSVC120_vc:IO61X_CanPort.obj
 0001:00071060       ??F?$_List_iterator@V?$_List_val@U?$_List_simple_types@V?$IO61X_BufferFifo@UIO61X_CanMessage_T@@@@@std@@@std@@@std@@QAEAAV01@XZ 10072060 f i IO61X_Library_MSVC120_vc:IO61X_CanPort.obj
 0001:00071070       ??_G?$IO61X_BufferFifo@UIO61X_CanMessage_T@@@@QAEPAXI@Z 10072070 f i IO61X_Library_MSVC120_vc:IO61X_CanPort.obj
 0001:000710a0       ??_EIO61X_CanPort@@UAEPAXI@Z 100720a0 f i IO61X_Library_MSVC120_vc:IO61X_CanPort.obj
 0001:000710a0       ??_GIO61X_CanPort@@UAEPAXI@Z 100720a0 f i IO61X_Library_MSVC120_vc:IO61X_CanPort.obj
 0001:000710e0       ?AddMessageToBuffer@?$IO61X_BufferFifo@UIO61X_CanMessage_T@@@@QAE_NPBUIO61X_CanMessage_T@@@Z 100720e0 f i IO61X_Library_MSVC120_vc:IO61X_CanPort.obj
 0001:00071130       ?AllocateBuffer_spin@IO61X_CanPort@@UAEPAX_NI@Z 10072130 f   IO61X_Library_MSVC120_vc:IO61X_CanPort.obj
 0001:00071230       ?ClearBufferList@IO61X_CanPort@@UAE_NXZ 10072230 f   IO61X_Library_MSVC120_vc:IO61X_CanPort.obj
 0001:00071250       ?GetMessageFromBuffer@?$IO61X_BufferFifo@UIO61X_CanMessage_T@@@@QAEPAUIO61X_CanMessage_T@@XZ 10072250 f i IO61X_Library_MSVC120_vc:IO61X_CanPort.obj
 0001:00071280       ?Receive_spin@IO61X_CanPort@@UAE_NH@Z 10072280 f i IO61X_Library_MSVC120_vc:IO61X_CanPort.obj
 0001:00071290       ?Send_spin@IO61X_CanPort@@UAE_NXZ 10072290 f   IO61X_Library_MSVC120_vc:IO61X_CanPort.obj
 0001:000713c0       ?UpdateBuffer_spin@IO61X_CanPort@@UAE_NPAX0@Z 100723c0 f   IO61X_Library_MSVC120_vc:IO61X_CanPort.obj
 0001:000714b0       ?_Buyheadnode@?$_List_alloc@$0A@U?$_List_base_types@V?$IO61X_BufferFifo@UIO61X_CanMessage_T@@@@V?$allocator@V?$IO61X_BufferFifo@UIO61X_CanMessage_T@@@@@std@@@std@@@std@@QAEPAU?$_List_node@V?$IO61X_BufferFifo@UIO61X_CanMessage_T@@@@PAX@2@XZ 100724b0 f i IO61X_Library_MSVC120_vc:IO61X_CanPort.obj
 0001:000714c0       ?_Buynode0@?$_List_alloc@$0A@U?$_List_base_types@V?$IO61X_BufferFifo@UIO61X_CanMessage_T@@@@V?$allocator@V?$IO61X_BufferFifo@UIO61X_CanMessage_T@@@@@std@@@std@@@std@@QAEPAU?$_List_node@V?$IO61X_BufferFifo@UIO61X_CanMessage_T@@@@PAX@2@PAU32@0@Z 100724c0 f i IO61X_Library_MSVC120_vc:IO61X_CanPort.obj
 0001:00071500       ?_Freeheadnode@?$_List_alloc@$0A@U?$_List_base_types@V?$IO61X_BufferFifo@UIO61X_CanMessage_T@@@@V?$allocator@V?$IO61X_BufferFifo@UIO61X_CanMessage_T@@@@@std@@@std@@@std@@QAEXPAU?$_List_node@V?$IO61X_BufferFifo@UIO61X_CanMessage_T@@@@PAX@2@@Z 10072500 f i IO61X_Library_MSVC120_vc:IO61X_CanPort.obj
 0001:00071520       ?_Freenode@?$_List_buy@V?$IO61X_BufferFifo@UIO61X_CanMessage_T@@@@V?$allocator@V?$IO61X_BufferFifo@UIO61X_CanMessage_T@@@@@std@@@std@@QAEXPAU?$_List_node@V?$IO61X_BufferFifo@UIO61X_CanMessage_T@@@@PAX@2@@Z 10072520 f i IO61X_Library_MSVC120_vc:IO61X_CanPort.obj
 0001:00071550       ?_Getal@?$_List_alloc@$0A@U?$_List_base_types@V?$IO61X_BufferFifo@UIO61X_CanMessage_T@@@@V?$allocator@V?$IO61X_BufferFifo@UIO61X_CanMessage_T@@@@@std@@@std@@@std@@QBE?AU?$_Wrap_alloc@V?$allocator@U?$_List_node@V?$IO61X_BufferFifo@UIO61X_CanMessage_T@@@@PAX@std@@@std@@@2@XZ 10072550 f i IO61X_Library_MSVC120_vc:IO61X_CanPort.obj
 0001:00071560       ?_Incsize@?$list@V?$IO61X_BufferFifo@UIO61X_CanMessage_T@@@@V?$allocator@V?$IO61X_BufferFifo@UIO61X_CanMessage_T@@@@@std@@@std@@QAEXI@Z 10072560 f i IO61X_Library_MSVC120_vc:IO61X_CanPort.obj
 0001:00071590       ?_Mynode@?$_List_unchecked_const_iterator@V?$_List_val@U?$_List_simple_types@V?$IO61X_BufferFifo@UIO61X_CanMessage_T@@@@@std@@@std@@U_Iterator_base0@2@@std@@QBEPAU?$_List_node@V?$IO61X_BufferFifo@UIO61X_CanMessage_T@@@@PAX@2@XZ 10072590 f i IO61X_Library_MSVC120_vc:IO61X_CanPort.obj
 0001:000715a0       ?_Myval@?$_List_val@U?$_List_simple_types@V?$IO61X_BufferFifo@UIO61X_CanMessage_T@@@@@std@@@std@@SAAAV?$IO61X_BufferFifo@UIO61X_CanMessage_T@@@@PAU?$_List_node@V?$IO61X_BufferFifo@UIO61X_CanMessage_T@@@@PAX@2@@Z 100725a0 f i IO61X_Library_MSVC120_vc:IO61X_CanPort.obj
 0001:000715b0       ?_Nextnode@?$_List_val@U?$_List_simple_types@V?$IO61X_BufferFifo@UIO61X_CanMessage_T@@@@@std@@@std@@SAAAPAU?$_List_node@V?$IO61X_BufferFifo@UIO61X_CanMessage_T@@@@PAX@2@PAU32@@Z 100725b0 f i IO61X_Library_MSVC120_vc:IO61X_CanPort.obj
 0001:000715c0       ?_Prevnode@?$_List_val@U?$_List_simple_types@V?$IO61X_BufferFifo@UIO61X_CanMessage_T@@@@@std@@@std@@SAAAPAU?$_List_node@V?$IO61X_BufferFifo@UIO61X_CanMessage_T@@@@PAX@2@PAU32@@Z 100725c0 f i IO61X_Library_MSVC120_vc:IO61X_CanPort.obj
 0001:000715d0       ?_Tidy@?$list@V?$IO61X_BufferFifo@UIO61X_CanMessage_T@@@@V?$allocator@V?$IO61X_BufferFifo@UIO61X_CanMessage_T@@@@@std@@@std@@QAEXXZ 100725d0 f i IO61X_Library_MSVC120_vc:IO61X_CanPort.obj
 0001:000715e0       ?_Unchecked_end@?$list@V?$IO61X_BufferFifo@UIO61X_CanMessage_T@@@@V?$allocator@V?$IO61X_BufferFifo@UIO61X_CanMessage_T@@@@@std@@@std@@QAE?AV?$_List_unchecked_iterator@V?$_List_val@U?$_List_simple_types@V?$IO61X_BufferFifo@UIO61X_CanMessage_T@@@@@std@@@std@@@2@XZ 100725e0 f i IO61X_Library_MSVC120_vc:IO61X_CanPort.obj
 0001:000715f0       ?allocate@?$_Wrap_alloc@V?$allocator@U?$_List_node@V?$IO61X_BufferFifo@UIO61X_CanMessage_T@@@@PAX@std@@@std@@@std@@QAEPAU?$_List_node@V?$IO61X_BufferFifo@UIO61X_CanMessage_T@@@@PAX@2@I@Z 100725f0 f i IO61X_Library_MSVC120_vc:IO61X_CanPort.obj
 0001:00071630       ?allocate@?$allocator@U?$_List_node@V?$IO61X_BufferFifo@UIO61X_CanMessage_T@@@@PAX@std@@@std@@QAEPAU?$_List_node@V?$IO61X_BufferFifo@UIO61X_CanMessage_T@@@@PAX@2@I@Z 10072630 f i IO61X_Library_MSVC120_vc:IO61X_CanPort.obj
 0001:00071670       ?atomic_load@std@@YAHPBUatomic_int@1@@Z 10072670 f i IO61X_Library_MSVC120_vc:IO61X_CanPort.obj
 0001:00071680       ?back@?$list@V?$IO61X_BufferFifo@UIO61X_CanMessage_T@@@@V?$allocator@V?$IO61X_BufferFifo@UIO61X_CanMessage_T@@@@@std@@@std@@QAEAAV?$IO61X_BufferFifo@UIO61X_CanMessage_T@@@@XZ 10072680 f i IO61X_Library_MSVC120_vc:IO61X_CanPort.obj
 0001:00071690       ?begin@?$list@V?$IO61X_BufferFifo@UIO61X_CanMessage_T@@@@V?$allocator@V?$IO61X_BufferFifo@UIO61X_CanMessage_T@@@@@std@@@std@@QAE?AV?$_List_iterator@V?$_List_val@U?$_List_simple_types@V?$IO61X_BufferFifo@UIO61X_CanMessage_T@@@@@std@@@std@@@2@XZ 10072690 f i IO61X_Library_MSVC120_vc:IO61X_CanPort.obj
 0001:000716a0       ?clear@?$list@V?$IO61X_BufferFifo@UIO61X_CanMessage_T@@@@V?$allocator@V?$IO61X_BufferFifo@UIO61X_CanMessage_T@@@@@std@@@std@@QAEXXZ 100726a0 f i IO61X_Library_MSVC120_vc:IO61X_CanPort.obj
 0001:000716f0       ?deallocate@?$_Wrap_alloc@V?$allocator@U?$_List_node@V?$IO61X_BufferFifo@UIO61X_CanMessage_T@@@@PAX@std@@@std@@@std@@QAEXPAU?$_List_node@V?$IO61X_BufferFifo@UIO61X_CanMessage_T@@@@PAX@2@I@Z 100726f0 f i IO61X_Library_MSVC120_vc:IO61X_CanPort.obj
 0001:00071710       ?deallocate@?$allocator@U?$_List_node@V?$IO61X_BufferFifo@UIO61X_CanMessage_T@@@@PAX@std@@@std@@QAEXPAU?$_List_node@V?$IO61X_BufferFifo@UIO61X_CanMessage_T@@@@PAX@2@I@Z 10072710 f i IO61X_Library_MSVC120_vc:IO61X_CanPort.obj
 0001:00071730       ?empty@?$list@V?$IO61X_BufferFifo@UIO61X_CanMessage_T@@@@V?$allocator@V?$IO61X_BufferFifo@UIO61X_CanMessage_T@@@@@std@@@std@@QBE_NXZ 10072730 f i IO61X_Library_MSVC120_vc:IO61X_CanPort.obj
 0001:00071740       ?end@?$list@V?$IO61X_BufferFifo@UIO61X_CanMessage_T@@@@V?$allocator@V?$IO61X_BufferFifo@UIO61X_CanMessage_T@@@@@std@@@std@@QAE?AV?$_List_iterator@V?$_List_val@U?$_List_simple_types@V?$IO61X_BufferFifo@UIO61X_CanMessage_T@@@@@std@@@std@@@2@XZ 10072740 f i IO61X_Library_MSVC120_vc:IO61X_CanPort.obj
 0001:00071750       ?getReadIdx@?$IO61X_BufferFifo@UIO61X_CanMessage_T@@@@QAEHXZ 10072750 f i IO61X_Library_MSVC120_vc:IO61X_CanPort.obj
 0001:00071760       ?getWriteIdx@?$IO61X_BufferFifo@UIO61X_CanMessage_T@@@@QAEHXZ 10072760 f i IO61X_Library_MSVC120_vc:IO61X_CanPort.obj
 0001:00071770       ?max_size@?$_Wrap_alloc@V?$allocator@U?$_List_node@V?$IO61X_BufferFifo@UIO61X_CanMessage_T@@@@PAX@std@@@std@@@std@@QBEIXZ 10072770 f i IO61X_Library_MSVC120_vc:IO61X_CanPort.obj
 0001:00071780       ?max_size@?$allocator@U?$_List_node@V?$IO61X_BufferFifo@UIO61X_CanMessage_T@@@@PAX@std@@@std@@QBEIXZ 10072780 f i IO61X_Library_MSVC120_vc:IO61X_CanPort.obj
 0001:00071790       ?max_size@?$allocator_traits@V?$allocator@U?$_List_node@V?$IO61X_BufferFifo@UIO61X_CanMessage_T@@@@PAX@std@@@std@@@std@@SAIABV?$allocator@U?$_List_node@V?$IO61X_BufferFifo@UIO61X_CanMessage_T@@@@PAX@std@@@2@@Z 10072790 f i IO61X_Library_MSVC120_vc:IO61X_CanPort.obj
 0001:000717a0       ?max_size@?$list@V?$IO61X_BufferFifo@UIO61X_CanMessage_T@@@@V?$allocator@V?$IO61X_BufferFifo@UIO61X_CanMessage_T@@@@@std@@@std@@QBEIXZ 100727a0 f i IO61X_Library_MSVC120_vc:IO61X_CanPort.obj
 0001:000717b0       ?push_back@?$list@V?$IO61X_BufferFifo@UIO61X_CanMessage_T@@@@V?$allocator@V?$IO61X_BufferFifo@UIO61X_CanMessage_T@@@@@std@@@std@@QAEX$$QAV?$IO61X_BufferFifo@UIO61X_CanMessage_T@@@@@Z 100727b0 f i IO61X_Library_MSVC120_vc:IO61X_CanPort.obj
 0001:00071800       ?setReadIdx@?$IO61X_BufferFifo@UIO61X_CanMessage_T@@@@QAEXH@Z 10072800 f i IO61X_Library_MSVC120_vc:IO61X_CanPort.obj
 0001:00071810       ?setWriteIdx@?$IO61X_BufferFifo@UIO61X_CanMessage_T@@@@QAEXH@Z 10072810 f i IO61X_Library_MSVC120_vc:IO61X_CanPort.obj
 0001:00071820       ??$_Allocate@U?$_List_node@V?$IO61X_BufferFifo@UIO61X_CanFdMessage_T@@@@PAX@std@@@std@@YAPAU?$_List_node@V?$IO61X_BufferFifo@UIO61X_CanFdMessage_T@@@@PAX@0@IPAU10@@Z 10072820 f i IO61X_Library_MSVC120_vc:IO61X_CanFdPort.obj
 0001:00071860       ??$_Buynode@V?$IO61X_BufferFifo@UIO61X_CanFdMessage_T@@@@@?$_List_buy@V?$IO61X_BufferFifo@UIO61X_CanFdMessage_T@@@@V?$allocator@V?$IO61X_BufferFifo@UIO61X_CanFdMessage_T@@@@@std@@@std@@QAEPAU?$_List_node@V?$IO61X_BufferFifo@UIO61X_CanFdMessage_T@@@@PAX@1@PAU21@0$$QAV?$IO61X_BufferFifo@UIO61X_CanFdMessage_T@@@@@Z 10072860 f i IO61X_Library_MSVC120_vc:IO61X_CanFdPort.obj
 0001:000718f0       ??$_Insert@V?$IO61X_BufferFifo@UIO61X_CanFdMessage_T@@@@@?$list@V?$IO61X_BufferFifo@UIO61X_CanFdMessage_T@@@@V?$allocator@V?$IO61X_BufferFifo@UIO61X_CanFdMessage_T@@@@@std@@@std@@QAEXV?$_List_unchecked_const_iterator@V?$_List_val@U?$_List_simple_types@V?$IO61X_BufferFifo@UIO61X_CanFdMessage_T@@@@@std@@@std@@U_Iterator_base0@2@@1@$$QAV?$IO61X_BufferFifo@UIO61X_CanFdMessage_T@@@@@Z 100728f0 f i IO61X_Library_MSVC120_vc:IO61X_CanFdPort.obj
 0001:00071940       ??$addressof@PAU?$_List_node@V?$IO61X_BufferFifo@UIO61X_CanFdMessage_T@@@@PAX@std@@@std@@YAPAPAU?$_List_node@V?$IO61X_BufferFifo@UIO61X_CanFdMessage_T@@@@PAX@0@AAPAU10@@Z 10072940 f i IO61X_Library_MSVC120_vc:IO61X_CanFdPort.obj
 0001:00071950       ??$addressof@V?$IO61X_BufferFifo@UIO61X_CanFdMessage_T@@@@@std@@YAPAV?$IO61X_BufferFifo@UIO61X_CanFdMessage_T@@@@AAV1@@Z 10072950 f i IO61X_Library_MSVC120_vc:IO61X_CanFdPort.obj
 0001:00071960       ??$construct@PAU?$_List_node@V?$IO61X_BufferFifo@UIO61X_CanFdMessage_T@@@@PAX@std@@AAPAU12@@?$_Wrap_alloc@V?$allocator@U?$_List_node@V?$IO61X_BufferFifo@UIO61X_CanFdMessage_T@@@@PAX@std@@@std@@@std@@QAEXPAPAU?$_List_node@V?$IO61X_BufferFifo@UIO61X_CanFdMessage_T@@@@PAX@1@AAPAU21@@Z 10072960 f i IO61X_Library_MSVC120_vc:IO61X_CanFdPort.obj
 0001:00071980       ??$construct@PAU?$_List_node@V?$IO61X_BufferFifo@UIO61X_CanFdMessage_T@@@@PAX@std@@AAPAU12@@?$allocator@U?$_List_node@V?$IO61X_BufferFifo@UIO61X_CanFdMessage_T@@@@PAX@std@@@std@@QAEXPAPAU?$_List_node@V?$IO61X_BufferFifo@UIO61X_CanFdMessage_T@@@@PAX@1@AAPAU21@@Z 10072980 f i IO61X_Library_MSVC120_vc:IO61X_CanFdPort.obj
 0001:000719a0       ??$construct@PAU?$_List_node@V?$IO61X_BufferFifo@UIO61X_CanFdMessage_T@@@@PAX@std@@AAPAU12@@?$allocator_traits@V?$allocator@U?$_List_node@V?$IO61X_BufferFifo@UIO61X_CanFdMessage_T@@@@PAX@std@@@std@@@std@@SAXAAV?$allocator@U?$_List_node@V?$IO61X_BufferFifo@UIO61X_CanFdMessage_T@@@@PAX@std@@@1@PAPAU?$_List_node@V?$IO61X_BufferFifo@UIO61X_CanFdMessage_T@@@@PAX@1@AAPAU31@@Z 100729a0 f i IO61X_Library_MSVC120_vc:IO61X_CanFdPort.obj
 0001:000719c0       ??$construct@V?$IO61X_BufferFifo@UIO61X_CanFdMessage_T@@@@V1@@?$_Wrap_alloc@V?$allocator@U?$_List_node@V?$IO61X_BufferFifo@UIO61X_CanFdMessage_T@@@@PAX@std@@@std@@@std@@QAEXPAV?$IO61X_BufferFifo@UIO61X_CanFdMessage_T@@@@$$QAV2@@Z 100729c0 f i IO61X_Library_MSVC120_vc:IO61X_CanFdPort.obj
 0001:00071a10       ??$construct@V?$IO61X_BufferFifo@UIO61X_CanFdMessage_T@@@@V1@@?$allocator@U?$_List_node@V?$IO61X_BufferFifo@UIO61X_CanFdMessage_T@@@@PAX@std@@@std@@QAEXPAV?$IO61X_BufferFifo@UIO61X_CanFdMessage_T@@@@$$QAV2@@Z 10072a10 f i IO61X_Library_MSVC120_vc:IO61X_CanFdPort.obj
 0001:00071a60       ??$construct@V?$IO61X_BufferFifo@UIO61X_CanFdMessage_T@@@@V1@@?$allocator_traits@V?$allocator@U?$_List_node@V?$IO61X_BufferFifo@UIO61X_CanFdMessage_T@@@@PAX@std@@@std@@@std@@SAXAAV?$allocator@U?$_List_node@V?$IO61X_BufferFifo@UIO61X_CanFdMessage_T@@@@PAX@std@@@1@PAV?$IO61X_BufferFifo@UIO61X_CanFdMessage_T@@@@$$QAV3@@Z 10072a60 f i IO61X_Library_MSVC120_vc:IO61X_CanFdPort.obj
 0001:00071ab0       ??$destroy@PAU?$_List_node@V?$IO61X_BufferFifo@UIO61X_CanFdMessage_T@@@@PAX@std@@@?$_Wrap_alloc@V?$allocator@U?$_List_node@V?$IO61X_BufferFifo@UIO61X_CanFdMessage_T@@@@PAX@std@@@std@@@std@@QAEXPAPAU?$_List_node@V?$IO61X_BufferFifo@UIO61X_CanFdMessage_T@@@@PAX@1@@Z 10072ab0 f i IO61X_Library_MSVC120_vc:IO61X_CanFdPort.obj
 0001:00071ac0       ??$destroy@PAU?$_List_node@V?$IO61X_BufferFifo@UIO61X_CanFdMessage_T@@@@PAX@std@@@?$allocator@U?$_List_node@V?$IO61X_BufferFifo@UIO61X_CanFdMessage_T@@@@PAX@std@@@std@@QAEXPAPAU?$_List_node@V?$IO61X_BufferFifo@UIO61X_CanFdMessage_T@@@@PAX@1@@Z 10072ac0 f i IO61X_Library_MSVC120_vc:IO61X_CanFdPort.obj
 0001:00071ad0       ??$destroy@PAU?$_List_node@V?$IO61X_BufferFifo@UIO61X_CanFdMessage_T@@@@PAX@std@@@?$allocator_traits@V?$allocator@U?$_List_node@V?$IO61X_BufferFifo@UIO61X_CanFdMessage_T@@@@PAX@std@@@std@@@std@@SAXAAV?$allocator@U?$_List_node@V?$IO61X_BufferFifo@UIO61X_CanFdMessage_T@@@@PAX@std@@@1@PAPAU?$_List_node@V?$IO61X_BufferFifo@UIO61X_CanFdMessage_T@@@@PAX@1@@Z 10072ad0 f i IO61X_Library_MSVC120_vc:IO61X_CanFdPort.obj
 0001:00071ae0       ??$destroy@V?$IO61X_BufferFifo@UIO61X_CanFdMessage_T@@@@@?$_Wrap_alloc@V?$allocator@U?$_List_node@V?$IO61X_BufferFifo@UIO61X_CanFdMessage_T@@@@PAX@std@@@std@@@std@@QAEXPAV?$IO61X_BufferFifo@UIO61X_CanFdMessage_T@@@@@Z 10072ae0 f i IO61X_Library_MSVC120_vc:IO61X_CanFdPort.obj
 0001:00071b00       ??$destroy@V?$IO61X_BufferFifo@UIO61X_CanFdMessage_T@@@@@?$allocator@U?$_List_node@V?$IO61X_BufferFifo@UIO61X_CanFdMessage_T@@@@PAX@std@@@std@@QAEXPAV?$IO61X_BufferFifo@UIO61X_CanFdMessage_T@@@@@Z 10072b00 f i IO61X_Library_MSVC120_vc:IO61X_CanFdPort.obj
 0001:00071b20       ??$destroy@V?$IO61X_BufferFifo@UIO61X_CanFdMessage_T@@@@@?$allocator_traits@V?$allocator@U?$_List_node@V?$IO61X_BufferFifo@UIO61X_CanFdMessage_T@@@@PAX@std@@@std@@@std@@SAXAAV?$allocator@U?$_List_node@V?$IO61X_BufferFifo@UIO61X_CanFdMessage_T@@@@PAX@std@@@1@PAV?$IO61X_BufferFifo@UIO61X_CanFdMessage_T@@@@@Z 10072b20 f i IO61X_Library_MSVC120_vc:IO61X_CanFdPort.obj
 0001:00071b40       ??$forward@AAPAU?$_List_node@V?$IO61X_BufferFifo@UIO61X_CanFdMessage_T@@@@PAX@std@@@std@@YAAAPAU?$_List_node@V?$IO61X_BufferFifo@UIO61X_CanFdMessage_T@@@@PAX@0@AAPAU10@@Z 10072b40 f i IO61X_Library_MSVC120_vc:IO61X_CanFdPort.obj
 0001:00071b50       ??$forward@V?$IO61X_BufferFifo@UIO61X_CanFdMessage_T@@@@@std@@YA$$QAV?$IO61X_BufferFifo@UIO61X_CanFdMessage_T@@@@AAV1@@Z 10072b50 f i IO61X_Library_MSVC120_vc:IO61X_CanFdPort.obj
 0001:00071b60       ??0?$IO61X_BufferFifo@UIO61X_CanFdMessage_T@@@@QAE@ABV0@@Z 10072b60 f i IO61X_Library_MSVC120_vc:IO61X_CanFdPort.obj
 0001:00071c10       ??0?$IO61X_BufferFifo@UIO61X_CanFdMessage_T@@@@QAE@IPAUIO61X_CanFdMessage_T@@@Z 10072c10 f i IO61X_Library_MSVC120_vc:IO61X_CanFdPort.obj
 0001:00071c90       ??0?$_List_alloc@$0A@U?$_List_base_types@V?$IO61X_BufferFifo@UIO61X_CanFdMessage_T@@@@V?$allocator@V?$IO61X_BufferFifo@UIO61X_CanFdMessage_T@@@@@std@@@std@@@std@@QAE@ABV?$allocator@V?$IO61X_BufferFifo@UIO61X_CanFdMessage_T@@@@@1@@Z 10072c90 f i IO61X_Library_MSVC120_vc:IO61X_CanFdPort.obj
 0001:00071cc0       ??0?$_List_buy@V?$IO61X_BufferFifo@UIO61X_CanFdMessage_T@@@@V?$allocator@V?$IO61X_BufferFifo@UIO61X_CanFdMessage_T@@@@@std@@@std@@QAE@ABV?$allocator@V?$IO61X_BufferFifo@UIO61X_CanFdMessage_T@@@@@1@@Z 10072cc0 f i IO61X_Library_MSVC120_vc:IO61X_CanFdPort.obj
 0001:00071cf0       ??0?$_List_const_iterator@V?$_List_val@U?$_List_simple_types@V?$IO61X_BufferFifo@UIO61X_CanFdMessage_T@@@@@std@@@std@@@std@@QAE@PAU?$_List_node@V?$IO61X_BufferFifo@UIO61X_CanFdMessage_T@@@@PAX@1@PBV?$_List_val@U?$_List_simple_types@V?$IO61X_BufferFifo@UIO61X_CanFdMessage_T@@@@@std@@@1@@Z 10072cf0 f i IO61X_Library_MSVC120_vc:IO61X_CanFdPort.obj
 0001:00071d00       ??0?$_List_iterator@V?$_List_val@U?$_List_simple_types@V?$IO61X_BufferFifo@UIO61X_CanFdMessage_T@@@@@std@@@std@@@std@@QAE@PAU?$_List_node@V?$IO61X_BufferFifo@UIO61X_CanFdMessage_T@@@@PAX@1@PBV?$_List_val@U?$_List_simple_types@V?$IO61X_BufferFifo@UIO61X_CanFdMessage_T@@@@@std@@@1@@Z 10072d00 f i IO61X_Library_MSVC120_vc:IO61X_CanFdPort.obj
 0001:00071d10       ??0?$_List_unchecked_const_iterator@V?$_List_val@U?$_List_simple_types@V?$IO61X_BufferFifo@UIO61X_CanFdMessage_T@@@@@std@@@std@@U_Iterator_base0@2@@std@@QAE@PAU?$_List_node@V?$IO61X_BufferFifo@UIO61X_CanFdMessage_T@@@@PAX@1@PBV?$_List_val@U?$_List_simple_types@V?$IO61X_BufferFifo@UIO61X_CanFdMessage_T@@@@@std@@@1@@Z 10072d10 f i IO61X_Library_MSVC120_vc:IO61X_CanFdPort.obj
 0001:00071d20       ??0?$_List_unchecked_iterator@V?$_List_val@U?$_List_simple_types@V?$IO61X_BufferFifo@UIO61X_CanFdMessage_T@@@@@std@@@std@@@std@@QAE@PAU?$_List_node@V?$IO61X_BufferFifo@UIO61X_CanFdMessage_T@@@@PAX@1@PBV?$_List_val@U?$_List_simple_types@V?$IO61X_BufferFifo@UIO61X_CanFdMessage_T@@@@@std@@@1@@Z 10072d20 f i IO61X_Library_MSVC120_vc:IO61X_CanFdPort.obj
 0001:00071d30       ??0?$_List_val@U?$_List_simple_types@V?$IO61X_BufferFifo@UIO61X_CanFdMessage_T@@@@@std@@@std@@QAE@XZ 10072d30 f i IO61X_Library_MSVC120_vc:IO61X_CanFdPort.obj
 0001:00071d40       ??0?$_Wrap_alloc@V?$allocator@U?$_List_node@V?$IO61X_BufferFifo@UIO61X_CanFdMessage_T@@@@PAX@std@@@std@@@std@@QAE@XZ 10072d40 f i IO61X_Library_MSVC120_vc:IO61X_CanFdPort.obj
 0001:00071d50       ??0?$allocator@U?$_List_node@V?$IO61X_BufferFifo@UIO61X_CanFdMessage_T@@@@PAX@std@@@std@@QAE@XZ 10072d50 f i IO61X_Library_MSVC120_vc:IO61X_CanFdPort.obj
 0001:00071d60       ??0?$allocator@V?$IO61X_BufferFifo@UIO61X_CanFdMessage_T@@@@@std@@QAE@XZ 10072d60 f i IO61X_Library_MSVC120_vc:IO61X_CanFdPort.obj
 0001:00071d70       ??0?$list@V?$IO61X_BufferFifo@UIO61X_CanFdMessage_T@@@@V?$allocator@V?$IO61X_BufferFifo@UIO61X_CanFdMessage_T@@@@@std@@@std@@QAE@XZ 10072d70 f i IO61X_Library_MSVC120_vc:IO61X_CanFdPort.obj
 0001:00071d90       ??0IO61X_CanFdPort@@QAE@II_N@Z 10072d90 f   IO61X_Library_MSVC120_vc:IO61X_CanFdPort.obj
 0001:00071e50       ??1?$IO61X_BufferFifo@UIO61X_CanFdMessage_T@@@@QAE@XZ 10072e50 f i IO61X_Library_MSVC120_vc:IO61X_CanFdPort.obj
 0001:00071e60       ??1?$_List_alloc@$0A@U?$_List_base_types@V?$IO61X_BufferFifo@UIO61X_CanFdMessage_T@@@@V?$allocator@V?$IO61X_BufferFifo@UIO61X_CanFdMessage_T@@@@@std@@@std@@@std@@QAE@XZ 10072e60 f i IO61X_Library_MSVC120_vc:IO61X_CanFdPort.obj
 0001:00071e70       ??1?$_List_buy@V?$IO61X_BufferFifo@UIO61X_CanFdMessage_T@@@@V?$allocator@V?$IO61X_BufferFifo@UIO61X_CanFdMessage_T@@@@@std@@@std@@QAE@XZ 10072e70 f i IO61X_Library_MSVC120_vc:IO61X_CanFdPort.obj
 0001:00071e80       ??1?$list@V?$IO61X_BufferFifo@UIO61X_CanFdMessage_T@@@@V?$allocator@V?$IO61X_BufferFifo@UIO61X_CanFdMessage_T@@@@@std@@@std@@QAE@XZ 10072e80 f i IO61X_Library_MSVC120_vc:IO61X_CanFdPort.obj
 0001:00071ea0       ??1IO61X_CanFdPort@@UAE@XZ 10072ea0 f   IO61X_Library_MSVC120_vc:IO61X_CanFdPort.obj
 0001:00071ee0       ??8?$_List_const_iterator@V?$_List_val@U?$_List_simple_types@V?$IO61X_BufferFifo@UIO61X_CanFdMessage_T@@@@@std@@@std@@@std@@QBE_NABV01@@Z 10072ee0 f i IO61X_Library_MSVC120_vc:IO61X_CanFdPort.obj
 0001:00071f00       ??9?$_List_const_iterator@V?$_List_val@U?$_List_simple_types@V?$IO61X_BufferFifo@UIO61X_CanFdMessage_T@@@@@std@@@std@@@std@@QBE_NABV01@@Z 10072f00 f i IO61X_Library_MSVC120_vc:IO61X_CanFdPort.obj
 0001:00071f20       ??D?$_List_const_iterator@V?$_List_val@U?$_List_simple_types@V?$IO61X_BufferFifo@UIO61X_CanFdMessage_T@@@@@std@@@std@@@std@@QBEABV?$IO61X_BufferFifo@UIO61X_CanFdMessage_T@@@@XZ 10072f20 f i IO61X_Library_MSVC120_vc:IO61X_CanFdPort.obj
 0001:00071f30       ??D?$_List_iterator@V?$_List_val@U?$_List_simple_types@V?$IO61X_BufferFifo@UIO61X_CanFdMessage_T@@@@@std@@@std@@@std@@QBEAAV?$IO61X_BufferFifo@UIO61X_CanFdMessage_T@@@@XZ 10072f30 f i IO61X_Library_MSVC120_vc:IO61X_CanFdPort.obj
 0001:00071f40       ??E?$_List_const_iterator@V?$_List_val@U?$_List_simple_types@V?$IO61X_BufferFifo@UIO61X_CanFdMessage_T@@@@@std@@@std@@@std@@QAEAAV01@XZ 10072f40 f i IO61X_Library_MSVC120_vc:IO61X_CanFdPort.obj
 0001:00071f50       ??E?$_List_iterator@V?$_List_val@U?$_List_simple_types@V?$IO61X_BufferFifo@UIO61X_CanFdMessage_T@@@@@std@@@std@@@std@@QAE?AV01@H@Z 10072f50 f i IO61X_Library_MSVC120_vc:IO61X_CanFdPort.obj
 0001:00071f70       ??E?$_List_iterator@V?$_List_val@U?$_List_simple_types@V?$IO61X_BufferFifo@UIO61X_CanFdMessage_T@@@@@std@@@std@@@std@@QAEAAV01@XZ 10072f70 f i IO61X_Library_MSVC120_vc:IO61X_CanFdPort.obj
 0001:00071f80       ??F?$_List_const_iterator@V?$_List_val@U?$_List_simple_types@V?$IO61X_BufferFifo@UIO61X_CanFdMessage_T@@@@@std@@@std@@@std@@QAEAAV01@XZ 10072f80 f i IO61X_Library_MSVC120_vc:IO61X_CanFdPort.obj
 0001:00071f90       ??F?$_List_iterator@V?$_List_val@U?$_List_simple_types@V?$IO61X_BufferFifo@UIO61X_CanFdMessage_T@@@@@std@@@std@@@std@@QAEAAV01@XZ 10072f90 f i IO61X_Library_MSVC120_vc:IO61X_CanFdPort.obj
 0001:00071fa0       ??_G?$IO61X_BufferFifo@UIO61X_CanFdMessage_T@@@@QAEPAXI@Z 10072fa0 f i IO61X_Library_MSVC120_vc:IO61X_CanFdPort.obj
 0001:00071fd0       ??_GIO61X_CanFdPort@@UAEPAXI@Z 10072fd0 f i IO61X_Library_MSVC120_vc:IO61X_CanFdPort.obj
 0001:00071fd0       ??_EIO61X_CanFdPort@@UAEPAXI@Z 10072fd0 f i IO61X_Library_MSVC120_vc:IO61X_CanFdPort.obj
 0001:00072020       ?AddMessageToBuffer@?$IO61X_BufferFifo@UIO61X_CanFdMessage_T@@@@QAE_NPBUIO61X_CanFdMessage_T@@@Z 10073020 f i IO61X_Library_MSVC120_vc:IO61X_CanFdPort.obj
 0001:00072090       ?AllocateBuffer_spin@IO61X_CanFdPort@@UAEPAX_NI@Z 10073090 f   IO61X_Library_MSVC120_vc:IO61X_CanFdPort.obj
 0001:00072190       ?ClearBufferList@IO61X_CanFdPort@@UAE_NXZ 10073190 f   IO61X_Library_MSVC120_vc:IO61X_CanFdPort.obj
 0001:000721b0       ?GetMessageFromBuffer@?$IO61X_BufferFifo@UIO61X_CanFdMessage_T@@@@QAEPAUIO61X_CanFdMessage_T@@XZ 100731b0 f i IO61X_Library_MSVC120_vc:IO61X_CanFdPort.obj
 0001:000721d0       ?Receive_spin@IO61X_CanFdPort@@UAE_NH@Z 100731d0 f i IO61X_Library_MSVC120_vc:IO61X_CanFdPort.obj
 0001:000721e0       ?Send_spin@IO61X_CanFdPort@@UAE_NXZ 100731e0 f   IO61X_Library_MSVC120_vc:IO61X_CanFdPort.obj
 0001:00072350       ?UpdateBuffer_spin@IO61X_CanFdPort@@UAE_NPAX0@Z 10073350 f   IO61X_Library_MSVC120_vc:IO61X_CanFdPort.obj
 0001:00072370       ?_Buyheadnode@?$_List_alloc@$0A@U?$_List_base_types@V?$IO61X_BufferFifo@UIO61X_CanFdMessage_T@@@@V?$allocator@V?$IO61X_BufferFifo@UIO61X_CanFdMessage_T@@@@@std@@@std@@@std@@QAEPAU?$_List_node@V?$IO61X_BufferFifo@UIO61X_CanFdMessage_T@@@@PAX@2@XZ 10073370 f i IO61X_Library_MSVC120_vc:IO61X_CanFdPort.obj
 0001:00072380       ?_Buynode0@?$_List_alloc@$0A@U?$_List_base_types@V?$IO61X_BufferFifo@UIO61X_CanFdMessage_T@@@@V?$allocator@V?$IO61X_BufferFifo@UIO61X_CanFdMessage_T@@@@@std@@@std@@@std@@QAEPAU?$_List_node@V?$IO61X_BufferFifo@UIO61X_CanFdMessage_T@@@@PAX@2@PAU32@0@Z 10073380 f i IO61X_Library_MSVC120_vc:IO61X_CanFdPort.obj
 0001:000723c0       ?_Freeheadnode@?$_List_alloc@$0A@U?$_List_base_types@V?$IO61X_BufferFifo@UIO61X_CanFdMessage_T@@@@V?$allocator@V?$IO61X_BufferFifo@UIO61X_CanFdMessage_T@@@@@std@@@std@@@std@@QAEXPAU?$_List_node@V?$IO61X_BufferFifo@UIO61X_CanFdMessage_T@@@@PAX@2@@Z 100733c0 f i IO61X_Library_MSVC120_vc:IO61X_CanFdPort.obj
 0001:000723e0       ?_Freenode@?$_List_buy@V?$IO61X_BufferFifo@UIO61X_CanFdMessage_T@@@@V?$allocator@V?$IO61X_BufferFifo@UIO61X_CanFdMessage_T@@@@@std@@@std@@QAEXPAU?$_List_node@V?$IO61X_BufferFifo@UIO61X_CanFdMessage_T@@@@PAX@2@@Z 100733e0 f i IO61X_Library_MSVC120_vc:IO61X_CanFdPort.obj
 0001:00072410       ?_Getal@?$_List_alloc@$0A@U?$_List_base_types@V?$IO61X_BufferFifo@UIO61X_CanFdMessage_T@@@@V?$allocator@V?$IO61X_BufferFifo@UIO61X_CanFdMessage_T@@@@@std@@@std@@@std@@QBE?AU?$_Wrap_alloc@V?$allocator@U?$_List_node@V?$IO61X_BufferFifo@UIO61X_CanFdMessage_T@@@@PAX@std@@@std@@@2@XZ 10073410 f i IO61X_Library_MSVC120_vc:IO61X_CanFdPort.obj
 0001:00072420       ?_Incsize@?$list@V?$IO61X_BufferFifo@UIO61X_CanFdMessage_T@@@@V?$allocator@V?$IO61X_BufferFifo@UIO61X_CanFdMessage_T@@@@@std@@@std@@QAEXI@Z 10073420 f i IO61X_Library_MSVC120_vc:IO61X_CanFdPort.obj
 0001:00072450       ?_Mynode@?$_List_unchecked_const_iterator@V?$_List_val@U?$_List_simple_types@V?$IO61X_BufferFifo@UIO61X_CanFdMessage_T@@@@@std@@@std@@U_Iterator_base0@2@@std@@QBEPAU?$_List_node@V?$IO61X_BufferFifo@UIO61X_CanFdMessage_T@@@@PAX@2@XZ 10073450 f i IO61X_Library_MSVC120_vc:IO61X_CanFdPort.obj
 0001:00072460       ?_Myval@?$_List_val@U?$_List_simple_types@V?$IO61X_BufferFifo@UIO61X_CanFdMessage_T@@@@@std@@@std@@SAAAV?$IO61X_BufferFifo@UIO61X_CanFdMessage_T@@@@PAU?$_List_node@V?$IO61X_BufferFifo@UIO61X_CanFdMessage_T@@@@PAX@2@@Z 10073460 f i IO61X_Library_MSVC120_vc:IO61X_CanFdPort.obj
 0001:00072470       ?_Nextnode@?$_List_val@U?$_List_simple_types@V?$IO61X_BufferFifo@UIO61X_CanFdMessage_T@@@@@std@@@std@@SAAAPAU?$_List_node@V?$IO61X_BufferFifo@UIO61X_CanFdMessage_T@@@@PAX@2@PAU32@@Z 10073470 f i IO61X_Library_MSVC120_vc:IO61X_CanFdPort.obj
 0001:00072480       ?_Prevnode@?$_List_val@U?$_List_simple_types@V?$IO61X_BufferFifo@UIO61X_CanFdMessage_T@@@@@std@@@std@@SAAAPAU?$_List_node@V?$IO61X_BufferFifo@UIO61X_CanFdMessage_T@@@@PAX@2@PAU32@@Z 10073480 f i IO61X_Library_MSVC120_vc:IO61X_CanFdPort.obj
 0001:00072490       ?_Tidy@?$list@V?$IO61X_BufferFifo@UIO61X_CanFdMessage_T@@@@V?$allocator@V?$IO61X_BufferFifo@UIO61X_CanFdMessage_T@@@@@std@@@std@@QAEXXZ 10073490 f i IO61X_Library_MSVC120_vc:IO61X_CanFdPort.obj
 0001:000724a0       ?_Unchecked_end@?$list@V?$IO61X_BufferFifo@UIO61X_CanFdMessage_T@@@@V?$allocator@V?$IO61X_BufferFifo@UIO61X_CanFdMessage_T@@@@@std@@@std@@QAE?AV?$_List_unchecked_iterator@V?$_List_val@U?$_List_simple_types@V?$IO61X_BufferFifo@UIO61X_CanFdMessage_T@@@@@std@@@std@@@2@XZ 100734a0 f i IO61X_Library_MSVC120_vc:IO61X_CanFdPort.obj
 0001:000724b0       ?_UpdateBufferForCan@IO61X_CanFdPort@@AAE_NPAX0@Z 100734b0 f   IO61X_Library_MSVC120_vc:IO61X_CanFdPort.obj
 0001:00072580       ?_UpdateBufferForFd@IO61X_CanFdPort@@AAE_NPAX0@Z 10073580 f   IO61X_Library_MSVC120_vc:IO61X_CanFdPort.obj
 0001:00072670       ?allocate@?$_Wrap_alloc@V?$allocator@U?$_List_node@V?$IO61X_BufferFifo@UIO61X_CanFdMessage_T@@@@PAX@std@@@std@@@std@@QAEPAU?$_List_node@V?$IO61X_BufferFifo@UIO61X_CanFdMessage_T@@@@PAX@2@I@Z 10073670 f i IO61X_Library_MSVC120_vc:IO61X_CanFdPort.obj
 0001:000726b0       ?allocate@?$allocator@U?$_List_node@V?$IO61X_BufferFifo@UIO61X_CanFdMessage_T@@@@PAX@std@@@std@@QAEPAU?$_List_node@V?$IO61X_BufferFifo@UIO61X_CanFdMessage_T@@@@PAX@2@I@Z 100736b0 f i IO61X_Library_MSVC120_vc:IO61X_CanFdPort.obj
 0001:000726f0       ?back@?$list@V?$IO61X_BufferFifo@UIO61X_CanFdMessage_T@@@@V?$allocator@V?$IO61X_BufferFifo@UIO61X_CanFdMessage_T@@@@@std@@@std@@QAEAAV?$IO61X_BufferFifo@UIO61X_CanFdMessage_T@@@@XZ 100736f0 f i IO61X_Library_MSVC120_vc:IO61X_CanFdPort.obj
 0001:00072700       ?begin@?$list@V?$IO61X_BufferFifo@UIO61X_CanFdMessage_T@@@@V?$allocator@V?$IO61X_BufferFifo@UIO61X_CanFdMessage_T@@@@@std@@@std@@QAE?AV?$_List_iterator@V?$_List_val@U?$_List_simple_types@V?$IO61X_BufferFifo@UIO61X_CanFdMessage_T@@@@@std@@@std@@@2@XZ 10073700 f i IO61X_Library_MSVC120_vc:IO61X_CanFdPort.obj
 0001:00072710       ?clear@?$list@V?$IO61X_BufferFifo@UIO61X_CanFdMessage_T@@@@V?$allocator@V?$IO61X_BufferFifo@UIO61X_CanFdMessage_T@@@@@std@@@std@@QAEXXZ 10073710 f i IO61X_Library_MSVC120_vc:IO61X_CanFdPort.obj
 0001:00072760       ?deallocate@?$_Wrap_alloc@V?$allocator@U?$_List_node@V?$IO61X_BufferFifo@UIO61X_CanFdMessage_T@@@@PAX@std@@@std@@@std@@QAEXPAU?$_List_node@V?$IO61X_BufferFifo@UIO61X_CanFdMessage_T@@@@PAX@2@I@Z 10073760 f i IO61X_Library_MSVC120_vc:IO61X_CanFdPort.obj
 0001:00072780       ?deallocate@?$allocator@U?$_List_node@V?$IO61X_BufferFifo@UIO61X_CanFdMessage_T@@@@PAX@std@@@std@@QAEXPAU?$_List_node@V?$IO61X_BufferFifo@UIO61X_CanFdMessage_T@@@@PAX@2@I@Z 10073780 f i IO61X_Library_MSVC120_vc:IO61X_CanFdPort.obj
 0001:000727a0       ?empty@?$list@V?$IO61X_BufferFifo@UIO61X_CanFdMessage_T@@@@V?$allocator@V?$IO61X_BufferFifo@UIO61X_CanFdMessage_T@@@@@std@@@std@@QBE_NXZ 100737a0 f i IO61X_Library_MSVC120_vc:IO61X_CanFdPort.obj
 0001:000727b0       ?end@?$list@V?$IO61X_BufferFifo@UIO61X_CanFdMessage_T@@@@V?$allocator@V?$IO61X_BufferFifo@UIO61X_CanFdMessage_T@@@@@std@@@std@@QAE?AV?$_List_iterator@V?$_List_val@U?$_List_simple_types@V?$IO61X_BufferFifo@UIO61X_CanFdMessage_T@@@@@std@@@std@@@2@XZ 100737b0 f i IO61X_Library_MSVC120_vc:IO61X_CanFdPort.obj
 0001:000727c0       ?getReadIdx@?$IO61X_BufferFifo@UIO61X_CanFdMessage_T@@@@QAEHXZ 100737c0 f i IO61X_Library_MSVC120_vc:IO61X_CanFdPort.obj
 0001:000727d0       ?getWriteIdx@?$IO61X_BufferFifo@UIO61X_CanFdMessage_T@@@@QAEHXZ 100737d0 f i IO61X_Library_MSVC120_vc:IO61X_CanFdPort.obj
 0001:000727e0       ?max_size@?$_Wrap_alloc@V?$allocator@U?$_List_node@V?$IO61X_BufferFifo@UIO61X_CanFdMessage_T@@@@PAX@std@@@std@@@std@@QBEIXZ 100737e0 f i IO61X_Library_MSVC120_vc:IO61X_CanFdPort.obj
 0001:000727f0       ?max_size@?$allocator@U?$_List_node@V?$IO61X_BufferFifo@UIO61X_CanFdMessage_T@@@@PAX@std@@@std@@QBEIXZ 100737f0 f i IO61X_Library_MSVC120_vc:IO61X_CanFdPort.obj
 0001:00072800       ?max_size@?$allocator_traits@V?$allocator@U?$_List_node@V?$IO61X_BufferFifo@UIO61X_CanFdMessage_T@@@@PAX@std@@@std@@@std@@SAIABV?$allocator@U?$_List_node@V?$IO61X_BufferFifo@UIO61X_CanFdMessage_T@@@@PAX@std@@@2@@Z 10073800 f i IO61X_Library_MSVC120_vc:IO61X_CanFdPort.obj
 0001:00072810       ?max_size@?$list@V?$IO61X_BufferFifo@UIO61X_CanFdMessage_T@@@@V?$allocator@V?$IO61X_BufferFifo@UIO61X_CanFdMessage_T@@@@@std@@@std@@QBEIXZ 10073810 f i IO61X_Library_MSVC120_vc:IO61X_CanFdPort.obj
 0001:00072820       ?push_back@?$list@V?$IO61X_BufferFifo@UIO61X_CanFdMessage_T@@@@V?$allocator@V?$IO61X_BufferFifo@UIO61X_CanFdMessage_T@@@@@std@@@std@@QAEX$$QAV?$IO61X_BufferFifo@UIO61X_CanFdMessage_T@@@@@Z 10073820 f i IO61X_Library_MSVC120_vc:IO61X_CanFdPort.obj
 0001:00072870       ?setReadIdx@?$IO61X_BufferFifo@UIO61X_CanFdMessage_T@@@@QAEXH@Z 10073870 f i IO61X_Library_MSVC120_vc:IO61X_CanFdPort.obj
 0001:00072880       ?setWriteIdx@?$IO61X_BufferFifo@UIO61X_CanFdMessage_T@@@@QAEXH@Z 10073880 f i IO61X_Library_MSVC120_vc:IO61X_CanFdPort.obj
 0001:00072890       ?IO61X_SetStatusHandling@@YA_NIE@Z 10073890 f   IO61X_Library_MSVC120_vc:IO61X_StatusManager.obj
 0001:00072910       ?IO61X_BusRecoveryThread@@YAPAXPAX@Z 10073910 f   IO61X_Library_MSVC120_vc:IO61X_ThreadManager.obj
 0001:00072a30       ?IO61X_CanBusRecovery@@YAXIE@Z 10073a30 f   IO61X_Library_MSVC120_vc:IO61X_ThreadManager.obj
 0001:00072cb0       ?IO61X_ClearBusRecoveryThread@@YAXI@Z 10073cb0 f   IO61X_Library_MSVC120_vc:IO61X_ThreadManager.obj
 0001:00072d70       ?IO61X_CreateBusRecoverySemaphore@@YA_NI@Z 10073d70 f   IO61X_Library_MSVC120_vc:IO61X_ThreadManager.obj
 0001:00072db0       ?IO61X_CreateBusRecoveryThread@@YA_NIEP6APAXPAX@Z@Z 10073db0 f   IO61X_Library_MSVC120_vc:IO61X_ThreadManager.obj
 0001:00072e20       ?IO61X_AllocateLinPortMemory@@YA_NIE@Z 10073e20 f   IO61X_Library_MSVC120_vc:IO61X_LinManager.obj
 0001:00072f00       ?IO61X_DoLinControllerInit@@YA_NIE@Z 10073f00 f   IO61X_Library_MSVC120_vc:IO61X_LinManager.obj
 0001:00072f40       ?IO61X_InitLin@@YA_NIEW4IO61X_PtMbxDirecVals_E@@I@Z 10073f40 f   IO61X_Library_MSVC120_vc:IO61X_LinManager.obj
 0001:000730c0       ?IO61X_LINRwwbAcqWrtIdx@@YAXIE@Z 100740c0 f   IO61X_Library_MSVC120_vc:IO61X_LinManager.obj
 0001:00073170       ?IO61X_LINRwwbRlsWrtIdx@@YAXIE@Z 10074170 f   IO61X_Library_MSVC120_vc:IO61X_LinManager.obj
 0001:000731a0       ?IO61X_LINSndRecPtStatInfo@@YA_NIW4IO61X_PtMbxDirecVals_E@@I@Z 100741a0 f   IO61X_Library_MSVC120_vc:IO61X_LinManager.obj
 0001:00073350       ?IO61X_ReadLinMessageFromReceiveQueue@@YAEPAUIO61X_ComMbxObj_T@@PAUIO61X_LinMessageObject_T@@@Z 10074350 f   IO61X_Library_MSVC120_vc:IO61X_LinManager.obj
 0001:000733a0       ?IO61X_SetLinPortValues@@YA_NIEEIEEW4IO61X_PortType_E@@@Z 100743a0 f   IO61X_Library_MSVC120_vc:IO61X_LinManager.obj
 0001:000734a0       ?IO61X_StartLin@@YA_NIEW4IO61X_PtMbxDirecVals_E@@I@Z 100744a0 f   IO61X_Library_MSVC120_vc:IO61X_LinManager.obj
 0001:000735d0       ?IO61X_StopLin@@YA_NIEW4IO61X_PtMbxDirecVals_E@@I@Z 100745d0 f   IO61X_Library_MSVC120_vc:IO61X_LinManager.obj
 0001:000736f0       ?IO61X_WriteLinMasterMessageToSendQueue@@YAEPBUIO61X_LinMessageObject_T@@PCIPAUIO61X_ComMbxObj_T@@@Z 100746f0 f   IO61X_Library_MSVC120_vc:IO61X_LinManager.obj
 0001:00073740       ??$?0AAIV?$IO61X_BufferFifo@UIO61X_LinMessage_T@@@@X@?$pair@HV?$IO61X_BufferFifo@UIO61X_LinMessage_T@@@@@std@@QAE@AAI$$QAV?$IO61X_BufferFifo@UIO61X_LinMessage_T@@@@@Z 10074740 f i IO61X_Library_MSVC120_vc:IO61X_LinPort.obj
 0001:00073760       ??$?0HV?$IO61X_BufferFifo@UIO61X_LinMessage_T@@@@X@?$pair@$$CBHV?$IO61X_BufferFifo@UIO61X_LinMessage_T@@@@@std@@QAE@$$QAU?$pair@HV?$IO61X_BufferFifo@UIO61X_LinMessage_T@@@@@1@@Z 10074760 f i IO61X_Library_MSVC120_vc:IO61X_LinPort.obj
 0001:00073780       ??$?0U?$pair@$$CBHV?$IO61X_BufferFifo@UIO61X_LinMessage_T@@@@@std@@@?$allocator@V?$_List_unchecked_iterator@V?$_List_val@U?$_List_simple_types@U?$pair@$$CBHV?$IO61X_BufferFifo@UIO61X_LinMessage_T@@@@@std@@@std@@@std@@@std@@@std@@QAE@ABV?$allocator@U?$pair@$$CBHV?$IO61X_BufferFifo@UIO61X_LinMessage_T@@@@@std@@@1@@Z 10074780 f i IO61X_Library_MSVC120_vc:IO61X_LinPort.obj
 0001:00073790       ??$?0V?$_List_iterator@V?$_List_val@U?$_List_simple_types@U?$pair@$$CBHV?$IO61X_BufferFifo@UIO61X_LinMessage_T@@@@@std@@@std@@@std@@@std@@_NX@?$pair@V?$_List_iterator@V?$_List_val@U?$_List_simple_types@U?$pair@$$CBHV?$IO61X_BufferFifo@UIO61X_LinMessage_T@@@@@std@@@std@@@std@@@std@@_N@std@@QAE@$$QAV?$_List_iterator@V?$_List_val@U?$_List_simple_types@U?$pair@$$CBHV?$IO61X_BufferFifo@UIO61X_LinMessage_T@@@@@std@@@std@@@std@@@1@$$QA_N@Z 10074790 f i IO61X_Library_MSVC120_vc:IO61X_LinPort.obj
 0001:000737b0       ??$?0V?$allocator@U?$pair@$$CBHV?$IO61X_BufferFifo@UIO61X_LinMessage_T@@@@@std@@@std@@@?$_Wrap_alloc@V?$allocator@V?$_List_unchecked_iterator@V?$_List_val@U?$_List_simple_types@U?$pair@$$CBHV?$IO61X_BufferFifo@UIO61X_LinMessage_T@@@@@std@@@std@@@std@@@std@@@std@@@std@@QAE@ABV?$allocator@U?$pair@$$CBHV?$IO61X_BufferFifo@UIO61X_LinMessage_T@@@@@std@@@1@@Z 100747b0 f i IO61X_Library_MSVC120_vc:IO61X_LinPort.obj
 0001:000737c0       ??$_Allocate@U?$_List_node@U?$pair@$$CBHV?$IO61X_BufferFifo@UIO61X_LinMessage_T@@@@@std@@PAX@std@@@std@@YAPAU?$_List_node@U?$pair@$$CBHV?$IO61X_BufferFifo@UIO61X_LinMessage_T@@@@@std@@PAX@0@IPAU10@@Z 100747c0 f i IO61X_Library_MSVC120_vc:IO61X_LinPort.obj
 0001:000737f0       ??$_Allocate@U?$_List_node@V?$IO61X_BufferFifo@UIO61X_LinMessage_T@@@@PAX@std@@@std@@YAPAU?$_List_node@V?$IO61X_BufferFifo@UIO61X_LinMessage_T@@@@PAX@0@IPAU10@@Z 100747f0 f i IO61X_Library_MSVC120_vc:IO61X_LinPort.obj
 0001:00073830       ??$_Allocate@V?$_List_unchecked_iterator@V?$_List_val@U?$_List_simple_types@U?$pair@$$CBHV?$IO61X_BufferFifo@UIO61X_LinMessage_T@@@@@std@@@std@@@std@@@std@@@std@@YAPAV?$_List_unchecked_iterator@V?$_List_val@U?$_List_simple_types@U?$pair@$$CBHV?$IO61X_BufferFifo@UIO61X_LinMessage_T@@@@@std@@@std@@@std@@@0@IPAV10@@Z 10074830 f i IO61X_Library_MSVC120_vc:IO61X_LinPort.obj
 0001:00073860       ??$_Buynode@U?$pair@HV?$IO61X_BufferFifo@UIO61X_LinMessage_T@@@@@std@@@?$_List_buy@U?$pair@$$CBHV?$IO61X_BufferFifo@UIO61X_LinMessage_T@@@@@std@@V?$allocator@U?$pair@$$CBHV?$IO61X_BufferFifo@UIO61X_LinMessage_T@@@@@std@@@2@@std@@QAEPAU?$_List_node@U?$pair@$$CBHV?$IO61X_BufferFifo@UIO61X_LinMessage_T@@@@@std@@PAX@1@PAU21@0$$QAU?$pair@HV?$IO61X_BufferFifo@UIO61X_LinMessage_T@@@@@1@@Z 10074860 f i IO61X_Library_MSVC120_vc:IO61X_LinPort.obj
 0001:00073900       ??$_Buynode@V?$IO61X_BufferFifo@UIO61X_LinMessage_T@@@@@?$_List_buy@V?$IO61X_BufferFifo@UIO61X_LinMessage_T@@@@V?$allocator@V?$IO61X_BufferFifo@UIO61X_LinMessage_T@@@@@std@@@std@@QAEPAU?$_List_node@V?$IO61X_BufferFifo@UIO61X_LinMessage_T@@@@PAX@1@PAU21@0$$QAV?$IO61X_BufferFifo@UIO61X_LinMessage_T@@@@@Z 10074900 f i IO61X_Library_MSVC120_vc:IO61X_LinPort.obj
 0001:00073990       ??$_Buynode_if_nil@AAU?$pair@$$CBHV?$IO61X_BufferFifo@UIO61X_LinMessage_T@@@@@std@@@?$_Hash@V?$_Umap_traits@HV?$IO61X_BufferFifo@UIO61X_LinMessage_T@@@@V?$_Uhash_compare@HU?$hash@H@std@@U?$equal_to@H@2@@std@@V?$allocator@U?$pair@$$CBHV?$IO61X_BufferFifo@UIO61X_LinMessage_T@@@@@std@@@3@$0A@@std@@@std@@IAE?AV?$_List_unchecked_iterator@V?$_List_val@U?$_List_simple_types@U?$pair@$$CBHV?$IO61X_BufferFifo@UIO61X_LinMessage_T@@@@@std@@@std@@@std@@@1@AAU?$pair@$$CBHV?$IO61X_BufferFifo@UIO61X_LinMessage_T@@@@@1@V21@@Z 10074990 f i IO61X_Library_MSVC120_vc:IO61X_LinPort.obj
 0001:000739a0       ??$_Copy_backward@PAV?$_List_unchecked_iterator@V?$_List_val@U?$_List_simple_types@U?$pair@$$CBHV?$IO61X_BufferFifo@UIO61X_LinMessage_T@@@@@std@@@std@@@std@@@std@@PAV12@@std@@YAPAV?$_List_unchecked_iterator@V?$_List_val@U?$_List_simple_types@U?$pair@$$CBHV?$IO61X_BufferFifo@UIO61X_LinMessage_T@@@@@std@@@std@@@std@@@0@PAV10@00@Z 100749a0 f i IO61X_Library_MSVC120_vc:IO61X_LinPort.obj
 0001:000739d0       ??$_Copy_backward@PAV?$_List_unchecked_iterator@V?$_List_val@U?$_List_simple_types@U?$pair@$$CBHV?$IO61X_BufferFifo@UIO61X_LinMessage_T@@@@@std@@@std@@@std@@@std@@PAV12@@std@@YAPAV?$_List_unchecked_iterator@V?$_List_val@U?$_List_simple_types@U?$pair@$$CBHV?$IO61X_BufferFifo@UIO61X_LinMessage_T@@@@@std@@@std@@@std@@@0@PAV10@00U_Nonscalar_ptr_iterator_tag@0@@Z 100749d0 f i IO61X_Library_MSVC120_vc:IO61X_LinPort.obj
 0001:00073a00       ??$_Destroy_range@U?$_Wrap_alloc@U?$_Wrap_alloc@V?$allocator@V?$_List_unchecked_iterator@V?$_List_val@U?$_List_simple_types@U?$pair@$$CBHV?$IO61X_BufferFifo@UIO61X_LinMessage_T@@@@@std@@@std@@@std@@@std@@@std@@@std@@@std@@@std@@YAXPAV?$_List_unchecked_iterator@V?$_List_val@U?$_List_simple_types@U?$pair@$$CBHV?$IO61X_BufferFifo@UIO61X_LinMessage_T@@@@@std@@@std@@@std@@@0@0AAU?$_Wrap_alloc@U?$_Wrap_alloc@V?$allocator@V?$_List_unchecked_iterator@V?$_List_val@U?$_List_simple_types@U?$pair@$$CBHV?$IO61X_BufferFifo@UIO61X_LinMessage_T@@@@@std@@@std@@@std@@@std@@@std@@@std@@@0@@Z 10074a00 f i IO61X_Library_MSVC120_vc:IO61X_LinPort.obj
 0001:00073a10       ??$_Destroy_range@U?$_Wrap_alloc@U?$_Wrap_alloc@V?$allocator@V?$_List_unchecked_iterator@V?$_List_val@U?$_List_simple_types@U?$pair@$$CBHV?$IO61X_BufferFifo@UIO61X_LinMessage_T@@@@@std@@@std@@@std@@@std@@@std@@@std@@@std@@@std@@YAXPAV?$_List_unchecked_iterator@V?$_List_val@U?$_List_simple_types@U?$pair@$$CBHV?$IO61X_BufferFifo@UIO61X_LinMessage_T@@@@@std@@@std@@@std@@@0@0AAU?$_Wrap_alloc@U?$_Wrap_alloc@V?$allocator@V?$_List_unchecked_iterator@V?$_List_val@U?$_List_simple_types@U?$pair@$$CBHV?$IO61X_BufferFifo@UIO61X_LinMessage_T@@@@@std@@@std@@@std@@@std@@@std@@@std@@@0@U_Nonscalar_ptr_iterator_tag@0@@Z 10074a10 f i IO61X_Library_MSVC120_vc:IO61X_LinPort.obj
 0001:00073a20       ??$_Fill@PAV?$_List_unchecked_iterator@V?$_List_val@U?$_List_simple_types@U?$pair@$$CBHV?$IO61X_BufferFifo@UIO61X_LinMessage_T@@@@@std@@@std@@@std@@@std@@V12@@std@@YAXPAV?$_List_unchecked_iterator@V?$_List_val@U?$_List_simple_types@U?$pair@$$CBHV?$IO61X_BufferFifo@UIO61X_LinMessage_T@@@@@std@@@std@@@std@@@0@0ABV10@@Z 10074a20 f i IO61X_Library_MSVC120_vc:IO61X_LinPort.obj
 0001:00073a60       ??$_Fn@U?$_Wrap_alloc@V?$allocator@V?$_List_unchecked_iterator@V?$_List_val@U?$_List_simple_types@U?$pair@$$CBHV?$IO61X_BufferFifo@UIO61X_LinMessage_T@@@@@std@@@std@@@std@@@std@@@std@@@std@@@_Alloc_max_size@std@@SAIHABU?$_Wrap_alloc@V?$allocator@V?$_List_unchecked_iterator@V?$_List_val@U?$_List_simple_types@U?$pair@$$CBHV?$IO61X_BufferFifo@UIO61X_LinMessage_T@@@@@std@@@std@@@std@@@std@@@std@@@1@@Z 10074a60 f i IO61X_Library_MSVC120_vc:IO61X_LinPort.obj
 0001:00073a70       ??$_Fn@U?$_Wrap_alloc@V?$allocator@V?$_List_unchecked_iterator@V?$_List_val@U?$_List_simple_types@U?$pair@$$CBHV?$IO61X_BufferFifo@UIO61X_LinMessage_T@@@@@std@@@std@@@std@@@std@@@std@@@std@@V?$_List_unchecked_iterator@V?$_List_val@U?$_List_simple_types@U?$pair@$$CBHV?$IO61X_BufferFifo@UIO61X_LinMessage_T@@@@@std@@@std@@@std@@@2@@_Alloc_destroy@std@@SAXHAAU?$_Wrap_alloc@V?$allocator@V?$_List_unchecked_iterator@V?$_List_val@U?$_List_simple_types@U?$pair@$$CBHV?$IO61X_BufferFifo@UIO61X_LinMessage_T@@@@@std@@@std@@@std@@@std@@@std@@@1@PAV?$_List_unchecked_iterator@V?$_List_val@U?$_List_simple_types@U?$pair@$$CBHV?$IO61X_BufferFifo@UIO61X_LinMessage_T@@@@@std@@@std@@@std@@@1@@Z 10074a70 f i IO61X_Library_MSVC120_vc:IO61X_LinPort.obj
 0001:00073a80       ??$_Fn@U?$_Wrap_alloc@V?$allocator@V?$_List_unchecked_iterator@V?$_List_val@U?$_List_simple_types@U?$pair@$$CBHV?$IO61X_BufferFifo@UIO61X_LinMessage_T@@@@@std@@@std@@@std@@@std@@@std@@@std@@V?$_List_unchecked_iterator@V?$_List_val@U?$_List_simple_types@U?$pair@$$CBHV?$IO61X_BufferFifo@UIO61X_LinMessage_T@@@@@std@@@std@@@std@@@2@ABV32@@_Alloc_construct@std@@SAXHAAU?$_Wrap_alloc@V?$allocator@V?$_List_unchecked_iterator@V?$_List_val@U?$_List_simple_types@U?$pair@$$CBHV?$IO61X_BufferFifo@UIO61X_LinMessage_T@@@@@std@@@std@@@std@@@std@@@std@@@1@PAV?$_List_unchecked_iterator@V?$_List_val@U?$_List_simple_types@U?$pair@$$CBHV?$IO61X_BufferFifo@UIO61X_LinMessage_T@@@@@std@@@std@@@std@@@1@ABV31@@Z 10074a80 f i IO61X_Library_MSVC120_vc:IO61X_LinPort.obj
 0001:00073aa0       ??$_Fn@U?$_Wrap_alloc@V?$allocator@V?$_List_unchecked_iterator@V?$_List_val@U?$_List_simple_types@U?$pair@$$CBHV?$IO61X_BufferFifo@UIO61X_LinMessage_T@@@@@std@@@std@@@std@@@std@@@std@@@std@@V?$_List_unchecked_iterator@V?$_List_val@U?$_List_simple_types@U?$pair@$$CBHV?$IO61X_BufferFifo@UIO61X_LinMessage_T@@@@@std@@@std@@@std@@@2@V32@@_Alloc_construct@std@@SAXHAAU?$_Wrap_alloc@V?$allocator@V?$_List_unchecked_iterator@V?$_List_val@U?$_List_simple_types@U?$pair@$$CBHV?$IO61X_BufferFifo@UIO61X_LinMessage_T@@@@@std@@@std@@@std@@@std@@@std@@@1@PAV?$_List_unchecked_iterator@V?$_List_val@U?$_List_simple_types@U?$pair@$$CBHV?$IO61X_BufferFifo@UIO61X_LinMessage_T@@@@@std@@@std@@@std@@@1@$$QAV31@@Z 10074aa0 f i IO61X_Library_MSVC120_vc:IO61X_LinPort.obj
 0001:00073ac0       ??$_Insert@AAU?$pair@$$CBHV?$IO61X_BufferFifo@UIO61X_LinMessage_T@@@@@std@@V?$_List_unchecked_iterator@V?$_List_val@U?$_List_simple_types@U?$pair@$$CBHV?$IO61X_BufferFifo@UIO61X_LinMessage_T@@@@@std@@@std@@@std@@@2@@?$_Hash@V?$_Umap_traits@HV?$IO61X_BufferFifo@UIO61X_LinMessage_T@@@@V?$_Uhash_compare@HU?$hash@H@std@@U?$equal_to@H@2@@std@@V?$allocator@U?$pair@$$CBHV?$IO61X_BufferFifo@UIO61X_LinMessage_T@@@@@std@@@3@$0A@@std@@@std@@IAE?AU?$pair@V?$_List_iterator@V?$_List_val@U?$_List_simple_types@U?$pair@$$CBHV?$IO61X_BufferFifo@UIO61X_LinMessage_T@@@@@std@@@std@@@std@@@std@@_N@1@AAU?$pair@$$CBHV?$IO61X_BufferFifo@UIO61X_LinMessage_T@@@@@1@V?$_List_unchecked_iterator@V?$_List_val@U?$_List_simple_types@U?$pair@$$CBHV?$IO61X_BufferFifo@UIO61X_LinMessage_T@@@@@std@@@std@@@std@@@1@@Z 10074ac0 f i IO61X_Library_MSVC120_vc:IO61X_LinPort.obj
 0001:00073bf0       ??$_Insert@U?$pair@HV?$IO61X_BufferFifo@UIO61X_LinMessage_T@@@@@std@@@?$list@U?$pair@$$CBHV?$IO61X_BufferFifo@UIO61X_LinMessage_T@@@@@std@@V?$allocator@U?$pair@$$CBHV?$IO61X_BufferFifo@UIO61X_LinMessage_T@@@@@std@@@2@@std@@QAEXV?$_List_unchecked_const_iterator@V?$_List_val@U?$_List_simple_types@U?$pair@$$CBHV?$IO61X_BufferFifo@UIO61X_LinMessage_T@@@@@std@@@std@@@std@@U_Iterator_base0@2@@1@$$QAU?$pair@HV?$IO61X_BufferFifo@UIO61X_LinMessage_T@@@@@1@@Z 10074bf0 f i IO61X_Library_MSVC120_vc:IO61X_LinPort.obj
 0001:00073c40       ??$_Insert@V?$IO61X_BufferFifo@UIO61X_LinMessage_T@@@@@?$list@V?$IO61X_BufferFifo@UIO61X_LinMessage_T@@@@V?$allocator@V?$IO61X_BufferFifo@UIO61X_LinMessage_T@@@@@std@@@std@@QAEXV?$_List_unchecked_const_iterator@V?$_List_val@U?$_List_simple_types@V?$IO61X_BufferFifo@UIO61X_LinMessage_T@@@@@std@@@std@@U_Iterator_base0@2@@1@$$QAV?$IO61X_BufferFifo@UIO61X_LinMessage_T@@@@@Z 10074c40 f i IO61X_Library_MSVC120_vc:IO61X_LinPort.obj
 0001:00073c90       ??$_Kfn@$$CBHV?$IO61X_BufferFifo@UIO61X_LinMessage_T@@@@@?$_Umap_traits@HV?$IO61X_BufferFifo@UIO61X_LinMessage_T@@@@V?$_Uhash_compare@HU?$hash@H@std@@U?$equal_to@H@2@@std@@V?$allocator@U?$pair@$$CBHV?$IO61X_BufferFifo@UIO61X_LinMessage_T@@@@@std@@@3@$0A@@std@@SAABHABU?$pair@$$CBHV?$IO61X_BufferFifo@UIO61X_LinMessage_T@@@@@1@@Z 10074c90 f i IO61X_Library_MSVC120_vc:IO61X_LinPort.obj
 0001:00073ca0       ??$_Ptr_cat@V?$_List_unchecked_iterator@V?$_List_val@U?$_List_simple_types@U?$pair@$$CBHV?$IO61X_BufferFifo@UIO61X_LinMessage_T@@@@@std@@@std@@@std@@@std@@V12@@std@@YA?AU_Nonscalar_ptr_iterator_tag@0@PAV?$_List_unchecked_iterator@V?$_List_val@U?$_List_simple_types@U?$pair@$$CBHV?$IO61X_BufferFifo@UIO61X_LinMessage_T@@@@@std@@@std@@@std@@@0@0@Z 10074ca0 f i IO61X_Library_MSVC120_vc:IO61X_LinPort.obj
 0001:00073cb0       ??$_Rechecked@PAV?$_List_unchecked_iterator@V?$_List_val@U?$_List_simple_types@U?$pair@$$CBHV?$IO61X_BufferFifo@UIO61X_LinMessage_T@@@@@std@@@std@@@std@@@std@@PAV12@@std@@YAAAPAV?$_List_unchecked_iterator@V?$_List_val@U?$_List_simple_types@U?$pair@$$CBHV?$IO61X_BufferFifo@UIO61X_LinMessage_T@@@@@std@@@std@@@std@@@0@AAPAV10@PAV10@@Z 10074cb0 f i IO61X_Library_MSVC120_vc:IO61X_LinPort.obj
 0001:00073cc0       ??$_Umove@PAV?$_List_unchecked_iterator@V?$_List_val@U?$_List_simple_types@U?$pair@$$CBHV?$IO61X_BufferFifo@UIO61X_LinMessage_T@@@@@std@@@std@@@std@@@std@@@?$vector@V?$_List_unchecked_iterator@V?$_List_val@U?$_List_simple_types@U?$pair@$$CBHV?$IO61X_BufferFifo@UIO61X_LinMessage_T@@@@@std@@@std@@@std@@@std@@U?$_Wrap_alloc@V?$allocator@V?$_List_unchecked_iterator@V?$_List_val@U?$_List_simple_types@U?$pair@$$CBHV?$IO61X_BufferFifo@UIO61X_LinMessage_T@@@@@std@@@std@@@std@@@std@@@std@@@2@@std@@IAEPAV?$_List_unchecked_iterator@V?$_List_val@U?$_List_simple_types@U?$pair@$$CBHV?$IO61X_BufferFifo@UIO61X_LinMessage_T@@@@@std@@@std@@@std@@@1@PAV21@00@Z 10074cc0 f i IO61X_Library_MSVC120_vc:IO61X_LinPort.obj
 0001:00073cf0       ??$_Unchecked@PAV?$_List_unchecked_iterator@V?$_List_val@U?$_List_simple_types@U?$pair@$$CBHV?$IO61X_BufferFifo@UIO61X_LinMessage_T@@@@@std@@@std@@@std@@@std@@@std@@YAPAV?$_List_unchecked_iterator@V?$_List_val@U?$_List_simple_types@U?$pair@$$CBHV?$IO61X_BufferFifo@UIO61X_LinMessage_T@@@@@std@@@std@@@std@@@0@PAV10@@Z 10074cf0 f i IO61X_Library_MSVC120_vc:IO61X_LinPort.obj
 0001:00073d00       ??$_Uninit_fill_n@PAV?$_List_unchecked_iterator@V?$_List_val@U?$_List_simple_types@U?$pair@$$CBHV?$IO61X_BufferFifo@UIO61X_LinMessage_T@@@@@std@@@std@@@std@@@std@@IV12@U?$_Wrap_alloc@V?$allocator@V?$_List_unchecked_iterator@V?$_List_val@U?$_List_simple_types@U?$pair@$$CBHV?$IO61X_BufferFifo@UIO61X_LinMessage_T@@@@@std@@@std@@@std@@@std@@@std@@@2@V12@@std@@YAXPAV?$_List_unchecked_iterator@V?$_List_val@U?$_List_simple_types@U?$pair@$$CBHV?$IO61X_BufferFifo@UIO61X_LinMessage_T@@@@@std@@@std@@@std@@@0@IPBV10@AAU?$_Wrap_alloc@U?$_Wrap_alloc@V?$allocator@V?$_List_unchecked_iterator@V?$_List_val@U?$_List_simple_types@U?$pair@$$CBHV?$IO61X_BufferFifo@UIO61X_LinMessage_T@@@@@std@@@std@@@std@@@std@@@std@@@std@@@0@0U_Nonscalar_ptr_iterator_tag@0@@Z 10074d00 f i IO61X_Library_MSVC120_vc:IO61X_LinPort.obj
 0001:00073d30       ??$_Uninit_move@PAV?$_List_unchecked_iterator@V?$_List_val@U?$_List_simple_types@U?$pair@$$CBHV?$IO61X_BufferFifo@UIO61X_LinMessage_T@@@@@std@@@std@@@std@@@std@@PAV12@U?$_Wrap_alloc@U?$_Wrap_alloc@V?$allocator@V?$_List_unchecked_iterator@V?$_List_val@U?$_List_simple_types@U?$pair@$$CBHV?$IO61X_BufferFifo@UIO61X_LinMessage_T@@@@@std@@@std@@@std@@@std@@@std@@@std@@@2@@std@@YAPAV?$_List_unchecked_iterator@V?$_List_val@U?$_List_simple_types@U?$pair@$$CBHV?$IO61X_BufferFifo@UIO61X_LinMessage_T@@@@@std@@@std@@@std@@@0@PAV10@00AAU?$_Wrap_alloc@U?$_Wrap_alloc@V?$allocator@V?$_List_unchecked_iterator@V?$_List_val@U?$_List_simple_types@U?$pair@$$CBHV?$IO61X_BufferFifo@UIO61X_LinMessage_T@@@@@std@@@std@@@std@@@std@@@std@@@std@@@0@@Z 10074d30 f i IO61X_Library_MSVC120_vc:IO61X_LinPort.obj
 0001:00073d60       ??$_Uninit_move@PAV?$_List_unchecked_iterator@V?$_List_val@U?$_List_simple_types@U?$pair@$$CBHV?$IO61X_BufferFifo@UIO61X_LinMessage_T@@@@@std@@@std@@@std@@@std@@PAV12@U?$_Wrap_alloc@V?$allocator@V?$_List_unchecked_iterator@V?$_List_val@U?$_List_simple_types@U?$pair@$$CBHV?$IO61X_BufferFifo@UIO61X_LinMessage_T@@@@@std@@@std@@@std@@@std@@@std@@@2@V12@@std@@YAPAV?$_List_unchecked_iterator@V?$_List_val@U?$_List_simple_types@U?$pair@$$CBHV?$IO61X_BufferFifo@UIO61X_LinMessage_T@@@@@std@@@std@@@std@@@0@PAV10@00AAU?$_Wrap_alloc@U?$_Wrap_alloc@V?$allocator@V?$_List_unchecked_iterator@V?$_List_val@U?$_List_simple_types@U?$pair@$$CBHV?$IO61X_BufferFifo@UIO61X_LinMessage_T@@@@@std@@@std@@@std@@@std@@@std@@@std@@@0@0U_Nonscalar_ptr_iterator_tag@0@@Z 10074d60 f i IO61X_Library_MSVC120_vc:IO61X_LinPort.obj
 0001:00073da0       ??$_Uninitialized_fill_n@PAV?$_List_unchecked_iterator@V?$_List_val@U?$_List_simple_types@U?$pair@$$CBHV?$IO61X_BufferFifo@UIO61X_LinMessage_T@@@@@std@@@std@@@std@@@std@@IV12@U?$_Wrap_alloc@U?$_Wrap_alloc@V?$allocator@V?$_List_unchecked_iterator@V?$_List_val@U?$_List_simple_types@U?$pair@$$CBHV?$IO61X_BufferFifo@UIO61X_LinMessage_T@@@@@std@@@std@@@std@@@std@@@std@@@std@@@2@@std@@YAXPAV?$_List_unchecked_iterator@V?$_List_val@U?$_List_simple_types@U?$pair@$$CBHV?$IO61X_BufferFifo@UIO61X_LinMessage_T@@@@@std@@@std@@@std@@@0@IPBV10@AAU?$_Wrap_alloc@U?$_Wrap_alloc@V?$allocator@V?$_List_unchecked_iterator@V?$_List_val@U?$_List_simple_types@U?$pair@$$CBHV?$IO61X_BufferFifo@UIO61X_LinMessage_T@@@@@std@@@std@@@std@@@std@@@std@@@std@@@0@@Z 10074da0 f i IO61X_Library_MSVC120_vc:IO61X_LinPort.obj
 0001:00073dd0       ??$_Uninitialized_move@PAV?$_List_unchecked_iterator@V?$_List_val@U?$_List_simple_types@U?$pair@$$CBHV?$IO61X_BufferFifo@UIO61X_LinMessage_T@@@@@std@@@std@@@std@@@std@@PAV12@U?$_Wrap_alloc@U?$_Wrap_alloc@V?$allocator@V?$_List_unchecked_iterator@V?$_List_val@U?$_List_simple_types@U?$pair@$$CBHV?$IO61X_BufferFifo@UIO61X_LinMessage_T@@@@@std@@@std@@@std@@@std@@@std@@@std@@@2@@std@@YAPAV?$_List_unchecked_iterator@V?$_List_val@U?$_List_simple_types@U?$pair@$$CBHV?$IO61X_BufferFifo@UIO61X_LinMessage_T@@@@@std@@@std@@@std@@@0@PAV10@00AAU?$_Wrap_alloc@U?$_Wrap_alloc@V?$allocator@V?$_List_unchecked_iterator@V?$_List_val@U?$_List_simple_types@U?$pair@$$CBHV?$IO61X_BufferFifo@UIO61X_LinMessage_T@@@@@std@@@std@@@std@@@std@@@std@@@std@@@0@@Z 10074dd0 f i IO61X_Library_MSVC120_vc:IO61X_LinPort.obj
 0001:00073df0       ??$_Val_type@PAV?$_List_unchecked_iterator@V?$_List_val@U?$_List_simple_types@U?$pair@$$CBHV?$IO61X_BufferFifo@UIO61X_LinMessage_T@@@@@std@@@std@@@std@@@std@@@std@@YAPAV?$_List_unchecked_iterator@V?$_List_val@U?$_List_simple_types@U?$pair@$$CBHV?$IO61X_BufferFifo@UIO61X_LinMessage_T@@@@@std@@@std@@@std@@@0@PAV10@@Z 10074df0 f i IO61X_Library_MSVC120_vc:IO61X_LinPort.obj
 0001:00073e00       ??$addressof@$$CBV?$_List_unchecked_iterator@V?$_List_val@U?$_List_simple_types@U?$pair@$$CBHV?$IO61X_BufferFifo@UIO61X_LinMessage_T@@@@@std@@@std@@@std@@@std@@@std@@YAPBV?$_List_unchecked_iterator@V?$_List_val@U?$_List_simple_types@U?$pair@$$CBHV?$IO61X_BufferFifo@UIO61X_LinMessage_T@@@@@std@@@std@@@std@@@0@ABV10@@Z 10074e00 f i IO61X_Library_MSVC120_vc:IO61X_LinPort.obj
 0001:00073e10       ??$addressof@PAU?$_List_node@U?$pair@$$CBHV?$IO61X_BufferFifo@UIO61X_LinMessage_T@@@@@std@@PAX@std@@@std@@YAPAPAU?$_List_node@U?$pair@$$CBHV?$IO61X_BufferFifo@UIO61X_LinMessage_T@@@@@std@@PAX@0@AAPAU10@@Z 10074e10 f i IO61X_Library_MSVC120_vc:IO61X_LinPort.obj
 0001:00073e20       ??$addressof@PAU?$_List_node@V?$IO61X_BufferFifo@UIO61X_LinMessage_T@@@@PAX@std@@@std@@YAPAPAU?$_List_node@V?$IO61X_BufferFifo@UIO61X_LinMessage_T@@@@PAX@0@AAPAU10@@Z 10074e20 f i IO61X_Library_MSVC120_vc:IO61X_LinPort.obj
 0001:00073e30       ??$addressof@U?$pair@$$CBHV?$IO61X_BufferFifo@UIO61X_LinMessage_T@@@@@std@@@std@@YAPAU?$pair@$$CBHV?$IO61X_BufferFifo@UIO61X_LinMessage_T@@@@@0@AAU10@@Z 10074e30 f i IO61X_Library_MSVC120_vc:IO61X_LinPort.obj
 0001:00073e40       ??$addressof@V?$IO61X_BufferFifo@UIO61X_LinMessage_T@@@@@std@@YAPAV?$IO61X_BufferFifo@UIO61X_LinMessage_T@@@@AAV1@@Z 10074e40 f i IO61X_Library_MSVC120_vc:IO61X_LinPort.obj
 0001:00073e50       ??$addressof@V?$_List_unchecked_iterator@V?$_List_val@U?$_List_simple_types@U?$pair@$$CBHV?$IO61X_BufferFifo@UIO61X_LinMessage_T@@@@@std@@@std@@@std@@@std@@@std@@YAPAV?$_List_unchecked_iterator@V?$_List_val@U?$_List_simple_types@U?$pair@$$CBHV?$IO61X_BufferFifo@UIO61X_LinMessage_T@@@@@std@@@std@@@std@@@0@AAV10@@Z 10074e50 f i IO61X_Library_MSVC120_vc:IO61X_LinPort.obj
 0001:00073e60       ??$construct@PAU?$_List_node@U?$pair@$$CBHV?$IO61X_BufferFifo@UIO61X_LinMessage_T@@@@@std@@PAX@std@@AAPAU12@@?$_Wrap_alloc@V?$allocator@U?$_List_node@U?$pair@$$CBHV?$IO61X_BufferFifo@UIO61X_LinMessage_T@@@@@std@@PAX@std@@@std@@@std@@QAEXPAPAU?$_List_node@U?$pair@$$CBHV?$IO61X_BufferFifo@UIO61X_LinMessage_T@@@@@std@@PAX@1@AAPAU21@@Z 10074e60 f i IO61X_Library_MSVC120_vc:IO61X_LinPort.obj
 0001:00073e80       ??$construct@PAU?$_List_node@U?$pair@$$CBHV?$IO61X_BufferFifo@UIO61X_LinMessage_T@@@@@std@@PAX@std@@AAPAU12@@?$allocator@U?$_List_node@U?$pair@$$CBHV?$IO61X_BufferFifo@UIO61X_LinMessage_T@@@@@std@@PAX@std@@@std@@QAEXPAPAU?$_List_node@U?$pair@$$CBHV?$IO61X_BufferFifo@UIO61X_LinMessage_T@@@@@std@@PAX@1@AAPAU21@@Z 10074e80 f i IO61X_Library_MSVC120_vc:IO61X_LinPort.obj
 0001:00073ea0       ??$construct@PAU?$_List_node@U?$pair@$$CBHV?$IO61X_BufferFifo@UIO61X_LinMessage_T@@@@@std@@PAX@std@@AAPAU12@@?$allocator_traits@V?$allocator@U?$_List_node@U?$pair@$$CBHV?$IO61X_BufferFifo@UIO61X_LinMessage_T@@@@@std@@PAX@std@@@std@@@std@@SAXAAV?$allocator@U?$_List_node@U?$pair@$$CBHV?$IO61X_BufferFifo@UIO61X_LinMessage_T@@@@@std@@PAX@std@@@1@PAPAU?$_List_node@U?$pair@$$CBHV?$IO61X_BufferFifo@UIO61X_LinMessage_T@@@@@std@@PAX@1@AAPAU31@@Z 10074ea0 f i IO61X_Library_MSVC120_vc:IO61X_LinPort.obj
 0001:00073ec0       ??$construct@PAU?$_List_node@V?$IO61X_BufferFifo@UIO61X_LinMessage_T@@@@PAX@std@@AAPAU12@@?$_Wrap_alloc@V?$allocator@U?$_List_node@V?$IO61X_BufferFifo@UIO61X_LinMessage_T@@@@PAX@std@@@std@@@std@@QAEXPAPAU?$_List_node@V?$IO61X_BufferFifo@UIO61X_LinMessage_T@@@@PAX@1@AAPAU21@@Z 10074ec0 f i IO61X_Library_MSVC120_vc:IO61X_LinPort.obj
 0001:00073ee0       ??$construct@PAU?$_List_node@V?$IO61X_BufferFifo@UIO61X_LinMessage_T@@@@PAX@std@@AAPAU12@@?$allocator@U?$_List_node@V?$IO61X_BufferFifo@UIO61X_LinMessage_T@@@@PAX@std@@@std@@QAEXPAPAU?$_List_node@V?$IO61X_BufferFifo@UIO61X_LinMessage_T@@@@PAX@1@AAPAU21@@Z 10074ee0 f i IO61X_Library_MSVC120_vc:IO61X_LinPort.obj
 0001:00073f00       ??$construct@PAU?$_List_node@V?$IO61X_BufferFifo@UIO61X_LinMessage_T@@@@PAX@std@@AAPAU12@@?$allocator_traits@V?$allocator@U?$_List_node@V?$IO61X_BufferFifo@UIO61X_LinMessage_T@@@@PAX@std@@@std@@@std@@SAXAAV?$allocator@U?$_List_node@V?$IO61X_BufferFifo@UIO61X_LinMessage_T@@@@PAX@std@@@1@PAPAU?$_List_node@V?$IO61X_BufferFifo@UIO61X_LinMessage_T@@@@PAX@1@AAPAU31@@Z 10074f00 f i IO61X_Library_MSVC120_vc:IO61X_LinPort.obj
 0001:00073f20       ??$construct@U?$pair@$$CBHV?$IO61X_BufferFifo@UIO61X_LinMessage_T@@@@@std@@U?$pair@HV?$IO61X_BufferFifo@UIO61X_LinMessage_T@@@@@2@@?$_Wrap_alloc@V?$allocator@U?$_List_node@U?$pair@$$CBHV?$IO61X_BufferFifo@UIO61X_LinMessage_T@@@@@std@@PAX@std@@@std@@@std@@QAEXPAU?$pair@$$CBHV?$IO61X_BufferFifo@UIO61X_LinMessage_T@@@@@1@$$QAU?$pair@HV?$IO61X_BufferFifo@UIO61X_LinMessage_T@@@@@1@@Z 10074f20 f i IO61X_Library_MSVC120_vc:IO61X_LinPort.obj
 0001:00073f80       ??$construct@U?$pair@$$CBHV?$IO61X_BufferFifo@UIO61X_LinMessage_T@@@@@std@@U?$pair@HV?$IO61X_BufferFifo@UIO61X_LinMessage_T@@@@@2@@?$allocator@U?$_List_node@U?$pair@$$CBHV?$IO61X_BufferFifo@UIO61X_LinMessage_T@@@@@std@@PAX@std@@@std@@QAEXPAU?$pair@$$CBHV?$IO61X_BufferFifo@UIO61X_LinMessage_T@@@@@1@$$QAU?$pair@HV?$IO61X_BufferFifo@UIO61X_LinMessage_T@@@@@1@@Z 10074f80 f i IO61X_Library_MSVC120_vc:IO61X_LinPort.obj
 0001:00073fe0       ??$construct@U?$pair@$$CBHV?$IO61X_BufferFifo@UIO61X_LinMessage_T@@@@@std@@U?$pair@HV?$IO61X_BufferFifo@UIO61X_LinMessage_T@@@@@2@@?$allocator_traits@V?$allocator@U?$_List_node@U?$pair@$$CBHV?$IO61X_BufferFifo@UIO61X_LinMessage_T@@@@@std@@PAX@std@@@std@@@std@@SAXAAV?$allocator@U?$_List_node@U?$pair@$$CBHV?$IO61X_BufferFifo@UIO61X_LinMessage_T@@@@@std@@PAX@std@@@1@PAU?$pair@$$CBHV?$IO61X_BufferFifo@UIO61X_LinMessage_T@@@@@1@$$QAU?$pair@HV?$IO61X_BufferFifo@UIO61X_LinMessage_T@@@@@1@@Z 10074fe0 f i IO61X_Library_MSVC120_vc:IO61X_LinPort.obj
 0001:00074040       ??$construct@V?$IO61X_BufferFifo@UIO61X_LinMessage_T@@@@V1@@?$_Wrap_alloc@V?$allocator@U?$_List_node@V?$IO61X_BufferFifo@UIO61X_LinMessage_T@@@@PAX@std@@@std@@@std@@QAEXPAV?$IO61X_BufferFifo@UIO61X_LinMessage_T@@@@$$QAV2@@Z 10075040 f i IO61X_Library_MSVC120_vc:IO61X_LinPort.obj
 0001:00074090       ??$construct@V?$IO61X_BufferFifo@UIO61X_LinMessage_T@@@@V1@@?$allocator@U?$_List_node@V?$IO61X_BufferFifo@UIO61X_LinMessage_T@@@@PAX@std@@@std@@QAEXPAV?$IO61X_BufferFifo@UIO61X_LinMessage_T@@@@$$QAV2@@Z 10075090 f i IO61X_Library_MSVC120_vc:IO61X_LinPort.obj
 0001:000740e0       ??$construct@V?$IO61X_BufferFifo@UIO61X_LinMessage_T@@@@V1@@?$allocator_traits@V?$allocator@U?$_List_node@V?$IO61X_BufferFifo@UIO61X_LinMessage_T@@@@PAX@std@@@std@@@std@@SAXAAV?$allocator@U?$_List_node@V?$IO61X_BufferFifo@UIO61X_LinMessage_T@@@@PAX@std@@@1@PAV?$IO61X_BufferFifo@UIO61X_LinMessage_T@@@@$$QAV3@@Z 100750e0 f i IO61X_Library_MSVC120_vc:IO61X_LinPort.obj
 0001:00074130       ??$construct@V?$_List_unchecked_iterator@V?$_List_val@U?$_List_simple_types@U?$pair@$$CBHV?$IO61X_BufferFifo@UIO61X_LinMessage_T@@@@@std@@@std@@@std@@@std@@ABV12@@?$_Wrap_alloc@U?$_Wrap_alloc@V?$allocator@V?$_List_unchecked_iterator@V?$_List_val@U?$_List_simple_types@U?$pair@$$CBHV?$IO61X_BufferFifo@UIO61X_LinMessage_T@@@@@std@@@std@@@std@@@std@@@std@@@std@@@std@@QAEXPAV?$_List_unchecked_iterator@V?$_List_val@U?$_List_simple_types@U?$pair@$$CBHV?$IO61X_BufferFifo@UIO61X_LinMessage_T@@@@@std@@@std@@@std@@@1@ABV21@@Z 10075130 f i IO61X_Library_MSVC120_vc:IO61X_LinPort.obj
 0001:00074150       ??$construct@V?$_List_unchecked_iterator@V?$_List_val@U?$_List_simple_types@U?$pair@$$CBHV?$IO61X_BufferFifo@UIO61X_LinMessage_T@@@@@std@@@std@@@std@@@std@@ABV12@@?$_Wrap_alloc@V?$allocator@V?$_List_unchecked_iterator@V?$_List_val@U?$_List_simple_types@U?$pair@$$CBHV?$IO61X_BufferFifo@UIO61X_LinMessage_T@@@@@std@@@std@@@std@@@std@@@std@@@std@@QAEXPAV?$_List_unchecked_iterator@V?$_List_val@U?$_List_simple_types@U?$pair@$$CBHV?$IO61X_BufferFifo@UIO61X_LinMessage_T@@@@@std@@@std@@@std@@@1@ABV21@@Z 10075150 f i IO61X_Library_MSVC120_vc:IO61X_LinPort.obj
 0001:00074170       ??$construct@V?$_List_unchecked_iterator@V?$_List_val@U?$_List_simple_types@U?$pair@$$CBHV?$IO61X_BufferFifo@UIO61X_LinMessage_T@@@@@std@@@std@@@std@@@std@@ABV12@@?$allocator_traits@U?$_Wrap_alloc@V?$allocator@V?$_List_unchecked_iterator@V?$_List_val@U?$_List_simple_types@U?$pair@$$CBHV?$IO61X_BufferFifo@UIO61X_LinMessage_T@@@@@std@@@std@@@std@@@std@@@std@@@std@@@std@@SAXAAU?$_Wrap_alloc@V?$allocator@V?$_List_unchecked_iterator@V?$_List_val@U?$_List_simple_types@U?$pair@$$CBHV?$IO61X_BufferFifo@UIO61X_LinMessage_T@@@@@std@@@std@@@std@@@std@@@std@@@1@PAV?$_List_unchecked_iterator@V?$_List_val@U?$_List_simple_types@U?$pair@$$CBHV?$IO61X_BufferFifo@UIO61X_LinMessage_T@@@@@std@@@std@@@std@@@1@ABV31@@Z 10075170 f i IO61X_Library_MSVC120_vc:IO61X_LinPort.obj
 0001:00074190       ??$construct@V?$_List_unchecked_iterator@V?$_List_val@U?$_List_simple_types@U?$pair@$$CBHV?$IO61X_BufferFifo@UIO61X_LinMessage_T@@@@@std@@@std@@@std@@@std@@ABV12@@?$allocator_traits@V?$allocator@V?$_List_unchecked_iterator@V?$_List_val@U?$_List_simple_types@U?$pair@$$CBHV?$IO61X_BufferFifo@UIO61X_LinMessage_T@@@@@std@@@std@@@std@@@std@@@std@@@std@@SAXAAV?$allocator@V?$_List_unchecked_iterator@V?$_List_val@U?$_List_simple_types@U?$pair@$$CBHV?$IO61X_BufferFifo@UIO61X_LinMessage_T@@@@@std@@@std@@@std@@@std@@@1@PAV?$_List_unchecked_iterator@V?$_List_val@U?$_List_simple_types@U?$pair@$$CBHV?$IO61X_BufferFifo@UIO61X_LinMessage_T@@@@@std@@@std@@@std@@@1@ABV31@@Z 10075190 f i IO61X_Library_MSVC120_vc:IO61X_LinPort.obj
 0001:000741b0       ??$construct@V?$_List_unchecked_iterator@V?$_List_val@U?$_List_simple_types@U?$pair@$$CBHV?$IO61X_BufferFifo@UIO61X_LinMessage_T@@@@@std@@@std@@@std@@@std@@V12@@?$_Wrap_alloc@U?$_Wrap_alloc@V?$allocator@V?$_List_unchecked_iterator@V?$_List_val@U?$_List_simple_types@U?$pair@$$CBHV?$IO61X_BufferFifo@UIO61X_LinMessage_T@@@@@std@@@std@@@std@@@std@@@std@@@std@@@std@@QAEXPAV?$_List_unchecked_iterator@V?$_List_val@U?$_List_simple_types@U?$pair@$$CBHV?$IO61X_BufferFifo@UIO61X_LinMessage_T@@@@@std@@@std@@@std@@@1@$$QAV21@@Z 100751b0 f i IO61X_Library_MSVC120_vc:IO61X_LinPort.obj
 0001:000741d0       ??$construct@V?$_List_unchecked_iterator@V?$_List_val@U?$_List_simple_types@U?$pair@$$CBHV?$IO61X_BufferFifo@UIO61X_LinMessage_T@@@@@std@@@std@@@std@@@std@@V12@@?$_Wrap_alloc@V?$allocator@V?$_List_unchecked_iterator@V?$_List_val@U?$_List_simple_types@U?$pair@$$CBHV?$IO61X_BufferFifo@UIO61X_LinMessage_T@@@@@std@@@std@@@std@@@std@@@std@@@std@@QAEXPAV?$_List_unchecked_iterator@V?$_List_val@U?$_List_simple_types@U?$pair@$$CBHV?$IO61X_BufferFifo@UIO61X_LinMessage_T@@@@@std@@@std@@@std@@@1@$$QAV21@@Z 100751d0 f i IO61X_Library_MSVC120_vc:IO61X_LinPort.obj
 0001:000741f0       ??$construct@V?$_List_unchecked_iterator@V?$_List_val@U?$_List_simple_types@U?$pair@$$CBHV?$IO61X_BufferFifo@UIO61X_LinMessage_T@@@@@std@@@std@@@std@@@std@@V12@@?$allocator@V?$_List_unchecked_iterator@V?$_List_val@U?$_List_simple_types@U?$pair@$$CBHV?$IO61X_BufferFifo@UIO61X_LinMessage_T@@@@@std@@@std@@@std@@@std@@@std@@QAEXPAV?$_List_unchecked_iterator@V?$_List_val@U?$_List_simple_types@U?$pair@$$CBHV?$IO61X_BufferFifo@UIO61X_LinMessage_T@@@@@std@@@std@@@std@@@1@$$QAV21@@Z 100751f0 f i IO61X_Library_MSVC120_vc:IO61X_LinPort.obj
 0001:00074210       ??$construct@V?$_List_unchecked_iterator@V?$_List_val@U?$_List_simple_types@U?$pair@$$CBHV?$IO61X_BufferFifo@UIO61X_LinMessage_T@@@@@std@@@std@@@std@@@std@@V12@@?$allocator_traits@U?$_Wrap_alloc@V?$allocator@V?$_List_unchecked_iterator@V?$_List_val@U?$_List_simple_types@U?$pair@$$CBHV?$IO61X_BufferFifo@UIO61X_LinMessage_T@@@@@std@@@std@@@std@@@std@@@std@@@std@@@std@@SAXAAU?$_Wrap_alloc@V?$allocator@V?$_List_unchecked_iterator@V?$_List_val@U?$_List_simple_types@U?$pair@$$CBHV?$IO61X_BufferFifo@UIO61X_LinMessage_T@@@@@std@@@std@@@std@@@std@@@std@@@1@PAV?$_List_unchecked_iterator@V?$_List_val@U?$_List_simple_types@U?$pair@$$CBHV?$IO61X_BufferFifo@UIO61X_LinMessage_T@@@@@std@@@std@@@std@@@1@$$QAV31@@Z 10075210 f i IO61X_Library_MSVC120_vc:IO61X_LinPort.obj
 0001:00074230       ??$construct@V?$_List_unchecked_iterator@V?$_List_val@U?$_List_simple_types@U?$pair@$$CBHV?$IO61X_BufferFifo@UIO61X_LinMessage_T@@@@@std@@@std@@@std@@@std@@V12@@?$allocator_traits@V?$allocator@V?$_List_unchecked_iterator@V?$_List_val@U?$_List_simple_types@U?$pair@$$CBHV?$IO61X_BufferFifo@UIO61X_LinMessage_T@@@@@std@@@std@@@std@@@std@@@std@@@std@@SAXAAV?$allocator@V?$_List_unchecked_iterator@V?$_List_val@U?$_List_simple_types@U?$pair@$$CBHV?$IO61X_BufferFifo@UIO61X_LinMessage_T@@@@@std@@@std@@@std@@@std@@@1@PAV?$_List_unchecked_iterator@V?$_List_val@U?$_List_simple_types@U?$pair@$$CBHV?$IO61X_BufferFifo@UIO61X_LinMessage_T@@@@@std@@@std@@@std@@@1@$$QAV31@@Z 10075230 f i IO61X_Library_MSVC120_vc:IO61X_LinPort.obj
 0001:00074250       ??$destroy@PAU?$_List_node@U?$pair@$$CBHV?$IO61X_BufferFifo@UIO61X_LinMessage_T@@@@@std@@PAX@std@@@?$_Wrap_alloc@V?$allocator@U?$_List_node@U?$pair@$$CBHV?$IO61X_BufferFifo@UIO61X_LinMessage_T@@@@@std@@PAX@std@@@std@@@std@@QAEXPAPAU?$_List_node@U?$pair@$$CBHV?$IO61X_BufferFifo@UIO61X_LinMessage_T@@@@@std@@PAX@1@@Z 10075250 f i IO61X_Library_MSVC120_vc:IO61X_LinPort.obj
 0001:00074260       ??$destroy@PAU?$_List_node@U?$pair@$$CBHV?$IO61X_BufferFifo@UIO61X_LinMessage_T@@@@@std@@PAX@std@@@?$allocator@U?$_List_node@U?$pair@$$CBHV?$IO61X_BufferFifo@UIO61X_LinMessage_T@@@@@std@@PAX@std@@@std@@QAEXPAPAU?$_List_node@U?$pair@$$CBHV?$IO61X_BufferFifo@UIO61X_LinMessage_T@@@@@std@@PAX@1@@Z 10075260 f i IO61X_Library_MSVC120_vc:IO61X_LinPort.obj
 0001:00074270       ??$destroy@PAU?$_List_node@U?$pair@$$CBHV?$IO61X_BufferFifo@UIO61X_LinMessage_T@@@@@std@@PAX@std@@@?$allocator_traits@V?$allocator@U?$_List_node@U?$pair@$$CBHV?$IO61X_BufferFifo@UIO61X_LinMessage_T@@@@@std@@PAX@std@@@std@@@std@@SAXAAV?$allocator@U?$_List_node@U?$pair@$$CBHV?$IO61X_BufferFifo@UIO61X_LinMessage_T@@@@@std@@PAX@std@@@1@PAPAU?$_List_node@U?$pair@$$CBHV?$IO61X_BufferFifo@UIO61X_LinMessage_T@@@@@std@@PAX@1@@Z 10075270 f i IO61X_Library_MSVC120_vc:IO61X_LinPort.obj
 0001:00074280       ??$destroy@PAU?$_List_node@V?$IO61X_BufferFifo@UIO61X_LinMessage_T@@@@PAX@std@@@?$_Wrap_alloc@V?$allocator@U?$_List_node@V?$IO61X_BufferFifo@UIO61X_LinMessage_T@@@@PAX@std@@@std@@@std@@QAEXPAPAU?$_List_node@V?$IO61X_BufferFifo@UIO61X_LinMessage_T@@@@PAX@1@@Z 10075280 f i IO61X_Library_MSVC120_vc:IO61X_LinPort.obj
 0001:00074290       ??$destroy@PAU?$_List_node@V?$IO61X_BufferFifo@UIO61X_LinMessage_T@@@@PAX@std@@@?$allocator@U?$_List_node@V?$IO61X_BufferFifo@UIO61X_LinMessage_T@@@@PAX@std@@@std@@QAEXPAPAU?$_List_node@V?$IO61X_BufferFifo@UIO61X_LinMessage_T@@@@PAX@1@@Z 10075290 f i IO61X_Library_MSVC120_vc:IO61X_LinPort.obj
 0001:000742a0       ??$destroy@PAU?$_List_node@V?$IO61X_BufferFifo@UIO61X_LinMessage_T@@@@PAX@std@@@?$allocator_traits@V?$allocator@U?$_List_node@V?$IO61X_BufferFifo@UIO61X_LinMessage_T@@@@PAX@std@@@std@@@std@@SAXAAV?$allocator@U?$_List_node@V?$IO61X_BufferFifo@UIO61X_LinMessage_T@@@@PAX@std@@@1@PAPAU?$_List_node@V?$IO61X_BufferFifo@UIO61X_LinMessage_T@@@@PAX@1@@Z 100752a0 f i IO61X_Library_MSVC120_vc:IO61X_LinPort.obj
 0001:000742b0       ??$destroy@U?$pair@$$CBHV?$IO61X_BufferFifo@UIO61X_LinMessage_T@@@@@std@@@?$_Wrap_alloc@V?$allocator@U?$_List_node@U?$pair@$$CBHV?$IO61X_BufferFifo@UIO61X_LinMessage_T@@@@@std@@PAX@std@@@std@@@std@@QAEXPAU?$pair@$$CBHV?$IO61X_BufferFifo@UIO61X_LinMessage_T@@@@@1@@Z 100752b0 f i IO61X_Library_MSVC120_vc:IO61X_LinPort.obj
 0001:000742d0       ??$destroy@U?$pair@$$CBHV?$IO61X_BufferFifo@UIO61X_LinMessage_T@@@@@std@@@?$allocator@U?$_List_node@U?$pair@$$CBHV?$IO61X_BufferFifo@UIO61X_LinMessage_T@@@@@std@@PAX@std@@@std@@QAEXPAU?$pair@$$CBHV?$IO61X_BufferFifo@UIO61X_LinMessage_T@@@@@1@@Z 100752d0 f i IO61X_Library_MSVC120_vc:IO61X_LinPort.obj
 0001:000742f0       ??$destroy@U?$pair@$$CBHV?$IO61X_BufferFifo@UIO61X_LinMessage_T@@@@@std@@@?$allocator_traits@V?$allocator@U?$_List_node@U?$pair@$$CBHV?$IO61X_BufferFifo@UIO61X_LinMessage_T@@@@@std@@PAX@std@@@std@@@std@@SAXAAV?$allocator@U?$_List_node@U?$pair@$$CBHV?$IO61X_BufferFifo@UIO61X_LinMessage_T@@@@@std@@PAX@std@@@1@PAU?$pair@$$CBHV?$IO61X_BufferFifo@UIO61X_LinMessage_T@@@@@1@@Z 100752f0 f i IO61X_Library_MSVC120_vc:IO61X_LinPort.obj
 0001:00074310       ??$destroy@V?$IO61X_BufferFifo@UIO61X_LinMessage_T@@@@@?$_Wrap_alloc@V?$allocator@U?$_List_node@V?$IO61X_BufferFifo@UIO61X_LinMessage_T@@@@PAX@std@@@std@@@std@@QAEXPAV?$IO61X_BufferFifo@UIO61X_LinMessage_T@@@@@Z 10075310 f i IO61X_Library_MSVC120_vc:IO61X_LinPort.obj
 0001:00074330       ??$destroy@V?$IO61X_BufferFifo@UIO61X_LinMessage_T@@@@@?$allocator@U?$_List_node@V?$IO61X_BufferFifo@UIO61X_LinMessage_T@@@@PAX@std@@@std@@QAEXPAV?$IO61X_BufferFifo@UIO61X_LinMessage_T@@@@@Z 10075330 f i IO61X_Library_MSVC120_vc:IO61X_LinPort.obj
 0001:00074350       ??$destroy@V?$IO61X_BufferFifo@UIO61X_LinMessage_T@@@@@?$allocator_traits@V?$allocator@U?$_List_node@V?$IO61X_BufferFifo@UIO61X_LinMessage_T@@@@PAX@std@@@std@@@std@@SAXAAV?$allocator@U?$_List_node@V?$IO61X_BufferFifo@UIO61X_LinMessage_T@@@@PAX@std@@@1@PAV?$IO61X_BufferFifo@UIO61X_LinMessage_T@@@@@Z 10075350 f i IO61X_Library_MSVC120_vc:IO61X_LinPort.obj
 0001:00074370       ??$destroy@V?$_List_unchecked_iterator@V?$_List_val@U?$_List_simple_types@U?$pair@$$CBHV?$IO61X_BufferFifo@UIO61X_LinMessage_T@@@@@std@@@std@@@std@@@std@@@?$_Wrap_alloc@U?$_Wrap_alloc@V?$allocator@V?$_List_unchecked_iterator@V?$_List_val@U?$_List_simple_types@U?$pair@$$CBHV?$IO61X_BufferFifo@UIO61X_LinMessage_T@@@@@std@@@std@@@std@@@std@@@std@@@std@@@std@@QAEXPAV?$_List_unchecked_iterator@V?$_List_val@U?$_List_simple_types@U?$pair@$$CBHV?$IO61X_BufferFifo@UIO61X_LinMessage_T@@@@@std@@@std@@@std@@@1@@Z 10075370 f i IO61X_Library_MSVC120_vc:IO61X_LinPort.obj
 0001:00074380       ??$destroy@V?$_List_unchecked_iterator@V?$_List_val@U?$_List_simple_types@U?$pair@$$CBHV?$IO61X_BufferFifo@UIO61X_LinMessage_T@@@@@std@@@std@@@std@@@std@@@?$_Wrap_alloc@V?$allocator@V?$_List_unchecked_iterator@V?$_List_val@U?$_List_simple_types@U?$pair@$$CBHV?$IO61X_BufferFifo@UIO61X_LinMessage_T@@@@@std@@@std@@@std@@@std@@@std@@@std@@QAEXPAV?$_List_unchecked_iterator@V?$_List_val@U?$_List_simple_types@U?$pair@$$CBHV?$IO61X_BufferFifo@UIO61X_LinMessage_T@@@@@std@@@std@@@std@@@1@@Z 10075380 f i IO61X_Library_MSVC120_vc:IO61X_LinPort.obj
 0001:00074390       ??$destroy@V?$_List_unchecked_iterator@V?$_List_val@U?$_List_simple_types@U?$pair@$$CBHV?$IO61X_BufferFifo@UIO61X_LinMessage_T@@@@@std@@@std@@@std@@@std@@@?$allocator@V?$_List_unchecked_iterator@V?$_List_val@U?$_List_simple_types@U?$pair@$$CBHV?$IO61X_BufferFifo@UIO61X_LinMessage_T@@@@@std@@@std@@@std@@@std@@@std@@QAEXPAV?$_List_unchecked_iterator@V?$_List_val@U?$_List_simple_types@U?$pair@$$CBHV?$IO61X_BufferFifo@UIO61X_LinMessage_T@@@@@std@@@std@@@std@@@1@@Z 10075390 f i IO61X_Library_MSVC120_vc:IO61X_LinPort.obj
 0001:000743a0       ??$destroy@V?$_List_unchecked_iterator@V?$_List_val@U?$_List_simple_types@U?$pair@$$CBHV?$IO61X_BufferFifo@UIO61X_LinMessage_T@@@@@std@@@std@@@std@@@std@@@?$allocator_traits@U?$_Wrap_alloc@V?$allocator@V?$_List_unchecked_iterator@V?$_List_val@U?$_List_simple_types@U?$pair@$$CBHV?$IO61X_BufferFifo@UIO61X_LinMessage_T@@@@@std@@@std@@@std@@@std@@@std@@@std@@@std@@SAXAAU?$_Wrap_alloc@V?$allocator@V?$_List_unchecked_iterator@V?$_List_val@U?$_List_simple_types@U?$pair@$$CBHV?$IO61X_BufferFifo@UIO61X_LinMessage_T@@@@@std@@@std@@@std@@@std@@@std@@@1@PAV?$_List_unchecked_iterator@V?$_List_val@U?$_List_simple_types@U?$pair@$$CBHV?$IO61X_BufferFifo@UIO61X_LinMessage_T@@@@@std@@@std@@@std@@@1@@Z 100753a0 f i IO61X_Library_MSVC120_vc:IO61X_LinPort.obj
 0001:000743b0       ??$destroy@V?$_List_unchecked_iterator@V?$_List_val@U?$_List_simple_types@U?$pair@$$CBHV?$IO61X_BufferFifo@UIO61X_LinMessage_T@@@@@std@@@std@@@std@@@std@@@?$allocator_traits@V?$allocator@V?$_List_unchecked_iterator@V?$_List_val@U?$_List_simple_types@U?$pair@$$CBHV?$IO61X_BufferFifo@UIO61X_LinMessage_T@@@@@std@@@std@@@std@@@std@@@std@@@std@@SAXAAV?$allocator@V?$_List_unchecked_iterator@V?$_List_val@U?$_List_simple_types@U?$pair@$$CBHV?$IO61X_BufferFifo@UIO61X_LinMessage_T@@@@@std@@@std@@@std@@@std@@@1@PAV?$_List_unchecked_iterator@V?$_List_val@U?$_List_simple_types@U?$pair@$$CBHV?$IO61X_BufferFifo@UIO61X_LinMessage_T@@@@@std@@@std@@@std@@@1@@Z 100753b0 f i IO61X_Library_MSVC120_vc:IO61X_LinPort.obj
 0001:000743c0       ??$emplace_front@U?$pair@HV?$IO61X_BufferFifo@UIO61X_LinMessage_T@@@@@std@@@?$list@U?$pair@$$CBHV?$IO61X_BufferFifo@UIO61X_LinMessage_T@@@@@std@@V?$allocator@U?$pair@$$CBHV?$IO61X_BufferFifo@UIO61X_LinMessage_T@@@@@std@@@2@@std@@QAEX$$QAU?$pair@HV?$IO61X_BufferFifo@UIO61X_LinMessage_T@@@@@1@@Z 100753c0 f i IO61X_Library_MSVC120_vc:IO61X_LinPort.obj
 0001:00074410       ??$fill@PAV?$_List_unchecked_iterator@V?$_List_val@U?$_List_simple_types@U?$pair@$$CBHV?$IO61X_BufferFifo@UIO61X_LinMessage_T@@@@@std@@@std@@@std@@@std@@V12@@std@@YAXPAV?$_List_unchecked_iterator@V?$_List_val@U?$_List_simple_types@U?$pair@$$CBHV?$IO61X_BufferFifo@UIO61X_LinMessage_T@@@@@std@@@std@@@std@@@0@0ABV10@@Z 10075410 f i IO61X_Library_MSVC120_vc:IO61X_LinPort.obj
 0001:00074450       ??$forward@AAI@std@@YAAAIAAI@Z 10075450 f i IO61X_Library_MSVC120_vc:IO61X_LinPort.obj
 0001:00074460       ??$forward@AAPAU?$_List_node@U?$pair@$$CBHV?$IO61X_BufferFifo@UIO61X_LinMessage_T@@@@@std@@PAX@std@@@std@@YAAAPAU?$_List_node@U?$pair@$$CBHV?$IO61X_BufferFifo@UIO61X_LinMessage_T@@@@@std@@PAX@0@AAPAU10@@Z 10075460 f i IO61X_Library_MSVC120_vc:IO61X_LinPort.obj
 0001:00074470       ??$forward@AAPAU?$_List_node@V?$IO61X_BufferFifo@UIO61X_LinMessage_T@@@@PAX@std@@@std@@YAAAPAU?$_List_node@V?$IO61X_BufferFifo@UIO61X_LinMessage_T@@@@PAX@0@AAPAU10@@Z 10075470 f i IO61X_Library_MSVC120_vc:IO61X_LinPort.obj
 0001:00074480       ??$forward@AAU?$pair@$$CBHV?$IO61X_BufferFifo@UIO61X_LinMessage_T@@@@@std@@@std@@YAAAU?$pair@$$CBHV?$IO61X_BufferFifo@UIO61X_LinMessage_T@@@@@0@AAU10@@Z 10075480 f i IO61X_Library_MSVC120_vc:IO61X_LinPort.obj
 0001:00074490       ??$forward@ABV?$_List_unchecked_iterator@V?$_List_val@U?$_List_simple_types@U?$pair@$$CBHV?$IO61X_BufferFifo@UIO61X_LinMessage_T@@@@@std@@@std@@@std@@@std@@@std@@YAABV?$_List_unchecked_iterator@V?$_List_val@U?$_List_simple_types@U?$pair@$$CBHV?$IO61X_BufferFifo@UIO61X_LinMessage_T@@@@@std@@@std@@@std@@@0@ABV10@@Z 10075490 f i IO61X_Library_MSVC120_vc:IO61X_LinPort.obj
 0001:000744a0       ??$forward@H@std@@YA$$QAHAAH@Z 100754a0 f i IO61X_Library_MSVC120_vc:IO61X_LinPort.obj
 0001:000744b0       ??$forward@U?$pair@HV?$IO61X_BufferFifo@UIO61X_LinMessage_T@@@@@std@@@std@@YA$$QAU?$pair@HV?$IO61X_BufferFifo@UIO61X_LinMessage_T@@@@@0@AAU10@@Z 100754b0 f i IO61X_Library_MSVC120_vc:IO61X_LinPort.obj
 0001:000744c0       ??$forward@V?$IO61X_BufferFifo@UIO61X_LinMessage_T@@@@@std@@YA$$QAV?$IO61X_BufferFifo@UIO61X_LinMessage_T@@@@AAV1@@Z 100754c0 f i IO61X_Library_MSVC120_vc:IO61X_LinPort.obj
 0001:000744d0       ??$forward@V?$_List_iterator@V?$_List_val@U?$_List_simple_types@U?$pair@$$CBHV?$IO61X_BufferFifo@UIO61X_LinMessage_T@@@@@std@@@std@@@std@@@std@@@std@@YA$$QAV?$_List_iterator@V?$_List_val@U?$_List_simple_types@U?$pair@$$CBHV?$IO61X_BufferFifo@UIO61X_LinMessage_T@@@@@std@@@std@@@std@@@0@AAV10@@Z 100754d0 f i IO61X_Library_MSVC120_vc:IO61X_LinPort.obj
 0001:000744e0       ??$forward@V?$_List_unchecked_iterator@V?$_List_val@U?$_List_simple_types@U?$pair@$$CBHV?$IO61X_BufferFifo@UIO61X_LinMessage_T@@@@@std@@@std@@@std@@@std@@@std@@YA$$QAV?$_List_unchecked_iterator@V?$_List_val@U?$_List_simple_types@U?$pair@$$CBHV?$IO61X_BufferFifo@UIO61X_LinMessage_T@@@@@std@@@std@@@std@@@0@AAV10@@Z 100754e0 f i IO61X_Library_MSVC120_vc:IO61X_LinPort.obj
 0001:000744f0       ??$forward@_N@std@@YA$$QA_NAA_N@Z 100754f0 f i IO61X_Library_MSVC120_vc:IO61X_LinPort.obj
 0001:00074500       ??$insert@U?$pair@HV?$IO61X_BufferFifo@UIO61X_LinMessage_T@@@@@std@@@?$_Hash@V?$_Umap_traits@HV?$IO61X_BufferFifo@UIO61X_LinMessage_T@@@@V?$_Uhash_compare@HU?$hash@H@std@@U?$equal_to@H@2@@std@@V?$allocator@U?$pair@$$CBHV?$IO61X_BufferFifo@UIO61X_LinMessage_T@@@@@std@@@3@$0A@@std@@@std@@QAE?AU?$pair@V?$_List_iterator@V?$_List_val@U?$_List_simple_types@U?$pair@$$CBHV?$IO61X_BufferFifo@UIO61X_LinMessage_T@@@@@std@@@std@@@std@@@std@@_N@1@$$QAU?$pair@HV?$IO61X_BufferFifo@UIO61X_LinMessage_T@@@@@1@@Z 10075500 f i IO61X_Library_MSVC120_vc:IO61X_LinPort.obj
 0001:00074560       ??0?$IO61X_BufferFifo@UIO61X_LinMessage_T@@@@QAE@ABV0@@Z 10075560 f i IO61X_Library_MSVC120_vc:IO61X_LinPort.obj
 0001:000745e0       ??0?$IO61X_BufferFifo@UIO61X_LinMessage_T@@@@QAE@IPAUIO61X_LinMessage_T@@@Z 100755e0 f i IO61X_Library_MSVC120_vc:IO61X_LinPort.obj
 0001:00074650       ??0?$_Hash@V?$_Umap_traits@HV?$IO61X_BufferFifo@UIO61X_LinMessage_T@@@@V?$_Uhash_compare@HU?$hash@H@std@@U?$equal_to@H@2@@std@@V?$allocator@U?$pair@$$CBHV?$IO61X_BufferFifo@UIO61X_LinMessage_T@@@@@std@@@3@$0A@@std@@@std@@QAE@ABV?$_Uhash_compare@HU?$hash@H@std@@U?$equal_to@H@2@@1@ABV?$allocator@U?$pair@$$CBHV?$IO61X_BufferFifo@UIO61X_LinMessage_T@@@@@std@@@1@@Z 10075650 f i IO61X_Library_MSVC120_vc:IO61X_LinPort.obj
 0001:00074700       ??0?$_Hash_oper1@$0A@U?$hash@H@std@@@std@@QAE@U?$hash@H@1@@Z 10075700 f i IO61X_Library_MSVC120_vc:IO61X_LinPort.obj
 0001:00074710       ??0?$_Hash_oper2@$0A@U?$hash@H@std@@U?$equal_to@H@2@@std@@QAE@U?$hash@H@1@U?$equal_to@H@1@@Z 10075710 f i IO61X_Library_MSVC120_vc:IO61X_LinPort.obj
 0001:00074720       ??0?$_List_alloc@$0A@U?$_List_base_types@U?$pair@$$CBHV?$IO61X_BufferFifo@UIO61X_LinMessage_T@@@@@std@@V?$allocator@U?$pair@$$CBHV?$IO61X_BufferFifo@UIO61X_LinMessage_T@@@@@std@@@2@@std@@@std@@QAE@ABV?$allocator@U?$pair@$$CBHV?$IO61X_BufferFifo@UIO61X_LinMessage_T@@@@@std@@@1@@Z 10075720 f i IO61X_Library_MSVC120_vc:IO61X_LinPort.obj
 0001:00074750       ??0?$_List_alloc@$0A@U?$_List_base_types@V?$IO61X_BufferFifo@UIO61X_LinMessage_T@@@@V?$allocator@V?$IO61X_BufferFifo@UIO61X_LinMessage_T@@@@@std@@@std@@@std@@QAE@ABV?$allocator@V?$IO61X_BufferFifo@UIO61X_LinMessage_T@@@@@1@@Z 10075750 f i IO61X_Library_MSVC120_vc:IO61X_LinPort.obj
 0001:00074780       ??0?$_List_buy@U?$pair@$$CBHV?$IO61X_BufferFifo@UIO61X_LinMessage_T@@@@@std@@V?$allocator@U?$pair@$$CBHV?$IO61X_BufferFifo@UIO61X_LinMessage_T@@@@@std@@@2@@std@@QAE@ABV?$allocator@U?$pair@$$CBHV?$IO61X_BufferFifo@UIO61X_LinMessage_T@@@@@std@@@1@@Z 10075780 f i IO61X_Library_MSVC120_vc:IO61X_LinPort.obj
 0001:000747b0       ??0?$_List_buy@V?$IO61X_BufferFifo@UIO61X_LinMessage_T@@@@V?$allocator@V?$IO61X_BufferFifo@UIO61X_LinMessage_T@@@@@std@@@std@@QAE@ABV?$allocator@V?$IO61X_BufferFifo@UIO61X_LinMessage_T@@@@@1@@Z 100757b0 f i IO61X_Library_MSVC120_vc:IO61X_LinPort.obj
 0001:000747e0       ??0?$_List_const_iterator@V?$_List_val@U?$_List_simple_types@U?$pair@$$CBHV?$IO61X_BufferFifo@UIO61X_LinMessage_T@@@@@std@@@std@@@std@@@std@@QAE@PAU?$_List_node@U?$pair@$$CBHV?$IO61X_BufferFifo@UIO61X_LinMessage_T@@@@@std@@PAX@1@PBV?$_List_val@U?$_List_simple_types@U?$pair@$$CBHV?$IO61X_BufferFifo@UIO61X_LinMessage_T@@@@@std@@@std@@@1@@Z 100757e0 f i IO61X_Library_MSVC120_vc:IO61X_LinPort.obj
 0001:000747f0       ??0?$_List_const_iterator@V?$_List_val@U?$_List_simple_types@U?$pair@$$CBHV?$IO61X_BufferFifo@UIO61X_LinMessage_T@@@@@std@@@std@@@std@@@std@@QAE@XZ 100757f0 f i IO61X_Library_MSVC120_vc:IO61X_LinPort.obj
 0001:00074800       ??0?$_List_const_iterator@V?$_List_val@U?$_List_simple_types@V?$IO61X_BufferFifo@UIO61X_LinMessage_T@@@@@std@@@std@@@std@@QAE@PAU?$_List_node@V?$IO61X_BufferFifo@UIO61X_LinMessage_T@@@@PAX@1@PBV?$_List_val@U?$_List_simple_types@V?$IO61X_BufferFifo@UIO61X_LinMessage_T@@@@@std@@@1@@Z 10075800 f i IO61X_Library_MSVC120_vc:IO61X_LinPort.obj
 0001:00074810       ??0?$_List_iterator@V?$_List_val@U?$_List_simple_types@U?$pair@$$CBHV?$IO61X_BufferFifo@UIO61X_LinMessage_T@@@@@std@@@std@@@std@@@std@@QAE@PAU?$_List_node@U?$pair@$$CBHV?$IO61X_BufferFifo@UIO61X_LinMessage_T@@@@@std@@PAX@1@PBV?$_List_val@U?$_List_simple_types@U?$pair@$$CBHV?$IO61X_BufferFifo@UIO61X_LinMessage_T@@@@@std@@@std@@@1@@Z 10075810 f i IO61X_Library_MSVC120_vc:IO61X_LinPort.obj
 0001:00074820       ??0?$_List_iterator@V?$_List_val@U?$_List_simple_types@U?$pair@$$CBHV?$IO61X_BufferFifo@UIO61X_LinMessage_T@@@@@std@@@std@@@std@@@std@@QAE@XZ 10075820 f i IO61X_Library_MSVC120_vc:IO61X_LinPort.obj
 0001:00074830       ??0?$_List_iterator@V?$_List_val@U?$_List_simple_types@V?$IO61X_BufferFifo@UIO61X_LinMessage_T@@@@@std@@@std@@@std@@QAE@PAU?$_List_node@V?$IO61X_BufferFifo@UIO61X_LinMessage_T@@@@PAX@1@PBV?$_List_val@U?$_List_simple_types@V?$IO61X_BufferFifo@UIO61X_LinMessage_T@@@@@std@@@1@@Z 10075830 f i IO61X_Library_MSVC120_vc:IO61X_LinPort.obj
 0001:00074840       ??0?$_List_unchecked_const_iterator@V?$_List_val@U?$_List_simple_types@U?$pair@$$CBHV?$IO61X_BufferFifo@UIO61X_LinMessage_T@@@@@std@@@std@@@std@@U_Iterator_base0@2@@std@@QAE@PAU?$_List_node@U?$pair@$$CBHV?$IO61X_BufferFifo@UIO61X_LinMessage_T@@@@@std@@PAX@1@PBV?$_List_val@U?$_List_simple_types@U?$pair@$$CBHV?$IO61X_BufferFifo@UIO61X_LinMessage_T@@@@@std@@@std@@@1@@Z 10075840 f i IO61X_Library_MSVC120_vc:IO61X_LinPort.obj
 0001:00074850       ??0?$_List_unchecked_const_iterator@V?$_List_val@U?$_List_simple_types@U?$pair@$$CBHV?$IO61X_BufferFifo@UIO61X_LinMessage_T@@@@@std@@@std@@@std@@U_Iterator_base0@2@@std@@QAE@XZ 10075850 f i IO61X_Library_MSVC120_vc:IO61X_LinPort.obj
 0001:00074860       ??0?$_List_unchecked_const_iterator@V?$_List_val@U?$_List_simple_types@V?$IO61X_BufferFifo@UIO61X_LinMessage_T@@@@@std@@@std@@U_Iterator_base0@2@@std@@QAE@PAU?$_List_node@V?$IO61X_BufferFifo@UIO61X_LinMessage_T@@@@PAX@1@PBV?$_List_val@U?$_List_simple_types@V?$IO61X_BufferFifo@UIO61X_LinMessage_T@@@@@std@@@1@@Z 10075860 f i IO61X_Library_MSVC120_vc:IO61X_LinPort.obj
 0001:00074870       ??0?$_List_unchecked_iterator@V?$_List_val@U?$_List_simple_types@U?$pair@$$CBHV?$IO61X_BufferFifo@UIO61X_LinMessage_T@@@@@std@@@std@@@std@@@std@@QAE@PAU?$_List_node@U?$pair@$$CBHV?$IO61X_BufferFifo@UIO61X_LinMessage_T@@@@@std@@PAX@1@PBV?$_List_val@U?$_List_simple_types@U?$pair@$$CBHV?$IO61X_BufferFifo@UIO61X_LinMessage_T@@@@@std@@@std@@@1@@Z 10075870 f i IO61X_Library_MSVC120_vc:IO61X_LinPort.obj
 0001:00074880       ??0?$_List_unchecked_iterator@V?$_List_val@U?$_List_simple_types@U?$pair@$$CBHV?$IO61X_BufferFifo@UIO61X_LinMessage_T@@@@@std@@@std@@@std@@@std@@QAE@XZ 10075880 f i IO61X_Library_MSVC120_vc:IO61X_LinPort.obj
 0001:00074890       ??0?$_List_unchecked_iterator@V?$_List_val@U?$_List_simple_types@V?$IO61X_BufferFifo@UIO61X_LinMessage_T@@@@@std@@@std@@@std@@QAE@PAU?$_List_node@V?$IO61X_BufferFifo@UIO61X_LinMessage_T@@@@PAX@1@PBV?$_List_val@U?$_List_simple_types@V?$IO61X_BufferFifo@UIO61X_LinMessage_T@@@@@std@@@1@@Z 10075890 f i IO61X_Library_MSVC120_vc:IO61X_LinPort.obj
 0001:000748a0       ??0?$_List_val@U?$_List_simple_types@U?$pair@$$CBHV?$IO61X_BufferFifo@UIO61X_LinMessage_T@@@@@std@@@std@@@std@@QAE@XZ 100758a0 f i IO61X_Library_MSVC120_vc:IO61X_LinPort.obj
 0001:000748b0       ??0?$_List_val@U?$_List_simple_types@V?$IO61X_BufferFifo@UIO61X_LinMessage_T@@@@@std@@@std@@QAE@XZ 100758b0 f i IO61X_Library_MSVC120_vc:IO61X_LinPort.obj
 0001:000748c0       ??0?$_Uhash_compare@HU?$hash@H@std@@U?$equal_to@H@2@@std@@QAE@U?$hash@H@1@U?$equal_to@H@1@@Z 100758c0 f i IO61X_Library_MSVC120_vc:IO61X_LinPort.obj
 0001:000748d0       ??0?$_Umap_traits@HV?$IO61X_BufferFifo@UIO61X_LinMessage_T@@@@V?$_Uhash_compare@HU?$hash@H@std@@U?$equal_to@H@2@@std@@V?$allocator@U?$pair@$$CBHV?$IO61X_BufferFifo@UIO61X_LinMessage_T@@@@@std@@@3@$0A@@std@@QAE@ABV?$_Uhash_compare@HU?$hash@H@std@@U?$equal_to@H@2@@1@@Z 100758d0 f i IO61X_Library_MSVC120_vc:IO61X_LinPort.obj
 0001:000748e0       ??0?$_Vector_alloc@$0A@U?$_Vec_base_types@V?$_List_unchecked_iterator@V?$_List_val@U?$_List_simple_types@U?$pair@$$CBHV?$IO61X_BufferFifo@UIO61X_LinMessage_T@@@@@std@@@std@@@std@@@std@@U?$_Wrap_alloc@V?$allocator@V?$_List_unchecked_iterator@V?$_List_val@U?$_List_simple_types@U?$pair@$$CBHV?$IO61X_BufferFifo@UIO61X_LinMessage_T@@@@@std@@@std@@@std@@@std@@@std@@@2@@std@@@std@@QAE@ABU?$_Wrap_alloc@V?$allocator@V?$_List_unchecked_iterator@V?$_List_val@U?$_List_simple_types@U?$pair@$$CBHV?$IO61X_BufferFifo@UIO61X_LinMessage_T@@@@@std@@@std@@@std@@@std@@@std@@@1@@Z 100758e0 f i IO61X_Library_MSVC120_vc:IO61X_LinPort.obj
 0001:00074900       ??0?$_Vector_const_iterator@V?$_Vector_val@U?$_Simple_types@V?$_List_unchecked_iterator@V?$_List_val@U?$_List_simple_types@U?$pair@$$CBHV?$IO61X_BufferFifo@UIO61X_LinMessage_T@@@@@std@@@std@@@std@@@std@@@std@@@std@@@std@@QAE@PAV?$_List_unchecked_iterator@V?$_List_val@U?$_List_simple_types@U?$pair@$$CBHV?$IO61X_BufferFifo@UIO61X_LinMessage_T@@@@@std@@@std@@@std@@@1@PBU_Container_base0@1@@Z 10075900 f i IO61X_Library_MSVC120_vc:IO61X_LinPort.obj
 0001:00074910       ??0?$_Vector_iterator@V?$_Vector_val@U?$_Simple_types@V?$_List_unchecked_iterator@V?$_List_val@U?$_List_simple_types@U?$pair@$$CBHV?$IO61X_BufferFifo@UIO61X_LinMessage_T@@@@@std@@@std@@@std@@@std@@@std@@@std@@@std@@QAE@PAV?$_List_unchecked_iterator@V?$_List_val@U?$_List_simple_types@U?$pair@$$CBHV?$IO61X_BufferFifo@UIO61X_LinMessage_T@@@@@std@@@std@@@std@@@1@PBU_Container_base0@1@@Z 10075910 f i IO61X_Library_MSVC120_vc:IO61X_LinPort.obj
 0001:00074920       ??0?$_Vector_val@U?$_Simple_types@V?$_List_unchecked_iterator@V?$_List_val@U?$_List_simple_types@U?$pair@$$CBHV?$IO61X_BufferFifo@UIO61X_LinMessage_T@@@@@std@@@std@@@std@@@std@@@std@@@std@@QAE@XZ 10075920 f i IO61X_Library_MSVC120_vc:IO61X_LinPort.obj
 0001:00074940       ??0?$_Wrap_alloc@U?$_Wrap_alloc@V?$allocator@V?$_List_unchecked_iterator@V?$_List_val@U?$_List_simple_types@U?$pair@$$CBHV?$IO61X_BufferFifo@UIO61X_LinMessage_T@@@@@std@@@std@@@std@@@std@@@std@@@std@@@std@@QAE@XZ 10075940 f i IO61X_Library_MSVC120_vc:IO61X_LinPort.obj
 0001:00074950       ??0?$_Wrap_alloc@V?$allocator@U?$_List_node@U?$pair@$$CBHV?$IO61X_BufferFifo@UIO61X_LinMessage_T@@@@@std@@PAX@std@@@std@@@std@@QAE@XZ 10075950 f i IO61X_Library_MSVC120_vc:IO61X_LinPort.obj
 0001:00074960       ??0?$_Wrap_alloc@V?$allocator@U?$_List_node@V?$IO61X_BufferFifo@UIO61X_LinMessage_T@@@@PAX@std@@@std@@@std@@QAE@XZ 10075960 f i IO61X_Library_MSVC120_vc:IO61X_LinPort.obj
 0001:00074970       ??0?$_Wrap_alloc@V?$allocator@V?$_List_unchecked_iterator@V?$_List_val@U?$_List_simple_types@U?$pair@$$CBHV?$IO61X_BufferFifo@UIO61X_LinMessage_T@@@@@std@@@std@@@std@@@std@@@std@@@std@@QAE@XZ 10075970 f i IO61X_Library_MSVC120_vc:IO61X_LinPort.obj
 0001:00074980       ??0?$allocator@U?$_List_node@U?$pair@$$CBHV?$IO61X_BufferFifo@UIO61X_LinMessage_T@@@@@std@@PAX@std@@@std@@QAE@XZ 10075980 f i IO61X_Library_MSVC120_vc:IO61X_LinPort.obj
 0001:00074990       ??0?$allocator@U?$_List_node@V?$IO61X_BufferFifo@UIO61X_LinMessage_T@@@@PAX@std@@@std@@QAE@XZ 10075990 f i IO61X_Library_MSVC120_vc:IO61X_LinPort.obj
 0001:000749a0       ??0?$allocator@U?$pair@$$CBHV?$IO61X_BufferFifo@UIO61X_LinMessage_T@@@@@std@@@std@@QAE@XZ 100759a0 f i IO61X_Library_MSVC120_vc:IO61X_LinPort.obj
 0001:000749b0       ??0?$allocator@V?$IO61X_BufferFifo@UIO61X_LinMessage_T@@@@@std@@QAE@XZ 100759b0 f i IO61X_Library_MSVC120_vc:IO61X_LinPort.obj
 0001:000749c0       ??0?$allocator@V?$_List_unchecked_iterator@V?$_List_val@U?$_List_simple_types@U?$pair@$$CBHV?$IO61X_BufferFifo@UIO61X_LinMessage_T@@@@@std@@@std@@@std@@@std@@@std@@QAE@XZ 100759c0 f i IO61X_Library_MSVC120_vc:IO61X_LinPort.obj
 0001:000749d0       ??0?$list@U?$pair@$$CBHV?$IO61X_BufferFifo@UIO61X_LinMessage_T@@@@@std@@V?$allocator@U?$pair@$$CBHV?$IO61X_BufferFifo@UIO61X_LinMessage_T@@@@@std@@@2@@std@@QAE@ABV?$allocator@U?$pair@$$CBHV?$IO61X_BufferFifo@UIO61X_LinMessage_T@@@@@std@@@1@@Z 100759d0 f i IO61X_Library_MSVC120_vc:IO61X_LinPort.obj
 0001:00074a00       ??0?$list@V?$IO61X_BufferFifo@UIO61X_LinMessage_T@@@@V?$allocator@V?$IO61X_BufferFifo@UIO61X_LinMessage_T@@@@@std@@@std@@QAE@XZ 10075a00 f i IO61X_Library_MSVC120_vc:IO61X_LinPort.obj
 0001:00074a20       ??0?$pair@V?$_List_iterator@V?$_List_val@U?$_List_simple_types@U?$pair@$$CBHV?$IO61X_BufferFifo@UIO61X_LinMessage_T@@@@@std@@@std@@@std@@@std@@_N@std@@QAE@XZ 10075a20 f i IO61X_Library_MSVC120_vc:IO61X_LinPort.obj
 0001:00074a30       ??0?$unordered_map@HV?$IO61X_BufferFifo@UIO61X_LinMessage_T@@@@U?$hash@H@std@@U?$equal_to@H@3@V?$allocator@U?$pair@$$CBHV?$IO61X_BufferFifo@UIO61X_LinMessage_T@@@@@std@@@3@@std@@QAE@XZ 10075a30 f i IO61X_Library_MSVC120_vc:IO61X_LinPort.obj
 0001:00074a50       ??0?$vector@V?$_List_unchecked_iterator@V?$_List_val@U?$_List_simple_types@U?$pair@$$CBHV?$IO61X_BufferFifo@UIO61X_LinMessage_T@@@@@std@@@std@@@std@@@std@@U?$_Wrap_alloc@V?$allocator@V?$_List_unchecked_iterator@V?$_List_val@U?$_List_simple_types@U?$pair@$$CBHV?$IO61X_BufferFifo@UIO61X_LinMessage_T@@@@@std@@@std@@@std@@@std@@@std@@@2@@std@@QAE@ABU?$_Wrap_alloc@V?$allocator@V?$_List_unchecked_iterator@V?$_List_val@U?$_List_simple_types@U?$pair@$$CBHV?$IO61X_BufferFifo@UIO61X_LinMessage_T@@@@@std@@@std@@@std@@@std@@@std@@@1@@Z 10075a50 f i IO61X_Library_MSVC120_vc:IO61X_LinPort.obj
 0001:00074a70       ??0IO61X_LinPort@@QAE@II_N@Z 10075a70 f   IO61X_Library_MSVC120_vc:IO61X_LinPort.obj
 0001:00074b60       ??1?$IO61X_BufferFifo@UIO61X_LinMessage_T@@@@QAE@XZ 10075b60 f i IO61X_Library_MSVC120_vc:IO61X_LinPort.obj
 0001:00074b70       ??1?$_Hash@V?$_Umap_traits@HV?$IO61X_BufferFifo@UIO61X_LinMessage_T@@@@V?$_Uhash_compare@HU?$hash@H@std@@U?$equal_to@H@2@@std@@V?$allocator@U?$pair@$$CBHV?$IO61X_BufferFifo@UIO61X_LinMessage_T@@@@@std@@@3@$0A@@std@@@std@@QAE@XZ 10075b70 f i IO61X_Library_MSVC120_vc:IO61X_LinPort.obj
 0001:00074bb0       ??1?$_List_alloc@$0A@U?$_List_base_types@U?$pair@$$CBHV?$IO61X_BufferFifo@UIO61X_LinMessage_T@@@@@std@@V?$allocator@U?$pair@$$CBHV?$IO61X_BufferFifo@UIO61X_LinMessage_T@@@@@std@@@2@@std@@@std@@QAE@XZ 10075bb0 f i IO61X_Library_MSVC120_vc:IO61X_LinPort.obj
 0001:00074bc0       ??1?$_List_alloc@$0A@U?$_List_base_types@V?$IO61X_BufferFifo@UIO61X_LinMessage_T@@@@V?$allocator@V?$IO61X_BufferFifo@UIO61X_LinMessage_T@@@@@std@@@std@@@std@@QAE@XZ 10075bc0 f i IO61X_Library_MSVC120_vc:IO61X_LinPort.obj
 0001:00074bd0       ??1?$_List_buy@U?$pair@$$CBHV?$IO61X_BufferFifo@UIO61X_LinMessage_T@@@@@std@@V?$allocator@U?$pair@$$CBHV?$IO61X_BufferFifo@UIO61X_LinMessage_T@@@@@std@@@2@@std@@QAE@XZ 10075bd0 f i IO61X_Library_MSVC120_vc:IO61X_LinPort.obj
 0001:00074be0       ??1?$_List_buy@V?$IO61X_BufferFifo@UIO61X_LinMessage_T@@@@V?$allocator@V?$IO61X_BufferFifo@UIO61X_LinMessage_T@@@@@std@@@std@@QAE@XZ 10075be0 f i IO61X_Library_MSVC120_vc:IO61X_LinPort.obj
 0001:00074bf0       ??1?$list@U?$pair@$$CBHV?$IO61X_BufferFifo@UIO61X_LinMessage_T@@@@@std@@V?$allocator@U?$pair@$$CBHV?$IO61X_BufferFifo@UIO61X_LinMessage_T@@@@@std@@@2@@std@@QAE@XZ 10075bf0 f i IO61X_Library_MSVC120_vc:IO61X_LinPort.obj
 0001:00074c10       ??1?$list@V?$IO61X_BufferFifo@UIO61X_LinMessage_T@@@@V?$allocator@V?$IO61X_BufferFifo@UIO61X_LinMessage_T@@@@@std@@@std@@QAE@XZ 10075c10 f i IO61X_Library_MSVC120_vc:IO61X_LinPort.obj
 0001:00074c30       ??1?$pair@$$CBHV?$IO61X_BufferFifo@UIO61X_LinMessage_T@@@@@std@@QAE@XZ 10075c30 f i IO61X_Library_MSVC120_vc:IO61X_LinPort.obj
 0001:00074c40       ??1?$pair@HV?$IO61X_BufferFifo@UIO61X_LinMessage_T@@@@@std@@QAE@XZ 10075c40 f i IO61X_Library_MSVC120_vc:IO61X_LinPort.obj
 0001:00074c50       ??1?$unordered_map@HV?$IO61X_BufferFifo@UIO61X_LinMessage_T@@@@U?$hash@H@std@@U?$equal_to@H@3@V?$allocator@U?$pair@$$CBHV?$IO61X_BufferFifo@UIO61X_LinMessage_T@@@@@std@@@3@@std@@QAE@XZ 10075c50 f i IO61X_Library_MSVC120_vc:IO61X_LinPort.obj
 0001:00074c90       ??1?$vector@V?$_List_unchecked_iterator@V?$_List_val@U?$_List_simple_types@U?$pair@$$CBHV?$IO61X_BufferFifo@UIO61X_LinMessage_T@@@@@std@@@std@@@std@@@std@@U?$_Wrap_alloc@V?$allocator@V?$_List_unchecked_iterator@V?$_List_val@U?$_List_simple_types@U?$pair@$$CBHV?$IO61X_BufferFifo@UIO61X_LinMessage_T@@@@@std@@@std@@@std@@@std@@@std@@@2@@std@@QAE@XZ 10075c90 f i IO61X_Library_MSVC120_vc:IO61X_LinPort.obj
 0001:00074cc0       ??1IO61X_LinPort@@UAE@XZ   10075cc0 f   IO61X_Library_MSVC120_vc:IO61X_LinPort.obj
 0001:00074d20       ??4?$pair@V?$_List_iterator@V?$_List_val@U?$_List_simple_types@U?$pair@$$CBHV?$IO61X_BufferFifo@UIO61X_LinMessage_T@@@@@std@@@std@@@std@@@std@@_N@std@@QAEAAU01@$$QAU01@@Z 10075d20 f i IO61X_Library_MSVC120_vc:IO61X_LinPort.obj
 0001:00074d40       ??8?$_List_const_iterator@V?$_List_val@U?$_List_simple_types@U?$pair@$$CBHV?$IO61X_BufferFifo@UIO61X_LinMessage_T@@@@@std@@@std@@@std@@@std@@QBE_NABV01@@Z 10075d40 f i IO61X_Library_MSVC120_vc:IO61X_LinPort.obj
 0001:00074d60       ??8?$_List_const_iterator@V?$_List_val@U?$_List_simple_types@V?$IO61X_BufferFifo@UIO61X_LinMessage_T@@@@@std@@@std@@@std@@QBE_NABV01@@Z 10075d60 f i IO61X_Library_MSVC120_vc:IO61X_LinPort.obj
 0001:00074d80       ??8?$_List_unchecked_const_iterator@V?$_List_val@U?$_List_simple_types@U?$pair@$$CBHV?$IO61X_BufferFifo@UIO61X_LinMessage_T@@@@@std@@@std@@@std@@U_Iterator_base0@2@@std@@QBE_NABV01@@Z 10075d80 f i IO61X_Library_MSVC120_vc:IO61X_LinPort.obj
 0001:00074da0       ??9?$_List_const_iterator@V?$_List_val@U?$_List_simple_types@U?$pair@$$CBHV?$IO61X_BufferFifo@UIO61X_LinMessage_T@@@@@std@@@std@@@std@@@std@@QBE_NABV01@@Z 10075da0 f i IO61X_Library_MSVC120_vc:IO61X_LinPort.obj
 0001:00074dc0       ??9?$_List_const_iterator@V?$_List_val@U?$_List_simple_types@V?$IO61X_BufferFifo@UIO61X_LinMessage_T@@@@@std@@@std@@@std@@QBE_NABV01@@Z 10075dc0 f i IO61X_Library_MSVC120_vc:IO61X_LinPort.obj
 0001:00074de0       ??9?$_List_unchecked_const_iterator@V?$_List_val@U?$_List_simple_types@U?$pair@$$CBHV?$IO61X_BufferFifo@UIO61X_LinMessage_T@@@@@std@@@std@@@std@@U_Iterator_base0@2@@std@@QBE_NABV01@@Z 10075de0 f i IO61X_Library_MSVC120_vc:IO61X_LinPort.obj
 0001:00074e00       ??A?$vector@V?$_List_unchecked_iterator@V?$_List_val@U?$_List_simple_types@U?$pair@$$CBHV?$IO61X_BufferFifo@UIO61X_LinMessage_T@@@@@std@@@std@@@std@@@std@@U?$_Wrap_alloc@V?$allocator@V?$_List_unchecked_iterator@V?$_List_val@U?$_List_simple_types@U?$pair@$$CBHV?$IO61X_BufferFifo@UIO61X_LinMessage_T@@@@@std@@@std@@@std@@@std@@@std@@@2@@std@@QAEAAV?$_List_unchecked_iterator@V?$_List_val@U?$_List_simple_types@U?$pair@$$CBHV?$IO61X_BufferFifo@UIO61X_LinMessage_T@@@@@std@@@std@@@std@@@1@I@Z 10075e00 f i IO61X_Library_MSVC120_vc:IO61X_LinPort.obj
 0001:00074e10       ??C?$_List_iterator@V?$_List_val@U?$_List_simple_types@U?$pair@$$CBHV?$IO61X_BufferFifo@UIO61X_LinMessage_T@@@@@std@@@std@@@std@@@std@@QBEPAU?$pair@$$CBHV?$IO61X_BufferFifo@UIO61X_LinMessage_T@@@@@1@XZ 10075e10 f i IO61X_Library_MSVC120_vc:IO61X_LinPort.obj
 0001:00074e20       ??D?$_List_const_iterator@V?$_List_val@U?$_List_simple_types@U?$pair@$$CBHV?$IO61X_BufferFifo@UIO61X_LinMessage_T@@@@@std@@@std@@@std@@@std@@QBEABU?$pair@$$CBHV?$IO61X_BufferFifo@UIO61X_LinMessage_T@@@@@1@XZ 10075e20 f i IO61X_Library_MSVC120_vc:IO61X_LinPort.obj
 0001:00074e30       ??D?$_List_const_iterator@V?$_List_val@U?$_List_simple_types@V?$IO61X_BufferFifo@UIO61X_LinMessage_T@@@@@std@@@std@@@std@@QBEABV?$IO61X_BufferFifo@UIO61X_LinMessage_T@@@@XZ 10075e30 f i IO61X_Library_MSVC120_vc:IO61X_LinPort.obj
 0001:00074e40       ??D?$_List_iterator@V?$_List_val@U?$_List_simple_types@U?$pair@$$CBHV?$IO61X_BufferFifo@UIO61X_LinMessage_T@@@@@std@@@std@@@std@@@std@@QBEAAU?$pair@$$CBHV?$IO61X_BufferFifo@UIO61X_LinMessage_T@@@@@1@XZ 10075e40 f i IO61X_Library_MSVC120_vc:IO61X_LinPort.obj
 0001:00074e50       ??D?$_List_iterator@V?$_List_val@U?$_List_simple_types@V?$IO61X_BufferFifo@UIO61X_LinMessage_T@@@@@std@@@std@@@std@@QBEAAV?$IO61X_BufferFifo@UIO61X_LinMessage_T@@@@XZ 10075e50 f i IO61X_Library_MSVC120_vc:IO61X_LinPort.obj
 0001:00074e60       ??D?$_List_unchecked_const_iterator@V?$_List_val@U?$_List_simple_types@U?$pair@$$CBHV?$IO61X_BufferFifo@UIO61X_LinMessage_T@@@@@std@@@std@@@std@@U_Iterator_base0@2@@std@@QBEABU?$pair@$$CBHV?$IO61X_BufferFifo@UIO61X_LinMessage_T@@@@@1@XZ 10075e60 f i IO61X_Library_MSVC120_vc:IO61X_LinPort.obj
 0001:00074e70       ??D?$_List_unchecked_iterator@V?$_List_val@U?$_List_simple_types@U?$pair@$$CBHV?$IO61X_BufferFifo@UIO61X_LinMessage_T@@@@@std@@@std@@@std@@@std@@QBEAAU?$pair@$$CBHV?$IO61X_BufferFifo@UIO61X_LinMessage_T@@@@@1@XZ 10075e70 f i IO61X_Library_MSVC120_vc:IO61X_LinPort.obj
 0001:00074e80       ??E?$_List_const_iterator@V?$_List_val@U?$_List_simple_types@U?$pair@$$CBHV?$IO61X_BufferFifo@UIO61X_LinMessage_T@@@@@std@@@std@@@std@@@std@@QAE?AV01@H@Z 10075e80 f i IO61X_Library_MSVC120_vc:IO61X_LinPort.obj
 0001:00074ea0       ??E?$_List_const_iterator@V?$_List_val@U?$_List_simple_types@U?$pair@$$CBHV?$IO61X_BufferFifo@UIO61X_LinMessage_T@@@@@std@@@std@@@std@@@std@@QAEAAV01@XZ 10075ea0 f i IO61X_Library_MSVC120_vc:IO61X_LinPort.obj
 0001:00074eb0       ??E?$_List_const_iterator@V?$_List_val@U?$_List_simple_types@V?$IO61X_BufferFifo@UIO61X_LinMessage_T@@@@@std@@@std@@@std@@QAEAAV01@XZ 10075eb0 f i IO61X_Library_MSVC120_vc:IO61X_LinPort.obj
 0001:00074ec0       ??E?$_List_iterator@V?$_List_val@U?$_List_simple_types@V?$IO61X_BufferFifo@UIO61X_LinMessage_T@@@@@std@@@std@@@std@@QAE?AV01@H@Z 10075ec0 f i IO61X_Library_MSVC120_vc:IO61X_LinPort.obj
 0001:00074ee0       ??E?$_List_iterator@V?$_List_val@U?$_List_simple_types@V?$IO61X_BufferFifo@UIO61X_LinMessage_T@@@@@std@@@std@@@std@@QAEAAV01@XZ 10075ee0 f i IO61X_Library_MSVC120_vc:IO61X_LinPort.obj
 0001:00074ef0       ??E?$_List_unchecked_const_iterator@V?$_List_val@U?$_List_simple_types@U?$pair@$$CBHV?$IO61X_BufferFifo@UIO61X_LinMessage_T@@@@@std@@@std@@@std@@U_Iterator_base0@2@@std@@QAEAAV01@XZ 10075ef0 f i IO61X_Library_MSVC120_vc:IO61X_LinPort.obj
 0001:00074f00       ??E?$_List_unchecked_iterator@V?$_List_val@U?$_List_simple_types@U?$pair@$$CBHV?$IO61X_BufferFifo@UIO61X_LinMessage_T@@@@@std@@@std@@@std@@@std@@QAEAAV01@XZ 10075f00 f i IO61X_Library_MSVC120_vc:IO61X_LinPort.obj
 0001:00074f10       ??F?$_List_const_iterator@V?$_List_val@U?$_List_simple_types@V?$IO61X_BufferFifo@UIO61X_LinMessage_T@@@@@std@@@std@@@std@@QAEAAV01@XZ 10075f10 f i IO61X_Library_MSVC120_vc:IO61X_LinPort.obj
 0001:00074f20       ??F?$_List_iterator@V?$_List_val@U?$_List_simple_types@V?$IO61X_BufferFifo@UIO61X_LinMessage_T@@@@@std@@@std@@@std@@QAEAAV01@XZ 10075f20 f i IO61X_Library_MSVC120_vc:IO61X_LinPort.obj
 0001:00074f30       ??F?$_List_unchecked_const_iterator@V?$_List_val@U?$_List_simple_types@U?$pair@$$CBHV?$IO61X_BufferFifo@UIO61X_LinMessage_T@@@@@std@@@std@@@std@@U_Iterator_base0@2@@std@@QAEAAV01@XZ 10075f30 f i IO61X_Library_MSVC120_vc:IO61X_LinPort.obj
 0001:00074f40       ??F?$_List_unchecked_iterator@V?$_List_val@U?$_List_simple_types@U?$pair@$$CBHV?$IO61X_BufferFifo@UIO61X_LinMessage_T@@@@@std@@@std@@@std@@@std@@QAEAAV01@XZ 10075f40 f i IO61X_Library_MSVC120_vc:IO61X_LinPort.obj
 0001:00074f50       ??H?$_Vector_iterator@V?$_Vector_val@U?$_Simple_types@V?$_List_unchecked_iterator@V?$_List_val@U?$_List_simple_types@U?$pair@$$CBHV?$IO61X_BufferFifo@UIO61X_LinMessage_T@@@@@std@@@std@@@std@@@std@@@std@@@std@@@std@@QBE?AV01@H@Z 10075f50 f i IO61X_Library_MSVC120_vc:IO61X_LinPort.obj
 0001:00074f70       ??R?$_Bitwise_hash@H@std@@QBEIABH@Z 10075f70 f i IO61X_Library_MSVC120_vc:IO61X_LinPort.obj
 0001:00074fb0       ??R?$_Uhash_compare@HU?$hash@H@std@@U?$equal_to@H@2@@std@@QBEIABH@Z 10075fb0 f i IO61X_Library_MSVC120_vc:IO61X_LinPort.obj
 0001:00074ff0       ??R?$_Uhash_compare@HU?$hash@H@std@@U?$equal_to@H@2@@std@@QBE_NABH0@Z 10075ff0 f i IO61X_Library_MSVC120_vc:IO61X_LinPort.obj
 0001:00075010       ??R?$equal_to@H@std@@QBE_NABH0@Z 10076010 f i IO61X_Library_MSVC120_vc:IO61X_LinPort.obj
 0001:00075030       ??Y?$_Vector_const_iterator@V?$_Vector_val@U?$_Simple_types@V?$_List_unchecked_iterator@V?$_List_val@U?$_List_simple_types@U?$pair@$$CBHV?$IO61X_BufferFifo@UIO61X_LinMessage_T@@@@@std@@@std@@@std@@@std@@@std@@@std@@@std@@QAEAAV01@H@Z 10076030 f i IO61X_Library_MSVC120_vc:IO61X_LinPort.obj
 0001:00075050       ??Y?$_Vector_iterator@V?$_Vector_val@U?$_Simple_types@V?$_List_unchecked_iterator@V?$_List_val@U?$_List_simple_types@U?$pair@$$CBHV?$IO61X_BufferFifo@UIO61X_LinMessage_T@@@@@std@@@std@@@std@@@std@@@std@@@std@@@std@@QAEAAV01@H@Z 10076050 f i IO61X_Library_MSVC120_vc:IO61X_LinPort.obj
 0001:00075070       ??_G?$IO61X_BufferFifo@UIO61X_LinMessage_T@@@@QAEPAXI@Z 10076070 f i IO61X_Library_MSVC120_vc:IO61X_LinPort.obj
 0001:000750a0       ??_G?$pair@$$CBHV?$IO61X_BufferFifo@UIO61X_LinMessage_T@@@@@std@@QAEPAXI@Z 100760a0 f i IO61X_Library_MSVC120_vc:IO61X_LinPort.obj
 0001:000750d0       ??_EIO61X_LinPort@@UAEPAXI@Z 100760d0 f i IO61X_Library_MSVC120_vc:IO61X_LinPort.obj
 0001:000750d0       ??_GIO61X_LinPort@@UAEPAXI@Z 100760d0 f i IO61X_Library_MSVC120_vc:IO61X_LinPort.obj
 0001:00075100       ?AddMessageToBuffer@?$IO61X_BufferFifo@UIO61X_LinMessage_T@@@@QAE_NPBUIO61X_LinMessage_T@@@Z 10076100 f i IO61X_Library_MSVC120_vc:IO61X_LinPort.obj
 0001:00075140       ?AllocateBuffer_spin@IO61X_LinPort@@UAEPAX_NI@Z 10076140 f   IO61X_Library_MSVC120_vc:IO61X_LinPort.obj
 0001:000753a0       ?CalculateFullProtID@IO61X_LinPort@@AAEEE@Z 100763a0 f   IO61X_Library_MSVC120_vc:IO61X_LinPort.obj
 0001:000753b0       ?ClearBufferList@IO61X_LinPort@@UAE_NXZ 100763b0 f   IO61X_Library_MSVC120_vc:IO61X_LinPort.obj
 0001:00075420       ?GetBufferData@IO61X_LinPort@@QAE_NIPAHPAI11PAE@Z 10076420 f   IO61X_Library_MSVC120_vc:IO61X_LinPort.obj
 0001:00075500       ?GetLatestMessageFromBuffer@?$IO61X_BufferFifo@UIO61X_LinMessage_T@@@@QAEPAUIO61X_LinMessage_T@@XZ 10076500 f i IO61X_Library_MSVC120_vc:IO61X_LinPort.obj
 0001:00075560       ?GetMessageFromBuffer@?$IO61X_BufferFifo@UIO61X_LinMessage_T@@@@QAEPAUIO61X_LinMessage_T@@XZ 10076560 f i IO61X_Library_MSVC120_vc:IO61X_LinPort.obj
 0001:00075580       ?IO61X_LINRwwbAcquireWriteIndex@IO61X_LinPort@@AAEXXZ 10076580 f   IO61X_Library_MSVC120_vc:IO61X_LinPort.obj
 0001:000755e0       ?IO61X_LINRwwbReleaseWriteIndex@IO61X_LinPort@@AAEXXZ 100765e0 f   IO61X_Library_MSVC120_vc:IO61X_LinPort.obj
 0001:00075610       ?Receive_spin@IO61X_LinPort@@UAE_NH@Z 10076610 f   IO61X_Library_MSVC120_vc:IO61X_LinPort.obj
 0001:00075790       ?Send_spin@IO61X_LinPort@@UAE_NXZ 10076790 f   IO61X_Library_MSVC120_vc:IO61X_LinPort.obj
 0001:000759b0       ?UpdateBuffer_spin@IO61X_LinPort@@UAE_NPAX0@Z 100769b0 f   IO61X_Library_MSVC120_vc:IO61X_LinPort.obj
 0001:00075b10       ?UpdateRwwb@IO61X_LinPort@@QAEXEEEE@Z 10076b10 f   IO61X_Library_MSVC120_vc:IO61X_LinPort.obj
 0001:00075c50       ?_Begin@?$_Hash@V?$_Umap_traits@HV?$IO61X_BufferFifo@UIO61X_LinMessage_T@@@@V?$_Uhash_compare@HU?$hash@H@std@@U?$equal_to@H@2@@std@@V?$allocator@U?$pair@$$CBHV?$IO61X_BufferFifo@UIO61X_LinMessage_T@@@@@std@@@3@$0A@@std@@@std@@IAE?AV?$_List_unchecked_iterator@V?$_List_val@U?$_List_simple_types@U?$pair@$$CBHV?$IO61X_BufferFifo@UIO61X_LinMessage_T@@@@@std@@@std@@@std@@@2@I@Z 10076c50 f i IO61X_Library_MSVC120_vc:IO61X_LinPort.obj
 0001:00075c70       ?_Buyheadnode@?$_List_alloc@$0A@U?$_List_base_types@U?$pair@$$CBHV?$IO61X_BufferFifo@UIO61X_LinMessage_T@@@@@std@@V?$allocator@U?$pair@$$CBHV?$IO61X_BufferFifo@UIO61X_LinMessage_T@@@@@std@@@2@@std@@@std@@QAEPAU?$_List_node@U?$pair@$$CBHV?$IO61X_BufferFifo@UIO61X_LinMessage_T@@@@@std@@PAX@2@XZ 10076c70 f i IO61X_Library_MSVC120_vc:IO61X_LinPort.obj
 0001:00075c80       ?_Buyheadnode@?$_List_alloc@$0A@U?$_List_base_types@V?$IO61X_BufferFifo@UIO61X_LinMessage_T@@@@V?$allocator@V?$IO61X_BufferFifo@UIO61X_LinMessage_T@@@@@std@@@std@@@std@@QAEPAU?$_List_node@V?$IO61X_BufferFifo@UIO61X_LinMessage_T@@@@PAX@2@XZ 10076c80 f i IO61X_Library_MSVC120_vc:IO61X_LinPort.obj
 0001:00075c90       ?_Buynode0@?$_List_alloc@$0A@U?$_List_base_types@U?$pair@$$CBHV?$IO61X_BufferFifo@UIO61X_LinMessage_T@@@@@std@@V?$allocator@U?$pair@$$CBHV?$IO61X_BufferFifo@UIO61X_LinMessage_T@@@@@std@@@2@@std@@@std@@QAEPAU?$_List_node@U?$pair@$$CBHV?$IO61X_BufferFifo@UIO61X_LinMessage_T@@@@@std@@PAX@2@PAU32@0@Z 10076c90 f i IO61X_Library_MSVC120_vc:IO61X_LinPort.obj
 0001:00075cd0       ?_Buynode0@?$_List_alloc@$0A@U?$_List_base_types@V?$IO61X_BufferFifo@UIO61X_LinMessage_T@@@@V?$allocator@V?$IO61X_BufferFifo@UIO61X_LinMessage_T@@@@@std@@@std@@@std@@QAEPAU?$_List_node@V?$IO61X_BufferFifo@UIO61X_LinMessage_T@@@@PAX@2@PAU32@0@Z 10076cd0 f i IO61X_Library_MSVC120_vc:IO61X_LinPort.obj
 0001:00075d10       ?_Check_size@?$_Hash@V?$_Umap_traits@HV?$IO61X_BufferFifo@UIO61X_LinMessage_T@@@@V?$_Uhash_compare@HU?$hash@H@std@@U?$equal_to@H@2@@std@@V?$allocator@U?$pair@$$CBHV?$IO61X_BufferFifo@UIO61X_LinMessage_T@@@@@std@@@3@$0A@@std@@@std@@IAEXXZ 10076d10 f i IO61X_Library_MSVC120_vc:IO61X_LinPort.obj
 0001:00075dd0       ?_Destroy@?$vector@V?$_List_unchecked_iterator@V?$_List_val@U?$_List_simple_types@U?$pair@$$CBHV?$IO61X_BufferFifo@UIO61X_LinMessage_T@@@@@std@@@std@@@std@@@std@@U?$_Wrap_alloc@V?$allocator@V?$_List_unchecked_iterator@V?$_List_val@U?$_List_simple_types@U?$pair@$$CBHV?$IO61X_BufferFifo@UIO61X_LinMessage_T@@@@@std@@@std@@@std@@@std@@@std@@@2@@std@@IAEXPAV?$_List_unchecked_iterator@V?$_List_val@U?$_List_simple_types@U?$pair@$$CBHV?$IO61X_BufferFifo@UIO61X_LinMessage_T@@@@@std@@@std@@@std@@@2@0@Z 10076dd0 f i IO61X_Library_MSVC120_vc:IO61X_LinPort.obj
 0001:00075de0       ?_Destroy_if_not_nil@?$_Hash@V?$_Umap_traits@HV?$IO61X_BufferFifo@UIO61X_LinMessage_T@@@@V?$_Uhash_compare@HU?$hash@H@std@@U?$equal_to@H@2@@std@@V?$allocator@U?$pair@$$CBHV?$IO61X_BufferFifo@UIO61X_LinMessage_T@@@@@std@@@3@$0A@@std@@@std@@IAEXV?$_List_unchecked_iterator@V?$_List_val@U?$_List_simple_types@U?$pair@$$CBHV?$IO61X_BufferFifo@UIO61X_LinMessage_T@@@@@std@@@std@@@std@@@2@@Z 10076de0 f i IO61X_Library_MSVC120_vc:IO61X_LinPort.obj
 0001:00075e20       ?_End@?$_Hash@V?$_Umap_traits@HV?$IO61X_BufferFifo@UIO61X_LinMessage_T@@@@V?$_Uhash_compare@HU?$hash@H@std@@U?$equal_to@H@2@@std@@V?$allocator@U?$pair@$$CBHV?$IO61X_BufferFifo@UIO61X_LinMessage_T@@@@@std@@@3@$0A@@std@@@std@@IAE?AV?$_List_unchecked_iterator@V?$_List_val@U?$_List_simple_types@U?$pair@$$CBHV?$IO61X_BufferFifo@UIO61X_LinMessage_T@@@@@std@@@std@@@std@@@2@I@Z 10076e20 f i IO61X_Library_MSVC120_vc:IO61X_LinPort.obj
 0001:00075e40       ?_Freeheadnode@?$_List_alloc@$0A@U?$_List_base_types@U?$pair@$$CBHV?$IO61X_BufferFifo@UIO61X_LinMessage_T@@@@@std@@V?$allocator@U?$pair@$$CBHV?$IO61X_BufferFifo@UIO61X_LinMessage_T@@@@@std@@@2@@std@@@std@@QAEXPAU?$_List_node@U?$pair@$$CBHV?$IO61X_BufferFifo@UIO61X_LinMessage_T@@@@@std@@PAX@2@@Z 10076e40 f i IO61X_Library_MSVC120_vc:IO61X_LinPort.obj
 0001:00075e60       ?_Freeheadnode@?$_List_alloc@$0A@U?$_List_base_types@V?$IO61X_BufferFifo@UIO61X_LinMessage_T@@@@V?$allocator@V?$IO61X_BufferFifo@UIO61X_LinMessage_T@@@@@std@@@std@@@std@@QAEXPAU?$_List_node@V?$IO61X_BufferFifo@UIO61X_LinMessage_T@@@@PAX@2@@Z 10076e60 f i IO61X_Library_MSVC120_vc:IO61X_LinPort.obj
 0001:00075e80       ?_Freenode@?$_List_buy@U?$pair@$$CBHV?$IO61X_BufferFifo@UIO61X_LinMessage_T@@@@@std@@V?$allocator@U?$pair@$$CBHV?$IO61X_BufferFifo@UIO61X_LinMessage_T@@@@@std@@@2@@std@@QAEXPAU?$_List_node@U?$pair@$$CBHV?$IO61X_BufferFifo@UIO61X_LinMessage_T@@@@@std@@PAX@2@@Z 10076e80 f i IO61X_Library_MSVC120_vc:IO61X_LinPort.obj
 0001:00075eb0       ?_Freenode@?$_List_buy@V?$IO61X_BufferFifo@UIO61X_LinMessage_T@@@@V?$allocator@V?$IO61X_BufferFifo@UIO61X_LinMessage_T@@@@@std@@@std@@QAEXPAU?$_List_node@V?$IO61X_BufferFifo@UIO61X_LinMessage_T@@@@PAX@2@@Z 10076eb0 f i IO61X_Library_MSVC120_vc:IO61X_LinPort.obj
 0001:00075ee0       ?_Getal@?$_List_alloc@$0A@U?$_List_base_types@U?$pair@$$CBHV?$IO61X_BufferFifo@UIO61X_LinMessage_T@@@@@std@@V?$allocator@U?$pair@$$CBHV?$IO61X_BufferFifo@UIO61X_LinMessage_T@@@@@std@@@2@@std@@@std@@QBE?AU?$_Wrap_alloc@V?$allocator@U?$_List_node@U?$pair@$$CBHV?$IO61X_BufferFifo@UIO61X_LinMessage_T@@@@@std@@PAX@std@@@std@@@2@XZ 10076ee0 f i IO61X_Library_MSVC120_vc:IO61X_LinPort.obj
 0001:00075ef0       ?_Getal@?$_List_alloc@$0A@U?$_List_base_types@V?$IO61X_BufferFifo@UIO61X_LinMessage_T@@@@V?$allocator@V?$IO61X_BufferFifo@UIO61X_LinMessage_T@@@@@std@@@std@@@std@@QBE?AU?$_Wrap_alloc@V?$allocator@U?$_List_node@V?$IO61X_BufferFifo@UIO61X_LinMessage_T@@@@PAX@std@@@std@@@2@XZ 10076ef0 f i IO61X_Library_MSVC120_vc:IO61X_LinPort.obj
 0001:00075f00       ?_Getal@?$_Vector_alloc@$0A@U?$_Vec_base_types@V?$_List_unchecked_iterator@V?$_List_val@U?$_List_simple_types@U?$pair@$$CBHV?$IO61X_BufferFifo@UIO61X_LinMessage_T@@@@@std@@@std@@@std@@@std@@U?$_Wrap_alloc@V?$allocator@V?$_List_unchecked_iterator@V?$_List_val@U?$_List_simple_types@U?$pair@$$CBHV?$IO61X_BufferFifo@UIO61X_LinMessage_T@@@@@std@@@std@@@std@@@std@@@std@@@2@@std@@@std@@QBE?AU?$_Wrap_alloc@U?$_Wrap_alloc@V?$allocator@V?$_List_unchecked_iterator@V?$_List_val@U?$_List_simple_types@U?$pair@$$CBHV?$IO61X_BufferFifo@UIO61X_LinMessage_T@@@@@std@@@std@@@std@@@std@@@std@@@std@@@2@XZ 10076f00 f i IO61X_Library_MSVC120_vc:IO61X_LinPort.obj
 0001:00075f10       ?_Gethash@?$_Hash_oper1@$0A@U?$hash@H@std@@@std@@QBE?AU?$hash@H@2@XZ 10076f10 f i IO61X_Library_MSVC120_vc:IO61X_LinPort.obj
 0001:00075f20       ?_Getkeyeq@?$_Hash_oper2@$0A@U?$hash@H@std@@U?$equal_to@H@2@@std@@QBE?AU?$equal_to@H@2@XZ 10076f20 f i IO61X_Library_MSVC120_vc:IO61X_LinPort.obj
 0001:00075f30       ?_Grow_to@?$vector@V?$_List_unchecked_iterator@V?$_List_val@U?$_List_simple_types@U?$pair@$$CBHV?$IO61X_BufferFifo@UIO61X_LinMessage_T@@@@@std@@@std@@@std@@@std@@U?$_Wrap_alloc@V?$allocator@V?$_List_unchecked_iterator@V?$_List_val@U?$_List_simple_types@U?$pair@$$CBHV?$IO61X_BufferFifo@UIO61X_LinMessage_T@@@@@std@@@std@@@std@@@std@@@std@@@2@@std@@IBEII@Z 10076f30 f i IO61X_Library_MSVC120_vc:IO61X_LinPort.obj
 0001:00075f70       ?_Hash_seq@std@@YAIPBEI@Z  10076f70 f i IO61X_Library_MSVC120_vc:IO61X_LinPort.obj
 0001:00075fa0       ?_Hashval@?$_Hash@V?$_Umap_traits@HV?$IO61X_BufferFifo@UIO61X_LinMessage_T@@@@V?$_Uhash_compare@HU?$hash@H@std@@U?$equal_to@H@2@@std@@V?$allocator@U?$pair@$$CBHV?$IO61X_BufferFifo@UIO61X_LinMessage_T@@@@@std@@@3@$0A@@std@@@std@@IBEIABH@Z 10076fa0 f i IO61X_Library_MSVC120_vc:IO61X_LinPort.obj
 0001:00076000       ?_Incsize@?$list@U?$pair@$$CBHV?$IO61X_BufferFifo@UIO61X_LinMessage_T@@@@@std@@V?$allocator@U?$pair@$$CBHV?$IO61X_BufferFifo@UIO61X_LinMessage_T@@@@@std@@@2@@std@@QAEXI@Z 10077000 f i IO61X_Library_MSVC120_vc:IO61X_LinPort.obj
 0001:00076030       ?_Incsize@?$list@V?$IO61X_BufferFifo@UIO61X_LinMessage_T@@@@V?$allocator@V?$IO61X_BufferFifo@UIO61X_LinMessage_T@@@@@std@@@std@@QAEXI@Z 10077030 f i IO61X_Library_MSVC120_vc:IO61X_LinPort.obj
 0001:00076060       ?_Init@?$_Hash@V?$_Umap_traits@HV?$IO61X_BufferFifo@UIO61X_LinMessage_T@@@@V?$_Uhash_compare@HU?$hash@H@std@@U?$equal_to@H@2@@std@@V?$allocator@U?$pair@$$CBHV?$IO61X_BufferFifo@UIO61X_LinMessage_T@@@@@std@@@3@$0A@@std@@@std@@IAEXI@Z 10077060 f i IO61X_Library_MSVC120_vc:IO61X_LinPort.obj
 0001:000760a0       ?_Insert_bucket@?$_Hash@V?$_Umap_traits@HV?$IO61X_BufferFifo@UIO61X_LinMessage_T@@@@V?$_Uhash_compare@HU?$hash@H@std@@U?$equal_to@H@2@@std@@V?$allocator@U?$pair@$$CBHV?$IO61X_BufferFifo@UIO61X_LinMessage_T@@@@@std@@@3@$0A@@std@@@std@@IAEXV?$_List_unchecked_iterator@V?$_List_val@U?$_List_simple_types@U?$pair@$$CBHV?$IO61X_BufferFifo@UIO61X_LinMessage_T@@@@@std@@@std@@@std@@@2@0I@Z 100770a0 f i IO61X_Library_MSVC120_vc:IO61X_LinPort.obj
 0001:00076100       ?_Insert_n@?$vector@V?$_List_unchecked_iterator@V?$_List_val@U?$_List_simple_types@U?$pair@$$CBHV?$IO61X_BufferFifo@UIO61X_LinMessage_T@@@@@std@@@std@@@std@@@std@@U?$_Wrap_alloc@V?$allocator@V?$_List_unchecked_iterator@V?$_List_val@U?$_List_simple_types@U?$pair@$$CBHV?$IO61X_BufferFifo@UIO61X_LinMessage_T@@@@@std@@@std@@@std@@@std@@@std@@@2@@std@@IAE?AV?$_Vector_iterator@V?$_Vector_val@U?$_Simple_types@V?$_List_unchecked_iterator@V?$_List_val@U?$_List_simple_types@U?$pair@$$CBHV?$IO61X_BufferFifo@UIO61X_LinMessage_T@@@@@std@@@std@@@std@@@std@@@std@@@std@@@2@V?$_Vector_const_iterator@V?$_Vector_val@U?$_Simple_types@V?$_List_unchecked_iterator@V?$_List_val@U?$_List_simple_types@U?$pair@$$CBHV?$IO61X_BufferFifo@UIO61X_LinMessage_T@@@@@std@@@std@@@std@@@std@@@std@@@std@@@2@IABV?$_List_unchecked_iterator@V?$_List_val@U?$_List_simple_types@U?$pair@$$CBHV?$IO61X_BufferFifo@UIO61X_LinMessage_T@@@@@std@@@std@@@std@@@2@@Z 10077100 f i IO61X_Library_MSVC120_vc:IO61X_LinPort.obj
 0001:00076370       ?_Make_iter@?$_Hash@V?$_Umap_traits@HV?$IO61X_BufferFifo@UIO61X_LinMessage_T@@@@V?$_Uhash_compare@HU?$hash@H@std@@U?$equal_to@H@2@@std@@V?$allocator@U?$pair@$$CBHV?$IO61X_BufferFifo@UIO61X_LinMessage_T@@@@@std@@@3@$0A@@std@@@std@@QBE?AV?$_List_iterator@V?$_List_val@U?$_List_simple_types@U?$pair@$$CBHV?$IO61X_BufferFifo@UIO61X_LinMessage_T@@@@@std@@@std@@@std@@@2@V?$_List_unchecked_const_iterator@V?$_List_val@U?$_List_simple_types@U?$pair@$$CBHV?$IO61X_BufferFifo@UIO61X_LinMessage_T@@@@@std@@@std@@@std@@U_Iterator_base0@2@@2@@Z 10077370 f i IO61X_Library_MSVC120_vc:IO61X_LinPort.obj
 0001:00076380       ?_Make_iter@?$list@U?$pair@$$CBHV?$IO61X_BufferFifo@UIO61X_LinMessage_T@@@@@std@@V?$allocator@U?$pair@$$CBHV?$IO61X_BufferFifo@UIO61X_LinMessage_T@@@@@std@@@2@@std@@QBE?AV?$_List_iterator@V?$_List_val@U?$_List_simple_types@U?$pair@$$CBHV?$IO61X_BufferFifo@UIO61X_LinMessage_T@@@@@std@@@std@@@std@@@2@V?$_List_const_iterator@V?$_List_val@U?$_List_simple_types@U?$pair@$$CBHV?$IO61X_BufferFifo@UIO61X_LinMessage_T@@@@@std@@@std@@@std@@@2@@Z 10077380 f i IO61X_Library_MSVC120_vc:IO61X_LinPort.obj
 0001:00076390       ?_Make_iter@?$list@U?$pair@$$CBHV?$IO61X_BufferFifo@UIO61X_LinMessage_T@@@@@std@@V?$allocator@U?$pair@$$CBHV?$IO61X_BufferFifo@UIO61X_LinMessage_T@@@@@std@@@2@@std@@QBE?AV?$_List_iterator@V?$_List_val@U?$_List_simple_types@U?$pair@$$CBHV?$IO61X_BufferFifo@UIO61X_LinMessage_T@@@@@std@@@std@@@std@@@2@V?$_List_unchecked_const_iterator@V?$_List_val@U?$_List_simple_types@U?$pair@$$CBHV?$IO61X_BufferFifo@UIO61X_LinMessage_T@@@@@std@@@std@@@std@@U_Iterator_base0@2@@2@@Z 10077390 f i IO61X_Library_MSVC120_vc:IO61X_LinPort.obj
 0001:000763a0       ?_Mynode@?$_List_unchecked_const_iterator@V?$_List_val@U?$_List_simple_types@U?$pair@$$CBHV?$IO61X_BufferFifo@UIO61X_LinMessage_T@@@@@std@@@std@@@std@@U_Iterator_base0@2@@std@@QBEPAU?$_List_node@U?$pair@$$CBHV?$IO61X_BufferFifo@UIO61X_LinMessage_T@@@@@std@@PAX@2@XZ 100773a0 f i IO61X_Library_MSVC120_vc:IO61X_LinPort.obj
 0001:000763b0       ?_Mynode@?$_List_unchecked_const_iterator@V?$_List_val@U?$_List_simple_types@V?$IO61X_BufferFifo@UIO61X_LinMessage_T@@@@@std@@@std@@U_Iterator_base0@2@@std@@QBEPAU?$_List_node@V?$IO61X_BufferFifo@UIO61X_LinMessage_T@@@@PAX@2@XZ 100773b0 f i IO61X_Library_MSVC120_vc:IO61X_LinPort.obj
 0001:000763c0       ?_Myval@?$_List_val@U?$_List_simple_types@U?$pair@$$CBHV?$IO61X_BufferFifo@UIO61X_LinMessage_T@@@@@std@@@std@@@std@@SAAAU?$pair@$$CBHV?$IO61X_BufferFifo@UIO61X_LinMessage_T@@@@@2@PAU?$_List_node@U?$pair@$$CBHV?$IO61X_BufferFifo@UIO61X_LinMessage_T@@@@@std@@PAX@2@@Z 100773c0 f i IO61X_Library_MSVC120_vc:IO61X_LinPort.obj
 0001:000763d0       ?_Myval@?$_List_val@U?$_List_simple_types@V?$IO61X_BufferFifo@UIO61X_LinMessage_T@@@@@std@@@std@@SAAAV?$IO61X_BufferFifo@UIO61X_LinMessage_T@@@@PAU?$_List_node@V?$IO61X_BufferFifo@UIO61X_LinMessage_T@@@@PAX@2@@Z 100773d0 f i IO61X_Library_MSVC120_vc:IO61X_LinPort.obj
 0001:000763e0       ?_Nextnode@?$_List_val@U?$_List_simple_types@U?$pair@$$CBHV?$IO61X_BufferFifo@UIO61X_LinMessage_T@@@@@std@@@std@@@std@@SAAAPAU?$_List_node@U?$pair@$$CBHV?$IO61X_BufferFifo@UIO61X_LinMessage_T@@@@@std@@PAX@2@PAU32@@Z 100773e0 f i IO61X_Library_MSVC120_vc:IO61X_LinPort.obj
 0001:000763f0       ?_Nextnode@?$_List_val@U?$_List_simple_types@V?$IO61X_BufferFifo@UIO61X_LinMessage_T@@@@@std@@@std@@SAAAPAU?$_List_node@V?$IO61X_BufferFifo@UIO61X_LinMessage_T@@@@PAX@2@PAU32@@Z 100773f0 f i IO61X_Library_MSVC120_vc:IO61X_LinPort.obj
 0001:00076400       ?_Orphan_all@_Container_base0@std@@QAEXXZ 10077400 f i IO61X_Library_MSVC120_vc:IO61X_LinPort.obj
 0001:00076410       ?_Orphan_range@?$vector@V?$_List_unchecked_iterator@V?$_List_val@U?$_List_simple_types@U?$pair@$$CBHV?$IO61X_BufferFifo@UIO61X_LinMessage_T@@@@@std@@@std@@@std@@@std@@U?$_Wrap_alloc@V?$allocator@V?$_List_unchecked_iterator@V?$_List_val@U?$_List_simple_types@U?$pair@$$CBHV?$IO61X_BufferFifo@UIO61X_LinMessage_T@@@@@std@@@std@@@std@@@std@@@std@@@2@@std@@IBEXPAV?$_List_unchecked_iterator@V?$_List_val@U?$_List_simple_types@U?$pair@$$CBHV?$IO61X_BufferFifo@UIO61X_LinMessage_T@@@@@std@@@std@@@std@@@2@0@Z 10077410 f i IO61X_Library_MSVC120_vc:IO61X_LinPort.obj
 0001:00076420       ?_Prevnode@?$_List_val@U?$_List_simple_types@U?$pair@$$CBHV?$IO61X_BufferFifo@UIO61X_LinMessage_T@@@@@std@@@std@@@std@@SAAAPAU?$_List_node@U?$pair@$$CBHV?$IO61X_BufferFifo@UIO61X_LinMessage_T@@@@@std@@PAX@2@PAU32@@Z 10077420 f i IO61X_Library_MSVC120_vc:IO61X_LinPort.obj
 0001:00076430       ?_Prevnode@?$_List_val@U?$_List_simple_types@V?$IO61X_BufferFifo@UIO61X_LinMessage_T@@@@@std@@@std@@SAAAPAU?$_List_node@V?$IO61X_BufferFifo@UIO61X_LinMessage_T@@@@PAX@2@PAU32@@Z 10077430 f i IO61X_Library_MSVC120_vc:IO61X_LinPort.obj
 0001:00076440       ?_Reinsert@?$_Hash@V?$_Umap_traits@HV?$IO61X_BufferFifo@UIO61X_LinMessage_T@@@@V?$_Uhash_compare@HU?$hash@H@std@@U?$equal_to@H@2@@std@@V?$allocator@U?$pair@$$CBHV?$IO61X_BufferFifo@UIO61X_LinMessage_T@@@@@std@@@3@$0A@@std@@@std@@IAEXXZ 10077440 f i IO61X_Library_MSVC120_vc:IO61X_LinPort.obj
 0001:00076480       ?_Tidy@?$list@U?$pair@$$CBHV?$IO61X_BufferFifo@UIO61X_LinMessage_T@@@@@std@@V?$allocator@U?$pair@$$CBHV?$IO61X_BufferFifo@UIO61X_LinMessage_T@@@@@std@@@2@@std@@QAEXXZ 10077480 f i IO61X_Library_MSVC120_vc:IO61X_LinPort.obj
 0001:00076490       ?_Tidy@?$list@V?$IO61X_BufferFifo@UIO61X_LinMessage_T@@@@V?$allocator@V?$IO61X_BufferFifo@UIO61X_LinMessage_T@@@@@std@@@std@@QAEXXZ 10077490 f i IO61X_Library_MSVC120_vc:IO61X_LinPort.obj
 0001:000764a0       ?_Tidy@?$vector@V?$_List_unchecked_iterator@V?$_List_val@U?$_List_simple_types@U?$pair@$$CBHV?$IO61X_BufferFifo@UIO61X_LinMessage_T@@@@@std@@@std@@@std@@@std@@U?$_Wrap_alloc@V?$allocator@V?$_List_unchecked_iterator@V?$_List_val@U?$_List_simple_types@U?$pair@$$CBHV?$IO61X_BufferFifo@UIO61X_LinMessage_T@@@@@std@@@std@@@std@@@std@@@std@@@2@@std@@IAEXXZ 100774a0 f i IO61X_Library_MSVC120_vc:IO61X_LinPort.obj
 0001:000764d0       ?_Ufill@?$vector@V?$_List_unchecked_iterator@V?$_List_val@U?$_List_simple_types@U?$pair@$$CBHV?$IO61X_BufferFifo@UIO61X_LinMessage_T@@@@@std@@@std@@@std@@@std@@U?$_Wrap_alloc@V?$allocator@V?$_List_unchecked_iterator@V?$_List_val@U?$_List_simple_types@U?$pair@$$CBHV?$IO61X_BufferFifo@UIO61X_LinMessage_T@@@@@std@@@std@@@std@@@std@@@std@@@2@@std@@IAEPAV?$_List_unchecked_iterator@V?$_List_val@U?$_List_simple_types@U?$pair@$$CBHV?$IO61X_BufferFifo@UIO61X_LinMessage_T@@@@@std@@@std@@@std@@@2@PAV32@IPBV32@@Z 100774d0 f i IO61X_Library_MSVC120_vc:IO61X_LinPort.obj
 0001:00076500       ?_Unchecked_begin@?$_Hash@V?$_Umap_traits@HV?$IO61X_BufferFifo@UIO61X_LinMessage_T@@@@V?$_Uhash_compare@HU?$hash@H@std@@U?$equal_to@H@2@@std@@V?$allocator@U?$pair@$$CBHV?$IO61X_BufferFifo@UIO61X_LinMessage_T@@@@@std@@@3@$0A@@std@@@std@@QAE?AV?$_List_unchecked_iterator@V?$_List_val@U?$_List_simple_types@U?$pair@$$CBHV?$IO61X_BufferFifo@UIO61X_LinMessage_T@@@@@std@@@std@@@std@@@2@XZ 10077500 f i IO61X_Library_MSVC120_vc:IO61X_LinPort.obj
 0001:00076510       ?_Unchecked_begin@?$list@U?$pair@$$CBHV?$IO61X_BufferFifo@UIO61X_LinMessage_T@@@@@std@@V?$allocator@U?$pair@$$CBHV?$IO61X_BufferFifo@UIO61X_LinMessage_T@@@@@std@@@2@@std@@QAE?AV?$_List_unchecked_iterator@V?$_List_val@U?$_List_simple_types@U?$pair@$$CBHV?$IO61X_BufferFifo@UIO61X_LinMessage_T@@@@@std@@@std@@@std@@@2@XZ 10077510 f i IO61X_Library_MSVC120_vc:IO61X_LinPort.obj
 0001:00076520       ?_Unchecked_end@?$_Hash@V?$_Umap_traits@HV?$IO61X_BufferFifo@UIO61X_LinMessage_T@@@@V?$_Uhash_compare@HU?$hash@H@std@@U?$equal_to@H@2@@std@@V?$allocator@U?$pair@$$CBHV?$IO61X_BufferFifo@UIO61X_LinMessage_T@@@@@std@@@3@$0A@@std@@@std@@QAE?AV?$_List_unchecked_iterator@V?$_List_val@U?$_List_simple_types@U?$pair@$$CBHV?$IO61X_BufferFifo@UIO61X_LinMessage_T@@@@@std@@@std@@@std@@@2@XZ 10077520 f i IO61X_Library_MSVC120_vc:IO61X_LinPort.obj
 0001:00076530       ?_Unchecked_end@?$list@U?$pair@$$CBHV?$IO61X_BufferFifo@UIO61X_LinMessage_T@@@@@std@@V?$allocator@U?$pair@$$CBHV?$IO61X_BufferFifo@UIO61X_LinMessage_T@@@@@std@@@2@@std@@QAE?AV?$_List_unchecked_iterator@V?$_List_val@U?$_List_simple_types@U?$pair@$$CBHV?$IO61X_BufferFifo@UIO61X_LinMessage_T@@@@@std@@@std@@@std@@@2@XZ 10077530 f i IO61X_Library_MSVC120_vc:IO61X_LinPort.obj
 0001:00076540       ?_Unchecked_end@?$list@V?$IO61X_BufferFifo@UIO61X_LinMessage_T@@@@V?$allocator@V?$IO61X_BufferFifo@UIO61X_LinMessage_T@@@@@std@@@std@@QAE?AV?$_List_unchecked_iterator@V?$_List_val@U?$_List_simple_types@V?$IO61X_BufferFifo@UIO61X_LinMessage_T@@@@@std@@@std@@@2@XZ 10077540 f i IO61X_Library_MSVC120_vc:IO61X_LinPort.obj
 0001:00076550       ?_Unchecked_splice@?$list@U?$pair@$$CBHV?$IO61X_BufferFifo@UIO61X_LinMessage_T@@@@@std@@V?$allocator@U?$pair@$$CBHV?$IO61X_BufferFifo@UIO61X_LinMessage_T@@@@@std@@@2@@std@@QAEXV?$_List_unchecked_const_iterator@V?$_List_val@U?$_List_simple_types@U?$pair@$$CBHV?$IO61X_BufferFifo@UIO61X_LinMessage_T@@@@@std@@@std@@@std@@U_Iterator_base0@2@@2@00@Z 10077550 f i IO61X_Library_MSVC120_vc:IO61X_LinPort.obj
 0001:000765a0       ?_Unlinknode@?$list@U?$pair@$$CBHV?$IO61X_BufferFifo@UIO61X_LinMessage_T@@@@@std@@V?$allocator@U?$pair@$$CBHV?$IO61X_BufferFifo@UIO61X_LinMessage_T@@@@@std@@@2@@std@@QAEPAU?$_List_node@U?$pair@$$CBHV?$IO61X_BufferFifo@UIO61X_LinMessage_T@@@@@std@@PAX@2@V?$_List_const_iterator@V?$_List_val@U?$_List_simple_types@U?$pair@$$CBHV?$IO61X_BufferFifo@UIO61X_LinMessage_T@@@@@std@@@std@@@std@@@2@@Z 100775a0 f i IO61X_Library_MSVC120_vc:IO61X_LinPort.obj
 0001:000765c0       ?_Unused_capacity@?$vector@V?$_List_unchecked_iterator@V?$_List_val@U?$_List_simple_types@U?$pair@$$CBHV?$IO61X_BufferFifo@UIO61X_LinMessage_T@@@@@std@@@std@@@std@@@std@@U?$_Wrap_alloc@V?$allocator@V?$_List_unchecked_iterator@V?$_List_val@U?$_List_simple_types@U?$pair@$$CBHV?$IO61X_BufferFifo@UIO61X_LinMessage_T@@@@@std@@@std@@@std@@@std@@@std@@@2@@std@@QBEIXZ 100775c0 f i IO61X_Library_MSVC120_vc:IO61X_LinPort.obj
 0001:000765d0       ?_Vec_hi@?$_Hash@V?$_Umap_traits@HV?$IO61X_BufferFifo@UIO61X_LinMessage_T@@@@V?$_Uhash_compare@HU?$hash@H@std@@U?$equal_to@H@2@@std@@V?$allocator@U?$pair@$$CBHV?$IO61X_BufferFifo@UIO61X_LinMessage_T@@@@@std@@@3@$0A@@std@@@std@@IAEAAV?$_List_unchecked_iterator@V?$_List_val@U?$_List_simple_types@U?$pair@$$CBHV?$IO61X_BufferFifo@UIO61X_LinMessage_T@@@@@std@@@std@@@std@@@2@I@Z 100775d0 f i IO61X_Library_MSVC120_vc:IO61X_LinPort.obj
 0001:000765f0       ?_Vec_lo@?$_Hash@V?$_Umap_traits@HV?$IO61X_BufferFifo@UIO61X_LinMessage_T@@@@V?$_Uhash_compare@HU?$hash@H@std@@U?$equal_to@H@2@@std@@V?$allocator@U?$pair@$$CBHV?$IO61X_BufferFifo@UIO61X_LinMessage_T@@@@@std@@@3@$0A@@std@@@std@@IAEAAV?$_List_unchecked_iterator@V?$_List_val@U?$_List_simple_types@U?$pair@$$CBHV?$IO61X_BufferFifo@UIO61X_LinMessage_T@@@@@std@@@std@@@std@@@2@I@Z 100775f0 f i IO61X_Library_MSVC120_vc:IO61X_LinPort.obj
 0001:00076600       ?_Xlen@?$vector@V?$_List_unchecked_iterator@V?$_List_val@U?$_List_simple_types@U?$pair@$$CBHV?$IO61X_BufferFifo@UIO61X_LinMessage_T@@@@@std@@@std@@@std@@@std@@U?$_Wrap_alloc@V?$allocator@V?$_List_unchecked_iterator@V?$_List_val@U?$_List_simple_types@U?$pair@$$CBHV?$IO61X_BufferFifo@UIO61X_LinMessage_T@@@@@std@@@std@@@std@@@std@@@std@@@2@@std@@IBEXXZ 10077600 f i IO61X_Library_MSVC120_vc:IO61X_LinPort.obj
 0001:00076610       ?allocate@?$_Wrap_alloc@U?$_Wrap_alloc@V?$allocator@V?$_List_unchecked_iterator@V?$_List_val@U?$_List_simple_types@U?$pair@$$CBHV?$IO61X_BufferFifo@UIO61X_LinMessage_T@@@@@std@@@std@@@std@@@std@@@std@@@std@@@std@@QAEPAV?$_List_unchecked_iterator@V?$_List_val@U?$_List_simple_types@U?$pair@$$CBHV?$IO61X_BufferFifo@UIO61X_LinMessage_T@@@@@std@@@std@@@std@@@2@I@Z 10077610 f i IO61X_Library_MSVC120_vc:IO61X_LinPort.obj
 0001:00076650       ?allocate@?$_Wrap_alloc@V?$allocator@U?$_List_node@U?$pair@$$CBHV?$IO61X_BufferFifo@UIO61X_LinMessage_T@@@@@std@@PAX@std@@@std@@@std@@QAEPAU?$_List_node@U?$pair@$$CBHV?$IO61X_BufferFifo@UIO61X_LinMessage_T@@@@@std@@PAX@2@I@Z 10077650 f i IO61X_Library_MSVC120_vc:IO61X_LinPort.obj
 0001:00076690       ?allocate@?$_Wrap_alloc@V?$allocator@U?$_List_node@V?$IO61X_BufferFifo@UIO61X_LinMessage_T@@@@PAX@std@@@std@@@std@@QAEPAU?$_List_node@V?$IO61X_BufferFifo@UIO61X_LinMessage_T@@@@PAX@2@I@Z 10077690 f i IO61X_Library_MSVC120_vc:IO61X_LinPort.obj
 0001:000766d0       ?allocate@?$_Wrap_alloc@V?$allocator@V?$_List_unchecked_iterator@V?$_List_val@U?$_List_simple_types@U?$pair@$$CBHV?$IO61X_BufferFifo@UIO61X_LinMessage_T@@@@@std@@@std@@@std@@@std@@@std@@@std@@QAEPAV?$_List_unchecked_iterator@V?$_List_val@U?$_List_simple_types@U?$pair@$$CBHV?$IO61X_BufferFifo@UIO61X_LinMessage_T@@@@@std@@@std@@@std@@@2@I@Z 100776d0 f i IO61X_Library_MSVC120_vc:IO61X_LinPort.obj
 0001:00076710       ?allocate@?$allocator@U?$_List_node@U?$pair@$$CBHV?$IO61X_BufferFifo@UIO61X_LinMessage_T@@@@@std@@PAX@std@@@std@@QAEPAU?$_List_node@U?$pair@$$CBHV?$IO61X_BufferFifo@UIO61X_LinMessage_T@@@@@std@@PAX@2@I@Z 10077710 f i IO61X_Library_MSVC120_vc:IO61X_LinPort.obj
 0001:00076750       ?allocate@?$allocator@U?$_List_node@V?$IO61X_BufferFifo@UIO61X_LinMessage_T@@@@PAX@std@@@std@@QAEPAU?$_List_node@V?$IO61X_BufferFifo@UIO61X_LinMessage_T@@@@PAX@2@I@Z 10077750 f i IO61X_Library_MSVC120_vc:IO61X_LinPort.obj
 0001:00076790       ?allocate@?$allocator@V?$_List_unchecked_iterator@V?$_List_val@U?$_List_simple_types@U?$pair@$$CBHV?$IO61X_BufferFifo@UIO61X_LinMessage_T@@@@@std@@@std@@@std@@@std@@@std@@QAEPAV?$_List_unchecked_iterator@V?$_List_val@U?$_List_simple_types@U?$pair@$$CBHV?$IO61X_BufferFifo@UIO61X_LinMessage_T@@@@@std@@@std@@@std@@@2@I@Z 10077790 f i IO61X_Library_MSVC120_vc:IO61X_LinPort.obj
 0001:000767d0       ?assign@?$vector@V?$_List_unchecked_iterator@V?$_List_val@U?$_List_simple_types@U?$pair@$$CBHV?$IO61X_BufferFifo@UIO61X_LinMessage_T@@@@@std@@@std@@@std@@@std@@U?$_Wrap_alloc@V?$allocator@V?$_List_unchecked_iterator@V?$_List_val@U?$_List_simple_types@U?$pair@$$CBHV?$IO61X_BufferFifo@UIO61X_LinMessage_T@@@@@std@@@std@@@std@@@std@@@std@@@2@@std@@QAEXIABV?$_List_unchecked_iterator@V?$_List_val@U?$_List_simple_types@U?$pair@$$CBHV?$IO61X_BufferFifo@UIO61X_LinMessage_T@@@@@std@@@std@@@std@@@2@@Z 100777d0 f i IO61X_Library_MSVC120_vc:IO61X_LinPort.obj
 0001:000767f0       ?at@?$unordered_map@HV?$IO61X_BufferFifo@UIO61X_LinMessage_T@@@@U?$hash@H@std@@U?$equal_to@H@3@V?$allocator@U?$pair@$$CBHV?$IO61X_BufferFifo@UIO61X_LinMessage_T@@@@@std@@@3@@std@@QAEAAV?$IO61X_BufferFifo@UIO61X_LinMessage_T@@@@ABH@Z 100777f0 f i IO61X_Library_MSVC120_vc:IO61X_LinPort.obj
 0001:00076820       ?back@?$list@V?$IO61X_BufferFifo@UIO61X_LinMessage_T@@@@V?$allocator@V?$IO61X_BufferFifo@UIO61X_LinMessage_T@@@@@std@@@std@@QAEAAV?$IO61X_BufferFifo@UIO61X_LinMessage_T@@@@XZ 10077820 f i IO61X_Library_MSVC120_vc:IO61X_LinPort.obj
 0001:00076830       ?begin@?$list@U?$pair@$$CBHV?$IO61X_BufferFifo@UIO61X_LinMessage_T@@@@@std@@V?$allocator@U?$pair@$$CBHV?$IO61X_BufferFifo@UIO61X_LinMessage_T@@@@@std@@@2@@std@@QAE?AV?$_List_iterator@V?$_List_val@U?$_List_simple_types@U?$pair@$$CBHV?$IO61X_BufferFifo@UIO61X_LinMessage_T@@@@@std@@@std@@@std@@@2@XZ 10077830 f i IO61X_Library_MSVC120_vc:IO61X_LinPort.obj
 0001:00076840       ?begin@?$list@V?$IO61X_BufferFifo@UIO61X_LinMessage_T@@@@V?$allocator@V?$IO61X_BufferFifo@UIO61X_LinMessage_T@@@@@std@@@std@@QAE?AV?$_List_iterator@V?$_List_val@U?$_List_simple_types@V?$IO61X_BufferFifo@UIO61X_LinMessage_T@@@@@std@@@std@@@2@XZ 10077840 f i IO61X_Library_MSVC120_vc:IO61X_LinPort.obj
 0001:00076850       ?begin@?$vector@V?$_List_unchecked_iterator@V?$_List_val@U?$_List_simple_types@U?$pair@$$CBHV?$IO61X_BufferFifo@UIO61X_LinMessage_T@@@@@std@@@std@@@std@@@std@@U?$_Wrap_alloc@V?$allocator@V?$_List_unchecked_iterator@V?$_List_val@U?$_List_simple_types@U?$pair@$$CBHV?$IO61X_BufferFifo@UIO61X_LinMessage_T@@@@@std@@@std@@@std@@@std@@@std@@@2@@std@@QAE?AV?$_Vector_iterator@V?$_Vector_val@U?$_Simple_types@V?$_List_unchecked_iterator@V?$_List_val@U?$_List_simple_types@U?$pair@$$CBHV?$IO61X_BufferFifo@UIO61X_LinMessage_T@@@@@std@@@std@@@std@@@std@@@std@@@std@@@2@XZ 10077850 f i IO61X_Library_MSVC120_vc:IO61X_LinPort.obj
 0001:00076860       ?bucket_count@?$_Hash@V?$_Umap_traits@HV?$IO61X_BufferFifo@UIO61X_LinMessage_T@@@@V?$_Uhash_compare@HU?$hash@H@std@@U?$equal_to@H@2@@std@@V?$allocator@U?$pair@$$CBHV?$IO61X_BufferFifo@UIO61X_LinMessage_T@@@@@std@@@3@$0A@@std@@@std@@QBEIXZ 10077860 f i IO61X_Library_MSVC120_vc:IO61X_LinPort.obj
 0001:00076870       ?capacity@?$vector@V?$_List_unchecked_iterator@V?$_List_val@U?$_List_simple_types@U?$pair@$$CBHV?$IO61X_BufferFifo@UIO61X_LinMessage_T@@@@@std@@@std@@@std@@@std@@U?$_Wrap_alloc@V?$allocator@V?$_List_unchecked_iterator@V?$_List_val@U?$_List_simple_types@U?$pair@$$CBHV?$IO61X_BufferFifo@UIO61X_LinMessage_T@@@@@std@@@std@@@std@@@std@@@std@@@2@@std@@QBEIXZ 10077870 f i IO61X_Library_MSVC120_vc:IO61X_LinPort.obj
 0001:00076880       ?clear@?$_Hash@V?$_Umap_traits@HV?$IO61X_BufferFifo@UIO61X_LinMessage_T@@@@V?$_Uhash_compare@HU?$hash@H@std@@U?$equal_to@H@2@@std@@V?$allocator@U?$pair@$$CBHV?$IO61X_BufferFifo@UIO61X_LinMessage_T@@@@@std@@@3@$0A@@std@@@std@@QAEXXZ 10077880 f i IO61X_Library_MSVC120_vc:IO61X_LinPort.obj
 0001:000768c0       ?clear@?$list@U?$pair@$$CBHV?$IO61X_BufferFifo@UIO61X_LinMessage_T@@@@@std@@V?$allocator@U?$pair@$$CBHV?$IO61X_BufferFifo@UIO61X_LinMessage_T@@@@@std@@@2@@std@@QAEXXZ 100778c0 f i IO61X_Library_MSVC120_vc:IO61X_LinPort.obj
 0001:00076910       ?clear@?$list@V?$IO61X_BufferFifo@UIO61X_LinMessage_T@@@@V?$allocator@V?$IO61X_BufferFifo@UIO61X_LinMessage_T@@@@@std@@@std@@QAEXXZ 10077910 f i IO61X_Library_MSVC120_vc:IO61X_LinPort.obj
 0001:00076960       ?clear@?$vector@V?$_List_unchecked_iterator@V?$_List_val@U?$_List_simple_types@U?$pair@$$CBHV?$IO61X_BufferFifo@UIO61X_LinMessage_T@@@@@std@@@std@@@std@@@std@@U?$_Wrap_alloc@V?$allocator@V?$_List_unchecked_iterator@V?$_List_val@U?$_List_simple_types@U?$pair@$$CBHV?$IO61X_BufferFifo@UIO61X_LinMessage_T@@@@@std@@@std@@@std@@@std@@@std@@@2@@std@@QAEXXZ 10077960 f i IO61X_Library_MSVC120_vc:IO61X_LinPort.obj
 0001:00076970       ?construct@?$allocator@V?$_List_unchecked_iterator@V?$_List_val@U?$_List_simple_types@U?$pair@$$CBHV?$IO61X_BufferFifo@UIO61X_LinMessage_T@@@@@std@@@std@@@std@@@std@@@std@@QAEXPAV?$_List_unchecked_iterator@V?$_List_val@U?$_List_simple_types@U?$pair@$$CBHV?$IO61X_BufferFifo@UIO61X_LinMessage_T@@@@@std@@@std@@@std@@@2@ABV32@@Z 10077970 f i IO61X_Library_MSVC120_vc:IO61X_LinPort.obj
 0001:00076990       ?deallocate@?$_Wrap_alloc@U?$_Wrap_alloc@V?$allocator@V?$_List_unchecked_iterator@V?$_List_val@U?$_List_simple_types@U?$pair@$$CBHV?$IO61X_BufferFifo@UIO61X_LinMessage_T@@@@@std@@@std@@@std@@@std@@@std@@@std@@@std@@QAEXPAV?$_List_unchecked_iterator@V?$_List_val@U?$_List_simple_types@U?$pair@$$CBHV?$IO61X_BufferFifo@UIO61X_LinMessage_T@@@@@std@@@std@@@std@@@2@I@Z 10077990 f i IO61X_Library_MSVC120_vc:IO61X_LinPort.obj
 0001:000769b0       ?deallocate@?$_Wrap_alloc@V?$allocator@U?$_List_node@U?$pair@$$CBHV?$IO61X_BufferFifo@UIO61X_LinMessage_T@@@@@std@@PAX@std@@@std@@@std@@QAEXPAU?$_List_node@U?$pair@$$CBHV?$IO61X_BufferFifo@UIO61X_LinMessage_T@@@@@std@@PAX@2@I@Z 100779b0 f i IO61X_Library_MSVC120_vc:IO61X_LinPort.obj
 0001:000769d0       ?deallocate@?$_Wrap_alloc@V?$allocator@U?$_List_node@V?$IO61X_BufferFifo@UIO61X_LinMessage_T@@@@PAX@std@@@std@@@std@@QAEXPAU?$_List_node@V?$IO61X_BufferFifo@UIO61X_LinMessage_T@@@@PAX@2@I@Z 100779d0 f i IO61X_Library_MSVC120_vc:IO61X_LinPort.obj
 0001:000769f0       ?deallocate@?$_Wrap_alloc@V?$allocator@V?$_List_unchecked_iterator@V?$_List_val@U?$_List_simple_types@U?$pair@$$CBHV?$IO61X_BufferFifo@UIO61X_LinMessage_T@@@@@std@@@std@@@std@@@std@@@std@@@std@@QAEXPAV?$_List_unchecked_iterator@V?$_List_val@U?$_List_simple_types@U?$pair@$$CBHV?$IO61X_BufferFifo@UIO61X_LinMessage_T@@@@@std@@@std@@@std@@@2@I@Z 100779f0 f i IO61X_Library_MSVC120_vc:IO61X_LinPort.obj
 0001:00076a10       ?deallocate@?$allocator@U?$_List_node@U?$pair@$$CBHV?$IO61X_BufferFifo@UIO61X_LinMessage_T@@@@@std@@PAX@std@@@std@@QAEXPAU?$_List_node@U?$pair@$$CBHV?$IO61X_BufferFifo@UIO61X_LinMessage_T@@@@@std@@PAX@2@I@Z 10077a10 f i IO61X_Library_MSVC120_vc:IO61X_LinPort.obj
 0001:00076a30       ?deallocate@?$allocator@U?$_List_node@V?$IO61X_BufferFifo@UIO61X_LinMessage_T@@@@PAX@std@@@std@@QAEXPAU?$_List_node@V?$IO61X_BufferFifo@UIO61X_LinMessage_T@@@@PAX@2@I@Z 10077a30 f i IO61X_Library_MSVC120_vc:IO61X_LinPort.obj
 0001:00076a50       ?deallocate@?$allocator@V?$_List_unchecked_iterator@V?$_List_val@U?$_List_simple_types@U?$pair@$$CBHV?$IO61X_BufferFifo@UIO61X_LinMessage_T@@@@@std@@@std@@@std@@@std@@@std@@QAEXPAV?$_List_unchecked_iterator@V?$_List_val@U?$_List_simple_types@U?$pair@$$CBHV?$IO61X_BufferFifo@UIO61X_LinMessage_T@@@@@std@@@std@@@std@@@2@I@Z 10077a50 f i IO61X_Library_MSVC120_vc:IO61X_LinPort.obj
 0001:00076a70       ?empty@?$_Hash@V?$_Umap_traits@HV?$IO61X_BufferFifo@UIO61X_LinMessage_T@@@@V?$_Uhash_compare@HU?$hash@H@std@@U?$equal_to@H@2@@std@@V?$allocator@U?$pair@$$CBHV?$IO61X_BufferFifo@UIO61X_LinMessage_T@@@@@std@@@3@$0A@@std@@@std@@QBE_NXZ 10077a70 f i IO61X_Library_MSVC120_vc:IO61X_LinPort.obj
 0001:00076a80       ?empty@?$list@U?$pair@$$CBHV?$IO61X_BufferFifo@UIO61X_LinMessage_T@@@@@std@@V?$allocator@U?$pair@$$CBHV?$IO61X_BufferFifo@UIO61X_LinMessage_T@@@@@std@@@2@@std@@QBE_NXZ 10077a80 f i IO61X_Library_MSVC120_vc:IO61X_LinPort.obj
 0001:00076a90       ?empty@?$list@V?$IO61X_BufferFifo@UIO61X_LinMessage_T@@@@V?$allocator@V?$IO61X_BufferFifo@UIO61X_LinMessage_T@@@@@std@@@std@@QBE_NXZ 10077a90 f i IO61X_Library_MSVC120_vc:IO61X_LinPort.obj
 0001:00076aa0       ?end@?$_Hash@V?$_Umap_traits@HV?$IO61X_BufferFifo@UIO61X_LinMessage_T@@@@V?$_Uhash_compare@HU?$hash@H@std@@U?$equal_to@H@2@@std@@V?$allocator@U?$pair@$$CBHV?$IO61X_BufferFifo@UIO61X_LinMessage_T@@@@@std@@@3@$0A@@std@@@std@@QAE?AV?$_List_iterator@V?$_List_val@U?$_List_simple_types@U?$pair@$$CBHV?$IO61X_BufferFifo@UIO61X_LinMessage_T@@@@@std@@@std@@@std@@@2@XZ 10077aa0 f i IO61X_Library_MSVC120_vc:IO61X_LinPort.obj
 0001:00076ab0       ?end@?$list@U?$pair@$$CBHV?$IO61X_BufferFifo@UIO61X_LinMessage_T@@@@@std@@V?$allocator@U?$pair@$$CBHV?$IO61X_BufferFifo@UIO61X_LinMessage_T@@@@@std@@@2@@std@@QAE?AV?$_List_iterator@V?$_List_val@U?$_List_simple_types@U?$pair@$$CBHV?$IO61X_BufferFifo@UIO61X_LinMessage_T@@@@@std@@@std@@@std@@@2@XZ 10077ab0 f i IO61X_Library_MSVC120_vc:IO61X_LinPort.obj
 0001:00076ac0       ?end@?$list@V?$IO61X_BufferFifo@UIO61X_LinMessage_T@@@@V?$allocator@V?$IO61X_BufferFifo@UIO61X_LinMessage_T@@@@@std@@@std@@QAE?AV?$_List_iterator@V?$_List_val@U?$_List_simple_types@V?$IO61X_BufferFifo@UIO61X_LinMessage_T@@@@@std@@@std@@@2@XZ 10077ac0 f i IO61X_Library_MSVC120_vc:IO61X_LinPort.obj
 0001:00076ad0       ?erase@?$list@U?$pair@$$CBHV?$IO61X_BufferFifo@UIO61X_LinMessage_T@@@@@std@@V?$allocator@U?$pair@$$CBHV?$IO61X_BufferFifo@UIO61X_LinMessage_T@@@@@std@@@2@@std@@QAE?AV?$_List_iterator@V?$_List_val@U?$_List_simple_types@U?$pair@$$CBHV?$IO61X_BufferFifo@UIO61X_LinMessage_T@@@@@std@@@std@@@std@@@2@V?$_List_const_iterator@V?$_List_val@U?$_List_simple_types@U?$pair@$$CBHV?$IO61X_BufferFifo@UIO61X_LinMessage_T@@@@@std@@@std@@@std@@@2@@Z 10077ad0 f i IO61X_Library_MSVC120_vc:IO61X_LinPort.obj
 0001:00076b20       ?find@?$_Hash@V?$_Umap_traits@HV?$IO61X_BufferFifo@UIO61X_LinMessage_T@@@@V?$_Uhash_compare@HU?$hash@H@std@@U?$equal_to@H@2@@std@@V?$allocator@U?$pair@$$CBHV?$IO61X_BufferFifo@UIO61X_LinMessage_T@@@@@std@@@3@$0A@@std@@@std@@QAE?AV?$_List_iterator@V?$_List_val@U?$_List_simple_types@U?$pair@$$CBHV?$IO61X_BufferFifo@UIO61X_LinMessage_T@@@@@std@@@std@@@std@@@2@ABH@Z 10077b20 f i IO61X_Library_MSVC120_vc:IO61X_LinPort.obj
 0001:00076b40       ?front@?$list@U?$pair@$$CBHV?$IO61X_BufferFifo@UIO61X_LinMessage_T@@@@@std@@V?$allocator@U?$pair@$$CBHV?$IO61X_BufferFifo@UIO61X_LinMessage_T@@@@@std@@@2@@std@@QAEAAU?$pair@$$CBHV?$IO61X_BufferFifo@UIO61X_LinMessage_T@@@@@2@XZ 10077b40 f i IO61X_Library_MSVC120_vc:IO61X_LinPort.obj
 0001:00076b50       ?getReadIdx@?$IO61X_BufferFifo@UIO61X_LinMessage_T@@@@QAEHXZ 10077b50 f i IO61X_Library_MSVC120_vc:IO61X_LinPort.obj
 0001:00076b60       ?getWriteIdx@?$IO61X_BufferFifo@UIO61X_LinMessage_T@@@@QAEHXZ 10077b60 f i IO61X_Library_MSVC120_vc:IO61X_LinPort.obj
 0001:00076b70       ?insert@?$vector@V?$_List_unchecked_iterator@V?$_List_val@U?$_List_simple_types@U?$pair@$$CBHV?$IO61X_BufferFifo@UIO61X_LinMessage_T@@@@@std@@@std@@@std@@@std@@U?$_Wrap_alloc@V?$allocator@V?$_List_unchecked_iterator@V?$_List_val@U?$_List_simple_types@U?$pair@$$CBHV?$IO61X_BufferFifo@UIO61X_LinMessage_T@@@@@std@@@std@@@std@@@std@@@std@@@2@@std@@QAE?AV?$_Vector_iterator@V?$_Vector_val@U?$_Simple_types@V?$_List_unchecked_iterator@V?$_List_val@U?$_List_simple_types@U?$pair@$$CBHV?$IO61X_BufferFifo@UIO61X_LinMessage_T@@@@@std@@@std@@@std@@@std@@@std@@@std@@@2@V?$_Vector_const_iterator@V?$_Vector_val@U?$_Simple_types@V?$_List_unchecked_iterator@V?$_List_val@U?$_List_simple_types@U?$pair@$$CBHV?$IO61X_BufferFifo@UIO61X_LinMessage_T@@@@@std@@@std@@@std@@@std@@@std@@@std@@@2@IABV?$_List_unchecked_iterator@V?$_List_val@U?$_List_simple_types@U?$pair@$$CBHV?$IO61X_BufferFifo@UIO61X_LinMessage_T@@@@@std@@@std@@@std@@@2@@Z 10077b70 f i IO61X_Library_MSVC120_vc:IO61X_LinPort.obj
 0001:00076b90       ?load_factor@?$_Hash@V?$_Umap_traits@HV?$IO61X_BufferFifo@UIO61X_LinMessage_T@@@@V?$_Uhash_compare@HU?$hash@H@std@@U?$equal_to@H@2@@std@@V?$allocator@U?$pair@$$CBHV?$IO61X_BufferFifo@UIO61X_LinMessage_T@@@@@std@@@3@$0A@@std@@@std@@QBEMXZ 10077b90 f i IO61X_Library_MSVC120_vc:IO61X_LinPort.obj
 0001:00076be0       ?lower_bound@?$_Hash@V?$_Umap_traits@HV?$IO61X_BufferFifo@UIO61X_LinMessage_T@@@@V?$_Uhash_compare@HU?$hash@H@std@@U?$equal_to@H@2@@std@@V?$allocator@U?$pair@$$CBHV?$IO61X_BufferFifo@UIO61X_LinMessage_T@@@@@std@@@3@$0A@@std@@@std@@QAE?AV?$_List_iterator@V?$_List_val@U?$_List_simple_types@U?$pair@$$CBHV?$IO61X_BufferFifo@UIO61X_LinMessage_T@@@@@std@@@std@@@std@@@2@ABH@Z 10077be0 f i IO61X_Library_MSVC120_vc:IO61X_LinPort.obj
 0001:00076c90       ?max_load_factor@?$_Hash@V?$_Umap_traits@HV?$IO61X_BufferFifo@UIO61X_LinMessage_T@@@@V?$_Uhash_compare@HU?$hash@H@std@@U?$equal_to@H@2@@std@@V?$allocator@U?$pair@$$CBHV?$IO61X_BufferFifo@UIO61X_LinMessage_T@@@@@std@@@3@$0A@@std@@@std@@QBEMXZ 10077c90 f i IO61X_Library_MSVC120_vc:IO61X_LinPort.obj
 0001:00076ca0       ?max_size@?$_Wrap_alloc@U?$_Wrap_alloc@V?$allocator@V?$_List_unchecked_iterator@V?$_List_val@U?$_List_simple_types@U?$pair@$$CBHV?$IO61X_BufferFifo@UIO61X_LinMessage_T@@@@@std@@@std@@@std@@@std@@@std@@@std@@@std@@QBEIXZ 10077ca0 f i IO61X_Library_MSVC120_vc:IO61X_LinPort.obj
 0001:00076cb0       ?max_size@?$_Wrap_alloc@V?$allocator@U?$_List_node@U?$pair@$$CBHV?$IO61X_BufferFifo@UIO61X_LinMessage_T@@@@@std@@PAX@std@@@std@@@std@@QBEIXZ 10077cb0 f i IO61X_Library_MSVC120_vc:IO61X_LinPort.obj
 0001:00076cc0       ?max_size@?$_Wrap_alloc@V?$allocator@U?$_List_node@V?$IO61X_BufferFifo@UIO61X_LinMessage_T@@@@PAX@std@@@std@@@std@@QBEIXZ 10077cc0 f i IO61X_Library_MSVC120_vc:IO61X_LinPort.obj
 0001:00076cd0       ?max_size@?$_Wrap_alloc@V?$allocator@V?$_List_unchecked_iterator@V?$_List_val@U?$_List_simple_types@U?$pair@$$CBHV?$IO61X_BufferFifo@UIO61X_LinMessage_T@@@@@std@@@std@@@std@@@std@@@std@@@std@@QBEIXZ 10077cd0 f i IO61X_Library_MSVC120_vc:IO61X_LinPort.obj
 0001:00076ce0       ?max_size@?$allocator@U?$_List_node@U?$pair@$$CBHV?$IO61X_BufferFifo@UIO61X_LinMessage_T@@@@@std@@PAX@std@@@std@@QBEIXZ 10077ce0 f i IO61X_Library_MSVC120_vc:IO61X_LinPort.obj
 0001:00076cf0       ?max_size@?$allocator@U?$_List_node@V?$IO61X_BufferFifo@UIO61X_LinMessage_T@@@@PAX@std@@@std@@QBEIXZ 10077cf0 f i IO61X_Library_MSVC120_vc:IO61X_LinPort.obj
 0001:00076d00       ?max_size@?$allocator@V?$_List_unchecked_iterator@V?$_List_val@U?$_List_simple_types@U?$pair@$$CBHV?$IO61X_BufferFifo@UIO61X_LinMessage_T@@@@@std@@@std@@@std@@@std@@@std@@QBEIXZ 10077d00 f i IO61X_Library_MSVC120_vc:IO61X_LinPort.obj
 0001:00076d10       ?max_size@?$allocator_traits@U?$_Wrap_alloc@V?$allocator@V?$_List_unchecked_iterator@V?$_List_val@U?$_List_simple_types@U?$pair@$$CBHV?$IO61X_BufferFifo@UIO61X_LinMessage_T@@@@@std@@@std@@@std@@@std@@@std@@@std@@@std@@SAIABU?$_Wrap_alloc@V?$allocator@V?$_List_unchecked_iterator@V?$_List_val@U?$_List_simple_types@U?$pair@$$CBHV?$IO61X_BufferFifo@UIO61X_LinMessage_T@@@@@std@@@std@@@std@@@std@@@std@@@2@@Z 10077d10 f i IO61X_Library_MSVC120_vc:IO61X_LinPort.obj
 0001:00076d20       ?max_size@?$allocator_traits@V?$allocator@U?$_List_node@U?$pair@$$CBHV?$IO61X_BufferFifo@UIO61X_LinMessage_T@@@@@std@@PAX@std@@@std@@@std@@SAIABV?$allocator@U?$_List_node@U?$pair@$$CBHV?$IO61X_BufferFifo@UIO61X_LinMessage_T@@@@@std@@PAX@std@@@2@@Z 10077d20 f i IO61X_Library_MSVC120_vc:IO61X_LinPort.obj
 0001:00076d30       ?max_size@?$allocator_traits@V?$allocator@U?$_List_node@V?$IO61X_BufferFifo@UIO61X_LinMessage_T@@@@PAX@std@@@std@@@std@@SAIABV?$allocator@U?$_List_node@V?$IO61X_BufferFifo@UIO61X_LinMessage_T@@@@PAX@std@@@2@@Z 10077d30 f i IO61X_Library_MSVC120_vc:IO61X_LinPort.obj
 0001:00076d40       ?max_size@?$allocator_traits@V?$allocator@V?$_List_unchecked_iterator@V?$_List_val@U?$_List_simple_types@U?$pair@$$CBHV?$IO61X_BufferFifo@UIO61X_LinMessage_T@@@@@std@@@std@@@std@@@std@@@std@@@std@@SAIABV?$allocator@V?$_List_unchecked_iterator@V?$_List_val@U?$_List_simple_types@U?$pair@$$CBHV?$IO61X_BufferFifo@UIO61X_LinMessage_T@@@@@std@@@std@@@std@@@std@@@2@@Z 10077d40 f i IO61X_Library_MSVC120_vc:IO61X_LinPort.obj
 0001:00076d50       ?max_size@?$list@U?$pair@$$CBHV?$IO61X_BufferFifo@UIO61X_LinMessage_T@@@@@std@@V?$allocator@U?$pair@$$CBHV?$IO61X_BufferFifo@UIO61X_LinMessage_T@@@@@std@@@2@@std@@QBEIXZ 10077d50 f i IO61X_Library_MSVC120_vc:IO61X_LinPort.obj
 0001:00076d60       ?max_size@?$list@V?$IO61X_BufferFifo@UIO61X_LinMessage_T@@@@V?$allocator@V?$IO61X_BufferFifo@UIO61X_LinMessage_T@@@@@std@@@std@@QBEIXZ 10077d60 f i IO61X_Library_MSVC120_vc:IO61X_LinPort.obj
 0001:00076d70       ?max_size@?$vector@V?$_List_unchecked_iterator@V?$_List_val@U?$_List_simple_types@U?$pair@$$CBHV?$IO61X_BufferFifo@UIO61X_LinMessage_T@@@@@std@@@std@@@std@@@std@@U?$_Wrap_alloc@V?$allocator@V?$_List_unchecked_iterator@V?$_List_val@U?$_List_simple_types@U?$pair@$$CBHV?$IO61X_BufferFifo@UIO61X_LinMessage_T@@@@@std@@@std@@@std@@@std@@@std@@@2@@std@@QBEIXZ 10077d70 f i IO61X_Library_MSVC120_vc:IO61X_LinPort.obj
 0001:00076d80       ?pointer_to@?$pointer_traits@PAU?$pair@$$CBHV?$IO61X_BufferFifo@UIO61X_LinMessage_T@@@@@std@@@std@@SAPAU?$pair@$$CBHV?$IO61X_BufferFifo@UIO61X_LinMessage_T@@@@@2@AAU32@@Z 10077d80 f i IO61X_Library_MSVC120_vc:IO61X_LinPort.obj
 0001:00076d90       ?push_back@?$list@V?$IO61X_BufferFifo@UIO61X_LinMessage_T@@@@V?$allocator@V?$IO61X_BufferFifo@UIO61X_LinMessage_T@@@@@std@@@std@@QAEX$$QAV?$IO61X_BufferFifo@UIO61X_LinMessage_T@@@@@Z 10077d90 f i IO61X_Library_MSVC120_vc:IO61X_LinPort.obj
 0001:00076de0       ?setReadIdx@?$IO61X_BufferFifo@UIO61X_LinMessage_T@@@@QAEXH@Z 10077de0 f i IO61X_Library_MSVC120_vc:IO61X_LinPort.obj
 0001:00076df0       ?setWriteIdx@?$IO61X_BufferFifo@UIO61X_LinMessage_T@@@@QAEXH@Z 10077df0 f i IO61X_Library_MSVC120_vc:IO61X_LinPort.obj
 0001:00076e00       ?size@?$_Hash@V?$_Umap_traits@HV?$IO61X_BufferFifo@UIO61X_LinMessage_T@@@@V?$_Uhash_compare@HU?$hash@H@std@@U?$equal_to@H@2@@std@@V?$allocator@U?$pair@$$CBHV?$IO61X_BufferFifo@UIO61X_LinMessage_T@@@@@std@@@3@$0A@@std@@@std@@QBEIXZ 10077e00 f i IO61X_Library_MSVC120_vc:IO61X_LinPort.obj
 0001:00076e10       ?size@?$list@U?$pair@$$CBHV?$IO61X_BufferFifo@UIO61X_LinMessage_T@@@@@std@@V?$allocator@U?$pair@$$CBHV?$IO61X_BufferFifo@UIO61X_LinMessage_T@@@@@std@@@2@@std@@QBEIXZ 10077e10 f i IO61X_Library_MSVC120_vc:IO61X_LinPort.obj
 0001:00076e20       ?size@?$list@V?$IO61X_BufferFifo@UIO61X_LinMessage_T@@@@V?$allocator@V?$IO61X_BufferFifo@UIO61X_LinMessage_T@@@@@std@@@std@@QBEIXZ 10077e20 f i IO61X_Library_MSVC120_vc:IO61X_LinPort.obj
 0001:00076e30       ?size@?$vector@V?$_List_unchecked_iterator@V?$_List_val@U?$_List_simple_types@U?$pair@$$CBHV?$IO61X_BufferFifo@UIO61X_LinMessage_T@@@@@std@@@std@@@std@@@std@@U?$_Wrap_alloc@V?$allocator@V?$_List_unchecked_iterator@V?$_List_val@U?$_List_simple_types@U?$pair@$$CBHV?$IO61X_BufferFifo@UIO61X_LinMessage_T@@@@@std@@@std@@@std@@@std@@@std@@@2@@std@@QBEIXZ 10077e30 f i IO61X_Library_MSVC120_vc:IO61X_LinPort.obj
 0001:00076e40       ?waitForSemaphore@@YAHPAXN@Z 10077e40 f   IO61X_Library_MSVC120_vc:SlrtOSManagement.obj
 0001:00076e70       ?IO61X_DoesFileExist@@YA_NPBD@Z 10077e70 f   IO61X_Library_MSVC120_vc:IO61X_CommonManager.obj
 0001:00076ea0       ?IO61X_GetFwFileName@@YA_NPBDPAD@Z 10077ea0 f   IO61X_Library_MSVC120_vc:IO61X_CommonManager.obj
 0001:00076ec0       ?IO61X_GetFwInfoValues@@YA_NPBDPAD11@Z 10077ec0 f   IO61X_Library_MSVC120_vc:IO61X_CommonManager.obj
 0001:00076fe0       ?IO61X_GetPciValues@@YA_NPBDPAUPciDeviceStruct@@@Z 10077fe0 f   IO61X_Library_MSVC120_vc:IO61X_CommonManager.obj
 0001:00077110       ?IO61X_VerifyMailboxTag@@YA_NII@Z 10078110 f   IO61X_Library_MSVC120_vc:IO61X_CommonManager.obj
 0001:00077140       ?IO61X_ReceiveConfigurationPacket_new@@YA_NPBUIO61X_PciObject_T@@IIGIPAX@Z 10078140 f   IO61X_Library_MSVC120_vc:IO61X_CommunicationManager.obj
 0001:00077330       ?IO61X_SendConfigurationPacket@@YA_NPBUIO61X_PciObject_T@@PAUIO61X_CommonRequestPacket_T@@@Z 10078330 f   IO61X_Library_MSVC120_vc:IO61X_CommunicationManager.obj
 0001:000773d0       __heap_alloc               100783d0 f i LIBCMT:malloc.obj
 0001:0007740d       _malloc                    1007840d f   LIBCMT:malloc.obj
 0001:0007749f       _free                      1007849f f   LIBCMT:free.obj
 0001:000774d7       __fpmath                   100784d7 f   LIBCMT:fpinit.obj
 0001:000774ee       ___setfflag                100784ee f   LIBCMT:fpinit.obj
 0001:00077501       __cfltcvt_init             10078501 f   LIBCMT:fpinit.obj
 0001:00077561       _calloc                    10078561 f   LIBCMT:calloc.obj
 0001:000775b0       __ftoui3                   100785b0 f   LIBCMT:ftol3.obj
 0001:000775bf       __ftoul3                   100785bf f   LIBCMT:ftol3.obj
 0001:000775ce       __ftol3                    100785ce f   LIBCMT:ftol3.obj
 0001:000775db       __ftol3_NaN                100785db f   LIBCMT:ftol3.obj
 0001:000775f3       __ftol3_work               100785f3 f   LIBCMT:ftol3.obj
 0001:00077679       __ftol3_common             10078679 f   LIBCMT:ftol3.obj
 0001:0007773b       __ftol3_arg_error          1007873b f   LIBCMT:ftol3.obj
 0001:0007774d       __ftol3_except             1007874d f   LIBCMT:ftol3.obj
 0001:0007778f       __dtoui3                   1007878f f   LIBCMT:ftol3.obj
 0001:0007779e       __dtoul3                   1007879e f   LIBCMT:ftol3.obj
 0001:000777ad       __dtol3                    100787ad f   LIBCMT:ftol3.obj
 0001:000777ba       __dtol3_NaN                100787ba f   LIBCMT:ftol3.obj
 0001:000777d7       __dtol3_work               100787d7 f   LIBCMT:ftol3.obj
 0001:000778bc       __ultod3                   100788bc f   LIBCMT:ftol3.obj
 0001:0007794d       __ltod3                    1007894d f   LIBCMT:ftol3.obj
 0001:00077980       _memcpy                    10078980 f   LIBCMT:memcpy.obj
 0001:00077fc4       ___raise_securityfailure   10078fc4 f   LIBCMT:gs_report.obj
 0001:00078001       ___report_gsfailure        10079001 f   LIBCMT:gs_report.obj
 0001:000780fc       ___report_rangecheckfailure 100790fc f   LIBCMT:gs_report.obj
 0001:00078108       ___report_securityfailure  10079108 f   LIBCMT:gs_report.obj
 0001:000781d8       ___report_securityfailureEx 100791d8 f   LIBCMT:gs_report.obj
 0001:000782ee       ___copy_path_to_wide_string 100792ee f   LIBCMT:crt0dat.obj
 0001:000783a0       ___copy_to_char            100793a0 f   LIBCMT:crt0dat.obj
 0001:00078455       ___crtCorExitProcess       10079455 f   LIBCMT:crt0dat.obj
 0001:00078489       ___crtExitProcess          10079489 f   LIBCMT:crt0dat.obj
 0001:0007849f       ___freeCrtMemory           1007949f f   LIBCMT:crt0dat.obj
 0001:000785ac       __amsg_exit                100795ac f   LIBCMT:crt0dat.obj
 0001:000785c8       __c_exit                   100795c8 f   LIBCMT:crt0dat.obj
 0001:000785d7       __cexit                    100795d7 f   LIBCMT:crt0dat.obj
 0001:000785e6       __cinit                    100795e6 f   LIBCMT:crt0dat.obj
 0001:0007866a       __exit                     1007966a f   LIBCMT:crt0dat.obj
 0001:0007867e       __exit_app                 1007967e f   LIBCMT:crt0dat.obj
 0001:0007868c       __get_pgmptr               1007968c f   LIBCMT:crt0dat.obj
 0001:000786bb       __get_wpgmptr              100796bb f   LIBCMT:crt0dat.obj
 0001:000786ea       __init_pointers            100796ea f   LIBCMT:crt0dat.obj
 0001:00078758       __initterm_e               10079758 f   LIBCMT:crt0dat.obj
 0001:0007877a       __lockexit                 1007977a f   LIBCMT:crt0dat.obj
 0001:00078783       __unlockexit               10079783 f   LIBCMT:crt0dat.obj
 0001:000788bb       _exit                      100798bb f   LIBCMT:crt0dat.obj
 0001:000788cf       _realloc                   100798cf f   LIBCMT:realloc.obj
 0001:00078980       _memmove                   10079980 f   LIBCMT:memmove.obj
 0001:00078fd0       _strchr                    10079fd0 f   LIBCMT:strchr.obj
 0001:0007903e       ___from_strstr_to_strchr   1007a03e     LIBCMT:strchr.obj
 0001:00079100       _strncat                   1007a100 f   LIBCMT:strncat.obj
 0001:00079240       _strncpy                   1007a240 f   LIBCMT:strncpy.obj
 0001:00079364       ___initstdio               1007a364 f   LIBCMT:_file.obj
 0001:000793d7       ___endstdio                1007a3d7 f   LIBCMT:_file.obj
 0001:000793fe       ___iob_func                1007a3fe f   LIBCMT:_file.obj
 0001:00079404       __lock_file                1007a404 f   LIBCMT:_file.obj
 0001:00079443       __lock_file2               1007a443 f   LIBCMT:_file.obj
 0001:00079473       __unlock_file              1007a473 f   LIBCMT:_file.obj
 0001:000794ad       __unlock_file2             1007a4ad f   LIBCMT:_file.obj
 0001:000794da       __fclose_nolock            1007a4da f   LIBCMT:fclose.obj
 0001:00079546       _fclose                    1007a546 f   LIBCMT:fclose.obj
 0001:000795bd       __fsopen                   1007a5bd f   LIBCMT:fopen.obj
 0001:00079681       _fopen                     1007a681 f   LIBCMT:fopen.obj
 0001:00079696       _fopen_s                   1007a696 f   LIBCMT:fopen.obj
 0001:000796db       __fprintf_l                1007a6db f   LIBCMT:fprintf.obj
 0001:000796f5       __fprintf_p                1007a6f5 f   LIBCMT:fprintf.obj
 0001:0007970e       __fprintf_p_l              1007a70e f   LIBCMT:fprintf.obj
 0001:00079728       __fprintf_s_l              1007a728 f   LIBCMT:fprintf.obj
 0001:00079742       _fprintf                   1007a742 f   LIBCMT:fprintf.obj
 0001:00079854       _fprintf_s                 1007a854 f   LIBCMT:fprintf.obj
 0001:0007986d       __fread_nolock             1007a86d f   LIBCMT:fread.obj
 0001:00079888       __fread_nolock_s           1007a888 f   LIBCMT:fread.obj
 0001:00079a4d       _fread                     1007aa4d f   LIBCMT:fread.obj
 0001:00079a68       _fread_s                   1007aa68 f   LIBCMT:fread.obj
 0001:00079af9       __fwrite_nolock            1007aaf9 f   LIBCMT:fwrite.obj
 0001:00079c52       _fwrite                    1007ac52 f   LIBCMT:fwrite.obj
 0001:00079cd4       __get_printf_count_output  1007acd4 f   LIBCMT:printf.obj
 0001:00079ce9       __printf_l                 1007ace9 f   LIBCMT:printf.obj
 0001:00079d00       __printf_p                 1007ad00 f   LIBCMT:printf.obj
 0001:00079d16       __printf_p_l               1007ad16 f   LIBCMT:printf.obj
 0001:00079d2d       __printf_s_l               1007ad2d f   LIBCMT:printf.obj
 0001:00079d44       __set_printf_count_output  1007ad44 f   LIBCMT:printf.obj
 0001:00079d6c       _printf                    1007ad6c f   LIBCMT:printf.obj
 0001:00079e1b       _printf_s                  1007ae1b f   LIBCMT:printf.obj
 0001:00079e31       __unlink                   1007ae31 f   LIBCMT:unlink.obj
 0001:00079e3a       _remove                    1007ae3a f   LIBCMT:unlink.obj
 0001:00079e7c       _rewind                    1007ae7c f   LIBCMT:rewind.obj
 0001:00079f3b       __scprintf                 1007af3b f   LIBCMT:sprintf.obj
 0001:00079f4e       __scprintf_l               1007af4e f   LIBCMT:sprintf.obj
 0001:00079f65       __scprintf_p               1007af65 f   LIBCMT:sprintf.obj
 0001:00079f78       __scprintf_p_l             1007af78 f   LIBCMT:sprintf.obj
 0001:00079f8f       __snprintf_s               1007af8f f   LIBCMT:sprintf.obj
 0001:00079fae       __snprintf_s_l             1007afae f   LIBCMT:sprintf.obj
 0001:00079fce       __sprintf_l                1007afce f   LIBCMT:sprintf.obj
 0001:00079fe8       __sprintf_p                1007afe8 f   LIBCMT:sprintf.obj
 0001:0007a004       __sprintf_p_l              1007b004 f   LIBCMT:sprintf.obj
 0001:0007a021       __sprintf_s_l              1007b021 f   LIBCMT:sprintf.obj
 0001:0007a03e       _sprintf                   1007b03e f   LIBCMT:sprintf.obj
 0001:0007a0c2       _sprintf_s                 1007b0c2 f   LIBCMT:sprintf.obj
 0001:0007a0de       _ldexp                     1007b0de f   LIBCMT:ldexp.obj
 0001:0007a2ca       @__security_check_cookie@4 1007b2ca f   LIBCMT:secchk.obj
 0001:0007a2e0       _memset                    1007b2e0 f   LIBCMT:memset.obj
 0001:0007a370       ___isa_available_init      1007b370 f   LIBCMT:cpu_disp.obj
 0001:0007a4e9       __invoke_watson_if_error   1007b4e9 f i LIBCMT:wassert.obj
 0001:0007a509       __wassert                  1007b509 f   LIBCMT:wassert.obj
 0001:0007abad       __CRT_INIT@12              1007bbad f   LIBCMT:dllcrt0.obj
 0001:0007ad1f       __DllMainCRTStartup@12     1007bd1f f   LIBCMT:dllcrt0.obj
 0001:0007ae50       ___DllXcptFilter           1007be50 f   LIBCMT:dllcrt0.obj
 0001:0007ae75       __get_purecall_handler     1007be75 f   LIBCMT:purevirt.obj
 0001:0007ae82       __purecall                 1007be82 f   LIBCMT:purevirt.obj
 0001:0007aea4       __set_purecall_handler     1007bea4 f   LIBCMT:purevirt.obj
 0001:0007aec9       ??0bad_alloc@std@@QAE@ABV01@@Z 1007bec9 f i LIBCMT:new.obj
 0001:0007aee4       ??0bad_alloc@std@@QAE@XZ   1007bee4 f i LIBCMT:new.obj
 0001:0007af0a       ??1bad_alloc@std@@UAE@XZ   1007bf0a f i LIBCMT:new.obj
 0001:0007af15       ??2@YAPAXI@Z               1007bf15 f   LIBCMT:new.obj
 0001:0007af66       ??_Gbad_alloc@std@@UAEPAXI@Z 1007bf66 f i LIBCMT:new.obj
 0001:0007af66       ??_Ebad_alloc@std@@UAEPAXI@Z 1007bf66 f i LIBCMT:new.obj
 0001:0007af8b       ??3@YAXPAX@Z               1007bf8b f   LIBCMT:delete.obj
 0001:0007af90       ___onexitinit              1007bf90 f   LIBCMT:onexit.obj
 0001:0007afbf       __onexit                   1007bfbf f   LIBCMT:onexit.obj
 0001:0007b0bb       _atexit                    1007c0bb f   LIBCMT:onexit.obj
 0001:0007b0d0       __cabs                     1007c0d0 f   LIBCMT:hypot.obj
 0001:0007b0ef       __hypot                    1007c0ef f   LIBCMT:hypot.obj
 0001:0007b35a       __CxxThrowException@8      1007c35a f   LIBCMT:throw.obj
 0001:0007b48d       ?_CallCatchBlock2@@YAPAXPAUEHRegistrationNode@@PBU_s_FuncInfo@@PAXHK@Z 1007c48d f   LIBCMT:_trnsctrl_.obj
 0001:0007b4ed       ?_CallMemberFunction0@@YGXPAX0@Z 1007c4ed f   LIBCMT:_trnsctrl_.obj
 0001:0007b4f4       ?_CallMemberFunction1@@YGXPAX00@Z 1007c4f4 f   LIBCMT:_trnsctrl_.obj
 0001:0007b4fb       ?_CallMemberFunction2@@YGXPAX00H@Z 1007c4fb f   LIBCMT:_trnsctrl_.obj
 0001:0007b502       ?_CallSETranslator@@YAHPAUEHExceptionRecord@@PAUEHRegistrationNode@@PAX2PBU_s_FuncInfo@@H1@Z 1007c502 f   LIBCMT:_trnsctrl_.obj
 0001:0007b5d9       ?_GetRangeOfTrysToCheck@@YAPBU_s_TryBlockMapEntry@@PBU_s_FuncInfo@@HHPAI1@Z 1007c5d9 f   LIBCMT:_trnsctrl_.obj
 0001:0007b657       ?_JumpToContinuation@@YGXPAXPAUEHRegistrationNode@@@Z 1007c657 f   LIBCMT:_trnsctrl_.obj
 0001:0007b689       ?_UnwindNestedFrames@@YGXPAUEHRegistrationNode@@PAUEHExceptionRecord@@@Z 1007c689 f   LIBCMT:_trnsctrl_.obj
 0001:0007b6de       __CreateFrameInfo          1007c6de f   LIBCMT:_trnsctrl_.obj
 0001:0007b708       __FindAndUnlinkFrame       1007c708 f   LIBCMT:_trnsctrl_.obj
 0001:0007b758       __IsExceptionObjectToBeDestroyed 1007c758 f   LIBCMT:_trnsctrl_.obj
 0001:0007b781       ___CxxFrameHandler         1007c781 f   LIBCMT:_trnsctrl_.obj
 0001:0007b7b7       ___CxxFrameHandler2        1007c7b7 f   LIBCMT:_trnsctrl_.obj
 0001:0007b7ed       ___CxxFrameHandler3        1007c7ed f   LIBCMT:_trnsctrl_.obj
 0001:0007b823       ___CxxLongjmpUnwind@4      1007c823 f   LIBCMT:_trnsctrl_.obj
 0001:0007b840       ??0type_info@@AAE@ABV0@@Z  1007c840 f   LIBCMT:typinfo.obj
 0001:0007b84b       ??1type_info@@UAE@XZ       1007c84b f   LIBCMT:typinfo.obj
 0001:0007b859       ??4type_info@@AAEAAV0@ABV0@@Z 1007c859 f   LIBCMT:typinfo.obj
 0001:0007b85e       ??8type_info@@QBE_NABV0@@Z 1007c85e f   LIBCMT:typinfo.obj
 0001:0007b87c       ??9type_info@@QBE_NABV0@@Z 1007c87c f   LIBCMT:typinfo.obj
 0001:0007b89b       ??_Etype_info@@UAEPAXI@Z   1007c89b f i LIBCMT:typinfo.obj
 0001:0007b89b       ??_Gtype_info@@UAEPAXI@Z   1007c89b f i LIBCMT:typinfo.obj
 0001:0007b8ba       ?_name_internal_method@type_info@@QBEPBDPAU__type_info_node@@@Z 1007c8ba f   LIBCMT:typinfo.obj
 0001:0007b8cc       ?_type_info_dtor_internal_method@type_info@@QAEXXZ 1007c8cc f   LIBCMT:typinfo.obj
 0001:0007b8d4       ?before@type_info@@QBE_NABV1@@Z 1007c8d4 f   LIBCMT:typinfo.obj
 0001:0007b8f4       ?name@type_info@@QBEPBDPAU__type_info_node@@@Z 1007c8f4 f   LIBCMT:typinfo.obj
 0001:0007b906       ?raw_name@type_info@@QBEPBDXZ 1007c906 f   LIBCMT:typinfo.obj
 0001:0007b90a       __fflush_nolock            1007c90a f   LIBCMT:fflush.obj
 0001:0007b950       __flush                    1007c950 f   LIBCMT:fflush.obj
 0001:0007b9b4       __flushall                 1007c9b4 f   LIBCMT:fflush.obj
 0001:0007b9bd       _fflush                    1007c9bd f   LIBCMT:fflush.obj
 0001:0007bafa       __getc_nolock              1007cafa f   LIBCMT:fgetc.obj
 0001:0007bb1c       _fgetc                     1007cb1c f   LIBCMT:fgetc.obj
 0001:0007bc15       _getc                      1007cc15 f   LIBCMT:fgetc.obj
 0001:0007bd0e       _fgetpos                   1007cd0e f   LIBCMT:fgetpos.obj
 0001:0007bd63       _fputc                     1007cd63 f   LIBCMT:fputc.obj
 0001:0007be64       _putc                      1007ce64 f   LIBCMT:fputc.obj
 0001:0007bf65       _fsetpos                   1007cf65 f   LIBCMT:fsetpos.obj
 0001:0007bf9e       __fseeki64                 1007cf9e f   LIBCMT:fseeki64.obj
 0001:0007c024       __fseeki64_nolock          1007d024 f   LIBCMT:fseeki64.obj
 0001:0007c0d5       _setvbuf                   1007d0d5 f   LIBCMT:setvbuf.obj
 0001:0007c1db       __ungetc_nolock            1007d1db f   LIBCMT:ungetc.obj
 0001:0007c2bb       _ungetc                    1007d2bb f   LIBCMT:ungetc.obj
 0001:0007c32b       __snprintf                 1007d32b f   LIBCMT:snprintf.obj
 0001:0007c3d7       __snprintf_l               1007d3d7 f   LIBCMT:snprintf.obj
 0001:0007c3f4       __vscprintf                1007d3f4 f   LIBCMT:vsprintf.obj
 0001:0007c40e       __vscprintf_helper         1007d40e f   LIBCMT:vsprintf.obj
 0001:0007c46a       __vscprintf_l              1007d46a f   LIBCMT:vsprintf.obj
 0001:0007c485       __vscprintf_p              1007d485 f   LIBCMT:vsprintf.obj
 0001:0007c49f       __vscprintf_p_l            1007d49f f   LIBCMT:vsprintf.obj
 0001:0007c4ba       __vsprintf_l               1007d4ba f   LIBCMT:vsprintf.obj
 0001:0007c53e       _vsprintf                  1007d53e f   LIBCMT:vsprintf.obj
 0001:0007c556       _memcpy_s                  1007d556 f   LIBCMT:memcpy_s.obj
 0001:0007c5d5       ??0__non_rtti_object@std@@QAE@ABV01@@Z 1007d5d5 f   LIBCMT:stdexcpt.obj
 0001:0007c5f0       ??0__non_rtti_object@std@@QAE@PBD@Z 1007d5f0 f   LIBCMT:stdexcpt.obj
 0001:0007c60b       ??0bad_cast@std@@QAE@ABV01@@Z 1007d60b f   LIBCMT:stdexcpt.obj
 0001:0007c626       ??0bad_cast@std@@QAE@PBD@Z 1007d626 f   LIBCMT:stdexcpt.obj
 0001:0007c642       ??0bad_typeid@std@@QAE@ABV01@@Z 1007d642 f   LIBCMT:stdexcpt.obj
 0001:0007c65d       ??0bad_typeid@std@@QAE@PBD@Z 1007d65d f   LIBCMT:stdexcpt.obj
 0001:0007c679       ??0exception@std@@QAE@ABQBD@Z 1007d679 f   LIBCMT:stdexcpt.obj
 0001:0007c69e       ??0exception@std@@QAE@ABQBDH@Z 1007d69e f   LIBCMT:stdexcpt.obj
 0001:0007c6b9       ??0exception@std@@QAE@ABV01@@Z 1007d6b9 f   LIBCMT:stdexcpt.obj
 0001:0007c6dc       ??0exception@std@@QAE@XZ   1007d6dc f   LIBCMT:stdexcpt.obj
 0001:0007c6ed       ??1__non_rtti_object@std@@UAE@XZ 1007d6ed f   LIBCMT:stdexcpt.obj
 0001:0007c6f8       ??1bad_cast@std@@UAE@XZ    1007d6f8 f   LIBCMT:stdexcpt.obj
 0001:0007c703       ??1bad_typeid@std@@UAE@XZ  1007d703 f   LIBCMT:stdexcpt.obj
 0001:0007c70e       ??1exception@std@@UAE@XZ   1007d70e f   LIBCMT:stdexcpt.obj
 0001:0007c719       ??4exception@std@@QAEAAV01@ABV01@@Z 1007d719 f   LIBCMT:stdexcpt.obj
 0001:0007c74c       ??_G__non_rtti_object@std@@UAEPAXI@Z 1007d74c f i LIBCMT:stdexcpt.obj
 0001:0007c74c       ??_E__non_rtti_object@std@@UAEPAXI@Z 1007d74c f i LIBCMT:stdexcpt.obj
 0001:0007c771       ??_Gbad_cast@std@@UAEPAXI@Z 1007d771 f i LIBCMT:stdexcpt.obj
 0001:0007c771       ??_Ebad_cast@std@@UAEPAXI@Z 1007d771 f i LIBCMT:stdexcpt.obj
 0001:0007c796       ??_Ebad_typeid@std@@UAEPAXI@Z 1007d796 f i LIBCMT:stdexcpt.obj
 0001:0007c796       ??_Gbad_typeid@std@@UAEPAXI@Z 1007d796 f i LIBCMT:stdexcpt.obj
 0001:0007c7bb       ??_Eexception@std@@UAEPAXI@Z 1007d7bb f i LIBCMT:stdexcpt.obj
 0001:0007c7bb       ??_Gexception@std@@UAEPAXI@Z 1007d7bb f i LIBCMT:stdexcpt.obj
 0001:0007c7e0       ?_Copy_str@exception@std@@AAEXPBD@Z 1007d7e0 f   LIBCMT:stdexcpt.obj
 0001:0007c81e       ?_Tidy@exception@std@@AAEXXZ 1007d81e f   LIBCMT:stdexcpt.obj
 0001:0007c83a       ?what@exception@std@@UBEPBDXZ 1007d83a f   LIBCMT:stdexcpt.obj
 0001:0007c847       ??_V@YAXPAX@Z              1007d847 f   LIBCMT:delete2.obj
 0001:0007c84c       ??_U@YAPAXI@Z              1007d84c f   LIBCMT:new2.obj
 0001:0007c860       _floor                     1007d860 f   LIBCMT:floor_pentium4.obj
 0001:0007c8a0       __floor_pentium4           1007d8a0 f   LIBCMT:floor_pentium4.obj
 0001:0007c981       ?_query_new_handler@@YAP6AHI@ZXZ 1007d981 f   LIBCMT:handler.obj
 0001:0007c98e       ?_set_new_handler@@YAP6AHI@ZH@Z 1007d98e f   LIBCMT:handler.obj
 0001:0007c997       ?_set_new_handler@@YAP6AHI@ZP6AHI@Z@Z 1007d997 f   LIBCMT:handler.obj
 0001:0007c9cc       __callnewh                 1007d9cc f   LIBCMT:handler.obj
 0001:0007c9f2       __initp_heap_handler       1007d9f2 f   LIBCMT:handler.obj
 0001:0007c9ff       __FF_MSGBANNER             1007d9ff f   LIBCMT:crt0msg.obj
 0001:0007ca38       __GET_RTERRMSG             1007da38 f   LIBCMT:crt0msg.obj
 0001:0007ca5c       __NMSG_WRITE               1007da5c f   LIBCMT:crt0msg.obj
 0001:0007cc19       ___doserrno                1007dc19 f   LIBCMT:dosmap.obj
 0001:0007cc2c       __dosmaperr                1007dc2c f   LIBCMT:dosmap.obj
 0001:0007cc4d       __errno                    1007dc4d f   LIBCMT:dosmap.obj
 0001:0007cc60       __get_doserrno             1007dc60 f   LIBCMT:dosmap.obj
 0001:0007cc83       __get_errno                1007dc83 f   LIBCMT:dosmap.obj
 0001:0007cca6       __get_errno_from_oserr     1007dca6 f   LIBCMT:dosmap.obj
 0001:0007cce7       __set_doserrno             1007dce7 f   LIBCMT:dosmap.obj
 0001:0007cd06       __set_errno                1007dd06 f   LIBCMT:dosmap.obj
 0001:0007cd25       __get_heap_handle          1007dd25 f   LIBCMT:heapinit.obj
 0001:0007cd2b       __heap_init                1007dd2b f   LIBCMT:heapinit.obj
 0001:0007cd40       __heap_term                1007dd40 f   LIBCMT:heapinit.obj
 0001:0007cd48       ??0_LocaleUpdate@@QAE@PAUlocaleinfo_struct@@@Z 1007dd48 f i LIBCMT:cvt.obj
 0001:0007cdd0       ??1_LocaleUpdate@@QAE@XZ   1007ddd0 f i LIBCMT:cvt.obj
 0001:0007cdde       ?GetLocaleT@_LocaleUpdate@@QAEPAUlocaleinfo_struct@@XZ 1007ddde f i LIBCMT:cvt.obj
 0001:0007cde1       ?strrchr@@YAPADPADH@Z      1007dde1 f i LIBCMT:cvt.obj
 0001:0007cdea       __cfltcvt                  1007ddea f   LIBCMT:cvt.obj
 0001:0007ce0b       __cfltcvt_l                1007de0b f   LIBCMT:cvt.obj
 0001:0007ce91       __cftoa                    1007de91 f   LIBCMT:cvt.obj
 0001:0007ceaf       __cftoa_l                  1007deaf f   LIBCMT:cvt.obj
 0001:0007d20b       __cftoe                    1007e20b f   LIBCMT:cvt.obj
 0001:0007d37a       __cftoe_l                  1007e37a f   LIBCMT:cvt.obj
 0001:0007d448       __cftof                    1007e448 f   LIBCMT:cvt.obj
 0001:0007d54f       __cftof_l                  1007e54f f   LIBCMT:cvt.obj
 0001:0007d610       __cftog                    1007e610 f   LIBCMT:cvt.obj
 0001:0007d62e       __cftog_l                  1007e62e f   LIBCMT:cvt.obj
 0001:0007d72d       __cropzeros                1007e72d f   LIBCMT:cvt.obj
 0001:0007d73e       __cropzeros_l              1007e73e f   LIBCMT:cvt.obj
 0001:0007d7be       __fassign                  1007e7be f   LIBCMT:cvt.obj
 0001:0007d7d6       __fassign_l                1007e7d6 f   LIBCMT:cvt.obj
 0001:0007d818       __forcdecpt                1007e818 f   LIBCMT:cvt.obj
 0001:0007d829       __forcdecpt_l              1007e829 f   LIBCMT:cvt.obj
 0001:0007d89d       __positive                 1007e89d f   LIBCMT:cvt.obj
 0001:0007d8df       __setdefaultprecision      1007e8df f   LIBCMT:fp8.obj
 0001:0007d906       __initp_misc_cfltcvt_tab   1007e906 f   LIBCMT:cmiscdat.obj
 0001:0007d925       __calloc_impl              1007e925 f   LIBCMT:calloc_impl.obj
 0001:0007d99f       __errcode                  1007e99f f   LIBCMT:fpexcept.obj
 0001:0007d9d1       __except1                  1007e9d1 f   LIBCMT:fpexcept.obj
 0001:0007da99       __except2                  1007ea99 f   LIBCMT:fpexcept.obj
 0001:0007db99       __handle_exc               1007eb99 f   LIBCMT:fpexcept.obj
 0001:0007dd77       __handle_qnan1             1007ed77 f   LIBCMT:fpexcept.obj
 0001:0007ddc7       __handle_qnan2             1007edc7 f   LIBCMT:fpexcept.obj
 0001:0007de27       __raise_exc                1007ee27 f   LIBCMT:fpexcept.obj
 0001:0007de48       __raise_exc_ex             1007ee48 f   LIBCMT:fpexcept.obj
 0001:0007e12d       __raise_excf               1007f12d f   LIBCMT:fpexcept.obj
 0001:0007e14e       __set_errno_from_matherr   1007f14e f   LIBCMT:fpexcept.obj
 0001:0007e17b       __umatherr                 1007f17b f   LIBCMT:fpexcept.obj
 0001:0007e21b       __crt_debugger_hook        1007f21b f   LIBCMT:dbghook.obj
 0001:0007e250       ___crtCloseThreadpoolTimer 1007f250 f   LIBCMT:winapisupp.obj
 0001:0007e267       ___crtCloseThreadpoolWait  1007f267 f   LIBCMT:winapisupp.obj
 0001:0007e27e       ___crtCreateEventExW       1007f27e f   LIBCMT:winapisupp.obj
 0001:0007e2b9       ___crtCreateSemaphoreExW   1007f2b9 f   LIBCMT:winapisupp.obj
 0001:0007e2f3       ___crtCreateSymbolicLinkW  1007f2f3 f   LIBCMT:winapisupp.obj
 0001:0007e31c       ___crtCreateThreadpoolTimer 1007f31c f   LIBCMT:winapisupp.obj
 0001:0007e33d       ___crtCreateThreadpoolWait 1007f33d f   LIBCMT:winapisupp.obj
 0001:0007e35e       ___crtFlsAlloc             1007f35e f   LIBCMT:winapisupp.obj
 0001:0007e37c       ___crtFlsFree              1007f37c f   LIBCMT:winapisupp.obj
 0001:0007e39b       ___crtFlsGetValue          1007f39b f   LIBCMT:winapisupp.obj
 0001:0007e3ba       ___crtFlsSetValue          1007f3ba f   LIBCMT:winapisupp.obj
 0001:0007e3dc       ___crtFlushProcessWriteBuffers 1007f3dc f   LIBCMT:winapisupp.obj
 0001:0007e3ec       ___crtFreeLibraryWhenCallbackReturns 1007f3ec f   LIBCMT:winapisupp.obj
 0001:0007e406       ___crtGetCurrentProcessorNumber 1007f406 f   LIBCMT:winapisupp.obj
 0001:0007e418       ___crtGetFileInformationByHandleEx 1007f418 f   LIBCMT:winapisupp.obj
 0001:0007e444       ___crtGetLogicalProcessorInformation 1007f444 f   LIBCMT:winapisupp.obj
 0001:0007e46a       ___crtGetShowWindowMode    1007f46a f   LIBCMT:winapisupp.obj
 0001:0007e48d       ___crtGetTickCount64       1007f48d f   LIBCMT:winapisupp.obj
 0001:0007e4a5       ___crtInitializeCriticalSectionEx 1007f4a5 f   LIBCMT:winapisupp.obj
 0001:0007e4d3       ___crtIsPackagedApp        1007f4d3 f   LIBCMT:winapisupp.obj
 0001:0007e513       ___crtLoadWinApiPointers   1007f513 f   LIBCMT:winapisupp.obj
 0001:0007e79e       ___crtSetFileInformationByHandle 1007f79e f   LIBCMT:winapisupp.obj
 0001:0007e7ca       ___crtSetThreadStackGuarantee 1007f7ca f   LIBCMT:winapisupp.obj
 0001:0007e7e5       ___crtSetThreadpoolTimer   1007f7e5 f   LIBCMT:winapisupp.obj
 0001:0007e805       ___crtSetThreadpoolWait    1007f805 f   LIBCMT:winapisupp.obj
 0001:0007e822       ___crtSetUnhandledExceptionFilter 1007f822 f   LIBCMT:winapisupp.obj
 0001:0007e830       ___crtSleep                1007f830 f   LIBCMT:winapisupp.obj
 0001:0007e83e       ___crtTerminateProcess     1007f83e f   LIBCMT:winapisupp.obj
 0001:0007e853       ___crtUnhandledException   1007f853 f   LIBCMT:winapisupp.obj
 0001:0007e869       ___crtWaitForThreadpoolTimerCallbacks 1007f869 f   LIBCMT:winapisupp.obj
 0001:0007e883       ?_invalid_parameter@@YAXPBG00II@Z 1007f883 f   LIBCMT:invarg.obj
 0001:0007e888       ?_invoke_watson@@YAXPBG00II@Z 1007f888 f   LIBCMT:invarg.obj
 0001:0007e8a0       __call_reportfault         1007f8a0 f   LIBCMT:invarg.obj
 0001:0007e9c5       __get_invalid_parameter_handler 1007f9c5 f   LIBCMT:invarg.obj
 0001:0007e9d2       __initp_misc_invarg        1007f9d2 f   LIBCMT:invarg.obj
 0001:0007e9df       __invalid_parameter        1007f9df f   LIBCMT:invarg.obj
 0001:0007ea0a       __invalid_parameter_noinfo 1007fa0a f   LIBCMT:invarg.obj
 0001:0007ea1a       __invalid_parameter_noinfo_noreturn 1007fa1a f   LIBCMT:invarg.obj
 0001:0007ea35       __invoke_watson            1007fa35 f   LIBCMT:invarg.obj
 0001:0007ea60       __set_invalid_parameter_handler 1007fa60 f   LIBCMT:invarg.obj
 0001:0007ea85       __RTC_Initialize           1007fa85 f   LIBCMT:initsect.obj
 0001:0007eaa5       __RTC_Terminate            1007faa5 f   LIBCMT:initsect.obj
 0001:0007eac5       __lock                     1007fac5 f   LIBCMT:mlock.obj
 0001:0007eaf9       __lockerr_exit             1007faf9 f   LIBCMT:mlock.obj
 0001:0007eb19       __mtdeletelocks            1007fb19 f   LIBCMT:mlock.obj
 0001:0007eb6d       __mtinitlocknum            1007fb6d f   LIBCMT:mlock.obj
 0001:0007ec16       __mtinitlocks              1007fc16 f   LIBCMT:mlock.obj
 0001:0007ec4f       __unlock                   1007fc4f f   LIBCMT:mlock.obj
 0001:0007ec70       __FindPESection            1007fc70 f   LIBCMT:pesect.obj
 0001:0007ecc0       __IsNonwritableInCurrentImage 1007fcc0 f   LIBCMT:pesect.obj
 0001:0007ed80       __ValidateImageBase        1007fd80 f   LIBCMT:pesect.obj
 0001:0007edb1       __calloc_crt               1007fdb1 f   LIBCMT:crtheap.obj
 0001:0007edf9       __malloc_crt               1007fdf9 f   LIBCMT:crtheap.obj
 0001:0007ee40       __realloc_crt              1007fe40 f   LIBCMT:crtheap.obj
 0001:0007ee8a       __recalloc_crt             1007fe8a f   LIBCMT:crtheap.obj
 0001:0007eed8       __set_malloc_crt_max_wait  1007fed8 f   LIBCMT:crtheap.obj
 0001:0007eeeb       _wait_a_bit                1007feeb f i LIBCMT:crtheap.obj
 0001:0007ef0f       ?_inconsistency@@YAXXZ     1007ff0f f   LIBCMT:hooks.obj
 0001:0007ef47       ?terminate@@YAXXZ          1007ff47 f   LIBCMT:hooks.obj
 0001:0007ef7b       ?unexpected@@YAXXZ         1007ff7b f   LIBCMT:hooks.obj
 0001:0007ef8e       __initp_eh_hooks           1007ff8e f   LIBCMT:hooks.obj
 0001:0007ef9f       ___getlocaleinfo           1007ff9f f   LIBCMT:inithelp.obj
 0001:0007f178       __initp_misc_purevirt      10080178 f   LIBCMT:inithelp.obj
 0001:0007f185       ___fpecode                 10080185 f   LIBCMT:winsig.obj
 0001:0007f18e       ___get_sigabrt             1008018e f   LIBCMT:winsig.obj
 0001:0007f19b       ___pxcptinfoptrs           1008019b f   LIBCMT:winsig.obj
 0001:0007f1a4       __initp_misc_winsig        100801a4 f   LIBCMT:winsig.obj
 0001:0007f265       _raise                     10080265 f   LIBCMT:winsig.obj
 0001:0007f45a       _signal                    1008045a f   LIBCMT:winsig.obj
 0001:0007f6b1       __initp_misc_rand_s        100806b1 f   LIBCMT:rand_s.obj
 0001:0007f6be       _rand_s                    100806be f   LIBCMT:rand_s.obj
 0001:0007f7d0       __SEH_prolog4              100807d0 f   LIBCMT:sehprolg4.obj
 0001:0007f815       __SEH_epilog4              10080815 f   LIBCMT:sehprolg4.obj
 0001:0007f870       __except_handler4          10080870 f   LIBCMT:chandler4.obj
 0001:0007fa04       ___initmbctable            10080a04 f   LIBCMT:mbctype.obj
 0001:0007fcbb       ___updatetmbcinfo          10080cbb f   LIBCMT:mbctype.obj
 0001:0007fd61       __getmbcp                  10080d61 f   LIBCMT:mbctype.obj
 0001:0007fd92       __setmbcp                  10080d92 f   LIBCMT:mbctype.obj
 0001:0007ff3a       __setmbcp_nolock           10080f3a f   LIBCMT:mbctype.obj
 0001:00080125       __ftbuf                    10081125 f   LIBCMT:_sftbuf.obj
 0001:00080156       __stbuf                    10081156 f   LIBCMT:_sftbuf.obj
 0001:000801fc       __fcloseall                100811fc f   LIBCMT:closeall.obj
 0001:00080299       __fileno                   10081299 f   LIBCMT:fileno.obj
 0001:000802bd       __close                    100812bd f   LIBCMT:close.obj
 0001:00080398       __close_nolock             10081398 f   LIBCMT:close.obj
 0001:00080432       __freebuf                  10081432 f   LIBCMT:_freebuf.obj
 0001:00080462       __getstream                10081462 f   LIBCMT:stream.obj
 0001:00080581       __openfile                 10081581 f   LIBCMT:_open.obj
 0001:00080800       __local_unwind4            10081800 f   LIBCMT:exsup4.obj
 0001:000808d6       __seh_longjmp_unwind4@4    100818d6 f   LIBCMT:exsup4.obj
 0001:000808f2       @_EH4_CallFilterFunc@8     100818f2 f   LIBCMT:exsup4.obj
 0001:00080909       @_EH4_TransferToHandler@8  10081909 f   LIBCMT:exsup4.obj
 0001:00080922       @_EH4_GlobalUnwind2@8      10081922 f   LIBCMT:exsup4.obj
 0001:0008093b       @_EH4_LocalUnwind@16       1008193b f   LIBCMT:exsup4.obj
 0001:00080952       __vfprintf_l               10081952 f   LIBCMT:vfprintf.obj
 0001:00080970       __vfprintf_p               10081970 f   LIBCMT:vfprintf.obj
 0001:0008098d       __vfprintf_p_l             1008198d f   LIBCMT:vfprintf.obj
 0001:000809ab       __vfprintf_s_l             100819ab f   LIBCMT:vfprintf.obj
 0001:000809c9       _vfprintf                  100819c9 f   LIBCMT:vfprintf.obj
 0001:000809e6       _vfprintf_helper           100819e6 f   LIBCMT:vfprintf.obj
 0001:00080af7       _vfprintf_s                10081af7 f   LIBCMT:vfprintf.obj
 0001:00080b14       __output_l                 10081b14 f   LIBCMT:output.obj
 0001:00081694       _get_int64_arg             10082694 f i LIBCMT:output.obj
 0001:000816a7       _get_int_arg               100826a7 f i LIBCMT:output.obj
 0001:000816b7       _get_short_arg             100826b7 f i LIBCMT:output.obj
 0001:000817b4       __ioinit                   100827b4 f   LIBCMT:ioinit.obj
 0001:00081a68       __ioterm                   10082a68 f   LIBCMT:ioinit.obj
 0001:00081aba       __filbuf                   10082aba f   LIBCMT:_filbuf.obj
 0001:00081bdb       __read                     10082bdb f   LIBCMT:read.obj
 0001:00081cef       __read_nolock              10082cef f   LIBCMT:read.obj
 0001:00082480       __flsbuf                   10083480 f   LIBCMT:_flsbuf.obj
 0001:000825cf       __write                    100835cf f   LIBCMT:write.obj
 0001:000826be       __write_nolock             100836be f   LIBCMT:write.obj
 0001:00082f23       __vprintf_l                10083f23 f   LIBCMT:vprintf.obj
 0001:00082f3e       __vprintf_p                10083f3e f   LIBCMT:vprintf.obj
 0001:00082f58       __vprintf_p_l              10083f58 f   LIBCMT:vprintf.obj
 0001:00082f73       __vprintf_s_l              10083f73 f   LIBCMT:vprintf.obj
 0001:00082f8e       _vprintf                   10083f8e f   LIBCMT:vprintf.obj
 0001:00082fa8       _vprintf_helper            10083fa8 f   LIBCMT:vprintf.obj
 0001:00083035       _vprintf_s                 10084035 f   LIBCMT:vprintf.obj
 0001:0008304f       __wremove                  1008404f f   LIBCMT:wunlink.obj
 0001:0008307d       __wunlink                  1008407d f   LIBCMT:wunlink.obj
 0001:00083086       __lseek                    10084086 f   LIBCMT:lseek.obj
 0001:00083175       __lseek_nolock             10084175 f   LIBCMT:lseek.obj
 0001:0008321c       __vsnprintf_c              1008421c f   LIBCMT:vsnprnc.obj
 0001:00083243       __vsnprintf_c_l            10084243 f   LIBCMT:vsnprnc.obj
 0001:0008326b       __vsnprintf_helper         1008426b f   LIBCMT:vsnprnc.obj
 0001:00083335       __vsnprintf_s              10084335 f   LIBCMT:vsnprnc.obj
 0001:00083353       __vsnprintf_s_l            10084353 f   LIBCMT:vsnprnc.obj
 0001:00083453       __vsprintf_p               10084453 f   LIBCMT:vsnprnc.obj
 0001:0008347a       __vsprintf_p_l             1008447a f   LIBCMT:vsnprnc.obj
 0001:000834a2       __vsprintf_s_l             100844a2 f   LIBCMT:vsnprnc.obj
 0001:00083517       _vsprintf_s                10084517 f   LIBCMT:vsnprnc.obj
 0001:00083532       __chgsign                  10084532 f   LIBCMT:ieeemisc.obj
 0001:0008355f       __chgsignf                 1008455f f   LIBCMT:ieeemisc.obj
 0001:00083580       __copysign                 10084580 f   LIBCMT:ieeemisc.obj
 0001:000835a8       __copysignf                100845a8 f   LIBCMT:ieeemisc.obj
 0001:000835c4       __finite                   100845c4 f   LIBCMT:ieeemisc.obj
 0001:000835dc       __fpclass                  100845dc f   LIBCMT:ieeemisc.obj
 0001:00083678       __isnan                    10084678 f   LIBCMT:ieeemisc.obj
 0001:000836ab       __logb                     100846ab f   LIBCMT:ieeemisc.obj
 0001:0008378c       __nextafter                1008478c f   LIBCMT:ieeemisc.obj
 0001:00083a2c       __scalb                    10084a2c f   LIBCMT:ieeemisc.obj
 0001:00083a44       __add_exp                  10084a44 f   LIBCMT:util.obj
 0001:00083a73       __decomp                   10084a73 f   LIBCMT:util.obj
 0001:00083b45       __get_exp                  10084b45 f   LIBCMT:util.obj
 0001:00083b5e       __set_bexp                 10084b5e f   LIBCMT:util.obj
 0001:00083b87       __set_exp                  10084b87 f   LIBCMT:util.obj
 0001:00083bb6       __sptype                   10084bb6 f   LIBCMT:util.obj
 0001:00083c11       ___clrfp_sse2              10084c11 f   LIBCMT:fpctrl.obj
 0001:00083c32       ___ctrlfp_sse2             10084c32 f   LIBCMT:fpctrl.obj
 0001:00083c6b       ___fclrf_sse2              10084c6b f   LIBCMT:fpctrl.obj
 0001:00083c88       ___get_fpsr_sse2           10084c88 f   LIBCMT:fpctrl.obj
 0001:00083ca4       ___set_fpsr_sse2           10084ca4 f   LIBCMT:fpctrl.obj
 0001:00083d1a       ___set_statfp_sse2         10084d1a f   LIBCMT:fpctrl.obj
 0001:00083d33       ___statfp_sse2             10084d33 f   LIBCMT:fpctrl.obj
 0001:00083d48       __clrfp                    10084d48 f   LIBCMT:fpctrl.obj
 0001:00083d59       __ctrlfp                   10084d59 f   LIBCMT:fpctrl.obj
 0001:00083d84       __set_statfp               10084d84 f   LIBCMT:fpctrl.obj
 0001:00083ddc       __statfp                   10084ddc f   LIBCMT:fpctrl.obj
 0001:00083dec       __VEC_memset               10084dec f   LIBCMT:p4_memset.obj
 0001:00083eb4       _wcscat_s                  10084eb4 f   LIBCMT:wcscat_s.obj
 0001:00083f20       _wcscpy_s                  10084f20 f   LIBCMT:wcscpy_s.obj
 0001:00083f7c       _wcslen                    10084f7c f   LIBCMT:wcslen.obj
 0001:00083f95       _wcsncat_s                 10084f95 f   LIBCMT:wcsncat_s.obj
 0001:00084063       __set_abort_behavior       10085063 f   LIBCMT:abort.obj
 0001:00084082       _abort                     10085082 f   LIBCMT:abort.obj
 0001:000840c5       ___set_app_type            100850c5 f   LIBCMT:errmode.obj
 0001:000840d2       __set_error_mode           100850d2 f   LIBCMT:errmode.obj
 0001:0008422e       __i64tow_s                 1008522e f   LIBCMT:xtows.obj
 0001:0008425f       __itow_s                   1008525f f   LIBCMT:xtows.obj
 0001:00084288       __ltow_s                   10085288 f   LIBCMT:xtows.obj
 0001:000842b2       __ui64tow_s                100852b2 f   LIBCMT:xtows.obj
 0001:000842cd       __ultow_s                  100852cd f   LIBCMT:xtows.obj
 0001:000843d8       __fwprintf_l               100853d8 f   LIBCMT:fwprintf.obj
 0001:000843f2       __fwprintf_p               100853f2 f   LIBCMT:fwprintf.obj
 0001:0008440b       __fwprintf_p_l             1008540b f   LIBCMT:fwprintf.obj
 0001:00084425       __fwprintf_s_l             10085425 f   LIBCMT:fwprintf.obj
 0001:0008443f       _fwprintf                  1008543f f   LIBCMT:fwprintf.obj
 0001:000844d3       _fwprintf_s                100854d3 f   LIBCMT:fwprintf.obj
 0001:000844ec       __vsnwprintf_s             100854ec f   LIBCMT:vswprnc.obj
 0001:0008450a       __vsnwprintf_s_l           1008550a f   LIBCMT:vswprnc.obj
 0001:0008460e       __vswprintf_c              1008560e f   LIBCMT:vswprnc.obj
 0001:00084635       __vswprintf_c_l            10085635 f   LIBCMT:vswprnc.obj
 0001:0008465d       __vswprintf_helper         1008565d f   LIBCMT:vswprnc.obj
 0001:00084758       __vswprintf_p              10085758 f   LIBCMT:vswprnc.obj
 0001:0008477f       __vswprintf_p_l            1008577f f   LIBCMT:vswprnc.obj
 0001:000847a7       __vswprintf_s_l            100857a7 f   LIBCMT:vswprnc.obj
 0001:0008481e       _vswprintf_s               1008581e f   LIBCMT:vswprnc.obj
 0001:00084839       ___crtMessageBoxW          10085839 f   LIBCMT:crtmboxw.obj
 0001:00084a1f       ___crtMessageBoxWaitThreadW@4 10085a1f f   LIBCMT:crtmboxw.obj
 0001:00084a3d       __XcptFilter               10085a3d f   LIBCMT:winxfltr.obj
 0001:00084b98       ___CppXcptFilter           10085b98 f   LIBCMT:winxfltr.obj
 0001:00084bea       ___get_flsindex            10085bea f   LIBCMT:tidtable.obj
 0001:00084bf0       ___threadhandle            10085bf0 f   LIBCMT:tidtable.obj
 0001:00084bf6       ___threadid                10085bf6 f   LIBCMT:tidtable.obj
 0001:00084bfc       __freefls@4                10085bfc f   LIBCMT:tidtable.obj
 0001:00084d31       __freeptd                  10085d31 f   LIBCMT:tidtable.obj
 0001:00084d67       __getptd                   10085d67 f   LIBCMT:tidtable.obj
 0001:00084d7f       __getptd_noexit            10085d7f f   LIBCMT:tidtable.obj
 0001:00084dee       __initptd                  10085dee f   LIBCMT:tidtable.obj
 0001:00084ea1       __mtinit                   10085ea1 f   LIBCMT:tidtable.obj
 0001:00084f17       __mtterm                   10085f17 f   LIBCMT:tidtable.obj
 0001:00084f34       __set_pgmptr               10085f34 f i LIBCMT:stdargv.obj
 0001:00084f41       __setargv                  10085f41 f   LIBCMT:stdargv.obj
 0001:00085170       __setenvp                  10086170 f   LIBCMT:stdenvp.obj
 0001:00085251       ___security_init_cookie    10086251 f   LIBCMT:gs_support.obj
 0001:000852ed       ___crtGetEnvironmentStringsA 100862ed f   LIBCMT:a_env.obj
 0001:0008537a       __msize                    1008637a f   LIBCMT:msize.obj
 0001:000853b0       __CIsqrt                   100863b0 f   LIBCMT:sqrt.obj
 0001:000853c4       _sqrt                      100863c4     LIBCMT:sqrt.obj
 0001:00085470       __CallSettingFrame@12      10086470 f   LIBCMT:lowhelpr.obj
 0001:00085497       __NLG_Return               10086497     LIBCMT:lowhelpr.obj
 0001:000854bc       ___DestructExceptionObject 100864bc f   LIBCMT:frame.obj
 0001:00085547       ??0bad_exception@std@@QAE@ABV01@@Z 10086547 f i LIBCMT:frame.obj
 0001:00085562       ??0bad_exception@std@@QAE@PBD@Z 10086562 f i LIBCMT:frame.obj
 0001:0008557e       ??1bad_exception@std@@UAE@XZ 1008657e f i LIBCMT:frame.obj
 0001:00085589       ??_Ebad_exception@std@@UAEPAXI@Z 10086589 f i LIBCMT:frame.obj
 0001:00085589       ??_Gbad_exception@std@@UAEPAXI@Z 10086589 f i LIBCMT:frame.obj
 0001:00085df6       ?__uncaught_exception@@YA_NXZ 10086df6 f   LIBCMT:frame.obj
 0001:00085e07       ?_is_exception_typeof@@YAHABVtype_info@@PAU_EXCEPTION_POINTERS@@@Z 10086e07 f   LIBCMT:frame.obj
 0001:00085e8e       __SetWinRTOutOfMemoryExceptionCallback 10086e8e f   LIBCMT:frame.obj
 0001:00085e9b       ___AdjustPointer           10086e9b f   LIBCMT:frame.obj
 0001:00085ec0       ___BuildCatchObject        10086ec0 f   LIBCMT:frame.obj
 0001:00085f4e       ___BuildCatchObjectHelper  10086f4e f   LIBCMT:frame.obj
 0001:00086110       ___CxxDetectRethrow        10087110 f   LIBCMT:frame.obj
 0001:0008615f       ___CxxExceptionFilter      1008715f f   LIBCMT:frame.obj
 0001:000862b9       ___CxxQueryExceptionSize   100872b9 f   LIBCMT:frame.obj
 0001:000862bd       ___CxxRegisterExceptionObject 100872bd f   LIBCMT:frame.obj
 0001:00086374       ___CxxUnregisterExceptionObject 10087374 f   LIBCMT:frame.obj
 0001:000864b1       ___FrameUnwindFilter       100874b1 f   LIBCMT:frame.obj
 0001:000864ff       ___FrameUnwindToState      100874ff f   LIBCMT:frame.obj
 0001:000865d8       ___GetPlatformExceptionInfo 100875d8 f   LIBCMT:frame.obj
 0001:0008662d       ___InternalCxxFrameHandler 1008762d f   LIBCMT:frame.obj
 0001:0008670e       ___TypeMatch               1008770e f   LIBCMT:frame.obj
 0001:00086780       _strcmp                    10087780 f   LIBCMT:strcmp.obj
 0001:0008680c       ?_Name_base@type_info@@CAPBDPBV1@PAU__type_info_node@@@Z 1008780c f   LIBCMT:typname.obj
 0001:000868fd       ?_Name_base_internal@type_info@@CAPBDPBV1@PAU__type_info_node@@@Z 100878fd f   LIBCMT:typname.obj
 0001:00086a07       ?_Type_info_dtor@type_info@@CAXPAV1@@Z 10087a07 f   LIBCMT:typname.obj
 0001:00086a78       ?_Type_info_dtor_internal@type_info@@CAXPAV1@@Z 10087a78 f   LIBCMT:typname.obj
 0001:00086ae9       ___clean_type_info_names_internal 10087ae9 f   LIBCMT:typname.obj
 0001:00086b3c       ___unDNameHelper           10087b3c f   LIBCMT:typname.obj
 0001:00086b6a       __commit                   10087b6a f   LIBCMT:commit.obj
 0001:00086c53       __ftelli64                 10087c53 f   LIBCMT:ftelli64.obj
 0001:00086cce       __ftelli64_nolock          10087cce f   LIBCMT:ftelli64.obj
 0001:000870a3       __lseeki64                 100880a3 f   LIBCMT:lseeki64.obj
 0001:0008719f       __lseeki64_nolock          1008819f f   LIBCMT:lseeki64.obj
 0001:00087212       __getbuf                   10088212 f   LIBCMT:_getbuf.obj
 0001:00087258       __vsnprintf                10088258 f   LIBCMT:vsnprint.obj
 0001:00087273       __vsnprintf_l              10088273 f   LIBCMT:vsnprint.obj
 0001:0008731f       __output_p_l               1008831f f   LIBCMT:outputp.obj
 0001:00088657       __validate_param_reuseA    10089657 f   LIBCMT:outputp.obj
 0001:0008878d       _get_crtdouble_arg         1008978d f i LIBCMT:outputp.obj
 0001:0008888c       _strcpy_s                  1008988c f   LIBCMT:strcpy_s.obj
 0001:000888f0       _strlen                    100898f0 f   LIBCMT:strlen.obj
 0001:0008897b       ___libm_error_support      1008997b f   LIBCMT:libm_error.obj
 0001:00088c63       ___libm_setusermatherr     10089c63 f   LIBCMT:libm_error.obj
 0001:00088c8f       __sse2_mathfcns_init       10089c8f f   LIBCMT:mathfcns.obj
 0001:00088c9e       __set_SSE2_enable          10089c9e f   LIBCMT:mathfcns.obj
 0001:00088cbd       __floor_default            10089cbd f   LIBCMT:floor.obj
 0001:00088d94       _wcsncpy_s                 10089d94 f   LIBCMT:wcsncpy_s.obj
 0001:00088e52       ___addlocaleref            10089e52 f   LIBCMT:localref.obj
 0001:00088ee7       ___freetlocinfo            10089ee7 f   LIBCMT:localref.obj
 0001:00089041       ___removelocaleref         1008a041 f   LIBCMT:localref.obj
 0001:000890e1       ___updatetlocinfo          1008a0e1 f   LIBCMT:localref.obj
 0001:00089161       __updatetlocinfoEx_nolock  1008a161 f   LIBCMT:localref.obj
 0001:000891ac       ___isascii                 1008a1ac f i LIBCMT:_ctype.obj
 0001:000891bc       ___iscsym                  1008a1bc f i LIBCMT:_ctype.obj
 0001:000891dc       ___iscsymf                 1008a1dc f i LIBCMT:_ctype.obj
 0001:000891f9       ___toascii                 1008a1f9 f i LIBCMT:_ctype.obj
 0001:00089204       __isalnum_l                1008a204 f i LIBCMT:_ctype.obj
 0001:0008925c       __isalpha_l                1008a25c f i LIBCMT:_ctype.obj
 0001:000892b4       __isblank_l                1008a2b4 f i LIBCMT:_ctype.obj
 0001:0008930e       __iscntrl_l                1008a30e f i LIBCMT:_ctype.obj
 0001:00089360       __iscsym_l                 1008a360 f i LIBCMT:_ctype.obj
 0001:00089381       __iscsymf_l                1008a381 f i LIBCMT:_ctype.obj
 0001:000893a2       __isdigit_l                1008a3a2 f i LIBCMT:_ctype.obj
 0001:000893f4       __isgraph_l                1008a3f4 f i LIBCMT:_ctype.obj
 0001:0008944c       __islower_l                1008a44c f i LIBCMT:_ctype.obj
 0001:0008949e       __isprint_l                1008a49e f i LIBCMT:_ctype.obj
 0001:000894f6       __ispunct_l                1008a4f6 f i LIBCMT:_ctype.obj
 0001:00089548       __isspace_l                1008a548 f i LIBCMT:_ctype.obj
 0001:0008959a       __isupper_l                1008a59a f i LIBCMT:_ctype.obj
 0001:000895ec       __isxdigit_l               1008a5ec f i LIBCMT:_ctype.obj
 0001:00089644       _isalnum                   1008a644 f i LIBCMT:_ctype.obj
 0001:00089671       _isalpha                   1008a671 f i LIBCMT:_ctype.obj
 0001:0008969e       _isblank                   1008a69e f i LIBCMT:_ctype.obj
 0001:000896d3       _iscntrl                   1008a6d3 f i LIBCMT:_ctype.obj
 0001:000896fe       _isdigit                   1008a6fe f i LIBCMT:_ctype.obj
 0001:00089729       _isgraph                   1008a729 f i LIBCMT:_ctype.obj
 0001:00089756       _islower                   1008a756 f i LIBCMT:_ctype.obj
 0001:00089781       _isprint                   1008a781 f i LIBCMT:_ctype.obj
 0001:000897ae       _ispunct                   1008a7ae f i LIBCMT:_ctype.obj
 0001:000897d9       _isspace                   1008a7d9 f i LIBCMT:_ctype.obj
 0001:00089804       _isupper                   1008a804 f i LIBCMT:_ctype.obj
 0001:0008982f       _isxdigit                  1008a82f f i LIBCMT:_ctype.obj
 0001:0008985c       __tolower                  1008a85c f   LIBCMT:tolower.obj
 0001:00089867       __tolower_l                1008a867 f   LIBCMT:tolower.obj
 0001:000899aa       _tolower                   1008a9aa f   LIBCMT:tolower.obj
 0001:000899e0       _strrchr                   1008a9e0 f   LIBCMT:strrchr.obj
 0001:00089b17       __fptostr                  1008ab17 f   LIBCMT:_fptostr.obj
 0001:00089bc7       ___crt_atoflt_l            1008abc7 f   LIBCMT:atodbl.obj
 0001:00089c6b       __atodbl                   1008ac6b f   LIBCMT:atodbl.obj
 0001:00089c80       __atodbl_l                 1008ac80 f   LIBCMT:atodbl.obj
 0001:00089d0e       __atoflt                   1008ad0e f   LIBCMT:atodbl.obj
 0001:00089d23       __atoflt_l                 1008ad23 f   LIBCMT:atodbl.obj
 0001:00089d3b       __atoldbl                  1008ad3b f   LIBCMT:atodbl.obj
 0001:00089d50       __atoldbl_l                1008ad50 f   LIBCMT:atodbl.obj
 0001:00089ddf       ___dtold                   1008addf f   LIBCMT:cfout.obj
 0001:00089ea7       __fltout2                  1008aea7 f   LIBCMT:cfout.obj
 0001:00089f40       __alldvrm                  1008af40 f   LIBCMT:lldvrm.obj
 0001:0008a020       __aullshr                  1008b020 f   LIBCMT:ullshr.obj
 0001:0008a03f       __get_output_format        1008b03f f   LIBCMT:outputformat.obj
 0001:0008a045       __set_output_format        1008b045 f   LIBCMT:outputformat.obj
 0001:0008a077       __controlfp_s              1008b077 f   LIBCMT:contrlfp.obj
 0001:0008a0d4       __fptrap                   1008b0d4 f   LIBCMT:crt0fp.obj
 0001:0008a0dd       __matherr                  1008b0dd f   LIBCMT:matherr.obj
 0001:0008a0e0       __recalloc                 1008b0e0 f   LIBCMT:recalloc.obj
 0001:0008a149       _strncpy_s                 1008b149 f   LIBCMT:strncpy_s.obj
 0001:0008a2d1       __MallocaIsSizeInRange     1008b2d1 f i LIBCMT:a_loc.obj
 0001:0008a2e2       __MarkAllocaS              1008b2e2 f i LIBCMT:a_loc.obj
 0001:0008a2f6       ___crtGetLocaleInfoA       1008b2f6 f   LIBCMT:a_loc.obj
 0001:0008a330       __freea                    1008b330 f i LIBCMT:a_loc.obj
 0001:0008a34e       _GetTableIndexFromLcid     1008b34e f   LIBCMT:winapinls.obj
 0001:0008a383       _GetTableIndexFromLocaleName 1008b383 f   LIBCMT:winapinls.obj
 0001:0008a3d1       ___crtCompareStringEx      1008b3d1 f   LIBCMT:winapinls.obj
 0001:0008a41d       ___crtDownlevelLCIDToLocaleName 1008b41d f   LIBCMT:winapinls.obj
 0001:0008a499       ___crtDownlevelLocaleNameToLCID 1008b499 f   LIBCMT:winapinls.obj
 0001:0008a4d7       ___crtEnumSystemLocalesEx  1008b4d7 f   LIBCMT:winapinls.obj
 0001:0008a514       ___crtGetDateFormatEx      1008b514 f   LIBCMT:winapinls.obj
 0001:0008a55d       ___crtGetLocaleInfoEx      1008b55d f   LIBCMT:winapinls.obj
 0001:0008a58c       ___crtGetTimeFormatEx      1008b58c f   LIBCMT:winapinls.obj
 0001:0008a5c1       ___crtGetUserDefaultLocaleName 1008b5c1 f   LIBCMT:winapinls.obj
 0001:0008a5ec       ___crtIsValidLocaleName    1008b5ec f   LIBCMT:winapinls.obj
 0001:0008a617       ___crtLCMapStringEx        1008b617 f   LIBCMT:winapinls.obj
 0001:0008a663       ___wcsnicmp_ascii          1008b663 f   LIBCMT:winapinls.obj
 0001:0008a8f5       ___crtLCMapStringA         1008b8f5 f   LIBCMT:a_map.obj
 0001:0008aa33       ___crtGetStringTypeA       1008ba33 f   LIBCMT:a_str.obj
 0001:0008aa73       __isatty                   1008ba73 f   LIBCMT:isatty.obj
 0001:0008aac7       ___lock_fhandle            1008bac7 f   LIBCMT:osfinfo.obj
 0001:0008ab55       __alloc_osfhnd             1008bb55 f   LIBCMT:osfinfo.obj
 0001:0008acfe       __free_osfhnd              1008bcfe f   LIBCMT:osfinfo.obj
 0001:0008ad84       __get_osfhandle            1008bd84 f   LIBCMT:osfinfo.obj
 0001:0008adeb       __open_osfhandle           1008bdeb f   LIBCMT:osfinfo.obj
 0001:0008af01       __set_osfhnd               1008bf01 f   LIBCMT:osfinfo.obj
 0001:0008af83       __unlock_fhandle           1008bf83 f   LIBCMT:osfinfo.obj
 0001:0008afa9       __open                     1008bfa9 f   LIBCMT:open.obj
 0001:0008b059       __sopen                    1008c059 f   LIBCMT:open.obj
 0001:0008b08c       __sopen_helper             1008c08c f   LIBCMT:open.obj
 0001:0008b155       __sopen_nolock             1008c155 f   LIBCMT:open.obj
 0001:0008b1a3       __sopen_s                  1008c1a3 f   LIBCMT:open.obj
 0001:0008b1c1       __mbsnbcmp                 1008c1c1 f   LIBCMT:mbsnbcmp.obj
 0001:0008b1d9       __mbsnbcmp_l               1008c1d9 f   LIBCMT:mbsnbcmp.obj
 0001:0008b2f0       __mbsnbicmp                1008c2f0 f   LIBCMT:mbsnbicm.obj
 0001:0008b308       __mbsnbicmp_l              1008c308 f   LIBCMT:mbsnbicm.obj
 0001:0008b4d0       __global_unwind2           1008c4d0 f   LIBCMT:exsup.obj
 0001:0008b535       __local_unwind2            1008c535 f   LIBCMT:exsup.obj
 0001:0008b5b9       __abnormal_termination     1008c5b9 f   LIBCMT:exsup.obj
 0001:0008b5dc       __NLG_Notify1              1008c5dc f   LIBCMT:exsup.obj
 0001:0008b5e5       __NLG_Notify               1008c5e5 f   LIBCMT:exsup.obj
 0001:0008b5fc       __NLG_Dispatch             1008c5fc     LIBCMT:exsup.obj
 0001:0008b5fc       __NLG_Dispatch2            1008c5fc     LIBCMT:exsup.obj
 0001:0008b604       __NLG_Call                 1008c604 f   LIBCMT:exsup.obj
 0001:0008b606       __NLG_Return2              1008c606     LIBCMT:exsup.obj
 0001:0008b607       __output_s_l               1008c607 f   LIBCMT:outputs.obj
 0001:0008c28f       ___iswcsym                 1008d28f f i LIBCMT:_wctype.obj
 0001:0008c2b3       ___iswcsymf                1008d2b3 f i LIBCMT:_wctype.obj
 0001:0008c2d7       __isleadbyte_l             1008d2d7 f i LIBCMT:_wctype.obj
 0001:0008c311       __iswalnum_l               1008d311 f i LIBCMT:_wctype.obj
 0001:0008c325       __iswalpha_l               1008d325 f i LIBCMT:_wctype.obj
 0001:0008c339       __iswblank_l               1008d339 f i LIBCMT:_wctype.obj
 0001:0008c354       __iswcntrl_l               1008d354 f i LIBCMT:_wctype.obj
 0001:0008c365       __iswcsym_l                1008d365 f i LIBCMT:_wctype.obj
 0001:0008c389       __iswcsymf_l               1008d389 f i LIBCMT:_wctype.obj
 0001:0008c3ad       __iswdigit_l               1008d3ad f i LIBCMT:_wctype.obj
 0001:0008c3be       __iswgraph_l               1008d3be f i LIBCMT:_wctype.obj
 0001:0008c3d2       __iswlower_l               1008d3d2 f i LIBCMT:_wctype.obj
 0001:0008c3e3       __iswprint_l               1008d3e3 f i LIBCMT:_wctype.obj
 0001:0008c3f7       __iswpunct_l               1008d3f7 f i LIBCMT:_wctype.obj
 0001:0008c408       __iswspace_l               1008d408 f i LIBCMT:_wctype.obj
 0001:0008c419       __iswupper_l               1008d419 f i LIBCMT:_wctype.obj
 0001:0008c42a       __iswxdigit_l              1008d42a f i LIBCMT:_wctype.obj
 0001:0008c43e       _isleadbyte                1008d43e f i LIBCMT:_wctype.obj
 0001:0008c44f       _iswalnum                  1008d44f f i LIBCMT:_wctype.obj
 0001:0008c463       _iswalpha                  1008d463 f i LIBCMT:_wctype.obj
 0001:0008c477       _iswascii                  1008d477 f i LIBCMT:_wctype.obj
 0001:0008c489       _iswblank                  1008d489 f i LIBCMT:_wctype.obj
 0001:0008c4a4       _iswcntrl                  1008d4a4 f i LIBCMT:_wctype.obj
 0001:0008c4b5       _iswdigit                  1008d4b5 f i LIBCMT:_wctype.obj
 0001:0008c4c6       _iswgraph                  1008d4c6 f i LIBCMT:_wctype.obj
 0001:0008c4da       _iswlower                  1008d4da f i LIBCMT:_wctype.obj
 0001:0008c4eb       _iswprint                  1008d4eb f i LIBCMT:_wctype.obj
 0001:0008c4ff       _iswpunct                  1008d4ff f i LIBCMT:_wctype.obj
 0001:0008c510       _iswspace                  1008d510 f i LIBCMT:_wctype.obj
 0001:0008c521       _iswupper                  1008d521 f i LIBCMT:_wctype.obj
 0001:0008c532       _iswxdigit                 1008d532 f i LIBCMT:_wctype.obj
 0001:0008c546       __wctomb_l                 1008d546 f   LIBCMT:wctomb.obj
 0001:0008c595       __wctomb_s_l               1008d595 f   LIBCMT:wctomb.obj
 0001:0008c6b9       _wctomb                    1008d6b9 f   LIBCMT:wctomb.obj
 0001:0008c6ec       _wctomb_s                  1008d6ec f   LIBCMT:wctomb.obj
 0001:0008c710       __aulldvrm                 1008d710 f   LIBCMT:ulldvrm.obj
 0001:0008c7a5       __mbtowc_l                 1008d7a5 f   LIBCMT:mbtowc.obj
 0001:0008c89a       _mbtowc                    1008d89a f   LIBCMT:mbtowc.obj
 0001:0008c8b2       __putwch                   1008d8b2 f   LIBCMT:putwch.obj
 0001:0008c8fe       __putwch_nolock            1008d8fe f   LIBCMT:putwch.obj
 0001:0008c950       __chkstk                   1008d950 f   LIBCMT:chkstk.obj
 0001:0008c950       __alloca_probe             1008d950 f   LIBCMT:chkstk.obj
 0001:0008c97b       __vfwprintf_l              1008d97b f   LIBCMT:vfwprint.obj
 0001:0008c999       __vfwprintf_p              1008d999 f   LIBCMT:vfwprint.obj
 0001:0008c9b6       __vfwprintf_p_l            1008d9b6 f   LIBCMT:vfwprint.obj
 0001:0008c9d4       __vfwprintf_s_l            1008d9d4 f   LIBCMT:vfwprint.obj
 0001:0008c9f2       _vfwprintf                 1008d9f2 f   LIBCMT:vfwprint.obj
 0001:0008ca0f       _vfwprintf_helper          1008da0f f   LIBCMT:vfwprint.obj
 0001:0008caa2       _vfwprintf_s               1008daa2 f   LIBCMT:vfwprint.obj
 0001:0008cabf       __woutput_l                1008dabf f   LIBCMT:woutput.obj
 0001:0008d79e       __woutput_s_l              1008e79e f   LIBCMT:woutputs.obj
 0001:0008e4b5       __validate_param_reuseW    1008f4b5 f   LIBCMT:woutputp.obj
 0001:0008e62d       __woutput_p_l              1008f62d f   LIBCMT:woutputp.obj
 0001:0008fa56       __ismbbalnum               10090a56 f   LIBCMT:ismbbyte.obj
 0001:0008fa6f       __ismbbalnum_l             10090a6f f   LIBCMT:ismbbyte.obj
 0001:0008fa89       __ismbbalpha               10090a89 f   LIBCMT:ismbbyte.obj
 0001:0008faa2       __ismbbalpha_l             10090aa2 f   LIBCMT:ismbbyte.obj
 0001:0008fabc       __ismbbblank               10090abc f   LIBCMT:ismbbyte.obj
 0001:0008fadd       __ismbbblank_l             10090add f   LIBCMT:ismbbyte.obj
 0001:0008faff       __ismbbgraph               10090aff f   LIBCMT:ismbbyte.obj
 0001:0008fb18       __ismbbgraph_l             10090b18 f   LIBCMT:ismbbyte.obj
 0001:0008fb32       __ismbbkalnum              10090b32 f   LIBCMT:ismbbyte.obj
 0001:0008fb48       __ismbbkalnum_l            10090b48 f   LIBCMT:ismbbyte.obj
 0001:0008fb5f       __ismbbkana                10090b5f f   LIBCMT:ismbbyte.obj
 0001:0008fb70       __ismbbkana_l              10090b70 f   LIBCMT:ismbbyte.obj
 0001:0008fbbc       __ismbbkprint              10090bbc f   LIBCMT:ismbbyte.obj
 0001:0008fbd2       __ismbbkprint_l            10090bd2 f   LIBCMT:ismbbyte.obj
 0001:0008fbe9       __ismbbkpunct              10090be9 f   LIBCMT:ismbbyte.obj
 0001:0008fbff       __ismbbkpunct_l            10090bff f   LIBCMT:ismbbyte.obj
 0001:0008fc16       __ismbblead                10090c16 f   LIBCMT:ismbbyte.obj
 0001:0008fc2c       __ismbblead_l              10090c2c f   LIBCMT:ismbbyte.obj
 0001:0008fc43       __ismbbprint               10090c43 f   LIBCMT:ismbbyte.obj
 0001:0008fc5c       __ismbbprint_l             10090c5c f   LIBCMT:ismbbyte.obj
 0001:0008fc76       __ismbbpunct               10090c76 f   LIBCMT:ismbbyte.obj
 0001:0008fc8c       __ismbbpunct_l             10090c8c f   LIBCMT:ismbbyte.obj
 0001:0008fca3       __ismbbtrail               10090ca3 f   LIBCMT:ismbbyte.obj
 0001:0008fcb9       __ismbbtrail_l             10090cb9 f   LIBCMT:ismbbyte.obj
 0001:0008fcd0       __trandisp1                10090cd0 f   LIBCMT:87disp.obj
 0001:0008fd37       __trandisp2                10090d37 f   LIBCMT:87disp.obj
 0001:0008fdc3       __rttospopde               10090dc3     LIBCMT:87disp.obj
 0001:0008fdc8       __rttospop                 10090dc8     LIBCMT:87disp.obj
 0001:0008fdca       __rtnospop                 10090dca     LIBCMT:87disp.obj
 0001:0008fdcc       __rttosnpop                10090dcc     LIBCMT:87disp.obj
 0001:0008fdcd       __rtnospopde               10090dcd     LIBCMT:87disp.obj
 0001:0008fdd4       __rtzeropop                10090dd4     LIBCMT:87disp.obj
 0001:0008fdd6       __rtzeronpop               10090dd6     LIBCMT:87disp.obj
 0001:0008fddb       __rtonepop                 10090ddb     LIBCMT:87disp.obj
 0001:0008fddd       __rtonenpop                10090ddd     LIBCMT:87disp.obj
 0001:0008fde2       __tosnan1                  10090de2     LIBCMT:87disp.obj
 0001:0008fe0d       __nosnan2                  10090e0d     LIBCMT:87disp.obj
 0001:0008fe0f       __tosnan2                  10090e0f     LIBCMT:87disp.obj
 0001:0008fe37       __nan2                     10090e37     LIBCMT:87disp.obj
 0001:0008fe76       __rtindfpop                10090e76     LIBCMT:87disp.obj
 0001:0008fe78       __rtindfnpop               10090e78     LIBCMT:87disp.obj
 0001:0008fe89       __rttosnpopde              10090e89     LIBCMT:87disp.obj
 0001:0008fe93       __rtchsifneg               10090e93     LIBCMT:87disp.obj
 0001:0008fea0       __startTwoArgErrorHandling 10090ea0 f   LIBCMT:genexcep.obj
 0001:0008feb7       __startOneArgErrorHandling 10090eb7 f   LIBCMT:genexcep.obj
 0001:0008ff00       __twoToTOS                 10090f00 f   LIBCMT:common.obj
 0001:0008ff15       __load_CW                  10090f15 f   LIBCMT:common.obj
 0001:0008ff2c       __convertTOStoQNaN         10090f2c f   LIBCMT:common.obj
 0001:0008ff45       __fload_withFB             10090f45 f   LIBCMT:common.obj
 0001:0008ff88       __checkTOS_withFB          10090f88 f   LIBCMT:common.obj
 0001:0008ff9e       __fast_exit                10090f9e f   LIBCMT:common.obj
 0001:0008ffab       __math_exit                10090fab f   LIBCMT:common.obj
 0001:0008ffd5       __check_overflow_exit      10090fd5 f   LIBCMT:common.obj
 0001:0008ffe9       __check_range_exit         10090fe9 f   LIBCMT:common.obj
 0001:0009008c       ?_ValidateExecute@@YAHP6GHXZ@Z 1009108c f   LIBCMT:validate.obj
 0001:0009009b       ?_ValidateRead@@YAHPBXI@Z  1009109b f   LIBCMT:validate.obj
 0001:000900aa       ?_ValidateWrite@@YAHPAXI@Z 100910aa f   LIBCMT:validate.obj
 0001:000900b9       __EH_epilog3               100910b9 f   LIBCMT:ehprolg3.obj
 0001:000900cd       __EH_epilog3_GS            100910cd f   LIBCMT:ehprolg3.obj
 0001:000900dc       __EH_epilog3_catch_GS      100910dc f   LIBCMT:ehprolg3.obj
 0001:000900eb       __EH_prolog3               100910eb f   LIBCMT:ehprolg3.obj
 0001:0009011e       __EH_prolog3_GS            1009111e f   LIBCMT:ehprolg3.obj
 0001:00090154       __EH_prolog3_catch         10091154 f   LIBCMT:ehprolg3.obj
 0001:0009018a       __EH_prolog3_catch_GS      1009118a f   LIBCMT:ehprolg3.obj
 0001:000901c3       ??0Block@_HeapManager@@QAE@XZ 100911c3 f i LIBCMT:undname.obj
 0001:000901c9       ??0DName@@QAE@AAPBDD@Z     100911c9 f   LIBCMT:undname.obj
 0001:00090282       ??0DName@@QAE@ABV0@@Z      10091282 f i LIBCMT:undname.obj
 0001:00090298       ??0DName@@QAE@D@Z          10091298 f   LIBCMT:undname.obj
 0001:000902c4       ??0DName@@QAE@PAV0@@Z      100912c4 f   LIBCMT:undname.obj
 0001:00090311       ??0DName@@QAE@PBD@Z        10091311 f   LIBCMT:undname.obj
 0001:0009034b       ??0DName@@QAE@W4DNameStatus@@@Z 1009134b f   LIBCMT:undname.obj
 0001:0009038e       ??0DName@@QAE@XZ           1009138e f i LIBCMT:undname.obj
 0001:0009039f       ??0DName@@QAE@_J@Z         1009139f f   LIBCMT:undname.obj
 0001:00090432       ??0DName@@QAE@_K@Z         10091432 f   LIBCMT:undname.obj
 0001:0009049f       ??0DNameNode@@IAE@XZ       1009149f f   LIBCMT:undname.obj
 0001:000904a8       ??0DNameStatusNode@@AAE@W4DNameStatus@@@Z 100914a8 f   LIBCMT:undname.obj
 0001:000904cb       ??0Replicator@@QAE@XZ      100914cb f i LIBCMT:undname.obj
 0001:000904d1       ??0UnDecorator@@QAE@PADPBDHP6APADJ@ZK@Z 100914d1 f i LIBCMT:undname.obj
 0001:0009053a       ??0charNode@@QAE@D@Z       1009153a f   LIBCMT:undname.obj
 0001:0009054f       ??0pDNameNode@@QAE@PAVDName@@@Z 1009154f f   LIBCMT:undname.obj
 0001:00090577       ??0pairNode@@QAE@PAVDNameNode@@0@Z 10091577 f   LIBCMT:undname.obj
 0001:00090596       ??0pcharNode@@QAE@PBDH@Z   10091596 f   LIBCMT:undname.obj
 0001:000905ed       ??2@YAPAXIAAV_HeapManager@@H@Z 100915ed f i LIBCMT:undname.obj
 0001:00090602       ??4DName@@QAEAAV0@ABV0@@Z  10091602 f   LIBCMT:undname.obj
 0001:00090618       ??4DName@@QAEAAV0@D@Z      10091618 f i LIBCMT:undname.obj
 0001:00090644       ??4DName@@QAEAAV0@PAV0@@Z  10091644 f   LIBCMT:undname.obj
 0001:0009068d       ??4DName@@QAEAAV0@PBD@Z    1009168d f   LIBCMT:undname.obj
 0001:000906bf       ??4DName@@QAEAAV0@W4DNameStatus@@@Z 100916bf f   LIBCMT:undname.obj
 0001:000906f4       ??AReplicator@@QBE?AVDName@@H@Z 100916f4 f   LIBCMT:undname.obj
 0001:00090730       ??BUnDecorator@@QAEPADXZ   10091730 f i LIBCMT:undname.obj
 0001:000908af       ??H@YA?AVDName@@DABV0@@Z   100918af f i LIBCMT:undname.obj
 0001:000908d3       ??H@YA?AVDName@@PBDABV0@@Z 100918d3 f i LIBCMT:undname.obj
 0001:000908f7       ??H@YA?AVDName@@W4DNameStatus@@ABV0@@Z 100918f7 f i LIBCMT:undname.obj
 0001:0009091b       ??HDName@@QBE?AV0@ABV0@@Z  1009191b f   LIBCMT:undname.obj
 0001:0009093d       ??HDName@@QBE?AV0@D@Z      1009193d f   LIBCMT:undname.obj
 0001:0009095f       ??HDName@@QBE?AV0@PAV0@@Z  1009195f f   LIBCMT:undname.obj
 0001:00090981       ??HDName@@QBE?AV0@PBD@Z    10091981 f   LIBCMT:undname.obj
 0001:000909a3       ??HDName@@QBE?AV0@W4DNameStatus@@@Z 100919a3 f   LIBCMT:undname.obj
 0001:000909c5       ??YDName@@QAEAAV0@ABV0@@Z  100919c5 f   LIBCMT:undname.obj
 0001:00090a08       ??YDName@@QAEAAV0@D@Z      10091a08 f   LIBCMT:undname.obj
 0001:00090a58       ??YDName@@QAEAAV0@PAV0@@Z  10091a58 f   LIBCMT:undname.obj
 0001:00090abd       ??YDName@@QAEAAV0@PBD@Z    10091abd f   LIBCMT:undname.obj
 0001:00090b1e       ??YDName@@QAEAAV0@W4DNameStatus@@@Z 10091b1e f   LIBCMT:undname.obj
 0001:00090b5e       ??YReplicator@@QAEAAV0@ABVDName@@@Z 10091b5e f   LIBCMT:undname.obj
 0001:00090ba8       ??_5DName@@QAEAAV0@ABV0@@Z 10091ba8 f   LIBCMT:undname.obj
 0001:00090bc4       ?Constructor@_HeapManager@@QAEXP6APAXI@ZP6AXPAX@Z@Z 10091bc4 f i LIBCMT:undname.obj
 0001:00090be1       ?Destructor@_HeapManager@@QAEXXZ 10091be1 f i LIBCMT:undname.obj
 0001:00090c07       ?UScore@UnDecorator@@SAPBDW4Tokens@@@Z 10091c07 f   LIBCMT:undname.obj
 0001:00090c24       ?append@DName@@AAEXPAVDNameNode@@@Z 10091c24 f   LIBCMT:undname.obj
 0001:00090c6a       ?composeDeclaration@UnDecorator@@CA?AVDName@@ABV2@@Z 10091c6a f i LIBCMT:undname.obj
 0001:000919a0       ?doAccessSpecifiers@UnDecorator@@SAHXZ 100929a0 f i LIBCMT:undname.obj
 0001:000919ae       ?doAllocationLanguage@UnDecorator@@SAHXZ 100929ae f i LIBCMT:undname.obj
 0001:000919bc       ?doAllocationModel@UnDecorator@@SAHXZ 100929bc f i LIBCMT:undname.obj
 0001:000919ca       ?doEcsu@UnDecorator@@SAHXZ 100929ca f i LIBCMT:undname.obj
 0001:000919d8       ?doEllipsis@UnDecorator@@SAHXZ 100929d8 f i LIBCMT:undname.obj
 0001:000919e6       ?doFunctionReturns@UnDecorator@@SAHXZ 100929e6 f i LIBCMT:undname.obj
 0001:000919f4       ?doMSKeywords@UnDecorator@@SAHXZ 100929f4 f i LIBCMT:undname.obj
 0001:00091a01       ?doMemberTypes@UnDecorator@@SAHXZ 10092a01 f i LIBCMT:undname.obj
 0001:00091a0f       ?doNameOnly@UnDecorator@@SAHXZ 10092a0f f i LIBCMT:undname.obj
 0001:00091a1a       ?doNoIdentCharCheck@UnDecorator@@SAHXZ 10092a1a f i LIBCMT:undname.obj
 0001:00091a25       ?doPchar@DName@@AAEXPBDH@Z 10092a25 f   LIBCMT:undname.obj
 0001:00091aad       ?doPtr64@UnDecorator@@SAHXZ 10092aad f i LIBCMT:undname.obj
 0001:00091abb       ?doRestrictionSpec@UnDecorator@@SAHXZ 10092abb f i LIBCMT:undname.obj
 0001:00091ac9       ?doThisTypes@UnDecorator@@SAHXZ 10092ac9 f i LIBCMT:undname.obj
 0001:00091adb       ?doThrowTypes@UnDecorator@@SAHXZ 10092adb f i LIBCMT:undname.obj
 0001:00091ae9       ?doTypeOnly@UnDecorator@@SAHXZ 10092ae9 f i LIBCMT:undname.obj
 0001:00091af4       ?doUnderScore@UnDecorator@@SAHXZ 10092af4 f i LIBCMT:undname.obj
 0001:00091aff       ?getArgumentList@UnDecorator@@CA?AVDName@@XZ 10092aff f   LIBCMT:undname.obj
 0001:00091c0b       ?getArgumentTypes@UnDecorator@@CA?AVDName@@XZ 10092c0b f   LIBCMT:undname.obj
 0001:00091ce9       ?getArrayType@UnDecorator@@CA?AVDName@@ABV2@@Z 10092ce9 f i LIBCMT:undname.obj
 0001:00091eeb       ?getBasedType@UnDecorator@@CA?AVDName@@XZ 10092eeb f   LIBCMT:undname.obj
 0001:00091f82       ?getBasicDataType@UnDecorator@@CA?AVDName@@ABV2@@Z 10092f82 f   LIBCMT:undname.obj
 0001:00092359       ?getCallIndex@UnDecorator@@CA?AVDName@@XZ 10093359 f i LIBCMT:undname.obj
 0001:0009236d       ?getCallingConvention@UnDecorator@@CA?AVDName@@XZ 1009336d f   LIBCMT:undname.obj
 0001:0009242c       ?getDataIndirectType@UnDecorator@@CA?AVDName@@ABV2@PBD0H@Z 1009342c f   LIBCMT:undname.obj
 0001:000929c9       ?getDataIndirectType@UnDecorator@@CA?AVDName@@XZ 100939c9 f i LIBCMT:undname.obj
 0001:00092a02       ?getDataType@UnDecorator@@CA?AVDName@@PAV2@@Z 10093a02 f   LIBCMT:undname.obj
 0001:00092ad4       ?getDecoratedName@UnDecorator@@CA?AVDName@@XZ 10093ad4 f   LIBCMT:undname.obj
 0001:00092d20       ?getDimension@UnDecorator@@CA?AVDName@@_N@Z 10093d20 f   LIBCMT:undname.obj
 0001:00092e57       ?getDispatchTarget@UnDecorator@@CA?AVDName@@XZ 10093e57 f   LIBCMT:undname.obj
 0001:00092eb2       ?getDisplacement@UnDecorator@@CA?AVDName@@XZ 10093eb2 f i LIBCMT:undname.obj
 0001:00092ec6       ?getECSUDataType@UnDecorator@@CA?AVDName@@XZ 10093ec6 f   LIBCMT:undname.obj
 0001:00092fd9       ?getECSUName@UnDecorator@@CA?AVDName@@XZ 10093fd9 f i LIBCMT:undname.obj
 0001:00092fea       ?getEnumType@UnDecorator@@CA?AVDName@@XZ 10093fea f i LIBCMT:undname.obj
 0001:000930ce       ?getExtendedDataIndirectType@UnDecorator@@CA?AVDName@@AAPBDAA_NH@Z 100940ce f   LIBCMT:undname.obj
 0001:00093273       ?getExternalDataType@UnDecorator@@CA?AVDName@@ABV2@@Z 10094273 f i LIBCMT:undname.obj
 0001:000932ec       ?getFunctionIndirectType@UnDecorator@@CA?AVDName@@ABV2@@Z 100942ec f   LIBCMT:undname.obj
 0001:000936e2       ?getGuardNumber@UnDecorator@@CA?AVDName@@XZ 100946e2 f i LIBCMT:undname.obj
 0001:000936f6       ?getLastChar@DName@@QBEDXZ 100946f6 f i LIBCMT:undname.obj
 0001:00093704       ?getLastChar@DNameStatusNode@@UBEDXZ 10094704 f i LIBCMT:undname.obj
 0001:00093710       ?getLastChar@charNode@@UBEDXZ 10094710 f i LIBCMT:undname.obj
 0001:00093714       ?getLastChar@pDNameNode@@UBEDXZ 10094714 f i LIBCMT:undname.obj
 0001:00093729       ?getLastChar@pairNode@@UBEDXZ 10094729 f i LIBCMT:undname.obj
 0001:00093743       ?getLastChar@pcharNode@@UBEDXZ 10094743 f i LIBCMT:undname.obj
 0001:00093755       ?getLexicalFrame@UnDecorator@@CA?AVDName@@XZ 10094755 f i LIBCMT:undname.obj
 0001:00093792       ?getMemory@_HeapManager@@QAEPAXIH@Z 10094792 f   LIBCMT:undname.obj
 0001:00093817       ?getNumberOfDimensions@UnDecorator@@CAHXZ 10094817 f   LIBCMT:undname.obj
 0001:00093878       ?getOperatorName@UnDecorator@@CA?AVDName@@_NPA_N@Z 10094878 f i LIBCMT:undname.obj
 0001:00093e52       ?getPointerType@UnDecorator@@CA?AVDName@@ABV2@0@Z 10094e52 f i LIBCMT:undname.obj
 0001:00093e70       ?getPointerTypeArray@UnDecorator@@CA?AVDName@@ABV2@0@Z 10094e70 f i LIBCMT:undname.obj
 0001:00093e8e       ?getPrimaryDataType@UnDecorator@@CA?AVDName@@ABV2@@Z 10094e8e f   LIBCMT:undname.obj
 0001:00094046       ?getPtrRefDataType@UnDecorator@@CA?AVDName@@ABV2@H@Z 10095046 f i LIBCMT:undname.obj
 0001:00094130       ?getPtrRefType@UnDecorator@@CA?AVDName@@ABV2@0PBD@Z 10095130 f   LIBCMT:undname.obj
 0001:0009422c       ?getReferenceType@UnDecorator@@CA?AVDName@@ABV2@0PBD@Z 1009522c f i LIBCMT:undname.obj
 0001:00094248       ?getRestrictionSpec@UnDecorator@@CA?AVDName@@XZ 10095248 f   LIBCMT:undname.obj
 0001:00094336       ?getReturnType@UnDecorator@@CA?AVDName@@PAV2@@Z 10095336 f   LIBCMT:undname.obj
 0001:00094365       ?getScope@UnDecorator@@CA?AVDName@@XZ 10095365 f   LIBCMT:undname.obj
 0001:0009473c       ?getScopedName@UnDecorator@@CA?AVDName@@XZ 1009573c f   LIBCMT:undname.obj
 0001:00094837       ?getSignedDimension@UnDecorator@@CA?AVDName@@XZ 10095837 f   LIBCMT:undname.obj
 0001:0009488a       ?getStorageConvention@UnDecorator@@CA?AVDName@@XZ 1009588a f i LIBCMT:undname.obj
 0001:0009489b       ?getString@DName@@QBEPADPAD0@Z 1009589b f i LIBCMT:undname.obj
 0001:000948b1       ?getString@DName@@QBEPADPADH@Z 100958b1 f i LIBCMT:undname.obj
 0001:0009490f       ?getString@DNameStatusNode@@UBEPADPAD0@Z 1009590f f i LIBCMT:undname.obj
 0001:00094936       ?getString@charNode@@UBEPADPAD0@Z 10095936 f i LIBCMT:undname.obj
 0001:0009494b       ?getString@pDNameNode@@UBEPADPAD0@Z 1009594b f i LIBCMT:undname.obj
 0001:00094968       ?getString@pairNode@@UBEPADPAD0@Z 10095968 f i LIBCMT:undname.obj
 0001:00094992       ?getString@pcharNode@@UBEPADPAD0@Z 10095992 f i LIBCMT:undname.obj
 0001:000949ad       ?getStringEncoding@UnDecorator@@CA?AVDName@@PADH@Z 100959ad f   LIBCMT:undname.obj
 0001:00094a50       ?getStringHelper@@YAPADPAD00H@Z 10095a50 f i LIBCMT:undname.obj
 0001:00094a85       ?getSymbolName@UnDecorator@@CA?AVDName@@XZ 10095a85 f i LIBCMT:undname.obj
 0001:00094acd       ?getTemplateArgumentList@UnDecorator@@CA?AVDName@@XZ 10095acd f   LIBCMT:undname.obj
 0001:00094d46       ?getTemplateConstant@UnDecorator@@CA?AVDName@@XZ 10095d46 f   LIBCMT:undname.obj
 0001:00095041       ?getTemplateName@UnDecorator@@CA?AVDName@@_N@Z 10096041 f   LIBCMT:undname.obj
 0001:0009519b       ?getThisType@UnDecorator@@CA?AVDName@@XZ 1009619b f i LIBCMT:undname.obj
 0001:000951d5       ?getThrowTypes@UnDecorator@@CA?AVDName@@XZ 100961d5 f   LIBCMT:undname.obj
 0001:0009525f       ?getTypeEncoding@UnDecorator@@CAHXZ 1009625f f i LIBCMT:undname.obj
 0001:0009574f       ?getVCallThunkType@UnDecorator@@CA?AVDName@@XZ 1009674f f i LIBCMT:undname.obj
 0001:0009578a       ?getVbTableType@UnDecorator@@CA?AVDName@@ABV2@@Z 1009678a f i LIBCMT:undname.obj
 0001:0009579f       ?getVdispMapType@UnDecorator@@CA?AVDName@@ABV2@@Z 1009679f f i LIBCMT:undname.obj
 0001:000957f5       ?getVfTableType@UnDecorator@@CA?AVDName@@ABV2@@Z 100967f5 f i LIBCMT:undname.obj
 0001:0009595a       ?getZName@UnDecorator@@CA?AVDName@@_N0@Z 1009695a f   LIBCMT:undname.obj
 0001:00095b84       ?haveTemplateParameters@UnDecorator@@SAHXZ 10096b84 f i LIBCMT:undname.obj
 0001:00095b8f       ?isArray@DName@@QBEHXZ     10096b8f f i LIBCMT:undname.obj
 0001:00095b99       ?isComArray@DName@@QBEHXZ  10096b99 f i LIBCMT:undname.obj
 0001:00095ba3       ?isEmpty@DName@@QBEHXZ     10096ba3 f i LIBCMT:undname.obj
 0001:00095bab       ?isFull@Replicator@@QBEHXZ 10096bab f i LIBCMT:undname.obj
 0001:00095bb4       ?isNoTE@DName@@QBEHXZ      10096bb4 f i LIBCMT:undname.obj
 0001:00095bbe       ?isPinPtr@DName@@QBEHXZ    10096bbe f i LIBCMT:undname.obj
 0001:00095bc8       ?isPtrRef@DName@@QBEHXZ    10096bc8 f i LIBCMT:undname.obj
 0001:00095bd2       ?isUDC@DName@@QBEHXZ       10096bd2 f i LIBCMT:undname.obj
 0001:00095be3       ?isUDTThunk@DName@@QBEHXZ  10096be3 f i LIBCMT:undname.obj
 0001:00095bf4       ?isVCallThunk@DName@@QBEHXZ 10096bf4 f i LIBCMT:undname.obj
 0001:00095bfe       ?isValid@DName@@QBEHXZ     10096bfe f i LIBCMT:undname.obj
 0001:00095c08       ?length@DName@@QBEHXZ      10096c08 f i LIBCMT:undname.obj
 0001:00095c15       ?length@DNameStatusNode@@UBEHXZ 10096c15 f i LIBCMT:undname.obj
 0001:00095c19       ?length@charNode@@UBEHXZ   10096c19 f i LIBCMT:undname.obj
 0001:00095c1d       ?length@pDNameNode@@UBEHXZ 10096c1d f i LIBCMT:undname.obj
 0001:00095c31       ?length@pairNode@@UBEHXZ   10096c31 f i LIBCMT:undname.obj
 0001:00095c5a       ?length@pcharNode@@UBEHXZ  10096c5a f i LIBCMT:undname.obj
 0001:00095c5e       ?make@DNameStatusNode@@SAPAV1@W4DNameStatus@@@Z 10096c5e f i LIBCMT:undname.obj
 0001:00095ce4       ?setIsArray@DName@@QAEXXZ  10096ce4 f i LIBCMT:undname.obj
 0001:00095cec       ?setIsComArray@DName@@QAEXXZ 10096cec f i LIBCMT:undname.obj
 0001:00095cf4       ?setIsNoTE@DName@@QAEXXZ   10096cf4 f i LIBCMT:undname.obj
 0001:00095cfc       ?setIsPinPtr@DName@@QAEXXZ 10096cfc f i LIBCMT:undname.obj
 0001:00095d04       ?setIsUDC@DName@@QAEXXZ    10096d04 f i LIBCMT:undname.obj
 0001:00095d11       ?setIsVCallThunk@DName@@QAEXXZ 10096d11 f i LIBCMT:undname.obj
 0001:00095d19       ?setPtrRef@DName@@QAEAAV1@XZ 10096d19 f i LIBCMT:undname.obj
 0001:00095d23       ?status@DName@@QBE?AW4DNameStatus@@XZ 10096d23 f i LIBCMT:undname.obj
 0001:00095d8b       ___unDName                 10096d8b f   LIBCMT:undname.obj
 0001:00095e2e       ___unDNameEx               10096e2e f   LIBCMT:undname.obj
 0001:000960f5       __strtol_l                 100970f5 f   LIBCMT:strtol.obj
 0001:00096110       __strtoul_l                10097110 f   LIBCMT:strtol.obj
 0001:0009612b       _strtol                    1009712b f   LIBCMT:strtol.obj
 0001:00096155       _strtoul                   10097155 f   LIBCMT:strtol.obj
 0001:0009617f       __frnd                     1009717f f   LIBCMT:frnd.obj
 0001:00096193       ___free_lconv_mon          10097193 f   LIBCMT:initmon.obj
 0001:0009628f       ___init_monetary           1009728f f   LIBCMT:initmon.obj
 0001:00096668       ___free_lconv_num          10097668 f   LIBCMT:initnum.obj
 0001:000966cf       ___init_numeric            100976cf f   LIBCMT:initnum.obj
 0001:0009690d       ___free_lc_time            1009790d f   LIBCMT:inittime.obj
 0001:00096c8d       ___init_time               10097c8d f   LIBCMT:inittime.obj
 0001:000974fc       _localeconv                100984fc f   LIBCMT:lconv.obj
 0001:00097522       __isctype                  10098522 f   LIBCMT:isctype.obj
 0001:00097551       __isctype_l                10098551 f   LIBCMT:isctype.obj
 0001:00097602       ___init_dummy              10098602 f   LIBCMT:wsetloca.obj
 0001:00097605       __locterm                  10098605 f   LIBCMT:wsetloca.obj
 0001:00097657       ____setlc_active_func      10098657 f   LIBCMT:wsetloca.obj
 0001:0009765d       ____unguarded_readlc_active_add_func 1009865d f   LIBCMT:wsetloca.obj
 0001:00097663       ___copy_locale_name        10098663 f   LIBCMT:wsetloca.obj
 0001:000976c7       ___create_locale           100986c7 f   LIBCMT:wsetloca.obj
 0001:000976d0       ___free_locale             100986d0 f   LIBCMT:wsetloca.obj
 0001:000976d5       ___get_current_locale      100986d5 f   LIBCMT:wsetloca.obj
 0001:000976da       ___lc_lctowcs              100986da f   LIBCMT:wsetloca.obj
 0001:00097748       ___lc_wcstolc              10098748 f   LIBCMT:wsetloca.obj
 0001:00097874       __configthreadlocale       10098874 f   LIBCMT:wsetloca.obj
 0001:000978fa       __create_locale            100988fa f   LIBCMT:wsetloca.obj
 0001:0009795c       __expandlocale             1009895c f   LIBCMT:wsetloca.obj
 0001:00097c53       __free_locale              10098c53 f   LIBCMT:wsetloca.obj
 0001:00097d0a       __get_current_locale       10098d0a f   LIBCMT:wsetloca.obj
 0001:00097db9       __wcreate_locale           10098db9 f   LIBCMT:wsetloca.obj
 0001:00097e90       __wcscats                  10098e90 f   LIBCMT:wsetloca.obj
 0001:00097ecf       __wsetlocale               10098ecf f   LIBCMT:wsetloca.obj
 0001:00098811       __CopyMan                  10099811 f i LIBCMT:intrncvt.obj
 0001:0009882e       __FillZeroMan              1009982e f i LIBCMT:intrncvt.obj
 0001:0009883d       __IncMan                   1009983d f i LIBCMT:intrncvt.obj
 0001:0009889f       __IsZeroMan                1009989f f i LIBCMT:intrncvt.obj
 0001:000988bc       __RoundMan                 100998bc f i LIBCMT:intrncvt.obj
 0001:000989bd       __ShrMan                   100999bd f i LIBCMT:intrncvt.obj
 0001:00098a4b       __ZeroTail                 10099a4b f i LIBCMT:intrncvt.obj
 0001:00098a93       ___addl                    10099a93 f i LIBCMT:intrncvt.obj
 0001:00098ab7       __ld12cvt                  10099ab7 f i LIBCMT:intrncvt.obj
 0001:00099022       __ld12tod                  1009a022 f   LIBCMT:intrncvt.obj
 0001:00099594       __ld12tof                  1009a594 f   LIBCMT:intrncvt.obj
 0001:00099b06       __ld12told                 1009ab06 f   LIBCMT:intrncvt.obj
 0001:00099bd5       ___STRINGTOLD_L            1009abd5 f   LIBCMT:strgtold.obj
 0001:00099c30       ___ld12mul                 1009ac30 f i LIBCMT:strgtold.obj
 0001:00099efc       ___multtenpow12            1009aefc f i LIBCMT:strgtold.obj
 0001:0009a24f       ___shl_12                  1009b24f f i LIBCMT:strgtold.obj
 0001:0009a280       ___shr_12                  1009b280 f i LIBCMT:strgtold.obj
 0001:0009a2b0       ___strgtold12_l            1009b2b0 f   LIBCMT:strgtold.obj
 0001:0009aa58       _$I10_OUTPUT               1009ba58 f   LIBCMT:x10fout.obj
 0001:0009b42c       ___add_12                  1009c42c f i LIBCMT:x10fout.obj
 0001:0009b49e       ___pctype_func             1009c49e f   LIBCMT:ctype.obj
 0001:0009b4c7       ___pwctype_func            1009c4c7 f   LIBCMT:ctype.obj
 0001:0009b607       ___control87_2             1009c607 f   LIBCMT:ieee87.obj
 0001:0009bc7b       __clearfp                  1009cc7b f   LIBCMT:ieee87.obj
 0001:0009bd5b       __control87                1009cd5b f i LIBCMT:ieee87.obj
 0001:0009c05d       __controlfp                1009d05d f   LIBCMT:ieee87.obj
 0001:0009c368       __fpreset                  1009d368 f   LIBCMT:ieee87.obj
 0001:0009c435       __set_controlfp            1009d435 f   LIBCMT:ieee87.obj
 0001:0009c4a8       __statusfp                 1009d4a8 f   LIBCMT:ieee87.obj
 0001:0009c542       __statusfp2                1009d542 f   LIBCMT:ieee87.obj
 0001:0009c5b0       __alloca_probe_16          1009d5b0 f   LIBCMT:alloca16.obj
 0001:0009c5c6       __alloca_probe_8           1009d5c6     LIBCMT:alloca16.obj
 0001:0009c5dc       _wcsnlen                   1009d5dc f   LIBCMT:wcslen_s.obj
 0001:0009c683       __wopen                    1009d683 f   LIBCMT:wopen.obj
 0001:0009c733       __wsopen                   1009d733 f   LIBCMT:wopen.obj
 0001:0009c766       __wsopen_helper            1009d766 f   LIBCMT:wopen.obj
 0001:0009c82f       __wsopen_nolock            1009d82f f   LIBCMT:wopen.obj
 0001:0009cf82       __wsopen_s                 1009df82 f   LIBCMT:wopen.obj
 0001:0009cfa0       _strncmp                   1009dfa0 f   LIBCMT:strncmp.obj
 0001:0009d018       __strnicmp                 1009e018 f   LIBCMT:strnicmp.obj
 0001:0009d083       __strnicmp_l               1009e083 f   LIBCMT:strnicmp.obj
 0001:0009d134       __iswctype_l               1009e134 f   LIBCMT:iswctype.obj
 0001:0009d146       _is_wctype                 1009e146 f   LIBCMT:iswctype.obj
 0001:0009d14f       _iswctype                  1009e14f f   LIBCMT:iswctype.obj
 0001:0009d1a5       ____lc_codepage_func       1009e1a5 f   LIBCMT:initctyp.obj
 0001:0009d1cb       ____lc_collate_cp_func     1009e1cb f   LIBCMT:initctyp.obj
 0001:0009d1f1       ____lc_locale_name_func    1009e1f1 f   LIBCMT:initctyp.obj
 0001:0009d219       ____mb_cur_max_func        1009e219 f   LIBCMT:initctyp.obj
 0001:0009d23f       ____mb_cur_max_l_func      1009e23f f   LIBCMT:initctyp.obj
 0001:0009d256       ___init_ctype              1009e256 f   LIBCMT:initctyp.obj
 0001:0009d5ee       ___termconout              1009e5ee f   LIBCMT:initcon.obj
 0001:0009d605       ___initconout              1009e605 f   LIBCMT:initcon.obj
 0001:0009d624       __fputwc_nolock            1009e624 f   LIBCMT:fputwc.obj
 0001:0009d7aa       _fputwc                    1009e7aa f   LIBCMT:fputwc.obj
 0001:0009d821       _putwc                     1009e821 f   LIBCMT:fputwc.obj
 0001:0009da0b       __wcstol_l                 1009ea0b f   LIBCMT:wcstol.obj
 0001:0009da23       __wcstoul_l                1009ea23 f   LIBCMT:wcstol.obj
 0001:0009da3b       _wcstol                    1009ea3b f   LIBCMT:wcstol.obj
 0001:0009da53       _wcstoul                   1009ea53 f   LIBCMT:wcstol.obj
 0001:0009da6b       __87except                 1009ea6b f   LIBCMT:87except.obj
 0001:0009db74       __atoi64                   1009eb74 f   LIBCMT:atox.obj
 0001:0009db88       __atoi64_l                 1009eb88 f   LIBCMT:atox.obj
 0001:0009db9f       __atoi_l                   1009eb9f f   LIBCMT:atox.obj
 0001:0009dba8       __atol_l                   1009eba8 f   LIBCMT:atox.obj
 0001:0009dbbf       __atoll_l                  1009ebbf f   LIBCMT:atox.obj
 0001:0009dbd6       _atoi                      1009ebd6 f   LIBCMT:atox.obj
 0001:0009dbdf       _atol                      1009ebdf f   LIBCMT:atox.obj
 0001:0009dbf3       _atoll                     1009ebf3 f   LIBCMT:atox.obj
 0001:0009dc07       ___init_collate            1009ec07 f   LIBCMT:initcoll.obj
 0001:0009dd27       _memcmp                    1009ed27 f   LIBCMT:memcmp.obj
 0001:000a0c3b       _wcscmp                    100a1c3b f   LIBCMT:wcscmp.obj
 0001:000a0c79       _wcscspn                   100a1c79 f   LIBCMT:wcscspn.obj
 0001:000a0cc4       _wcsncmp                   100a1cc4 f   LIBCMT:wcsncmp.obj
 0001:000a0cfa       _wcspbrk                   100a1cfa f   LIBCMT:wcspbrk.obj
 0001:000a12fe       ___get_qualified_locale    100a22fe f   LIBCMT:getqloc.obj
 0001:000a1b6e       ___get_qualified_locale_downlevel 100a2b6e f   LIBCMT:getqloc_downlevel.obj
 0001:000a1d8a       ___mtold12                 100a2d8a f   LIBCMT:mantold.obj
 0001:000a1f6a       __chsize                   100a2f6a f   LIBCMT:chsize.obj
 0001:000a1f84       __chsize_nolock            100a2f84 f   LIBCMT:chsize.obj
 0001:000a213a       __chsize_s                 100a313a f   LIBCMT:chsize.obj
 0001:000a2228       __get_fmode                100a3228 f   LIBCMT:setmode.obj
 0001:000a2252       __set_fmode                100a3252 f   LIBCMT:setmode.obj
 0001:000a228d       __setmode                  100a328d f   LIBCMT:setmode.obj
 0001:000a2392       __setmode_nolock           100a3392 f   LIBCMT:setmode.obj
 0001:000a2460       ___ascii_strnicmp          100a3460 f   LIBCMT:_strnicm.obj
 0001:000a24c1       __flswbuf                  100a34c1 f   LIBCMT:_flswbuf.obj
 0001:000a2623       __wchartodigit             100a3623 f   LIBCMT:wchtodig.obj
 0001:000a2a32       __strtof_l                 100a3a32 f   LIBCMT:strtoq.obj
 0001:000a2a52       __strtoi64                 100a3a52 f   LIBCMT:strtoq.obj
 0001:000a2a7c       __strtoi64_l               100a3a7c f   LIBCMT:strtoq.obj
 0001:000a2a97       __strtoimax_l              100a3a97 f   LIBCMT:strtoq.obj
 0001:000a2aa0       __strtold_l                100a3aa0 f   LIBCMT:strtoq.obj
 0001:000a2aa9       __strtoll_l                100a3aa9 f   LIBCMT:strtoq.obj
 0001:000a2ab2       __strtoui64                100a3ab2 f   LIBCMT:strtoq.obj
 0001:000a2adc       __strtoui64_l              100a3adc f   LIBCMT:strtoq.obj
 0001:000a2af7       __strtoull_l               100a3af7 f   LIBCMT:strtoq.obj
 0001:000a2b00       __strtoumax_l              100a3b00 f   LIBCMT:strtoq.obj
 0001:000a2b09       _strtof                    100a3b09 f   LIBCMT:strtoq.obj
 0001:000a2b28       _strtoimax                 100a3b28 f   LIBCMT:strtoq.obj
 0001:000a2b31       _strtold                   100a3b31 f   LIBCMT:strtoq.obj
 0001:000a2b3a       _strtoll                   100a3b3a f   LIBCMT:strtoq.obj
 0001:000a2b43       _strtoull                  100a3b43 f   LIBCMT:strtoq.obj
 0001:000a2b4c       _strtoumax                 100a3b4c f   LIBCMT:strtoq.obj
 0001:000a2b55       __wtoi                     100a3b55 f   LIBCMT:wtox.obj
 0001:000a2b5e       __wtoi64                   100a3b5e f   LIBCMT:wtox.obj
 0001:000a2b72       __wtoi64_l                 100a3b72 f   LIBCMT:wtox.obj
 0001:000a2b89       __wtoi_l                   100a3b89 f   LIBCMT:wtox.obj
 0001:000a2b92       __wtol                     100a3b92 f   LIBCMT:wtox.obj
 0001:000a2ba6       __wtol_l                   100a3ba6 f   LIBCMT:wtox.obj
 0001:000a2bbd       __wtoll                    100a3bbd f   LIBCMT:wtox.obj
 0001:000a2bd1       __wtoll_l                  100a3bd1 f   LIBCMT:wtox.obj
 0001:000a2be8       _wcschr                    100a3be8 f   LIBCMT:wcschr.obj
 0001:000a2c96       __wcsicmp                  100a3c96 f   LIBCMT:wcsicmp.obj
 0001:000a2d29       __wcsicmp_l                100a3d29 f   LIBCMT:wcsicmp.obj
 0001:000a2e04       __wcsnicmp                 100a3e04 f   LIBCMT:wcsnicmp.obj
 0001:000a2eba       __wcsnicmp_l               100a3eba f   LIBCMT:wcsnicmp.obj
 0001:000a2fb3       __strtod_l                 100a3fb3 f   LIBCMT:strtod.obj
 0001:000a30ca       _strtod                    100a40ca f   LIBCMT:strtod.obj
 0001:000a30e0       __allmul                   100a40e0 f   LIBCMT:llmul.obj
 0001:000a33e4       __wcstof_l                 100a43e4 f   LIBCMT:wcstoq.obj
 0001:000a3497       __wcstoi64                 100a4497 f   LIBCMT:wcstoq.obj
 0001:000a34c1       __wcstoi64_l               100a44c1 f   LIBCMT:wcstoq.obj
 0001:000a34dc       __wcstoimax_l              100a44dc f   LIBCMT:wcstoq.obj
 0001:000a34e5       __wcstold_l                100a44e5 f   LIBCMT:wcstoq.obj
 0001:000a34ee       __wcstoll_l                100a44ee f   LIBCMT:wcstoq.obj
 0001:000a34f7       __wcstoui64                100a44f7 f   LIBCMT:wcstoq.obj
 0001:000a3521       __wcstoui64_l              100a4521 f   LIBCMT:wcstoq.obj
 0001:000a353c       __wcstoull_l               100a453c f   LIBCMT:wcstoq.obj
 0001:000a3545       __wcstoumax_l              100a4545 f   LIBCMT:wcstoq.obj
 0001:000a354e       _wcstof                    100a454e f   LIBCMT:wcstoq.obj
 0001:000a3563       _wcstoimax                 100a4563 f   LIBCMT:wcstoq.obj
 0001:000a356c       _wcstold                   100a456c f   LIBCMT:wcstoq.obj
 0001:000a3575       _wcstoll                   100a4575 f   LIBCMT:wcstoq.obj
 0001:000a357e       _wcstoull                  100a457e f   LIBCMT:wcstoq.obj
 0001:000a3587       _wcstoumax                 100a4587 f   LIBCMT:wcstoq.obj
 0001:000a3590       __towlower_l               100a4590 f   LIBCMT:towlower.obj
 0001:000a3641       _towlower                  100a4641 f   LIBCMT:towlower.obj
 0001:000a3652       __fltin2                   100a4652 f   LIBCMT:cfin.obj
 0001:000a3700       __wcstod_l                 100a4700 f   LIBCMT:wcstod.obj
 0001:000a37fb       _wcstod                    100a47fb f   LIBCMT:wcstod.obj
 0001:000a3810       ___crtLCMapStringW         100a4810 f   LIBCMT:w_map.obj
 0001:000a383f       __wfltin2                  100a483f f   LIBCMT:wcfin.obj
 0001:000a38e8       ___WSTRINGTOLD_L           100a48e8 f   LIBCMT:wstrgtold.obj
 0001:000a3943       ___wstrgtold12_l           100a4943 f   LIBCMT:wstrgtold.obj
 0001:000a4193       ??0bad_function_call@std@@QAE@ABV01@@Z 100a5193 f i libcpmt:xthrow.obj
 0001:000a41ae       ??0bad_function_call@std@@QAE@PBD@Z 100a51ae f i libcpmt:xthrow.obj
 0001:000a41c2       ??0length_error@std@@QAE@ABV01@@Z 100a51c2 f i libcpmt:xthrow.obj
 0001:000a41dd       ??0length_error@std@@QAE@PBD@Z 100a51dd f i libcpmt:xthrow.obj
 0001:000a41ff       ??0out_of_range@std@@QAE@ABV01@@Z 100a51ff f i libcpmt:xthrow.obj
 0001:000a421a       ??0out_of_range@std@@QAE@PBD@Z 100a521a f i libcpmt:xthrow.obj
 0001:000a423c       ??0overflow_error@std@@QAE@ABV01@@Z 100a523c f i libcpmt:xthrow.obj
 0001:000a4257       ??0overflow_error@std@@QAE@PBD@Z 100a5257 f i libcpmt:xthrow.obj
 0001:000a4279       ??0regex_error@std@@QAE@ABV01@@Z 100a5279 f i libcpmt:xthrow.obj
 0001:000a429d       ??0regex_error@std@@QAE@W4error_type@regex_constants@1@@Z 100a529d f i libcpmt:xthrow.obj
 0001:000a42cd       ??1bad_function_call@std@@UAE@XZ 100a52cd f i libcpmt:xthrow.obj
 0001:000a42d2       ??1length_error@std@@UAE@XZ 100a52d2 f i libcpmt:xthrow.obj
 0001:000a42d7       ??1out_of_range@std@@UAE@XZ 100a52d7 f i libcpmt:xthrow.obj
 0001:000a42dc       ??1overflow_error@std@@UAE@XZ 100a52dc f i libcpmt:xthrow.obj
 0001:000a42e1       ??1regex_error@std@@UAE@XZ 100a52e1 f i libcpmt:xthrow.obj
 0001:000a42e6       ??_Gbad_function_call@std@@UAEPAXI@Z 100a52e6 f i libcpmt:xthrow.obj
 0001:000a42e6       ??_Ebad_function_call@std@@UAEPAXI@Z 100a52e6 f i libcpmt:xthrow.obj
 0001:000a4305       ??_Elength_error@std@@UAEPAXI@Z 100a5305 f i libcpmt:xthrow.obj
 0001:000a4305       ??_Glength_error@std@@UAEPAXI@Z 100a5305 f i libcpmt:xthrow.obj
 0001:000a4324       ??_Gout_of_range@std@@UAEPAXI@Z 100a5324 f i libcpmt:xthrow.obj
 0001:000a4324       ??_Eout_of_range@std@@UAEPAXI@Z 100a5324 f i libcpmt:xthrow.obj
 0001:000a4343       ??_Goverflow_error@std@@UAEPAXI@Z 100a5343 f i libcpmt:xthrow.obj
 0001:000a4343       ??_Eoverflow_error@std@@UAEPAXI@Z 100a5343 f i libcpmt:xthrow.obj
 0001:000a4362       ??_Gregex_error@std@@UAEPAXI@Z 100a5362 f i libcpmt:xthrow.obj
 0001:000a4362       ??_Eregex_error@std@@UAEPAXI@Z 100a5362 f i libcpmt:xthrow.obj
 0001:000a4381       ?_Stringify@regex_error@std@@CAPBDW4error_type@regex_constants@2@@Z 100a5381 f i libcpmt:xthrow.obj
 0001:000a4441       ?_Xbad_alloc@std@@YAXXZ    100a5441 f   libcpmt:xthrow.obj
 0001:000a4472       ?_Xbad_function_call@std@@YAXXZ 100a5472 f   libcpmt:xthrow.obj
 0001:000a4496       ?_Xinvalid_argument@std@@YAXPBD@Z 100a5496 f   libcpmt:xthrow.obj
 0001:000a44c4       ?_Xlength_error@std@@YAXPBD@Z 100a54c4 f   libcpmt:xthrow.obj
 0001:000a44f2       ?_Xout_of_range@std@@YAXPBD@Z 100a54f2 f   libcpmt:xthrow.obj
 0001:000a4520       ?_Xoverflow_error@std@@YAXPBD@Z 100a5520 f   libcpmt:xthrow.obj
 0001:000a454e       ?_Xregex_error@std@@YAXW4error_type@regex_constants@1@@Z 100a554e f   libcpmt:xthrow.obj
 0001:000a456e       ?_Xruntime_error@std@@YAXPBD@Z 100a556e f   libcpmt:xthrow.obj
 0001:000a459c       ?what@bad_function_call@std@@UBEPBDXZ 100a559c f i libcpmt:xthrow.obj
 0001:000a45a2       ?_Syserror_map@std@@YAPBDH@Z 100a55a2 f   libcpmt:syserror.obj
 0001:000a45cc       ?_Winerror_map@std@@YAPBDH@Z 100a55cc f   libcpmt:syserror.obj
 0001:000a45f6       ??0_Init_locks@std@@QAE@XZ 100a55f6 f   libcpmt:xlock.obj
 0001:000a4624       ??0_Lockit@std@@QAE@H@Z    100a5624 f   libcpmt:xlock.obj
 0001:000a4657       ??0_Lockit@std@@QAE@XZ     100a5657 f   libcpmt:xlock.obj
 0001:000a4669       ??1_Init_locks@std@@QAE@XZ 100a5669 f   libcpmt:xlock.obj
 0001:000a4691       ??1_Lockit@std@@QAE@XZ     100a5691 f   libcpmt:xlock.obj
 0001:000a46b5       ?_Init_locks_ctor@_Init_locks@std@@CAXPAV12@@Z 100a56b5 f   libcpmt:xlock.obj
 0001:000a46dd       ?_Init_locks_dtor@_Init_locks@std@@CAXPAV12@@Z 100a56dd f   libcpmt:xlock.obj
 0001:000a4705       ?_Lockit_ctor@_Lockit@std@@CAXPAV12@@Z 100a5705 f   libcpmt:xlock.obj
 0001:000a4711       ?_Lockit_ctor@_Lockit@std@@CAXPAV12@H@Z 100a5711 f   libcpmt:xlock.obj
 0001:000a473d       ?_Lockit_ctor@_Lockit@std@@SAXH@Z 100a573d f   libcpmt:xlock.obj
 0001:000a4764       ?_Lockit_dtor@_Lockit@std@@CAXPAV12@@Z 100a5764 f   libcpmt:xlock.obj
 0001:000a477b       ?_Lockit_dtor@_Lockit@std@@SAXH@Z 100a577b f   libcpmt:xlock.obj
 0001:000a47a2       ?uncaught_exception@std@@YA_NXZ 100a57a2 f   libcpmt:uncaught.obj
 0001:000a47a7       __Getctype                 100a57a7 f   libcpmt:_tolower.obj
 0001:000a4813       __Tolower                  100a5813 f   libcpmt:_tolower.obj
 0001:000a4912       __Toupper                  100a5912 f   libcpmt:_toupper.obj
 0001:000a4a11       ??0?$_Yarn@D@std@@QAE@PBD@Z 100a5a11 f i libcpmt:locale0.obj
 0001:000a4a2d       ??0_Fac_node@std@@QAE@PAU01@PAV_Facet_base@1@@Z 100a5a2d f i libcpmt:locale0.obj
 0001:000a4a41       ??0_Locimp@locale@std@@AAE@ABV012@@Z 100a5a41 f i libcpmt:locale0.obj
 0001:000a4aab       ??0_Locimp@locale@std@@AAE@_N@Z 100a5aab f i libcpmt:locale0.obj
 0001:000a4ae8       ??0locale@std@@AAE@PAV_Locimp@01@@Z 100a5ae8 f i libcpmt:locale0.obj
 0001:000a4af6       ??0locale@std@@QAE@W4_Uninitialized@1@@Z 100a5af6 f i libcpmt:locale0.obj
 0001:000a4afb       ??1_Fac_node@std@@QAE@XZ   100a5afb f i libcpmt:locale0.obj
 0001:000a4b10       ??1_Fac_tidy_reg_t@std@@QAE@XZ 100a5b10 f i libcpmt:locale0.obj
 0001:000a4b34       ??1_Locimp@locale@std@@MAE@XZ 100a5b34 f i libcpmt:locale0.obj
 0001:000a4b5f       ??4?$_Yarn@D@std@@QAEAAV01@PBD@Z 100a5b5f f i libcpmt:locale0.obj
 0001:000a4bb3       ??_G_Fac_node@std@@QAEPAXI@Z 100a5bb3 f i libcpmt:locale0.obj
 0001:000a4bd2       ??_G_Locimp@locale@std@@MAEPAXI@Z 100a5bd2 f i libcpmt:locale0.obj
 0001:000a4bd2       ??_E_Locimp@locale@std@@MAEPAXI@Z 100a5bd2 f i libcpmt:locale0.obj
 0001:000a4bf1       ?_C_str@?$_Yarn@D@std@@QBEPBDXZ 100a5bf1 f i libcpmt:locale0.obj
 0001:000a4bfb       ?_Empty@?$_Yarn@D@std@@QBE_NXZ 100a5bfb f i libcpmt:locale0.obj
 0001:000a4c03       ?_Facet_Register@std@@YAXPAV_Facet_base@1@@Z 100a5c03 f   libcpmt:locale0.obj
 0001:000a4c2b       ?_Getgloballocale@locale@std@@CAPAV_Locimp@12@XZ 100a5c2b f   libcpmt:locale0.obj
 0001:000a4c31       ?_Init@locale@std@@CAPAV_Locimp@12@_N@Z 100a5c31 f   libcpmt:locale0.obj
 0001:000a4cad       ?_Locimp_dtor@_Locimp@locale@std@@CAXPAV123@@Z 100a5cad f   libcpmt:locale0.obj
 0001:000a4d06       ?_Locinfo_ctor@_Locinfo@std@@SAXPAV12@PBD@Z 100a5d06 f   libcpmt:locale0.obj
 0001:000a4d51       ?_Locinfo_dtor@_Locinfo@std@@SAXPAV12@@Z 100a5d51 f   libcpmt:locale0.obj
 0001:000a4d73       ?_New_Locimp@_Locimp@locale@std@@CAPAV123@ABV123@@Z 100a5d73 f   libcpmt:locale0.obj
 0001:000a4da3       ?_New_Locimp@_Locimp@locale@std@@CAPAV123@_N@Z 100a5da3 f   libcpmt:locale0.obj
 0001:000a4dc2       ?_Setgloballocale@locale@std@@CAXPAX@Z 100a5dc2 f   libcpmt:locale0.obj
 0001:000a4dea       ?classic@locale@std@@SAABV12@XZ 100a5dea f   libcpmt:locale0.obj
 0001:000a4df8       ?empty@locale@std@@SA?AV12@XZ 100a5df8 f   libcpmt:locale0.obj
 0001:000a4e1b       __Deletegloballocale       100a5e1b f   libcpmt:locale0.obj
 0001:000a4e66       ?_Addstd@ios_base@std@@SAXPAV12@@Z 100a5e66 f   libcpmt:ios.obj
 0001:000a4eb7       ?_Callfns@ios_base@std@@AAEXW4event@12@@Z 100a5eb7 f i libcpmt:ios.obj
 0001:000a4edc       ?_Ios_base_dtor@ios_base@std@@CAXPAV12@@Z 100a5edc f   libcpmt:ios.obj
 0001:000a4f19       ?_Tidy@ios_base@std@@AAEXXZ 100a5f19 f i libcpmt:ios.obj
 0001:000a4f5b       ??$_Xfiopen@D@std@@YAPAU_iobuf@@PBDHH@Z 100a5f5b f i libcpmt:fiopen.obj
 0001:000a4ffd       ??$_Xfiopen@_W@std@@YAPAU_iobuf@@PB_WHH@Z 100a5ffd f i libcpmt:fiopen.obj
 0001:000a509f       ?_Fiopen@std@@YAPAU_iobuf@@PBDHH@Z 100a609f f   libcpmt:fiopen.obj
 0001:000a50a8       ?_Fiopen@std@@YAPAU_iobuf@@PBGHH@Z 100a60a8 f   libcpmt:fiopen.obj
 0001:000a50b1       ?_Fiopen@std@@YAPAU_iobuf@@PB_WHH@Z 100a60b1 f   libcpmt:fiopen.obj
 0001:000a50ba       ?_Xfsopen@std@@YAPAU_iobuf@@PBDHH@Z 100a60ba f   libcpmt:fiopen.obj
 0001:000a50d7       ?_Xfsopen@std@@YAPAU_iobuf@@PB_WHH@Z 100a60d7 f   libcpmt:fiopen.obj
 0001:000a50f4       __Mtxdst                   100a60f4 f   libcpmt:xmtx.obj
 0001:000a5102       __Mtxinit                  100a6102 f   libcpmt:xmtx.obj
 0001:000a5119       __Mtxlock                  100a6119 f   libcpmt:xmtx.obj
 0001:000a5127       __Mtxunlock                100a6127 f   libcpmt:xmtx.obj
 0001:000a5135       __Once                     100a6135 f   libcpmt:xmtx.obj
 0001:000a516a       ??1_Init_atexit@@QAE@XZ    100a616a f i libcpmt:iosptrs.obj
 0001:000a5193       ?_Atexit@@YAXP6AXXZ@Z      100a6193 f   libcpmt:iosptrs.obj
 0001:000a51c1       ??$?8DD@std@@YA_NABV?$allocator@D@0@0@Z 100a61c1 f i libcpmt:locale.obj
 0001:000a51c4       ??$?8DU?$char_traits@D@std@@@std@@YA_NABV?$istreambuf_iterator@DU?$char_traits@D@std@@@0@0@Z 100a61c4 f i libcpmt:locale.obj
 0001:000a51d4       ??$?8V?$allocator@D@std@@V01@@std@@YA_NABU?$_Wrap_alloc@V?$allocator@D@std@@@0@0@Z 100a61d4 f i libcpmt:locale.obj
 0001:000a51d7       ??$?9DD@std@@YA_NABV?$allocator@D@0@0@Z 100a61d7 f i libcpmt:locale.obj
 0001:000a51da       ??$?9DU?$char_traits@D@std@@@std@@YA_NABV?$istreambuf_iterator@DU?$char_traits@D@std@@@0@0@Z 100a61da f i libcpmt:locale.obj
 0001:000a51f3       ??$?9V?$allocator@D@std@@V01@@std@@YA_NABU?$_Wrap_alloc@V?$allocator@D@std@@@0@0@Z 100a61f3 f i libcpmt:locale.obj
 0001:000a51f6       ??$_Find_elem@D@std@@YAIPADD@Z 100a61f6 f i libcpmt:locale.obj
 0001:000a5218       ??$_Getloctxt@DV?$istreambuf_iterator@DU?$char_traits@D@std@@@std@@@std@@YAHAAV?$istreambuf_iterator@DU?$char_traits@D@std@@@0@0IPBD@Z 100a6218 f i libcpmt:locale.obj
 0001:000a5392       ??$_Getvals@D@?$numpunct@D@std@@IAEXDPBUlconv@@U_Cvtvec@@@Z 100a6392 f i libcpmt:locale.obj
 0001:000a53ab       ??$_Maklocchr@D@std@@YADDPADABU_Cvtvec@@@Z 100a63ab f i libcpmt:locale.obj
 0001:000a53b3       ??$_Maklocstr@D@std@@YAPADPBDPADABU_Cvtvec@@@Z 100a63b3 f i libcpmt:locale.obj
 0001:000a53e1       ??$use_facet@V?$num_get@DV?$istreambuf_iterator@DU?$char_traits@D@std@@@std@@@std@@@std@@YAABV?$num_get@DV?$istreambuf_iterator@DU?$char_traits@D@std@@@std@@@0@ABVlocale@0@@Z 100a63e1 f i libcpmt:locale.obj
 0001:000a547a       ??$use_facet@V?$num_put@DV?$ostreambuf_iterator@DU?$char_traits@D@std@@@std@@@std@@@std@@YAABV?$num_put@DV?$ostreambuf_iterator@DU?$char_traits@D@std@@@std@@@0@ABVlocale@0@@Z 100a647a f i libcpmt:locale.obj
 0001:000a5513       ??$use_facet@V?$numpunct@D@std@@@std@@YAABV?$numpunct@D@0@ABVlocale@0@@Z 100a6513 f i libcpmt:locale.obj
 0001:000a55ac       ??0?$num_get@DV?$istreambuf_iterator@DU?$char_traits@D@std@@@std@@@std@@QAE@ABV_Locinfo@1@I@Z 100a65ac f i libcpmt:locale.obj
 0001:000a55c1       ??0?$num_put@DV?$ostreambuf_iterator@DU?$char_traits@D@std@@@std@@@std@@QAE@ABV_Locinfo@1@I@Z 100a65c1 f i libcpmt:locale.obj
 0001:000a55d6       ??0?$numpunct@D@std@@QAE@ABV_Locinfo@1@I_N@Z 100a65d6 f i libcpmt:locale.obj
 0001:000a560c       ??1?$num_get@DV?$istreambuf_iterator@DU?$char_traits@D@std@@@std@@@std@@MAE@XZ 100a660c f i libcpmt:locale.obj
 0001:000a5613       ??1?$num_put@DV?$ostreambuf_iterator@DU?$char_traits@D@std@@@std@@@std@@MAE@XZ 100a6613 f i libcpmt:locale.obj
 0001:000a561a       ??1?$numpunct@D@std@@MAE@XZ 100a661a f i libcpmt:locale.obj
 0001:000a5630       ??4?$basic_string@DU?$char_traits@D@std@@V?$allocator@D@2@@std@@QAEAAV01@ABV01@@Z 100a6630 f i libcpmt:locale.obj
 0001:000a564e       ??4?$ostreambuf_iterator@DU?$char_traits@D@std@@@std@@QAEAAV01@D@Z 100a664e f i libcpmt:locale.obj
 0001:000a5672       ??A?$basic_string@DU?$char_traits@D@std@@V?$allocator@D@2@@std@@QAEAADI@Z 100a6672 f i libcpmt:locale.obj
 0001:000a5686       ??A?$basic_string@DU?$char_traits@D@std@@V?$allocator@D@2@@std@@QBEABDI@Z 100a6686 f i libcpmt:locale.obj
 0001:000a569a       ??D?$istreambuf_iterator@DU?$char_traits@D@std@@@std@@QBEDXZ 100a669a f i libcpmt:locale.obj
 0001:000a56ad       ??D?$ostreambuf_iterator@DU?$char_traits@D@std@@@std@@QAEAAV01@XZ 100a66ad f i libcpmt:locale.obj
 0001:000a56b0       ??E?$istreambuf_iterator@DU?$char_traits@D@std@@@std@@QAEAAV01@XZ 100a66b0 f i libcpmt:locale.obj
 0001:000a56bc       ??E?$ostreambuf_iterator@DU?$char_traits@D@std@@@std@@QAEAAV01@XZ 100a66bc f i libcpmt:locale.obj
 0001:000a56bf       ??Y?$basic_string@DU?$char_traits@D@std@@V?$allocator@D@2@@std@@QAEAAV01@ABV01@@Z 100a66bf f i libcpmt:locale.obj
 0001:000a56d2       ??Y?$basic_string@DU?$char_traits@D@std@@V?$allocator@D@2@@std@@QAEAAV01@D@Z 100a66d2 f i libcpmt:locale.obj
 0001:000a56e3       ??_G?$num_get@DV?$istreambuf_iterator@DU?$char_traits@D@std@@@std@@@std@@MAEPAXI@Z 100a66e3 f i libcpmt:locale.obj
 0001:000a56e3       ??_E?$num_get@DV?$istreambuf_iterator@DU?$char_traits@D@std@@@std@@@std@@MAEPAXI@Z 100a66e3 f i libcpmt:locale.obj
 0001:000a5703       ??_G?$num_put@DV?$ostreambuf_iterator@DU?$char_traits@D@std@@@std@@@std@@MAEPAXI@Z 100a6703 f i libcpmt:locale.obj
 0001:000a5703       ??_E?$num_put@DV?$ostreambuf_iterator@DU?$char_traits@D@std@@@std@@@std@@MAEPAXI@Z 100a6703 f i libcpmt:locale.obj
 0001:000a5723       ??_G?$numpunct@D@std@@MAEPAXI@Z 100a6723 f i libcpmt:locale.obj
 0001:000a5723       ??_E?$numpunct@D@std@@MAEPAXI@Z 100a6723 f i libcpmt:locale.obj
 0001:000a574e       ?_Addfac@_Locimp@locale@std@@AAEXPAVfacet@23@I@Z 100a674e f i libcpmt:locale.obj
 0001:000a5764       ?_Change_alloc@?$_String_alloc@$0A@U?$_String_base_types@DV?$allocator@D@std@@@std@@@std@@QAEXABU?$_Wrap_alloc@V?$allocator@D@std@@@2@@Z 100a6764 f i libcpmt:locale.obj
 0001:000a5767       ?_Ffmt@?$num_put@DV?$ostreambuf_iterator@DU?$char_traits@D@std@@@std@@@std@@ABAPADPADDH@Z 100a6767 f i libcpmt:locale.obj
 0001:000a57fc       ?_Fput@?$num_put@DV?$ostreambuf_iterator@DU?$char_traits@D@std@@@std@@@std@@ABA?AV?$ostreambuf_iterator@DU?$char_traits@D@std@@@2@V32@AAVios_base@2@DPBDIIII@Z 100a67fc f i libcpmt:locale.obj
 0001:000a5b54       ?_Getcat@?$num_get@DV?$istreambuf_iterator@DU?$char_traits@D@std@@@std@@@std@@SAIPAPBVfacet@locale@2@PBV42@@Z 100a6b54 f i libcpmt:locale.obj
 0001:000a5bbc       ?_Getcat@?$num_put@DV?$ostreambuf_iterator@DU?$char_traits@D@std@@@std@@@std@@SAIPAPBVfacet@locale@2@PBV42@@Z 100a6bbc f i libcpmt:locale.obj
 0001:000a5c24       ?_Getcat@?$numpunct@D@std@@SAIPAPBVfacet@locale@2@PBV42@@Z 100a6c24 f i libcpmt:locale.obj
 0001:000a5c9f       ?_Getcvt@_Locinfo@std@@QBE?AU_Cvtvec@@XZ 100a6c9f f i libcpmt:locale.obj
 0001:000a5cc5       ?_Getfalse@_Locinfo@std@@QBEPBDXZ 100a6cc5 f i libcpmt:locale.obj
 0001:000a5ccb       ?_Getffld@?$num_get@DV?$istreambuf_iterator@DU?$char_traits@D@std@@@std@@@std@@ABAHPADAAV?$istreambuf_iterator@DU?$char_traits@D@std@@@2@1AAVios_base@2@PAH@Z 100a6ccb f i libcpmt:locale.obj
 0001:000a6272       ?_Getffldx@?$num_get@DV?$istreambuf_iterator@DU?$char_traits@D@std@@@std@@@std@@ABAHPADAAV?$istreambuf_iterator@DU?$char_traits@D@std@@@2@1AAVios_base@2@PAH@Z 100a7272 f i libcpmt:locale.obj
 0001:000a6866       ?_Getifld@?$num_get@DV?$istreambuf_iterator@DU?$char_traits@D@std@@@std@@@std@@ABAHPADAAV?$istreambuf_iterator@DU?$char_traits@D@std@@@2@1HABVlocale@2@@Z 100a7866 f i libcpmt:locale.obj
 0001:000a6ba3       ?_Getlconv@_Locinfo@std@@QBEPBUlconv@@XZ 100a7ba3 f i libcpmt:locale.obj
 0001:000a6ba8       ?_Getname@_Locinfo@std@@QBEPBDXZ 100a7ba8 f i libcpmt:locale.obj
 0001:000a6bb3       ?_Gettrue@_Locinfo@std@@QBEPBDXZ 100a7bb3 f i libcpmt:locale.obj
 0001:000a6bb9       ?_Ifmt@?$num_put@DV?$ostreambuf_iterator@DU?$char_traits@D@std@@@std@@@std@@ABAPADPADPBDH@Z 100a7bb9 f i libcpmt:locale.obj
 0001:000a6c2f       ?_Inc@?$istreambuf_iterator@DU?$char_traits@D@std@@@std@@AAEXXZ 100a7c2f f i libcpmt:locale.obj
 0001:000a6c51       ?_Init@?$num_get@DV?$istreambuf_iterator@DU?$char_traits@D@std@@@std@@@std@@IAEXABV_Locinfo@2@@Z 100a7c51 f i libcpmt:locale.obj
 0001:000a6c54       ?_Init@?$num_put@DV?$ostreambuf_iterator@DU?$char_traits@D@std@@@std@@@std@@IAEXABV_Locinfo@2@@Z 100a7c54 f i libcpmt:locale.obj
 0001:000a6c57       ?_Init@?$numpunct@D@std@@IAEXABV_Locinfo@2@_N@Z 100a7c57 f i libcpmt:locale.obj
 0001:000a6d19       ?_Iput@?$num_put@DV?$ostreambuf_iterator@DU?$char_traits@D@std@@@std@@@std@@ABA?AV?$ostreambuf_iterator@DU?$char_traits@D@std@@@2@V32@AAVios_base@2@DPADI@Z 100a7d19 f i libcpmt:locale.obj
 0001:000a6fb8       ?_Locimp_Addfac@_Locimp@locale@std@@CAXPAV123@PAVfacet@23@I@Z 100a7fb8 f   libcpmt:locale.obj
 0001:000a7051       ?_Locimp_ctor@_Locimp@locale@std@@CAXPAV123@ABV123@@Z 100a8051 f   libcpmt:locale.obj
 0001:000a70f4       ?_Locinfo_Addcats@_Locinfo@std@@SAAAV12@PAV12@HPBD@Z 100a80f4 f   libcpmt:locale.obj
 0001:000a7190       ?_Locinfo_ctor@_Locinfo@std@@SAXPAV12@HPBD@Z 100a8190 f   libcpmt:locale.obj
 0001:000a71c6       ?_Makeloc@_Locimp@locale@std@@CAPAV123@ABV_Locinfo@3@HPAV123@PBV23@@Z 100a81c6 f   libcpmt:locale.obj
 0001:000a740e       ?_Peek@?$istreambuf_iterator@DU?$char_traits@D@std@@@std@@ABEDXZ 100a840e f i libcpmt:locale.obj
 0001:000a7432       ?_Put@?$num_put@DV?$ostreambuf_iterator@DU?$char_traits@D@std@@@std@@@std@@ABA?AV?$ostreambuf_iterator@DU?$char_traits@D@std@@@2@V32@PBDI@Z 100a8432 f i libcpmt:locale.obj
 0001:000a7463       ?_Rep@?$num_put@DV?$ostreambuf_iterator@DU?$char_traits@D@std@@@std@@@std@@ABA?AV?$ostreambuf_iterator@DU?$char_traits@D@std@@@2@V32@DI@Z 100a8463 f i libcpmt:locale.obj
 0001:000a748d       ?_Tidy@?$numpunct@D@std@@AAEXXZ 100a848d f i libcpmt:locale.obj
 0001:000a74ad       ?assign@?$basic_string@DU?$char_traits@D@std@@V?$allocator@D@2@@std@@QAEAAV12@$$QAV12@@Z 100a84ad f i libcpmt:locale.obj
 0001:000a74d2       ?assign@?$basic_string@DU?$char_traits@D@std@@V?$allocator@D@2@@std@@QAEAAV12@ABV12@@Z 100a84d2 f i libcpmt:locale.obj
 0001:000a74e5       ?decimal_point@?$numpunct@D@std@@QBEDXZ 100a84e5 f i libcpmt:locale.obj
 0001:000a74ea       ?do_decimal_point@?$numpunct@D@std@@MBEDXZ 100a84ea f i libcpmt:locale.obj
 0001:000a74ee       ?do_falsename@?$numpunct@D@std@@MBE?AV?$basic_string@DU?$char_traits@D@std@@V?$allocator@D@2@@2@XZ 100a84ee f i libcpmt:locale.obj
 0001:000a750a       ?do_get@?$num_get@DV?$istreambuf_iterator@DU?$char_traits@D@std@@@std@@@std@@MBE?AV?$istreambuf_iterator@DU?$char_traits@D@std@@@2@V32@0AAVios_base@2@AAHAAG@Z 100a850a f i libcpmt:locale.obj
 0001:000a75d3       ?do_get@?$num_get@DV?$istreambuf_iterator@DU?$char_traits@D@std@@@std@@@std@@MBE?AV?$istreambuf_iterator@DU?$char_traits@D@std@@@2@V32@0AAVios_base@2@AAHAAI@Z 100a85d3 f i libcpmt:locale.obj
 0001:000a7698       ?do_get@?$num_get@DV?$istreambuf_iterator@DU?$char_traits@D@std@@@std@@@std@@MBE?AV?$istreambuf_iterator@DU?$char_traits@D@std@@@2@V32@0AAVios_base@2@AAHAAJ@Z 100a8698 f i libcpmt:locale.obj
 0001:000a7748       ?do_get@?$num_get@DV?$istreambuf_iterator@DU?$char_traits@D@std@@@std@@@std@@MBE?AV?$istreambuf_iterator@DU?$char_traits@D@std@@@2@V32@0AAVios_base@2@AAHAAK@Z 100a8748 f i libcpmt:locale.obj
 0001:000a77f8       ?do_get@?$num_get@DV?$istreambuf_iterator@DU?$char_traits@D@std@@@std@@@std@@MBE?AV?$istreambuf_iterator@DU?$char_traits@D@std@@@2@V32@0AAVios_base@2@AAHAAM@Z 100a87f8 f i libcpmt:locale.obj
 0001:000a78b8       ?do_get@?$num_get@DV?$istreambuf_iterator@DU?$char_traits@D@std@@@std@@@std@@MBE?AV?$istreambuf_iterator@DU?$char_traits@D@std@@@2@V32@0AAVios_base@2@AAHAAN@Z 100a88b8 f i libcpmt:locale.obj
 0001:000a797b       ?do_get@?$num_get@DV?$istreambuf_iterator@DU?$char_traits@D@std@@@std@@@std@@MBE?AV?$istreambuf_iterator@DU?$char_traits@D@std@@@2@V32@0AAVios_base@2@AAHAAO@Z 100a897b f i libcpmt:locale.obj
 0001:000a7a3e       ?do_get@?$num_get@DV?$istreambuf_iterator@DU?$char_traits@D@std@@@std@@@std@@MBE?AV?$istreambuf_iterator@DU?$char_traits@D@std@@@2@V32@0AAVios_base@2@AAHAAPAX@Z 100a8a3e f i libcpmt:locale.obj
 0001:000a7af0       ?do_get@?$num_get@DV?$istreambuf_iterator@DU?$char_traits@D@std@@@std@@@std@@MBE?AV?$istreambuf_iterator@DU?$char_traits@D@std@@@2@V32@0AAVios_base@2@AAHAA_J@Z 100a8af0 f i libcpmt:locale.obj
 0001:000a7ba5       ?do_get@?$num_get@DV?$istreambuf_iterator@DU?$char_traits@D@std@@@std@@@std@@MBE?AV?$istreambuf_iterator@DU?$char_traits@D@std@@@2@V32@0AAVios_base@2@AAHAA_K@Z 100a8ba5 f i libcpmt:locale.obj
 0001:000a7c5a       ?do_get@?$num_get@DV?$istreambuf_iterator@DU?$char_traits@D@std@@@std@@@std@@MBE?AV?$istreambuf_iterator@DU?$char_traits@D@std@@@2@V32@0AAVios_base@2@AAHAA_N@Z 100a8c5a f i libcpmt:locale.obj
 0001:000a7e10       ?do_grouping@?$numpunct@D@std@@MBE?AV?$basic_string@DU?$char_traits@D@std@@V?$allocator@D@2@@2@XZ 100a8e10 f i libcpmt:locale.obj
 0001:000a7e2c       ?do_put@?$num_put@DV?$ostreambuf_iterator@DU?$char_traits@D@std@@@std@@@std@@MBE?AV?$ostreambuf_iterator@DU?$char_traits@D@std@@@2@V32@AAVios_base@2@DJ@Z 100a8e2c f i libcpmt:locale.obj
 0001:000a7e99       ?do_put@?$num_put@DV?$ostreambuf_iterator@DU?$char_traits@D@std@@@std@@@std@@MBE?AV?$ostreambuf_iterator@DU?$char_traits@D@std@@@2@V32@AAVios_base@2@DK@Z 100a8e99 f i libcpmt:locale.obj
 0001:000a7f06       ?do_put@?$num_put@DV?$ostreambuf_iterator@DU?$char_traits@D@std@@@std@@@std@@MBE?AV?$ostreambuf_iterator@DU?$char_traits@D@std@@@2@V32@AAVios_base@2@DN@Z 100a8f06 f i libcpmt:locale.obj
 0001:000a80be       ?do_put@?$num_put@DV?$ostreambuf_iterator@DU?$char_traits@D@std@@@std@@@std@@MBE?AV?$ostreambuf_iterator@DU?$char_traits@D@std@@@2@V32@AAVios_base@2@DO@Z 100a90be f i libcpmt:locale.obj
 0001:000a825c       ?do_put@?$num_put@DV?$ostreambuf_iterator@DU?$char_traits@D@std@@@std@@@std@@MBE?AV?$ostreambuf_iterator@DU?$char_traits@D@std@@@2@V32@AAVios_base@2@DPBX@Z 100a925c f i libcpmt:locale.obj
 0001:000a82b9       ?do_put@?$num_put@DV?$ostreambuf_iterator@DU?$char_traits@D@std@@@std@@@std@@MBE?AV?$ostreambuf_iterator@DU?$char_traits@D@std@@@2@V32@AAVios_base@2@D_J@Z 100a92b9 f i libcpmt:locale.obj
 0001:000a8329       ?do_put@?$num_put@DV?$ostreambuf_iterator@DU?$char_traits@D@std@@@std@@@std@@MBE?AV?$ostreambuf_iterator@DU?$char_traits@D@std@@@2@V32@AAVios_base@2@D_K@Z 100a9329 f i libcpmt:locale.obj
 0001:000a8399       ?do_put@?$num_put@DV?$ostreambuf_iterator@DU?$char_traits@D@std@@@std@@@std@@MBE?AV?$ostreambuf_iterator@DU?$char_traits@D@std@@@2@V32@AAVios_base@2@D_N@Z 100a9399 f i libcpmt:locale.obj
 0001:000a84f8       ?do_thousands_sep@?$numpunct@D@std@@MBEDXZ 100a94f8 f i libcpmt:locale.obj
 0001:000a84fc       ?do_truename@?$numpunct@D@std@@MBE?AV?$basic_string@DU?$char_traits@D@std@@V?$allocator@D@2@@2@XZ 100a94fc f i libcpmt:locale.obj
 0001:000a8518       ?equal@?$istreambuf_iterator@DU?$char_traits@D@std@@@std@@QBE_NABV12@@Z 100a9518 f i libcpmt:locale.obj
 0001:000a8553       ?falsename@?$numpunct@D@std@@QBE?AV?$basic_string@DU?$char_traits@D@std@@V?$allocator@D@2@@2@XZ 100a9553 f i libcpmt:locale.obj
 0001:000a856c       ?get_allocator@?$basic_string@DU?$char_traits@D@std@@V?$allocator@D@2@@std@@QBE?AV?$allocator@D@2@XZ 100a956c f i libcpmt:locale.obj
 0001:000a8576       ?global@locale@std@@SA?AV12@ABV12@@Z 100a9576 f   libcpmt:locale.obj
 0001:000a8630       ?grouping@?$numpunct@D@std@@QBE?AV?$basic_string@DU?$char_traits@D@std@@V?$allocator@D@2@@2@XZ 100a9630 f i libcpmt:locale.obj
 0001:000a8649       ?insert@?$basic_string@DU?$char_traits@D@std@@V?$allocator@D@2@@std@@QAEAAV12@IID@Z 100a9649 f i libcpmt:locale.obj
 0001:000a86f5       ?precision@ios_base@std@@QBE_JXZ 100a96f5 f i libcpmt:locale.obj
 0001:000a86fc       ?sbumpc@?$basic_streambuf@DU?$char_traits@D@std@@@std@@QAEHXZ 100a96fc f i libcpmt:locale.obj
 0001:000a8726       ?sgetc@?$basic_streambuf@DU?$char_traits@D@std@@@std@@QAEHXZ 100a9726 f i libcpmt:locale.obj
 0001:000a8745       ?thousands_sep@?$numpunct@D@std@@QBEDXZ 100a9745 f i libcpmt:locale.obj
 0001:000a874a       ?truename@?$numpunct@D@std@@QBE?AV?$basic_string@DU?$char_traits@D@std@@V?$allocator@D@2@@2@XZ 100a974a f i libcpmt:locale.obj
 0001:000a8763       ?widen@?$ctype@D@std@@QBEPBDPBD0PAD@Z 100a9763 f i libcpmt:locale.obj
 0001:000a876c       _ldexpf                    100a976c f i libcpmt:locale.obj
 0001:000a878a       _ldexpl                    100a978a f i libcpmt:locale.obj
 0001:000a87a2       __Getcvt                   100a97a2 f   libcpmt:xwctomb.obj
 0001:000a880b       __Wcrtomb                  100a980b f   libcpmt:xwctomb.obj
 0001:000a8869       ___Wcrtomb_lk              100a9869 f   libcpmt:xwctomb.obj
 0001:000a8872       ??$?8GG@std@@YA_NABV?$allocator@G@0@0@Z 100a9872 f i libcpmt:wlocale.obj
 0001:000a8875       ??$?8GU?$char_traits@G@std@@@std@@YA_NABV?$istreambuf_iterator@GU?$char_traits@G@std@@@0@0@Z 100a9875 f i libcpmt:wlocale.obj
 0001:000a8885       ??$?8V?$allocator@G@std@@V01@@std@@YA_NABU?$_Wrap_alloc@V?$allocator@G@std@@@0@0@Z 100a9885 f i libcpmt:wlocale.obj
 0001:000a8888       ??$?8V?$allocator@_W@std@@V01@@std@@YA_NABU?$_Wrap_alloc@V?$allocator@_W@std@@@0@0@Z 100a9888 f i libcpmt:wlocale.obj
 0001:000a888b       ??$?8_WU?$char_traits@_W@std@@@std@@YA_NABV?$istreambuf_iterator@_WU?$char_traits@_W@std@@@0@0@Z 100a988b f i libcpmt:wlocale.obj
 0001:000a889b       ??$?8_W_W@std@@YA_NABV?$allocator@_W@0@0@Z 100a989b f i libcpmt:wlocale.obj
 0001:000a889e       ??$?9GG@std@@YA_NABV?$allocator@G@0@0@Z 100a989e f i libcpmt:wlocale.obj
 0001:000a88a1       ??$?9GU?$char_traits@G@std@@@std@@YA_NABV?$istreambuf_iterator@GU?$char_traits@G@std@@@0@0@Z 100a98a1 f i libcpmt:wlocale.obj
 0001:000a88ba       ??$?9V?$allocator@G@std@@V01@@std@@YA_NABU?$_Wrap_alloc@V?$allocator@G@std@@@0@0@Z 100a98ba f i libcpmt:wlocale.obj
 0001:000a88bd       ??$?9V?$allocator@_W@std@@V01@@std@@YA_NABU?$_Wrap_alloc@V?$allocator@_W@std@@@0@0@Z 100a98bd f i libcpmt:wlocale.obj
 0001:000a88c0       ??$?9_WU?$char_traits@_W@std@@@std@@YA_NABV?$istreambuf_iterator@_WU?$char_traits@_W@std@@@0@0@Z 100a98c0 f i libcpmt:wlocale.obj
 0001:000a88d9       ??$?9_W_W@std@@YA_NABV?$allocator@_W@0@0@Z 100a98d9 f i libcpmt:wlocale.obj
 0001:000a88dc       ??$_Allocate@G@std@@YAPAGIPAG@Z 100a98dc f i libcpmt:wlocale.obj
 0001:000a8907       ??$_Allocate@_W@std@@YAPA_WIPA_W@Z 100a9907 f i libcpmt:wlocale.obj
 0001:000a8932       ??$_Copy_impl@PA_WV?$ostreambuf_iterator@GU?$char_traits@G@std@@@std@@@std@@YA?AV?$ostreambuf_iterator@GU?$char_traits@G@std@@@0@PA_W0V10@@Z 100a9932 f i libcpmt:wlocale.obj
 0001:000a8954       ??$_Copy_impl@PA_WV?$ostreambuf_iterator@GU?$char_traits@G@std@@@std@@@std@@YA?AV?$ostreambuf_iterator@GU?$char_traits@G@std@@@0@PA_W0V10@U_Nonscalar_ptr_iterator_tag@0@@Z 100a9954 f i libcpmt:wlocale.obj
 0001:000a8999       ??$_Copy_impl@PA_WV?$ostreambuf_iterator@_WU?$char_traits@_W@std@@@std@@@std@@YA?AV?$ostreambuf_iterator@_WU?$char_traits@_W@std@@@0@PA_W0V10@@Z 100a9999 f i libcpmt:wlocale.obj
 0001:000a89bb       ??$_Copy_impl@PA_WV?$ostreambuf_iterator@_WU?$char_traits@_W@std@@@std@@@std@@YA?AV?$ostreambuf_iterator@_WU?$char_traits@_W@std@@@0@PA_W0V10@U_Nonscalar_ptr_iterator_tag@0@@Z 100a99bb f i libcpmt:wlocale.obj
 0001:000a8a00       ??$_Find_elem@G@std@@YAIPAGG@Z 100a9a00 f i libcpmt:wlocale.obj
 0001:000a8a24       ??$_Find_elem@_W@std@@YAIPA_W_W@Z 100a9a24 f i libcpmt:wlocale.obj
 0001:000a8a48       ??$_Getloctxt@DV?$istreambuf_iterator@GU?$char_traits@G@std@@@std@@@std@@YAHAAV?$istreambuf_iterator@GU?$char_traits@G@std@@@0@0IPBD@Z 100a9a48 f i libcpmt:wlocale.obj
 0001:000a8bca       ??$_Getloctxt@DV?$istreambuf_iterator@_WU?$char_traits@_W@std@@@std@@@std@@YAHAAV?$istreambuf_iterator@_WU?$char_traits@_W@std@@@0@0IPBD@Z 100a9bca f i libcpmt:wlocale.obj
 0001:000a8d4c       ??$_Getloctxt@GV?$istreambuf_iterator@GU?$char_traits@G@std@@@std@@@std@@YAHAAV?$istreambuf_iterator@GU?$char_traits@G@std@@@0@0IPBG@Z 100a9d4c f i libcpmt:wlocale.obj
 0001:000a8ed6       ??$_Getloctxt@_WV?$istreambuf_iterator@_WU?$char_traits@_W@std@@@std@@@std@@YAHAAV?$istreambuf_iterator@_WU?$char_traits@_W@std@@@0@0IPB_W@Z 100a9ed6 f i libcpmt:wlocale.obj
 0001:000a9060       ??$_Getvals@G@?$_Mpunct@G@std@@IAEXGPBUlconv@@@Z 100aa060 f i libcpmt:wlocale.obj
 0001:000a90f2       ??$_Getvals@G@?$numpunct@G@std@@IAEXGPBUlconv@@U_Cvtvec@@@Z 100aa0f2 f i libcpmt:wlocale.obj
 0001:000a9156       ??$_Getvals@G@?$time_get@GV?$istreambuf_iterator@GU?$char_traits@G@std@@@std@@@std@@IAEXGABV_Locinfo@1@@Z 100aa156 f i libcpmt:wlocale.obj
 0001:000a91c3       ??$_Getvals@_W@?$_Mpunct@_W@std@@IAEX_WPBUlconv@@@Z 100aa1c3 f i libcpmt:wlocale.obj
 0001:000a922f       ??$_Getvals@_W@?$numpunct@_W@std@@IAEX_WPBUlconv@@U_Cvtvec@@@Z 100aa22f f i libcpmt:wlocale.obj
 0001:000a924d       ??$_Getvals@_W@?$time_get@_WV?$istreambuf_iterator@_WU?$char_traits@_W@std@@@std@@@std@@IAEX_WABV_Locinfo@1@@Z 100aa24d f i libcpmt:wlocale.obj
 0001:000a92a8       ??$_LStrcoll@G@std@@YAHPBG000PBU_Collvec@@@Z 100aa2a8 f i libcpmt:wlocale.obj
 0001:000a92f5       ??$_LStrcoll@_W@std@@YAHPB_W000PBU_Collvec@@@Z 100aa2f5 f i libcpmt:wlocale.obj
 0001:000a92fe       ??$_LStrxfrm@G@std@@YAIPAG0PBG1PBU_Collvec@@@Z 100aa2fe f i libcpmt:wlocale.obj
 0001:000a9331       ??$_LStrxfrm@_W@std@@YAIPA_W0PB_W1PBU_Collvec@@@Z 100aa331 f i libcpmt:wlocale.obj
 0001:000a933a       ??$_Maklocchr@G@std@@YAGDPAGABU_Cvtvec@@@Z 100aa33a f i libcpmt:wlocale.obj
 0001:000a9368       ??$_Maklocchr@_W@std@@YA_WDPA_WABU_Cvtvec@@@Z 100aa368 f i libcpmt:wlocale.obj
 0001:000a9396       ??$_Maklocstr@G@std@@YAPAGPBDPAGABU_Cvtvec@@@Z 100aa396 f i libcpmt:wlocale.obj
 0001:000a942f       ??$_Maklocstr@_W@std@@YAPA_WPBDPA_WABU_Cvtvec@@@Z 100aa42f f i libcpmt:wlocale.obj
 0001:000a94c8       ??$_Ptr_cat@PA_WV?$ostreambuf_iterator@GU?$char_traits@G@std@@@std@@@std@@YA?AU_Nonscalar_ptr_iterator_tag@0@AAPA_WAAV?$ostreambuf_iterator@GU?$char_traits@G@std@@@0@@Z 100aa4c8 f i libcpmt:wlocale.obj
 0001:000a94d3       ??$_Ptr_cat@PA_WV?$ostreambuf_iterator@_WU?$char_traits@_W@std@@@std@@@std@@YA?AU_Nonscalar_ptr_iterator_tag@0@AAPA_WAAV?$ostreambuf_iterator@_WU?$char_traits@_W@std@@@0@@Z 100aa4d3 f i libcpmt:wlocale.obj
 0001:000a94de       ??$_Rechecked@V?$ostreambuf_iterator@GU?$char_traits@G@std@@@std@@V12@@std@@YAAAV?$ostreambuf_iterator@GU?$char_traits@G@std@@@0@AAV10@V10@@Z 100aa4de f i libcpmt:wlocale.obj
 0001:000a94f1       ??$_Rechecked@V?$ostreambuf_iterator@_WU?$char_traits@_W@std@@@std@@V12@@std@@YAAAV?$ostreambuf_iterator@_WU?$char_traits@_W@std@@@0@AAV10@V10@@Z 100aa4f1 f i libcpmt:wlocale.obj
 0001:000a9504       ??$_Unchecked@PA_W@std@@YAPA_WPA_W@Z 100aa504 f i libcpmt:wlocale.obj
 0001:000a950c       ??$_Unchecked@V?$ostreambuf_iterator@GU?$char_traits@G@std@@@std@@@std@@YA?AV?$ostreambuf_iterator@GU?$char_traits@G@std@@@0@V10@@Z 100aa50c f i libcpmt:wlocale.obj
 0001:000a951f       ??$_Unchecked@V?$ostreambuf_iterator@_WU?$char_traits@_W@std@@@std@@@std@@YA?AV?$ostreambuf_iterator@_WU?$char_traits@_W@std@@@0@V10@@Z 100aa51f f i libcpmt:wlocale.obj
 0001:000a9532       ??$addressof@G@std@@YAPAGAAG@Z 100aa532 f i libcpmt:wlocale.obj
 0001:000a953a       ??$addressof@_W@std@@YAPA_WAA_W@Z 100aa53a f i libcpmt:wlocale.obj
 0001:000a9542       ??$assign@V?$_String_iterator@V?$_String_val@U?$_Simple_types@G@std@@@std@@@std@@@?$basic_string@GU?$char_traits@G@std@@V?$allocator@G@2@@std@@QAEAAV01@V?$_String_iterator@V?$_String_val@U?$_Simple_types@G@std@@@std@@@1@0@Z 100aa542 f i libcpmt:wlocale.obj
 0001:000a9574       ??$assign@V?$_String_iterator@V?$_String_val@U?$_Simple_types@_W@std@@@std@@@std@@@?$basic_string@_WU?$char_traits@_W@std@@V?$allocator@_W@2@@std@@QAEAAV01@V?$_String_iterator@V?$_String_val@U?$_Simple_types@_W@std@@@std@@@1@0@Z 100aa574 f i libcpmt:wlocale.obj
 0001:000a95a6       ??$construct@PAGAAPAG@?$_Wrap_alloc@V?$allocator@G@std@@@std@@QAEXPAPAGAAPAG@Z 100aa5a6 f i libcpmt:wlocale.obj
 0001:000a95bb       ??$construct@PAGAAPAG@?$allocator@G@std@@QAEXPAPAGAAPAG@Z 100aa5bb f i libcpmt:wlocale.obj
 0001:000a95d0       ??$construct@PAGAAPAG@?$allocator_traits@V?$allocator@G@std@@@std@@SAXAAV?$allocator@G@1@PAPAGAAPAG@Z 100aa5d0 f i libcpmt:wlocale.obj
 0001:000a95e3       ??$construct@PA_WAAPA_W@?$_Wrap_alloc@V?$allocator@_W@std@@@std@@QAEXPAPA_WAAPA_W@Z 100aa5e3 f i libcpmt:wlocale.obj
 0001:000a95f8       ??$construct@PA_WAAPA_W@?$allocator@_W@std@@QAEXPAPA_WAAPA_W@Z 100aa5f8 f i libcpmt:wlocale.obj
 0001:000a960d       ??$construct@PA_WAAPA_W@?$allocator_traits@V?$allocator@_W@std@@@std@@SAXAAV?$allocator@_W@1@PAPA_WAAPA_W@Z 100aa60d f i libcpmt:wlocale.obj
 0001:000a9620       ??$copy@PA_WV?$ostreambuf_iterator@GU?$char_traits@G@std@@@std@@@std@@YA?AV?$ostreambuf_iterator@GU?$char_traits@G@std@@@0@PA_W0V10@@Z 100aa620 f i libcpmt:wlocale.obj
 0001:000a9650       ??$copy@PA_WV?$ostreambuf_iterator@_WU?$char_traits@_W@std@@@std@@@std@@YA?AV?$ostreambuf_iterator@_WU?$char_traits@_W@std@@@0@PA_W0V10@@Z 100aa650 f i libcpmt:wlocale.obj
 0001:000a9680       ??$destroy@PAG@?$_Wrap_alloc@V?$allocator@G@std@@@std@@QAEXPAPAG@Z 100aa680 f i libcpmt:wlocale.obj
 0001:000a9683       ??$destroy@PAG@?$allocator@G@std@@QAEXPAPAG@Z 100aa683 f i libcpmt:wlocale.obj
 0001:000a9686       ??$destroy@PAG@?$allocator_traits@V?$allocator@G@std@@@std@@SAXAAV?$allocator@G@1@PAPAG@Z 100aa686 f i libcpmt:wlocale.obj
 0001:000a9687       ??$destroy@PA_W@?$_Wrap_alloc@V?$allocator@_W@std@@@std@@QAEXPAPA_W@Z 100aa687 f i libcpmt:wlocale.obj
 0001:000a968a       ??$destroy@PA_W@?$allocator@_W@std@@QAEXPAPA_W@Z 100aa68a f i libcpmt:wlocale.obj
 0001:000a968d       ??$destroy@PA_W@?$allocator_traits@V?$allocator@_W@std@@@std@@SAXAAV?$allocator@_W@1@PAPA_W@Z 100aa68d f i libcpmt:wlocale.obj
 0001:000a968e       ??$forward@AAPAG@std@@YAAAPAGAAPAG@Z 100aa68e f i libcpmt:wlocale.obj
 0001:000a9696       ??$forward@AAPA_W@std@@YAAAPA_WAAPA_W@Z 100aa696 f i libcpmt:wlocale.obj
 0001:000a969e       ??$forward@V?$basic_string@GU?$char_traits@G@std@@V?$allocator@G@2@@std@@@std@@YA$$QAV?$basic_string@GU?$char_traits@G@std@@V?$allocator@G@2@@0@AAV10@@Z 100aa69e f i libcpmt:wlocale.obj
 0001:000a96a6       ??$forward@V?$basic_string@_WU?$char_traits@_W@std@@V?$allocator@_W@2@@std@@@std@@YA$$QAV?$basic_string@_WU?$char_traits@_W@std@@V?$allocator@_W@2@@0@AAV10@@Z 100aa6a6 f i libcpmt:wlocale.obj
 0001:000a96ae       ??$use_facet@V?$codecvt@GDH@std@@@std@@YAABV?$codecvt@GDH@0@ABVlocale@0@@Z 100aa6ae f i libcpmt:wlocale.obj
 0001:000a9747       ??$use_facet@V?$codecvt@_WDH@std@@@std@@YAABV?$codecvt@_WDH@0@ABVlocale@0@@Z 100aa747 f i libcpmt:wlocale.obj
 0001:000a97e0       ??$use_facet@V?$collate@G@std@@@std@@YAABV?$collate@G@0@ABVlocale@0@@Z 100aa7e0 f i libcpmt:wlocale.obj
 0001:000a9879       ??$use_facet@V?$collate@_W@std@@@std@@YAABV?$collate@_W@0@ABVlocale@0@@Z 100aa879 f i libcpmt:wlocale.obj
 0001:000a9912       ??$use_facet@V?$ctype@G@std@@@std@@YAABV?$ctype@G@0@ABVlocale@0@@Z 100aa912 f i libcpmt:wlocale.obj
 0001:000a99ab       ??$use_facet@V?$ctype@_W@std@@@std@@YAABV?$ctype@_W@0@ABVlocale@0@@Z 100aa9ab f i libcpmt:wlocale.obj
 0001:000a9a44       ??$use_facet@V?$messages@G@std@@@std@@YAABV?$messages@G@0@ABVlocale@0@@Z 100aaa44 f i libcpmt:wlocale.obj
 0001:000a9add       ??$use_facet@V?$messages@_W@std@@@std@@YAABV?$messages@_W@0@ABVlocale@0@@Z 100aaadd f i libcpmt:wlocale.obj
 0001:000a9b76       ??$use_facet@V?$money_get@GV?$istreambuf_iterator@GU?$char_traits@G@std@@@std@@@std@@@std@@YAABV?$money_get@GV?$istreambuf_iterator@GU?$char_traits@G@std@@@std@@@0@ABVlocale@0@@Z 100aab76 f i libcpmt:wlocale.obj
 0001:000a9c0f       ??$use_facet@V?$money_get@_WV?$istreambuf_iterator@_WU?$char_traits@_W@std@@@std@@@std@@@std@@YAABV?$money_get@_WV?$istreambuf_iterator@_WU?$char_traits@_W@std@@@std@@@0@ABVlocale@0@@Z 100aac0f f i libcpmt:wlocale.obj
 0001:000a9ca8       ??$use_facet@V?$money_put@GV?$ostreambuf_iterator@GU?$char_traits@G@std@@@std@@@std@@@std@@YAABV?$money_put@GV?$ostreambuf_iterator@GU?$char_traits@G@std@@@std@@@0@ABVlocale@0@@Z 100aaca8 f i libcpmt:wlocale.obj
 0001:000a9d41       ??$use_facet@V?$money_put@_WV?$ostreambuf_iterator@_WU?$char_traits@_W@std@@@std@@@std@@@std@@YAABV?$money_put@_WV?$ostreambuf_iterator@_WU?$char_traits@_W@std@@@std@@@0@ABVlocale@0@@Z 100aad41 f i libcpmt:wlocale.obj
 0001:000a9dda       ??$use_facet@V?$moneypunct@G$00@std@@@std@@YAABV?$moneypunct@G$00@0@ABVlocale@0@@Z 100aadda f i libcpmt:wlocale.obj
 0001:000a9e73       ??$use_facet@V?$moneypunct@G$0A@@std@@@std@@YAABV?$moneypunct@G$0A@@0@ABVlocale@0@@Z 100aae73 f i libcpmt:wlocale.obj
 0001:000a9f0c       ??$use_facet@V?$moneypunct@_W$00@std@@@std@@YAABV?$moneypunct@_W$00@0@ABVlocale@0@@Z 100aaf0c f i libcpmt:wlocale.obj
 0001:000a9fa5       ??$use_facet@V?$moneypunct@_W$0A@@std@@@std@@YAABV?$moneypunct@_W$0A@@0@ABVlocale@0@@Z 100aafa5 f i libcpmt:wlocale.obj
 0001:000aa03e       ??$use_facet@V?$num_get@GV?$istreambuf_iterator@GU?$char_traits@G@std@@@std@@@std@@@std@@YAABV?$num_get@GV?$istreambuf_iterator@GU?$char_traits@G@std@@@std@@@0@ABVlocale@0@@Z 100ab03e f i libcpmt:wlocale.obj
 0001:000aa0d7       ??$use_facet@V?$num_get@_WV?$istreambuf_iterator@_WU?$char_traits@_W@std@@@std@@@std@@@std@@YAABV?$num_get@_WV?$istreambuf_iterator@_WU?$char_traits@_W@std@@@std@@@0@ABVlocale@0@@Z 100ab0d7 f i libcpmt:wlocale.obj
 0001:000aa170       ??$use_facet@V?$num_put@GV?$ostreambuf_iterator@GU?$char_traits@G@std@@@std@@@std@@@std@@YAABV?$num_put@GV?$ostreambuf_iterator@GU?$char_traits@G@std@@@std@@@0@ABVlocale@0@@Z 100ab170 f i libcpmt:wlocale.obj
 0001:000aa209       ??$use_facet@V?$num_put@_WV?$ostreambuf_iterator@_WU?$char_traits@_W@std@@@std@@@std@@@std@@YAABV?$num_put@_WV?$ostreambuf_iterator@_WU?$char_traits@_W@std@@@std@@@0@ABVlocale@0@@Z 100ab209 f i libcpmt:wlocale.obj
 0001:000aa2a2       ??$use_facet@V?$numpunct@G@std@@@std@@YAABV?$numpunct@G@0@ABVlocale@0@@Z 100ab2a2 f i libcpmt:wlocale.obj
 0001:000aa33b       ??$use_facet@V?$numpunct@_W@std@@@std@@YAABV?$numpunct@_W@0@ABVlocale@0@@Z 100ab33b f i libcpmt:wlocale.obj
 0001:000aa3d4       ??$use_facet@V?$time_get@GV?$istreambuf_iterator@GU?$char_traits@G@std@@@std@@@std@@@std@@YAABV?$time_get@GV?$istreambuf_iterator@GU?$char_traits@G@std@@@std@@@0@ABVlocale@0@@Z 100ab3d4 f i libcpmt:wlocale.obj
 0001:000aa46d       ??$use_facet@V?$time_get@_WV?$istreambuf_iterator@_WU?$char_traits@_W@std@@@std@@@std@@@std@@YAABV?$time_get@_WV?$istreambuf_iterator@_WU?$char_traits@_W@std@@@std@@@0@ABVlocale@0@@Z 100ab46d f i libcpmt:wlocale.obj
 0001:000aa506       ??$use_facet@V?$time_put@GV?$ostreambuf_iterator@GU?$char_traits@G@std@@@std@@@std@@@std@@YAABV?$time_put@GV?$ostreambuf_iterator@GU?$char_traits@G@std@@@std@@@0@ABVlocale@0@@Z 100ab506 f i libcpmt:wlocale.obj
 0001:000aa59f       ??$use_facet@V?$time_put@_WV?$ostreambuf_iterator@_WU?$char_traits@_W@std@@@std@@@std@@@std@@YAABV?$time_put@_WV?$ostreambuf_iterator@_WU?$char_traits@_W@std@@@std@@@0@ABVlocale@0@@Z 100ab59f f i libcpmt:wlocale.obj
 0001:000aa638       ??0?$_Mpunct@G@std@@QAE@ABV_Locinfo@1@I_N1@Z 100ab638 f i libcpmt:wlocale.obj
 0001:000aa674       ??0?$_Mpunct@_W@std@@QAE@ABV_Locinfo@1@I_N1@Z 100ab674 f i libcpmt:wlocale.obj
 0001:000aa6b0       ??0?$_String_alloc@$0A@U?$_String_base_types@GV?$allocator@G@std@@@std@@@std@@QAE@ABV?$allocator@G@1@@Z 100ab6b0 f i libcpmt:wlocale.obj
 0001:000aa6bd       ??0?$_String_alloc@$0A@U?$_String_base_types@_WV?$allocator@_W@std@@@std@@@std@@QAE@ABV?$allocator@_W@1@@Z 100ab6bd f i libcpmt:wlocale.obj
 0001:000aa6ca       ??0?$_String_const_iterator@V?$_String_val@U?$_Simple_types@G@std@@@std@@@std@@QAE@PBGPBU_Container_base0@1@@Z 100ab6ca f i libcpmt:wlocale.obj
 0001:000aa6d8       ??0?$_String_const_iterator@V?$_String_val@U?$_Simple_types@G@std@@@std@@@std@@QAE@XZ 100ab6d8 f i libcpmt:wlocale.obj
 0001:000aa6de       ??0?$_String_const_iterator@V?$_String_val@U?$_Simple_types@_W@std@@@std@@@std@@QAE@PB_WPBU_Container_base0@1@@Z 100ab6de f i libcpmt:wlocale.obj
 0001:000aa6ec       ??0?$_String_const_iterator@V?$_String_val@U?$_Simple_types@_W@std@@@std@@@std@@QAE@XZ 100ab6ec f i libcpmt:wlocale.obj
 0001:000aa6f2       ??0?$_String_iterator@V?$_String_val@U?$_Simple_types@G@std@@@std@@@std@@QAE@PAGPBU_Container_base0@1@@Z 100ab6f2 f i libcpmt:wlocale.obj
 0001:000aa700       ??0?$_String_iterator@V?$_String_val@U?$_Simple_types@_W@std@@@std@@@std@@QAE@PA_WPBU_Container_base0@1@@Z 100ab700 f i libcpmt:wlocale.obj
 0001:000aa70e       ??0?$_String_val@U?$_Simple_types@G@std@@@std@@QAE@XZ 100ab70e f i libcpmt:wlocale.obj
 0001:000aa719       ??0?$_String_val@U?$_Simple_types@_W@std@@@std@@QAE@XZ 100ab719 f i libcpmt:wlocale.obj
 0001:000aa724       ??0?$_Wrap_alloc@V?$allocator@G@std@@@std@@QAE@ABV?$allocator@G@1@@Z 100ab724 f i libcpmt:wlocale.obj
 0001:000aa729       ??0?$_Wrap_alloc@V?$allocator@G@std@@@std@@QAE@XZ 100ab729 f i libcpmt:wlocale.obj
 0001:000aa72c       ??0?$_Wrap_alloc@V?$allocator@_W@std@@@std@@QAE@ABV?$allocator@_W@1@@Z 100ab72c f i libcpmt:wlocale.obj
 0001:000aa731       ??0?$_Wrap_alloc@V?$allocator@_W@std@@@std@@QAE@XZ 100ab731 f i libcpmt:wlocale.obj
 0001:000aa734       ??0?$allocator@G@std@@QAE@ABV01@@Z 100ab734 f i libcpmt:wlocale.obj
 0001:000aa739       ??0?$allocator@G@std@@QAE@XZ 100ab739 f i libcpmt:wlocale.obj
 0001:000aa73c       ??0?$allocator@_W@std@@QAE@ABV01@@Z 100ab73c f i libcpmt:wlocale.obj
 0001:000aa741       ??0?$allocator@_W@std@@QAE@XZ 100ab741 f i libcpmt:wlocale.obj
 0001:000aa744       ??0?$basic_string@GU?$char_traits@G@std@@V?$allocator@G@2@@std@@QAE@$$QAV01@@Z 100ab744 f i libcpmt:wlocale.obj
 0001:000aa769       ??0?$basic_string@GU?$char_traits@G@std@@V?$allocator@G@2@@std@@QAE@ABV01@@Z 100ab769 f i libcpmt:wlocale.obj
 0001:000aa791       ??0?$basic_string@GU?$char_traits@G@std@@V?$allocator@G@2@@std@@QAE@IG@Z 100ab791 f i libcpmt:wlocale.obj
 0001:000aa7b9       ??0?$basic_string@GU?$char_traits@G@std@@V?$allocator@G@2@@std@@QAE@PBG@Z 100ab7b9 f i libcpmt:wlocale.obj
 0001:000aa7de       ??0?$basic_string@GU?$char_traits@G@std@@V?$allocator@G@2@@std@@QAE@PBGI@Z 100ab7de f i libcpmt:wlocale.obj
 0001:000aa806       ??0?$basic_string@GU?$char_traits@G@std@@V?$allocator@G@2@@std@@QAE@XZ 100ab806 f i libcpmt:wlocale.obj
 0001:000aa819       ??0?$basic_string@_WU?$char_traits@_W@std@@V?$allocator@_W@2@@std@@QAE@$$QAV01@@Z 100ab819 f i libcpmt:wlocale.obj
 0001:000aa83e       ??0?$basic_string@_WU?$char_traits@_W@std@@V?$allocator@_W@2@@std@@QAE@ABV01@@Z 100ab83e f i libcpmt:wlocale.obj
 0001:000aa866       ??0?$basic_string@_WU?$char_traits@_W@std@@V?$allocator@_W@2@@std@@QAE@I_W@Z 100ab866 f i libcpmt:wlocale.obj
 0001:000aa88e       ??0?$basic_string@_WU?$char_traits@_W@std@@V?$allocator@_W@2@@std@@QAE@PB_W@Z 100ab88e f i libcpmt:wlocale.obj
 0001:000aa8b3       ??0?$basic_string@_WU?$char_traits@_W@std@@V?$allocator@_W@2@@std@@QAE@PB_WI@Z 100ab8b3 f i libcpmt:wlocale.obj
 0001:000aa8db       ??0?$basic_string@_WU?$char_traits@_W@std@@V?$allocator@_W@2@@std@@QAE@XZ 100ab8db f i libcpmt:wlocale.obj
 0001:000aa8ee       ??0?$codecvt@GDH@std@@QAE@ABV_Locinfo@1@I@Z 100ab8ee f i libcpmt:wlocale.obj
 0001:000aa924       ??0?$codecvt@_WDH@std@@QAE@ABV_Locinfo@1@I@Z 100ab924 f i libcpmt:wlocale.obj
 0001:000aa95a       ??0?$collate@G@std@@QAE@ABV_Locinfo@1@I@Z 100ab95a f i libcpmt:wlocale.obj
 0001:000aa97e       ??0?$collate@_W@std@@QAE@ABV_Locinfo@1@I@Z 100ab97e f i libcpmt:wlocale.obj
 0001:000aa9a2       ??0?$ctype@G@std@@QAE@ABV_Locinfo@1@I@Z 100ab9a2 f i libcpmt:wlocale.obj
 0001:000aa9c3       ??0?$ctype@_W@std@@QAE@ABV_Locinfo@1@I@Z 100ab9c3 f i libcpmt:wlocale.obj
 0001:000aa9e4       ??0?$messages@G@std@@QAE@ABV_Locinfo@1@I@Z 100ab9e4 f i libcpmt:wlocale.obj
 0001:000aa9f9       ??0?$messages@_W@std@@QAE@ABV_Locinfo@1@I@Z 100ab9f9 f i libcpmt:wlocale.obj
 0001:000aaa0e       ??0?$money_get@GV?$istreambuf_iterator@GU?$char_traits@G@std@@@std@@@std@@QAE@ABV_Locinfo@1@I@Z 100aba0e f i libcpmt:wlocale.obj
 0001:000aaa23       ??0?$money_get@_WV?$istreambuf_iterator@_WU?$char_traits@_W@std@@@std@@@std@@QAE@ABV_Locinfo@1@I@Z 100aba23 f i libcpmt:wlocale.obj
 0001:000aaa38       ??0?$money_put@GV?$ostreambuf_iterator@GU?$char_traits@G@std@@@std@@@std@@QAE@ABV_Locinfo@1@I@Z 100aba38 f i libcpmt:wlocale.obj
 0001:000aaa4d       ??0?$money_put@_WV?$ostreambuf_iterator@_WU?$char_traits@_W@std@@@std@@@std@@QAE@ABV_Locinfo@1@I@Z 100aba4d f i libcpmt:wlocale.obj
 0001:000aaa62       ??0?$moneypunct@G$00@std@@QAE@ABV_Locinfo@1@I_N@Z 100aba62 f i libcpmt:wlocale.obj
 0001:000aaa85       ??0?$moneypunct@G$0A@@std@@QAE@ABV_Locinfo@1@I_N@Z 100aba85 f i libcpmt:wlocale.obj
 0001:000aaaa8       ??0?$moneypunct@_W$00@std@@QAE@ABV_Locinfo@1@I_N@Z 100abaa8 f i libcpmt:wlocale.obj
 0001:000aaacb       ??0?$moneypunct@_W$0A@@std@@QAE@ABV_Locinfo@1@I_N@Z 100abacb f i libcpmt:wlocale.obj
 0001:000aaaee       ??0?$num_get@GV?$istreambuf_iterator@GU?$char_traits@G@std@@@std@@@std@@QAE@ABV_Locinfo@1@I@Z 100abaee f i libcpmt:wlocale.obj
 0001:000aab03       ??0?$num_get@_WV?$istreambuf_iterator@_WU?$char_traits@_W@std@@@std@@@std@@QAE@ABV_Locinfo@1@I@Z 100abb03 f i libcpmt:wlocale.obj
 0001:000aab18       ??0?$num_put@GV?$ostreambuf_iterator@GU?$char_traits@G@std@@@std@@@std@@QAE@ABV_Locinfo@1@I@Z 100abb18 f i libcpmt:wlocale.obj
 0001:000aab2d       ??0?$num_put@_WV?$ostreambuf_iterator@_WU?$char_traits@_W@std@@@std@@@std@@QAE@ABV_Locinfo@1@I@Z 100abb2d f i libcpmt:wlocale.obj
 0001:000aab42       ??0?$numpunct@G@std@@QAE@ABV_Locinfo@1@I_N@Z 100abb42 f i libcpmt:wlocale.obj
 0001:000aab78       ??0?$numpunct@_W@std@@QAE@ABV_Locinfo@1@I_N@Z 100abb78 f i libcpmt:wlocale.obj
 0001:000aabae       ??0?$time_get@GV?$istreambuf_iterator@GU?$char_traits@G@std@@@std@@@std@@QAE@ABV_Locinfo@1@I@Z 100abbae f i libcpmt:wlocale.obj
 0001:000aabe1       ??0?$time_get@_WV?$istreambuf_iterator@_WU?$char_traits@_W@std@@@std@@@std@@QAE@ABV_Locinfo@1@I@Z 100abbe1 f i libcpmt:wlocale.obj
 0001:000aac14       ??0?$time_put@GV?$ostreambuf_iterator@GU?$char_traits@G@std@@@std@@@std@@QAE@ABV_Locinfo@1@I@Z 100abc14 f i libcpmt:wlocale.obj
 0001:000aac39       ??0?$time_put@_WV?$ostreambuf_iterator@_WU?$char_traits@_W@std@@@std@@@std@@QAE@ABV_Locinfo@1@I@Z 100abc39 f i libcpmt:wlocale.obj
 0001:000aac5e       ??0_Timevec@std@@QAE@PAX@Z 100abc5e f i libcpmt:wlocale.obj
 0001:000aac6c       ??0messages_base@std@@QAE@I@Z 100abc6c f i libcpmt:wlocale.obj
 0001:000aac81       ??0money_base@std@@QAE@I@Z 100abc81 f i libcpmt:wlocale.obj
 0001:000aac96       ??0time_base@std@@QAE@I@Z  100abc96 f i libcpmt:wlocale.obj
 0001:000aacab       ??1?$_Mpunct@G@std@@MAE@XZ 100abcab f i libcpmt:wlocale.obj
 0001:000aacc1       ??1?$_Mpunct@_W@std@@MAE@XZ 100abcc1 f i libcpmt:wlocale.obj
 0001:000aacd7       ??1?$basic_string@GU?$char_traits@G@std@@V?$allocator@G@2@@std@@QAE@XZ 100abcd7 f i libcpmt:wlocale.obj
 0001:000aace1       ??1?$basic_string@_WU?$char_traits@_W@std@@V?$allocator@_W@2@@std@@QAE@XZ 100abce1 f i libcpmt:wlocale.obj
 0001:000aaceb       ??1?$codecvt@GDH@std@@MAE@XZ 100abceb f i libcpmt:wlocale.obj
 0001:000aacf2       ??1?$codecvt@_WDH@std@@MAE@XZ 100abcf2 f i libcpmt:wlocale.obj
 0001:000aacf9       ??1?$collate@G@std@@MAE@XZ 100abcf9 f i libcpmt:wlocale.obj
 0001:000aad13       ??1?$collate@_W@std@@MAE@XZ 100abd13 f i libcpmt:wlocale.obj
 0001:000aad2d       ??1?$ctype@G@std@@MAE@XZ   100abd2d f i libcpmt:wlocale.obj
 0001:000aad56       ??1?$ctype@_W@std@@MAE@XZ  100abd56 f i libcpmt:wlocale.obj
 0001:000aad7f       ??1?$messages@G@std@@MAE@XZ 100abd7f f i libcpmt:wlocale.obj
 0001:000aad86       ??1?$messages@_W@std@@MAE@XZ 100abd86 f i libcpmt:wlocale.obj
 0001:000aad8d       ??1?$money_get@GV?$istreambuf_iterator@GU?$char_traits@G@std@@@std@@@std@@MAE@XZ 100abd8d f i libcpmt:wlocale.obj
 0001:000aad94       ??1?$money_get@_WV?$istreambuf_iterator@_WU?$char_traits@_W@std@@@std@@@std@@MAE@XZ 100abd94 f i libcpmt:wlocale.obj
 0001:000aad9b       ??1?$money_put@GV?$ostreambuf_iterator@GU?$char_traits@G@std@@@std@@@std@@MAE@XZ 100abd9b f i libcpmt:wlocale.obj
 0001:000aada2       ??1?$money_put@_WV?$ostreambuf_iterator@_WU?$char_traits@_W@std@@@std@@@std@@MAE@XZ 100abda2 f i libcpmt:wlocale.obj
 0001:000aada9       ??1?$moneypunct@G$00@std@@MAE@XZ 100abda9 f i libcpmt:wlocale.obj
 0001:000aadbf       ??1?$moneypunct@G$0A@@std@@MAE@XZ 100abdbf f i libcpmt:wlocale.obj
 0001:000aadd5       ??1?$moneypunct@_W$00@std@@MAE@XZ 100abdd5 f i libcpmt:wlocale.obj
 0001:000aadeb       ??1?$moneypunct@_W$0A@@std@@MAE@XZ 100abdeb f i libcpmt:wlocale.obj
 0001:000aae01       ??1?$num_get@GV?$istreambuf_iterator@GU?$char_traits@G@std@@@std@@@std@@MAE@XZ 100abe01 f i libcpmt:wlocale.obj
 0001:000aae08       ??1?$num_get@_WV?$istreambuf_iterator@_WU?$char_traits@_W@std@@@std@@@std@@MAE@XZ 100abe08 f i libcpmt:wlocale.obj
 0001:000aae0f       ??1?$num_put@GV?$ostreambuf_iterator@GU?$char_traits@G@std@@@std@@@std@@MAE@XZ 100abe0f f i libcpmt:wlocale.obj
 0001:000aae16       ??1?$num_put@_WV?$ostreambuf_iterator@_WU?$char_traits@_W@std@@@std@@@std@@MAE@XZ 100abe16 f i libcpmt:wlocale.obj
 0001:000aae1d       ??1?$numpunct@G@std@@MAE@XZ 100abe1d f i libcpmt:wlocale.obj
 0001:000aae33       ??1?$numpunct@_W@std@@MAE@XZ 100abe33 f i libcpmt:wlocale.obj
 0001:000aae49       ??1?$time_get@GV?$istreambuf_iterator@GU?$char_traits@G@std@@@std@@@std@@MAE@XZ 100abe49 f i libcpmt:wlocale.obj
 0001:000aae5f       ??1?$time_get@_WV?$istreambuf_iterator@_WU?$char_traits@_W@std@@@std@@@std@@MAE@XZ 100abe5f f i libcpmt:wlocale.obj
 0001:000aae75       ??1?$time_put@GV?$ostreambuf_iterator@GU?$char_traits@G@std@@@std@@@std@@MAE@XZ 100abe75 f i libcpmt:wlocale.obj
 0001:000aae8f       ??1?$time_put@_WV?$ostreambuf_iterator@_WU?$char_traits@_W@std@@@std@@@std@@MAE@XZ 100abe8f f i libcpmt:wlocale.obj
 0001:000aaea9       ??1_Timevec@std@@QAE@XZ    100abea9 f i libcpmt:wlocale.obj
 0001:000aaeb2       ??1messages_base@std@@UAE@XZ 100abeb2 f i libcpmt:wlocale.obj
 0001:000aaeb9       ??1money_base@std@@UAE@XZ  100abeb9 f i libcpmt:wlocale.obj
 0001:000aaec0       ??1time_base@std@@UAE@XZ   100abec0 f i libcpmt:wlocale.obj
 0001:000aaec7       ??4?$_Yarn@_W@std@@QAEAAV01@PB_W@Z 100abec7 f i libcpmt:wlocale.obj
 0001:000aaf20       ??4?$basic_string@GU?$char_traits@G@std@@V?$allocator@G@2@@std@@QAEAAV01@$$QAV01@@Z 100abf20 f i libcpmt:wlocale.obj
 0001:000aaf45       ??4?$basic_string@GU?$char_traits@G@std@@V?$allocator@G@2@@std@@QAEAAV01@ABV01@@Z 100abf45 f i libcpmt:wlocale.obj
 0001:000aaf63       ??4?$basic_string@_WU?$char_traits@_W@std@@V?$allocator@_W@2@@std@@QAEAAV01@$$QAV01@@Z 100abf63 f i libcpmt:wlocale.obj
 0001:000aaf88       ??4?$basic_string@_WU?$char_traits@_W@std@@V?$allocator@_W@2@@std@@QAEAAV01@ABV01@@Z 100abf88 f i libcpmt:wlocale.obj
 0001:000aafa6       ??4?$ostreambuf_iterator@GU?$char_traits@G@std@@@std@@QAEAAV01@G@Z 100abfa6 f i libcpmt:wlocale.obj
 0001:000aafcf       ??4?$ostreambuf_iterator@_WU?$char_traits@_W@std@@@std@@QAEAAV01@_W@Z 100abfcf f i libcpmt:wlocale.obj
 0001:000aaff8       ??4_Timevec@std@@QAEAAV01@ABV01@@Z 100abff8 f i libcpmt:wlocale.obj
 0001:000ab00b       ??8?$_String_const_iterator@V?$_String_val@U?$_Simple_types@G@std@@@std@@@std@@QBE_NABV01@@Z 100ac00b f i libcpmt:wlocale.obj
 0001:000ab01e       ??8?$_String_const_iterator@V?$_String_val@U?$_Simple_types@_W@std@@@std@@@std@@QBE_NABV01@@Z 100ac01e f i libcpmt:wlocale.obj
 0001:000ab031       ??9?$_String_const_iterator@V?$_String_val@U?$_Simple_types@G@std@@@std@@@std@@QBE_NABV01@@Z 100ac031 f i libcpmt:wlocale.obj
 0001:000ab044       ??9?$_String_const_iterator@V?$_String_val@U?$_Simple_types@_W@std@@@std@@@std@@QBE_NABV01@@Z 100ac044 f i libcpmt:wlocale.obj
 0001:000ab057       ??A?$basic_string@GU?$char_traits@G@std@@V?$allocator@G@2@@std@@QAEAAGI@Z 100ac057 f i libcpmt:wlocale.obj
 0001:000ab06c       ??A?$basic_string@GU?$char_traits@G@std@@V?$allocator@G@2@@std@@QBEABGI@Z 100ac06c f i libcpmt:wlocale.obj
 0001:000ab081       ??A?$basic_string@_WU?$char_traits@_W@std@@V?$allocator@_W@2@@std@@QAEAA_WI@Z 100ac081 f i libcpmt:wlocale.obj
 0001:000ab096       ??A?$basic_string@_WU?$char_traits@_W@std@@V?$allocator@_W@2@@std@@QBEAB_WI@Z 100ac096 f i libcpmt:wlocale.obj
 0001:000ab0ab       ??D?$_String_const_iterator@V?$_String_val@U?$_Simple_types@G@std@@@std@@@std@@QBEABGXZ 100ac0ab f i libcpmt:wlocale.obj
 0001:000ab0ae       ??D?$_String_const_iterator@V?$_String_val@U?$_Simple_types@_W@std@@@std@@@std@@QBEAB_WXZ 100ac0ae f i libcpmt:wlocale.obj
 0001:000ab0b1       ??D?$_String_iterator@V?$_String_val@U?$_Simple_types@G@std@@@std@@@std@@QBEAAGXZ 100ac0b1 f i libcpmt:wlocale.obj
 0001:000ab0b4       ??D?$_String_iterator@V?$_String_val@U?$_Simple_types@_W@std@@@std@@@std@@QBEAA_WXZ 100ac0b4 f i libcpmt:wlocale.obj
 0001:000ab0b7       ??D?$istreambuf_iterator@GU?$char_traits@G@std@@@std@@QBEGXZ 100ac0b7 f i libcpmt:wlocale.obj
 0001:000ab0cb       ??D?$istreambuf_iterator@_WU?$char_traits@_W@std@@@std@@QBE_WXZ 100ac0cb f i libcpmt:wlocale.obj
 0001:000ab0df       ??D?$ostreambuf_iterator@GU?$char_traits@G@std@@@std@@QAEAAV01@XZ 100ac0df f i libcpmt:wlocale.obj
 0001:000ab0e2       ??D?$ostreambuf_iterator@_WU?$char_traits@_W@std@@@std@@QAEAAV01@XZ 100ac0e2 f i libcpmt:wlocale.obj
 0001:000ab0e5       ??E?$_String_const_iterator@V?$_String_val@U?$_Simple_types@G@std@@@std@@@std@@QAEAAV01@XZ 100ac0e5 f i libcpmt:wlocale.obj
 0001:000ab0eb       ??E?$_String_const_iterator@V?$_String_val@U?$_Simple_types@_W@std@@@std@@@std@@QAEAAV01@XZ 100ac0eb f i libcpmt:wlocale.obj
 0001:000ab0f1       ??E?$istreambuf_iterator@GU?$char_traits@G@std@@@std@@QAEAAV01@XZ 100ac0f1 f i libcpmt:wlocale.obj
 0001:000ab0fd       ??E?$istreambuf_iterator@_WU?$char_traits@_W@std@@@std@@QAEAAV01@XZ 100ac0fd f i libcpmt:wlocale.obj
 0001:000ab109       ??E?$ostreambuf_iterator@GU?$char_traits@G@std@@@std@@QAEAAV01@H@Z 100ac109 f i libcpmt:wlocale.obj
 0001:000ab10e       ??E?$ostreambuf_iterator@GU?$char_traits@G@std@@@std@@QAEAAV01@XZ 100ac10e f i libcpmt:wlocale.obj
 0001:000ab111       ??E?$ostreambuf_iterator@_WU?$char_traits@_W@std@@@std@@QAEAAV01@H@Z 100ac111 f i libcpmt:wlocale.obj
 0001:000ab116       ??E?$ostreambuf_iterator@_WU?$char_traits@_W@std@@@std@@QAEAAV01@XZ 100ac116 f i libcpmt:wlocale.obj
 0001:000ab119       ??G?$_String_const_iterator@V?$_String_val@U?$_Simple_types@G@std@@@std@@@std@@QBEHABV01@@Z 100ac119 f i libcpmt:wlocale.obj
 0001:000ab129       ??G?$_String_const_iterator@V?$_String_val@U?$_Simple_types@_W@std@@@std@@@std@@QBEHABV01@@Z 100ac129 f i libcpmt:wlocale.obj
 0001:000ab139       ??G?$_String_iterator@V?$_String_val@U?$_Simple_types@G@std@@@std@@@std@@QBE?AV01@H@Z 100ac139 f i libcpmt:wlocale.obj
 0001:000ab14e       ??G?$_String_iterator@V?$_String_val@U?$_Simple_types@G@std@@@std@@@std@@QBEHABV?$_String_const_iterator@V?$_String_val@U?$_Simple_types@G@std@@@std@@@1@@Z 100ac14e f i libcpmt:wlocale.obj
 0001:000ab15e       ??G?$_String_iterator@V?$_String_val@U?$_Simple_types@_W@std@@@std@@@std@@QBE?AV01@H@Z 100ac15e f i libcpmt:wlocale.obj
 0001:000ab173       ??G?$_String_iterator@V?$_String_val@U?$_Simple_types@_W@std@@@std@@@std@@QBEHABV?$_String_const_iterator@V?$_String_val@U?$_Simple_types@_W@std@@@std@@@1@@Z 100ac173 f i libcpmt:wlocale.obj
 0001:000ab183       ??H?$_String_iterator@V?$_String_val@U?$_Simple_types@G@std@@@std@@@std@@QBE?AV01@H@Z 100ac183 f i libcpmt:wlocale.obj
 0001:000ab197       ??H?$_String_iterator@V?$_String_val@U?$_Simple_types@_W@std@@@std@@@std@@QBE?AV01@H@Z 100ac197 f i libcpmt:wlocale.obj
 0001:000ab1ab       ??Y?$_String_const_iterator@V?$_String_val@U?$_Simple_types@G@std@@@std@@@std@@QAEAAV01@H@Z 100ac1ab f i libcpmt:wlocale.obj
 0001:000ab1bb       ??Y?$_String_const_iterator@V?$_String_val@U?$_Simple_types@_W@std@@@std@@@std@@QAEAAV01@H@Z 100ac1bb f i libcpmt:wlocale.obj
 0001:000ab1cb       ??Y?$_String_iterator@V?$_String_val@U?$_Simple_types@G@std@@@std@@@std@@QAEAAV01@H@Z 100ac1cb f i libcpmt:wlocale.obj
 0001:000ab1db       ??Y?$_String_iterator@V?$_String_val@U?$_Simple_types@_W@std@@@std@@@std@@QAEAAV01@H@Z 100ac1db f i libcpmt:wlocale.obj
 0001:000ab1eb       ??Y?$basic_string@GU?$char_traits@G@std@@V?$allocator@G@2@@std@@QAEAAV01@ABV01@@Z 100ac1eb f i libcpmt:wlocale.obj
 0001:000ab1fe       ??Y?$basic_string@GU?$char_traits@G@std@@V?$allocator@G@2@@std@@QAEAAV01@G@Z 100ac1fe f i libcpmt:wlocale.obj
 0001:000ab20f       ??Y?$basic_string@_WU?$char_traits@_W@std@@V?$allocator@_W@2@@std@@QAEAAV01@ABV01@@Z 100ac20f f i libcpmt:wlocale.obj
 0001:000ab222       ??Y?$basic_string@_WU?$char_traits@_W@std@@V?$allocator@_W@2@@std@@QAEAAV01@_W@Z 100ac222 f i libcpmt:wlocale.obj
 0001:000ab233       ??Z?$_String_iterator@V?$_String_val@U?$_Simple_types@G@std@@@std@@@std@@QAEAAV01@H@Z 100ac233 f i libcpmt:wlocale.obj
 0001:000ab245       ??Z?$_String_iterator@V?$_String_val@U?$_Simple_types@_W@std@@@std@@@std@@QAEAAV01@H@Z 100ac245 f i libcpmt:wlocale.obj
 0001:000ab257       ??_E?$_Mpunct@G@std@@MAEPAXI@Z 100ac257 f i libcpmt:wlocale.obj
 0001:000ab257       ??_G?$_Mpunct@G@std@@MAEPAXI@Z 100ac257 f i libcpmt:wlocale.obj
 0001:000ab282       ??_E?$_Mpunct@_W@std@@MAEPAXI@Z 100ac282 f i libcpmt:wlocale.obj
 0001:000ab282       ??_G?$_Mpunct@_W@std@@MAEPAXI@Z 100ac282 f i libcpmt:wlocale.obj
 0001:000ab2ad       ??_G?$codecvt@GDH@std@@MAEPAXI@Z 100ac2ad f i libcpmt:wlocale.obj
 0001:000ab2ad       ??_E?$codecvt@GDH@std@@MAEPAXI@Z 100ac2ad f i libcpmt:wlocale.obj
 0001:000ab2cd       ??_G?$codecvt@_WDH@std@@MAEPAXI@Z 100ac2cd f i libcpmt:wlocale.obj
 0001:000ab2cd       ??_E?$codecvt@_WDH@std@@MAEPAXI@Z 100ac2cd f i libcpmt:wlocale.obj
 0001:000ab2ed       ??_G?$collate@G@std@@MAEPAXI@Z 100ac2ed f i libcpmt:wlocale.obj
 0001:000ab2ed       ??_E?$collate@G@std@@MAEPAXI@Z 100ac2ed f i libcpmt:wlocale.obj
 0001:000ab30c       ??_E?$collate@_W@std@@MAEPAXI@Z 100ac30c f i libcpmt:wlocale.obj
 0001:000ab30c       ??_G?$collate@_W@std@@MAEPAXI@Z 100ac30c f i libcpmt:wlocale.obj
 0001:000ab32b       ??_G?$ctype@G@std@@MAEPAXI@Z 100ac32b f i libcpmt:wlocale.obj
 0001:000ab32b       ??_E?$ctype@G@std@@MAEPAXI@Z 100ac32b f i libcpmt:wlocale.obj
 0001:000ab34a       ??_G?$ctype@_W@std@@MAEPAXI@Z 100ac34a f i libcpmt:wlocale.obj
 0001:000ab34a       ??_E?$ctype@_W@std@@MAEPAXI@Z 100ac34a f i libcpmt:wlocale.obj
 0001:000ab369       ??_G?$messages@G@std@@MAEPAXI@Z 100ac369 f i libcpmt:wlocale.obj
 0001:000ab369       ??_E?$messages@G@std@@MAEPAXI@Z 100ac369 f i libcpmt:wlocale.obj
 0001:000ab389       ??_E?$messages@_W@std@@MAEPAXI@Z 100ac389 f i libcpmt:wlocale.obj
 0001:000ab389       ??_G?$messages@_W@std@@MAEPAXI@Z 100ac389 f i libcpmt:wlocale.obj
 0001:000ab3a9       ??_G?$money_get@GV?$istreambuf_iterator@GU?$char_traits@G@std@@@std@@@std@@MAEPAXI@Z 100ac3a9 f i libcpmt:wlocale.obj
 0001:000ab3a9       ??_E?$money_get@GV?$istreambuf_iterator@GU?$char_traits@G@std@@@std@@@std@@MAEPAXI@Z 100ac3a9 f i libcpmt:wlocale.obj
 0001:000ab3c9       ??_G?$money_get@_WV?$istreambuf_iterator@_WU?$char_traits@_W@std@@@std@@@std@@MAEPAXI@Z 100ac3c9 f i libcpmt:wlocale.obj
 0001:000ab3c9       ??_E?$money_get@_WV?$istreambuf_iterator@_WU?$char_traits@_W@std@@@std@@@std@@MAEPAXI@Z 100ac3c9 f i libcpmt:wlocale.obj
 0001:000ab3e9       ??_E?$money_put@GV?$ostreambuf_iterator@GU?$char_traits@G@std@@@std@@@std@@MAEPAXI@Z 100ac3e9 f i libcpmt:wlocale.obj
 0001:000ab3e9       ??_G?$money_put@GV?$ostreambuf_iterator@GU?$char_traits@G@std@@@std@@@std@@MAEPAXI@Z 100ac3e9 f i libcpmt:wlocale.obj
 0001:000ab409       ??_G?$money_put@_WV?$ostreambuf_iterator@_WU?$char_traits@_W@std@@@std@@@std@@MAEPAXI@Z 100ac409 f i libcpmt:wlocale.obj
 0001:000ab409       ??_E?$money_put@_WV?$ostreambuf_iterator@_WU?$char_traits@_W@std@@@std@@@std@@MAEPAXI@Z 100ac409 f i libcpmt:wlocale.obj
 0001:000ab429       ??_E?$moneypunct@G$00@std@@MAEPAXI@Z 100ac429 f i libcpmt:wlocale.obj
 0001:000ab429       ??_G?$moneypunct@G$00@std@@MAEPAXI@Z 100ac429 f i libcpmt:wlocale.obj
 0001:000ab454       ??_E?$moneypunct@G$0A@@std@@MAEPAXI@Z 100ac454 f i libcpmt:wlocale.obj
 0001:000ab454       ??_G?$moneypunct@G$0A@@std@@MAEPAXI@Z 100ac454 f i libcpmt:wlocale.obj
 0001:000ab47f       ??_G?$moneypunct@_W$00@std@@MAEPAXI@Z 100ac47f f i libcpmt:wlocale.obj
 0001:000ab47f       ??_E?$moneypunct@_W$00@std@@MAEPAXI@Z 100ac47f f i libcpmt:wlocale.obj
 0001:000ab4aa       ??_E?$moneypunct@_W$0A@@std@@MAEPAXI@Z 100ac4aa f i libcpmt:wlocale.obj
 0001:000ab4aa       ??_G?$moneypunct@_W$0A@@std@@MAEPAXI@Z 100ac4aa f i libcpmt:wlocale.obj
 0001:000ab4d5       ??_E?$num_get@GV?$istreambuf_iterator@GU?$char_traits@G@std@@@std@@@std@@MAEPAXI@Z 100ac4d5 f i libcpmt:wlocale.obj
 0001:000ab4d5       ??_G?$num_get@GV?$istreambuf_iterator@GU?$char_traits@G@std@@@std@@@std@@MAEPAXI@Z 100ac4d5 f i libcpmt:wlocale.obj
 0001:000ab4f5       ??_G?$num_get@_WV?$istreambuf_iterator@_WU?$char_traits@_W@std@@@std@@@std@@MAEPAXI@Z 100ac4f5 f i libcpmt:wlocale.obj
 0001:000ab4f5       ??_E?$num_get@_WV?$istreambuf_iterator@_WU?$char_traits@_W@std@@@std@@@std@@MAEPAXI@Z 100ac4f5 f i libcpmt:wlocale.obj
 0001:000ab515       ??_E?$num_put@GV?$ostreambuf_iterator@GU?$char_traits@G@std@@@std@@@std@@MAEPAXI@Z 100ac515 f i libcpmt:wlocale.obj
 0001:000ab515       ??_G?$num_put@GV?$ostreambuf_iterator@GU?$char_traits@G@std@@@std@@@std@@MAEPAXI@Z 100ac515 f i libcpmt:wlocale.obj
 0001:000ab535       ??_G?$num_put@_WV?$ostreambuf_iterator@_WU?$char_traits@_W@std@@@std@@@std@@MAEPAXI@Z 100ac535 f i libcpmt:wlocale.obj
 0001:000ab535       ??_E?$num_put@_WV?$ostreambuf_iterator@_WU?$char_traits@_W@std@@@std@@@std@@MAEPAXI@Z 100ac535 f i libcpmt:wlocale.obj
 0001:000ab555       ??_G?$numpunct@G@std@@MAEPAXI@Z 100ac555 f i libcpmt:wlocale.obj
 0001:000ab555       ??_E?$numpunct@G@std@@MAEPAXI@Z 100ac555 f i libcpmt:wlocale.obj
 0001:000ab580       ??_E?$numpunct@_W@std@@MAEPAXI@Z 100ac580 f i libcpmt:wlocale.obj
 0001:000ab580       ??_G?$numpunct@_W@std@@MAEPAXI@Z 100ac580 f i libcpmt:wlocale.obj
 0001:000ab5ab       ??_G?$time_get@GV?$istreambuf_iterator@GU?$char_traits@G@std@@@std@@@std@@MAEPAXI@Z 100ac5ab f i libcpmt:wlocale.obj
 0001:000ab5ab       ??_E?$time_get@GV?$istreambuf_iterator@GU?$char_traits@G@std@@@std@@@std@@MAEPAXI@Z 100ac5ab f i libcpmt:wlocale.obj
 0001:000ab5d6       ??_E?$time_get@_WV?$istreambuf_iterator@_WU?$char_traits@_W@std@@@std@@@std@@MAEPAXI@Z 100ac5d6 f i libcpmt:wlocale.obj
 0001:000ab5d6       ??_G?$time_get@_WV?$istreambuf_iterator@_WU?$char_traits@_W@std@@@std@@@std@@MAEPAXI@Z 100ac5d6 f i libcpmt:wlocale.obj
 0001:000ab601       ??_G?$time_put@GV?$ostreambuf_iterator@GU?$char_traits@G@std@@@std@@@std@@MAEPAXI@Z 100ac601 f i libcpmt:wlocale.obj
 0001:000ab601       ??_E?$time_put@GV?$ostreambuf_iterator@GU?$char_traits@G@std@@@std@@@std@@MAEPAXI@Z 100ac601 f i libcpmt:wlocale.obj
 0001:000ab620       ??_G?$time_put@_WV?$ostreambuf_iterator@_WU?$char_traits@_W@std@@@std@@@std@@MAEPAXI@Z 100ac620 f i libcpmt:wlocale.obj
 0001:000ab620       ??_E?$time_put@_WV?$ostreambuf_iterator@_WU?$char_traits@_W@std@@@std@@@std@@MAEPAXI@Z 100ac620 f i libcpmt:wlocale.obj
 0001:000ab63f       ??_Emessages_base@std@@UAEPAXI@Z 100ac63f f i libcpmt:wlocale.obj
 0001:000ab63f       ??_Gmessages_base@std@@UAEPAXI@Z 100ac63f f i libcpmt:wlocale.obj
 0001:000ab65f       ??_Gmoney_base@std@@UAEPAXI@Z 100ac65f f i libcpmt:wlocale.obj
 0001:000ab65f       ??_Emoney_base@std@@UAEPAXI@Z 100ac65f f i libcpmt:wlocale.obj
 0001:000ab67f       ??_Gtime_base@std@@UAEPAXI@Z 100ac67f f i libcpmt:wlocale.obj
 0001:000ab67f       ??_Etime_base@std@@UAEPAXI@Z 100ac67f f i libcpmt:wlocale.obj
 0001:000ab69f       ?_Assign_rv@?$basic_string@GU?$char_traits@G@std@@V?$allocator@G@2@@std@@QAEX$$QAV12@@Z 100ac69f f i libcpmt:wlocale.obj
 0001:000ab6ed       ?_Assign_rv@?$basic_string@_WU?$char_traits@_W@std@@V?$allocator@_W@2@@std@@QAEX$$QAV12@@Z 100ac6ed f i libcpmt:wlocale.obj
 0001:000ab73b       ?_C_str@?$_Yarn@_W@std@@QBEPB_WXZ 100ac73b f i libcpmt:wlocale.obj
 0001:000ab745       ?_Change_alloc@?$_String_alloc@$0A@U?$_String_base_types@GV?$allocator@G@std@@@std@@@std@@QAEXABU?$_Wrap_alloc@V?$allocator@G@std@@@2@@Z 100ac745 f i libcpmt:wlocale.obj
 0001:000ab748       ?_Change_alloc@?$_String_alloc@$0A@U?$_String_base_types@_WV?$allocator@_W@std@@@std@@@std@@QAEXABU?$_Wrap_alloc@V?$allocator@_W@std@@@2@@Z 100ac748 f i libcpmt:wlocale.obj
 0001:000ab74b       ?_Chassign@?$basic_string@GU?$char_traits@G@std@@V?$allocator@G@2@@std@@QAEXIIG@Z 100ac74b f i libcpmt:wlocale.obj
 0001:000ab78c       ?_Chassign@?$basic_string@_WU?$char_traits@_W@std@@V?$allocator@_W@2@@std@@QAEXII_W@Z 100ac78c f i libcpmt:wlocale.obj
 0001:000ab7cd       ?_Compat@?$_String_const_iterator@V?$_String_val@U?$_Simple_types@G@std@@@std@@@std@@QBEXABV12@@Z 100ac7cd f i libcpmt:wlocale.obj
 0001:000ab7d0       ?_Compat@?$_String_const_iterator@V?$_String_val@U?$_Simple_types@_W@std@@@std@@@std@@QBEXABV12@@Z 100ac7d0 f i libcpmt:wlocale.obj
 0001:000ab7d3       ?_Copy@?$basic_string@GU?$char_traits@G@std@@V?$allocator@G@2@@std@@QAEXII@Z 100ac7d3 f i libcpmt:wlocale.obj
 0001:000ab8c3       ?_Copy@?$basic_string@_WU?$char_traits@_W@std@@V?$allocator@_W@2@@std@@QAEXII@Z 100ac8c3 f i libcpmt:wlocale.obj
 0001:000ab9b3       ?_Donarrow@?$ctype@G@std@@IBEDGD@Z 100ac9b3 f i libcpmt:wlocale.obj
 0001:000ab9fb       ?_Donarrow@?$ctype@_W@std@@IBED_WD@Z 100ac9fb f i libcpmt:wlocale.obj
 0001:000aba43       ?_Dowiden@?$ctype@G@std@@IBEGD@Z 100aca43 f i libcpmt:wlocale.obj
 0001:000aba79       ?_Dowiden@?$ctype@_W@std@@IBE_WD@Z 100aca79 f i libcpmt:wlocale.obj
 0001:000abaaf       ?_Empty@?$_Yarn@_W@std@@QBE_NXZ 100acaaf f i libcpmt:wlocale.obj
 0001:000abab7       ?_Eos@?$basic_string@GU?$char_traits@G@std@@V?$allocator@G@2@@std@@QAEXI@Z 100acab7 f i libcpmt:wlocale.obj
 0001:000abad2       ?_Eos@?$basic_string@_WU?$char_traits@_W@std@@V?$allocator@_W@2@@std@@QAEXI@Z 100acad2 f i libcpmt:wlocale.obj
 0001:000abaed       ?_Ffmt@?$num_put@GV?$ostreambuf_iterator@GU?$char_traits@G@std@@@std@@@std@@ABAPADPADDH@Z 100acaed f i libcpmt:wlocale.obj
 0001:000abb82       ?_Ffmt@?$num_put@_WV?$ostreambuf_iterator@_WU?$char_traits@_W@std@@@std@@@std@@ABAPADPADDH@Z 100acb82 f i libcpmt:wlocale.obj
 0001:000abc17       ?_Fput@?$num_put@GV?$ostreambuf_iterator@GU?$char_traits@G@std@@@std@@@std@@ABA?AV?$ostreambuf_iterator@GU?$char_traits@G@std@@@2@V32@AAVios_base@2@GPBDIIII@Z 100acc17 f i libcpmt:wlocale.obj
 0001:000abf7a       ?_Fput@?$num_put@_WV?$ostreambuf_iterator@_WU?$char_traits@_W@std@@@std@@@std@@ABA?AV?$ostreambuf_iterator@_WU?$char_traits@_W@std@@@2@V32@AAVios_base@2@_WPBDIIII@Z 100acf7a f i libcpmt:wlocale.obj
 0001:000ac2dd       ?_Getal@?$_String_alloc@$0A@U?$_String_base_types@GV?$allocator@G@std@@@std@@@std@@QBE?AU?$_Wrap_alloc@V?$allocator@G@std@@@2@XZ 100ad2dd f i libcpmt:wlocale.obj
 0001:000ac2e7       ?_Getal@?$_String_alloc@$0A@U?$_String_base_types@_WV?$allocator@_W@std@@@std@@@std@@QBE?AU?$_Wrap_alloc@V?$allocator@_W@std@@@2@XZ 100ad2e7 f i libcpmt:wlocale.obj
 0001:000ac2f1       ?_Getcat@?$codecvt@GDH@std@@SAIPAPBVfacet@locale@2@PBV42@@Z 100ad2f1 f i libcpmt:wlocale.obj
 0001:000ac357       ?_Getcat@?$codecvt@_WDH@std@@SAIPAPBVfacet@locale@2@PBV42@@Z 100ad357 f i libcpmt:wlocale.obj
 0001:000ac3bd       ?_Getcat@?$collate@G@std@@SAIPAPBVfacet@locale@2@PBV42@@Z 100ad3bd f i libcpmt:wlocale.obj
 0001:000ac463       ?_Getcat@?$collate@_W@std@@SAIPAPBVfacet@locale@2@PBV42@@Z 100ad463 f i libcpmt:wlocale.obj
 0001:000ac509       ?_Getcat@?$ctype@G@std@@SAIPAPBVfacet@locale@2@PBV42@@Z 100ad509 f i libcpmt:wlocale.obj
 0001:000ac579       ?_Getcat@?$ctype@_W@std@@SAIPAPBVfacet@locale@2@PBV42@@Z 100ad579 f i libcpmt:wlocale.obj
 0001:000ac5e9       ?_Getcat@?$messages@G@std@@SAIPAPBVfacet@locale@2@PBV42@@Z 100ad5e9 f i libcpmt:wlocale.obj
 0001:000ac651       ?_Getcat@?$messages@_W@std@@SAIPAPBVfacet@locale@2@PBV42@@Z 100ad651 f i libcpmt:wlocale.obj
 0001:000ac6b9       ?_Getcat@?$money_get@GV?$istreambuf_iterator@GU?$char_traits@G@std@@@std@@@std@@SAIPAPBVfacet@locale@2@PBV42@@Z 100ad6b9 f i libcpmt:wlocale.obj
 0001:000ac721       ?_Getcat@?$money_get@_WV?$istreambuf_iterator@_WU?$char_traits@_W@std@@@std@@@std@@SAIPAPBVfacet@locale@2@PBV42@@Z 100ad721 f i libcpmt:wlocale.obj
 0001:000ac789       ?_Getcat@?$money_put@GV?$ostreambuf_iterator@GU?$char_traits@G@std@@@std@@@std@@SAIPAPBVfacet@locale@2@PBV42@@Z 100ad789 f i libcpmt:wlocale.obj
 0001:000ac7f1       ?_Getcat@?$money_put@_WV?$ostreambuf_iterator@_WU?$char_traits@_W@std@@@std@@@std@@SAIPAPBVfacet@locale@2@PBV42@@Z 100ad7f1 f i libcpmt:wlocale.obj
 0001:000ac859       ?_Getcat@?$moneypunct@G$00@std@@SAIPAPBVfacet@locale@2@PBV42@@Z 100ad859 f i libcpmt:wlocale.obj
 0001:000ac8dd       ?_Getcat@?$moneypunct@G$0A@@std@@SAIPAPBVfacet@locale@2@PBV42@@Z 100ad8dd f i libcpmt:wlocale.obj
 0001:000ac962       ?_Getcat@?$moneypunct@_W$00@std@@SAIPAPBVfacet@locale@2@PBV42@@Z 100ad962 f i libcpmt:wlocale.obj
 0001:000ac9e6       ?_Getcat@?$moneypunct@_W$0A@@std@@SAIPAPBVfacet@locale@2@PBV42@@Z 100ad9e6 f i libcpmt:wlocale.obj
 0001:000aca6b       ?_Getcat@?$num_get@GV?$istreambuf_iterator@GU?$char_traits@G@std@@@std@@@std@@SAIPAPBVfacet@locale@2@PBV42@@Z 100ada6b f i libcpmt:wlocale.obj
 0001:000acad3       ?_Getcat@?$num_get@_WV?$istreambuf_iterator@_WU?$char_traits@_W@std@@@std@@@std@@SAIPAPBVfacet@locale@2@PBV42@@Z 100adad3 f i libcpmt:wlocale.obj
 0001:000acb3b       ?_Getcat@?$num_put@GV?$ostreambuf_iterator@GU?$char_traits@G@std@@@std@@@std@@SAIPAPBVfacet@locale@2@PBV42@@Z 100adb3b f i libcpmt:wlocale.obj
 0001:000acba3       ?_Getcat@?$num_put@_WV?$ostreambuf_iterator@_WU?$char_traits@_W@std@@@std@@@std@@SAIPAPBVfacet@locale@2@PBV42@@Z 100adba3 f i libcpmt:wlocale.obj
 0001:000acc0b       ?_Getcat@?$numpunct@G@std@@SAIPAPBVfacet@locale@2@PBV42@@Z 100adc0b f i libcpmt:wlocale.obj
 0001:000acc86       ?_Getcat@?$numpunct@_W@std@@SAIPAPBVfacet@locale@2@PBV42@@Z 100adc86 f i libcpmt:wlocale.obj
 0001:000acd01       ?_Getcat@?$time_get@GV?$istreambuf_iterator@GU?$char_traits@G@std@@@std@@@std@@SAIPAPBVfacet@locale@2@PBV42@@Z 100add01 f i libcpmt:wlocale.obj
 0001:000acd6d       ?_Getcat@?$time_get@_WV?$istreambuf_iterator@_WU?$char_traits@_W@std@@@std@@@std@@SAIPAPBVfacet@locale@2@PBV42@@Z 100add6d f i libcpmt:wlocale.obj
 0001:000acdd9       ?_Getcat@?$time_put@GV?$ostreambuf_iterator@GU?$char_traits@G@std@@@std@@@std@@SAIPAPBVfacet@locale@2@PBV42@@Z 100addd9 f i libcpmt:wlocale.obj
 0001:000ace4d       ?_Getcat@?$time_put@_WV?$ostreambuf_iterator@_WU?$char_traits@_W@std@@@std@@@std@@SAIPAPBVfacet@locale@2@PBV42@@Z 100ade4d f i libcpmt:wlocale.obj
 0001:000acec1       ?_Getcoll@_Locinfo@std@@QBE?AU_Collvec@@XZ 100adec1 f i libcpmt:wlocale.obj
 0001:000aced7       ?_Getdateorder@_Locinfo@std@@QBEHXZ 100aded7 f i libcpmt:wlocale.obj
 0001:000acedc       ?_Getdays@_Locinfo@std@@QBEPBDXZ 100adedc f i libcpmt:wlocale.obj
 0001:000acf15       ?_Getffld@?$num_get@GV?$istreambuf_iterator@GU?$char_traits@G@std@@@std@@@std@@ABAHPADAAV?$istreambuf_iterator@GU?$char_traits@G@std@@@2@1AAVios_base@2@PAH@Z 100adf15 f i libcpmt:wlocale.obj
 0001:000ad4ef       ?_Getffld@?$num_get@_WV?$istreambuf_iterator@_WU?$char_traits@_W@std@@@std@@@std@@ABAHPADAAV?$istreambuf_iterator@_WU?$char_traits@_W@std@@@2@1AAVios_base@2@PAH@Z 100ae4ef f i libcpmt:wlocale.obj
 0001:000adac9       ?_Getffldx@?$num_get@GV?$istreambuf_iterator@GU?$char_traits@G@std@@@std@@@std@@ABAHPADAAV?$istreambuf_iterator@GU?$char_traits@G@std@@@2@1AAVios_base@2@PAH@Z 100aeac9 f i libcpmt:wlocale.obj
 0001:000ae16e       ?_Getffldx@?$num_get@_WV?$istreambuf_iterator@_WU?$char_traits@_W@std@@@std@@@std@@ABAHPADAAV?$istreambuf_iterator@_WU?$char_traits@_W@std@@@2@1AAVios_base@2@PAH@Z 100af16e f i libcpmt:wlocale.obj
 0001:000ae813       ?_Getfmt@?$time_get@GV?$istreambuf_iterator@GU?$char_traits@G@std@@@std@@@std@@IBE?AV?$istreambuf_iterator@GU?$char_traits@G@std@@@2@V32@0AAVios_base@2@AAHPAUtm@@PBD@Z 100af813 f i libcpmt:wlocale.obj
 0001:000ae91f       ?_Getfmt@?$time_get@_WV?$istreambuf_iterator@_WU?$char_traits@_W@std@@@std@@@std@@IBE?AV?$istreambuf_iterator@_WU?$char_traits@_W@std@@@2@V32@0AAVios_base@2@AAHPAUtm@@PBD@Z 100af91f f i libcpmt:wlocale.obj
 0001:000aea2b       ?_Getifld@?$num_get@GV?$istreambuf_iterator@GU?$char_traits@G@std@@@std@@@std@@ABAHPADAAV?$istreambuf_iterator@GU?$char_traits@G@std@@@2@1HABVlocale@2@@Z 100afa2b f i libcpmt:wlocale.obj
 0001:000aedb1       ?_Getifld@?$num_get@_WV?$istreambuf_iterator@_WU?$char_traits@_W@std@@@std@@@std@@ABAHPADAAV?$istreambuf_iterator@_WU?$char_traits@_W@std@@@2@1HABVlocale@2@@Z 100afdb1 f i libcpmt:wlocale.obj
 0001:000af137       ?_Getint@?$time_get@GV?$istreambuf_iterator@GU?$char_traits@G@std@@@std@@@std@@ABAHAAV?$istreambuf_iterator@GU?$char_traits@G@std@@@2@0HHAAHABV?$ctype@G@2@@Z 100b0137 f i libcpmt:wlocale.obj
 0001:000af2b1       ?_Getint@?$time_get@_WV?$istreambuf_iterator@_WU?$char_traits@_W@std@@@std@@@std@@ABAHAAV?$istreambuf_iterator@_WU?$char_traits@_W@std@@@2@0HHAAHABV?$ctype@_W@2@@Z 100b02b1 f i libcpmt:wlocale.obj
 0001:000af42b       ?_Getmfld@?$money_get@GV?$istreambuf_iterator@GU?$char_traits@G@std@@@std@@@std@@ABE?AV?$basic_string@DU?$char_traits@D@std@@V?$allocator@D@2@@2@AAV?$istreambuf_iterator@GU?$char_traits@G@std@@@2@0_NAAVios_base@2@PAG@Z 100b042b f i libcpmt:wlocale.obj
 0001:000afe8f       ?_Getmfld@?$money_get@_WV?$istreambuf_iterator@_WU?$char_traits@_W@std@@@std@@@std@@ABE?AV?$basic_string@DU?$char_traits@D@std@@V?$allocator@D@2@@2@AAV?$istreambuf_iterator@_WU?$char_traits@_W@std@@@2@0_NAAVios_base@2@PA_W@Z 100b0e8f f i libcpmt:wlocale.obj
 0001:000b08f3       ?_Getmonths@_Locinfo@std@@QBEPBDXZ 100b18f3 f i libcpmt:wlocale.obj
 0001:000b092c       ?_Getptr@_Timevec@std@@QBEPAXXZ 100b192c f i libcpmt:wlocale.obj
 0001:000b092f       ?_Gnavail@?$basic_streambuf@GU?$char_traits@G@std@@@std@@IBE_JXZ 100b192f f i libcpmt:wlocale.obj
 0001:000b0941       ?_Gnavail@?$basic_streambuf@_WU?$char_traits@_W@std@@@std@@IBE_JXZ 100b1941 f i libcpmt:wlocale.obj
 0001:000b0953       ?_Gninc@?$basic_streambuf@GU?$char_traits@G@std@@@std@@IAEPAGXZ 100b1953 f i libcpmt:wlocale.obj
 0001:000b0963       ?_Gninc@?$basic_streambuf@_WU?$char_traits@_W@std@@@std@@IAEPA_WXZ 100b1963 f i libcpmt:wlocale.obj
 0001:000b0973       ?_Grow@?$basic_string@GU?$char_traits@G@std@@V?$allocator@G@2@@std@@QAE_NI_N@Z 100b1973 f i libcpmt:wlocale.obj
 0001:000b09dc       ?_Grow@?$basic_string@_WU?$char_traits@_W@std@@V?$allocator@_W@2@@std@@QAE_NI_N@Z 100b19dc f i libcpmt:wlocale.obj
 0001:000b0a45       ?_Ifmt@?$num_put@GV?$ostreambuf_iterator@GU?$char_traits@G@std@@@std@@@std@@ABAPADPADPBDH@Z 100b1a45 f i libcpmt:wlocale.obj
 0001:000b0abb       ?_Ifmt@?$num_put@_WV?$ostreambuf_iterator@_WU?$char_traits@_W@std@@@std@@@std@@ABAPADPADPBDH@Z 100b1abb f i libcpmt:wlocale.obj
 0001:000b0b31       ?_Inc@?$istreambuf_iterator@GU?$char_traits@G@std@@@std@@AAEXXZ 100b1b31 f i libcpmt:wlocale.obj
 0001:000b0b58       ?_Inc@?$istreambuf_iterator@_WU?$char_traits@_W@std@@@std@@AAEXXZ 100b1b58 f i libcpmt:wlocale.obj
 0001:000b0b7f       ?_Init@?$_Mpunct@G@std@@IAEXABV_Locinfo@2@_N@Z 100b1b7f f i libcpmt:wlocale.obj
 0001:000b0c68       ?_Init@?$_Mpunct@_W@std@@IAEXABV_Locinfo@2@_N@Z 100b1c68 f i libcpmt:wlocale.obj
 0001:000b0d51       ?_Init@?$codecvt@GDH@std@@IAEXABV_Locinfo@2@@Z 100b1d51 f i libcpmt:wlocale.obj
 0001:000b0d77       ?_Init@?$codecvt@_WDH@std@@IAEXABV_Locinfo@2@@Z 100b1d77 f i libcpmt:wlocale.obj
 0001:000b0d9d       ?_Init@?$collate@G@std@@IAEXABV_Locinfo@2@@Z 100b1d9d f i libcpmt:wlocale.obj
 0001:000b0daf       ?_Init@?$collate@_W@std@@IAEXABV_Locinfo@2@@Z 100b1daf f i libcpmt:wlocale.obj
 0001:000b0dc1       ?_Init@?$ctype@G@std@@IAEXABV_Locinfo@2@@Z 100b1dc1 f i libcpmt:wlocale.obj
 0001:000b0dfc       ?_Init@?$ctype@_W@std@@IAEXABV_Locinfo@2@@Z 100b1dfc f i libcpmt:wlocale.obj
 0001:000b0e37       ?_Init@?$messages@G@std@@IAEXABV_Locinfo@2@@Z 100b1e37 f i libcpmt:wlocale.obj
 0001:000b0e3a       ?_Init@?$messages@_W@std@@IAEXABV_Locinfo@2@@Z 100b1e3a f i libcpmt:wlocale.obj
 0001:000b0e3d       ?_Init@?$money_get@GV?$istreambuf_iterator@GU?$char_traits@G@std@@@std@@@std@@IAEXABV_Locinfo@2@@Z 100b1e3d f i libcpmt:wlocale.obj
 0001:000b0e40       ?_Init@?$money_get@_WV?$istreambuf_iterator@_WU?$char_traits@_W@std@@@std@@@std@@IAEXABV_Locinfo@2@@Z 100b1e40 f i libcpmt:wlocale.obj
 0001:000b0e43       ?_Init@?$money_put@GV?$ostreambuf_iterator@GU?$char_traits@G@std@@@std@@@std@@IAEXABV_Locinfo@2@@Z 100b1e43 f i libcpmt:wlocale.obj
 0001:000b0e46       ?_Init@?$money_put@_WV?$ostreambuf_iterator@_WU?$char_traits@_W@std@@@std@@@std@@IAEXABV_Locinfo@2@@Z 100b1e46 f i libcpmt:wlocale.obj
 0001:000b0e49       ?_Init@?$num_get@GV?$istreambuf_iterator@GU?$char_traits@G@std@@@std@@@std@@IAEXABV_Locinfo@2@@Z 100b1e49 f i libcpmt:wlocale.obj
 0001:000b0e4c       ?_Init@?$num_get@_WV?$istreambuf_iterator@_WU?$char_traits@_W@std@@@std@@@std@@IAEXABV_Locinfo@2@@Z 100b1e4c f i libcpmt:wlocale.obj
 0001:000b0e4f       ?_Init@?$num_put@GV?$ostreambuf_iterator@GU?$char_traits@G@std@@@std@@@std@@IAEXABV_Locinfo@2@@Z 100b1e4f f i libcpmt:wlocale.obj
 0001:000b0e52       ?_Init@?$num_put@_WV?$ostreambuf_iterator@_WU?$char_traits@_W@std@@@std@@@std@@IAEXABV_Locinfo@2@@Z 100b1e52 f i libcpmt:wlocale.obj
 0001:000b0e55       ?_Init@?$numpunct@G@std@@IAEXABV_Locinfo@2@_N@Z 100b1e55 f i libcpmt:wlocale.obj
 0001:000b0f4e       ?_Init@?$numpunct@_W@std@@IAEXABV_Locinfo@2@_N@Z 100b1f4e f i libcpmt:wlocale.obj
 0001:000b1042       ?_Init@?$time_get@GV?$istreambuf_iterator@GU?$char_traits@G@std@@@std@@@std@@IAEXABV_Locinfo@2@@Z 100b2042 f i libcpmt:wlocale.obj
 0001:000b108c       ?_Init@?$time_get@_WV?$istreambuf_iterator@_WU?$char_traits@_W@std@@@std@@@std@@IAEXABV_Locinfo@2@@Z 100b208c f i libcpmt:wlocale.obj
 0001:000b10d6       ?_Init@?$time_put@GV?$ostreambuf_iterator@GU?$char_traits@G@std@@@std@@@std@@IAEXABV_Locinfo@2@@Z 100b20d6 f i libcpmt:wlocale.obj
 0001:000b1101       ?_Init@?$time_put@_WV?$ostreambuf_iterator@_WU?$char_traits@_W@std@@@std@@@std@@IAEXABV_Locinfo@2@@Z 100b2101 f i libcpmt:wlocale.obj
 0001:000b112c       ?_Inside@?$basic_string@GU?$char_traits@G@std@@V?$allocator@G@2@@std@@QAE_NPBG@Z 100b212c f i libcpmt:wlocale.obj
 0001:000b1168       ?_Inside@?$basic_string@_WU?$char_traits@_W@std@@V?$allocator@_W@2@@std@@QAE_NPB_W@Z 100b2168 f i libcpmt:wlocale.obj
 0001:000b11a4       ?_Iput@?$num_put@GV?$ostreambuf_iterator@GU?$char_traits@G@std@@@std@@@std@@ABA?AV?$ostreambuf_iterator@GU?$char_traits@G@std@@@2@V32@AAVios_base@2@GPADI@Z 100b21a4 f i libcpmt:wlocale.obj
 0001:000b144a       ?_Iput@?$num_put@_WV?$ostreambuf_iterator@_WU?$char_traits@_W@std@@@std@@@std@@ABA?AV?$ostreambuf_iterator@_WU?$char_traits@_W@std@@@2@V32@AAVios_base@2@_WPADI@Z 100b244a f i libcpmt:wlocale.obj
 0001:000b16f0       ?_Makeushloc@_Locimp@locale@std@@CAXABV_Locinfo@3@HPAV123@PBV23@@Z 100b26f0 f   libcpmt:wlocale.obj
 0001:000b1c9a       ?_Makewloc@_Locimp@locale@std@@CAXABV_Locinfo@3@HPAV123@PBV23@@Z 100b2c9a f   libcpmt:wlocale.obj
 0001:000b2244       ?_Maklocwcs@std@@YAPA_WPB_W@Z 100b3244 f i libcpmt:wlocale.obj
 0001:000b2282       ?_Makpat@?$_Mpunct@G@std@@AAEXAAUpattern@money_base@2@III@Z 100b3282 f i libcpmt:wlocale.obj
 0001:000b22cc       ?_Makpat@?$_Mpunct@_W@std@@AAEXAAUpattern@money_base@2@III@Z 100b32cc f i libcpmt:wlocale.obj
 0001:000b2316       ?_Myptr@?$_String_val@U?$_Simple_types@G@std@@@std@@QAEPAGXZ 100b3316 f i libcpmt:wlocale.obj
 0001:000b2321       ?_Myptr@?$_String_val@U?$_Simple_types@G@std@@@std@@QBEPBGXZ 100b3321 f i libcpmt:wlocale.obj
 0001:000b232c       ?_Myptr@?$_String_val@U?$_Simple_types@_W@std@@@std@@QAEPA_WXZ 100b332c f i libcpmt:wlocale.obj
 0001:000b2337       ?_Myptr@?$_String_val@U?$_Simple_types@_W@std@@@std@@QBEPB_WXZ 100b3337 f i libcpmt:wlocale.obj
 0001:000b2342       ?_Pdif@?$basic_string@GU?$char_traits@G@std@@V?$allocator@G@2@@std@@SAIV?$_String_const_iterator@V?$_String_val@U?$_Simple_types@G@std@@@std@@@2@0@Z 100b3342 f i libcpmt:wlocale.obj
 0001:000b2355       ?_Pdif@?$basic_string@_WU?$char_traits@_W@std@@V?$allocator@_W@2@@std@@SAIV?$_String_const_iterator@V?$_String_val@U?$_Simple_types@_W@std@@@std@@@2@0@Z 100b3355 f i libcpmt:wlocale.obj
 0001:000b2368       ?_Peek@?$istreambuf_iterator@GU?$char_traits@G@std@@@std@@ABEGXZ 100b3368 f i libcpmt:wlocale.obj
 0001:000b2396       ?_Peek@?$istreambuf_iterator@_WU?$char_traits@_W@std@@@std@@ABE_WXZ 100b3396 f i libcpmt:wlocale.obj
 0001:000b23c4       ?_Pnavail@?$basic_streambuf@GU?$char_traits@G@std@@@std@@IBE_JXZ 100b33c4 f i libcpmt:wlocale.obj
 0001:000b23d6       ?_Pnavail@?$basic_streambuf@_WU?$char_traits@_W@std@@@std@@IBE_JXZ 100b33d6 f i libcpmt:wlocale.obj
 0001:000b23e8       ?_Pninc@?$basic_streambuf@GU?$char_traits@G@std@@@std@@IAEPAGXZ 100b33e8 f i libcpmt:wlocale.obj
 0001:000b23f8       ?_Pninc@?$basic_streambuf@_WU?$char_traits@_W@std@@@std@@IAEPA_WXZ 100b33f8 f i libcpmt:wlocale.obj
 0001:000b2408       ?_Put@?$money_put@GV?$ostreambuf_iterator@GU?$char_traits@G@std@@@std@@@std@@CA?AV?$ostreambuf_iterator@GU?$char_traits@G@std@@@2@V32@V?$_String_const_iterator@V?$_String_val@U?$_Simple_types@G@std@@@std@@@2@I@Z 100b3408 f i libcpmt:wlocale.obj
 0001:000b243f       ?_Put@?$money_put@_WV?$ostreambuf_iterator@_WU?$char_traits@_W@std@@@std@@@std@@CA?AV?$ostreambuf_iterator@_WU?$char_traits@_W@std@@@2@V32@V?$_String_const_iterator@V?$_String_val@U?$_Simple_types@_W@std@@@std@@@2@I@Z 100b343f f i libcpmt:wlocale.obj
 0001:000b2476       ?_Put@?$num_put@GV?$ostreambuf_iterator@GU?$char_traits@G@std@@@std@@@std@@ABA?AV?$ostreambuf_iterator@GU?$char_traits@G@std@@@2@V32@PBGI@Z 100b3476 f i libcpmt:wlocale.obj
 0001:000b24a9       ?_Put@?$num_put@_WV?$ostreambuf_iterator@_WU?$char_traits@_W@std@@@std@@@std@@ABA?AV?$ostreambuf_iterator@_WU?$char_traits@_W@std@@@2@V32@PB_WI@Z 100b34a9 f i libcpmt:wlocale.obj
 0001:000b24dc       ?_Putmfld@?$money_put@GV?$ostreambuf_iterator@GU?$char_traits@G@std@@@std@@@std@@ABE?AV?$ostreambuf_iterator@GU?$char_traits@G@std@@@2@V32@_NAAVios_base@2@G1V?$basic_string@GU?$char_traits@G@std@@V?$allocator@G@2@@2@G@Z 100b34dc f i libcpmt:wlocale.obj
 0001:000b2a41       ?_Putmfld@?$money_put@_WV?$ostreambuf_iterator@_WU?$char_traits@_W@std@@@std@@@std@@ABE?AV?$ostreambuf_iterator@_WU?$char_traits@_W@std@@@2@V32@_NAAVios_base@2@_W1V?$basic_string@_WU?$char_traits@_W@std@@V?$allocator@_W@2@@2@3@Z 100b3a41 f i libcpmt:wlocale.obj
 0001:000b2fa6       ?_Rep@?$money_put@GV?$ostreambuf_iterator@GU?$char_traits@G@std@@@std@@@std@@CA?AV?$ostreambuf_iterator@GU?$char_traits@G@std@@@2@V32@GI@Z 100b3fa6 f i libcpmt:wlocale.obj
 0001:000b2fd0       ?_Rep@?$money_put@_WV?$ostreambuf_iterator@_WU?$char_traits@_W@std@@@std@@@std@@CA?AV?$ostreambuf_iterator@_WU?$char_traits@_W@std@@@2@V32@_WI@Z 100b3fd0 f i libcpmt:wlocale.obj
 0001:000b2ffa       ?_Rep@?$num_put@GV?$ostreambuf_iterator@GU?$char_traits@G@std@@@std@@@std@@ABA?AV?$ostreambuf_iterator@GU?$char_traits@G@std@@@2@V32@GI@Z 100b3ffa f i libcpmt:wlocale.obj
 0001:000b3024       ?_Rep@?$num_put@_WV?$ostreambuf_iterator@_WU?$char_traits@_W@std@@@std@@@std@@ABA?AV?$ostreambuf_iterator@_WU?$char_traits@_W@std@@@2@V32@_WI@Z 100b4024 f i libcpmt:wlocale.obj
 0001:000b304e       ?_Tidy@?$_Mpunct@G@std@@AAEXXZ 100b404e f i libcpmt:wlocale.obj
 0001:000b3076       ?_Tidy@?$_Mpunct@_W@std@@AAEXXZ 100b4076 f i libcpmt:wlocale.obj
 0001:000b309e       ?_Tidy@?$basic_string@GU?$char_traits@G@std@@V?$allocator@G@2@@std@@QAEX_NI@Z 100b409e f i libcpmt:wlocale.obj
 0001:000b30e4       ?_Tidy@?$basic_string@_WU?$char_traits@_W@std@@V?$allocator@_W@2@@std@@QAEX_NI@Z 100b40e4 f i libcpmt:wlocale.obj
 0001:000b312a       ?_Tidy@?$numpunct@G@std@@AAEXXZ 100b412a f i libcpmt:wlocale.obj
 0001:000b314a       ?_Tidy@?$numpunct@_W@std@@AAEXXZ 100b414a f i libcpmt:wlocale.obj
 0001:000b316a       ?_Tidy@?$time_get@GV?$istreambuf_iterator@GU?$char_traits@G@std@@@std@@@std@@AAEXXZ 100b416a f i libcpmt:wlocale.obj
 0001:000b318a       ?_Tidy@?$time_get@_WV?$istreambuf_iterator@_WU?$char_traits@_W@std@@@std@@@std@@AAEXXZ 100b418a f i libcpmt:wlocale.obj
 0001:000b31aa       ?_W_Getdays@_Locinfo@std@@QBEPBGXZ 100b41aa f i libcpmt:wlocale.obj
 0001:000b31e3       ?_W_Getmonths@_Locinfo@std@@QBEPBGXZ 100b41e3 f i libcpmt:wlocale.obj
 0001:000b321c       ?_W_Gettnames@_Locinfo@std@@QBE?AV_Timevec@2@XZ 100b421c f i libcpmt:wlocale.obj
 0001:000b3236       ?_Xlen@?$basic_string@GU?$char_traits@G@std@@V?$allocator@G@2@@std@@QBEXXZ 100b4236 f i libcpmt:wlocale.obj
 0001:000b3241       ?_Xlen@?$basic_string@_WU?$char_traits@_W@std@@V?$allocator@_W@2@@std@@QBEXXZ 100b4241 f i libcpmt:wlocale.obj
 0001:000b324c       ?_Xran@?$basic_string@GU?$char_traits@G@std@@V?$allocator@G@2@@std@@QBEXXZ 100b424c f i libcpmt:wlocale.obj
 0001:000b3257       ?_Xran@?$basic_string@_WU?$char_traits@_W@std@@V?$allocator@_W@2@@std@@QBEXXZ 100b4257 f i libcpmt:wlocale.obj
 0001:000b3262       ?allocate@?$_Wrap_alloc@V?$allocator@G@std@@@std@@QAEPAGI@Z 100b4262 f i libcpmt:wlocale.obj
 0001:000b3275       ?allocate@?$_Wrap_alloc@V?$allocator@_W@std@@@std@@QAEPA_WI@Z 100b4275 f i libcpmt:wlocale.obj
 0001:000b3288       ?allocate@?$allocator@G@std@@QAEPAGI@Z 100b4288 f i libcpmt:wlocale.obj
 0001:000b329b       ?allocate@?$allocator@_W@std@@QAEPA_WI@Z 100b429b f i libcpmt:wlocale.obj
 0001:000b32ae       ?append@?$basic_string@GU?$char_traits@G@std@@V?$allocator@G@2@@std@@QAEAAV12@ABV12@@Z 100b42ae f i libcpmt:wlocale.obj
 0001:000b32c1       ?append@?$basic_string@GU?$char_traits@G@std@@V?$allocator@G@2@@std@@QAEAAV12@ABV12@II@Z 100b42c1 f i libcpmt:wlocale.obj
 0001:000b3366       ?append@?$basic_string@GU?$char_traits@G@std@@V?$allocator@G@2@@std@@QAEAAV12@IG@Z 100b4366 f i libcpmt:wlocale.obj
 0001:000b33c9       ?append@?$basic_string@_WU?$char_traits@_W@std@@V?$allocator@_W@2@@std@@QAEAAV12@ABV12@@Z 100b43c9 f i libcpmt:wlocale.obj
 0001:000b33dc       ?append@?$basic_string@_WU?$char_traits@_W@std@@V?$allocator@_W@2@@std@@QAEAAV12@ABV12@II@Z 100b43dc f i libcpmt:wlocale.obj
 0001:000b3481       ?append@?$basic_string@_WU?$char_traits@_W@std@@V?$allocator@_W@2@@std@@QAEAAV12@I_W@Z 100b4481 f i libcpmt:wlocale.obj
 0001:000b34e4       ?assign@?$basic_string@GU?$char_traits@G@std@@V?$allocator@G@2@@std@@QAEAAV12@$$QAV12@@Z 100b44e4 f i libcpmt:wlocale.obj
 0001:000b3509       ?assign@?$basic_string@GU?$char_traits@G@std@@V?$allocator@G@2@@std@@QAEAAV12@ABV12@@Z 100b4509 f i libcpmt:wlocale.obj
 0001:000b351c       ?assign@?$basic_string@GU?$char_traits@G@std@@V?$allocator@G@2@@std@@QAEAAV12@ABV12@II@Z 100b451c f i libcpmt:wlocale.obj
 0001:000b35b0       ?assign@?$basic_string@GU?$char_traits@G@std@@V?$allocator@G@2@@std@@QAEAAV12@IG@Z 100b45b0 f i libcpmt:wlocale.obj
 0001:000b3600       ?assign@?$basic_string@GU?$char_traits@G@std@@V?$allocator@G@2@@std@@QAEAAV12@PBG@Z 100b4600 f i libcpmt:wlocale.obj
 0001:000b3627       ?assign@?$basic_string@GU?$char_traits@G@std@@V?$allocator@G@2@@std@@QAEAAV12@PBGI@Z 100b4627 f i libcpmt:wlocale.obj
 0001:000b36a0       ?assign@?$basic_string@_WU?$char_traits@_W@std@@V?$allocator@_W@2@@std@@QAEAAV12@$$QAV12@@Z 100b46a0 f i libcpmt:wlocale.obj
 0001:000b36c5       ?assign@?$basic_string@_WU?$char_traits@_W@std@@V?$allocator@_W@2@@std@@QAEAAV12@ABV12@@Z 100b46c5 f i libcpmt:wlocale.obj
 0001:000b36d8       ?assign@?$basic_string@_WU?$char_traits@_W@std@@V?$allocator@_W@2@@std@@QAEAAV12@ABV12@II@Z 100b46d8 f i libcpmt:wlocale.obj
 0001:000b376c       ?assign@?$basic_string@_WU?$char_traits@_W@std@@V?$allocator@_W@2@@std@@QAEAAV12@I_W@Z 100b476c f i libcpmt:wlocale.obj
 0001:000b37bc       ?assign@?$basic_string@_WU?$char_traits@_W@std@@V?$allocator@_W@2@@std@@QAEAAV12@PB_W@Z 100b47bc f i libcpmt:wlocale.obj
 0001:000b37e3       ?assign@?$basic_string@_WU?$char_traits@_W@std@@V?$allocator@_W@2@@std@@QAEAAV12@PB_WI@Z 100b47e3 f i libcpmt:wlocale.obj
 0001:000b385c       ?assign@?$char_traits@G@std@@SAPAGPAGIG@Z 100b485c f i libcpmt:wlocale.obj
 0001:000b3872       ?assign@?$char_traits@G@std@@SAXAAGABG@Z 100b4872 f i libcpmt:wlocale.obj
 0001:000b3883       ?assign@?$char_traits@_W@std@@SAPA_WPA_WI_W@Z 100b4883 f i libcpmt:wlocale.obj
 0001:000b3899       ?assign@?$char_traits@_W@std@@SAXAA_WAB_W@Z 100b4899 f i libcpmt:wlocale.obj
 0001:000b38aa       ?begin@?$basic_string@GU?$char_traits@G@std@@V?$allocator@G@2@@std@@QAE?AV?$_String_iterator@V?$_String_val@U?$_Simple_types@G@std@@@std@@@2@XZ 100b48aa f i libcpmt:wlocale.obj
 0001:000b38be       ?begin@?$basic_string@_WU?$char_traits@_W@std@@V?$allocator@_W@2@@std@@QAE?AV?$_String_iterator@V?$_String_val@U?$_Simple_types@_W@std@@@std@@@2@XZ 100b48be f i libcpmt:wlocale.obj
 0001:000b38d2       ?c_str@?$basic_string@GU?$char_traits@G@std@@V?$allocator@G@2@@std@@QBEPBGXZ 100b48d2 f i libcpmt:wlocale.obj
 0001:000b38dd       ?c_str@?$basic_string@_WU?$char_traits@_W@std@@V?$allocator@_W@2@@std@@QBEPB_WXZ 100b48dd f i libcpmt:wlocale.obj
 0001:000b38e8       ?copy@?$char_traits@G@std@@SAPAGPAGPBGI@Z 100b48e8 f i libcpmt:wlocale.obj
 0001:000b390a       ?copy@?$char_traits@_W@std@@SAPA_WPA_WPB_WI@Z 100b490a f i libcpmt:wlocale.obj
 0001:000b392c       ?curr_symbol@?$_Mpunct@G@std@@QBE?AV?$basic_string@GU?$char_traits@G@std@@V?$allocator@G@2@@2@XZ 100b492c f i libcpmt:wlocale.obj
 0001:000b3945       ?curr_symbol@?$_Mpunct@_W@std@@QBE?AV?$basic_string@_WU?$char_traits@_W@std@@V?$allocator@_W@2@@2@XZ 100b4945 f i libcpmt:wlocale.obj
 0001:000b395e       ?date_order@?$time_get@GV?$istreambuf_iterator@GU?$char_traits@G@std@@@std@@@std@@QBE?AW4dateorder@time_base@2@XZ 100b495e f i libcpmt:wlocale.obj
 0001:000b3963       ?date_order@?$time_get@_WV?$istreambuf_iterator@_WU?$char_traits@_W@std@@@std@@@std@@QBE?AW4dateorder@time_base@2@XZ 100b4963 f i libcpmt:wlocale.obj
 0001:000b3968       ?deallocate@?$_Wrap_alloc@V?$allocator@G@std@@@std@@QAEXPAGI@Z 100b4968 f i libcpmt:wlocale.obj
 0001:000b3978       ?deallocate@?$_Wrap_alloc@V?$allocator@_W@std@@@std@@QAEXPA_WI@Z 100b4978 f i libcpmt:wlocale.obj
 0001:000b3988       ?deallocate@?$allocator@G@std@@QAEXPAGI@Z 100b4988 f i libcpmt:wlocale.obj
 0001:000b3998       ?deallocate@?$allocator@_W@std@@QAEXPA_WI@Z 100b4998 f i libcpmt:wlocale.obj
 0001:000b39a8       ?decimal_point@?$_Mpunct@G@std@@QBEGXZ 100b49a8 f i libcpmt:wlocale.obj
 0001:000b39ad       ?decimal_point@?$_Mpunct@_W@std@@QBE_WXZ 100b49ad f i libcpmt:wlocale.obj
 0001:000b39b2       ?decimal_point@?$numpunct@G@std@@QBEGXZ 100b49b2 f i libcpmt:wlocale.obj
 0001:000b39b7       ?decimal_point@?$numpunct@_W@std@@QBE_WXZ 100b49b7 f i libcpmt:wlocale.obj
 0001:000b39bc       ?do_always_noconv@?$codecvt@GDH@std@@MBE_NXZ 100b49bc f i libcpmt:wlocale.obj
 0001:000b39bf       ?do_always_noconv@?$codecvt@_WDH@std@@MBE_NXZ 100b49bf f i libcpmt:wlocale.obj
 0001:000b39c2       ?do_close@?$messages@G@std@@MBEXH@Z 100b49c2 f i libcpmt:wlocale.obj
 0001:000b39c5       ?do_close@?$messages@_W@std@@MBEXH@Z 100b49c5 f i libcpmt:wlocale.obj
 0001:000b39c8       ?do_compare@?$collate@G@std@@MBEHPBG000@Z 100b49c8 f i libcpmt:wlocale.obj
 0001:000b39f9       ?do_compare@?$collate@_W@std@@MBEHPB_W000@Z 100b49f9 f i libcpmt:wlocale.obj
 0001:000b3a2a       ?do_curr_symbol@?$_Mpunct@G@std@@MBE?AV?$basic_string@GU?$char_traits@G@std@@V?$allocator@G@2@@2@XZ 100b4a2a f i libcpmt:wlocale.obj
 0001:000b3a46       ?do_curr_symbol@?$_Mpunct@_W@std@@MBE?AV?$basic_string@_WU?$char_traits@_W@std@@V?$allocator@_W@2@@2@XZ 100b4a46 f i libcpmt:wlocale.obj
 0001:000b3a62       ?do_date_order@?$time_get@GV?$istreambuf_iterator@GU?$char_traits@G@std@@@std@@@std@@MBE?AW4dateorder@time_base@2@XZ 100b4a62 f i libcpmt:wlocale.obj
 0001:000b3a66       ?do_date_order@?$time_get@_WV?$istreambuf_iterator@_WU?$char_traits@_W@std@@@std@@@std@@MBE?AW4dateorder@time_base@2@XZ 100b4a66 f i libcpmt:wlocale.obj
 0001:000b3a6a       ?do_decimal_point@?$_Mpunct@G@std@@MBEGXZ 100b4a6a f i libcpmt:wlocale.obj
 0001:000b3a6f       ?do_decimal_point@?$_Mpunct@_W@std@@MBE_WXZ 100b4a6f f i libcpmt:wlocale.obj
 0001:000b3a74       ?do_decimal_point@?$numpunct@G@std@@MBEGXZ 100b4a74 f i libcpmt:wlocale.obj
 0001:000b3a79       ?do_decimal_point@?$numpunct@_W@std@@MBE_WXZ 100b4a79 f i libcpmt:wlocale.obj
 0001:000b3a7e       ?do_encoding@?$codecvt@GDH@std@@MBEHXZ 100b4a7e f i libcpmt:wlocale.obj
 0001:000b3a81       ?do_encoding@?$codecvt@_WDH@std@@MBEHXZ 100b4a81 f i libcpmt:wlocale.obj
 0001:000b3a84       ?do_falsename@?$numpunct@G@std@@MBE?AV?$basic_string@GU?$char_traits@G@std@@V?$allocator@G@2@@2@XZ 100b4a84 f i libcpmt:wlocale.obj
 0001:000b3aa0       ?do_falsename@?$numpunct@_W@std@@MBE?AV?$basic_string@_WU?$char_traits@_W@std@@V?$allocator@_W@2@@2@XZ 100b4aa0 f i libcpmt:wlocale.obj
 0001:000b3abc       ?do_frac_digits@?$_Mpunct@G@std@@MBEHXZ 100b4abc f i libcpmt:wlocale.obj
 0001:000b3ac0       ?do_frac_digits@?$_Mpunct@_W@std@@MBEHXZ 100b4ac0 f i libcpmt:wlocale.obj
 0001:000b3ac4       ?do_get@?$messages@G@std@@MBE?AV?$basic_string@GU?$char_traits@G@std@@V?$allocator@G@2@@2@HHHABV32@@Z 100b4ac4 f i libcpmt:wlocale.obj
 0001:000b3ae0       ?do_get@?$messages@_W@std@@MBE?AV?$basic_string@_WU?$char_traits@_W@std@@V?$allocator@_W@2@@2@HHHABV32@@Z 100b4ae0 f i libcpmt:wlocale.obj
 0001:000b3afc       ?do_get@?$money_get@GV?$istreambuf_iterator@GU?$char_traits@G@std@@@std@@@std@@MBE?AV?$istreambuf_iterator@GU?$char_traits@G@std@@@2@V32@0_NAAVios_base@2@AAHAAO@Z 100b4afc f i libcpmt:wlocale.obj
 0001:000b3ba8       ?do_get@?$money_get@GV?$istreambuf_iterator@GU?$char_traits@G@std@@@std@@@std@@MBE?AV?$istreambuf_iterator@GU?$char_traits@G@std@@@2@V32@0_NAAVios_base@2@AAHAAV?$basic_string@GU?$char_traits@G@std@@V?$allocator@G@2@@2@@Z 100b4ba8 f i libcpmt:wlocale.obj
 0001:000b3c84       ?do_get@?$money_get@_WV?$istreambuf_iterator@_WU?$char_traits@_W@std@@@std@@@std@@MBE?AV?$istreambuf_iterator@_WU?$char_traits@_W@std@@@2@V32@0_NAAVios_base@2@AAHAAO@Z 100b4c84 f i libcpmt:wlocale.obj
 0001:000b3d30       ?do_get@?$money_get@_WV?$istreambuf_iterator@_WU?$char_traits@_W@std@@@std@@@std@@MBE?AV?$istreambuf_iterator@_WU?$char_traits@_W@std@@@2@V32@0_NAAVios_base@2@AAHAAV?$basic_string@_WU?$char_traits@_W@std@@V?$allocator@_W@2@@2@@Z 100b4d30 f i libcpmt:wlocale.obj
 0001:000b3e0c       ?do_get@?$num_get@GV?$istreambuf_iterator@GU?$char_traits@G@std@@@std@@@std@@MBE?AV?$istreambuf_iterator@GU?$char_traits@G@std@@@2@V32@0AAVios_base@2@AAHAAG@Z 100b4e0c f i libcpmt:wlocale.obj
 0001:000b3ed5       ?do_get@?$num_get@GV?$istreambuf_iterator@GU?$char_traits@G@std@@@std@@@std@@MBE?AV?$istreambuf_iterator@GU?$char_traits@G@std@@@2@V32@0AAVios_base@2@AAHAAI@Z 100b4ed5 f i libcpmt:wlocale.obj
 0001:000b3f9a       ?do_get@?$num_get@GV?$istreambuf_iterator@GU?$char_traits@G@std@@@std@@@std@@MBE?AV?$istreambuf_iterator@GU?$char_traits@G@std@@@2@V32@0AAVios_base@2@AAHAAJ@Z 100b4f9a f i libcpmt:wlocale.obj
 0001:000b404a       ?do_get@?$num_get@GV?$istreambuf_iterator@GU?$char_traits@G@std@@@std@@@std@@MBE?AV?$istreambuf_iterator@GU?$char_traits@G@std@@@2@V32@0AAVios_base@2@AAHAAK@Z 100b504a f i libcpmt:wlocale.obj
 0001:000b40fa       ?do_get@?$num_get@GV?$istreambuf_iterator@GU?$char_traits@G@std@@@std@@@std@@MBE?AV?$istreambuf_iterator@GU?$char_traits@G@std@@@2@V32@0AAVios_base@2@AAHAAM@Z 100b50fa f i libcpmt:wlocale.obj
 0001:000b41ba       ?do_get@?$num_get@GV?$istreambuf_iterator@GU?$char_traits@G@std@@@std@@@std@@MBE?AV?$istreambuf_iterator@GU?$char_traits@G@std@@@2@V32@0AAVios_base@2@AAHAAN@Z 100b51ba f i libcpmt:wlocale.obj
 0001:000b427d       ?do_get@?$num_get@GV?$istreambuf_iterator@GU?$char_traits@G@std@@@std@@@std@@MBE?AV?$istreambuf_iterator@GU?$char_traits@G@std@@@2@V32@0AAVios_base@2@AAHAAO@Z 100b527d f i libcpmt:wlocale.obj
 0001:000b4340       ?do_get@?$num_get@GV?$istreambuf_iterator@GU?$char_traits@G@std@@@std@@@std@@MBE?AV?$istreambuf_iterator@GU?$char_traits@G@std@@@2@V32@0AAVios_base@2@AAHAAPAX@Z 100b5340 f i libcpmt:wlocale.obj
 0001:000b43f2       ?do_get@?$num_get@GV?$istreambuf_iterator@GU?$char_traits@G@std@@@std@@@std@@MBE?AV?$istreambuf_iterator@GU?$char_traits@G@std@@@2@V32@0AAVios_base@2@AAHAA_J@Z 100b53f2 f i libcpmt:wlocale.obj
 0001:000b44a7       ?do_get@?$num_get@GV?$istreambuf_iterator@GU?$char_traits@G@std@@@std@@@std@@MBE?AV?$istreambuf_iterator@GU?$char_traits@G@std@@@2@V32@0AAVios_base@2@AAHAA_K@Z 100b54a7 f i libcpmt:wlocale.obj
 0001:000b455c       ?do_get@?$num_get@GV?$istreambuf_iterator@GU?$char_traits@G@std@@@std@@@std@@MBE?AV?$istreambuf_iterator@GU?$char_traits@G@std@@@2@V32@0AAVios_base@2@AAHAA_N@Z 100b555c f i libcpmt:wlocale.obj
 0001:000b4714       ?do_get@?$num_get@_WV?$istreambuf_iterator@_WU?$char_traits@_W@std@@@std@@@std@@MBE?AV?$istreambuf_iterator@_WU?$char_traits@_W@std@@@2@V32@0AAVios_base@2@AAHAAG@Z 100b5714 f i libcpmt:wlocale.obj
 0001:000b47dd       ?do_get@?$num_get@_WV?$istreambuf_iterator@_WU?$char_traits@_W@std@@@std@@@std@@MBE?AV?$istreambuf_iterator@_WU?$char_traits@_W@std@@@2@V32@0AAVios_base@2@AAHAAI@Z 100b57dd f i libcpmt:wlocale.obj
 0001:000b48a2       ?do_get@?$num_get@_WV?$istreambuf_iterator@_WU?$char_traits@_W@std@@@std@@@std@@MBE?AV?$istreambuf_iterator@_WU?$char_traits@_W@std@@@2@V32@0AAVios_base@2@AAHAAJ@Z 100b58a2 f i libcpmt:wlocale.obj
 0001:000b4952       ?do_get@?$num_get@_WV?$istreambuf_iterator@_WU?$char_traits@_W@std@@@std@@@std@@MBE?AV?$istreambuf_iterator@_WU?$char_traits@_W@std@@@2@V32@0AAVios_base@2@AAHAAK@Z 100b5952 f i libcpmt:wlocale.obj
 0001:000b4a02       ?do_get@?$num_get@_WV?$istreambuf_iterator@_WU?$char_traits@_W@std@@@std@@@std@@MBE?AV?$istreambuf_iterator@_WU?$char_traits@_W@std@@@2@V32@0AAVios_base@2@AAHAAM@Z 100b5a02 f i libcpmt:wlocale.obj
 0001:000b4ac2       ?do_get@?$num_get@_WV?$istreambuf_iterator@_WU?$char_traits@_W@std@@@std@@@std@@MBE?AV?$istreambuf_iterator@_WU?$char_traits@_W@std@@@2@V32@0AAVios_base@2@AAHAAN@Z 100b5ac2 f i libcpmt:wlocale.obj
 0001:000b4b85       ?do_get@?$num_get@_WV?$istreambuf_iterator@_WU?$char_traits@_W@std@@@std@@@std@@MBE?AV?$istreambuf_iterator@_WU?$char_traits@_W@std@@@2@V32@0AAVios_base@2@AAHAAO@Z 100b5b85 f i libcpmt:wlocale.obj
 0001:000b4c48       ?do_get@?$num_get@_WV?$istreambuf_iterator@_WU?$char_traits@_W@std@@@std@@@std@@MBE?AV?$istreambuf_iterator@_WU?$char_traits@_W@std@@@2@V32@0AAVios_base@2@AAHAAPAX@Z 100b5c48 f i libcpmt:wlocale.obj
 0001:000b4cfa       ?do_get@?$num_get@_WV?$istreambuf_iterator@_WU?$char_traits@_W@std@@@std@@@std@@MBE?AV?$istreambuf_iterator@_WU?$char_traits@_W@std@@@2@V32@0AAVios_base@2@AAHAA_J@Z 100b5cfa f i libcpmt:wlocale.obj
 0001:000b4daf       ?do_get@?$num_get@_WV?$istreambuf_iterator@_WU?$char_traits@_W@std@@@std@@@std@@MBE?AV?$istreambuf_iterator@_WU?$char_traits@_W@std@@@2@V32@0AAVios_base@2@AAHAA_K@Z 100b5daf f i libcpmt:wlocale.obj
 0001:000b4e64       ?do_get@?$num_get@_WV?$istreambuf_iterator@_WU?$char_traits@_W@std@@@std@@@std@@MBE?AV?$istreambuf_iterator@_WU?$char_traits@_W@std@@@2@V32@0AAVios_base@2@AAHAA_N@Z 100b5e64 f i libcpmt:wlocale.obj
 0001:000b501c       ?do_get@?$time_get@GV?$istreambuf_iterator@GU?$char_traits@G@std@@@std@@@std@@MBE?AV?$istreambuf_iterator@GU?$char_traits@G@std@@@2@V32@0AAVios_base@2@AAHPAUtm@@DD@Z 100b601c f i libcpmt:wlocale.obj
 0001:000b5385       ?do_get@?$time_get@_WV?$istreambuf_iterator@_WU?$char_traits@_W@std@@@std@@@std@@MBE?AV?$istreambuf_iterator@_WU?$char_traits@_W@std@@@2@V32@0AAVios_base@2@AAHPAUtm@@DD@Z 100b6385 f i libcpmt:wlocale.obj
 0001:000b56ee       ?do_get_date@?$time_get@GV?$istreambuf_iterator@GU?$char_traits@G@std@@@std@@@std@@MBE?AV?$istreambuf_iterator@GU?$char_traits@G@std@@@2@V32@0AAVios_base@2@AAHPAUtm@@@Z 100b66ee f i libcpmt:wlocale.obj
 0001:000b5b41       ?do_get_date@?$time_get@_WV?$istreambuf_iterator@_WU?$char_traits@_W@std@@@std@@@std@@MBE?AV?$istreambuf_iterator@_WU?$char_traits@_W@std@@@2@V32@0AAVios_base@2@AAHPAUtm@@@Z 100b6b41 f i libcpmt:wlocale.obj
 0001:000b5f94       ?do_get_monthname@?$time_get@GV?$istreambuf_iterator@GU?$char_traits@G@std@@@std@@@std@@MBE?AV?$istreambuf_iterator@GU?$char_traits@G@std@@@2@V32@0AAVios_base@2@AAHPAUtm@@@Z 100b6f94 f i libcpmt:wlocale.obj
 0001:000b5fd4       ?do_get_monthname@?$time_get@_WV?$istreambuf_iterator@_WU?$char_traits@_W@std@@@std@@@std@@MBE?AV?$istreambuf_iterator@_WU?$char_traits@_W@std@@@2@V32@0AAVios_base@2@AAHPAUtm@@@Z 100b6fd4 f i libcpmt:wlocale.obj
 0001:000b6014       ?do_get_time@?$time_get@GV?$istreambuf_iterator@GU?$char_traits@G@std@@@std@@@std@@MBE?AV?$istreambuf_iterator@GU?$char_traits@G@std@@@2@V32@0AAVios_base@2@AAHPAUtm@@@Z 100b7014 f i libcpmt:wlocale.obj
 0001:000b6116       ?do_get_time@?$time_get@_WV?$istreambuf_iterator@_WU?$char_traits@_W@std@@@std@@@std@@MBE?AV?$istreambuf_iterator@_WU?$char_traits@_W@std@@@2@V32@0AAVios_base@2@AAHPAUtm@@@Z 100b7116 f i libcpmt:wlocale.obj
 0001:000b6218       ?do_get_weekday@?$time_get@GV?$istreambuf_iterator@GU?$char_traits@G@std@@@std@@@std@@MBE?AV?$istreambuf_iterator@GU?$char_traits@G@std@@@2@V32@0AAVios_base@2@AAHPAUtm@@@Z 100b7218 f i libcpmt:wlocale.obj
 0001:000b6258       ?do_get_weekday@?$time_get@_WV?$istreambuf_iterator@_WU?$char_traits@_W@std@@@std@@@std@@MBE?AV?$istreambuf_iterator@_WU?$char_traits@_W@std@@@2@V32@0AAVios_base@2@AAHPAUtm@@@Z 100b7258 f i libcpmt:wlocale.obj
 0001:000b6298       ?do_get_year@?$time_get@GV?$istreambuf_iterator@GU?$char_traits@G@std@@@std@@@std@@MBE?AV?$istreambuf_iterator@GU?$char_traits@G@std@@@2@V32@0AAVios_base@2@AAHPAUtm@@@Z 100b7298 f i libcpmt:wlocale.obj
 0001:000b6330       ?do_get_year@?$time_get@_WV?$istreambuf_iterator@_WU?$char_traits@_W@std@@@std@@@std@@MBE?AV?$istreambuf_iterator@_WU?$char_traits@_W@std@@@2@V32@0AAVios_base@2@AAHPAUtm@@@Z 100b7330 f i libcpmt:wlocale.obj
 0001:000b63c8       ?do_grouping@?$_Mpunct@G@std@@MBE?AV?$basic_string@DU?$char_traits@D@std@@V?$allocator@D@2@@2@XZ 100b73c8 f i libcpmt:wlocale.obj
 0001:000b63e4       ?do_grouping@?$_Mpunct@_W@std@@MBE?AV?$basic_string@DU?$char_traits@D@std@@V?$allocator@D@2@@2@XZ 100b73e4 f i libcpmt:wlocale.obj
 0001:000b6400       ?do_grouping@?$numpunct@G@std@@MBE?AV?$basic_string@DU?$char_traits@D@std@@V?$allocator@D@2@@2@XZ 100b7400 f i libcpmt:wlocale.obj
 0001:000b641c       ?do_grouping@?$numpunct@_W@std@@MBE?AV?$basic_string@DU?$char_traits@D@std@@V?$allocator@D@2@@2@XZ 100b741c f i libcpmt:wlocale.obj
 0001:000b6438       ?do_hash@?$collate@G@std@@MBEJPBG0@Z 100b7438 f i libcpmt:wlocale.obj
 0001:000b6453       ?do_hash@?$collate@_W@std@@MBEJPB_W0@Z 100b7453 f i libcpmt:wlocale.obj
 0001:000b646e       ?do_in@?$codecvt@GDH@std@@MBEHAAHPBD1AAPBDPAG3AAPAG@Z 100b746e f i libcpmt:wlocale.obj
 0001:000b6508       ?do_in@?$codecvt@_WDH@std@@MBEHAAHPBD1AAPBDPA_W3AAPA_W@Z 100b7508 f i libcpmt:wlocale.obj
 0001:000b65a2       ?do_is@?$ctype@G@std@@MBEPBGPBG0PAF@Z 100b75a2 f i libcpmt:wlocale.obj
 0001:000b65be       ?do_is@?$ctype@G@std@@MBE_NFG@Z 100b75be f i libcpmt:wlocale.obj
 0001:000b65dd       ?do_is@?$ctype@_W@std@@MBEPB_WPB_W0PAF@Z 100b75dd f i libcpmt:wlocale.obj
 0001:000b65f9       ?do_is@?$ctype@_W@std@@MBE_NF_W@Z 100b75f9 f i libcpmt:wlocale.obj
 0001:000b6618       ?do_length@?$codecvt@GDH@std@@MBEHAAHPBD1I@Z 100b7618 f i libcpmt:wlocale.obj
 0001:000b668f       ?do_length@?$codecvt@_WDH@std@@MBEHAAHPBD1I@Z 100b768f f i libcpmt:wlocale.obj
 0001:000b6706       ?do_max_length@?$codecvt@GDH@std@@MBEHXZ 100b7706 f i libcpmt:wlocale.obj
 0001:000b670a       ?do_max_length@?$codecvt@_WDH@std@@MBEHXZ 100b770a f i libcpmt:wlocale.obj
 0001:000b670e       ?do_narrow@?$ctype@G@std@@MBEDGD@Z 100b770e f i libcpmt:wlocale.obj
 0001:000b6717       ?do_narrow@?$ctype@G@std@@MBEPBGPBG0DPAD@Z 100b7717 f i libcpmt:wlocale.obj
 0001:000b676a       ?do_narrow@?$ctype@_W@std@@MBED_WD@Z 100b776a f i libcpmt:wlocale.obj
 0001:000b6773       ?do_narrow@?$ctype@_W@std@@MBEPB_WPB_W0DPAD@Z 100b7773 f i libcpmt:wlocale.obj
 0001:000b67c6       ?do_neg_format@?$_Mpunct@G@std@@MBE?AUpattern@money_base@2@XZ 100b77c6 f i libcpmt:wlocale.obj
 0001:000b67d5       ?do_neg_format@?$_Mpunct@_W@std@@MBE?AUpattern@money_base@2@XZ 100b77d5 f i libcpmt:wlocale.obj
 0001:000b67e4       ?do_negative_sign@?$_Mpunct@G@std@@MBE?AV?$basic_string@GU?$char_traits@G@std@@V?$allocator@G@2@@2@XZ 100b77e4 f i libcpmt:wlocale.obj
 0001:000b6800       ?do_negative_sign@?$_Mpunct@_W@std@@MBE?AV?$basic_string@_WU?$char_traits@_W@std@@V?$allocator@_W@2@@2@XZ 100b7800 f i libcpmt:wlocale.obj
 0001:000b681c       ?do_open@?$messages@G@std@@MBEHABV?$basic_string@DU?$char_traits@D@std@@V?$allocator@D@2@@2@ABVlocale@2@@Z 100b781c f i libcpmt:wlocale.obj
 0001:000b6822       ?do_open@?$messages@_W@std@@MBEHABV?$basic_string@DU?$char_traits@D@std@@V?$allocator@D@2@@2@ABVlocale@2@@Z 100b7822 f i libcpmt:wlocale.obj
 0001:000b6828       ?do_out@?$codecvt@GDH@std@@MBEHAAHPBG1AAPBGPAD3AAPAD@Z 100b7828 f i libcpmt:wlocale.obj
 0001:000b691d       ?do_out@?$codecvt@_WDH@std@@MBEHAAHPB_W1AAPB_WPAD3AAPAD@Z 100b791d f i libcpmt:wlocale.obj
 0001:000b6a12       ?do_pos_format@?$_Mpunct@G@std@@MBE?AUpattern@money_base@2@XZ 100b7a12 f i libcpmt:wlocale.obj
 0001:000b6a21       ?do_pos_format@?$_Mpunct@_W@std@@MBE?AUpattern@money_base@2@XZ 100b7a21 f i libcpmt:wlocale.obj
 0001:000b6a30       ?do_positive_sign@?$_Mpunct@G@std@@MBE?AV?$basic_string@GU?$char_traits@G@std@@V?$allocator@G@2@@2@XZ 100b7a30 f i libcpmt:wlocale.obj
 0001:000b6a4c       ?do_positive_sign@?$_Mpunct@_W@std@@MBE?AV?$basic_string@_WU?$char_traits@_W@std@@V?$allocator@_W@2@@2@XZ 100b7a4c f i libcpmt:wlocale.obj
 0001:000b6a68       ?do_put@?$money_put@GV?$ostreambuf_iterator@GU?$char_traits@G@std@@@std@@@std@@MBE?AV?$ostreambuf_iterator@GU?$char_traits@G@std@@@2@V32@_NAAVios_base@2@GABV?$basic_string@GU?$char_traits@G@std@@V?$allocator@G@2@@2@@Z 100b7a68 f i libcpmt:wlocale.obj
 0001:000b6b87       ?do_put@?$money_put@GV?$ostreambuf_iterator@GU?$char_traits@G@std@@@std@@@std@@MBE?AV?$ostreambuf_iterator@GU?$char_traits@G@std@@@2@V32@_NAAVios_base@2@GO@Z 100b7b87 f i libcpmt:wlocale.obj
 0001:000b6ce8       ?do_put@?$money_put@_WV?$ostreambuf_iterator@_WU?$char_traits@_W@std@@@std@@@std@@MBE?AV?$ostreambuf_iterator@_WU?$char_traits@_W@std@@@2@V32@_NAAVios_base@2@_WABV?$basic_string@_WU?$char_traits@_W@std@@V?$allocator@_W@2@@2@@Z 100b7ce8 f i libcpmt:wlocale.obj
 0001:000b6e07       ?do_put@?$money_put@_WV?$ostreambuf_iterator@_WU?$char_traits@_W@std@@@std@@@std@@MBE?AV?$ostreambuf_iterator@_WU?$char_traits@_W@std@@@2@V32@_NAAVios_base@2@_WO@Z 100b7e07 f i libcpmt:wlocale.obj
 0001:000b6f68       ?do_put@?$num_put@GV?$ostreambuf_iterator@GU?$char_traits@G@std@@@std@@@std@@MBE?AV?$ostreambuf_iterator@GU?$char_traits@G@std@@@2@V32@AAVios_base@2@GJ@Z 100b7f68 f i libcpmt:wlocale.obj
 0001:000b6fd5       ?do_put@?$num_put@GV?$ostreambuf_iterator@GU?$char_traits@G@std@@@std@@@std@@MBE?AV?$ostreambuf_iterator@GU?$char_traits@G@std@@@2@V32@AAVios_base@2@GK@Z 100b7fd5 f i libcpmt:wlocale.obj
 0001:000b7042       ?do_put@?$num_put@GV?$ostreambuf_iterator@GU?$char_traits@G@std@@@std@@@std@@MBE?AV?$ostreambuf_iterator@GU?$char_traits@G@std@@@2@V32@AAVios_base@2@GN@Z 100b8042 f i libcpmt:wlocale.obj
 0001:000b71fa       ?do_put@?$num_put@GV?$ostreambuf_iterator@GU?$char_traits@G@std@@@std@@@std@@MBE?AV?$ostreambuf_iterator@GU?$char_traits@G@std@@@2@V32@AAVios_base@2@GO@Z 100b81fa f i libcpmt:wlocale.obj
 0001:000b7398       ?do_put@?$num_put@GV?$ostreambuf_iterator@GU?$char_traits@G@std@@@std@@@std@@MBE?AV?$ostreambuf_iterator@GU?$char_traits@G@std@@@2@V32@AAVios_base@2@GPBX@Z 100b8398 f i libcpmt:wlocale.obj
 0001:000b73f5       ?do_put@?$num_put@GV?$ostreambuf_iterator@GU?$char_traits@G@std@@@std@@@std@@MBE?AV?$ostreambuf_iterator@GU?$char_traits@G@std@@@2@V32@AAVios_base@2@G_J@Z 100b83f5 f i libcpmt:wlocale.obj
 0001:000b7465       ?do_put@?$num_put@GV?$ostreambuf_iterator@GU?$char_traits@G@std@@@std@@@std@@MBE?AV?$ostreambuf_iterator@GU?$char_traits@G@std@@@2@V32@AAVios_base@2@G_K@Z 100b8465 f i libcpmt:wlocale.obj
 0001:000b74d5       ?do_put@?$num_put@GV?$ostreambuf_iterator@GU?$char_traits@G@std@@@std@@@std@@MBE?AV?$ostreambuf_iterator@GU?$char_traits@G@std@@@2@V32@AAVios_base@2@G_N@Z 100b84d5 f i libcpmt:wlocale.obj
 0001:000b7637       ?do_put@?$num_put@_WV?$ostreambuf_iterator@_WU?$char_traits@_W@std@@@std@@@std@@MBE?AV?$ostreambuf_iterator@_WU?$char_traits@_W@std@@@2@V32@AAVios_base@2@_WJ@Z 100b8637 f i libcpmt:wlocale.obj
 0001:000b76a4       ?do_put@?$num_put@_WV?$ostreambuf_iterator@_WU?$char_traits@_W@std@@@std@@@std@@MBE?AV?$ostreambuf_iterator@_WU?$char_traits@_W@std@@@2@V32@AAVios_base@2@_WK@Z 100b86a4 f i libcpmt:wlocale.obj
 0001:000b7711       ?do_put@?$num_put@_WV?$ostreambuf_iterator@_WU?$char_traits@_W@std@@@std@@@std@@MBE?AV?$ostreambuf_iterator@_WU?$char_traits@_W@std@@@2@V32@AAVios_base@2@_WN@Z 100b8711 f i libcpmt:wlocale.obj
 0001:000b78c9       ?do_put@?$num_put@_WV?$ostreambuf_iterator@_WU?$char_traits@_W@std@@@std@@@std@@MBE?AV?$ostreambuf_iterator@_WU?$char_traits@_W@std@@@2@V32@AAVios_base@2@_WO@Z 100b88c9 f i libcpmt:wlocale.obj
 0001:000b7a67       ?do_put@?$num_put@_WV?$ostreambuf_iterator@_WU?$char_traits@_W@std@@@std@@@std@@MBE?AV?$ostreambuf_iterator@_WU?$char_traits@_W@std@@@2@V32@AAVios_base@2@_WPBX@Z 100b8a67 f i libcpmt:wlocale.obj
 0001:000b7ac4       ?do_put@?$num_put@_WV?$ostreambuf_iterator@_WU?$char_traits@_W@std@@@std@@@std@@MBE?AV?$ostreambuf_iterator@_WU?$char_traits@_W@std@@@2@V32@AAVios_base@2@_W_J@Z 100b8ac4 f i libcpmt:wlocale.obj
 0001:000b7b34       ?do_put@?$num_put@_WV?$ostreambuf_iterator@_WU?$char_traits@_W@std@@@std@@@std@@MBE?AV?$ostreambuf_iterator@_WU?$char_traits@_W@std@@@2@V32@AAVios_base@2@_W_K@Z 100b8b34 f i libcpmt:wlocale.obj
 0001:000b7ba4       ?do_put@?$num_put@_WV?$ostreambuf_iterator@_WU?$char_traits@_W@std@@@std@@@std@@MBE?AV?$ostreambuf_iterator@_WU?$char_traits@_W@std@@@2@V32@AAVios_base@2@_W_N@Z 100b8ba4 f i libcpmt:wlocale.obj
 0001:000b7d06       ?do_put@?$time_put@GV?$ostreambuf_iterator@GU?$char_traits@G@std@@@std@@@std@@MBE?AV?$ostreambuf_iterator@GU?$char_traits@G@std@@@2@V32@AAVios_base@2@GPBUtm@@DD@Z 100b8d06 f i libcpmt:wlocale.obj
 0001:000b7de0       ?do_put@?$time_put@_WV?$ostreambuf_iterator@_WU?$char_traits@_W@std@@@std@@@std@@MBE?AV?$ostreambuf_iterator@_WU?$char_traits@_W@std@@@2@V32@AAVios_base@2@_WPBUtm@@DD@Z 100b8de0 f i libcpmt:wlocale.obj
 0001:000b7eba       ?do_scan_is@?$ctype@G@std@@MBEPBGFPBG0@Z 100b8eba f i libcpmt:wlocale.obj
 0001:000b7ee8       ?do_scan_is@?$ctype@_W@std@@MBEPB_WFPB_W0@Z 100b8ee8 f i libcpmt:wlocale.obj
 0001:000b7f16       ?do_scan_not@?$ctype@G@std@@MBEPBGFPBG0@Z 100b8f16 f i libcpmt:wlocale.obj
 0001:000b7f44       ?do_scan_not@?$ctype@_W@std@@MBEPB_WFPB_W0@Z 100b8f44 f i libcpmt:wlocale.obj
 0001:000b7f72       ?do_thousands_sep@?$_Mpunct@G@std@@MBEGXZ 100b8f72 f i libcpmt:wlocale.obj
 0001:000b7f77       ?do_thousands_sep@?$_Mpunct@_W@std@@MBE_WXZ 100b8f77 f i libcpmt:wlocale.obj
 0001:000b7f7c       ?do_thousands_sep@?$numpunct@G@std@@MBEGXZ 100b8f7c f i libcpmt:wlocale.obj
 0001:000b7f81       ?do_thousands_sep@?$numpunct@_W@std@@MBE_WXZ 100b8f81 f i libcpmt:wlocale.obj
 0001:000b7f86       ?do_tolower@?$ctype@G@std@@MBEGG@Z 100b8f86 f i libcpmt:wlocale.obj
 0001:000b7f9b       ?do_tolower@?$ctype@G@std@@MBEPBGPAGPBG@Z 100b8f9b f i libcpmt:wlocale.obj
 0001:000b7fe2       ?do_tolower@?$ctype@_W@std@@MBEPB_WPA_WPB_W@Z 100b8fe2 f i libcpmt:wlocale.obj
 0001:000b8029       ?do_tolower@?$ctype@_W@std@@MBE_W_W@Z 100b9029 f i libcpmt:wlocale.obj
 0001:000b803e       ?do_toupper@?$ctype@G@std@@MBEGG@Z 100b903e f i libcpmt:wlocale.obj
 0001:000b8053       ?do_toupper@?$ctype@G@std@@MBEPBGPAGPBG@Z 100b9053 f i libcpmt:wlocale.obj
 0001:000b809a       ?do_toupper@?$ctype@_W@std@@MBEPB_WPA_WPB_W@Z 100b909a f i libcpmt:wlocale.obj
 0001:000b80e1       ?do_toupper@?$ctype@_W@std@@MBE_W_W@Z 100b90e1 f i libcpmt:wlocale.obj
 0001:000b80f6       ?do_transform@?$collate@G@std@@MBE?AV?$basic_string@GU?$char_traits@G@std@@V?$allocator@G@2@@2@PBG0@Z 100b90f6 f i libcpmt:wlocale.obj
 0001:000b8184       ?do_transform@?$collate@_W@std@@MBE?AV?$basic_string@_WU?$char_traits@_W@std@@V?$allocator@_W@2@@2@PB_W0@Z 100b9184 f i libcpmt:wlocale.obj
 0001:000b8212       ?do_truename@?$numpunct@G@std@@MBE?AV?$basic_string@GU?$char_traits@G@std@@V?$allocator@G@2@@2@XZ 100b9212 f i libcpmt:wlocale.obj
 0001:000b822e       ?do_truename@?$numpunct@_W@std@@MBE?AV?$basic_string@_WU?$char_traits@_W@std@@V?$allocator@_W@2@@2@XZ 100b922e f i libcpmt:wlocale.obj
 0001:000b824a       ?do_unshift@?$codecvt@GDH@std@@MBEHAAHPAD1AAPAD@Z 100b924a f i libcpmt:wlocale.obj
 0001:000b82d0       ?do_unshift@?$codecvt@_WDH@std@@MBEHAAHPAD1AAPAD@Z 100b92d0 f i libcpmt:wlocale.obj
 0001:000b8356       ?do_widen@?$ctype@G@std@@MBEGD@Z 100b9356 f i libcpmt:wlocale.obj
 0001:000b835f       ?do_widen@?$ctype@G@std@@MBEPBDPBD0PAG@Z 100b935f f i libcpmt:wlocale.obj
 0001:000b83ad       ?do_widen@?$ctype@_W@std@@MBEPBDPBD0PA_W@Z 100b93ad f i libcpmt:wlocale.obj
 0001:000b83fb       ?do_widen@?$ctype@_W@std@@MBE_WD@Z 100b93fb f i libcpmt:wlocale.obj
 0001:000b8404       ?empty@?$basic_string@GU?$char_traits@G@std@@V?$allocator@G@2@@std@@QBE_NXZ 100b9404 f i libcpmt:wlocale.obj
 0001:000b840d       ?empty@?$basic_string@_WU?$char_traits@_W@std@@V?$allocator@_W@2@@std@@QBE_NXZ 100b940d f i libcpmt:wlocale.obj
 0001:000b8416       ?end@?$basic_string@GU?$char_traits@G@std@@V?$allocator@G@2@@std@@QAE?AV?$_String_iterator@V?$_String_val@U?$_Simple_types@G@std@@@std@@@2@XZ 100b9416 f i libcpmt:wlocale.obj
 0001:000b8434       ?end@?$basic_string@_WU?$char_traits@_W@std@@V?$allocator@_W@2@@std@@QAE?AV?$_String_iterator@V?$_String_val@U?$_Simple_types@_W@std@@@std@@@2@XZ 100b9434 f i libcpmt:wlocale.obj
 0001:000b8452       ?eof@?$char_traits@G@std@@SAGXZ 100b9452 f i libcpmt:wlocale.obj
 0001:000b8458       ?eof@?$char_traits@_W@std@@SAGXZ 100b9458 f i libcpmt:wlocale.obj
 0001:000b845e       ?eq_int_type@?$char_traits@G@std@@SA_NABG0@Z 100b945e f i libcpmt:wlocale.obj
 0001:000b8474       ?eq_int_type@?$char_traits@_W@std@@SA_NABG0@Z 100b9474 f i libcpmt:wlocale.obj
 0001:000b848a       ?equal@?$istreambuf_iterator@GU?$char_traits@G@std@@@std@@QBE_NABV12@@Z 100b948a f i libcpmt:wlocale.obj
 0001:000b84c5       ?equal@?$istreambuf_iterator@_WU?$char_traits@_W@std@@@std@@QBE_NABV12@@Z 100b94c5 f i libcpmt:wlocale.obj
 0001:000b8500       ?erase@?$basic_string@GU?$char_traits@G@std@@V?$allocator@G@2@@std@@QAEAAV12@I@Z 100b9500 f i libcpmt:wlocale.obj
 0001:000b8533       ?erase@?$basic_string@GU?$char_traits@G@std@@V?$allocator@G@2@@std@@QAEAAV12@II@Z 100b9533 f i libcpmt:wlocale.obj
 0001:000b85b7       ?erase@?$basic_string@_WU?$char_traits@_W@std@@V?$allocator@_W@2@@std@@QAEAAV12@I@Z 100b95b7 f i libcpmt:wlocale.obj
 0001:000b85ea       ?erase@?$basic_string@_WU?$char_traits@_W@std@@V?$allocator@_W@2@@std@@QAEAAV12@II@Z 100b95ea f i libcpmt:wlocale.obj
 0001:000b866e       ?falsename@?$numpunct@G@std@@QBE?AV?$basic_string@GU?$char_traits@G@std@@V?$allocator@G@2@@2@XZ 100b966e f i libcpmt:wlocale.obj
 0001:000b8687       ?falsename@?$numpunct@_W@std@@QBE?AV?$basic_string@_WU?$char_traits@_W@std@@V?$allocator@_W@2@@2@XZ 100b9687 f i libcpmt:wlocale.obj
 0001:000b86a0       ?frac_digits@?$_Mpunct@G@std@@QBEHXZ 100b96a0 f i libcpmt:wlocale.obj
 0001:000b86a5       ?frac_digits@?$_Mpunct@_W@std@@QBEHXZ 100b96a5 f i libcpmt:wlocale.obj
 0001:000b86aa       ?get_allocator@?$basic_string@GU?$char_traits@G@std@@V?$allocator@G@2@@std@@QBE?AV?$allocator@G@2@XZ 100b96aa f i libcpmt:wlocale.obj
 0001:000b86b4       ?get_allocator@?$basic_string@_WU?$char_traits@_W@std@@V?$allocator@_W@2@@std@@QBE?AV?$allocator@_W@2@XZ 100b96b4 f i libcpmt:wlocale.obj
 0001:000b86be       ?get_monthname@?$time_get@GV?$istreambuf_iterator@GU?$char_traits@G@std@@@std@@@std@@QBE?AV?$istreambuf_iterator@GU?$char_traits@G@std@@@2@V32@0AAVios_base@2@AAHPAUtm@@@Z 100b96be f i libcpmt:wlocale.obj
 0001:000b86e5       ?get_monthname@?$time_get@_WV?$istreambuf_iterator@_WU?$char_traits@_W@std@@@std@@@std@@QBE?AV?$istreambuf_iterator@_WU?$char_traits@_W@std@@@2@V32@0AAVios_base@2@AAHPAUtm@@@Z 100b96e5 f i libcpmt:wlocale.obj
 0001:000b870c       ?get_weekday@?$time_get@GV?$istreambuf_iterator@GU?$char_traits@G@std@@@std@@@std@@QBE?AV?$istreambuf_iterator@GU?$char_traits@G@std@@@2@V32@0AAVios_base@2@AAHPAUtm@@@Z 100b970c f i libcpmt:wlocale.obj
 0001:000b8733       ?get_weekday@?$time_get@_WV?$istreambuf_iterator@_WU?$char_traits@_W@std@@@std@@@std@@QBE?AV?$istreambuf_iterator@_WU?$char_traits@_W@std@@@2@V32@0AAVios_base@2@AAHPAUtm@@@Z 100b9733 f i libcpmt:wlocale.obj
 0001:000b875a       ?get_year@?$time_get@GV?$istreambuf_iterator@GU?$char_traits@G@std@@@std@@@std@@QBE?AV?$istreambuf_iterator@GU?$char_traits@G@std@@@2@V32@0AAVios_base@2@AAHPAUtm@@@Z 100b975a f i libcpmt:wlocale.obj
 0001:000b8781       ?get_year@?$time_get@_WV?$istreambuf_iterator@_WU?$char_traits@_W@std@@@std@@@std@@QBE?AV?$istreambuf_iterator@_WU?$char_traits@_W@std@@@2@V32@0AAVios_base@2@AAHPAUtm@@@Z 100b9781 f i libcpmt:wlocale.obj
 0001:000b87a8       ?gptr@?$basic_streambuf@GU?$char_traits@G@std@@@std@@IBEPAGXZ 100b97a8 f i libcpmt:wlocale.obj
 0001:000b87ae       ?gptr@?$basic_streambuf@_WU?$char_traits@_W@std@@@std@@IBEPA_WXZ 100b97ae f i libcpmt:wlocale.obj
 0001:000b87b4       ?grouping@?$_Mpunct@G@std@@QBE?AV?$basic_string@DU?$char_traits@D@std@@V?$allocator@D@2@@2@XZ 100b97b4 f i libcpmt:wlocale.obj
 0001:000b87cd       ?grouping@?$_Mpunct@_W@std@@QBE?AV?$basic_string@DU?$char_traits@D@std@@V?$allocator@D@2@@2@XZ 100b97cd f i libcpmt:wlocale.obj
 0001:000b87e6       ?grouping@?$numpunct@G@std@@QBE?AV?$basic_string@DU?$char_traits@D@std@@V?$allocator@D@2@@2@XZ 100b97e6 f i libcpmt:wlocale.obj
 0001:000b87ff       ?grouping@?$numpunct@_W@std@@QBE?AV?$basic_string@DU?$char_traits@D@std@@V?$allocator@D@2@@2@XZ 100b97ff f i libcpmt:wlocale.obj
 0001:000b8818       ?insert@?$basic_string@GU?$char_traits@G@std@@V?$allocator@G@2@@std@@QAEAAV12@IIG@Z 100b9818 f i libcpmt:wlocale.obj
 0001:000b88c9       ?insert@?$basic_string@_WU?$char_traits@_W@std@@V?$allocator@_W@2@@std@@QAEAAV12@II_W@Z 100b98c9 f i libcpmt:wlocale.obj
 0001:000b897a       ?is@?$ctype@G@std@@QBE_NFG@Z 100b997a f i libcpmt:wlocale.obj
 0001:000b8983       ?is@?$ctype@_W@std@@QBE_NF_W@Z 100b9983 f i libcpmt:wlocale.obj
 0001:000b898c       ?length@?$char_traits@G@std@@SAIPBG@Z 100b998c f i libcpmt:wlocale.obj
 0001:000b89a2       ?length@?$char_traits@_W@std@@SAIPB_W@Z 100b99a2 f i libcpmt:wlocale.obj
 0001:000b89b8       ?max_size@?$_Wrap_alloc@V?$allocator@G@std@@@std@@QBEIXZ 100b99b8 f i libcpmt:wlocale.obj
 0001:000b89be       ?max_size@?$_Wrap_alloc@V?$allocator@_W@std@@@std@@QBEIXZ 100b99be f i libcpmt:wlocale.obj
 0001:000b89c4       ?max_size@?$allocator@G@std@@QBEIXZ 100b99c4 f i libcpmt:wlocale.obj
 0001:000b89ca       ?max_size@?$allocator@_W@std@@QBEIXZ 100b99ca f i libcpmt:wlocale.obj
 0001:000b89d0       ?max_size@?$allocator_traits@V?$allocator@G@std@@@std@@SAIABV?$allocator@G@2@@Z 100b99d0 f i libcpmt:wlocale.obj
 0001:000b89d6       ?max_size@?$allocator_traits@V?$allocator@_W@std@@@std@@SAIABV?$allocator@_W@2@@Z 100b99d6 f i libcpmt:wlocale.obj
 0001:000b89dc       ?max_size@?$basic_string@GU?$char_traits@G@std@@V?$allocator@G@2@@std@@QBEIXZ 100b99dc f i libcpmt:wlocale.obj
 0001:000b89e2       ?max_size@?$basic_string@_WU?$char_traits@_W@std@@V?$allocator@_W@2@@std@@QBEIXZ 100b99e2 f i libcpmt:wlocale.obj
 0001:000b89e8       ?move@?$char_traits@G@std@@SAPAGPAGPBGI@Z 100b99e8 f i libcpmt:wlocale.obj
 0001:000b8a0a       ?move@?$char_traits@_W@std@@SAPA_WPA_WPB_WI@Z 100b9a0a f i libcpmt:wlocale.obj
 0001:000b8a2c       ?name@locale@std@@QBE?AV?$basic_string@DU?$char_traits@D@std@@V?$allocator@D@2@@2@XZ 100b9a2c f i libcpmt:wlocale.obj
 0001:000b8aab       ?narrow@?$ctype@G@std@@QBEDGD@Z 100b9aab f i libcpmt:wlocale.obj
 0001:000b8ab4       ?narrow@?$ctype@_W@std@@QBED_WD@Z 100b9ab4 f i libcpmt:wlocale.obj
 0001:000b8abd       ?neg_format@?$_Mpunct@G@std@@QBE?AUpattern@money_base@2@XZ 100b9abd f i libcpmt:wlocale.obj
 0001:000b8acf       ?neg_format@?$_Mpunct@_W@std@@QBE?AUpattern@money_base@2@XZ 100b9acf f i libcpmt:wlocale.obj
 0001:000b8ae1       ?negative_sign@?$_Mpunct@G@std@@QBE?AV?$basic_string@GU?$char_traits@G@std@@V?$allocator@G@2@@2@XZ 100b9ae1 f i libcpmt:wlocale.obj
 0001:000b8afa       ?negative_sign@?$_Mpunct@_W@std@@QBE?AV?$basic_string@_WU?$char_traits@_W@std@@V?$allocator@_W@2@@2@XZ 100b9afa f i libcpmt:wlocale.obj
 0001:000b8b13       ?pos_format@?$_Mpunct@G@std@@QBE?AUpattern@money_base@2@XZ 100b9b13 f i libcpmt:wlocale.obj
 0001:000b8b25       ?pos_format@?$_Mpunct@_W@std@@QBE?AUpattern@money_base@2@XZ 100b9b25 f i libcpmt:wlocale.obj
 0001:000b8b37       ?positive_sign@?$_Mpunct@G@std@@QBE?AV?$basic_string@GU?$char_traits@G@std@@V?$allocator@G@2@@2@XZ 100b9b37 f i libcpmt:wlocale.obj
 0001:000b8b50       ?positive_sign@?$_Mpunct@_W@std@@QBE?AV?$basic_string@_WU?$char_traits@_W@std@@V?$allocator@_W@2@@2@XZ 100b9b50 f i libcpmt:wlocale.obj
 0001:000b8b69       ?replace@?$basic_string@GU?$char_traits@G@std@@V?$allocator@G@2@@std@@QAEAAV12@IIABV12@II@Z 100b9b69 f i libcpmt:wlocale.obj
 0001:000b8e72       ?replace@?$basic_string@GU?$char_traits@G@std@@V?$allocator@G@2@@std@@QAEAAV12@IIPBGI@Z 100b9e72 f i libcpmt:wlocale.obj
 0001:000b8fe7       ?replace@?$basic_string@GU?$char_traits@G@std@@V?$allocator@G@2@@std@@QAEAAV12@V?$_String_const_iterator@V?$_String_val@U?$_Simple_types@G@std@@@std@@@2@0V?$_String_iterator@V?$_String_val@U?$_Simple_types@G@std@@@std@@@2@1@Z 100b9fe7 f i libcpmt:wlocale.obj
 0001:000b9071       ?replace@?$basic_string@_WU?$char_traits@_W@std@@V?$allocator@_W@2@@std@@QAEAAV12@IIABV12@II@Z 100ba071 f i libcpmt:wlocale.obj
 0001:000b937a       ?replace@?$basic_string@_WU?$char_traits@_W@std@@V?$allocator@_W@2@@std@@QAEAAV12@IIPB_WI@Z 100ba37a f i libcpmt:wlocale.obj
 0001:000b94ef       ?replace@?$basic_string@_WU?$char_traits@_W@std@@V?$allocator@_W@2@@std@@QAEAAV12@V?$_String_const_iterator@V?$_String_val@U?$_Simple_types@_W@std@@@std@@@2@0V?$_String_iterator@V?$_String_val@U?$_Simple_types@_W@std@@@std@@@2@1@Z 100ba4ef f i libcpmt:wlocale.obj
 0001:000b9579       ?resize@?$basic_string@GU?$char_traits@G@std@@V?$allocator@G@2@@std@@QAEXI@Z 100ba579 f i libcpmt:wlocale.obj
 0001:000b958a       ?resize@?$basic_string@GU?$char_traits@G@std@@V?$allocator@G@2@@std@@QAEXIG@Z 100ba58a f i libcpmt:wlocale.obj
 0001:000b95b8       ?resize@?$basic_string@_WU?$char_traits@_W@std@@V?$allocator@_W@2@@std@@QAEXI@Z 100ba5b8 f i libcpmt:wlocale.obj
 0001:000b95c9       ?resize@?$basic_string@_WU?$char_traits@_W@std@@V?$allocator@_W@2@@std@@QAEXI_W@Z 100ba5c9 f i libcpmt:wlocale.obj
 0001:000b95f7       ?sbumpc@?$basic_streambuf@GU?$char_traits@G@std@@@std@@QAEGXZ 100ba5f7 f i libcpmt:wlocale.obj
 0001:000b9625       ?sbumpc@?$basic_streambuf@_WU?$char_traits@_W@std@@@std@@QAEGXZ 100ba625 f i libcpmt:wlocale.obj
 0001:000b9653       ?select_on_container_copy_construction@?$_Wrap_alloc@V?$allocator@G@std@@@std@@QBE?AU12@XZ 100ba653 f i libcpmt:wlocale.obj
 0001:000b965d       ?select_on_container_copy_construction@?$_Wrap_alloc@V?$allocator@_W@std@@@std@@QBE?AU12@XZ 100ba65d f i libcpmt:wlocale.obj
 0001:000b9667       ?select_on_container_copy_construction@?$allocator@G@std@@QBE?AV12@XZ 100ba667 f i libcpmt:wlocale.obj
 0001:000b9671       ?select_on_container_copy_construction@?$allocator@_W@std@@QBE?AV12@XZ 100ba671 f i libcpmt:wlocale.obj
 0001:000b967b       ?select_on_container_copy_construction@?$allocator_traits@V?$allocator@G@std@@@std@@SA?AV?$allocator@G@2@ABV32@@Z 100ba67b f i libcpmt:wlocale.obj
 0001:000b9683       ?select_on_container_copy_construction@?$allocator_traits@V?$allocator@_W@std@@@std@@SA?AV?$allocator@_W@2@ABV32@@Z 100ba683 f i libcpmt:wlocale.obj
 0001:000b968b       ?sgetc@?$basic_streambuf@GU?$char_traits@G@std@@@std@@QAEGXZ 100ba68b f i libcpmt:wlocale.obj
 0001:000b96ae       ?sgetc@?$basic_streambuf@_WU?$char_traits@_W@std@@@std@@QAEGXZ 100ba6ae f i libcpmt:wlocale.obj
 0001:000b96d1       ?size@?$basic_string@GU?$char_traits@G@std@@V?$allocator@G@2@@std@@QBEIXZ 100ba6d1 f i libcpmt:wlocale.obj
 0001:000b96d5       ?size@?$basic_string@_WU?$char_traits@_W@std@@V?$allocator@_W@2@@std@@QBEIXZ 100ba6d5 f i libcpmt:wlocale.obj
 0001:000b96d9       ?sputc@?$basic_streambuf@GU?$char_traits@G@std@@@std@@QAEGG@Z 100ba6d9 f i libcpmt:wlocale.obj
 0001:000b9714       ?sputc@?$basic_streambuf@_WU?$char_traits@_W@std@@@std@@QAEG_W@Z 100ba714 f i libcpmt:wlocale.obj
 0001:000b974f       ?thousands_sep@?$_Mpunct@G@std@@QBEGXZ 100ba74f f i libcpmt:wlocale.obj
 0001:000b9754       ?thousands_sep@?$_Mpunct@_W@std@@QBE_WXZ 100ba754 f i libcpmt:wlocale.obj
 0001:000b9759       ?thousands_sep@?$numpunct@G@std@@QBEGXZ 100ba759 f i libcpmt:wlocale.obj
 0001:000b975e       ?thousands_sep@?$numpunct@_W@std@@QBE_WXZ 100ba75e f i libcpmt:wlocale.obj
 0001:000b9763       ?to_char_type@?$char_traits@G@std@@SAGABG@Z 100ba763 f i libcpmt:wlocale.obj
 0001:000b976e       ?to_char_type@?$char_traits@_W@std@@SA_WABG@Z 100ba76e f i libcpmt:wlocale.obj
 0001:000b9779       ?to_int_type@?$char_traits@G@std@@SAGABG@Z 100ba779 f i libcpmt:wlocale.obj
 0001:000b9784       ?to_int_type@?$char_traits@_W@std@@SAGAB_W@Z 100ba784 f i libcpmt:wlocale.obj
 0001:000b978f       ?truename@?$numpunct@G@std@@QBE?AV?$basic_string@GU?$char_traits@G@std@@V?$allocator@G@2@@2@XZ 100ba78f f i libcpmt:wlocale.obj
 0001:000b97a8       ?truename@?$numpunct@_W@std@@QBE?AV?$basic_string@_WU?$char_traits@_W@std@@V?$allocator@_W@2@@2@XZ 100ba7a8 f i libcpmt:wlocale.obj
 0001:000b97c1       ?widen@?$ctype@G@std@@QBEGD@Z 100ba7c1 f i libcpmt:wlocale.obj
 0001:000b97ca       ?widen@?$ctype@G@std@@QBEPBDPBD0PAG@Z 100ba7ca f i libcpmt:wlocale.obj
 0001:000b97d3       ?widen@?$ctype@_W@std@@QBEPBDPBD0PA_W@Z 100ba7d3 f i libcpmt:wlocale.obj
 0001:000b97dc       ?widen@?$ctype@_W@std@@QBE_WD@Z 100ba7dc f i libcpmt:wlocale.obj
 0001:000b97e5       _wmemcpy                   100ba7e5 f i libcpmt:wlocale.obj
 0001:000b97fe       _wmemmove                  100ba7fe f i libcpmt:wlocale.obj
 0001:000b9817       _wmemset                   100ba817 f i libcpmt:wlocale.obj
 0001:000b9841       ??$_Copy_impl@PADV?$ostreambuf_iterator@DU?$char_traits@D@std@@@std@@@std@@YA?AV?$ostreambuf_iterator@DU?$char_traits@D@std@@@0@PAD0V10@@Z 100ba841 f i libcpmt:xlocale.obj
 0001:000b9863       ??$_Copy_impl@PADV?$ostreambuf_iterator@DU?$char_traits@D@std@@@std@@@std@@YA?AV?$ostreambuf_iterator@DU?$char_traits@D@std@@@0@PAD0V10@U_Nonscalar_ptr_iterator_tag@0@@Z 100ba863 f i libcpmt:xlocale.obj
 0001:000b98a3       ??$_Getvals@D@?$_Mpunct@D@std@@IAEXDPBUlconv@@@Z 100ba8a3 f i libcpmt:xlocale.obj
 0001:000b991f       ??$_Getvals@D@?$time_get@DV?$istreambuf_iterator@DU?$char_traits@D@std@@@std@@@std@@IAEXDABV_Locinfo@1@@Z 100ba91f f i libcpmt:xlocale.obj
 0001:000b998c       ??$_LStrcoll@D@std@@YAHPBD000PBU_Collvec@@@Z 100ba98c f i libcpmt:xlocale.obj
 0001:000b9995       ??$_LStrxfrm@D@std@@YAIPAD0PBD1PBU_Collvec@@@Z 100ba995 f i libcpmt:xlocale.obj
 0001:000b999e       ??$_Ptr_cat@PADV?$ostreambuf_iterator@DU?$char_traits@D@std@@@std@@@std@@YA?AU_Nonscalar_ptr_iterator_tag@0@AAPADAAV?$ostreambuf_iterator@DU?$char_traits@D@std@@@0@@Z 100ba99e f i libcpmt:xlocale.obj
 0001:000b99a9       ??$_Rechecked@V?$ostreambuf_iterator@DU?$char_traits@D@std@@@std@@V12@@std@@YAAAV?$ostreambuf_iterator@DU?$char_traits@D@std@@@0@AAV10@V10@@Z 100ba9a9 f i libcpmt:xlocale.obj
 0001:000b99bc       ??$_Unchecked@PAD@std@@YAPADPAD@Z 100ba9bc f i libcpmt:xlocale.obj
 0001:000b99c4       ??$_Unchecked@V?$ostreambuf_iterator@DU?$char_traits@D@std@@@std@@@std@@YA?AV?$ostreambuf_iterator@DU?$char_traits@D@std@@@0@V10@@Z 100ba9c4 f i libcpmt:xlocale.obj
 0001:000b99d7       ??$assign@V?$_String_iterator@V?$_String_val@U?$_Simple_types@D@std@@@std@@@std@@@?$basic_string@DU?$char_traits@D@std@@V?$allocator@D@2@@std@@QAEAAV01@V?$_String_iterator@V?$_String_val@U?$_Simple_types@D@std@@@std@@@1@0@Z 100ba9d7 f i libcpmt:xlocale.obj
 0001:000b9a08       ??$copy@PADV?$ostreambuf_iterator@DU?$char_traits@D@std@@@std@@@std@@YA?AV?$ostreambuf_iterator@DU?$char_traits@D@std@@@0@PAD0V10@@Z 100baa08 f i libcpmt:xlocale.obj
 0001:000b9a38       ??$use_facet@V?$collate@D@std@@@std@@YAABV?$collate@D@0@ABVlocale@0@@Z 100baa38 f i libcpmt:xlocale.obj
 0001:000b9ad1       ??$use_facet@V?$messages@D@std@@@std@@YAABV?$messages@D@0@ABVlocale@0@@Z 100baad1 f i libcpmt:xlocale.obj
 0001:000b9b6a       ??$use_facet@V?$money_get@DV?$istreambuf_iterator@DU?$char_traits@D@std@@@std@@@std@@@std@@YAABV?$money_get@DV?$istreambuf_iterator@DU?$char_traits@D@std@@@std@@@0@ABVlocale@0@@Z 100bab6a f i libcpmt:xlocale.obj
 0001:000b9c03       ??$use_facet@V?$money_put@DV?$ostreambuf_iterator@DU?$char_traits@D@std@@@std@@@std@@@std@@YAABV?$money_put@DV?$ostreambuf_iterator@DU?$char_traits@D@std@@@std@@@0@ABVlocale@0@@Z 100bac03 f i libcpmt:xlocale.obj
 0001:000b9c9c       ??$use_facet@V?$moneypunct@D$00@std@@@std@@YAABV?$moneypunct@D$00@0@ABVlocale@0@@Z 100bac9c f i libcpmt:xlocale.obj
 0001:000b9d35       ??$use_facet@V?$moneypunct@D$0A@@std@@@std@@YAABV?$moneypunct@D$0A@@0@ABVlocale@0@@Z 100bad35 f i libcpmt:xlocale.obj
 0001:000b9dce       ??$use_facet@V?$time_get@DV?$istreambuf_iterator@DU?$char_traits@D@std@@@std@@@std@@@std@@YAABV?$time_get@DV?$istreambuf_iterator@DU?$char_traits@D@std@@@std@@@0@ABVlocale@0@@Z 100badce f i libcpmt:xlocale.obj
 0001:000b9e67       ??$use_facet@V?$time_put@DV?$ostreambuf_iterator@DU?$char_traits@D@std@@@std@@@std@@@std@@YAABV?$time_put@DV?$ostreambuf_iterator@DU?$char_traits@D@std@@@std@@@0@ABVlocale@0@@Z 100bae67 f i libcpmt:xlocale.obj
 0001:000b9f00       ??0?$_Mpunct@D@std@@QAE@ABV_Locinfo@1@I_N1@Z 100baf00 f i libcpmt:xlocale.obj
 0001:000b9f3c       ??0?$_String_const_iterator@V?$_String_val@U?$_Simple_types@D@std@@@std@@@std@@QAE@XZ 100baf3c f i libcpmt:xlocale.obj
 0001:000b9f42       ??0?$basic_string@DU?$char_traits@D@std@@V?$allocator@D@2@@std@@QAE@PBDI@Z 100baf42 f i libcpmt:xlocale.obj
 0001:000b9f68       ??0?$collate@D@std@@QAE@ABV_Locinfo@1@I@Z 100baf68 f i libcpmt:xlocale.obj
 0001:000b9f8c       ??0?$messages@D@std@@QAE@ABV_Locinfo@1@I@Z 100baf8c f i libcpmt:xlocale.obj
 0001:000b9fa1       ??0?$money_get@DV?$istreambuf_iterator@DU?$char_traits@D@std@@@std@@@std@@QAE@ABV_Locinfo@1@I@Z 100bafa1 f i libcpmt:xlocale.obj
 0001:000b9fb6       ??0?$money_put@DV?$ostreambuf_iterator@DU?$char_traits@D@std@@@std@@@std@@QAE@ABV_Locinfo@1@I@Z 100bafb6 f i libcpmt:xlocale.obj
 0001:000b9fcb       ??0?$moneypunct@D$00@std@@QAE@ABV_Locinfo@1@I_N@Z 100bafcb f i libcpmt:xlocale.obj
 0001:000b9fee       ??0?$moneypunct@D$0A@@std@@QAE@ABV_Locinfo@1@I_N@Z 100bafee f i libcpmt:xlocale.obj
 0001:000ba011       ??0?$time_get@DV?$istreambuf_iterator@DU?$char_traits@D@std@@@std@@@std@@QAE@ABV_Locinfo@1@I@Z 100bb011 f i libcpmt:xlocale.obj
 0001:000ba044       ??0?$time_put@DV?$ostreambuf_iterator@DU?$char_traits@D@std@@@std@@@std@@QAE@ABV_Locinfo@1@I@Z 100bb044 f i libcpmt:xlocale.obj
 0001:000ba069       ??1?$_Mpunct@D@std@@MAE@XZ 100bb069 f i libcpmt:xlocale.obj
 0001:000ba07f       ??1?$collate@D@std@@MAE@XZ 100bb07f f i libcpmt:xlocale.obj
 0001:000ba099       ??1?$messages@D@std@@MAE@XZ 100bb099 f i libcpmt:xlocale.obj
 0001:000ba0a0       ??1?$money_get@DV?$istreambuf_iterator@DU?$char_traits@D@std@@@std@@@std@@MAE@XZ 100bb0a0 f i libcpmt:xlocale.obj
 0001:000ba0a7       ??1?$money_put@DV?$ostreambuf_iterator@DU?$char_traits@D@std@@@std@@@std@@MAE@XZ 100bb0a7 f i libcpmt:xlocale.obj
 0001:000ba0ae       ??1?$moneypunct@D$00@std@@MAE@XZ 100bb0ae f i libcpmt:xlocale.obj
 0001:000ba0c4       ??1?$moneypunct@D$0A@@std@@MAE@XZ 100bb0c4 f i libcpmt:xlocale.obj
 0001:000ba0da       ??1?$time_get@DV?$istreambuf_iterator@DU?$char_traits@D@std@@@std@@@std@@MAE@XZ 100bb0da f i libcpmt:xlocale.obj
 0001:000ba0f0       ??1?$time_put@DV?$ostreambuf_iterator@DU?$char_traits@D@std@@@std@@@std@@MAE@XZ 100bb0f0 f i libcpmt:xlocale.obj
 0001:000ba10a       ??4?$basic_string@DU?$char_traits@D@std@@V?$allocator@D@2@@std@@QAEAAV01@$$QAV01@@Z 100bb10a f i libcpmt:xlocale.obj
 0001:000ba12f       ??8?$_String_const_iterator@V?$_String_val@U?$_Simple_types@D@std@@@std@@@std@@QBE_NABV01@@Z 100bb12f f i libcpmt:xlocale.obj
 0001:000ba142       ??9?$_String_const_iterator@V?$_String_val@U?$_Simple_types@D@std@@@std@@@std@@QBE_NABV01@@Z 100bb142 f i libcpmt:xlocale.obj
 0001:000ba155       ??E?$_String_const_iterator@V?$_String_val@U?$_Simple_types@D@std@@@std@@@std@@QAEAAV01@XZ 100bb155 f i libcpmt:xlocale.obj
 0001:000ba15a       ??E?$ostreambuf_iterator@DU?$char_traits@D@std@@@std@@QAEAAV01@H@Z 100bb15a f i libcpmt:xlocale.obj
 0001:000ba15f       ??G?$_String_const_iterator@V?$_String_val@U?$_Simple_types@D@std@@@std@@@std@@QBEHABV01@@Z 100bb15f f i libcpmt:xlocale.obj
 0001:000ba16d       ??G?$_String_iterator@V?$_String_val@U?$_Simple_types@D@std@@@std@@@std@@QBE?AV01@H@Z 100bb16d f i libcpmt:xlocale.obj
 0001:000ba17e       ??G?$_String_iterator@V?$_String_val@U?$_Simple_types@D@std@@@std@@@std@@QBEHABV?$_String_const_iterator@V?$_String_val@U?$_Simple_types@D@std@@@std@@@1@@Z 100bb17e f i libcpmt:xlocale.obj
 0001:000ba18c       ??H?$_String_iterator@V?$_String_val@U?$_Simple_types@D@std@@@std@@@std@@QBE?AV01@H@Z 100bb18c f i libcpmt:xlocale.obj
 0001:000ba19d       ??Y?$_String_const_iterator@V?$_String_val@U?$_Simple_types@D@std@@@std@@@std@@QAEAAV01@H@Z 100bb19d f i libcpmt:xlocale.obj
 0001:000ba1ab       ??Y?$_String_iterator@V?$_String_val@U?$_Simple_types@D@std@@@std@@@std@@QAEAAV01@H@Z 100bb1ab f i libcpmt:xlocale.obj
 0001:000ba1b9       ??Z?$_String_iterator@V?$_String_val@U?$_Simple_types@D@std@@@std@@@std@@QAEAAV01@H@Z 100bb1b9 f i libcpmt:xlocale.obj
 0001:000ba1c7       ??_E?$_Mpunct@D@std@@MAEPAXI@Z 100bb1c7 f i libcpmt:xlocale.obj
 0001:000ba1c7       ??_G?$_Mpunct@D@std@@MAEPAXI@Z 100bb1c7 f i libcpmt:xlocale.obj
 0001:000ba1f2       ??_G?$collate@D@std@@MAEPAXI@Z 100bb1f2 f i libcpmt:xlocale.obj
 0001:000ba1f2       ??_E?$collate@D@std@@MAEPAXI@Z 100bb1f2 f i libcpmt:xlocale.obj
 0001:000ba211       ??_G?$messages@D@std@@MAEPAXI@Z 100bb211 f i libcpmt:xlocale.obj
 0001:000ba211       ??_E?$messages@D@std@@MAEPAXI@Z 100bb211 f i libcpmt:xlocale.obj
 0001:000ba231       ??_E?$money_get@DV?$istreambuf_iterator@DU?$char_traits@D@std@@@std@@@std@@MAEPAXI@Z 100bb231 f i libcpmt:xlocale.obj
 0001:000ba231       ??_G?$money_get@DV?$istreambuf_iterator@DU?$char_traits@D@std@@@std@@@std@@MAEPAXI@Z 100bb231 f i libcpmt:xlocale.obj
 0001:000ba251       ??_G?$money_put@DV?$ostreambuf_iterator@DU?$char_traits@D@std@@@std@@@std@@MAEPAXI@Z 100bb251 f i libcpmt:xlocale.obj
 0001:000ba251       ??_E?$money_put@DV?$ostreambuf_iterator@DU?$char_traits@D@std@@@std@@@std@@MAEPAXI@Z 100bb251 f i libcpmt:xlocale.obj
 0001:000ba271       ??_E?$moneypunct@D$00@std@@MAEPAXI@Z 100bb271 f i libcpmt:xlocale.obj
 0001:000ba271       ??_G?$moneypunct@D$00@std@@MAEPAXI@Z 100bb271 f i libcpmt:xlocale.obj
 0001:000ba29c       ??_G?$moneypunct@D$0A@@std@@MAEPAXI@Z 100bb29c f i libcpmt:xlocale.obj
 0001:000ba29c       ??_E?$moneypunct@D$0A@@std@@MAEPAXI@Z 100bb29c f i libcpmt:xlocale.obj
 0001:000ba2c7       ??_G?$time_get@DV?$istreambuf_iterator@DU?$char_traits@D@std@@@std@@@std@@MAEPAXI@Z 100bb2c7 f i libcpmt:xlocale.obj
 0001:000ba2c7       ??_E?$time_get@DV?$istreambuf_iterator@DU?$char_traits@D@std@@@std@@@std@@MAEPAXI@Z 100bb2c7 f i libcpmt:xlocale.obj
 0001:000ba2f2       ??_G?$time_put@DV?$ostreambuf_iterator@DU?$char_traits@D@std@@@std@@@std@@MAEPAXI@Z 100bb2f2 f i libcpmt:xlocale.obj
 0001:000ba2f2       ??_E?$time_put@DV?$ostreambuf_iterator@DU?$char_traits@D@std@@@std@@@std@@MAEPAXI@Z 100bb2f2 f i libcpmt:xlocale.obj
 0001:000ba311       ?_Compat@?$_String_const_iterator@V?$_String_val@U?$_Simple_types@D@std@@@std@@@std@@QBEXABV12@@Z 100bb311 f i libcpmt:xlocale.obj
 0001:000ba314       ?_Getcat@?$collate@D@std@@SAIPAPBVfacet@locale@2@PBV42@@Z 100bb314 f i libcpmt:xlocale.obj
 0001:000ba3ba       ?_Getcat@?$messages@D@std@@SAIPAPBVfacet@locale@2@PBV42@@Z 100bb3ba f i libcpmt:xlocale.obj
 0001:000ba422       ?_Getcat@?$money_get@DV?$istreambuf_iterator@DU?$char_traits@D@std@@@std@@@std@@SAIPAPBVfacet@locale@2@PBV42@@Z 100bb422 f i libcpmt:xlocale.obj
 0001:000ba48a       ?_Getcat@?$money_put@DV?$ostreambuf_iterator@DU?$char_traits@D@std@@@std@@@std@@SAIPAPBVfacet@locale@2@PBV42@@Z 100bb48a f i libcpmt:xlocale.obj
 0001:000ba4f2       ?_Getcat@?$moneypunct@D$00@std@@SAIPAPBVfacet@locale@2@PBV42@@Z 100bb4f2 f i libcpmt:xlocale.obj
 0001:000ba576       ?_Getcat@?$moneypunct@D$0A@@std@@SAIPAPBVfacet@locale@2@PBV42@@Z 100bb576 f i libcpmt:xlocale.obj
 0001:000ba5fb       ?_Getcat@?$time_get@DV?$istreambuf_iterator@DU?$char_traits@D@std@@@std@@@std@@SAIPAPBVfacet@locale@2@PBV42@@Z 100bb5fb f i libcpmt:xlocale.obj
 0001:000ba667       ?_Getcat@?$time_put@DV?$ostreambuf_iterator@DU?$char_traits@D@std@@@std@@@std@@SAIPAPBVfacet@locale@2@PBV42@@Z 100bb667 f i libcpmt:xlocale.obj
 0001:000ba6db       ?_Getfmt@?$time_get@DV?$istreambuf_iterator@DU?$char_traits@D@std@@@std@@@std@@IBE?AV?$istreambuf_iterator@DU?$char_traits@D@std@@@2@V32@0AAVios_base@2@AAHPAUtm@@PBD@Z 100bb6db f i libcpmt:xlocale.obj
 0001:000ba7e6       ?_Getint@?$time_get@DV?$istreambuf_iterator@DU?$char_traits@D@std@@@std@@@std@@ABAHAAV?$istreambuf_iterator@DU?$char_traits@D@std@@@2@0HHAAHABV?$ctype@D@2@@Z 100bb7e6 f i libcpmt:xlocale.obj
 0001:000ba970       ?_Getmfld@?$money_get@DV?$istreambuf_iterator@DU?$char_traits@D@std@@@std@@@std@@ABE?AV?$basic_string@DU?$char_traits@D@std@@V?$allocator@D@2@@2@AAV?$istreambuf_iterator@DU?$char_traits@D@std@@@2@0_NAAVios_base@2@PAD@Z 100bb970 f i libcpmt:xlocale.obj
 0001:000bb3c0       ?_Gettnames@_Locinfo@std@@QBE?AV_Timevec@2@XZ 100bc3c0 f i libcpmt:xlocale.obj
 0001:000bb3da       ?_Init@?$_Mpunct@D@std@@IAEXABV_Locinfo@2@_N@Z 100bc3da f i libcpmt:xlocale.obj
 0001:000bb4c3       ?_Init@?$collate@D@std@@IAEXABV_Locinfo@2@@Z 100bc4c3 f i libcpmt:xlocale.obj
 0001:000bb4d5       ?_Init@?$messages@D@std@@IAEXABV_Locinfo@2@@Z 100bc4d5 f i libcpmt:xlocale.obj
 0001:000bb4d8       ?_Init@?$money_get@DV?$istreambuf_iterator@DU?$char_traits@D@std@@@std@@@std@@IAEXABV_Locinfo@2@@Z 100bc4d8 f i libcpmt:xlocale.obj
 0001:000bb4db       ?_Init@?$money_put@DV?$ostreambuf_iterator@DU?$char_traits@D@std@@@std@@@std@@IAEXABV_Locinfo@2@@Z 100bc4db f i libcpmt:xlocale.obj
 0001:000bb4de       ?_Init@?$time_get@DV?$istreambuf_iterator@DU?$char_traits@D@std@@@std@@@std@@IAEXABV_Locinfo@2@@Z 100bc4de f i libcpmt:xlocale.obj
 0001:000bb528       ?_Init@?$time_put@DV?$ostreambuf_iterator@DU?$char_traits@D@std@@@std@@@std@@IAEXABV_Locinfo@2@@Z 100bc528 f i libcpmt:xlocale.obj
 0001:000bb553       ?_Makexloc@_Locimp@locale@std@@CAXABV_Locinfo@3@HPAV123@PBV23@@Z 100bc553 f   libcpmt:xlocale.obj
 0001:000bb8d7       ?_Makpat@?$_Mpunct@D@std@@AAEXAAUpattern@money_base@2@III@Z 100bc8d7 f i libcpmt:xlocale.obj
 0001:000bb921       ?_Pdif@?$basic_string@DU?$char_traits@D@std@@V?$allocator@D@2@@std@@SAIV?$_String_const_iterator@V?$_String_val@U?$_Simple_types@D@std@@@std@@@2@0@Z 100bc921 f i libcpmt:xlocale.obj
 0001:000bb932       ?_Put@?$money_put@DV?$ostreambuf_iterator@DU?$char_traits@D@std@@@std@@@std@@CA?AV?$ostreambuf_iterator@DU?$char_traits@D@std@@@2@V32@V?$_String_const_iterator@V?$_String_val@U?$_Simple_types@D@std@@@std@@@2@I@Z 100bc932 f i libcpmt:xlocale.obj
 0001:000bb967       ?_Putmfld@?$money_put@DV?$ostreambuf_iterator@DU?$char_traits@D@std@@@std@@@std@@ABE?AV?$ostreambuf_iterator@DU?$char_traits@D@std@@@2@V32@_NAAVios_base@2@D1V?$basic_string@DU?$char_traits@D@std@@V?$allocator@D@2@@2@D@Z 100bc967 f i libcpmt:xlocale.obj
 0001:000bbeb5       ?_Rep@?$money_put@DV?$ostreambuf_iterator@DU?$char_traits@D@std@@@std@@@std@@CA?AV?$ostreambuf_iterator@DU?$char_traits@D@std@@@2@V32@DI@Z 100bceb5 f i libcpmt:xlocale.obj
 0001:000bbedf       ?_Tidy@?$_Mpunct@D@std@@AAEXXZ 100bcedf f i libcpmt:xlocale.obj
 0001:000bbf07       ?_Tidy@?$time_get@DV?$istreambuf_iterator@DU?$char_traits@D@std@@@std@@@std@@AAEXXZ 100bcf07 f i libcpmt:xlocale.obj
 0001:000bbf27       ?curr_symbol@?$_Mpunct@D@std@@QBE?AV?$basic_string@DU?$char_traits@D@std@@V?$allocator@D@2@@2@XZ 100bcf27 f i libcpmt:xlocale.obj
 0001:000bbf40       ?date_order@?$time_get@DV?$istreambuf_iterator@DU?$char_traits@D@std@@@std@@@std@@QBE?AW4dateorder@time_base@2@XZ 100bcf40 f i libcpmt:xlocale.obj
 0001:000bbf45       ?decimal_point@?$_Mpunct@D@std@@QBEDXZ 100bcf45 f i libcpmt:xlocale.obj
 0001:000bbf4a       ?do_close@?$messages@D@std@@MBEXH@Z 100bcf4a f i libcpmt:xlocale.obj
 0001:000bbf4d       ?do_compare@?$collate@D@std@@MBEHPBD000@Z 100bcf4d f i libcpmt:xlocale.obj
 0001:000bbf7e       ?do_curr_symbol@?$_Mpunct@D@std@@MBE?AV?$basic_string@DU?$char_traits@D@std@@V?$allocator@D@2@@2@XZ 100bcf7e f i libcpmt:xlocale.obj
 0001:000bbf9a       ?do_date_order@?$time_get@DV?$istreambuf_iterator@DU?$char_traits@D@std@@@std@@@std@@MBE?AW4dateorder@time_base@2@XZ 100bcf9a f i libcpmt:xlocale.obj
 0001:000bbf9e       ?do_decimal_point@?$_Mpunct@D@std@@MBEDXZ 100bcf9e f i libcpmt:xlocale.obj
 0001:000bbfa2       ?do_frac_digits@?$_Mpunct@D@std@@MBEHXZ 100bcfa2 f i libcpmt:xlocale.obj
 0001:000bbfa6       ?do_get@?$messages@D@std@@MBE?AV?$basic_string@DU?$char_traits@D@std@@V?$allocator@D@2@@2@HHHABV32@@Z 100bcfa6 f i libcpmt:xlocale.obj
 0001:000bbfc2       ?do_get@?$money_get@DV?$istreambuf_iterator@DU?$char_traits@D@std@@@std@@@std@@MBE?AV?$istreambuf_iterator@DU?$char_traits@D@std@@@2@V32@0_NAAVios_base@2@AAHAAO@Z 100bcfc2 f i libcpmt:xlocale.obj
 0001:000bc06e       ?do_get@?$money_get@DV?$istreambuf_iterator@DU?$char_traits@D@std@@@std@@@std@@MBE?AV?$istreambuf_iterator@DU?$char_traits@D@std@@@2@V32@0_NAAVios_base@2@AAHAAV?$basic_string@DU?$char_traits@D@std@@V?$allocator@D@2@@2@@Z 100bd06e f i libcpmt:xlocale.obj
 0001:000bc142       ?do_get@?$time_get@DV?$istreambuf_iterator@DU?$char_traits@D@std@@@std@@@std@@MBE?AV?$istreambuf_iterator@DU?$char_traits@D@std@@@2@V32@0AAVios_base@2@AAHPAUtm@@DD@Z 100bd142 f i libcpmt:xlocale.obj
 0001:000bc4ab       ?do_get_date@?$time_get@DV?$istreambuf_iterator@DU?$char_traits@D@std@@@std@@@std@@MBE?AV?$istreambuf_iterator@DU?$char_traits@D@std@@@2@V32@0AAVios_base@2@AAHPAUtm@@@Z 100bd4ab f i libcpmt:xlocale.obj
 0001:000bc912       ?do_get_monthname@?$time_get@DV?$istreambuf_iterator@DU?$char_traits@D@std@@@std@@@std@@MBE?AV?$istreambuf_iterator@DU?$char_traits@D@std@@@2@V32@0AAVios_base@2@AAHPAUtm@@@Z 100bd912 f i libcpmt:xlocale.obj
 0001:000bc952       ?do_get_time@?$time_get@DV?$istreambuf_iterator@DU?$char_traits@D@std@@@std@@@std@@MBE?AV?$istreambuf_iterator@DU?$char_traits@D@std@@@2@V32@0AAVios_base@2@AAHPAUtm@@@Z 100bd952 f i libcpmt:xlocale.obj
 0001:000bca54       ?do_get_weekday@?$time_get@DV?$istreambuf_iterator@DU?$char_traits@D@std@@@std@@@std@@MBE?AV?$istreambuf_iterator@DU?$char_traits@D@std@@@2@V32@0AAVios_base@2@AAHPAUtm@@@Z 100bda54 f i libcpmt:xlocale.obj
 0001:000bca94       ?do_get_year@?$time_get@DV?$istreambuf_iterator@DU?$char_traits@D@std@@@std@@@std@@MBE?AV?$istreambuf_iterator@DU?$char_traits@D@std@@@2@V32@0AAVios_base@2@AAHPAUtm@@@Z 100bda94 f i libcpmt:xlocale.obj
 0001:000bcb2c       ?do_grouping@?$_Mpunct@D@std@@MBE?AV?$basic_string@DU?$char_traits@D@std@@V?$allocator@D@2@@2@XZ 100bdb2c f i libcpmt:xlocale.obj
 0001:000bcb48       ?do_hash@?$collate@D@std@@MBEJPBD0@Z 100bdb48 f i libcpmt:xlocale.obj
 0001:000bcb60       ?do_neg_format@?$_Mpunct@D@std@@MBE?AUpattern@money_base@2@XZ 100bdb60 f i libcpmt:xlocale.obj
 0001:000bcb6f       ?do_negative_sign@?$_Mpunct@D@std@@MBE?AV?$basic_string@DU?$char_traits@D@std@@V?$allocator@D@2@@2@XZ 100bdb6f f i libcpmt:xlocale.obj
 0001:000bcb8b       ?do_open@?$messages@D@std@@MBEHABV?$basic_string@DU?$char_traits@D@std@@V?$allocator@D@2@@2@ABVlocale@2@@Z 100bdb8b f i libcpmt:xlocale.obj
 0001:000bcb91       ?do_pos_format@?$_Mpunct@D@std@@MBE?AUpattern@money_base@2@XZ 100bdb91 f i libcpmt:xlocale.obj
 0001:000bcba0       ?do_positive_sign@?$_Mpunct@D@std@@MBE?AV?$basic_string@DU?$char_traits@D@std@@V?$allocator@D@2@@2@XZ 100bdba0 f i libcpmt:xlocale.obj
 0001:000bcbbc       ?do_put@?$money_put@DV?$ostreambuf_iterator@DU?$char_traits@D@std@@@std@@@std@@MBE?AV?$ostreambuf_iterator@DU?$char_traits@D@std@@@2@V32@_NAAVios_base@2@DABV?$basic_string@DU?$char_traits@D@std@@V?$allocator@D@2@@2@@Z 100bdbbc f i libcpmt:xlocale.obj
 0001:000bcce8       ?do_put@?$money_put@DV?$ostreambuf_iterator@DU?$char_traits@D@std@@@std@@@std@@MBE?AV?$ostreambuf_iterator@DU?$char_traits@D@std@@@2@V32@_NAAVios_base@2@DO@Z 100bdce8 f i libcpmt:xlocale.obj
 0001:000bce45       ?do_put@?$time_put@DV?$ostreambuf_iterator@DU?$char_traits@D@std@@@std@@@std@@MBE?AV?$ostreambuf_iterator@DU?$char_traits@D@std@@@2@V32@AAVios_base@2@DPBUtm@@DD@Z 100bde45 f i libcpmt:xlocale.obj
 0001:000bcf12       ?do_thousands_sep@?$_Mpunct@D@std@@MBEDXZ 100bdf12 f i libcpmt:xlocale.obj
 0001:000bcf16       ?do_transform@?$collate@D@std@@MBE?AV?$basic_string@DU?$char_traits@D@std@@V?$allocator@D@2@@2@PBD0@Z 100bdf16 f i libcpmt:xlocale.obj
 0001:000bcf9e       ?end@?$basic_string@DU?$char_traits@D@std@@V?$allocator@D@2@@std@@QAE?AV?$_String_iterator@V?$_String_val@U?$_Simple_types@D@std@@@std@@@2@XZ 100bdf9e f i libcpmt:xlocale.obj
 0001:000bcfbb       ?frac_digits@?$_Mpunct@D@std@@QBEHXZ 100bdfbb f i libcpmt:xlocale.obj
 0001:000bcfc0       ?get_monthname@?$time_get@DV?$istreambuf_iterator@DU?$char_traits@D@std@@@std@@@std@@QBE?AV?$istreambuf_iterator@DU?$char_traits@D@std@@@2@V32@0AAVios_base@2@AAHPAUtm@@@Z 100bdfc0 f i libcpmt:xlocale.obj
 0001:000bcfe7       ?get_weekday@?$time_get@DV?$istreambuf_iterator@DU?$char_traits@D@std@@@std@@@std@@QBE?AV?$istreambuf_iterator@DU?$char_traits@D@std@@@2@V32@0AAVios_base@2@AAHPAUtm@@@Z 100bdfe7 f i libcpmt:xlocale.obj
 0001:000bd00e       ?get_year@?$time_get@DV?$istreambuf_iterator@DU?$char_traits@D@std@@@std@@@std@@QBE?AV?$istreambuf_iterator@DU?$char_traits@D@std@@@2@V32@0AAVios_base@2@AAHPAUtm@@@Z 100be00e f i libcpmt:xlocale.obj
 0001:000bd035       ?grouping@?$_Mpunct@D@std@@QBE?AV?$basic_string@DU?$char_traits@D@std@@V?$allocator@D@2@@2@XZ 100be035 f i libcpmt:xlocale.obj
 0001:000bd04e       ?is@?$ctype@D@std@@QBE_NFD@Z 100be04e f i libcpmt:xlocale.obj
 0001:000bd06c       ?narrow@?$ctype@D@std@@QBEDDD@Z 100be06c f i libcpmt:xlocale.obj
 0001:000bd075       ?neg_format@?$_Mpunct@D@std@@QBE?AUpattern@money_base@2@XZ 100be075 f i libcpmt:xlocale.obj
 0001:000bd087       ?negative_sign@?$_Mpunct@D@std@@QBE?AV?$basic_string@DU?$char_traits@D@std@@V?$allocator@D@2@@2@XZ 100be087 f i libcpmt:xlocale.obj
 0001:000bd0a0       ?pos_format@?$_Mpunct@D@std@@QBE?AUpattern@money_base@2@XZ 100be0a0 f i libcpmt:xlocale.obj
 0001:000bd0b2       ?positive_sign@?$_Mpunct@D@std@@QBE?AV?$basic_string@DU?$char_traits@D@std@@V?$allocator@D@2@@2@XZ 100be0b2 f i libcpmt:xlocale.obj
 0001:000bd0cb       ?replace@?$basic_string@DU?$char_traits@D@std@@V?$allocator@D@2@@std@@QAEAAV12@IIABV12@II@Z 100be0cb f i libcpmt:xlocale.obj
 0001:000bd3e8       ?replace@?$basic_string@DU?$char_traits@D@std@@V?$allocator@D@2@@std@@QAEAAV12@IIPBDI@Z 100be3e8 f i libcpmt:xlocale.obj
 0001:000bd541       ?replace@?$basic_string@DU?$char_traits@D@std@@V?$allocator@D@2@@std@@QAEAAV12@V?$_String_const_iterator@V?$_String_val@U?$_Simple_types@D@std@@@std@@@2@0V?$_String_iterator@V?$_String_val@U?$_Simple_types@D@std@@@std@@@2@1@Z 100be541 f i libcpmt:xlocale.obj
 0001:000bd5c1       ?resize@?$basic_string@DU?$char_traits@D@std@@V?$allocator@D@2@@std@@QAEXI@Z 100be5c1 f i libcpmt:xlocale.obj
 0001:000bd5d2       ?resize@?$basic_string@DU?$char_traits@D@std@@V?$allocator@D@2@@std@@QAEXID@Z 100be5d2 f i libcpmt:xlocale.obj
 0001:000bd5fe       ?thousands_sep@?$_Mpunct@D@std@@QBEDXZ 100be5fe f i libcpmt:xlocale.obj
 0001:000bd603       __Stof                     100be603 f   libcpmt:xstof.obj
 0001:000bd61b       __Stofx                    100be61b f   libcpmt:xstof.obj
 0001:000bd82d       __Stod                     100be82d f   libcpmt:xstod.obj
 0001:000bd845       __Stodx                    100be845 f   libcpmt:xstod.obj
 0001:000bdaae       __Stold                    100beaae f   libcpmt:xstold.obj
 0001:000bdac6       __Stoldx                   100beac6 f   libcpmt:xstold.obj
 0001:000bdd2f       __Stolx                    100bed2f f   libcpmt:xstol.obj
 0001:000bddcf       __Stoul                    100bedcf f   libcpmt:xstoul.obj
 0001:000bdde7       __Stoulx                   100bede7 f   libcpmt:xstoul.obj
 0001:000bdf63       __Stoll                    100bef63 f   libcpmt:xstoll.obj
 0001:000bdf7b       __Stollx                   100bef7b f   libcpmt:xstoll.obj
 0001:000be043       __Stoull                   100bf043 f   libcpmt:xstoull.obj
 0001:000be05b       __Stoullx                  100bf05b f   libcpmt:xstoull.obj
 0001:000be246       __Getcoll                  100bf246 f   libcpmt:xstrcoll.obj
 0001:000be267       __Strcoll                  100bf267 f   libcpmt:xstrcoll.obj
 0001:000be2fc       __Getdateorder             100bf2fc f   libcpmt:xdateord.obj
 0001:000be346       __Mbrtowc                  100bf346 f   libcpmt:xmbtowc.obj
 0001:000be49d       __Wcscoll                  100bf49d f   libcpmt:xwcscoll.obj
 0001:000be577       __Wcsxfrm                  100bf577 f   libcpmt:xwcsxfrm.obj
 0001:000be639       __Getwctype                100bf639 f   libcpmt:xgetwctype.obj
 0001:000be65d       __Getwctypes               100bf65d f   libcpmt:xgetwctype.obj
 0001:000be67c       __Towlower                 100bf67c f   libcpmt:xtowlower.obj
 0001:000be6e8       __Towupper                 100bf6e8 f   libcpmt:xtowupper.obj
 0001:000be758       __Strxfrm                  100bf758 f   libcpmt:xstrxfrm.obj
 0001:000be7fe       __Stopfx                   100bf7fe f   libcpmt:xstopfx.obj
 0001:000be938       __Stoflt                   100bf938 f   libcpmt:xstoflt.obj
 0001:000beb8b       __Stoxflt                  100bfb8b f   libcpmt:xstoxflt.obj
 0001:000bee15       __FDtest                   100bfe15 f   libcpmt:xfdtest.obj
 0001:000bee61       __FPlsw                    100bfe61 f   libcpmt:xfdtest.obj
 0001:000bee69       __FPmsw                    100bfe69 f   libcpmt:xfdtest.obj
 0001:000bee74       __FDscale                  100bfe74 f   libcpmt:xfdscale.obj
 0001:000bf00e       __FXp_addh                 100c000e f   libcpmt:xfprec.obj
 0001:000bf32f       __FXp_addx                 100c032f f   libcpmt:xfprec.obj
 0001:000bf372       __FXp_getw                 100c0372 f   libcpmt:xfprec.obj
 0001:000bf434       __FXp_invx                 100c0434 f   libcpmt:xfprec.obj
 0001:000bf531       __FXp_ldexpx               100c0531 f   libcpmt:xfprec.obj
 0001:000bf573       __FXp_movx                 100c0573 f   libcpmt:xfprec.obj
 0001:000bf590       __FXp_mulh                 100c0590 f   libcpmt:xfprec.obj
 0001:000bf71a       __FXp_mulx                 100c071a f   libcpmt:xfprec.obj
 0001:000bf7ee       __FXp_setn                 100c07ee f   libcpmt:xfprec.obj
 0001:000bf855       __FXp_setw                 100c0855 f   libcpmt:xfprec.obj
 0001:000bf8d9       __FXp_sqrtx                100c08d9 f   libcpmt:xfprec.obj
 0001:000bf9ff       __FXp_subx                 100c09ff f   libcpmt:xfprec.obj
 0001:000bfa44       __FDtento                  100c0a44 f   libcpmt:xfdtento.obj
 0001:000bfb6b       __Dtest                    100c0b6b f   libcpmt:xdtest.obj
 0001:000bfbcd       __Plsw                     100c0bcd f   libcpmt:xdtest.obj
 0001:000bfbd5       __Pmsw                     100c0bd5 f   libcpmt:xdtest.obj
 0001:000bfbe0       __Dscale                   100c0be0 f   libcpmt:xdscale.obj
 0001:000bfe47       __Xp_addh                  100c0e47 f   libcpmt:xprec.obj
 0001:000c014d       __Xp_addx                  100c114d f   libcpmt:xprec.obj
 0001:000c0191       __Xp_getw                  100c1191 f   libcpmt:xprec.obj
 0001:000c0242       __Xp_invx                  100c1242 f   libcpmt:xprec.obj
 0001:000c0338       __Xp_ldexpx                100c1338 f   libcpmt:xprec.obj
 0001:000c0374       __Xp_movx                  100c1374 f   libcpmt:xprec.obj
 0001:000c0391       __Xp_mulh                  100c1391 f   libcpmt:xprec.obj
 0001:000c050f       __Xp_mulx                  100c150f f   libcpmt:xprec.obj
 0001:000c05e2       __Xp_setn                  100c15e2 f   libcpmt:xprec.obj
 0001:000c060a       __Xp_setw                  100c160a f   libcpmt:xprec.obj
 0001:000c06f8       __Xp_sqrtx                 100c16f8 f   libcpmt:xprec.obj
 0001:000c0808       __Xp_subx                  100c1808 f   libcpmt:xprec.obj
 0001:000c084e       __Dtento                   100c184e f   libcpmt:xdtento.obj
 0001:000c0970       __LDtest                   100c1970 f   libcpmt:xldtest.obj
 0001:000c0979       __LPlsw                    100c1979 f   libcpmt:xldtest.obj
 0001:000c0981       __LPmsw                    100c1981 f   libcpmt:xldtest.obj
 0001:000c098c       __LDscale                  100c198c f   libcpmt:xldscale.obj
 0001:000c0995       __LXp_addh                 100c1995 f   libcpmt:xlprec.obj
 0001:000c0c9b       __LXp_addx                 100c1c9b f   libcpmt:xlprec.obj
 0001:000c0cdf       __LXp_getw                 100c1cdf f   libcpmt:xlprec.obj
 0001:000c0d90       __LXp_invx                 100c1d90 f   libcpmt:xlprec.obj
 0001:000c0e86       __LXp_ldexpx               100c1e86 f   libcpmt:xlprec.obj
 0001:000c0ec2       __LXp_movx                 100c1ec2 f   libcpmt:xlprec.obj
 0001:000c0edf       __LXp_mulh                 100c1edf f   libcpmt:xlprec.obj
 0001:000c105d       __LXp_mulx                 100c205d f   libcpmt:xlprec.obj
 0001:000c1130       __LXp_setn                 100c2130 f   libcpmt:xlprec.obj
 0001:000c1158       __LXp_setw                 100c2158 f   libcpmt:xlprec.obj
 0001:000c1246       __LXp_sqrtx                100c2246 f   libcpmt:xlprec.obj
 0001:000c1356       __LXp_subx                 100c2356 f   libcpmt:xlprec.obj
 0001:000c139c       _sqrtl                     100c239c f i libcpmt:xlprec.obj
 0001:000c13b0       __LDtento                  100c23b0 f   libcpmt:xldtento.obj
 0001:000c14d2       __FDnorm                   100c24d2 f   libcpmt:xfdnorm.obj
 0001:000c159c       __Feraise                  100c259c f   libcpmt:xferaise.obj
 0001:000c15c5       __FDint                    100c25c5 f   libcpmt:xfdint.obj
 0001:000c168f       __FDunscale                100c268f f   libcpmt:xfdunsca.obj
 0001:000c1714       __Dnorm                    100c2714 f   libcpmt:xdnorm.obj
 0001:000c1885       __Dint                     100c2885 f   libcpmt:xdint.obj
 0001:000c1981       __Dunscale                 100c2981 f   libcpmt:xdunscal.obj
 0001:000c1a15       __LDint                    100c2a15 f   libcpmt:xldint.obj
 0001:000c1a1e       __LDunscale                100c2a1e f   libcpmt:xldunsca.obj
 0001:000c1a28       _GetModuleHandleA@4        100c2a28 f   kernel32:KERNEL32.dll
 0001:000c1a2e       _GetProcAddress@8          100c2a2e f   kernel32:KERNEL32.dll
 0001:000c1a34       _WaitForSingleObject@8     100c2a34 f   kernel32:KERNEL32.dll
 0001:000c1a3a       _HeapAlloc@12              100c2a3a f   kernel32:KERNEL32.dll
 0001:000c1a40       _GetLastError@0            100c2a40 f   kernel32:KERNEL32.dll
 0001:000c1a46       _HeapFree@12               100c2a46 f   kernel32:KERNEL32.dll
 0001:000c1a4c       _IsDebuggerPresent@0       100c2a4c f   kernel32:KERNEL32.dll
 0001:000c1a52       _IsProcessorFeaturePresent@4 100c2a52 f   kernel32:KERNEL32.dll
 0001:000c1a58       _EncodePointer@4           100c2a58 f   kernel32:KERNEL32.dll
 0001:000c1a5e       _DecodePointer@4           100c2a5e f   kernel32:KERNEL32.dll
 0001:000c1a64       _ExitProcess@4             100c2a64 f   kernel32:KERNEL32.dll
 0001:000c1a6a       _GetModuleHandleExW@12     100c2a6a f   kernel32:KERNEL32.dll
 0001:000c1a70       _AreFileApisANSI@0         100c2a70 f   kernel32:KERNEL32.dll
 0001:000c1a76       _MultiByteToWideChar@24    100c2a76 f   kernel32:KERNEL32.dll
 0001:000c1a7c       _WideCharToMultiByte@32    100c2a7c f   kernel32:KERNEL32.dll
 0001:000c1a82       _HeapReAlloc@16            100c2a82 f   kernel32:KERNEL32.dll
 0001:000c1a88       _EnterCriticalSection@4    100c2a88 f   kernel32:KERNEL32.dll
 0001:000c1a8e       _LeaveCriticalSection@4    100c2a8e f   kernel32:KERNEL32.dll
 0001:000c1a94       _GetStdHandle@4            100c2a94 f   kernel32:KERNEL32.dll
 0001:000c1a9a       _GetFileType@4             100c2a9a f   kernel32:KERNEL32.dll
 0001:000c1aa0       _GetModuleFileNameW@12     100c2aa0 f   kernel32:KERNEL32.dll
 0001:000c1aa6       _WriteConsoleW@20          100c2aa6 f   kernel32:KERNEL32.dll
 0001:000c1aac       _GetCommandLineA@0         100c2aac f   kernel32:KERNEL32.dll
 0001:000c1ab2       _GetCurrentThreadId@0      100c2ab2 f   kernel32:KERNEL32.dll
 0001:000c1ab8       _RaiseException@16         100c2ab8 f   kernel32:KERNEL32.dll
 0001:000c1abe       _RtlUnwind@16              100c2abe f   kernel32:KERNEL32.dll
 0001:000c1ac4       _WriteFile@20              100c2ac4 f   kernel32:KERNEL32.dll
 0001:000c1aca       _GetProcessHeap@0          100c2aca f   kernel32:KERNEL32.dll
 0001:000c1ad0       _UnhandledExceptionFilter@4 100c2ad0 f   kernel32:KERNEL32.dll
 0001:000c1ad6       _SetUnhandledExceptionFilter@4 100c2ad6 f   kernel32:KERNEL32.dll
 0001:000c1adc       _SetLastError@4            100c2adc f   kernel32:KERNEL32.dll
 0001:000c1ae2       _InitializeCriticalSectionAndSpinCount@8 100c2ae2 f   kernel32:KERNEL32.dll
 0001:000c1ae8       _CreateEventW@16           100c2ae8 f   kernel32:KERNEL32.dll
 0001:000c1aee       _Sleep@4                   100c2aee f   kernel32:KERNEL32.dll
 0001:000c1af4       _GetCurrentProcess@0       100c2af4 f   kernel32:KERNEL32.dll
 0001:000c1afa       _TerminateProcess@8        100c2afa f   kernel32:KERNEL32.dll
 0001:000c1b00       _TlsAlloc@0                100c2b00 f   kernel32:KERNEL32.dll
 0001:000c1b06       _TlsGetValue@4             100c2b06 f   kernel32:KERNEL32.dll
 0001:000c1b0c       _TlsSetValue@8             100c2b0c f   kernel32:KERNEL32.dll
 0001:000c1b12       _TlsFree@4                 100c2b12 f   kernel32:KERNEL32.dll
 0001:000c1b18       _GetStartupInfoW@4         100c2b18 f   kernel32:KERNEL32.dll
 0001:000c1b1e       _GetTickCount@0            100c2b1e f   kernel32:KERNEL32.dll
 0001:000c1b24       _GetModuleHandleW@4        100c2b24 f   kernel32:KERNEL32.dll
 0001:000c1b2a       _CreateSemaphoreW@16       100c2b2a f   kernel32:KERNEL32.dll
 0001:000c1b30       _DeleteCriticalSection@4   100c2b30 f   kernel32:KERNEL32.dll
 0001:000c1b36       _FatalAppExitA@8           100c2b36 f   kernel32:KERNEL32.dll
 0001:000c1b3c       _SetConsoleCtrlHandler@8   100c2b3c f   kernel32:KERNEL32.dll
 0001:000c1b42       _FreeLibrary@4             100c2b42 f   kernel32:KERNEL32.dll
 0001:000c1b48       _LoadLibraryExW@12         100c2b48 f   kernel32:KERNEL32.dll
 0001:000c1b4e       _IsValidCodePage@4         100c2b4e f   kernel32:KERNEL32.dll
 0001:000c1b54       _GetACP@0                  100c2b54 f   kernel32:KERNEL32.dll
 0001:000c1b5a       _GetOEMCP@0                100c2b5a f   kernel32:KERNEL32.dll
 0001:000c1b60       _GetCPInfo@8               100c2b60 f   kernel32:KERNEL32.dll
 0001:000c1b66       _CloseHandle@4             100c2b66 f   kernel32:KERNEL32.dll
 0001:000c1b6c       _ReadFile@20               100c2b6c f   kernel32:KERNEL32.dll
 0001:000c1b72       _GetConsoleMode@8          100c2b72 f   kernel32:KERNEL32.dll
 0001:000c1b78       _ReadConsoleW@20           100c2b78 f   kernel32:KERNEL32.dll
 0001:000c1b7e       _GetConsoleCP@0            100c2b7e f   kernel32:KERNEL32.dll
 0001:000c1b84       _DeleteFileW@4             100c2b84 f   kernel32:KERNEL32.dll
 0001:000c1b8a       _SetFilePointerEx@20       100c2b8a f   kernel32:KERNEL32.dll
 0001:000c1b90       _OutputDebugStringW@4      100c2b90 f   kernel32:KERNEL32.dll
 0001:000c1b96       _GetCurrentThread@0        100c2b96 f   kernel32:KERNEL32.dll
 0001:000c1b9c       _GetModuleFileNameA@12     100c2b9c f   kernel32:KERNEL32.dll
 0001:000c1ba2       _QueryPerformanceCounter@4 100c2ba2 f   kernel32:KERNEL32.dll
 0001:000c1ba8       _GetCurrentProcessId@0     100c2ba8 f   kernel32:KERNEL32.dll
 0001:000c1bae       _GetSystemTimeAsFileTime@4 100c2bae f   kernel32:KERNEL32.dll
 0001:000c1bb4       _GetEnvironmentStringsW@0  100c2bb4 f   kernel32:KERNEL32.dll
 0001:000c1bba       _FreeEnvironmentStringsW@4 100c2bba f   kernel32:KERNEL32.dll
 0001:000c1bc0       _HeapSize@12               100c2bc0 f   kernel32:KERNEL32.dll
 0001:000c1bc6       _FlushFileBuffers@4        100c2bc6 f   kernel32:KERNEL32.dll
 0001:000c1bcc       _GetDateFormatW@24         100c2bcc f   kernel32:KERNEL32.dll
 0001:000c1bd2       _GetTimeFormatW@24         100c2bd2 f   kernel32:KERNEL32.dll
 0001:000c1bd8       _CompareStringW@24         100c2bd8 f   kernel32:KERNEL32.dll
 0001:000c1bde       _LCMapStringW@24           100c2bde f   kernel32:KERNEL32.dll
 0001:000c1be4       _GetLocaleInfoW@16         100c2be4 f   kernel32:KERNEL32.dll
 0001:000c1bea       _IsValidLocale@8           100c2bea f   kernel32:KERNEL32.dll
 0001:000c1bf0       _GetUserDefaultLCID@0      100c2bf0 f   kernel32:KERNEL32.dll
 0001:000c1bf6       _EnumSystemLocalesW@8      100c2bf6 f   kernel32:KERNEL32.dll
 0001:000c1bfc       _GetStringTypeW@16         100c2bfc f   kernel32:KERNEL32.dll
 0001:000c1c02       _SetStdHandle@8            100c2c02 f   kernel32:KERNEL32.dll
 0001:000c1c08       _CreateFileW@28            100c2c08 f   kernel32:KERNEL32.dll
 0001:000c1c0e       _SetEndOfFile@4            100c2c0e f   kernel32:KERNEL32.dll
 0001:000c1c20       ??$?6DU?$char_traits@D@std@@V?$allocator@D@1@@std@@YAAAV?$basic_ostream@DU?$char_traits@D@std@@@0@AAV10@ABV?$basic_string@DU?$char_traits@D@std@@V?$allocator@D@2@@0@@Z 100c2c20 f i libsg_MSVC120_vc:sg_common.obj
 0001:000c1f30       ??$_Uninit_move@PAV?$basic_string@DU?$char_traits@D@std@@V?$allocator@D@2@@std@@PAV12@V?$allocator@V?$basic_string@DU?$char_traits@D@std@@V?$allocator@D@2@@std@@@2@V12@@std@@YAPAV?$basic_string@DU?$char_traits@D@std@@V?$allocator@D@2@@0@PAV10@00AAU?$_Wrap_alloc@V?$allocator@V?$basic_string@DU?$char_traits@D@std@@V?$allocator@D@2@@std@@@std@@@0@0U_Nonscalar_ptr_iterator_tag@0@@Z 100c2f30 f i libsg_MSVC120_vc:sg_common.obj
 0001:000c1fc0       ??$endl@DU?$char_traits@D@std@@@std@@YAAAV?$basic_ostream@DU?$char_traits@D@std@@@0@AAV10@@Z 100c2fc0 f i libsg_MSVC120_vc:sg_common.obj
 0001:000c2060       ??1?$vector@V?$basic_string@DU?$char_traits@D@std@@V?$allocator@D@2@@std@@V?$allocator@V?$basic_string@DU?$char_traits@D@std@@V?$allocator@D@2@@std@@@2@@std@@QAE@XZ 100c3060 f i libsg_MSVC120_vc:sg_common.obj
 0001:000c20a0       ??6?$basic_ostream@DU?$char_traits@D@std@@@std@@QAEAAV01@I@Z 100c30a0 f i libsg_MSVC120_vc:sg_common.obj
 0001:000c22e0       ?_Destroy@?$vector@V?$basic_string@DU?$char_traits@D@std@@V?$allocator@D@2@@std@@V?$allocator@V?$basic_string@DU?$char_traits@D@std@@V?$allocator@D@2@@std@@@2@@std@@IAEXPAV?$basic_string@DU?$char_traits@D@std@@V?$allocator@D@2@@2@0@Z 100c32e0 f i libsg_MSVC120_vc:sg_common.obj
 0001:000c2320       ?_Reallocate@?$vector@V?$basic_string@DU?$char_traits@D@std@@V?$allocator@D@2@@std@@V?$allocator@V?$basic_string@DU?$char_traits@D@std@@V?$allocator@D@2@@std@@@2@@std@@IAEXI@Z 100c3320 f i libsg_MSVC120_vc:sg_common.obj
 0001:000c2410       ?_Reserve@?$vector@V?$basic_string@DU?$char_traits@D@std@@V?$allocator@D@2@@std@@V?$allocator@V?$basic_string@DU?$char_traits@D@std@@V?$allocator@D@2@@std@@@2@@std@@IAEXI@Z 100c3410 f i libsg_MSVC120_vc:sg_common.obj
 0001:000c24c0       ?dec@std@@YAAAVios_base@1@AAV21@@Z 100c34c0 f i libsg_MSVC120_vc:sg_common.obj
 0001:000c24e0       ?hex@std@@YAAAVios_base@1@AAV21@@Z 100c34e0 f i libsg_MSVC120_vc:sg_common.obj
 0001:000c2500       ?push_back@?$vector@V?$basic_string@DU?$char_traits@D@std@@V?$allocator@D@2@@std@@V?$allocator@V?$basic_string@DU?$char_traits@D@std@@V?$allocator@D@2@@std@@@2@@std@@QAEX$$QAV?$basic_string@DU?$char_traits@D@std@@V?$allocator@D@2@@2@@Z 100c3500 f i libsg_MSVC120_vc:sg_common.obj
 0001:000c2580       ?put@?$basic_ostream@DU?$char_traits@D@std@@@std@@QAEAAV12@D@Z 100c3580 f i libsg_MSVC120_vc:sg_common.obj
 0001:000c27d0       ?to_string@std@@YA?AV?$basic_string@DU?$char_traits@D@std@@V?$allocator@D@2@@1@_J@Z 100c37d0 f i libsg_MSVC120_vc:sg_common.obj
 0001:000c2850       _createEncryptedMacFile    100c3850 f   libsg_MSVC120_vc:sg_common.obj
 0001:000c28d0       _createHashValue           100c38d0 f   libsg_MSVC120_vc:sg_common.obj
 0001:000c2900       _getLowestBit              100c3900 f   libsg_MSVC120_vc:sg_common.obj
 0001:000c2920       _getPCIConfigData          100c3920 f   libsg_MSVC120_vc:sg_common.obj
 0001:000c2930       _getTargetAuthentication   100c3930 f   libsg_MSVC120_vc:sg_common.obj
 0001:000c3850       _printWarningMessage       100c4850 f   libsg_MSVC120_vc:sg_common.obj
 0001:000c3890       _readPciBar                100c4890 f   libsg_MSVC120_vc:sg_common.obj
 0001:000c39a0       _setPCIConfigAddress       100c49a0 f   libsg_MSVC120_vc:sg_common.obj
 0001:000c39e0       _setPCIConfigData          100c49e0 f   libsg_MSVC120_vc:sg_common.obj
 0001:000c3a00       _sg_checkTargetAuthentication 100c4a00 f   libsg_MSVC120_vc:sg_common.obj
 0001:000c3a30       _sg_createMutex            100c4a30 f   libsg_MSVC120_vc:sg_common.obj
 0001:000c3a50       _sg_createSemaphore        100c4a50 f   libsg_MSVC120_vc:sg_common.obj
 0001:000c3a70       _sg_createThread           100c4a70 f   libsg_MSVC120_vc:sg_common.obj
 0001:000c3aa0       _sg_destroyMutex           100c4aa0 f   libsg_MSVC120_vc:sg_common.obj
 0001:000c3ab0       _sg_destroySemaphore       100c4ab0 f   libsg_MSVC120_vc:sg_common.obj
 0001:000c3ad0       _sg_destroyThread          100c4ad0 f   libsg_MSVC120_vc:sg_common.obj
 0001:000c3b00       _sg_detectPciDevice        100c4b00 f   libsg_MSVC120_vc:sg_common.obj
 0001:000c3b30       _sg_doesFsNodeExist        100c4b30 f   libsg_MSVC120_vc:sg_common.obj
 0001:000c3b50       _sg_findPciDevice          100c4b50 f   libsg_MSVC120_vc:sg_common.obj
 0001:000c3dd0       _sg_fullFile               100c4dd0 f   libsg_MSVC120_vc:sg_common.obj
 0001:000c3e70       _sg_getConfigBaseDir       100c4e70 f   libsg_MSVC120_vc:sg_common.obj
 0001:000c3eb0       _sg_getElapsedTime         100c4eb0 f   libsg_MSVC120_vc:sg_common.obj
 0001:000c3ed0       _sg_getModelBaseDir        100c4ed0 f   libsg_MSVC120_vc:sg_common.obj
 0001:000c3f10       _sg_lockMutex              100c4f10 f   libsg_MSVC120_vc:sg_common.obj
 0001:000c3f20       _sg_mapIo                  100c4f20 f   libsg_MSVC120_vc:sg_common.obj
 0001:000c3f30       _sg_mapMemory              100c4f30 f   libsg_MSVC120_vc:sg_common.obj
 0001:000c3f60       _sg_releaseSemaphore       100c4f60 f   libsg_MSVC120_vc:sg_common.obj
 0001:000c3f80       _sg_setAbilities           100c4f80 f   libsg_MSVC120_vc:sg_common.obj
 0001:000c3f90       _sg_setDriveLetter         100c4f90 f   libsg_MSVC120_vc:sg_common.obj
 0001:000c3fa0       _sg_showPciDevice          100c4fa0 f   libsg_MSVC120_vc:sg_common.obj
 0001:000c4060       _sg_tryLockMutex           100c5060 f   libsg_MSVC120_vc:sg_common.obj
 0001:000c4080       _sg_unlockMutex            100c5080 f   libsg_MSVC120_vc:sg_common.obj
 0001:000c4090       _sg_waitForSemaphore       100c5090 f   libsg_MSVC120_vc:sg_common.obj
 0001:000c40b0       _sg_wait_ns                100c50b0 f   libsg_MSVC120_vc:sg_common.obj
 0001:000c4100       _sg_wait_s                 100c5100 f   libsg_MSVC120_vc:sg_common.obj
 0001:000c4120       ?compare@?$char_traits@D@std@@SAHPBD0I@Z 100c5120 f i libsg_MSVC120_vc:sg_target.obj
 0001:000c4190       ?find@?$basic_string@DU?$char_traits@D@std@@V?$allocator@D@2@@std@@QBEIPBDII@Z 100c5190 f i libsg_MSVC120_vc:sg_target.obj
 0001:000c4230       _sg_getCpuTemperature      100c5230 f   libsg_MSVC120_vc:sg_target.obj
 0001:000c4250       _sg_getTargetMatlabVersion 100c5250 f   libsg_MSVC120_vc:sg_target.obj
 0001:000c43e0       _sg_target_getHostLinkMac  100c53e0 f   libsg_MSVC120_vc:sg_target.obj
 0001:000c4420       _sg_target_getTccActivationTemp 100c5420 f   libsg_MSVC120_vc:sg_target.obj
 0001:000c4430       ?MurmurHash3_x64_128@@YAXPBXHIPAX@Z 100c5430 f   libsg_MSVC120_vc:MurmurHash3.obj
 0001:000c4880       ?MurmurHash3_x86_128@@YAXPBXHIPAX@Z 100c5880 f   libsg_MSVC120_vc:MurmurHash3.obj
 0001:000c4ba0       ?MurmurHash3_x86_32@@YAXPBXHIPAX@Z 100c5ba0 f   libsg_MSVC120_vc:MurmurHash3.obj
 0001:000c4c54       __wcsdup                   100c5c54 f   LIBCMT:wcsdup.obj
 0001:000c4ca7       __invoke_watson_if_oneof   100c5ca7 f i LIBCMT:setlocal.obj
 0001:000c4cd2       _setlocale                 100c5cd2 f   LIBCMT:setlocal.obj
 0001:000c4eb6       __fseek_nolock             100c5eb6 f   LIBCMT:fseek.obj
 0001:000c4f45       _fseek                     100c5f45 f   LIBCMT:fseek.obj
 0001:000c4fc8       __wfopen                   100c5fc8 f   LIBCMT:wfopen.obj
 0001:000c4fdd       __wfopen_s                 100c5fdd f   LIBCMT:wfopen.obj
 0001:000c5022       __wfsopen                  100c6022 f   LIBCMT:wfopen.obj
 0001:000c50f0       _strcspn                   100c60f0 f   LIBCMT:strcspn.obj
 0001:000c5136       __Getdays                  100c6136 f   LIBCMT:strftime.obj
 0001:000c513f       __Getdays_l                100c613f f   LIBCMT:strftime.obj
 0001:000c5226       __Getmonths                100c6226 f   LIBCMT:strftime.obj
 0001:000c522f       __Getmonths_l              100c622f f   LIBCMT:strftime.obj
 0001:000c5322       __Gettnames                100c6322 f   LIBCMT:strftime.obj
 0001:000c532b       __Strftime                 100c632b f   LIBCMT:strftime.obj
 0001:000c5349       __Strftime_l               100c6349 f   LIBCMT:strftime.obj
 0001:000c546c       __strftime_l               100c646c f   LIBCMT:strftime.obj
 0001:000c548a       _strftime                  100c648a f   LIBCMT:strftime.obj
 0001:000c5ec0       __W_Getdays                100c6ec0 f   LIBCMT:wcsftime.obj
 0001:000c5ec9       __W_Getdays_l              100c6ec9 f   LIBCMT:wcsftime.obj
 0001:000c5fe2       __W_Getmonths              100c6fe2 f   LIBCMT:wcsftime.obj
 0001:000c5feb       __W_Getmonths_l            100c6feb f   LIBCMT:wcsftime.obj
 0001:000c6104       __W_Gettnames              100c7104 f   LIBCMT:wcsftime.obj
 0001:000c610d       __W_Gettnames_l            100c710d f   LIBCMT:wcsftime.obj
 0001:000c67bc       __Wcsftime                 100c77bc f   LIBCMT:wcsftime.obj
 0001:000c67da       __Wcsftime_l               100c77da f   LIBCMT:wcsftime.obj
 0001:000c691d       __wcsftime_l               100c791d f   LIBCMT:wcsftime.obj
 0001:000c693b       _wcsftime                  100c793b f   LIBCMT:wcsftime.obj
 0001:000c6960       _memchr                    100c7960 f   LIBCMT:memchr.obj
 0001:000c6a10       __aulldiv                  100c7a10 f   LIBCMT:ulldiv.obj
 0001:000c6d1c       ___crtCompareStringA       100c7d1c f   LIBCMT:a_cmp.obj
 0001:000c6d5f       ___crtCompareStringW       100c7d5f f   LIBCMT:w_cmp.obj
 0001:000c6dc3       __ftell_nolock             100c7dc3 f   LIBCMT:ftell.obj
 0001:000c7153       _ftell                     100c8153 f   LIBCMT:ftell.obj
 0001:000c71bf       __access                   100c81bf f   LIBCMT:access.obj
 0001:000c71d5       __access_s                 100c81d5 f   LIBCMT:access.obj
 0001:000c7220       __libm_sse2_pow_precise    100c8220 f   LIBCMT:pow_sse2_precise.obj
 0001:000c7d90       __mbstowcs_l               100c8d90 f   LIBCMT:mbstowcs.obj
 0001:000c7d99       __mbstowcs_l_helper        100c8d99 f   LIBCMT:mbstowcs.obj
 0001:000c7efa       __mbstowcs_s_l             100c8efa f   LIBCMT:mbstowcs.obj
 0001:000c7fd8       _mbstowcs                  100c8fd8 f   LIBCMT:mbstowcs.obj
 0001:000c8000       _mbstowcs_s                100c9000 f   LIBCMT:mbstowcs.obj
 0001:000c8051       __wcstombs_l               100c9051 f   LIBCMT:wcstombs.obj
 0001:000c805a       __wcstombs_l_helper        100c905a f   LIBCMT:wcstombs.obj
 0001:000c82c1       __wcstombs_s_l             100c92c1 f   LIBCMT:wcstombs.obj
 0001:000c838c       _wcstombs                  100c938c f   LIBCMT:wcstombs.obj
 0001:000c83a4       _wcstombs_s                100c93a4 f   LIBCMT:wcstombs.obj
 0001:000c83c2       __wopenfile                100c93c2 f   LIBCMT:_wopen.obj
 0001:000c8660       ___tzset                   100c9660 f   LIBCMT:tzset.obj
 0001:000c86b0       __isindst                  100c96b0 f   LIBCMT:tzset.obj
 0001:000c88de       __set_daylight             100c98de f i LIBCMT:tzset.obj
 0001:000c88ed       __set_dstbias              100c98ed f i LIBCMT:tzset.obj
 0001:000c88fc       __set_timezone             100c98fc f i LIBCMT:tzset.obj
 0001:000c890b       __tzset                    100c990b f   LIBCMT:tzset.obj
 0001:000c8e59       ___daylight                100c9e59 f   LIBCMT:timeset.obj
 0001:000c8e5f       ___dstbias                 100c9e5f f   LIBCMT:timeset.obj
 0001:000c8e65       ___timezone                100c9e65 f   LIBCMT:timeset.obj
 0001:000c8e6b       ___tzname                  100c9e6b f   LIBCMT:timeset.obj
 0001:000c8e71       __get_daylight             100c9e71 f   LIBCMT:timeset.obj
 0001:000c8e9b       __get_dstbias              100c9e9b f   LIBCMT:timeset.obj
 0001:000c8ec5       __get_timezone             100c9ec5 f   LIBCMT:timeset.obj
 0001:000c8eef       __get_tzname               100c9eef f   LIBCMT:timeset.obj
 0001:000c8f82       __waccess                  100c9f82 f   LIBCMT:waccess.obj
 0001:000c8f98       __waccess_s                100c9f98 f   LIBCMT:waccess.obj
 0001:000c9040       _pow                       100ca040 f   LIBCMT:pow.obj
 0001:000c9080       __CIpow                    100ca080 f   LIBCMT:pow.obj
 0001:000c90bb       __CIpow_default            100ca0bb f   LIBCMT:pow.obj
 0001:000c90d4       __pow_default              100ca0d4     LIBCMT:pow.obj
 0001:000c92ca       __dupenv_s                 100ca2ca f   LIBCMT:getenv.obj
 0001:000c943d       __getenv_helper_nolock     100ca43d f   LIBCMT:getenv.obj
 0001:000c955c       _getenv                    100ca55c f   LIBCMT:getenv.obj
 0001:000c95dc       _getenv_s                  100ca5dc f   LIBCMT:getenv.obj
 0001:000c96b0       __CIpow_pentium4           100ca6b0 f   LIBCMT:pow_pentium4.obj
 0001:000c96c9       __pow_pentium4             100ca6c9     LIBCMT:pow_pentium4.obj
 0001:000ca221       __fFEXP                    100cb221     LIBCMT:87tran.obj
 0001:000ca278       __rtinfpopse               100cb278     LIBCMT:87tran.obj
 0001:000ca27a       __rtinfnpopse              100cb27a     LIBCMT:87tran.obj
 0001:000ca28a       __fFLN                     100cb28a     LIBCMT:87tran.obj
 0001:000ca33f       __rtinfpop                 100cb33f     LIBCMT:87tran.obj
 0001:000ca341       __rtinfnpop                100cb341     LIBCMT:87tran.obj
 0001:000ca35e       __ffexpm1                  100cb35e     LIBCMT:87tran.obj
 0001:000ca407       __d_inttype                100cb407 f   LIBCMT:powhlp.obj
 0001:000ca46f       __powhlp                   100cb46f f   LIBCMT:powhlp.obj
 0001:000ca5a5       _strnlen                   100cb5a5 f   LIBCMT:strlen_s.obj
 0001:000ca5c0       ___wtomb_environ           100cb5c0 f   LIBCMT:wtombenv.obj
 0001:000ca64f       __mbsnbicoll               100cb64f f   LIBCMT:mbsnbico.obj
 0001:000ca667       __mbsnbicoll_l             100cb667 f   LIBCMT:mbsnbico.obj
 0001:000ca71d       ___crtsetenv               100cb71d f   LIBCMT:setenv.obj
 0001:000caa20       __strnicoll                100cba20 f   LIBCMT:strnicol.obj
 0001:000caa47       __strnicoll_l              100cba47 f   LIBCMT:strnicol.obj
 0001:000cab0c       __strdup                   100cbb0c f   LIBCMT:strdup.obj
 0001:000cab5c       __mbschr                   100cbb5c f   LIBCMT:mbschr.obj
 0001:000cab71       __mbschr_l                 100cbb71 f   LIBCMT:mbschr.obj
 0001:000cac0e       ??0_Init_cout@std@@QAE@XZ  100cbc0e f i libcpmt:cout.obj
 0001:000cac67       ?tie@?$basic_ios@DU?$char_traits@D@std@@@std@@QAEPAV?$basic_ostream@DU?$char_traits@D@std@@@2@PAV32@@Z 100cbc67 f i libcpmt:cout.obj
 0001:000cac78       _FindFirstFileA@8          100cbc78 f   kernel32:KERNEL32.dll
 0001:000cac7e       _FindNextFileA@8           100cbc7e f   kernel32:KERNEL32.dll
 0001:000cac84       _ReleaseSemaphore@12       100cbc84 f   kernel32:KERNEL32.dll
 0001:000cac8a       _ReleaseMutex@4            100cbc8a f   kernel32:KERNEL32.dll
 0001:000cac90       _CreateMutexA@12           100cbc90 f   kernel32:KERNEL32.dll
 0001:000cac96       _CreateThread@24           100cbc96 f   kernel32:KERNEL32.dll
 0001:000cac9c       _TerminateThread@8         100cbc9c f   kernel32:KERNEL32.dll
 0001:000caca2       _CreateSemaphoreA@16       100cbca2 f   kernel32:KERNEL32.dll
 0001:000caca8       _GetTimeZoneInformation@4  100cbca8 f   kernel32:KERNEL32.dll
 0001:000cacae       _GetFileAttributesExW@12   100cbcae f   kernel32:KERNEL32.dll
 0001:000cacb4       _SetEnvironmentVariableA@8 100cbcb4 f   kernel32:KERNEL32.dll
 0001:000cacc0       _restoreInterrupts         100cbcc0 f   xpcruntime:xpcPCFunctions.obj
 0001:000cacd0       _rl32eGetTicksDouble       100cbcd0 f   xpcruntime:xpcPCFunctions.obj
 0001:000cad40       _saveAndDisableInterrupts  100cbd40 f   xpcruntime:xpcPCFunctions.obj
 0001:000cad60       _xPCSubtractTime           100cbd60 f   xpcruntime:xpcPCFunctions.obj
 0001:000cad80       _xpcSubtractTime           100cbd80 f   xpcruntime:xpcPCFunctions.obj
 0002:00000000       ___xc_a                    10103000     LIBCMT:crt0init.obj
 0002:0000048c       ___xc_z                    1010348c     LIBCMT:crt0init.obj
 0002:00000590       ___xi_a                    10103590     LIBCMT:crt0init.obj
 0002:000007ac       ___xi_z                    101037ac     LIBCMT:crt0init.obj
 0002:000008b0       ___xp_a                    101038b0     LIBCMT:crt0init.obj
 0002:00000bc4       ___xp_z                    10103bc4     LIBCMT:crt0init.obj
 0002:00000cc8       ___xt_a                    10103cc8     LIBCMT:crt0init.obj
 0002:00000dcc       ___xt_z                    10103dcc     LIBCMT:crt0init.obj
 0002:00000f08       ??_C@_07DGGOPEII@CANTest?$AA@ 10103f08     xpctarget.obj
 0002:00000f14       _ptsetfilename             10103f14     xpctarget.obj
 0002:00000f18       _xmlfile                   10103f18     xpctarget.obj
 0002:00000f20       ??_C@_03COLHFAIP@6?48?$AA@ 10103f20     xpctarget.obj
 0002:00000f24       ??_C@_01DNKMNLPK@?$HM?$AA@ 10103f24     xpctarget.obj
 0002:00000f28       __real@3fb999999999999a    10103f28     xpctarget.obj
 0002:00000f38       __real@407f400000000000    10103f38     xpctarget.obj
 0002:00000f48       _CANTest_BIOMAP            10103f48     appmappingData.obj
 0002:00001068       _CANTest_LBLMAP            10104068     appmappingData.obj
 0002:00001188       _CANTest_SIDMAP            10104188     appmappingData.obj
 0002:000012a8       _CANTest_SBIO              101042a8     appmappingData.obj
 0002:00001308       _CANTest_SLBL              10104308     appmappingData.obj
 0002:00001368       _CANTest_PTIDSMAP          10104368     appmappingData.obj
 0002:00001510       _CANTest_PTNAMESMAP        10104510     appmappingData.obj
 0002:000016b8       _CANTest_SPTMAP            101046b8     appmappingData.obj
 0002:0000178c       _CANTest_dtmap             1010478c     appmappingData.obj
 0002:000017b0       _appInfo                   101047b0     appmappingData.obj
 0002:000019b9       ??_C@_00CNPNBAHC@?$AA@     101049b9     appmappingData.obj
 0002:000019c0       __real@3cb0000000000000    101049c0     rt_matrx.obj
 0002:000019d0       __real@3fe0000000000000    101049d0     rt_matrx.obj
 0002:000019e0       __real@3ff0000000000000    101049e0     rt_matrx.obj
 0002:00002250       ??_C@_0DJ@FHKINPLE@Unexpected?5itemKind?5?$DN?5DATA_ITEM?5@ 10105250     rt_logging.obj
 0002:00002294       ??_C@_0DA@IEHFPFCJ@Unexpected?5itemKind?$DN?$CFd?5in?5rt_Pro@ 10105294     rt_logging.obj
 0002:000022d0       ??_C@_0DA@IFLHJPBO@Unexpected?5itemKind?$DN?$CFd?5in?5rt_Pro@ 101052d0     rt_logging.obj
 0002:0000230c       ??_C@_0DA@IAPIIJJL@Unexpected?5itemKind?$DN?$CFd?5in?5rt_Pro@ 1010530c     rt_logging.obj
 0002:00002348       ??_C@_0BE@LCIGPJIG@MATLAB?55?40?5MAT?9file?$AA@ 10105348     rt_logging.obj
 0002:00002360       ??_C@_0FB@PCJEAJIB@?$CK?$CK?$CK?5Log?5variable?5?$CFs?5has?5wrapped?5@ 10105360     rt_logging.obj
 0002:000023c8       ??_C@_0MG@NKMLMOGF@?$CK?$CK?$CK?5To?5avoid?5wrapping?0?5explicitl@ 101053c8     rt_logging.obj
 0002:000024b8       ??_C@_0N@IPAEOLLP@_rtw_tmw?4tmw?$AA@ 101054b8     rt_logging.obj
 0002:000024c8       ??_C@_04HDOCAJNK@?$CFs?$CFs?$AA@ 101054c8     rt_logging.obj
 0002:000024d0       ??_C@_03ELIABIOC@w?$CLb?$AA@ 101054d0     rt_logging.obj
 0002:000024d4       ??_C@_0BF@JPILDDFA@?$CK?$CK?$CK?5Error?5opening?5?$CFs?$AA@ 101054d4     rt_logging.obj
 0002:000024f0       ??_C@_0BK@EEMDELA@unable?5to?5open?5data?5file?6?$AA@ 101054f0     rt_logging.obj
 0002:00002510       ??_C@_04CGFJFPFD@none?$AA@ 10105510     rt_logging.obj
 0002:00002518       ??_C@_0EE@LCGFPNON@?$CK?$CK?$CK?5Error?5creating?5signals?5struc@ 10105518     rt_logging.obj
 0002:0000256c       ??_C@_0CE@NHECEDMK@?$CK?$CK?$CK?5Error?5creating?5log?5variable?5@ 1010556c     rt_logging.obj
 0002:00002598       ??_C@_0DB@IOCGKAGH@?$CK?$CK?$CK?5Errors?5occurred?5when?5startin@ 10105598     rt_logging.obj
 0002:000025d4       ??_C@_0BO@BBLOGEBK@?$CK?$CK?$CK?5Memory?5allocation?5error?4?6?$AA@ 101055d4     rt_logging.obj
 0002:000025f8       ??_C@_0N@LGFBAGEL@?5?$CIreal?5part?$CJ?$AA@ 101055f8     rt_logging.obj
 0002:00002608       ??_C@_0KH@CGNMHNFE@?5?5?5?5varName?5?5?5?5?5?5?5?5?5?5?$DN?5?$CFs?$CFs?6?5?5?5?5@ 10105608     rt_logging.obj
 0002:000026d0       ??_C@_0LE@OALKKEFM@?5?5?5?5varName?5?5?5?5?5?5?5?5?5?5?$DN?5?$CFs?5?$CIcompl@ 101056d0     rt_logging.obj
 0002:000027a8       ??_C@_0KF@JDDLEOKO@?5?5?5?5varName?5?5?5?5?5?5?5?5?5?5?$DN?5?$CFs?6?5?5?5?5nR@ 101057a8     rt_logging.obj
 0002:00002870       ??_C@_0DP@HPDMIOFM@?$CK?$CK?$CK?5Using?5a?5default?5buffer?5of?5si@ 10105870     rt_logging.obj
 0002:000028c0       ??_C@_0KE@JEFOLKNF@?6?$CK?$CK?$CK?5Memory?5required?5to?5log?5vari@ 101058c0     rt_logging.obj
 0002:00002988       ??_C@_0JP@DKLMHCBI@?$CK?$CK?$CK?5Details?3?6?5?5?5?5?5?5?5varName?5?5?5?5?5@ 10105988     rt_logging.obj
 0002:00002a48       ??_C@_0CM@CAMILBED@?$CK?$CK?$CK?5Error?5allocating?5memory?5for?5@ 10105a48     rt_logging.obj
 0002:00002a7c       ??_C@_0DF@BBCNMOPM@?$CK?$CK?$CK?5Error?5allocating?5memory?5for?5@ 10105a7c     rt_logging.obj
 0002:00002ac0       ??_C@_0JP@DBCLPCCI@?$CK?$CK?$CK?5Details?3?6?5?5?5?5?5?5?5varName?5?5?5?5?5@ 10105ac0     rt_logging.obj
 0002:00002b80       ??_C@_0FK@DPGAOBGA@?$CK?$CK?$CK?5Error?5allocating?5memory?5for?5@ 10105b80     rt_logging.obj
 0002:00002bec       ??_C@_0BI@GGDNPHLJ@?$CK?$CK?$CK?5Error?5writing?5to?5?$CFs?$AA@ 10105bec     rt_logging.obj
 0002:00002c08       ??_C@_0CB@IBGJGELG@?$CK?$CK?$CK?5Error?5writing?5?$CFs?5due?5to?3?5?$CFs?6@ 10105c08     rt_logging.obj
 0002:00002c30       ??_C@_0CN@FLMCHCPB@?$CK?$CK?$CK?5Error?5writing?5log?5variable?5?$CF@ 10105c30     rt_logging.obj
 0002:00002c68       ??_C@_0DH@GAJCNOJP@?$CK?$CK?$CK?5Error?5writing?5structure?5log?5@ 10105c68     rt_logging.obj
 0002:00002cac       ??_C@_0BD@POEALECL@?$CK?$CK?5created?5?$CFs?5?$CK?$CK?6?6?$AA@ 10105cac     rt_logging.obj
 0002:00002cc8       __real@0000000000000000    10105cc8     rt_logging.obj
 0002:00002cd8       __real@4020000000000000    10105cd8     rt_logging.obj
 0002:00002ce8       __real@41dfffffffc00000    10105ce8     rt_logging.obj
 0002:00002cf8       __real@41efffffffe00000    10105cf8     rt_logging.obj
 0002:00002d08       __real@4330000000000000    10105d08     rt_logging.obj
 0002:00002d18       __real@8000000000000000    10105d18     rt_logging.obj
 0002:00002d28       __real@bfbf9add3afd2773    10105d28     rt_logging.obj
 0002:00002d38       __real@bff0000000000000    10105d38     rt_logging.obj
 0002:00002d48       __real@c000000000000000    10105d48     rt_logging.obj
 0002:00002d60       __xmm@20202020202020202020202020202020 10105d60     rt_logging.obj
 0002:00002d80       __xmm@41f00000000000000000000000000000 10105d80     rt_logging.obj
 0002:00002d94       ??_C@_06FAENGAMN@DSTATE?$AA@ 10105d94     CANTest.obj
 0002:00002d9c       ??_C@_0BJ@NFEJJNHO@CANTest?1Mon_Cont?1LPFM?1d1?$AA@ 10105d9c     CANTest.obj
 0002:00002dbc       ??_C@_0BI@HIACJKBI@CANTest?1Mon_Cont?1LPFM?1d?$AA@ 10105dbc     CANTest.obj
 0002:00002dd8       _CANTest_M                 10105dd8     CANTest.obj
 0002:00002ddc       ??_C@_0BC@OJJPBDHH@FixedStepDiscrete?$AA@ 10105ddc     CANTest.obj
 0002:00002df4       ??_C@_04EPKDLPPB@tout?$AA@ 10105df4     CANTest.obj
 0002:00002dfc       ??_C@_04IKFDFCPA@xout?$AA@ 10105dfc     CANTest.obj
 0002:00002e04       ??_C@_03HBFGMJOD@rt_?$AA@  10105e04     CANTest.obj
 0002:00002e08       ??_C@_09BBCLLDMP@CAN?5Setup?$AA@ 10105e08     CANTest.obj
 0002:00002e14       ??_C@_0BJ@FHLCMGDD@CANTest?1DAQ_In?1CAN?5Setup?$AA@ 10105e14     CANTest.obj
 0002:00002e34       ??_C@_09EJDGHAME@CAN?5Read1?$AA@ 10105e34     CANTest.obj
 0002:00002e40       ??_C@_0BJ@PKPAFDI@CANTest?1DAQ_In?1CAN?5Read1?$AA@ 10105e40     CANTest.obj
 0002:00002e60       ??_C@_0L@BNCKLANN@CAN?5Write1?$AA@ 10105e60     CANTest.obj
 0002:00002e70       ??_C@_0CE@BLHJEHJM@CANTest?1DAQ_Out?1CANBoard?1CAN?5Wri@ 10105e70     CANTest.obj
 0002:00002ea0       __real@3f60624dd2f1a9fc    10105ea0     CANTest.obj
 0002:00002eb0       __real@4008000000000000    10105eb0     CANTest.obj
 0002:00002ec0       __real@401c000000000000    10105ec0     CANTest.obj
 0002:00002ed0       __real@4024000000000000    10105ed0     CANTest.obj
 0002:00002ee0       __real@402e000000000000    10105ee0     CANTest.obj
 0002:00002ef0       __real@4069000000000000    10105ef0     CANTest.obj
 0002:00002f00       __real@40e0000000000000    10105f00     CANTest.obj
 0002:00002f10       __real@40efffe000000000    10105f10     CANTest.obj
 0002:00002f20       __real@41f0000000000000    10105f20     CANTest.obj
 0002:00002f30       __real@c069000000000000    10105f30     CANTest.obj
 0002:00002f40       __xmm@00000000000000003f60624dd2f1a9fc 10105f40     CANTest.obj
 0002:00002f60       __xmm@000000a3000000170000002700000001 10105f60     CANTest.obj
 0002:000038d8       ??_C@_0BE@MNNBMEFJ@DAQ_In?1CAN?5Read1?1p1?$AA@ 101068d8     CANTest_capi.obj
 0002:000038f0       ??_C@_0BE@OGPMJHJK@DAQ_In?1CAN?5Read1?1p2?$AA@ 101068f0     CANTest_capi.obj
 0002:00003908       ??_C@_0BG@PFCKGPME@DAQ_In?1CAN?5Unpack2?1p1?$AA@ 10106908     CANTest_capi.obj
 0002:00003924       ??_C@_03JGNEPIDC@RPM?$AA@  10106924     CANTest_capi.obj
 0002:00003928       ??_C@_0BG@NOAHDMAH@DAQ_In?1CAN?5Unpack2?1p2?$AA@ 10106928     CANTest_capi.obj
 0002:00003944       ??_C@_02MIKLMMJE@TQ?$AA@   10106944     CANTest_capi.obj
 0002:00003948       ??_C@_0P@MLBKJILF@Mon_Cont?1ContM?$AA@ 10106948     CANTest_capi.obj
 0002:0000395c       ??_C@_08CIGKJJFI@ContMode?$AA@ 1010695c     CANTest_capi.obj
 0002:00003968       ??_C@_0BK@BKIKJDHD@DAQ_Out?1CANBoard?1Constant?$AA@ 10106968     CANTest_capi.obj
 0002:00003988       ??_C@_05GMBADOLI@Ready?$AA@ 10106988     CANTest_capi.obj
 0002:00003990       ??_C@_0BL@PELKNKH@DAQ_Out?1CANBoard?1Constant1?$AA@ 10106990     CANTest_capi.obj
 0002:000039b0       ??_C@_04ILOKDBOJ@Gear?$AA@ 101069b0     CANTest_capi.obj
 0002:000039b8       ??_C@_0BL@CEGGPOGE@DAQ_Out?1CANBoard?1Constant2?$AA@ 101069b8     CANTest_capi.obj
 0002:000039d8       ??_C@_03GHCKAFB@BMS?$AA@   101069d8     CANTest_capi.obj
 0002:000039dc       ??_C@_0BL@DNHNMPCF@DAQ_Out?1CANBoard?1Constant3?$AA@ 101069dc     CANTest_capi.obj
 0002:000039fc       ??_C@_08GLBEHMNM@PosTQLim?$AA@ 101069fc     CANTest_capi.obj
 0002:00003a08       ??_C@_0BL@HCDMFJOC@DAQ_Out?1CANBoard?1Constant4?$AA@ 10106a08     CANTest_capi.obj
 0002:00003a28       ??_C@_08NEHEBCK@NegTQLim?$AA@ 10106a28     CANTest_capi.obj
 0002:00003a34       ??_C@_0BK@ECBCLENL@DAQ_Out?1CANBoard?1CAN?5Pack?$AA@ 10106a34     CANTest_capi.obj
 0002:00003a54       ??_C@_0BD@CDBAFIAD@Mon_Cont?1LPFM?1gain?$AA@ 10106a54     CANTest_capi.obj
 0002:00003a6c       ??_C@_0BE@FPHHEGFA@Mon_Cont?1LPFM?1gain1?$AA@ 10106a6c     CANTest_capi.obj
 0002:00003a84       ??_C@_0BE@HEFKBFJD@Mon_Cont?1LPFM?1gain2?$AA@ 10106a84     CANTest_capi.obj
 0002:00003a9c       ??_C@_0BH@GPJEMOCG@Mon_Cont?1LPFM?1Product1?$AA@ 10106a9c     CANTest_capi.obj
 0002:00003ab8       ??_C@_0BI@BEDPBGIB@Mon_Cont?1LPFM?1Product11?$AA@ 10106ab8     CANTest_capi.obj
 0002:00003ad4       ??_C@_0BH@EELJJNOF@Mon_Cont?1LPFM?1Product2?$AA@ 10106ad4     CANTest_capi.obj
 0002:00003af0       ??_C@_0BD@JCOAGPMK@Mon_Cont?1LPFM?1Sum1?$AA@ 10106af0     CANTest_capi.obj
 0002:00003b08       ??_C@_0BD@LJMNDMAJ@Mon_Cont?1LPFM?1Sum2?$AA@ 10106b08     CANTest_capi.obj
 0002:00003b20       ??_C@_0BD@KANGANEI@Mon_Cont?1LPFM?1Sum3?$AA@ 10106b20     CANTest_capi.obj
 0002:00003b38       ??_C@_0BD@OPJHJLIP@Mon_Cont?1LPFM?1Sum4?$AA@ 10106b38     CANTest_capi.obj
 0002:00003b50       ??_C@_0BA@IOPEPKAJ@Mon_Cont?1LPFM?1d?$AA@ 10106b50     CANTest_capi.obj
 0002:00003b64       ??_C@_0BB@LPAPELOM@Mon_Cont?1LPFM?1d1?$AA@ 10106b64     CANTest_capi.obj
 0002:00003b78       ??_C@_0BB@GFOJNDKK@DAQ_In?1CAN?5Read1?$AA@ 10106b78     CANTest_capi.obj
 0002:00003b8c       ??_C@_02KKFPAPOP@P1?$AA@   10106b8c     CANTest_capi.obj
 0002:00003b90       ??_C@_02IBHCFMCM@P2?$AA@   10106b90     CANTest_capi.obj
 0002:00003b94       ??_C@_02JIGJGNGN@P3?$AA@   10106b94     CANTest_capi.obj
 0002:00003b98       ??_C@_02NHCIPLKK@P4?$AA@   10106b98     CANTest_capi.obj
 0002:00003b9c       ??_C@_02MODDMKOL@P5?$AA@   10106b9c     CANTest_capi.obj
 0002:00003ba0       ??_C@_02OFBOJJCI@P6?$AA@   10106ba0     CANTest_capi.obj
 0002:00003ba4       ??_C@_0BB@DNPEBAKB@DAQ_In?1CAN?5Setup?$AA@ 10106ba4     CANTest_capi.obj
 0002:00003bb8       ??_C@_02PMAFKIGJ@P7?$AA@   10106bb8     CANTest_capi.obj
 0002:00003bbc       ??_C@_02HLJNLEKG@P8?$AA@   10106bbc     CANTest_capi.obj
 0002:00003bc0       ??_C@_02GCIGIFOH@P9?$AA@   10106bc0     CANTest_capi.obj
 0002:00003bc4       ??_C@_03OPFJJGBF@P10?$AA@  10106bc4     CANTest_capi.obj
 0002:00003bc8       ??_C@_03PGECKHFE@P11?$AA@  10106bc8     CANTest_capi.obj
 0002:00003bcc       ??_C@_03NNGPPEJH@P12?$AA@  10106bcc     CANTest_capi.obj
 0002:00003bd0       ??_C@_03MEHEMFNG@P13?$AA@  10106bd0     CANTest_capi.obj
 0002:00003bd4       ??_C@_03ILDFFDBB@P14?$AA@  10106bd4     CANTest_capi.obj
 0002:00003bd8       ??_C@_03JCCOGCFA@P15?$AA@  10106bd8     CANTest_capi.obj
 0002:00003bdc       ??_C@_03LJADDBJD@P16?$AA@  10106bdc     CANTest_capi.obj
 0002:00003be0       ??_C@_03KABIAANC@P17?$AA@  10106be0     CANTest_capi.obj
 0002:00003be4       ??_C@_03CHIABMBN@P18?$AA@  10106be4     CANTest_capi.obj
 0002:00003be8       ??_C@_03DOJLCNFM@P19?$AA@  10106be8     CANTest_capi.obj
 0002:00003bec       ??_C@_03ONBPCIEM@P20?$AA@  10106bec     CANTest_capi.obj
 0002:00003bf0       ??_C@_03PEAEBJAN@P21?$AA@  10106bf0     CANTest_capi.obj
 0002:00003bf4       ??_C@_03NPCJEKMO@P22?$AA@  10106bf4     CANTest_capi.obj
 0002:00003bf8       ??_C@_03MGDCHLIP@P23?$AA@  10106bf8     CANTest_capi.obj
 0002:00003bfc       ??_C@_03IJHDONEI@P24?$AA@  10106bfc     CANTest_capi.obj
 0002:00003c00       ??_C@_0BD@GJOLMHBL@Mon_Cont?1Constant1?$AA@ 10106c00     CANTest_capi.obj
 0002:00003c18       ??_C@_05LPIJGKJ@Value?$AA@ 10106c18     CANTest_capi.obj
 0002:00003c20       ??_C@_0BC@LDHONOBD@Mon_Cont?1ContMode?$AA@ 10106c20     CANTest_capi.obj
 0002:00003c38       ??_C@_0P@BMHHLDKB@Mon_Cont?1TQCom?$AA@ 10106c38     CANTest_capi.obj
 0002:00003c4c       ??_C@_04OMOMKKFL@Gain?$AA@ 10106c4c     CANTest_capi.obj
 0002:00003c54       ??_C@_0BM@CEKODGPJ@DAQ_Out?1CANBoard?1CAN?5Write1?$AA@ 10106c54     CANTest_capi.obj
 0002:00003c78       ??_C@_0BI@BDJDFDIH@Mon_Cont?1LPFM?1Constant1?$AA@ 10106c78     CANTest_capi.obj
 0002:00003c94       ??_C@_0BB@CFEOEMDC@InitialCondition?$AA@ 10106c94     CANTest_capi.obj
 0002:00003ca8       ??_C@_02GPBJIKLE@Ts?$AA@   10106ca8     CANTest_capi.obj
 0002:00003cac       ??_C@_0O@PPAIJIHF@unsigned?5char?$AA@ 10106cac     CANTest_capi.obj
 0002:00003cbc       ??_C@_09JBMFCIMO@boolean_T?$AA@ 10106cbc     CANTest_capi.obj
 0002:00003cc8       ??_C@_07MMLECJPG@numeric?$AA@ 10106cc8     CANTest_capi.obj
 0002:00003cd4       ??_C@_0N@HINIGIGN@CAN_DATATYPE?$AA@ 10106cd4     CANTest_capi.obj
 0002:00003ce4       ??_C@_06BNJCAIGJ@double?$AA@ 10106ce4     CANTest_capi.obj
 0002:00003cec       ??_C@_06CNMIJIPB@real_T?$AA@ 10106cec     CANTest_capi.obj
 0002:00003cf4       ??_C@_05KNFBNCOH@float?$AA@ 10106cf4     CANTest_capi.obj
 0002:00003cfc       ??_C@_0DL@PGGFBBLM@Error?3?5task?5ID?5?$CFd?5is?5out?5of?5rang@ 10106cfc     CANTest_xcp_TET.obj
 0002:00003d48       __real@3e112e0be826d695    10106d48     CANTest_xcp_TET.obj
 0002:00003d58       __real@3f847ae147ae147b    10106d58     CANTest_xcp_TET.obj
 0002:00003d68       __real@3fefae147ae147ae    10106d68     CANTest_xcp_TET.obj
 0002:00003d78       _CAN_DATATYPE_GROUND       10106d78     can_datatype_ground.obj
 0002:00003d94       _serialfifoground          10106d94     xpc_datatype_ground.obj
 0002:00003da0       _bcmsg1553ground           10106da0     xpc_datatype_ground.obj
 0002:00003db0       _bcstatground              10106db0     xpc_datatype_ground.obj
 0002:00003dc8       _bmmsg1553ground           10106dc8     xpc_datatype_ground.obj
 0002:00003e04       ??_C@_0BI@INNPNFJN@Memory?5Allocation?5Error?$AA@ 10106e04     rtw_modelmap_utils.obj
 0002:00003e20       ??_C@_1HC@PKAJIAEN@?$AAC?$AA?3?$AA?2?$AAP?$AAR?$AAO?$AAG?$AAR?$AAA?$AA?$HO?$AA1?$AA?2?$AAM?$AAA?$AAT?$AAL?$AAA?$AAB?$AA?2?$AAR?$AA2?$AA0?$AA1?$AA8?$AAa?$AA?2?$AAr?$AAt?$AAw?$AA?2?$AAc?$AA?2@ 10106e20     rtw_modelmap_utils.obj
 0002:00003ea8       ??_C@_1CI@OEAJCJND@?$AAj?$AA?5?$AA?$DN?$AA?$DN?$AA?5?$AAe?$AAn?$AAc?$AAo?$AAd?$AAe?$AAd?$AAP?$AAa?$AAt?$AAh?$AAL?$AAe?$AAn?$AA?$AA@ 10106ea8     rtw_modelmap_utils.obj
 0002:00003ed8       ??_C@_1DC@NFAOIFKB@?$AAe?$AAn?$AAc?$AAo?$AAd?$AAe?$AAd?$AAP?$AAa?$AAt?$AAh?$AA?$FL?$AAj?$AA?9?$AA1?$AA?$FN?$AA?5?$AA?$DN?$AA?$DN?$AA?5?$AA?8?$AA?2?$AA0?$AA?8?$AA?$AA@ 10106ed8     rtw_modelmap_utils.obj
 0002:00003f14       ??_C@_1DI@FLNJGPEE@?$AAs?$AAi?$AAg?$AAC?$AAo?$AAm?$AAp?$AAl?$AAe?$AAx?$AAi?$AAt?$AAy?$AA?$FL?$AA?$CK?$AAs?$AAi?$AAg?$AAI?$AAd?$AAx?$AA?$FN?$AA?5?$AA?$CB?$AA?$DN?$AA?5?$AA1?$AA?$AA@ 10106f14     rtw_modelmap_utils.obj
 0002:00003f58       ??_C@_1KI@OFELMGBG@?$AA?$CI?$AA?$CI?$AA?$CI?$AAd?$AAa?$AAt?$AAa?$AAT?$AAy?$AAp?$AAe?$AAM?$AAa?$AAp?$AA?$CJ?$AA?$FL?$AA?$CI?$AA?$CI?$AA?$CI?$AAs?$AAt?$AAa?$AAt?$AAe?$AAs?$AA?$CJ?$AA?$FL?$AA?$CI?$AAi?$AA?$CJ?$AA?$FN?$AA?4@ 10106f58     rtw_modelmap_utils.obj
 0002:00004024       ??_C@_1DA@ILCMPHNE@?$AAf?$AAu?$AAl?$AAl?$AAP?$AAa?$AAt?$AAh?$AA?5?$AA?$CB?$AA?$DN?$AA?5?$AA?$CI?$AA?$CI?$AAv?$AAo?$AAi?$AAd?$AA?5?$AA?$CK?$AA?$CJ?$AA0?$AA?$CJ?$AA?$AA@ 10107024     rtw_modelmap_utils.obj
 0002:00004060       ??_C@_1CI@OEPPFCCA@?$AAp?$AAa?$AAt?$AAh?$AA?5?$AA?$CB?$AA?$DN?$AA?5?$AA?$CI?$AA?$CI?$AAv?$AAo?$AAi?$AAd?$AA?5?$AA?$CK?$AA?$CJ?$AA0?$AA?$CJ?$AA?$AA@ 10107060     rtw_modelmap_utils.obj
 0002:00004090       ??_C@_1FK@GLJIMFHB@?$AA?$CI?$AA?$CI?$AAm?$AAm?$AAi?$AA?$CJ?$AA?9?$AA?$DO?$AAI?$AAn?$AAs?$AAt?$AAa?$AAn?$AAc?$AAe?$AAM?$AAa?$AAp?$AA?4?$AAf?$AAu?$AAl?$AAl?$AAP?$AAa?$AAt?$AAh?$AA?$CJ?$AA?5?$AA?$DN?$AA?$DN@ 10107090     rtw_modelmap_utils.obj
 0002:000040fc       ??_C@_1DG@HPCJGNCE@?$AAm?$AAm?$AAi?$AAP?$AAa?$AAt?$AAh?$AA?$FL?$AAp?$AAa?$AAt?$AAh?$AAL?$AAe?$AAn?$AA?9?$AA1?$AA?$FN?$AA?5?$AA?$DN?$AA?$DN?$AA?5?$AA?8?$AA?2?$AA0?$AA?8?$AA?$AA@ 101070fc     rtw_modelmap_utils.obj
 0002:0000413c       ??_C@_1DM@DBAOGGOO@?$AAm?$AAm?$AAi?$AAP?$AAa?$AAt?$AAh?$AA?$FL?$AAm?$AAm?$AAi?$AAP?$AAa?$AAt?$AAh?$AAL?$AAe?$AAn?$AA?9?$AA1?$AA?$FN?$AA?5?$AA?$DN?$AA?$DN?$AA?5?$AA?8?$AA?2?$AA0?$AA?8?$AA?$AA@ 1010713c     rtw_modelmap_utils.obj
 0002:00004184       ??_C@_1DC@LHIAKAFE@?$AAb?$AAl?$AAo?$AAc?$AAk?$AAP?$AAa?$AAt?$AAh?$AA?5?$AA?$CB?$AA?$DN?$AA?5?$AA?$CI?$AA?$CI?$AAv?$AAo?$AAi?$AAd?$AA?5?$AA?$CK?$AA?$CJ?$AA0?$AA?$CJ?$AA?$AA@ 10107184     rtw_modelmap_utils.obj
 0002:000041c0       ??_C@_1GI@KIEJKPGC@?$AAf?$AAu?$AAl?$AAl?$AAS?$AAt?$AAa?$AAt?$AAe?$AAB?$AAl?$AAo?$AAc?$AAk?$AAP?$AAa?$AAt?$AAh?$AA?$FL?$AAf?$AAu?$AAl?$AAl?$AAS?$AAt?$AAa?$AAt?$AAe?$AAB?$AAl?$AAo?$AAc@ 101071c0     rtw_modelmap_utils.obj
 0002:00004240       ??_C@_1EE@DNPIBJHC@?$AA?$CI?$AA?$CI?$AAd?$AAi?$AAm?$AAM?$AAa?$AAp?$AA?$CJ?$AA?$FL?$AA?$CI?$AAm?$AAa?$AAp?$AAI?$AAd?$AAx?$AA?$CJ?$AA?$FN?$AA?4?$AAn?$AAu?$AAm?$AAD?$AAi?$AAm?$AAs?$AA?$CJ?$AA?5?$AA?$DN?$AA?$DN?$AA?5@ 10107240     rtw_modelmap_utils.obj
 0002:00004294       ??_C@_06JFOKFOED@CSTATE?$AA@ 10107294     rtw_modelmap_utils.obj
 0002:0000429c       ??_C@_1BI@LEBJNOGG@?$AAc?$AAs?$AAv?$AAI?$AAd?$AAx?$AA?5?$AA?$DO?$AA?$DN?$AA?5?$AA0?$AA?$AA@ 1010729c     rtw_modelmap_utils.obj
 0002:000042b8       ??_C@_1BA@KDMGHCHP@?$AAT?$AAI?$AAD?$AA?$DN?$AA?$DN?$AA?9?$AA1?$AA?$AA@ 101072b8     rtw_modelmap_utils.obj
 0002:000042cc       ??_C@_1DM@DHGKBPCE@?$AAs?$AAi?$AAg?$AAP?$AAa?$AAt?$AAh?$AA?$FL?$AAs?$AAi?$AAg?$AAP?$AAa?$AAt?$AAh?$AAL?$AAe?$AAn?$AA?9?$AA1?$AA?$FN?$AA?5?$AA?$DN?$AA?$DN?$AA?5?$AA?8?$AA?2?$AA0?$AA?8?$AA?$AA@ 101072cc     rtw_modelmap_utils.obj
 0002:00004314       ??_C@_0DI@LHHNDFGF@Check?5list?5of?5parameters?0?5?$CFi?5par@ 10107314     sg_IO613_setup_s.obj
 0002:00004358       ??_C@_0BK@FGCMAICJ@Protocol?5is?5not?5supported?$AA@ 10107358     sg_IO613_setup_s.obj
 0002:00004378       ??_C@_0CL@BGDFCID@module?5type?$DN?$CFd?5id?$DN?$CFd?5was?5not?5ini@ 10107378     sg_IO613_setup_s.obj
 0002:000043ac       ??_C@_0DN@MPIPMPFL@SG?5?$CFs?3?5Module?5?$CFi?0?5send?5CAN?5initi@ 101073ac     sg_IO613_setup_s.obj
 0002:000043f8       ??_C@_0DK@NGEPHCKA@SG?5?$CFs?3?5Module?5?$CFi?0?5send?5CAN?5termi@ 101073f8     sg_IO613_setup_s.obj
 0002:00004440       ??_C@_0CO@KLEJKMDK@SG?5?$CFs?3?5Module?5?$CFi?0?5stop?5CAN?5contr@ 10107440     sg_IO613_setup_s.obj
 0002:00004478       ??_C@_0BK@EBKJELMI@maxfunc?5?$DN?5?$CFd?5at?5?$FL?$CFd?0?5?$CFd?$FN?6?$AA@ 10107478     xpcruntime:xpcimports.obj
 0002:00004494       ??_C@_0CC@DMFKNLL@VendorId?5?$DN?50x?$CFx?0?5DeviceId?5?$DN?50x?$CFx@ 10107494     xpcruntime:xpcimports.obj
 0002:000044b8       ??_C@_0DH@OHCBLNMG@Subsystem?5Device?5ID?5?$DN?50x?$CFx?6Subsy@ 101074b8     xpcruntime:xpcimports.obj
 0002:000044f0       ??_C@_0BD@MMMMEFCM@Class?5Code?5?$DN?50x?$CFx?6?$AA@ 101074f0     xpcruntime:xpcimports.obj
 0002:00004504       ??_C@_0BE@OLDDDNHM@InterruptLine?5?$DN?5?$CFd?6?$AA@ 10107504     xpcruntime:xpcimports.obj
 0002:00004518       ??_C@_0CE@IBMFFAPN@bus?5?$DN?5?$CFd?0?5slot?5?$DN?5?$CFd?0?5function?5?$DN?5@ 10107518     xpcruntime:xpcimports.obj
 0002:0000453c       ??_C@_0CE@DGLLGDFH@?5?5?5?5Phys?5?5?5Virtual?5?5?5Length?5IO?1M@ 1010753c     xpcruntime:xpcimports.obj
 0002:00004560       ??_C@_0BI@FEOPLEMG@?$CF08x?5?$CF08x?5?$CF08x?5?5?5?5?5?5?$CFc?6?$AA@ 10107560     xpcruntime:xpcimports.obj
 0002:00004578       ??_C@_0BB@BNNCEDPC@rl32eScopeExists?$AA@ 10107578     xpcruntime:xpcimports.obj
 0002:0000458c       ??_C@_0BM@FJBFEGFG@rl32eScopeExists?5not?5found?6?$AA@ 1010758c     xpcruntime:xpcimports.obj
 0002:000045a8       ??_C@_0O@BNNGKJEA@rl32eDefScope?$AA@ 101075a8     xpcruntime:xpcimports.obj
 0002:000045b8       ??_C@_0BJ@CDNOENKA@rl32eDefScope?5not?5found?6?$AA@ 101075b8     xpcruntime:xpcimports.obj
 0002:000045d4       ??_C@_0P@CKNKILDP@rl32eAddSignal?$AA@ 101075d4     xpcruntime:xpcimports.obj
 0002:000045e4       ??_C@_0BK@GMJAJBAI@rl32eAddSignal?5not?5found?6?$AA@ 101075e4     xpcruntime:xpcimports.obj
 0002:00004600       ??_C@_0BB@LDMIHGCE@rl32eGetSignalNo?$AA@ 10107600     xpcruntime:xpcimports.obj
 0002:00004614       ??_C@_0BM@LGAMBAID@rl32eGetSignalNo?5not?5found?6?$AA@ 10107614     xpcruntime:xpcimports.obj
 0002:00004630       ??_C@_0O@CFDGALBP@rl32eSetScope?$AA@ 10107630     xpcruntime:xpcimports.obj
 0002:00004640       ??_C@_0BJ@JCLHHIN@rl32eSetScope?5not?5found?6?$AA@ 10107640     xpcruntime:xpcimports.obj
 0002:0000465c       ??_C@_0P@IKMCBMHH@xpceFSScopeSet?$AA@ 1010765c     xpcruntime:xpcimports.obj
 0002:0000466c       ??_C@_0BK@JODJPNNH@xpceFSScopeSet?5not?5found?6?$AA@ 1010766c     xpcruntime:xpcimports.obj
 0002:00004688       ??_C@_0BE@DLACEEJM@rl32eSetTargetScope?$AA@ 10107688     xpcruntime:xpcimports.obj
 0002:0000469c       ??_C@_0BP@JCHFMKPJ@rl32eSetTargetScope?5not?5found?6?$AA@ 1010769c     xpcruntime:xpcimports.obj
 0002:000046bc       ??_C@_0BJ@LIDLNDHC@rl32eSetTargetScopeSigFt?$AA@ 101076bc     xpcruntime:xpcimports.obj
 0002:000046d8       ??_C@_0CE@JLGHCFHI@rl32eSetTargetScopeSigFt?5not?5fou@ 101076d8     xpcruntime:xpcimports.obj
 0002:000046fc       ??_C@_0BI@JAPOIDNG@rl32eRestartAcquisition?$AA@ 101076fc     xpcruntime:xpcimports.obj
 0002:00004714       ??_C@_0CD@LLBEFFBO@rl32eRestartAcquisition?5not?5foun@ 10107714     xpcruntime:xpcimports.obj
 0002:00004738       ??_C@_0P@IEIIADJB@xpceScopeAcqOK?$AA@ 10107738     xpcruntime:xpcimports.obj
 0002:00004748       ??_C@_0BK@NJCKNFPN@xpceScopeAcqOK?5not?5found?6?$AA@ 10107748     xpcruntime:xpcimports.obj
 0002:00004764       ??_C@_0BA@IJINKAHF@xpceRegisterISR?$AA@ 10107764     xpcruntime:xpcimports.obj
 0002:00004774       ??_C@_0BL@NNDLOEJE@xpceRegisterISR?5not?5found?6?$AA@ 10107774     xpcruntime:xpcimports.obj
 0002:00004790       ??_C@_0BC@NLBADGKF@xpceDeRegisterISR?$AA@ 10107790     xpcruntime:xpcimports.obj
 0002:000047a4       ??_C@_0BN@DCAIKFFD@xpceDeRegisterISR?5not?5found?6?$AA@ 101077a4     xpcruntime:xpcimports.obj
 0002:000047c4       ??_C@_07JPMEPILD@xpcInpB?$AA@ 101077c4     xpcruntime:xpcimports.obj
 0002:000047cc       ??_C@_0BD@PGABEJOL@xpcInpB?5not?5found?6?$AA@ 101077cc     xpcruntime:xpcimports.obj
 0002:000047e0       ??_C@_07KIHBBOKH@xpcInpW?$AA@ 101077e0     xpcruntime:xpcimports.obj
 0002:000047e8       ??_C@_0BD@FPCJFMCC@xpcInpW?5not?5found?6?$AA@ 101077e8     xpcruntime:xpcimports.obj
 0002:000047fc       ??_C@_08KDIAJBOP@xpcInpDW?$AA@ 101077fc     xpcruntime:xpcimports.obj
 0002:00004808       ??_C@_0BE@PIELDNIL@xpcInpDW?5not?5found?6?$AA@ 10107808     xpcruntime:xpcimports.obj
 0002:0000481c       ??_C@_08PJFMOIGO@xpcOutpB?$AA@ 1010781c     xpcruntime:xpcimports.obj
 0002:00004828       ??_C@_0BE@HCKNCEKF@xpcOutpB?5not?5found?6?$AA@ 10107828     xpcruntime:xpcimports.obj
 0002:0000483c       ??_C@_08MOOJAOHK@xpcOutpW?$AA@ 1010783c     xpcruntime:xpcimports.obj
 0002:00004848       ??_C@_0BE@NLIFDBGM@xpcOutpW?5not?5found?6?$AA@ 10107848     xpcruntime:xpcimports.obj
 0002:0000485c       ??_C@_09FLIEKHJG@xpcOutpDW?$AA@ 1010785c     xpcruntime:xpcimports.obj
 0002:00004868       ??_C@_0BF@GJKLPNHB@xpcOutpDW?5not?5found?6?$AA@ 10107868     xpcruntime:xpcimports.obj
 0002:00004880       ??_C@_0BH@EHOLELHH@xpcReserveMemoryRegion?$AA@ 10107880     xpcruntime:xpcimports.obj
 0002:00004898       ??_C@_0CC@KAAAGPI@xpcReserveMemoryRegion?5not?5found@ 10107898     xpcruntime:xpcimports.obj
 0002:000048bc       ??_C@_0BA@JGPMHGAF@rl32eShowPCIDev?$AA@ 101078bc     xpcruntime:xpcimports.obj
 0002:000048cc       ??_C@_0BL@DDFFLNHI@rl32eShowPCIDev?5not?5found?6?$AA@ 101078cc     xpcruntime:xpcimports.obj
 0002:000048e8       ??_C@_0BB@KBCOJPFB@rl32eShowPCIInfo?$AA@ 101078e8     xpcruntime:xpcimports.obj
 0002:000048fc       ??_C@_0BM@IFDMAGLO@rl32eShowPCIInfo?5not?5found?6?$AA@ 101078fc     xpcruntime:xpcimports.obj
 0002:00004918       ??_C@_0BA@BGPAADB@rl32eGetPCIInfo?$AA@ 10107918     xpcruntime:xpcimports.obj
 0002:00004928       ??_C@_0BL@IGOMLDCK@rl32eGetPCIInfo?5not?5found?6?$AA@ 10107928     xpcruntime:xpcimports.obj
 0002:00004944       ??_C@_0BG@NJPFKFDP@rl32eGetPCIInfoAtSlot?$AA@ 10107944     xpcruntime:xpcimports.obj
 0002:0000495c       ??_C@_0CB@BBKIPMLA@rl32eGetPCIInfoAtSlot?5not?5found?6@ 1010795c     xpcruntime:xpcimports.obj
 0002:00004980       ??_C@_0BH@OKBOPNFG@xpceAssignPCIInterrupt?$AA@ 10107980     xpcruntime:xpcimports.obj
 0002:00004998       ??_C@_0CC@CDNDNJBJ@xpceAssignPCIInterrupt?5not?5found@ 10107998     xpcruntime:xpcimports.obj
 0002:000049bc       ??_C@_0BD@PCKOKHO@xpceGetSignalValue?$AA@ 101079bc     xpcruntime:xpcimports.obj
 0002:000049d0       ??_C@_0BO@GCBDJHMB@xpceGetSignalValue?5not?5found?6?$AA@ 101079d0     xpcruntime:xpcimports.obj
 0002:000049f0       ??_C@_0BB@BJONJAGA@xpceSetParameter?$AA@ 101079f0     xpcruntime:xpcimports.obj
 0002:00004a04       ??_C@_0BM@BJIKDLHA@xpceSetParameter?5not?5found?6?$AA@ 10107a04     xpcruntime:xpcimports.obj
 0002:00004a20       ??_C@_0BB@GNFDFMCM@xpceGetParameter?$AA@ 10107a20     xpcruntime:xpcimports.obj
 0002:00004a34       ??_C@_0BM@POHNKBC@xpceGetParameter?5not?5found?6?$AA@ 10107a34     xpcruntime:xpcimports.obj
 0002:00004a50       ??_C@_0BB@CEIJLFCD@xpceGetParamDims?$AA@ 10107a50     xpcruntime:xpcimports.obj
 0002:00004a64       ??_C@_0BM@OABDBKAO@xpceGetParamDims?5not?5found?6?$AA@ 10107a64     xpcruntime:xpcimports.obj
 0002:00004a80       ??_C@_0L@OCBLLHBM@xpceGetTET?$AA@ 10107a80     xpcruntime:xpcimports.obj
 0002:00004a8c       ??_C@_0BG@HNOFBOB@xpceGetTET?5not?5found?6?$AA@ 10107a8c     xpcruntime:xpcimports.obj
 0002:00004aa4       ??_C@_0P@OKGNGAGH@xpcIsModelInit?$AA@ 10107aa4     xpcruntime:xpcimports.obj
 0002:00004ab4       ??_C@_0BK@DHEMLBIM@xpcIsModelInit?5not?5found?6?$AA@ 10107ab4     xpcruntime:xpcimports.obj
 0002:00004ad0       ??_C@_0BH@KJJLCAOJ@xpcAllocPhysicalMemory?$AA@ 10107ad0     xpcruntime:xpcimports.obj
 0002:00004ae8       ??_C@_0CC@MOJPNHKL@xpcAllocPhysicalMemory?5not?5found@ 10107ae8     xpcruntime:xpcimports.obj
 0002:00004b0c       ??_C@_0BG@CBNPGAEL@xpcFreePhysicalMemory?$AA@ 10107b0c     xpcruntime:xpcimports.obj
 0002:00004b24       ??_C@_0CB@PKJEBPOG@xpcFreePhysicalMemory?5not?5found?6@ 10107b24     xpcruntime:xpcimports.obj
 0002:00004b48       ??_C@_0BC@JGKNLICL@xpcGetElapsedTime?$AA@ 10107b48     xpcruntime:xpcimports.obj
 0002:00004b5c       ??_C@_0BN@OEOAHCIO@xpcGetElapsedTime?5not?5found?6?$AA@ 10107b5c     xpcruntime:xpcimports.obj
 0002:00004b7c       ??_C@_0M@ICBLMODA@xpcBusyWait?$AA@ 10107b7c     xpcruntime:xpcimports.obj
 0002:00004b88       ??_C@_0BH@FBOPECBI@xpcBusyWait?5not?5found?6?$AA@ 10107b88     xpcruntime:xpcimports.obj
 0002:00004ba0       ??_C@_0N@LKKJEKKA@TBCreateSpin?$AA@ 10107ba0     xpcruntime:xpcimports.obj
 0002:00004bb0       ??_C@_0BI@FHKMLKOE@TBCreateSpin?5not?5found?6?$AA@ 10107bb0     xpcruntime:xpcimports.obj
 0002:00004bc8       ??_C@_0N@HOAJHNBD@TBDeleteSpin?$AA@ 10107bc8     xpcruntime:xpcimports.obj
 0002:00004bd8       ??_C@_0BI@BKCPAAG@TBDeleteSpin?5not?5found?6?$AA@ 10107bd8     xpcruntime:xpcimports.obj
 0002:00004bf0       ??_C@_0P@DAHDDBJG@TBTakeSpinFast?$AA@ 10107bf0     xpcruntime:xpcimports.obj
 0002:00004c00       ??_C@_0BK@NKAIBHGB@TBTakeSpinFast?5not?5found?6?$AA@ 10107c00     xpcruntime:xpcimports.obj
 0002:00004c1c       ??_C@_0P@FKNAAELA@TBGiveSpinFast?$AA@ 10107c1c     xpcruntime:xpcimports.obj
 0002:00004c2c       ??_C@_0BK@KGPJBJND@TBGiveSpinFast?5not?5found?6?$AA@ 10107c2c     xpcruntime:xpcimports.obj
 0002:00004c48       ??_C@_0BE@IIGBFDHK@xpceCreateSemaphore?$AA@ 10107c48     xpcruntime:xpcimports.obj
 0002:00004c5c       ??_C@_0BP@KFBAFFKJ@xpceCreateSemaphore?5not?5found?6?$AA@ 10107c5c     xpcruntime:xpcimports.obj
 0002:00004c7c       ??_C@_0BC@IFNIONKJ@xpceWaitSemaphore?$AA@ 10107c7c     xpcruntime:xpcimports.obj
 0002:00004c90       ??_C@_0BN@NMFAADIO@xpceWaitSemaphore?5not?5found?6?$AA@ 10107c90     xpcruntime:xpcimports.obj
 0002:00004cb0       ??_C@_0BE@NNDIOBKE@xpceSignalSemaphore?$AA@ 10107cb0     xpcruntime:xpcimports.obj
 0002:00004cc4       ??_C@_0BP@LBANMHJP@xpceSignalSemaphore?5not?5found?6?$AA@ 10107cc4     xpcruntime:xpcimports.obj
 0002:00004ce4       ??_C@_0BE@MEBEKOIM@xpceDeleteSemaphore?$AA@ 10107ce4     xpcruntime:xpcimports.obj
 0002:00004cf8       ??_C@_0BP@OFNCKOJH@xpceDeleteSemaphore?5not?5found?6?$AA@ 10107cf8     xpcruntime:xpcimports.obj
 0002:00004d18       ??_C@_0BD@MFNDMBOF@FindUsbVideoDevice?$AA@ 10107d18     xpcruntime:xpcimports.obj
 0002:00004d2c       ??_C@_0BO@POKLDHMI@FindUsbVideoDevice?5not?5found?6?$AA@ 10107d2c     xpcruntime:xpcimports.obj
 0002:00004d4c       ??_C@_0BA@PLPAPNAB@GetVideoConfigs?$AA@ 10107d4c     xpcruntime:xpcimports.obj
 0002:00004d5c       ??_C@_0BL@DALDHKHC@GetVideoConfigs?5not?5found?6?$AA@ 10107d5c     xpcruntime:xpcimports.obj
 0002:00004d78       ??_C@_0L@GBAEMHMH@StartVideo?$AA@ 10107d78     xpcruntime:xpcimports.obj
 0002:00004d84       ??_C@_0BG@HDCELEBP@StartVideo?5not?5found?6?$AA@ 10107d84     xpcruntime:xpcimports.obj
 0002:00004d9c       ??_C@_0BA@FDNPOCLN@ReadFrameBuffer?$AA@ 10107d9c     xpcruntime:xpcimports.obj
 0002:00004dac       ??_C@_0BL@JHGHPNBI@ReadFrameBuffer?5not?5found?6?$AA@ 10107dac     xpcruntime:xpcimports.obj
 0002:00004dc8       ??_C@_09FAHCLKAG@StopVideo?$AA@ 10107dc8     xpcruntime:xpcimports.obj
 0002:00004dd4       ??_C@_0BF@NKGKKADL@StopVideo?5not?5found?6?$AA@ 10107dd4     xpcruntime:xpcimports.obj
 0002:00004dec       ??_C@_0O@MCPKDLLL@ConvertUImage?$AA@ 10107dec     xpcruntime:xpcimports.obj
 0002:00004dfc       ??_C@_0BJ@PHJKOAFL@ConvertUImage?5not?5found?6?$AA@ 10107dfc     xpcruntime:xpcimports.obj
 0002:00004e18       ??_C@_0BD@NKCBPBJJ@CreateVideoDisplay?$AA@ 10107e18     xpcruntime:xpcimports.obj
 0002:00004e2c       ??_C@_0BO@HPPLLNFP@CreateVideoDisplay?5not?5found?6?$AA@ 10107e2c     xpcruntime:xpcimports.obj
 0002:00004e4c       ??_C@_0BE@KJCKGPHA@DestroyVideoDisplay?$AA@ 10107e4c     xpcruntime:xpcimports.obj
 0002:00004e60       ??_C@_0BP@FMGLJAIJ@DestroyVideoDisplay?5not?5found?6?$AA@ 10107e60     xpcruntime:xpcimports.obj
 0002:00004e80       ??_C@_0BC@HCMIMIDN@StartVideoDisplay?$AA@ 10107e80     xpcruntime:xpcimports.obj
 0002:00004e94       ??_C@_0BN@EFIEBGOO@StartVideoDisplay?5not?5found?6?$AA@ 10107e94     xpcruntime:xpcimports.obj
 0002:00004eb4       ??_C@_0BB@JBBLMILG@StopVideoDisplay?$AA@ 10107eb4     xpcruntime:xpcimports.obj
 0002:00004ec8       ??_C@_0BM@DBJBPLEL@StopVideoDisplay?5not?5found?6?$AA@ 10107ec8     xpcruntime:xpcimports.obj
 0002:00004ee4       ??_C@_0M@MFJEGMHC@StreamVideo?$AA@ 10107ee4     xpcruntime:xpcimports.obj
 0002:00004ef0       ??_C@_0BH@OINCDMLA@StreamVideo?5not?5found?6?$AA@ 10107ef0     xpcruntime:xpcimports.obj
 0002:00004f08       ??_C@_0N@IGGLCIGE@xpceaddEvent?$AA@ 10107f08     xpcruntime:xpcimports.obj
 0002:00004f18       ??_C@_0BI@NHJNFMKH@xpceaddEvent?5not?5found?6?$AA@ 10107f18     xpcruntime:xpcimports.obj
 0002:00004f30       ??_C@_0BC@MLJODBHJ@slrtStartProfiler?$AA@ 10107f30     xpcruntime:xpcimports.obj
 0002:00004f44       ??_C@_0BN@HLNCOKA@slrtStartProfiler?5not?5found?6?$AA@ 10107f44     xpcruntime:xpcimports.obj
 0002:00004f64       ??_C@_0BB@ONJONMCD@slrtStopProfiler?$AA@ 10107f64     xpcruntime:xpcimports.obj
 0002:00004f78       ??_C@_0BM@GAKJEGBA@slrtStopProfiler?5not?5found?6?$AA@ 10107f78     xpcruntime:xpcimports.obj
 0002:00004f94       ??_C@_0BF@EILBHBBF@slrtGetProfilerState?$AA@ 10107f94     xpcruntime:xpcimports.obj
 0002:00004fac       ??_C@_0CA@EDDFOCLE@slrtGetProfilerState?5not?5found?6?$AA@ 10107fac     xpcruntime:xpcimports.obj
 0002:00004fcc       ??_C@_0BB@HDPOIJAB@xpceDAQPostEvent?$AA@ 10107fcc     xpcruntime:xpcimports.obj
 0002:00004fe0       ??_C@_0BM@IHANBKGN@xpceDAQPostEvent?5not?5found?6?$AA@ 10107fe0     xpcruntime:xpcimports.obj
 0002:00004ffc       ??_C@_0BH@MBACMOD@xpceDAQUpdateTimeStamp?$AA@ 10107ffc     xpcruntime:xpcimports.obj
 0002:00005014       ??_C@_0CC@DAKBBINL@xpceDAQUpdateTimeStamp?5not?5found@ 10108014     xpcruntime:xpcimports.obj
 0002:00005038       ??_C@_0BD@HLALHPHI@slrtRegisterSignal?$AA@ 10108038     xpcruntime:xpcimports.obj
 0002:0000504c       ??_C@_0BO@BALEBHKF@slrtRegisterSignal?5not?5found?6?$AA@ 1010804c     xpcruntime:xpcimports.obj
 0002:0000506c       ??_C@_0O@DKILEOIJ@slrtLogSignal?$AA@ 1010806c     xpcruntime:xpcimports.obj
 0002:0000507c       ??_C@_0BJ@FMKKIEDD@slrtLogSignal?5not?5found?6?$AA@ 1010807c     xpcruntime:xpcimports.obj
 0002:00005098       ??_C@_0BG@CCHICKPN@slrteSetStepSizeDelta?$AA@ 10108098     xpcruntime:xpcimports.obj
 0002:000050b0       ??_C@_0CB@MKHINEIJ@slrteSetStepSizeDelta?5not?5found?6@ 101080b0     xpcruntime:xpcimports.obj
 0002:000050d4       ??_C@_0BI@CLNBLDKJ@slrteGetCurrentStepSize?$AA@ 101080d4     xpcruntime:xpcimports.obj
 0002:000050ec       ??_C@_0CD@GIOJPGJA@slrteGetCurrentStepSize?5not?5foun@ 101080ec     xpcruntime:xpcimports.obj
 0002:00005110       ??_C@_0BE@FCLCBOC@registerPTPTimeRead?$AA@ 10108110     xpcruntime:xpcimports.obj
 0002:00005124       ??_C@_0BP@LHPKAJIP@registerPTPTimeRead?5not?5found?6?$AA@ 10108124     xpcruntime:xpcimports.obj
 0002:00005144       ??_C@_0BG@KIGCDDJI@unRegisterPTPTimeRead?$AA@ 10108144     xpcruntime:xpcimports.obj
 0002:0000515c       ??_C@_0CB@MLFFBFCM@unRegisterPTPTimeRead?5not?5found?6@ 1010815c     xpcruntime:xpcimports.obj
 0002:00005180       ??_C@_0BB@IPMDDBHK@slTestInitialize?$AA@ 10108180     xpcruntime:xpcimports.obj
 0002:00005194       ??_C@_0BM@LAJFCCJH@slTestInitialize?5not?5found?6?$AA@ 10108194     xpcruntime:xpcimports.obj
 0002:000051b0       ??_C@_0BF@OOMPMEBC@slTestLogAssessments?$AA@ 101081b0     xpcruntime:xpcimports.obj
 0002:000051c8       ??_C@_0CA@FGJCEBAG@slTestLogAssessments?5not?5found?6?$AA@ 101081c8     xpcruntime:xpcimports.obj
 0002:000051e8       ??_C@_0BB@HJHKONHO@slTestEvalOnFail?$AA@ 101081e8     xpcruntime:xpcimports.obj
 0002:000051fc       ??_C@_0BM@JIKCFFNJ@slTestEvalOnFail?5not?5found?6?$AA@ 101081fc     xpcruntime:xpcimports.obj
 0002:00005218       ??_C@_0BA@LBHLABFP@slTestTerminate?$AA@ 10108218     xpcruntime:xpcimports.obj
 0002:00005228       ??_C@_0BL@EMFGKAPA@slTestTerminate?5not?5found?6?$AA@ 10108228     xpcruntime:xpcimports.obj
 0002:00005244       ??_C@_0BE@JPNPBBEO@slTestRegAssessment?$AA@ 10108244     xpcruntime:xpcimports.obj
 0002:00005258       ??_C@_0BP@FBDEJJJH@slTestRegAssessment?5not?5found?6?$AA@ 10108258     xpcruntime:xpcimports.obj
 0002:00005278       ??_C@_0O@NCLGDNIB@slrteSetupMSI?$AA@ 10108278     xpcruntime:xpcimports.obj
 0002:00005288       ??_C@_0BJ@HEFMECLM@slrteSetupMSI?5not?5found?6?$AA@ 10108288     xpcruntime:xpcimports.obj
 0002:000052a4       ??_C@_0BH@BPOLALHD@slrtGetCRBScratchSpace?$AA@ 101082a4     xpcruntime:xpcimports.obj
 0002:000052bc       ??_C@_0CC@KCKAJKKJ@slrtGetCRBScratchSpace?5not?5found@ 101082bc     xpcruntime:xpcimports.obj
 0002:000052e0       ??_C@_0BC@MKFDAKOL@slrtGetSgCRBSpace?$AA@ 101082e0     xpcruntime:xpcimports.obj
 0002:000052f4       ??_C@_0BN@JDPHPLHL@slrtGetSgCRBSpace?5not?5found?6?$AA@ 101082f4     xpcruntime:xpcimports.obj
 0002:00005314       ??_C@_0P@EPAPKLIF@slrtfsOpenFile?$AA@ 10108314     xpcruntime:xpcimports.obj
 0002:00005324       ??_C@_0BK@FIHCBOHG@slrtfsOpenFile?5not?5found?6?$AA@ 10108324     xpcruntime:xpcimports.obj
 0002:00005340       ??_C@_0BA@LILAFDDL@slrtfsCloseFile?$AA@ 10108340     xpcruntime:xpcimports.obj
 0002:00005350       ??_C@_0BL@DEGHJFIB@slrtfsCloseFile?5not?5found?6?$AA@ 10108350     xpcruntime:xpcimports.obj
 0002:0000536c       ??_C@_0BC@OKMJDIEH@slrtfsWriteToFile?$AA@ 1010836c     xpcruntime:xpcimports.obj
 0002:00005380       ??_C@_0BN@KCFLCLAH@slrtfsWriteToFile?5not?5found?6?$AA@ 10108380     xpcruntime:xpcimports.obj
 0002:000053a0       ??_C@_0BK@GIPNFFFF@slrtfsGetFileErrorMessage?$AA@ 101083a0     xpcruntime:xpcimports.obj
 0002:000053bc       ??_C@_0CF@BCBLMKLE@slrtfsGetFileErrorMessage?5not?5fo@ 101083bc     xpcruntime:xpcimports.obj
 0002:000053e4       ??_C@_0BD@ICBOKMK@slrtfsGetFileError?$AA@ 101083e4     xpcruntime:xpcimports.obj
 0002:000053f8       ??_C@_0BO@FNBANAE@slrtfsGetFileError?5not?5found?6?$AA@ 101083f8     xpcruntime:xpcimports.obj
 0002:00005418       ??_C@_0BE@PPAJMHJP@slrtfsOpenFileAsync?$AA@ 10108418     xpcruntime:xpcimports.obj
 0002:0000542c       ??_C@_0BP@HKBMMJOK@slrtfsOpenFileAsync?5not?5found?6?$AA@ 1010842c     xpcruntime:xpcimports.obj
 0002:0000544c       ??_C@_0BF@IGNDIBPF@slrtfsCloseFileAsync?$AA@ 1010844c     xpcruntime:xpcimports.obj
 0002:00005464       ??_C@_0CA@GJPFDBKN@slrtfsCloseFileAsync?5not?5found?6?$AA@ 10108464     xpcruntime:xpcimports.obj
 0002:00005484       ??_C@_0BE@IOLEBNB@slrtfsGetFileStatus?$AA@ 10108484     xpcruntime:xpcimports.obj
 0002:00005498       ??_C@_0BP@PEFHDGHL@slrtfsGetFileStatus?5not?5found?6?$AA@ 10108498     xpcruntime:xpcimports.obj
 0002:000054b8       ??_C@_0M@HKIJIMG@slrtfsFread?$AA@ 101084b8     xpcruntime:xpcimports.obj
 0002:000054c4       ??_C@_0BH@OOKBGONO@slrtfsFread?5not?5found?6?$AA@ 101084c4     xpcruntime:xpcimports.obj
 0002:000054dc       ??_C@_0BE@OGCMPLAP@slrtGetDefaultDrive?$AA@ 101084dc     xpcruntime:xpcimports.obj
 0002:000054f0       ??_C@_0BP@HKFGLHOE@slrtGetDefaultDrive?5not?5found?6?$AA@ 101084f0     xpcruntime:xpcimports.obj
 0002:00005510       ??_C@_0N@NAJIKFFI@slrtLogEvent?$AA@ 10108510     xpcruntime:xpcimports.obj
 0002:00005520       ??_C@_0BI@NKCEACND@slrtLogEvent?5not?5found?6?$AA@ 10108520     xpcruntime:xpcimports.obj
 0002:00005538       ??_C@_0N@IDKFJOHI@getlasterror?$AA@ 10108538     xpcruntime:xpcimports.obj
 0002:00005548       ??_C@_0BI@MIHMCHGL@getlasterror?5not?5found?6?$AA@ 10108548     xpcruntime:xpcimports.obj
 0002:00005560       ??_C@_0P@OKHGKJKN@geterrorstring?$AA@ 10108560     xpcruntime:xpcimports.obj
 0002:00005570       ??_C@_0BK@NOHFDMLP@geterrorstring?5not?5found?6?$AA@ 10108570     xpcruntime:xpcimports.obj
 0002:0000558c       ??_C@_0BD@HNFFKMGJ@slrtGetCPUTCelsius?$AA@ 1010858c     xpcruntime:xpcimports.obj
 0002:000055a0       ??_C@_0BO@LHBFKLIH@slrtGetCPUTCelsius?5not?5found?6?$AA@ 101085a0     xpcruntime:xpcimports.obj
 0002:000055c0       ??_C@_0M@OONCNCLM@slrtWarning?$AA@ 101085c0     xpcruntime:xpcimports.obj
 0002:000055cc       ??_C@_0BH@ICKGIEMB@slrtWarning?5not?5found?6?$AA@ 101085cc     xpcruntime:xpcimports.obj
 0002:000055e4       ??_C@_0M@JACEPOPN@registerNIC?$AA@ 101085e4     xpcruntime:xpcimports.obj
 0002:000055f0       ??_C@_0BH@JMDHJIAC@registerNIC?5not?5found?6?$AA@ 101085f0     xpcruntime:xpcimports.obj
 0002:00005608       ??_C@_0M@KBKHECFH@NICSetIface?$AA@ 10108608     xpcruntime:xpcimports.obj
 0002:00005614       ??_C@_0BH@NJAHOBA@NICSetIface?5not?5found?6?$AA@ 10108614     xpcruntime:xpcimports.obj
 0002:0000562c       ??_C@_0M@FAILFBCK@NICGetIface?$AA@ 1010862c     xpcruntime:xpcimports.obj
 0002:00005638       ??_C@_0BH@KDLLDOGM@NICGetIface?5not?5found?6?$AA@ 10108638     xpcruntime:xpcimports.obj
 0002:00005650       ??_C@_0L@JNFPDPO@releaseNIC?$AA@ 10108650     xpcruntime:xpcimports.obj
 0002:0000565c       ??_C@_0BG@EBGJANLA@releaseNIC?5not?5found?6?$AA@ 1010865c     xpcruntime:xpcimports.obj
 0002:00005674       ??_C@_0BC@HLDKJAG@SetIPTASKPriority?$AA@ 10108674     xpcruntime:xpcimports.obj
 0002:00005688       ??_C@_0BN@OGKMHHAE@SetIPTASKPriority?5not?5found?6?$AA@ 10108688     xpcruntime:xpcimports.obj
 0002:000056a8       ??_C@_0O@LHENMBDD@OpenInterface?$AA@ 101086a8     xpcruntime:xpcimports.obj
 0002:000056b8       ??_C@_0BJ@PFGDBKHB@OpenInterface?5not?5found?6?$AA@ 101086b8     xpcruntime:xpcimports.obj
 0002:000056d4       ??_C@_0P@IINFELKD@CloseInterface?$AA@ 101086d4     xpcruntime:xpcimports.obj
 0002:000056e4       ??_C@_0BK@PAPDNDBK@CloseInterface?5not?5found?6?$AA@ 101086e4     xpcruntime:xpcimports.obj
 0002:00005700       ??_C@_05LEFIAAOI@SetIP?$AA@ 10108700     xpcruntime:xpcimports.obj
 0002:00005708       ??_C@_0BB@CGLIBAMM@SetIP?5not?5found?6?$AA@ 10108708     xpcruntime:xpcimports.obj
 0002:0000571c       ??_C@_0BA@HIJJHHMD@AddGatewayRoute?$AA@ 1010871c     xpcruntime:xpcimports.obj
 0002:0000572c       ??_C@_0BL@BFCFMDMN@AddGatewayRoute?5not?5found?6?$AA@ 1010872c     xpcruntime:xpcimports.obj
 0002:00005748       ??_C@_0BC@OGIEOMEH@AddMulticastRoute?$AA@ 10108748     xpcruntime:xpcimports.obj
 0002:0000575c       ??_C@_0BN@IMNDPFCL@AddMulticastRoute?5not?5found?6?$AA@ 1010875c     xpcruntime:xpcimports.obj
 0002:0000577c       ??_C@_0M@PHMABFPI@DeleteRoute?$AA@ 1010877c     xpcruntime:xpcimports.obj
 0002:00005788       ??_C@_0BH@JPJGLLID@DeleteRoute?5not?5found?6?$AA@ 10108788     xpcruntime:xpcimports.obj
 0002:000057a0       ??_C@_0BA@FCDIMKIJ@GetHostTarIPAdd?$AA@ 101087a0     xpcruntime:xpcimports.obj
 0002:000057b0       ??_C@_0BL@MBKDGKBO@GetHostTarIPAdd?5not?5found?6?$AA@ 101087b0     xpcruntime:xpcimports.obj
 0002:000057cc       ??_C@_0M@HPMIPIBI@GetDCUUsage?$AA@ 101087cc     xpcruntime:xpcimports.obj
 0002:000057d8       ??_C@_0BH@EBLJKCJC@GetDCUUsage?5not?5found?6?$AA@ 101087d8     xpcruntime:xpcimports.obj
 0002:000057f0       ??_C@_06MPKMECK@accept?$AA@ 101087f0     xpcruntime:xpcimports.obj
 0002:000057f8       ??_C@_0BC@GBGIEMNO@accept?5not?5found?6?$AA@ 101087f8     xpcruntime:xpcimports.obj
 0002:0000580c       ??_C@_04NPNJNMMP@bind?$AA@ 1010880c     xpcruntime:xpcimports.obj
 0002:00005814       ??_C@_0BA@DAJNENLO@bind?5not?5found?6?$AA@ 10108814     xpcruntime:xpcimports.obj
 0002:00005824       ??_C@_0L@CKHNIFCM@setsockopt?$AA@ 10108824     xpcruntime:xpcimports.obj
 0002:00005830       ??_C@_0BG@MFIIOMFE@setsockopt?5not?5found?6?$AA@ 10108830     xpcruntime:xpcimports.obj
 0002:00005848       ??_C@_0M@ODDJDCDK@closesocket?$AA@ 10108848     xpcruntime:xpcimports.obj
 0002:00005854       ??_C@_0BH@JHGHMIL@closesocket?5not?5found?6?$AA@ 10108854     xpcruntime:xpcimports.obj
 0002:0000586c       ??_C@_07KAIBNCHO@connect?$AA@ 1010886c     xpcruntime:xpcimports.obj
 0002:00005874       ??_C@_0BD@MKLLMBM@connect?5not?5found?6?$AA@ 10108874     xpcruntime:xpcimports.obj
 0002:00005888       ??_C@_0M@PBPOCKDG@ioctlsocket?$AA@ 10108888     xpcruntime:xpcimports.obj
 0002:00005894       ??_C@_0BH@NFCNHHIH@ioctlsocket?5not?5found?6?$AA@ 10108894     xpcruntime:xpcimports.obj
 0002:000058ac       ??_C@_06OODDLKLE@listen?$AA@ 101088ac     xpcruntime:xpcimports.obj
 0002:000058b4       ??_C@_0BC@NHBILEKI@listen?5not?5found?6?$AA@ 101088b4     xpcruntime:xpcimports.obj
 0002:000058c8       ??_C@_08HMBBGFHE@recvfrom?$AA@ 101088c8     xpcruntime:xpcimports.obj
 0002:000058d4       ??_C@_0BE@BJAJFFLF@recvfrom?5not?5found?6?$AA@ 101088d4     xpcruntime:xpcimports.obj
 0002:000058e8       ??_C@_06MEPBGKEC@sendto?$AA@ 101088e8     xpcruntime:xpcimports.obj
 0002:000058f0       ??_C@_0BC@BHPIMDJO@sendto?5not?5found?6?$AA@ 101088f0     xpcruntime:xpcimports.obj
 0002:00005904       ??_C@_09JKBDEEOB@inet_addr?$AA@ 10108904     xpcruntime:xpcimports.obj
 0002:00005910       ??_C@_0BF@HKJPGECN@inet_addr?5not?5found?6?$AA@ 10108910     xpcruntime:xpcimports.obj
 0002:00005928       ??_C@_06HBELJPBO@socket?$AA@ 10108928     xpcruntime:xpcimports.obj
 0002:00005930       ??_C@_0BC@NAGFFJGA@socket?5not?5found?6?$AA@ 10108930     xpcruntime:xpcimports.obj
 0002:00005944       ??_C@_09ICJIFGNC@GetSocket?$AA@ 10108944     xpcruntime:xpcimports.obj
 0002:00005950       ??_C@_0BF@KDBCKMOJ@GetSocket?5not?5found?6?$AA@ 10108950     xpcruntime:xpcimports.obj
 0002:00005968       ??_C@_0P@KJEGJMJI@GetSocketState?$AA@ 10108968     xpcruntime:xpcimports.obj
 0002:00005978       ??_C@_0BK@IALBJHEB@GetSocketState?5not?5found?6?$AA@ 10108978     xpcruntime:xpcimports.obj
 0002:00005994       ??_C@_0L@MEAJHNHB@SocketSend?$AA@ 10108994     xpcruntime:xpcimports.obj
 0002:000059a0       ??_C@_0BG@EOCMBFJA@SocketSend?5not?5found?6?$AA@ 101089a0     xpcruntime:xpcimports.obj
 0002:000059b8       ??_C@_0O@PFPCLEMF@SocketReceive?$AA@ 101089b8     xpcruntime:xpcimports.obj
 0002:000059c8       ??_C@_0BJ@HIBADDFO@SocketReceive?5not?5found?6?$AA@ 101089c8     xpcruntime:xpcimports.obj
 0002:000059e4       ??_C@_0BD@OOGFNAIK@CreateServerSocket?$AA@ 101089e4     xpcruntime:xpcimports.obj
 0002:000059f8       ??_C@_0BO@GKIJHIPH@CreateServerSocket?5not?5found?6?$AA@ 101089f8     xpcruntime:xpcimports.obj
 0002:00005a18       ??_C@_0BB@KGHJGFFO@OpenServerListen?$AA@ 10108a18     xpcruntime:xpcimports.obj
 0002:00005a2c       ??_C@_0BM@NFMMLIO@OpenServerListen?5not?5found?6?$AA@ 10108a2c     xpcruntime:xpcimports.obj
 0002:00005a48       ??_C@_0BE@BAJLDJAH@ConnectServerSocket?$AA@ 10108a48     xpcruntime:xpcimports.obj
 0002:00005a5c       ??_C@_0BP@KJNODIKE@ConnectServerSocket?5not?5found?6?$AA@ 10108a5c     xpcruntime:xpcimports.obj
 0002:00005a7c       ??_C@_0BC@PLKKJDIM@CloseServerSocket?$AA@ 10108a7c     xpcruntime:xpcimports.obj
 0002:00005a90       ??_C@_0BN@KEJEPNMB@CloseServerSocket?5not?5found?6?$AA@ 10108a90     xpcruntime:xpcimports.obj
 0002:00005ab0       ??_C@_0BC@IHMNIGFJ@ResetServerSocket?$AA@ 10108ab0     xpcruntime:xpcimports.obj
 0002:00005ac4       ??_C@_0BN@NIOGJLCG@ResetServerSocket?5not?5found?6?$AA@ 10108ac4     xpcruntime:xpcimports.obj
 0002:00005ae4       ??_C@_0BD@MCLPKCPP@CreateClientSocket?$AA@ 10108ae4     xpcruntime:xpcimports.obj
 0002:00005af8       ??_C@_0BO@DILAGPFN@CreateClientSocket?5not?5found?6?$AA@ 10108af8     xpcruntime:xpcimports.obj
 0002:00005b18       ??_C@_0BB@DAPKNNLG@BindClientSocket?$AA@ 10108b18     xpcruntime:xpcimports.obj
 0002:00005b2c       ??_C@_0BM@LLLMMDFN@BindClientSocket?5not?5found?6?$AA@ 10108b2c     xpcruntime:xpcimports.obj
 0002:00005b48       ??_C@_0BE@DMEBELHC@ConnectClientSocket?$AA@ 10108b48     xpcruntime:xpcimports.obj
 0002:00005b5c       ??_C@_0BP@PLOHCPAO@ConnectClientSocket?5not?5found?6?$AA@ 10108b5c     xpcruntime:xpcimports.obj
 0002:00005b7c       ??_C@_0BC@NHHAOBPJ@CloseClientSocket?$AA@ 10108b7c     xpcruntime:xpcimports.obj
 0002:00005b90       ??_C@_0BN@PGKNOKGL@CloseClientSocket?5not?5found?6?$AA@ 10108b90     xpcruntime:xpcimports.obj
 0002:00005bb0       ??_C@_0BC@KLBHPECM@ResetClientSocket?$AA@ 10108bb0     xpcruntime:xpcimports.obj
 0002:00005bc4       ??_C@_0BN@IKNPIMIM@ResetClientSocket?5not?5found?6?$AA@ 10108bc4     xpcruntime:xpcimports.obj
 0002:00005be4       ??_C@_0M@IJOPFCCE@UDPOpenSend?$AA@ 10108be4     xpcruntime:xpcimports.obj
 0002:00005bf0       ??_C@_0BH@CCHBDPG@UDPOpenSend?5not?5found?6?$AA@ 10108bf0     xpcruntime:xpcimports.obj
 0002:00005c08       ??_C@_0P@MEPACHPD@UDPOpenReceive?$AA@ 10108c08     xpcruntime:xpcimports.obj
 0002:00005c18       ??_C@_0BK@PFMCPKIO@UDPOpenReceive?5not?5found?6?$AA@ 10108c18     xpcruntime:xpcimports.obj
 0002:00005c34       ??_C@_0BK@BGNLEHGA@UDPAddMulticastMembership?$AA@ 10108c34     xpcruntime:xpcimports.obj
 0002:00005c50       ??_C@_0CF@CAEMAELE@UDPAddMulticastMembership?5not?5fo@ 10108c50     xpcruntime:xpcimports.obj
 0002:00005c78       ??_C@_0N@NMMOLOEM@UDPCloseSend?$AA@ 10108c78     xpcruntime:xpcimports.obj
 0002:00005c88       ??_C@_0BI@ENKCOCDG@UDPCloseSend?5not?5found?6?$AA@ 10108c88     xpcruntime:xpcimports.obj
 0002:00005ca0       ??_C@_0BA@DMJGBBIA@UDPCloseReceive?$AA@ 10108ca0     xpcruntime:xpcimports.obj
 0002:00005cb0       ??_C@_0BL@PEBIMLNC@UDPCloseReceive?5not?5found?6?$AA@ 10108cb0     xpcruntime:xpcimports.obj
 0002:00005ccc       ??_C@_0P@NPOCJKPL@registerDFTask?$AA@ 10108ccc     xpcruntime:xpcimports.obj
 0002:00005cdc       ??_C@_0BK@JHOOFMMI@registerDFTask?5not?5found?6?$AA@ 10108cdc     xpcruntime:xpcimports.obj
 0002:00005cf8       ??_C@_0BB@ICCLEIPB@deregisterDFTask?$AA@ 10108cf8     xpcruntime:xpcimports.obj
 0002:00005d0c       ??_C@_0BM@PEOCAIDM@deregisterDFTask?5not?5found?6?$AA@ 10108d0c     xpcruntime:xpcimports.obj
 0002:00005d28       ??_C@_0O@PHHDMOJH@triggerDFTask?$AA@ 10108d28     xpcruntime:xpcimports.obj
 0002:00005d38       ??_C@_0BJ@IKKCFBJL@triggerDFTask?5not?5found?6?$AA@ 10108d38     xpcruntime:xpcimports.obj
 0002:00005d54       ??_C@_0O@IAHKGBOC@waitForDFTask?$AA@ 10108d54     xpcruntime:xpcimports.obj
 0002:00005d64       ??_C@_0BJ@FHLCNAKE@waitForDFTask?5not?5found?6?$AA@ 10108d64     xpcruntime:xpcimports.obj
 0002:00005d84       ??_7error_category@std@@6B@ 10108d84     IO61X_Library_MSVC120_vc:IO61X_iConcurrentExecution.obj
 0002:00005da0       ??_7_Generic_error_category@std@@6B@ 10108da0     IO61X_Library_MSVC120_vc:IO61X_iConcurrentExecution.obj
 0002:00005db8       ??_C@_07DCLBNMLN@generic?$AA@ 10108db8     IO61X_Library_MSVC120_vc:IO61X_iConcurrentExecution.obj
 0002:00005dc0       ??_C@_0O@BFJCFAAK@unknown?5error?$AA@ 10108dc0     IO61X_Library_MSVC120_vc:IO61X_iConcurrentExecution.obj
 0002:00005dd4       ??_7_Iostream_error_category@std@@6B@ 10108dd4     IO61X_Library_MSVC120_vc:IO61X_iConcurrentExecution.obj
 0002:00005dec       ??_C@_08LLGCOLLL@iostream?$AA@ 10108dec     IO61X_Library_MSVC120_vc:IO61X_iConcurrentExecution.obj
 0002:00005df8       ??_C@_0BG@PADBLCHM@iostream?5stream?5error?$AA@ 10108df8     IO61X_Library_MSVC120_vc:IO61X_iConcurrentExecution.obj
 0002:00005e14       ??_7_System_error_category@std@@6B@ 10108e14     IO61X_Library_MSVC120_vc:IO61X_iConcurrentExecution.obj
 0002:00005e2c       ??_C@_06FHFOAHML@system?$AA@ 10108e2c     IO61X_Library_MSVC120_vc:IO61X_iConcurrentExecution.obj
 0002:00005e34       ??_C@_0CO@HPPJBJJP@IO61X?3?5Stop?5init?3?5Create?5module?5@ 10108e34     IO61X_Library_MSVC120_vc:IO61X_iConcurrentExecution.obj
 0002:00005e64       ??_C@_05IKHNOFAI@IO611?$AA@ 10108e64     IO61X_Library_MSVC120_vc:IO61X_iConcurrentExecution.obj
 0002:00005e6c       ??_C@_09CGAELICL@Speedgoat?$AA@ 10108e6c     IO61X_Library_MSVC120_vc:IO61X_iConcurrentExecution.obj
 0002:00005e78       ??_C@_0CO@FBEPDOL@?$CFs?5IO611?3?5CAN?9Module?5?$CICAN?9HS?1LS?0@ 10108e78     IO61X_Library_MSVC120_vc:IO61X_iConcurrentExecution.obj
 0002:00005ea8       ??_C@_05KBFALGML@IO612?$AA@ 10108ea8     IO61X_Library_MSVC120_vc:IO61X_iConcurrentExecution.obj
 0002:00005eb0       ??_C@_0BO@LGELLPDA@?$CFs?5IO612?3?5CAN?9Module?5?$CICAN?9HS?$CJ?$AA@ 10108eb0     IO61X_Library_MSVC120_vc:IO61X_iConcurrentExecution.obj
 0002:00005ed0       ??_C@_05LIELIHIK@IO613?$AA@ 10108ed0     IO61X_Library_MSVC120_vc:IO61X_iConcurrentExecution.obj
 0002:00005ed8       ??_C@_0CG@HBAEMGF@?$CFs?5IO613?3?5CAN?9Module?5?$CICAN?9HS?0?5CA@ 10108ed8     IO61X_Library_MSVC120_vc:IO61X_iConcurrentExecution.obj
 0002:00005f00       ??_C@_05PHAKBBEN@IO614?$AA@ 10108f00     IO61X_Library_MSVC120_vc:IO61X_iConcurrentExecution.obj
 0002:00005f08       ??_C@_0CG@CLEFKGLI@?$CFs?5IO614?3?5CAN?9Module?5?$CICAN?9HS?1LS?0@ 10108f08     IO61X_Library_MSVC120_vc:IO61X_iConcurrentExecution.obj
 0002:00005f30       ??_C@_0N@KDLPGNFM@Protocol?3?5?$CFs?$AA@ 10108f30     IO61X_Library_MSVC120_vc:IO61X_iConcurrentExecution.obj
 0002:00005f40       ??_C@_02NBHMGPMG@SG?$AA@   10108f40     IO61X_Library_MSVC120_vc:IO61X_iConcurrentExecution.obj
 0002:00005f44       ??_C@_0CI@LCHIHHMB@?$CFs?5?$CFs?0?5ModuleID?5?$CFi?3?5PCI?5auto?9sea@ 10108f44     IO61X_Library_MSVC120_vc:IO61X_iConcurrentExecution.obj
 0002:00005f6c       ??_C@_0CG@MLFAEPCL@?$CFs?5?$CFs?0?5ModuleID?5?$CFi?3?5PCI?5?$DN?5?$FL?$CFi?5?$CFi@ 10108f6c     IO61X_Library_MSVC120_vc:IO61X_iConcurrentExecution.obj
 0002:00005f98       ??_C@_0EG@EBENGAJE@Initialization?5of?5the?5module?5cha@ 10108f98     IO61X_Library_MSVC120_vc:IO61X_iConcurrentExecution.obj
 0002:00005fe0       ??_C@_0FP@GCJDODBN@?$CFs?0?5ModuleID?5?$CFi?3?5Stop?5initializa@ 10108fe0     IO61X_Library_MSVC120_vc:IO61X_iConcurrentExecution.obj
 0002:00006040       ??_C@_0DJ@LOHGNCMC@?5Midx?5?$CFi?5module?5status?3?5?$CFi?5?5?9?5?$CI2@ 10109040     IO61X_Library_MSVC120_vc:IO61X_iConcurrentExecution.obj
 0002:0000607c       ??_C@_0DK@PKLDLFEJ@?5Midx?5?$CFi?5module?5status?3?5?$CFi?5?5?9?5?$CI2@ 1010907c     IO61X_Library_MSVC120_vc:IO61X_iConcurrentExecution.obj
 0002:000060b8       ??_C@_0CM@POKEONFH@?5Midx?5?$CFi?5module?5status?3?5?$CFi?5?5?9?5?$CI0@ 101090b8     IO61X_Library_MSVC120_vc:IO61X_iConcurrentExecution.obj
 0002:000060e8       ??_C@_0FG@BEHOJACO@?$CFs?5?$CFs?0?5ModuleID?5?$CFi?3?5Stop?5initial@ 101090e8     IO61X_Library_MSVC120_vc:IO61X_iConcurrentExecution.obj
 0002:00006140       ??_C@_0FB@IJAHJJML@?$CFs?5?$CFs?0?5ModuleID?5?$CFi?3?5Stop?5initial@ 10109140     IO61X_Library_MSVC120_vc:IO61X_iConcurrentExecution.obj
 0002:00006198       ??_C@_0FO@KLDFAJDM@?$CFs?5?$CFs?0?5ModuleID?5?$CFi?3?5Ch?3?5?$CFi?0?5CAN?9@ 10109198     IO61X_Library_MSVC120_vc:IO61X_iConcurrentExecution.obj
 0002:000061f8       ??_C@_0FJ@NEMKGECH@?$CFs?5?$CFs?0?5ModuleID?5?$CFi?3?5Stop?5initial@ 101091f8     IO61X_Library_MSVC120_vc:IO61X_iConcurrentExecution.obj
 0002:00006258       ??_C@_0FM@EIKMFGMH@?$CFs?5?$CFs?0?5ModuleID?5?$CFi?3?5Stop?5initial@ 10109258     IO61X_Library_MSVC120_vc:IO61X_iConcurrentExecution.obj
 0002:000062b4       ??_C@_0CJ@KCCCMIE@?5CAN?5controller?5of?5channel?5?$CFi?5is@ 101092b4     IO61X_Library_MSVC120_vc:IO61X_iConcurrentExecution.obj
 0002:000062e0       ??_C@_0DH@HHLJPGIF@?5CAN?5controller?5of?5channel?5?$CFi?5ha@ 101092e0     IO61X_Library_MSVC120_vc:IO61X_iConcurrentExecution.obj
 0002:00006318       ??_C@_0FB@FDPDMBNC@?$CFs?5?$CFs?0?5ModuleID?5?$CFi?3?5Ch?3?5?$CFi?0?5CAN?5@ 10109318     IO61X_Library_MSVC120_vc:IO61X_iConcurrentExecution.obj
 0002:00006370       ??_C@_0FJ@OCKFCHGI@?$CFs?5?$CFs?0?5ModuleID?5?$CFi?3?5Stop?5initial@ 10109370     IO61X_Library_MSVC120_vc:IO61X_iConcurrentExecution.obj
 0002:000063d0       ??_C@_0FM@DFDDPMAD@?$CFs?5?$CFs?0?5ModuleID?5?$CFi?3?5Stop?5initial@ 101093d0     IO61X_Library_MSVC120_vc:IO61X_iConcurrentExecution.obj
 0002:0000642c       ??_C@_0BM@IHNLLKI@?5LIN?5channel?5?$CFi?5is?5started?4?$AA@ 1010942c     IO61X_Library_MSVC120_vc:IO61X_iConcurrentExecution.obj
 0002:00006448       ??_C@_0FD@BPHCCJKC@?$CFs?5?$CFs?0?5ModuleID?5?$CFi?3?5Stop?5initial@ 10109448     IO61X_Library_MSVC120_vc:IO61X_iConcurrentExecution.obj
 0002:0000649c       ??_C@_0CL@CPEFIKHH@ReadCanMessage?5midx?$DN?$CFi?5pidx?$DN?$CFi?5r@ 1010949c     IO61X_Library_MSVC120_vc:IO61X_iConcurrentExecution.obj
 0002:000064c8       ??_C@_0BF@JHDCKNLK@?5read?5msg?5has?5dlc?$DN?$CFi?$AA@ 101094c8     IO61X_Library_MSVC120_vc:IO61X_iConcurrentExecution.obj
 0002:000064e0       ??_C@_0CN@ODKIBECA@ReadCanFdMessage?5midx?$DN?$CFi?5pidx?$DN?$CFi@ 101094e0     IO61X_Library_MSVC120_vc:IO61X_iConcurrentExecution.obj
 0002:00006510       ??_C@_0CO@NPJNMNEG@?5ReadCanFdMessage?5midx?$DN?$CFi?5pidx?$DN?$CF@ 10109510     IO61X_Library_MSVC120_vc:IO61X_iConcurrentExecution.obj
 0002:00006540       ??_C@_0FJ@EOHNBDEK@?$CFs?5?$CFs?0?5ModuleID?5?$CFi?3?5Stop?5initial@ 10109540     IO61X_Library_MSVC120_vc:IO61X_iConcurrentExecution.obj
 0002:0000659c       ??_C@_0BH@KFNADDDE@?5Is?5CAN?9FD?5channel?3?5?$CFi?$AA@ 1010959c     IO61X_Library_MSVC120_vc:IO61X_iConcurrentExecution.obj
 0002:000065b8       ??_C@_0FM@KDOHGIFN@?$CFs?5?$CFs?0?5ModuleID?5?$CFi?3?5Stop?5initial@ 101095b8     IO61X_Library_MSVC120_vc:IO61X_iConcurrentExecution.obj
 0002:00006618       ??_C@_0GD@CNGPFPIB@?$CFs?5?$CFs?0?5ModuleID?5?$CFi?3?5Stop?5initial@ 10109618     IO61X_Library_MSVC120_vc:IO61X_iConcurrentExecution.obj
 0002:00006680       ??_C@_0FJ@HIBCFAAF@?$CFs?5?$CFs?0?5ModuleID?5?$CFi?3?5Stop?5initial@ 10109680     IO61X_Library_MSVC120_vc:IO61X_iConcurrentExecution.obj
 0002:000066e0       ??_C@_0FM@NOHIMCJJ@?$CFs?5?$CFs?0?5ModuleID?5?$CFi?3?5Stop?5initial@ 101096e0     IO61X_Library_MSVC120_vc:IO61X_iConcurrentExecution.obj
 0002:00006740       ??_C@_0FO@IIIPINHB@?$CFs?5?$CFs?0?5ModuleID?5?$CFi?3?5Ch?3?5?$CFi?0?5LIN?5@ 10109740     IO61X_Library_MSVC120_vc:IO61X_iConcurrentExecution.obj
 0002:000067a0       ??_C@_0EE@JEPGAOEK@?$CFs?5?$CFs?0?5ModuleID?5?$CFi?3?5Ch?3?5?$CFi?0?5LIN?5@ 101097a0     IO61X_Library_MSVC120_vc:IO61X_iConcurrentExecution.obj
 0002:000067e8       ??_C@_0EJ@EDMHPHMF@?$CFs?5?$CFs?0?5ModuleID?5?$CFi?3?5Ch?3?5?$CFi?0?5LIN?5@ 101097e8     IO61X_Library_MSVC120_vc:IO61X_iConcurrentExecution.obj
 0002:00006838       ??_C@_0FF@GFDAIAPK@?$CFs?5?$CFs?0?5ModuleID?5?$CFi?3?5Stop?5initial@ 10109838     IO61X_Library_MSVC120_vc:IO61X_iConcurrentExecution.obj
 0002:00006890       ??_C@_0CD@OJPGODOF@Delete?5sender?5class?5of?5channel?3?5@ 10109890     IO61X_Library_MSVC120_vc:IO61X_iConcurrentExecution.obj
 0002:000068b4       ??_C@_0BM@GICLOAFC@pPort?$FL?$CFi?$FN?5after?5cleanup?3?5?$CFp?$AA@ 101098b4     IO61X_Library_MSVC120_vc:IO61X_iConcurrentExecution.obj
 0002:000068d0       ??_C@_0FF@JDOMCIP@?$CFs?5?$CFs?0?5ModuleID?5?$CFi?3?5Ch?3?5?$CFi?0?5CAN?5@ 101098d0     IO61X_Library_MSVC120_vc:IO61X_iConcurrentExecution.obj
 0002:00006928       ??_C@_0EB@IKNOLOPM@update?5buffer?5for?5modIdx?3?5?$CFi?5?9?5c@ 10109928     IO61X_Library_MSVC120_vc:IO61X_iConcurrentExecution.obj
 0002:0000696c       ??_C@_0CK@DADHBNDG@?5Update?5slave?5RWWB?5buffer?5with?5P@ 1010996c     IO61X_Library_MSVC120_vc:IO61X_iConcurrentExecution.obj
 0002:00006998       ??_C@_0CL@NICGPKGN@?5Update?5master?5RWWB?5buffer?5with?5@ 10109998     IO61X_Library_MSVC120_vc:IO61X_iConcurrentExecution.obj
 0002:000069c4       ??_C@_0DL@IECNHDBJ@?5mIdx?3?$CFi?5Activate?5status?5handlin@ 101099c4     IO61X_Library_MSVC120_vc:IO61X_iConcurrentExecution.obj
 0002:00006a00       ??_C@_0FE@BOLCOBEE@?$CFs?5?$CFs?0?5ModuleID?5?$CFi?3?5Stop?5initial@ 10109a00     IO61X_Library_MSVC120_vc:IO61X_iConcurrentExecution.obj
 0002:00006a54       ??_C@_0BM@PKFIHHDK@?$CFs?0?5create?5semaphore?5failed?$AA@ 10109a54     IO61X_Library_MSVC120_vc:IO61X_iConcurrentExecution.obj
 0002:00006a70       ??_C@_0BJ@BIIBHAJE@?$CFs?0?5create?5thread?5failed?$AA@ 10109a70     IO61X_Library_MSVC120_vc:IO61X_iConcurrentExecution.obj
 0002:00006a8c       ??_C@_0BJ@LBNIPIGG@?5Send?5status?5request?5LIN?$AA@ 10109a8c     IO61X_Library_MSVC120_vc:IO61X_iConcurrentExecution.obj
 0002:00006aa8       ??_C@_0BJ@KLDGNNBO@?5Receive?5status?5response?$AA@ 10109aa8     IO61X_Library_MSVC120_vc:IO61X_iConcurrentExecution.obj
 0002:00006ac4       ??_C@_0BH@GMGPOEOE@?5Status?5success?5?9?5?$CI?$CFi?$CJ?$AA@ 10109ac4     IO61X_Library_MSVC120_vc:IO61X_iConcurrentExecution.obj
 0002:00006adc       ??_C@_0BO@JODEOEC@?5Status?5?9?$DO?5Mode?3?5?$CFi?5?5?9?9?5?5?$CI?$CFi?$CJ?$AA@ 10109adc     IO61X_Library_MSVC120_vc:IO61X_iConcurrentExecution.obj
 0002:00006afc       ??_C@_0BN@NPAGNFID@?5Status?5?9?$DO?5BRP?3?5?$CFi?5?5?9?9?5?5?$CI?$CFi?$CJ?$AA@ 10109afc     IO61X_Library_MSVC120_vc:IO61X_iConcurrentExecution.obj
 0002:00006b1c       ??_C@_01EEMJAFIK@?6?$AA@   10109b1c     IO61X_Library_MSVC120_vc:IO61X_iConcurrentExecution.obj
 0002:00006b20       ??_C@_0BA@JFNIOLAK@string?5too?5long?$AA@ 10109b20     IO61X_Library_MSVC120_vc:IO61X_iConcurrentExecution.obj
 0002:00006b30       ??_C@_0BI@CFPLBAOH@invalid?5string?5position?$AA@ 10109b30     IO61X_Library_MSVC120_vc:IO61X_iConcurrentExecution.obj
 0002:00006b48       ??_C@_0CN@IBMHLJIN@Create?5global?5sender?5semaphore?5f@ 10109b48     IO61X_Library_MSVC120_vc:IO61X_GlobalSender.obj
 0002:00006b78       ??_C@_0EK@OABNKIO@?$CFs?5?$CFs?0?5ModuleID?5?$CFi?3?5?6Create?5send@ 10109b78     IO61X_Library_MSVC120_vc:IO61X_GlobalSender.obj
 0002:00006bc4       ??_C@_0DF@EIMPCBKK@Create?5global?5sender?5background?5@ 10109bc4     IO61X_Library_MSVC120_vc:IO61X_GlobalSender.obj
 0002:00006c00       ??_C@_0EH@BHEPDGFD@?$CFs?5?$CFs?0?5ModuleID?5?$CFi?3?5?6Create?5send@ 10109c00     IO61X_Library_MSVC120_vc:IO61X_GlobalSender.obj
 0002:00006c48       ??_C@_0CN@IEICINDA@Close?5handle?5for?5sender?5thread?5f@ 10109c48     IO61X_Library_MSVC120_vc:IO61X_GlobalSender.obj
 0002:00006c78       ??_C@_0CI@NMDKDNDH@Sender?5thread?5is?5terminated?4?5mod@ 10109c78     IO61X_Library_MSVC120_vc:IO61X_GlobalSender.obj
 0002:00006ca0       ??_C@_0EG@PKFHEILI@?5Timeout?5or?5error?5occurred?5while@ 10109ca0     IO61X_Library_MSVC120_vc:IO61X_GlobalSender.obj
 0002:00006ce8       ??_C@_0CO@FFGNAHJB@Close?5handle?5for?5sender?5semaphor@ 10109ce8     IO61X_Library_MSVC120_vc:IO61X_GlobalSender.obj
 0002:00006d18       ??_C@_0DO@CMBMABAE@?5Timeout?5or?5error?5occurred?5while@ 10109d18     IO61X_Library_MSVC120_vc:IO61X_GlobalSender.obj
 0002:00006d58       ??_C@_0BN@MBDCGEJD@?5end?5of?5thread?5for?5modIdx?5?$CFi?$AA@ 10109d58     IO61X_Library_MSVC120_vc:IO61X_GlobalSender.obj
 0002:00006d78       __real@3f50624dd2f1a9fc    10109d78     IO61X_Library_MSVC120_vc:IO61X_GlobalSender.obj
 0002:00006d80       __real@409f400000000000    10109d80     IO61X_Library_MSVC120_vc:IO61X_GlobalSender.obj
 0002:00006d8c       ??_7logic_error@std@@6B@   10109d8c     IO61X_Library_MSVC120_vc:IO61X_DriverObject.obj
 0002:00006d98       ??_7invalid_argument@std@@6B@ 10109d98     IO61X_Library_MSVC120_vc:IO61X_DriverObject.obj
 0002:00006da4       ??_7runtime_error@std@@6B@ 10109da4     IO61X_Library_MSVC120_vc:IO61X_DriverObject.obj
 0002:00006dac       ??_C@_0BA@ELKIONDK@bad?5locale?5name?$AA@ 10109dac     IO61X_Library_MSVC120_vc:IO61X_DriverObject.obj
 0002:00006dc0       ??_7_Facet_base@std@@6B@   10109dc0     IO61X_Library_MSVC120_vc:IO61X_DriverObject.obj
 0002:00006dd0       ??_7facet@locale@std@@6B@  10109dd0     IO61X_Library_MSVC120_vc:IO61X_DriverObject.obj
 0002:00006de0       ??_7codecvt_base@std@@6B@  10109de0     IO61X_Library_MSVC120_vc:IO61X_DriverObject.obj
 0002:00006dfc       ??_7ctype_base@std@@6B@    10109dfc     IO61X_Library_MSVC120_vc:IO61X_DriverObject.obj
 0002:00006e0c       ??_7?$ctype@D@std@@6B@     10109e0c     IO61X_Library_MSVC120_vc:IO61X_DriverObject.obj
 0002:00006e3c       ??_7_System_error@std@@6B@ 10109e3c     IO61X_Library_MSVC120_vc:IO61X_DriverObject.obj
 0002:00006e44       ??_C@_02LMMGGCAJ@?3?5?$AA@ 10109e44     IO61X_Library_MSVC120_vc:IO61X_DriverObject.obj
 0002:00006e4c       ??_7system_error@std@@6B@  10109e4c     IO61X_Library_MSVC120_vc:IO61X_DriverObject.obj
 0002:00006e58       ??_7failure@ios_base@std@@6B@ 10109e58     IO61X_Library_MSVC120_vc:IO61X_DriverObject.obj
 0002:00006e64       ??_7ios_base@std@@6B@      10109e64     IO61X_Library_MSVC120_vc:IO61X_DriverObject.obj
 0002:00006e68       ??_C@_0BF@PHHKMMFD@ios_base?3?3badbit?5set?$AA@ 10109e68     IO61X_Library_MSVC120_vc:IO61X_DriverObject.obj
 0002:00006e80       ??_C@_0BG@FMKFHCIL@ios_base?3?3failbit?5set?$AA@ 10109e80     IO61X_Library_MSVC120_vc:IO61X_DriverObject.obj
 0002:00006e98       ??_C@_0BF@OOHOMBOF@ios_base?3?3eofbit?5set?$AA@ 10109e98     IO61X_Library_MSVC120_vc:IO61X_DriverObject.obj
 0002:00006eb4       ??_7?$basic_ios@DU?$char_traits@D@std@@@std@@6B@ 10109eb4     IO61X_Library_MSVC120_vc:IO61X_DriverObject.obj
 0002:00006ebc       ??_7?$basic_streambuf@DU?$char_traits@D@std@@@std@@6B@ 10109ebc     IO61X_Library_MSVC120_vc:IO61X_DriverObject.obj
 0002:00006efc       ??_7?$basic_ostream@DU?$char_traits@D@std@@@std@@6B@ 10109efc     IO61X_Library_MSVC120_vc:IO61X_DriverObject.obj
 0002:00006f00       ??_8?$basic_ostream@DU?$char_traits@D@std@@@std@@7B@ 10109f00     IO61X_Library_MSVC120_vc:IO61X_DriverObject.obj
 0002:00006f08       ??_C@_0CL@MLCKCNAM@?5Destructor?5of?5the?5IO61X?5driver?5@ 10109f08     IO61X_Library_MSVC120_vc:IO61X_DriverObject.obj
 0002:00006f34       ??_C@_0L@GHEDMKJM@?5qtyPt?3?5?$CFi?$AA@ 10109f34     IO61X_Library_MSVC120_vc:IO61X_DriverObject.obj
 0002:00006f40       ??_C@_0DI@GIFLCGKE@?5Free?5channel?5?$CFi?5configuration?5p@ 10109f40     IO61X_Library_MSVC120_vc:IO61X_DriverObject.obj
 0002:00006f78       ??_C@_0CN@KDIHJNFN@?5Free?5channel?5array?5pointer?5of?5m@ 10109f78     IO61X_Library_MSVC120_vc:IO61X_DriverObject.obj
 0002:00006fa8       ??_C@_0DE@LKCLIJAB@?5Free?5channel?5status?5array?5point@ 10109fa8     IO61X_Library_MSVC120_vc:IO61X_DriverObject.obj
 0002:00006fdc       ??_C@_0BD@MADOGCNH@?5Free?5module?5array?$AA@ 10109fdc     IO61X_Library_MSVC120_vc:IO61X_DriverObject.obj
 0002:00006ff0       ??_C@_0BL@OFBPMCFM@?5Get?5next?5module?5index?3?5?$CFi?$AA@ 10109ff0     IO61X_Library_MSVC120_vc:IO61X_DriverObject.obj
 0002:0000700c       ??_C@_0N@LDGPNHPF@C?3?1IO61X?4log?$AA@ 1010a00c     IO61X_Library_MSVC120_vc:IO61X_DriverObject.obj
 0002:0000701c       ??_C@_0BJ@GPLPCFPM@buffer?5file?5already?5set?$CB?$AA@ 1010a01c     IO61X_Library_MSVC120_vc:IO61X_DriverObject.obj
 0002:0000703c       ??_7?$basic_filebuf@DU?$char_traits@D@std@@@std@@6B@ 1010a03c     IO61X_Library_MSVC120_vc:IO61X_DriverObject.obj
 0002:0000707c       ??_7?$basic_ofstream@DU?$char_traits@D@std@@@std@@6B@ 1010a07c     IO61X_Library_MSVC120_vc:IO61X_DriverObject.obj
 0002:00007080       ??_8?$basic_ofstream@DU?$char_traits@D@std@@@std@@7B@ 1010a080     IO61X_Library_MSVC120_vc:IO61X_DriverObject.obj
 0002:00007088       ??_C@_0GD@FPHFEDKK@Error?5?9?5IO61X_Logger?5could?5not?5o@ 1010a088     IO61X_Library_MSVC120_vc:IO61X_DriverObject.obj
 0002:000070ec       ??_C@_0CL@NFFLPONK@IO61X_Logger?5is?5writing?5to?5log?5f@ 1010a0ec     IO61X_Library_MSVC120_vc:IO61X_DriverObject.obj
 0002:00007118       ??_C@_0BM@HGJAMJFF@?$CF06i?7?$CF02i?3?$CF02i?3?$CF02i?4?$CF06i?7?$CFs?$AA@ 1010a118     IO61X_Library_MSVC120_vc:IO61X_DriverObject.obj
 0002:00007134       ??_C@_0M@JLENPOIA@Error?5?9?5?$CFs?6?$AA@ 1010a134     IO61X_Library_MSVC120_vc:IO61X_DriverObject.obj
 0002:00007140       ??_C@_0L@GOBGNBNP@Warn?5?9?5?$CFs?6?$AA@ 1010a140     IO61X_Library_MSVC120_vc:IO61X_DriverObject.obj
 0002:0000714c       ??_C@_03OFAPEBGM@?$CFs?6?$AA@ 1010a14c     IO61X_Library_MSVC120_vc:IO61X_DriverObject.obj
 0002:00007150       ??_C@_09KNGFFBCM@Dbg?5?9?5?$CFs?6?$AA@ 1010a150     IO61X_Library_MSVC120_vc:IO61X_DriverObject.obj
 0002:0000715c       ??_C@_0BC@KFMMCNJC@illegal?5log?5level?$AA@ 1010a15c     IO61X_Library_MSVC120_vc:IO61X_DriverObject.obj
 0002:00007174       ??_7?$codecvt@DDH@std@@6B@ 1010a174     IO61X_Library_MSVC120_vc:IO61X_DriverObject.obj
 0002:0000719c       ??_C@_08EPJLHIJG@bad?5cast?$AA@ 1010a19c     IO61X_Library_MSVC120_vc:IO61X_DriverObject.obj
 0002:000071a8       __real@4038000000000000    1010a1a8     IO61X_Library_MSVC120_vc:IO61X_DriverObject.obj
 0002:000071b0       __real@404e000000000000    1010a1b0     IO61X_Library_MSVC120_vc:IO61X_DriverObject.obj
 0002:000071b8       __real@40ac200000000000    1010a1b8     IO61X_Library_MSVC120_vc:IO61X_DriverObject.obj
 0002:000071c0       __real@412e848000000000    1010a1c0     IO61X_Library_MSVC120_vc:IO61X_DriverObject.obj
 0002:000071c8       ??_C@_0DA@FFIDKFAA@?$CFs?5?$CFs?0?5ModuleID?5?$CFi?3?5Stop?5init?3?5N@ 1010a1c8     IO61X_Library_MSVC120_vc:IO61X_ModuleManager.obj
 0002:000071f8       ??_C@_0CP@DANDMPJH@?$CFs?5?$CFs?0?5ModuleID?5?$CFi?3?5Stop?5init?3?5N@ 1010a1f8     IO61X_Library_MSVC120_vc:IO61X_ModuleManager.obj
 0002:00007228       ??_C@_0BL@BBNCCDAJ@wrong?5BL?5mailbox?5tag?3?5?$CF?44s?$AA@ 1010a228     IO61X_Library_MSVC120_vc:IO61X_ModuleManager.obj
 0002:00007244       ??_C@_0DC@EEOFINGB@?$CFs?5?$CFs?0?5ModuleID?5?$CFi?3?5Stop?5init?3?5B@ 1010a244     IO61X_Library_MSVC120_vc:IO61X_ModuleManager.obj
 0002:00007278       ??_C@_0CM@HDOFHFPL@?$CFs?5?$CFs?0?5ModuleID?5?$CFi?3?5Protocol?5not@ 1010a278     IO61X_Library_MSVC120_vc:IO61X_ModuleManager.obj
 0002:000072a4       ??_C@_0DB@OHJLEFIA@?$CFs?5?$CFs?0?5ModuleID?5?$CFi?3?5Is?5not?5avail@ 1010a2a4     IO61X_Library_MSVC120_vc:IO61X_ModuleManager.obj
 0002:000072d8       ??_C@_0CK@PFKCPLID@?$CFs?5?$CFs?0?5ModuleID?5?$CFi?3?5mmap?5PCI?5Bar@ 1010a2d8     IO61X_Library_MSVC120_vc:IO61X_ModuleManager.obj
 0002:00007304       ??_C@_0CK@PBFHCLLO@?$CFs?5?$CFs?0?5ModuleID?5?$CFi?3?5mmap?5PCI?5Bar@ 1010a304     IO61X_Library_MSVC120_vc:IO61X_ModuleManager.obj
 0002:00007330       ??_C@_0CJ@BJOMJDBB@?$CFs?5?$CFs?0?5ModuleID?5?$CFi?3?5allocate?5DMA@ 1010a330     IO61X_Library_MSVC120_vc:IO61X_ModuleManager.obj
 0002:0000735c       ??_C@_0CN@CMGLGAID@timeout?5occurred?5during?5attempt?5@ 1010a35c     IO61X_Library_MSVC120_vc:IO61X_ModuleManager.obj
 0002:0000738c       ??_C@_0DN@PELLPKBO@?$CFs?5?$CFs?0?5ModuleID?5?$CFi?3?5Stop?5init?3?5A@ 1010a38c     IO61X_Library_MSVC120_vc:IO61X_ModuleManager.obj
 0002:000073cc       ??_C@_0DD@HMFNOBCE@?$CFs?5?$CFs?0?5ModuleID?5?$CFi?3?5Stop?5init?3?5M@ 1010a3cc     IO61X_Library_MSVC120_vc:IO61X_ModuleManager.obj
 0002:00007400       ??_C@_0CP@BHLBLMEM@Register?5DMA?9?5?$DOpageSize?3?5?$CFi?5?5?9?9?5@ 1010a400     IO61X_Library_MSVC120_vc:IO61X_ModuleManager.obj
 0002:00007430       ??_C@_0CK@CPGHJOLF@register?5DMA?5?9?$DO?5i?3?5?$CFi?5?5?9?5?5?$CIpageC@ 1010a430     IO61X_Library_MSVC120_vc:IO61X_ModuleManager.obj
 0002:0000745c       ??_C@_0CD@IOHHOPGL@entrySizeTranslationTable?5?5?5?5?3?5?$CF@ 1010a45c     IO61X_Library_MSVC120_vc:IO61X_ModuleManager.obj
 0002:00007480       ??_C@_0CD@PEEBPJIH@startAddressTranslationTable?5?3?5?$CF@ 1010a480     IO61X_Library_MSVC120_vc:IO61X_ModuleManager.obj
 0002:000074a4       ??_C@_0CD@FBMAHJLH@endAddressTranslationTable?5?5?5?3?5?$CF@ 1010a4a4     IO61X_Library_MSVC120_vc:IO61X_ModuleManager.obj
 0002:000074c8       ??_C@_0CC@GDADBIJB@pTranslationTableStartAddress?3?5?$CF@ 1010a4c8     IO61X_Library_MSVC120_vc:IO61X_ModuleManager.obj
 0002:000074ec       ??_C@_0CI@CCBDOIMG@Send?5test?5communication?5command?5@ 1010a4ec     IO61X_Library_MSVC120_vc:IO61X_ModuleManager.obj
 0002:00007514       ??_C@_0CD@OLBFJCGJ@Module?5command?9mailbox?5test?5fail@ 1010a514     IO61X_Library_MSVC120_vc:IO61X_ModuleManager.obj
 0002:00007538       ??_C@_0CL@PPNFMCAG@Receive?5test?5communication?5comma@ 1010a538     IO61X_Library_MSVC120_vc:IO61X_ModuleManager.obj
 0002:00007564       ??_C@_0BC@EOJMNIH@DMA?5Memory?5Check?$AA?$AA@ 1010a564     IO61X_Library_MSVC120_vc:IO61X_ModuleManager.obj
 0002:00007578       ??_C@_0DA@CEFGGKPB@Send?5test?5command?5to?5read?5data?5f@ 1010a578     IO61X_Library_MSVC120_vc:IO61X_ModuleManager.obj
 0002:000075a8       ??_C@_0ED@NCEHGLKO@Test?5DMA?5read?5CMD?5failed?4?5Receiv@ 1010a5a8     IO61X_Library_MSVC120_vc:IO61X_ModuleManager.obj
 0002:000075f0       ??_C@_0ED@IFGFBKAD@Test?5DMA?5write?5CMD?5failed?4?5Writt@ 1010a5f0     IO61X_Library_MSVC120_vc:IO61X_ModuleManager.obj
 0002:00007634       ??_C@_0DB@EKOGLCJF@?$CFs?5?$CFs?0?5ModuleID?5?$CFi?3?5Stop?5init?3?5F@ 1010a634     IO61X_Library_MSVC120_vc:IO61X_ModuleManager.obj
 0002:00007668       ??_C@_0DA@BMDEBCMF@?$CFs?5?$CFs?0?5ModuleID?5?$CFi?3?5Stop?5init?3?5F@ 1010a668     IO61X_Library_MSVC120_vc:IO61X_ModuleManager.obj
 0002:00007698       ??_C@_0BI@NAPDGFCO@IO61X_StartFirmware?5ok?4?$AA@ 1010a698     IO61X_Library_MSVC120_vc:IO61X_ModuleManager.obj
 0002:000076b0       ??_C@_0CP@HDIABEHL@?$CFs?5?$CFs?0?5ModuleID?5?$CFi?3?5Stop?5init?3?5F@ 1010a6b0     IO61X_Library_MSVC120_vc:IO61X_ModuleManager.obj
 0002:000076e0       ??_C@_0CD@EFIBPAEF@?$CFs?5?$CFs?0?5ModuleID?5?$CFi?3?5FW?5is?5runnin@ 1010a6e0     IO61X_Library_MSVC120_vc:IO61X_ModuleManager.obj
 0002:00007704       ??_C@_0BG@CFKFAKJI@IO61X_GetFirmware?5ok?4?$AA@ 1010a704     IO61X_Library_MSVC120_vc:IO61X_ModuleManager.obj
 0002:0000771c       ??_C@_0BM@KGKGDPMP@IO61X_CheckFirmwareData?5ok?4?$AA@ 1010a71c     IO61X_Library_MSVC120_vc:IO61X_ModuleManager.obj
 0002:00007738       ??_C@_0L@ECCLJPGL@CAN?9IB200?$AA?$AA@ 1010a738     IO61X_Library_MSVC120_vc:IO61X_ModuleManager.obj
 0002:00007744       ??_C@_0BF@LMIMMHPA@Error?5?9?$DO?5HW?5name?3?5?$CFs?$AA@ 1010a744     IO61X_Library_MSVC120_vc:IO61X_ModuleManager.obj
 0002:0000775c       ??_C@_0DD@PLMLICKO@Error?5?9?$DO?5HW?5version?3?5?$CF?$CDX?4?5?$CF?$CDX?9?$CF?$CD@ 1010a75c     IO61X_Library_MSVC120_vc:IO61X_ModuleManager.obj
 0002:00007790       ??_C@_07DJOPIJFJ@VCI_FW?$AA?$AA@ 1010a790     IO61X_Library_MSVC120_vc:IO61X_ModuleManager.obj
 0002:00007798       ??_C@_0BF@FFLNBEOO@Error?5?9?$DO?5FW?5name?3?5?$CFs?$AA@ 1010a798     IO61X_Library_MSVC120_vc:IO61X_ModuleManager.obj
 0002:000077b0       ??_C@_0DD@ICCHKAPP@Error?5?9?$DO?5FW?5version?3?5?$CF?$CDX?4?5?$CF?$CDX?9?$CF?$CD@ 1010a7b0     IO61X_Library_MSVC120_vc:IO61X_ModuleManager.obj
 0002:000077e4       ??_C@_0CF@PINLFNNB@Error?5?9?$DO?5FW?5length?3?5?$CFi?5?5?$CIis?5not?5@ 1010a7e4     IO61X_Library_MSVC120_vc:IO61X_ModuleManager.obj
 0002:0000780c       ??_C@_0CF@NPJNIGKF@Send?5FW?5to?5module?5controller?5fai@ 1010a80c     IO61X_Library_MSVC120_vc:IO61X_ModuleManager.obj
 0002:00007834       ??_C@_0BB@FBOLPJLE@Start?5FW?5failed?4?$AA@ 1010a834     IO61X_Library_MSVC120_vc:IO61X_ModuleManager.obj
 0002:00007848       ??_C@_0CP@HOIAMECO@Check?5FW?5start?5?9?$DO?5tag?5of?5mailbox@ 1010a848     IO61X_Library_MSVC120_vc:IO61X_ModuleManager.obj
 0002:00007878       ??_C@_0DD@ODMKBJIE@?5Check?5FW?5start?5?9?$DO?5tag?5on?5comman@ 1010a878     IO61X_Library_MSVC120_vc:IO61X_ModuleManager.obj
 0002:000078ac       ??_C@_0DG@OIGAFPIM@?5Check?5FW?5start?5?9?$DO?5tag?5on?5comman@ 1010a8ac     IO61X_Library_MSVC120_vc:IO61X_ModuleManager.obj
 0002:000078e8       ??_C@_0EO@LLFOHEED@?5Check?5FW?5start?5?9?$DO?5DMA?5pre?9initi@ 1010a8e8     IO61X_Library_MSVC120_vc:IO61X_ModuleManager.obj
 0002:00007938       ??_C@_0N@KMFJDPFB@DMA?5size?3?5?$CFi?$AA@ 1010a938     IO61X_Library_MSVC120_vc:IO61X_ModuleManager.obj
 0002:00007948       ??_C@_0BG@FKOMHHH@run?5establish?5DMA?3?5?$CFi?$AA@ 1010a948     IO61X_Library_MSVC120_vc:IO61X_ModuleManager.obj
 0002:00007960       ??_C@_0DP@LHELCCP@?$CFs?5?$CFs?0?5ModuleID?5?$CFi?3?5Stop?5initial@ 1010a960     IO61X_Library_MSVC120_vc:IO61X_ModuleManager.obj
 0002:000079a0       ??_C@_0DO@GBJDNJEH@?$CFs?5?$CFs?0?5ModuleID?5?$CFi?3?5Stop?5initial@ 1010a9a0     IO61X_Library_MSVC120_vc:IO61X_ModuleManager.obj
 0002:000079e0       ??_C@_0P@JMPDDCLG@DMA?5failed?3?5?$CFi?$AA@ 1010a9e0     IO61X_Library_MSVC120_vc:IO61X_ModuleManager.obj
 0002:000079f0       ??_C@_0FM@MKMAPIOJ@?$CFs?5?$CFs?0?5ModuleID?5?$CFi?3?5Stop?5initial@ 1010a9f0     IO61X_Library_MSVC120_vc:IO61X_ModuleManager.obj
 0002:00007a4c       ??_C@_0CM@PAKPJBMN@?$CFi?5DMA?5tests?5are?5done?0?5isDmaTagA@ 1010aa4c     IO61X_Library_MSVC120_vc:IO61X_ModuleManager.obj
 0002:00007a78       ??_C@_0P@OFGBGADG@Tag?5on?5DMA?3?5?$CFs?$AA@ 1010aa78     IO61X_Library_MSVC120_vc:IO61X_ModuleManager.obj
 0002:00007a88       ??_C@_0BP@JBIFFOOA@Get?5DMA?5size?5failed?0?5size?5?$DN?50?4?$AA@ 1010aa88     IO61X_Library_MSVC120_vc:IO61X_ModuleManager.obj
 0002:00007aa8       ??_C@_0BF@EHKHKNIP@Get?5DMA?5size?5failed?4?$AA@ 1010aaa8     IO61X_Library_MSVC120_vc:IO61X_ModuleManager.obj
 0002:00007ac0       ??_C@_0BH@EGIBFFOF@?5Establish?5DMA?5failed?4?$AA@ 1010aac0     IO61X_Library_MSVC120_vc:IO61X_ModuleManager.obj
 0002:00007ad8       ??_C@_0EO@PBPCOHKP@?$CFs?5?$CFs?0?5ModuleID?5?$CFi?3?5Stop?5initial@ 1010aad8     IO61X_Library_MSVC120_vc:IO61X_ModuleManager.obj
 0002:00007b28       ??_C@_0FB@OLBMGLPN@?$CFs?5?$CFs?0?5ModuleID?5?$CFi?3?5Stop?5module?5@ 1010ab28     IO61X_Library_MSVC120_vc:IO61X_ModuleManager.obj
 0002:00007b7c       ??_C@_0BC@MHGPKAGN@Capa?5quantity?3?5?$CFi?$AA@ 1010ab7c     IO61X_Library_MSVC120_vc:IO61X_ModuleManager.obj
 0002:00007b90       ??_C@_0BG@HOIBJOBF@Channel?5?$CFi?3?5?$CF?$CDX?5?9?5?$CF?$CDX?$AA@ 1010ab90     IO61X_Library_MSVC120_vc:IO61X_ModuleManager.obj
 0002:00007ba8       ??_C@_0FM@JNPGDLDO@Quantity?5of?5channels?5?$CI?$CFi?$CJ?5mismat@ 1010aba8     IO61X_Library_MSVC120_vc:IO61X_ModuleManager.obj
 0002:00007c04       ??_C@_0BP@NPHEKLLM@Get?5module?5capabilities?5failed?$AA@ 1010ac04     IO61X_Library_MSVC120_vc:IO61X_ModuleManager.obj
 0002:00007c24       ??_C@_0BK@GKPGMPGC@check?5expansion?5for?5IO611?$AA@ 1010ac24     IO61X_Library_MSVC120_vc:IO61X_ModuleManager.obj
 0002:00007c40       ??_C@_0GB@EDEADJPA@?$CFs?5?$CFs?0?5ModuleID?5?$CFi?3?5Stop?5initial@ 1010ac40     IO61X_Library_MSVC120_vc:IO61X_ModuleManager.obj
 0002:00007ca8       ??_C@_0FH@GIKGPMBF@?$CFs?5?$CFs?0?5ModuleID?5?$CFi?3?5Stop?5initial@ 1010aca8     IO61X_Library_MSVC120_vc:IO61X_ModuleManager.obj
 0002:00007d00       ??_C@_0FH@BFNFPKEN@?$CFs?5?$CFs?0?5ModuleID?5?$CFi?3?5Stop?5initial@ 1010ad00     IO61X_Library_MSVC120_vc:IO61X_ModuleManager.obj
 0002:00007d58       ??_C@_0BL@EIKECGIK@?5check?5expansion?5for?5IO612?$AA@ 1010ad58     IO61X_Library_MSVC120_vc:IO61X_ModuleManager.obj
 0002:00007d78       ??_C@_0FH@CPECEDCL@?$CFs?5?$CFs?0?5ModuleID?5?$CFi?3?5Stop?5initial@ 1010ad78     IO61X_Library_MSVC120_vc:IO61X_ModuleManager.obj
 0002:00007dd0       ??_C@_0FH@FCDBEFHD@?$CFs?5?$CFs?0?5ModuleID?5?$CFi?3?5Stop?5initial@ 1010add0     IO61X_Library_MSVC120_vc:IO61X_ModuleManager.obj
 0002:00007e28       ??_C@_0CG@NILLNIFM@Module?5channel?5array?5is?5not?5avai@ 1010ae28     IO61X_Library_MSVC120_vc:IO61X_ModuleManager.obj
 0002:00007e50       ??_C@_0EH@DOKLOK@?5ChnIdx?$FL?$DN?$DNCapIdx?$FN?5?$CFi?5?$CI?$DNChannel?5?$CF@ 1010ae50     IO61X_Library_MSVC120_vc:IO61X_ModuleManager.obj
 0002:00007e98       ??_C@_0BL@EIHEGGGO@?5ptTypeOfs?5?5?5?5?5?5?5?5?5?5?5?5?3?5?$CFi?$AA@ 1010ae98     IO61X_Library_MSVC120_vc:IO61X_ModuleManager.obj
 0002:00007eb4       ??_C@_0BL@DMDIIFDL@?5ProtlHelpIdx?5?5?5?5?5?5?5?5?5?3?5?$CFi?$AA@ 1010aeb4     IO61X_Library_MSVC120_vc:IO61X_ModuleManager.obj
 0002:00007ed0       ??_C@_0BE@CJFICDOI@?5Snd?5offset?5?$CFi?3?5?$CF?$CDX?$AA@ 1010aed0     IO61X_Library_MSVC120_vc:IO61X_ModuleManager.obj
 0002:00007ee4       ??_C@_0BL@GNJILCCL@?5Snd?5number?5of?5objects?3?5?$CFi?$AA@ 1010aee4     IO61X_Library_MSVC120_vc:IO61X_ModuleManager.obj
 0002:00007f00       ??_C@_0BG@IMNHNIMK@?5Snd?5Mbx?5Tag?5?$CI?$CFi?$CJ?3?5?$CFs?$AA@ 1010af00     IO61X_Library_MSVC120_vc:IO61X_ModuleManager.obj
 0002:00007f18       ??_C@_0BE@CDPPKMJF@?5Rec?5offset?5?$CFi?3?5?$CF?$CDX?$AA@ 1010af18     IO61X_Library_MSVC120_vc:IO61X_ModuleManager.obj
 0002:00007f2c       ??_C@_0BL@KCHLAGCP@?5Rec?5number?5of?5objects?3?5?$CFi?$AA@ 1010af2c     IO61X_Library_MSVC120_vc:IO61X_ModuleManager.obj
 0002:00007f48       ??_C@_0BG@GLEBELGH@?5Rec?5Mbx?5Tag?5?$CI?$CFi?$CJ?3?5?$CFs?$AA@ 1010af48     IO61X_Library_MSVC120_vc:IO61X_ModuleManager.obj
 0002:00007f60       ??_C@_0CP@HLMNNILH@?5Find?5send?5queue?5for?5the?5channel@ 1010af60     IO61X_Library_MSVC120_vc:IO61X_ModuleManager.obj
 0002:00007f90       ??_C@_0DC@OEBFFOHM@?5Find?5receive?5queue?5for?5the?5chan@ 1010af90     IO61X_Library_MSVC120_vc:IO61X_ModuleManager.obj
 0002:00007fc4       ??_C@_0CK@NILADMDF@?5Channel?5?$CFi?5?5?9?5?5sndMbx?3?5?$CFp?5?5?9?9?5r@ 1010afc4     IO61X_Library_MSVC120_vc:IO61X_ModuleManager.obj
 0002:00007ff0       ??_C@_0BB@HDLHJEIE@?5Mailbox?5tag?3?5?$CFs?$AA@ 1010aff0     IO61X_Library_MSVC120_vc:IO61X_ModuleManager.obj
 0002:00008004       ??_C@_0DD@PKOAOLLG@?5Port?5?$CFi?5?5?9?5?5Rwwb1?3?5?$CFp?5?5?9?9?5Rwwb2@ 1010b004     IO61X_Library_MSVC120_vc:IO61X_ModuleManager.obj
 0002:00008038       ??_C@_0BK@NEOPDFJ@No?5RWWB?5buffer?5available?4?$AA@ 1010b038     IO61X_Library_MSVC120_vc:IO61X_ModuleManager.obj
 0002:00008054       ??_C@_0CJ@EIFCMMGO@CAN?5channel?5?$CFi?0?5start?5controller@ 1010b054     IO61X_Library_MSVC120_vc:IO61X_ModuleManager.obj
 0002:00008080       ??_C@_0CC@PJDKNLFI@?5Start?5time?5of?5the?5controller?3?5?$CF@ 1010b080     IO61X_Library_MSVC120_vc:IO61X_ModuleManager.obj
 0002:000080a4       ??_C@_06OMDKJLOD@VCI_FW?$AA@ 1010b0a4     IO61X_Library_MSVC120_vc:IO61X_ModuleManager.obj
 0002:000080ac       ??_C@_09JJAHAHCJ@CAN?9IB200?$AA@ 1010b0ac     IO61X_Library_MSVC120_vc:IO61X_ModuleManager.obj
 0002:000080b8       ??_C@_05CICAGBGK@_HEX_?$AA@ 1010b0b8     IO61X_Library_MSVC120_vc:IO61X_ModuleManager.obj
 0002:000080c0       __real@3f747ae147ae147b    1010b0c0     IO61X_Library_MSVC120_vc:IO61X_ModuleManager.obj
 0002:000080c8       __real@3fc999999999999a    1010b0c8     IO61X_Library_MSVC120_vc:IO61X_ModuleManager.obj
 0002:000080d0       __real@41cdcd6500000000    1010b0d0     IO61X_Library_MSVC120_vc:IO61X_ModuleManager.obj
 0002:000080d8       __real@41e65a0bc0000000    1010b0d8     IO61X_Library_MSVC120_vc:IO61X_ModuleManager.obj
 0002:000080e0       ??_C@_0BJ@HIEOFCE@?5OpMode?5?5?5?5?5?5?3?5?$CFi?5?9?9?5?$CF?$CDX?$AA@ 1010b0e0     IO61X_Library_MSVC120_vc:IO61X_CanManager.obj
 0002:000080fc       ??_C@_0BC@FLAODBAP@?5Timing?4Mode?5?3?5?$CFi?$AA@ 1010b0fc     IO61X_Library_MSVC120_vc:IO61X_CanManager.obj
 0002:00008110       ??_C@_0BC@GCMPEKFO@?5Timing?4BRP?5?5?3?5?$CFi?$AA@ 1010b110     IO61X_Library_MSVC120_vc:IO61X_CanManager.obj
 0002:00008124       ??_C@_0BC@LHHOEJPI@?5Timing?4SJW?5?5?3?5?$CFi?$AA@ 1010b124     IO61X_Library_MSVC120_vc:IO61X_CanManager.obj
 0002:00008138       ??_C@_0BC@ONMEDDKI@?5Timing?4TSEG1?3?5?$CFi?$AA@ 1010b138     IO61X_Library_MSVC120_vc:IO61X_CanManager.obj
 0002:0000814c       ??_C@_0BC@GLFAEBAG@?5Timing?4TSEG2?3?5?$CFi?$AA@ 1010b14c     IO61X_Library_MSVC120_vc:IO61X_CanManager.obj
 0002:00008160       ??_C@_0BC@DCDOKDIN@?5Timing?4TDO?5?5?3?5?$CFi?$AA@ 1010b160     IO61X_Library_MSVC120_vc:IO61X_CanManager.obj
 0002:00008174       ??_C@_0BM@PLPKBPGJ@IO61X_CanAllocatePortMemory?$AA@ 1010b174     IO61X_Library_MSVC120_vc:IO61X_CanManager.obj
 0002:00008190       ??_C@_0EE@NPNAHFFJ@Allocate?5memory?5for?5CAN?5channel?5@ 1010b190     IO61X_Library_MSVC120_vc:IO61X_CanManager.obj
 0002:000081d4       ??_C@_0DN@EHBDBFID@Allocate?5memory?5for?5CAN?5channel?5@ 1010b1d4     IO61X_Library_MSVC120_vc:IO61X_CanManager.obj
 0002:00008214       ??_C@_0BE@BONPKMMA@?5ExtOpMode?5?5?5?5?5?3?5?$CFi?$AA@ 1010b214     IO61X_Library_MSVC120_vc:IO61X_CanManager.obj
 0002:00008228       ??_C@_0BE@NIOAAGLK@?5TimingFD?4Mode?5?3?5?$CFi?$AA@ 1010b228     IO61X_Library_MSVC120_vc:IO61X_CanManager.obj
 0002:0000823c       ??_C@_0BE@OBCBHNOL@?5TimingFD?4BRP?5?5?3?5?$CFi?$AA@ 1010b23c     IO61X_Library_MSVC120_vc:IO61X_CanManager.obj
 0002:00008250       ??_C@_0BE@DEJAHOEN@?5TimingFD?4SJW?5?5?3?5?$CFi?$AA@ 1010b250     IO61X_Library_MSVC120_vc:IO61X_CanManager.obj
 0002:00008264       ??_C@_0BE@GOCKAEBN@?5TimingFD?4TSEG1?3?5?$CFi?$AA@ 1010b264     IO61X_Library_MSVC120_vc:IO61X_CanManager.obj
 0002:00008278       ??_C@_0BE@OILOHGLD@?5TimingFD?4TSEG2?3?5?$CFi?$AA@ 1010b278     IO61X_Library_MSVC120_vc:IO61X_CanManager.obj
 0002:0000828c       ??_C@_0BE@LBNAJEDI@?5TimingFD?4TDO?5?5?3?5?$CFi?$AA@ 1010b28c     IO61X_Library_MSVC120_vc:IO61X_CanManager.obj
 0002:000082a0       ??_C@_0DI@EEGJFJKH@Send?5init?5CAN?5controller?5command@ 1010b2a0     IO61X_Library_MSVC120_vc:IO61X_CanManager.obj
 0002:000082d8       ??_C@_0CK@LDKCBOIA@Init?5controller?5of?5CAN?5channel?5?$CF@ 1010b2d8     IO61X_Library_MSVC120_vc:IO61X_CanManager.obj
 0002:00008304       ??_C@_0DH@CPKNPEID@Set?5Standard?5Acceptance?5Mask?5of?5@ 1010b304     IO61X_Library_MSVC120_vc:IO61X_CanManager.obj
 0002:0000833c       ??_C@_0DH@MKAHLFCK@Set?5Extended?5Acceptance?5Mask?5of?5@ 1010b33c     IO61X_Library_MSVC120_vc:IO61X_CanManager.obj
 0002:00008374       ??_C@_0CE@CEFKEBID@?5number?5elements?5in?5read?5buffer?3@ 1010b374     IO61X_Library_MSVC120_vc:IO61X_CanManager.obj
 0002:00008398       ??_C@_0BL@GAIHPOE@?5Receive?5status?5successful?$AA@ 1010b398     IO61X_Library_MSVC120_vc:IO61X_CanManager.obj
 0002:000083b4       ??_C@_0O@PACICJLO@?5OpMode?5?5?3?5?$CFi?$AA@ 1010b3b4     IO61X_Library_MSVC120_vc:IO61X_CanManager.obj
 0002:000083c4       ??_C@_0O@IMDIFLIP@?5ExtMode?5?3?5?$CFi?$AA@ 1010b3c4     IO61X_Library_MSVC120_vc:IO61X_CanManager.obj
 0002:000083d4       ??_C@_0O@EHIKCHFE@?5BusLoad?5?3?5?$CFi?$AA@ 1010b3d4     IO61X_Library_MSVC120_vc:IO61X_CanManager.obj
 0002:000083e4       ??_C@_0BJ@MPLIDJGO@?5CtrlStat?3?5?$CF?$CDX?5?5?5?9?5?5?$CI?$CFi?$CJ?$AA@ 1010b3e4     IO61X_Library_MSVC120_vc:IO61X_CanManager.obj
 0002:00008400       __real@4059000000000000    1010b400     IO61X_Library_MSVC120_vc:IO61X_CanManager.obj
 0002:00008408       __real@419312d000000000    1010b408     IO61X_Library_MSVC120_vc:IO61X_CanManager.obj
 0002:00008414       ??_7IO61X_Port@@6B@        1010b414     IO61X_Library_MSVC120_vc:IO61X_Port.obj
 0002:00008430       ??_7IO61X_CanPort@@6B@     1010b430     IO61X_Library_MSVC120_vc:IO61X_CanPort.obj
 0002:00008448       ??_C@_0CA@LJEMIHJL@?5CAN?9m_pPortOperatingStatus?3?5?$CFi?$AA@ 1010b448     IO61X_Library_MSVC120_vc:IO61X_CanPort.obj
 0002:00008468       ??_C@_0DC@ICOJGLAG@?5Snd?$CI?$CFi?$CJ?5?9?$DO?5Id?3?5?$CFi?5?5?9?5?5Data?3?5?$CFi?5@ 1010b468     IO61X_Library_MSVC120_vc:IO61X_CanPort.obj
 0002:0000849c       ??_C@_0CH@CAKDPKAE@?5Send?5buffer?5full?0?5new?5message?5i@ 1010b49c     IO61X_Library_MSVC120_vc:IO61X_CanPort.obj
 0002:000084c4       ??_C@_0BB@MOGOBHAF@list?$DMT?$DO?5too?5long?$AA@ 1010b4c4     IO61X_Library_MSVC120_vc:IO61X_CanPort.obj
 0002:000084dc       ??_7IO61X_CanFdPort@@6B@   1010b4dc     IO61X_Library_MSVC120_vc:IO61X_CanFdPort.obj
 0002:000084f4       ??_C@_0CD@EDBJFMAB@?5Can?9FD?3?5m_pChnOperatingStatus?3?5@ 1010b4f4     IO61X_Library_MSVC120_vc:IO61X_CanFdPort.obj
 0002:00008518       ??_C@_0CD@KAICBPCE@?5Snd?9FD?$CI?$CFi?$CJ?5?9?$DO?5Id?3?5?$CFi?5?5?9?5?5Data?3?5@ 1010b518     IO61X_Library_MSVC120_vc:IO61X_CanFdPort.obj
 0002:0000853c       ??_C@_0CA@COKLLPNM@?5Snd?$CI?$CFi?$CJ?5?9?$DO?5Id?3?5?$CFi?5?5?9?5?5Data?3?5?$CFi?$AA@ 1010b53c     IO61X_Library_MSVC120_vc:IO61X_CanFdPort.obj
 0002:0000855c       ??_C@_0CE@LKGFPNFO@?51?5do?5channel?5reset?5to?5send?5msg?3@ 1010b55c     IO61X_Library_MSVC120_vc:IO61X_CanFdPort.obj
 0002:00008580       ??_C@_0DE@PBMMAPEG@midx?5?$CFi?5pidx?5?$CFi?3?52?5do?5channel?5re@ 1010b580     IO61X_Library_MSVC120_vc:IO61X_CanFdPort.obj
 0002:000085b4       ??_C@_0DC@MIIKPNLO@Allocate?5memory?5for?5status?5handl@ 1010b5b4     IO61X_Library_MSVC120_vc:IO61X_StatusManager.obj
 0002:000085e8       ??_C@_0DD@MGPKIDFK@?5Start?5thread?5for?5bus?5recovery?5o@ 1010b5e8     IO61X_Library_MSVC120_vc:IO61X_ThreadManager.obj
 0002:0000861c       ??_C@_0DI@EHKKLLFJ@?5Trigger?5bus?5recovery?5of?5module?5@ 1010b61c     IO61X_Library_MSVC120_vc:IO61X_ThreadManager.obj
 0002:00008658       ??_C@_0EP@NBFBDFHJ@?5Timeout?5or?5error?5occurred?5while@ 1010b658     IO61X_Library_MSVC120_vc:IO61X_ThreadManager.obj
 0002:000086a8       ??_C@_0DA@KHJGFNOK@?5Finish?5bus?5recovery?5thread?5of?5m@ 1010b6a8     IO61X_Library_MSVC120_vc:IO61X_ThreadManager.obj
 0002:000086d8       ??_C@_0CH@NNLDDICK@?5Thread?5for?5bus?5recovery?5is?5term@ 1010b6d8     IO61X_Library_MSVC120_vc:IO61X_ThreadManager.obj
 0002:00008700       ??_C@_0FB@EDPCAIGI@?5Timeout?5or?5error?5occurred?5while@ 1010b700     IO61X_Library_MSVC120_vc:IO61X_ThreadManager.obj
 0002:00008754       ??_C@_0BM@IHKMOCDG@IO61X_AllocateLinPortMemory?$AA@ 1010b754     IO61X_Library_MSVC120_vc:IO61X_LinManager.obj
 0002:00008770       ??_C@_0EE@KEBBMEEG@Allocate?5memory?5for?5LIN?5channel?5@ 1010b770     IO61X_Library_MSVC120_vc:IO61X_LinManager.obj
 0002:000087b4       ??_C@_0DN@OFONPBNE@Allocate?5memory?5for?5LIN?5channel?5@ 1010b7b4     IO61X_Library_MSVC120_vc:IO61X_LinManager.obj
 0002:000087f4       ??_C@_0CJ@OBMJACAP@Send?5init?5LIN?5controller?5command@ 1010b7f4     IO61X_Library_MSVC120_vc:IO61X_LinManager.obj
 0002:00008820       ??_C@_0DE@EAGKGLGD@Init?5LIN?5controller?5failed?5for?5L@ 1010b820     IO61X_Library_MSVC120_vc:IO61X_LinManager.obj
 0002:00008854       ??_C@_0DC@LIGLLDGH@?5Start?5LIN?5controller?5of?5channel@ 1010b854     IO61X_Library_MSVC120_vc:IO61X_LinManager.obj
 0002:00008888       ??_C@_0CJ@MMMPOLBN@?5get?5new?5status?5response?5?9?$DO?5?$CFi?5?9@ 1010b888     IO61X_Library_MSVC120_vc:IO61X_LinManager.obj
 0002:000088b8       ??_7IO61X_LinPort@@6B@     1010b8b8     IO61X_Library_MSVC120_vc:IO61X_LinPort.obj
 0002:000088d0       ??_C@_0BO@EGCCECIA@?5lin?5master?5send?5?5?9?5?5size?3?5?$CFi?$AA@ 1010b8d0     IO61X_Library_MSVC120_vc:IO61X_LinPort.obj
 0002:000088f0       ??_C@_0EF@HAICGCEN@Ma?9Snd?5?9?$DO?5WrtIdx?3?5?$CFi?5?9?5Id?3?5?$CFi?5?9?5@ 1010b8f0     IO61X_Library_MSVC120_vc:IO61X_LinPort.obj
 0002:00008938       ??_C@_0BM@NNLPADEO@?5Slave?5sender?5?9?5update?5RWWB?$AA@ 1010b938     IO61X_Library_MSVC120_vc:IO61X_LinPort.obj
 0002:00008954       ??_C@_0CN@CGLOBHBB@Slv?9Upd2?5?9?$DO?5pRwwb?$FL?$CFi?$FN?5?9?5Id?3?5?$CFi?5?9@ 1010b954     IO61X_Library_MSVC120_vc:IO61X_LinPort.obj
 0002:00008984       ??_C@_0CN@NABBNAPE@?5Lin?5Receive?5for?5midx?3?5?$CFi?5pidx?3?5@ 1010b984     IO61X_Library_MSVC120_vc:IO61X_LinPort.obj
 0002:000089b4       ??_C@_0CK@JFNDCLIP@?5LIN?5recv?5?9?5id?3?5?$CFi?5is?5element?5of@ 1010b9b4     IO61X_Library_MSVC120_vc:IO61X_LinPort.obj
 0002:000089e0       ??_C@_0DL@IBHLHGKN@?5LIN?5channel?5?$CFi?5?9?5msg?5lost?5?$CIbuff@ 1010b9e0     IO61X_Library_MSVC120_vc:IO61X_LinPort.obj
 0002:00008a1c       ??_C@_0DH@BEFEMNDH@?5LIN?5channel?5?$CFi?5?9?5msg?5with?5unkno@ 1010ba1c     IO61X_Library_MSVC120_vc:IO61X_LinPort.obj
 0002:00008a54       ??_C@_0DE@COCANJNC@?5Master?5receive?5an?5error?5?9?5type?3@ 1010ba54     IO61X_Library_MSVC120_vc:IO61X_LinPort.obj
 0002:00008a88       ??_C@_0FF@HGKJOIIG@LIN?5Upd?9Buf?5isMaster?3?5?$CFi?5?9?$DO?5WrtI@ 1010ba88     IO61X_Library_MSVC120_vc:IO61X_LinPort.obj
 0002:00008ae0       ??_C@_0DK@NCINICNB@?5Send?5buffer?5?$CIisMaster?3?$CFi?$CJ?5full?0@ 1010bae0     IO61X_Library_MSVC120_vc:IO61X_LinPort.obj
 0002:00008b1c       ??_C@_0CG@JLELDBBM@?5LIN?5pidx?5?$CFi?5allocate?5new?5send?5b@ 1010bb1c     IO61X_Library_MSVC120_vc:IO61X_LinPort.obj
 0002:00008b44       ??_C@_0DF@ONJOCOHM@?5LIN?5pidx?5?$CFi?5?9?5allocate?5new?5rece@ 1010bb44     IO61X_Library_MSVC120_vc:IO61X_LinPort.obj
 0002:00008b80       ??_C@_0EA@GFOAJJ@?5LIN?5pidx?5?$CFi?5?9?5cannot?5add?5messag@ 1010bb80     IO61X_Library_MSVC120_vc:IO61X_LinPort.obj
 0002:00008bc0       ??_C@_0CB@HOALPLKL@?5release?5rwwb?5?9?$DO?5rwwb_latest?3?5?$CFi@ 1010bbc0     IO61X_Library_MSVC120_vc:IO61X_LinPort.obj
 0002:00008be4       ??_C@_0CA@MMOGIFNF@invalid?5unordered_map?$DMK?0?5T?$DO?5key?$AA@ 1010bbe4     IO61X_Library_MSVC120_vc:IO61X_LinPort.obj
 0002:00008c04       ??_C@_0BD@OLBABOEK@vector?$DMT?$DO?5too?5long?$AA@ 1010bc04     IO61X_Library_MSVC120_vc:IO61X_LinPort.obj
 0002:00008c18       __real@408f400000000000    1010bc18     IO61X_Library_MSVC120_vc:SlrtOSManagement.obj
 0002:00008c20       ??_C@_01KDCPPGHE@r?$AA@    1010bc20     IO61X_Library_MSVC120_vc:IO61X_CommonManager.obj
 0002:00008c24       ??_C@_08FGIMKMMK@IO61X?4FW?$AA@ 1010bc24     IO61X_Library_MSVC120_vc:IO61X_CommonManager.obj
 0002:00008c30       ??_C@_09LNKODCMC@CAN?9IB410?$AA@ 1010bc30     IO61X_Library_MSVC120_vc:IO61X_CommonManager.obj
 0002:00008c3c       ??_C@_07KACCAJNE@VCI3_FW?$AA@ 1010bc3c     IO61X_Library_MSVC120_vc:IO61X_CommonManager.obj
 0002:00008c44       ??_C@_07DHBGGMLN@0?43?49?43?$AA@ 1010bc44     IO61X_Library_MSVC120_vc:IO61X_CommonManager.obj
 0002:00008c4c       ??_C@_0BP@GAIBGCK@?5Protocol?5?$CFs?5is?5not?5supported?4?$AA@ 1010bc4c     IO61X_Library_MSVC120_vc:IO61X_CommonManager.obj
 0002:00008c6c       ??_C@_0CL@CNDINDBP@Wrong?5mailbox?5tag?3?5?$CF?$CDX?5?5?9?5?5?$CIexpe@ 1010bc6c     IO61X_Library_MSVC120_vc:IO61X_CommonManager.obj
 0002:00008c98       ??_C@_0DH@DFHLJFIL@Send?5config?5packet?5to?5microcontr@ 1010bc98     IO61X_Library_MSVC120_vc:IO61X_CommunicationManager.obj
 0002:00008cd0       ??_C@_0DC@DCAKPOPO@Mailbox?5direction?5is?5not?5sending@ 1010bcd0     IO61X_Library_MSVC120_vc:IO61X_CommunicationManager.obj
 0002:00008d04       ??_C@_0DE@FFJJAHHN@Mailbox?5direction?5is?5not?5receivi@ 1010bd04     IO61X_Library_MSVC120_vc:IO61X_CommunicationManager.obj
 0002:00008d38       ??_C@_0BA@EFALFILH@Error?5Code?3?5?$CF?$CDX?$AA@ 1010bd38     IO61X_Library_MSVC120_vc:IO61X_CommunicationManager.obj
 0002:00008d48       ??_C@_0M@OKGPPKGC@counter?3?5?$CFi?$AA@ 1010bd48     IO61X_Library_MSVC120_vc:IO61X_CommunicationManager.obj
 0002:00008d54       ??_C@_0CC@PJMCGONE@readIndex?3?5?$CFi?5?5?9?$DO?5?5writeIndex?3?5?$CF@ 1010bd54     IO61X_Library_MSVC120_vc:IO61X_CommunicationManager.obj
 0002:00008d78       ??_C@_0DH@KMCMOMKN@Expected?5packet?5size?3?5?$CFi?5?5?9?$DO?5?5Re@ 1010bd78     IO61X_Library_MSVC120_vc:IO61X_CommunicationManager.obj
 0002:00008db0       ??_C@_0DK@NJKODLDL@Expected?5command?5code?3?5?$CFi?5?5?9?$DO?5?5R@ 1010bdb0     IO61X_Library_MSVC120_vc:IO61X_CommunicationManager.obj
 0002:00008df0       ??_C@_0EA@IBGFCMAI@Expected?5requestet?5channel?3?5?$CFi?5?5@ 1010bdf0     IO61X_Library_MSVC120_vc:IO61X_CommunicationManager.obj
 0002:00008e30       ??_C@_0DG@JNOEDLGP@Expected?5return?5code?3?50?5?5?9?$DO?5?5Ret@ 1010be30     IO61X_Library_MSVC120_vc:IO61X_CommunicationManager.obj
 0002:00008e68       ??_C@_0BH@LLJIFCCH@No?5packet?5was?5received?$AA@ 1010be68     IO61X_Library_MSVC120_vc:IO61X_CommunicationManager.obj
 0002:00008e80       __FPinit                   1010be80     LIBCMT:fpinit.obj
 0002:00008f1c       ??_C@_1BI@BGOHAHKC@?$AAm?$AAs?$AAc?$AAo?$AAr?$AAe?$AAe?$AA?4?$AAd?$AAl?$AAl?$AA?$AA@ 1010bf1c     LIBCMT:crt0dat.obj
 0002:00008f34       ??_C@_0P@MIGLKIOC@CorExitProcess?$AA@ 1010bf34     LIBCMT:crt0dat.obj
 0002:00008f44       ??_C@_17LGKOMLJ@?$AA?4?$AA?4?$AA?4?$AA?$AA@ 1010bf44     LIBCMT:wassert.obj
 0002:00008f4c       ??_C@_13LBAGMAIH@?$AA?6?$AA?$AA@ 1010bf4c     LIBCMT:wassert.obj
 0002:00008f50       ??_C@_15IABLJNFO@?$AA?6?$AA?6?$AA?$AA@ 1010bf50     LIBCMT:wassert.obj
 0002:00008f58       ??_C@_1CE@OJBNHDMO@?$AAA?$AAs?$AAs?$AAe?$AAr?$AAt?$AAi?$AAo?$AAn?$AA?5?$AAf?$AAa?$AAi?$AAl?$AAe?$AAd?$AA?$CB?$AA?$AA@ 1010bf58     LIBCMT:wassert.obj
 0002:00008f7c       ??_C@_1BE@PHKBBGE@?$AAP?$AAr?$AAo?$AAg?$AAr?$AAa?$AAm?$AA?3?$AA?5?$AA?$AA@ 1010bf7c     LIBCMT:wassert.obj
 0002:00008f90       ??_C@_1CO@EAEJAADC@?$AA?$DM?$AAp?$AAr?$AAo?$AAg?$AAr?$AAa?$AAm?$AA?5?$AAn?$AAa?$AAm?$AAe?$AA?5?$AAu?$AAn?$AAk?$AAn?$AAo?$AAw?$AAn?$AA?$DO?$AA?$AA@ 1010bf90     LIBCMT:wassert.obj
 0002:00008fc0       ??_C@_1O@HEMHKNDC@?$AAF?$AAi?$AAl?$AAe?$AA?3?$AA?5?$AA?$AA@ 1010bfc0     LIBCMT:wassert.obj
 0002:00008fd0       ??_C@_1O@KCAFKHJE@?$AAL?$AAi?$AAn?$AAe?$AA?3?$AA?5?$AA?$AA@ 1010bfd0     LIBCMT:wassert.obj
 0002:00008fe0       ??_C@_1BK@PEDCIPMA@?$AAE?$AAx?$AAp?$AAr?$AAe?$AAs?$AAs?$AAi?$AAo?$AAn?$AA?3?$AA?5?$AA?$AA@ 1010bfe0     LIBCMT:wassert.obj
 0002:00009000       ??_C@_1OA@EGMLFBHJ@?$AAF?$AAo?$AAr?$AA?5?$AAi?$AAn?$AAf?$AAo?$AAr?$AAm?$AAa?$AAt?$AAi?$AAo?$AAn?$AA?5?$AAo?$AAn?$AA?5?$AAh?$AAo?$AAw?$AA?5?$AAy?$AAo?$AAu?$AAr?$AA?5?$AAp?$AAr?$AAo?$AAg@ 1010c000     LIBCMT:wassert.obj
 0002:000090e0       ??_C@_1HK@POCJMFGK@?$AA?$CI?$AAP?$AAr?$AAe?$AAs?$AAs?$AA?5?$AAR?$AAe?$AAt?$AAr?$AAy?$AA?5?$AAt?$AAo?$AA?5?$AAd?$AAe?$AAb?$AAu?$AAg?$AA?5?$AAt?$AAh?$AAe?$AA?5?$AAa?$AAp?$AAp?$AAl?$AAi?$AAc@ 1010c0e0     LIBCMT:wassert.obj
 0002:00009160       ??_C@_1EK@MBDPDCGA@?$AAM?$AAi?$AAc?$AAr?$AAo?$AAs?$AAo?$AAf?$AAt?$AA?5?$AAV?$AAi?$AAs?$AAu?$AAa?$AAl?$AA?5?$AAC?$AA?$CL?$AA?$CL?$AA?5?$AAR?$AAu?$AAn?$AAt?$AAi?$AAm?$AAe?$AA?5?$AAL?$AAi?$AAb@ 1010c160     LIBCMT:wassert.obj
 0002:000091ac       __pDefaultRawDllMain       1010c1ac     LIBCMT:dllcrt0.obj
 0002:000091ac       __pRawDllMain              1010c1ac     LIBCMT:dllcrt0.obj
 0002:000091b0       ?value@?$integral_constant@_N$0A@@std@@2_NB 1010c1b0     LIBCMT:new.obj
 0002:000091b1       ?value@?$integral_constant@_N$00@std@@2_NB 1010c1b1     LIBCMT:new.obj
 0002:000091b8       ??_7bad_alloc@std@@6B@     1010c1b8     LIBCMT:new.obj
 0002:000091c0       ??_C@_0P@GHFPNOJB@bad?5allocation?$AA@ 1010c1c0     LIBCMT:new.obj
 0002:000091f0       ?ProcessDetach@NativeDll@<CrtImplementationDetails>@@0IB 1010c1f0     LIBCMT:_trnsctrl_.obj
 0002:000091f4       ?ProcessAttach@NativeDll@<CrtImplementationDetails>@@0IB 1010c1f4     LIBCMT:_trnsctrl_.obj
 0002:000091f8       ?ThreadAttach@NativeDll@<CrtImplementationDetails>@@0IB 1010c1f8     LIBCMT:_trnsctrl_.obj
 0002:000091fc       ?ThreadDetach@NativeDll@<CrtImplementationDetails>@@0IB 1010c1fc     LIBCMT:_trnsctrl_.obj
 0002:00009200       ?ProcessVerifier@NativeDll@<CrtImplementationDetails>@@0IB 1010c200     LIBCMT:_trnsctrl_.obj
 0002:00009208       ??_7type_info@@6B@         1010c208     LIBCMT:typinfo.obj
 0002:00009210       ??_7exception@std@@6B@     1010c210     LIBCMT:stdexcpt.obj
 0002:00009218       ??_C@_0BC@EOODALEL@Unknown?5exception?$AA@ 1010c218     LIBCMT:stdexcpt.obj
 0002:00009230       ??_7bad_cast@std@@6B@      1010c230     LIBCMT:stdexcpt.obj
 0002:0000923c       ??_7bad_typeid@std@@6B@    1010c23c     LIBCMT:stdexcpt.obj
 0002:00009248       ??_7__non_rtti_object@std@@6B@ 1010c248     LIBCMT:stdexcpt.obj
 0002:00009358       ??_C@_1FK@PGACCAFB@?$AAR?$AA6?$AA0?$AA0?$AA2?$AA?$AN?$AA?6?$AA?9?$AA?5?$AAf?$AAl?$AAo?$AAa?$AAt?$AAi?$AAn?$AAg?$AA?5?$AAp?$AAo?$AAi?$AAn?$AAt?$AA?5?$AAs?$AAu?$AAp?$AAp?$AAo?$AAr?$AAt?$AA?5@ 1010c358     LIBCMT:crt0msg.obj
 0002:000093b8       ??_C@_1FE@LLNEDJMD@?$AAR?$AA6?$AA0?$AA0?$AA8?$AA?$AN?$AA?6?$AA?9?$AA?5?$AAn?$AAo?$AAt?$AA?5?$AAe?$AAn?$AAo?$AAu?$AAg?$AAh?$AA?5?$AAs?$AAp?$AAa?$AAc?$AAe?$AA?5?$AAf?$AAo?$AAr?$AA?5?$AAa?$AAr@ 1010c3b8     LIBCMT:crt0msg.obj
 0002:00009410       ??_C@_1FI@HONFMGBI@?$AAR?$AA6?$AA0?$AA0?$AA9?$AA?$AN?$AA?6?$AA?9?$AA?5?$AAn?$AAo?$AAt?$AA?5?$AAe?$AAn?$AAo?$AAu?$AAg?$AAh?$AA?5?$AAs?$AAp?$AAa?$AAc?$AAe?$AA?5?$AAf?$AAo?$AAr?$AA?5?$AAe?$AAn@ 1010c410     LIBCMT:crt0msg.obj
 0002:00009468       ??_C@_1EG@BEHAGFJD@?$AAR?$AA6?$AA0?$AA1?$AA0?$AA?$AN?$AA?6?$AA?9?$AA?5?$AAa?$AAb?$AAo?$AAr?$AAt?$AA?$CI?$AA?$CJ?$AA?5?$AAh?$AAa?$AAs?$AA?5?$AAb?$AAe?$AAe?$AAn?$AA?5?$AAc?$AAa?$AAl?$AAl?$AAe?$AAd@ 1010c468     LIBCMT:crt0msg.obj
 0002:000094b0       ??_C@_1FI@LOGNIKDM@?$AAR?$AA6?$AA0?$AA1?$AA6?$AA?$AN?$AA?6?$AA?9?$AA?5?$AAn?$AAo?$AAt?$AA?5?$AAe?$AAn?$AAo?$AAu?$AAg?$AAh?$AA?5?$AAs?$AAp?$AAa?$AAc?$AAe?$AA?5?$AAf?$AAo?$AAr?$AA?5?$AAt?$AAh@ 1010c4b0     LIBCMT:crt0msg.obj
 0002:00009508       ??_C@_1FK@BEOGODMC@?$AAR?$AA6?$AA0?$AA1?$AA7?$AA?$AN?$AA?6?$AA?9?$AA?5?$AAu?$AAn?$AAe?$AAx?$AAp?$AAe?$AAc?$AAt?$AAe?$AAd?$AA?5?$AAm?$AAu?$AAl?$AAt?$AAi?$AAt?$AAh?$AAr?$AAe?$AAa?$AAd?$AA?5@ 1010c508     LIBCMT:crt0msg.obj
 0002:00009568       ??_C@_1EC@JIBHAOPH@?$AAR?$AA6?$AA0?$AA1?$AA8?$AA?$AN?$AA?6?$AA?9?$AA?5?$AAu?$AAn?$AAe?$AAx?$AAp?$AAe?$AAc?$AAt?$AAe?$AAd?$AA?5?$AAh?$AAe?$AAa?$AAp?$AA?5?$AAe?$AAr?$AAr?$AAo?$AAr?$AA?$AN?$AA?6@ 1010c568     LIBCMT:crt0msg.obj
 0002:000095b0       ??_C@_1FC@ECHBIFBC@?$AAR?$AA6?$AA0?$AA1?$AA9?$AA?$AN?$AA?6?$AA?9?$AA?5?$AAu?$AAn?$AAa?$AAb?$AAl?$AAe?$AA?5?$AAt?$AAo?$AA?5?$AAo?$AAp?$AAe?$AAn?$AA?5?$AAc?$AAo?$AAn?$AAs?$AAo?$AAl?$AAe?$AA?5@ 1010c5b0     LIBCMT:crt0msg.obj
 0002:00009608       ??_C@_1GK@FHCKBEFA@?$AAR?$AA6?$AA0?$AA2?$AA4?$AA?$AN?$AA?6?$AA?9?$AA?5?$AAn?$AAo?$AAt?$AA?5?$AAe?$AAn?$AAo?$AAu?$AAg?$AAh?$AA?5?$AAs?$AAp?$AAa?$AAc?$AAe?$AA?5?$AAf?$AAo?$AAr?$AA?5?$AA_?$AAo@ 1010c608     LIBCMT:crt0msg.obj
 0002:00009678       ??_C@_1EM@MAADIHMB@?$AAR?$AA6?$AA0?$AA2?$AA5?$AA?$AN?$AA?6?$AA?9?$AA?5?$AAp?$AAu?$AAr?$AAe?$AA?5?$AAv?$AAi?$AAr?$AAt?$AAu?$AAa?$AAl?$AA?5?$AAf?$AAu?$AAn?$AAc?$AAt?$AAi?$AAo?$AAn?$AA?5?$AAc@ 1010c678     LIBCMT:crt0msg.obj
 0002:000096c8       ??_C@_1GK@MCAAGJMO@?$AAR?$AA6?$AA0?$AA2?$AA6?$AA?$AN?$AA?6?$AA?9?$AA?5?$AAn?$AAo?$AAt?$AA?5?$AAe?$AAn?$AAo?$AAu?$AAg?$AAh?$AA?5?$AAs?$AAp?$AAa?$AAc?$AAe?$AA?5?$AAf?$AAo?$AAr?$AA?5?$AAs?$AAt@ 1010c6c8     LIBCMT:crt0msg.obj
 0002:00009738       ??_C@_1GK@MFGOKLAG@?$AAR?$AA6?$AA0?$AA2?$AA7?$AA?$AN?$AA?6?$AA?9?$AA?5?$AAn?$AAo?$AAt?$AA?5?$AAe?$AAn?$AAo?$AAu?$AAg?$AAh?$AA?5?$AAs?$AAp?$AAa?$AAc?$AAe?$AA?5?$AAf?$AAo?$AAr?$AA?5?$AAl?$AAo@ 1010c738     LIBCMT:crt0msg.obj
 0002:000097a8       ??_C@_1EK@HHFLMAOL@?$AAR?$AA6?$AA0?$AA2?$AA8?$AA?$AN?$AA?6?$AA?9?$AA?5?$AAu?$AAn?$AAa?$AAb?$AAl?$AAe?$AA?5?$AAt?$AAo?$AA?5?$AAi?$AAn?$AAi?$AAt?$AAi?$AAa?$AAl?$AAi?$AAz?$AAe?$AA?5?$AAh?$AAe@ 1010c7a8     LIBCMT:crt0msg.obj
 0002:000097f4       ??_C@_1DO@BMFCDCD@?$AAR?$AA6?$AA0?$AA3?$AA0?$AA?$AN?$AA?6?$AA?9?$AA?5?$AAC?$AAR?$AAT?$AA?5?$AAn?$AAo?$AAt?$AA?5?$AAi?$AAn?$AAi?$AAt?$AAi?$AAa?$AAl?$AAi?$AAz?$AAe?$AAd?$AA?$AN?$AA?6?$AA?$AA@ 1010c7f4     LIBCMT:crt0msg.obj
 0002:00009838       ??_C@_1MG@ENCOOIDF@?$AAR?$AA6?$AA0?$AA3?$AA1?$AA?$AN?$AA?6?$AA?9?$AA?5?$AAA?$AAt?$AAt?$AAe?$AAm?$AAp?$AAt?$AA?5?$AAt?$AAo?$AA?5?$AAi?$AAn?$AAi?$AAt?$AAi?$AAa?$AAl?$AAi?$AAz?$AAe?$AA?5?$AAt@ 1010c838     LIBCMT:crt0msg.obj
 0002:00009900       ??_C@_1GG@GOPILAJP@?$AAR?$AA6?$AA0?$AA3?$AA2?$AA?$AN?$AA?6?$AA?9?$AA?5?$AAn?$AAo?$AAt?$AA?5?$AAe?$AAn?$AAo?$AAu?$AAg?$AAh?$AA?5?$AAs?$AAp?$AAa?$AAc?$AAe?$AA?5?$AAf?$AAo?$AAr?$AA?5?$AAl?$AAo@ 1010c900     LIBCMT:crt0msg.obj
 0002:00009968       ??_C@_1BOO@KGEDBGAJ@?$AAR?$AA6?$AA0?$AA3?$AA3?$AA?$AN?$AA?6?$AA?9?$AA?5?$AAA?$AAt?$AAt?$AAe?$AAm?$AAp?$AAt?$AA?5?$AAt?$AAo?$AA?5?$AAu?$AAs?$AAe?$AA?5?$AAM?$AAS?$AAI?$AAL?$AA?5?$AAc?$AAo?$AAd@ 1010c968     LIBCMT:crt0msg.obj
 0002:00009b58       ??_C@_1GG@MKFPEKFO@?$AAR?$AA6?$AA0?$AA3?$AA4?$AA?$AN?$AA?6?$AA?9?$AA?5?$AAi?$AAn?$AAc?$AAo?$AAn?$AAs?$AAi?$AAs?$AAt?$AAe?$AAn?$AAt?$AA?5?$AAo?$AAn?$AAe?$AAx?$AAi?$AAt?$AA?5?$AAb?$AAe?$AAg@ 1010cb58     LIBCMT:crt0msg.obj
 0002:00009bc0       ??_C@_1BO@BFCDCGC@?$AAD?$AAO?$AAM?$AAA?$AAI?$AAN?$AA?5?$AAe?$AAr?$AAr?$AAo?$AAr?$AA?$AN?$AA?6?$AA?$AA@ 1010cbc0     LIBCMT:crt0msg.obj
 0002:00009be0       ??_C@_1BK@KMOMNAAI@?$AAS?$AAI?$AAN?$AAG?$AA?5?$AAe?$AAr?$AAr?$AAo?$AAr?$AA?$AN?$AA?6?$AA?$AA@ 1010cbe0     LIBCMT:crt0msg.obj
 0002:00009bfc       ??_C@_1BM@JBBEPPHI@?$AAT?$AAL?$AAO?$AAS?$AAS?$AA?5?$AAe?$AAr?$AAr?$AAo?$AAr?$AA?$AN?$AA?6?$AA?$AA@ 1010cbfc     LIBCMT:crt0msg.obj
 0002:00009c18       ??_C@_15JNBOKNOG@?$AA?$AN?$AA?6?$AA?$AA@ 1010cc18     LIBCMT:crt0msg.obj
 0002:00009c20       ??_C@_1BO@BKOMIGKJ@?$AAr?$AAu?$AAn?$AAt?$AAi?$AAm?$AAe?$AA?5?$AAe?$AAr?$AAr?$AAo?$AAr?$AA?5?$AA?$AA@ 1010cc20     LIBCMT:crt0msg.obj
 0002:00009c40       ??_C@_1DE@JNGNBFGO@?$AAR?$AAu?$AAn?$AAt?$AAi?$AAm?$AAe?$AA?5?$AAE?$AAr?$AAr?$AAo?$AAr?$AA?$CB?$AA?6?$AA?6?$AAP?$AAr?$AAo?$AAg?$AAr?$AAa?$AAm?$AA?3?$AA?5?$AA?$AA@ 1010cc40     LIBCMT:crt0msg.obj
 0002:00009c74       ??_C@_05KLBDPFGC@e?$CL000?$AA@ 1010cc74     LIBCMT:cvt.obj
 0002:00009c7c       ??_C@_04FJHINJAO@tanh?$AA@ 1010cc7c     LIBCMT:fpexcept.obj
 0002:00009c84       ??_C@_04FIHNOPOL@asin?$AA@ 1010cc84     LIBCMT:fpexcept.obj
 0002:00009c8c       ??_C@_04PDIFKINK@acos?$AA@ 1010cc8c     LIBCMT:fpexcept.obj
 0002:00009c94       ??_C@_04MLLJIGOK@atan?$AA@ 1010cc94     LIBCMT:fpexcept.obj
 0002:00009c9c       ??_C@_05KNGEOGJB@atan2?$AA@ 1010cc9c     LIBCMT:fpexcept.obj
 0002:00009ca4       ??_C@_04EIAKFFMI@sqrt?$AA@ 1010cca4     LIBCMT:fpexcept.obj
 0002:00009cac       ??_C@_03BLEJJJBH@sin?$AA@  1010ccac     LIBCMT:fpexcept.obj
 0002:00009cb0       ??_C@_03LALBNOCG@cos?$AA@  1010ccb0     LIBCMT:fpexcept.obj
 0002:00009cb4       ??_C@_03IIINPABG@tan?$AA@  1010ccb4     LIBCMT:fpexcept.obj
 0002:00009cb8       ??_C@_04GFPJNGEK@ceil?$AA@ 1010ccb8     LIBCMT:fpexcept.obj
 0002:00009cc0       ??_C@_05PBJFFIGL@floor?$AA@ 1010ccc0     LIBCMT:fpexcept.obj
 0002:00009cc8       ??_C@_04ODHECPBC@fabs?$AA@ 1010ccc8     LIBCMT:fpexcept.obj
 0002:00009cd0       ??_C@_04EHEDPDJG@modf?$AA@ 1010ccd0     LIBCMT:fpexcept.obj
 0002:00009cd8       ??_C@_05CEJMAHNP@ldexp?$AA@ 1010ccd8     LIBCMT:fpexcept.obj
 0002:00009ce0       ??_C@_05KBKMEMPO@_cabs?$AA@ 1010cce0     LIBCMT:fpexcept.obj
 0002:00009ce8       ??_C@_06MEIMCGCF@_hypot?$AA@ 1010cce8     LIBCMT:fpexcept.obj
 0002:00009cf0       ??_C@_04KEPJIHGP@fmod?$AA@ 1010ccf0     LIBCMT:fpexcept.obj
 0002:00009cf8       ??_C@_05GKKHEGJL@frexp?$AA@ 1010ccf8     LIBCMT:fpexcept.obj
 0002:00009d00       ??_C@_03MJLDFKDL@_y0?$AA@  1010cd00     LIBCMT:fpexcept.obj
 0002:00009d04       ??_C@_03NAKIGLHK@_y1?$AA@  1010cd04     LIBCMT:fpexcept.obj
 0002:00009d08       ??_C@_03ONILCKOB@_yn?$AA@  1010cd08     LIBCMT:fpexcept.obj
 0002:00009d0c       ??_C@_05JGDBENOH@_logb?$AA@ 1010cd0c     LIBCMT:fpexcept.obj
 0002:00009d14       ??_C@_0L@KDOEJCKC@_nextafter?$AA@ 1010cd14     LIBCMT:fpexcept.obj
 0002:00009d20       ??_C@_03KHJOGHMM@exp?$AA@  1010cd20     LIBCMT:fpexcept.obj
 0002:00009d24       ??_C@_03JGHBODFD@pow?$AA@  1010cd24     LIBCMT:fpexcept.obj
 0002:00009d28       ??_C@_03MGHMBJCF@log?$AA@  1010cd28     LIBCMT:fpexcept.obj
 0002:00009d2c       ??_C@_05HGHHAHAP@log10?$AA@ 1010cd2c     LIBCMT:fpexcept.obj
 0002:00009d34       ??_C@_04COOMCNPB@sinh?$AA@ 1010cd34     LIBCMT:fpexcept.obj
 0002:00009d3c       ??_C@_04HPJJNFIM@cosh?$AA@ 1010cd3c     LIBCMT:fpexcept.obj
 0002:00009d44       ??_C@_1BK@MGMFAEKH@?$AAk?$AAe?$AAr?$AAn?$AAe?$AAl?$AA3?$AA2?$AA?4?$AAd?$AAl?$AAl?$AA?$AA@ 1010cd44     LIBCMT:winapisupp.obj
 0002:00009d60       ??_C@_08KNHFBNJ@FlsAlloc?$AA@ 1010cd60     LIBCMT:winapisupp.obj
 0002:00009d6c       ??_C@_07PEJMOBNF@FlsFree?$AA@ 1010cd6c     LIBCMT:winapisupp.obj
 0002:00009d74       ??_C@_0M@GDNOONDI@FlsGetValue?$AA@ 1010cd74     LIBCMT:winapisupp.obj
 0002:00009d80       ??_C@_0M@JCPCPOEF@FlsSetValue?$AA@ 1010cd80     LIBCMT:winapisupp.obj
 0002:00009d8c       ??_C@_0BM@HCFOFFN@InitializeCriticalSectionEx?$AA@ 1010cd8c     LIBCMT:winapisupp.obj
 0002:00009da8       ??_C@_0P@DLHPPCNH@CreateEventExW?$AA@ 1010cda8     LIBCMT:winapisupp.obj
 0002:00009db8       ??_C@_0BD@KIEEOEEH@CreateSemaphoreExW?$AA@ 1010cdb8     LIBCMT:winapisupp.obj
 0002:00009dcc       ??_C@_0BI@BKLFFAPO@SetThreadStackGuarantee?$AA@ 1010cdcc     LIBCMT:winapisupp.obj
 0002:00009de4       ??_C@_0BG@OGFAJCKC@CreateThreadpoolTimer?$AA@ 1010cde4     LIBCMT:winapisupp.obj
 0002:00009dfc       ??_C@_0BD@LPLEMMDI@SetThreadpoolTimer?$AA@ 1010cdfc     LIBCMT:winapisupp.obj
 0002:00009e10       ??_C@_0CA@FMNJENH@WaitForThreadpoolTimerCallbacks?$AA@ 1010ce10     LIBCMT:winapisupp.obj
 0002:00009e30       ??_C@_0BF@DCFCCNOC@CloseThreadpoolTimer?$AA@ 1010ce30     LIBCMT:winapisupp.obj
 0002:00009e48       ??_C@_0BF@FLABGKKM@CreateThreadpoolWait?$AA@ 1010ce48     LIBCMT:winapisupp.obj
 0002:00009e60       ??_C@_0BC@MGCOHNA@SetThreadpoolWait?$AA@ 1010ce60     LIBCMT:winapisupp.obj
 0002:00009e74       ??_C@_0BE@OCIOMIMP@CloseThreadpoolWait?$AA@ 1010ce74     LIBCMT:winapisupp.obj
 0002:00009e88       ??_C@_0BJ@LKGHFHBO@FlushProcessWriteBuffers?$AA@ 1010ce88     LIBCMT:winapisupp.obj
 0002:00009ea4       ??_C@_0BP@KALKKPMO@FreeLibraryWhenCallbackReturns?$AA@ 1010cea4     LIBCMT:winapisupp.obj
 0002:00009ec4       ??_C@_0BK@DFNBACLA@GetCurrentProcessorNumber?$AA@ 1010cec4     LIBCMT:winapisupp.obj
 0002:00009ee0       ??_C@_0BP@KHGALBC@GetLogicalProcessorInformation?$AA@ 1010cee0     LIBCMT:winapisupp.obj
 0002:00009f00       ??_C@_0BE@FKKLLFLM@CreateSymbolicLinkW?$AA@ 1010cf00     LIBCMT:winapisupp.obj
 0002:00009f14       ??_C@_0BJ@OHNKDLIJ@SetDefaultDllDirectories?$AA@ 1010cf14     LIBCMT:winapisupp.obj
 0002:00009f30       ??_C@_0BE@LJANKFHF@EnumSystemLocalesEx?$AA@ 1010cf30     LIBCMT:winapisupp.obj
 0002:00009f44       ??_C@_0BA@IHGNDAEB@CompareStringEx?$AA@ 1010cf44     LIBCMT:winapisupp.obj
 0002:00009f54       ??_C@_0BA@EPCJIIPD@GetDateFormatEx?$AA@ 1010cf54     LIBCMT:winapisupp.obj
 0002:00009f64       ??_C@_0BA@ONOKGCMP@GetLocaleInfoEx?$AA@ 1010cf64     LIBCMT:winapisupp.obj
 0002:00009f74       ??_C@_0BA@CIJJKCJJ@GetTimeFormatEx?$AA@ 1010cf74     LIBCMT:winapisupp.obj
 0002:00009f84       ??_C@_0BJ@PBCCBIPI@GetUserDefaultLocaleName?$AA@ 1010cf84     LIBCMT:winapisupp.obj
 0002:00009fa0       ??_C@_0BC@CELBKLLA@IsValidLocaleName?$AA@ 1010cfa0     LIBCMT:winapisupp.obj
 0002:00009fb4       ??_C@_0O@KKBNKAPF@LCMapStringEx?$AA@ 1010cfb4     LIBCMT:winapisupp.obj
 0002:00009fc4       ??_C@_0BE@JOGNEJCI@GetCurrentPackageId?$AA@ 1010cfc4     LIBCMT:winapisupp.obj
 0002:00009fd8       ??_C@_0P@CDHHOHKP@GetTickCount64?$AA@ 1010cfd8     LIBCMT:winapisupp.obj
 0002:00009fe8       ??_C@_0BO@KPCLFDJJ@GetFileInformationByHandleExW?$AA@ 1010cfe8     LIBCMT:winapisupp.obj
 0002:0000a008       ??_C@_0BM@MHIDLABK@SetFileInformationByHandleW?$AA@ 1010d008     LIBCMT:winapisupp.obj
 0002:0000a024       ??_C@_1BK@GAEMIDIL@?$AAA?$AAD?$AAV?$AAA?$AAP?$AAI?$AA3?$AA2?$AA?4?$AAD?$AAL?$AAL?$AA?$AA@ 1010d024     LIBCMT:rand_s.obj
 0002:0000a040       ??_C@_0BC@JEAENNKH@SystemFunction036?$AA@ 1010d040     LIBCMT:rand_s.obj
 0002:0000a064       ??_C@_1M@HPNHIDJI@?$AAj?$AAa?$AA?9?$AAJ?$AAP?$AA?$AA@ 1010d064     LIBCMT:mbctype.obj
 0002:0000a070       ??_C@_1M@BIBDDEMK@?$AAz?$AAh?$AA?9?$AAC?$AAN?$AA?$AA@ 1010d070     LIBCMT:mbctype.obj
 0002:0000a07c       ??_C@_1M@JLOOOEGK@?$AAk?$AAo?$AA?9?$AAK?$AAR?$AA?$AA@ 1010d07c     LIBCMT:mbctype.obj
 0002:0000a088       ??_C@_1M@CLNBBOPM@?$AAz?$AAh?$AA?9?$AAT?$AAW?$AA?$AA@ 1010d088     LIBCMT:mbctype.obj
 0002:0000a0b4       ??_C@_06OJHGLDPL@?$CInull?$CJ?$AA@ 1010d0b4     LIBCMT:output.obj
 0002:0000a0bc       ??_C@_1O@CEDCILHN@?$AA?$CI?$AAn?$AAu?$AAl?$AAl?$AA?$CJ?$AA?$AA@ 1010d0bc     LIBCMT:output.obj
 0002:0000a0d0       ___lookuptable             1010d0d0     LIBCMT:output.obj
 0002:0000a12c       ??_C@_1BG@GOEBHBDC@?$AAU?$AAS?$AAE?$AAR?$AA3?$AA2?$AA?4?$AAD?$AAL?$AAL?$AA?$AA@ 1010d12c     LIBCMT:crtmboxw.obj
 0002:0000a144       ??_C@_0M@DLDCCGNP@MessageBoxW?$AA@ 1010d144     LIBCMT:crtmboxw.obj
 0002:0000a150       ??_C@_0BA@HNOPNCHB@GetActiveWindow?$AA@ 1010d150     LIBCMT:crtmboxw.obj
 0002:0000a160       ??_C@_0BD@HHGDFDBJ@GetLastActivePopup?$AA@ 1010d160     LIBCMT:crtmboxw.obj
 0002:0000a174       ??_C@_0BK@DEKFELLI@GetUserObjectInformationW?$AA@ 1010d174     LIBCMT:crtmboxw.obj
 0002:0000a190       ??_C@_0BI@DFKBFLJE@GetProcessWindowStation?$AA@ 1010d190     LIBCMT:crtmboxw.obj
 0002:0000a1a8       __XcptActTab               1010d1a8     LIBCMT:winxfltr.obj
 0002:0000a238       __XcptActTabCount          1010d238     LIBCMT:winxfltr.obj
 0002:0000a23c       __XcptActTabSize           1010d23c     LIBCMT:winxfltr.obj
 0002:0000a240       __First_FPE_Indx           1010d240     LIBCMT:winxfltr.obj
 0002:0000a244       __Num_FPE                  1010d244     LIBCMT:winxfltr.obj
 0002:0000a248       __pDestructExceptionObject 1010d248     LIBCMT:frame.obj
 0002:0000a250       ??_7bad_exception@std@@6B@ 1010d250     LIBCMT:frame.obj
 0002:0000a258       ??_C@_0O@DPKOEFFH@bad?5exception?$AA@ 1010d258     LIBCMT:frame.obj
 0002:0000a2d0       ??_C@_05EOHGHCHD@exp10?$AA@ 1010d2d0     LIBCMT:libm_error.obj
 0002:0000a2d8       ??_C@_03KOEHGMDN@Sun?$AA@  1010d2d8     LIBCMT:nlsdata.obj
 0002:0000a2dc       ??_C@_03PDAGKDH@Mon?$AA@   1010d2dc     LIBCMT:nlsdata.obj
 0002:0000a2e0       ??_C@_03NAGEINEP@Tue?$AA@  1010d2e0     LIBCMT:nlsdata.obj
 0002:0000a2e4       ??_C@_03MHOMLAJA@Wed?$AA@  1010d2e4     LIBCMT:nlsdata.obj
 0002:0000a2e8       ??_C@_03IOFIKPDN@Thu?$AA@  1010d2e8     LIBCMT:nlsdata.obj
 0002:0000a2ec       ??_C@_03IDIOELNC@Fri?$AA@  1010d2ec     LIBCMT:nlsdata.obj
 0002:0000a2f0       ??_C@_03FEFJNEK@Sat?$AA@   1010d2f0     LIBCMT:nlsdata.obj
 0002:0000a2f4       ??_C@_06OOPIFAJ@Sunday?$AA@ 1010d2f4     LIBCMT:nlsdata.obj
 0002:0000a2fc       ??_C@_06JLEDEDGH@Monday?$AA@ 1010d2fc     LIBCMT:nlsdata.obj
 0002:0000a304       ??_C@_07BAAGCFCM@Tuesday?$AA@ 1010d304     LIBCMT:nlsdata.obj
 0002:0000a30c       ??_C@_09DLIGFAKA@Wednesday?$AA@ 1010d30c     LIBCMT:nlsdata.obj
 0002:0000a318       ??_C@_08HACCIKIA@Thursday?$AA@ 1010d318     LIBCMT:nlsdata.obj
 0002:0000a324       ??_C@_06JECMNKMI@Friday?$AA@ 1010d324     LIBCMT:nlsdata.obj
 0002:0000a32c       ??_C@_08INBOOONO@Saturday?$AA@ 1010d32c     LIBCMT:nlsdata.obj
 0002:0000a338       ??_C@_03JIHJHPIE@Jan?$AA@  1010d338     LIBCMT:nlsdata.obj
 0002:0000a33c       ??_C@_03HJBDCHOM@Feb?$AA@  1010d33c     LIBCMT:nlsdata.obj
 0002:0000a340       ??_C@_03ODNJBKGA@Mar?$AA@  1010d340     LIBCMT:nlsdata.obj
 0002:0000a344       ??_C@_03LEOLGMJP@Apr?$AA@  1010d344     LIBCMT:nlsdata.obj
 0002:0000a348       ??_C@_03CNMDKL@May?$AA@    1010d348     LIBCMT:nlsdata.obj
 0002:0000a34c       ??_C@_03IDFGHECI@Jun?$AA@  1010d34c     LIBCMT:nlsdata.obj
 0002:0000a350       ??_C@_03LBGABGKK@Jul?$AA@  1010d350     LIBCMT:nlsdata.obj
 0002:0000a354       ??_C@_03IFJFEIGA@Aug?$AA@  1010d354     LIBCMT:nlsdata.obj
 0002:0000a358       ??_C@_03GGCAPAJC@Sep?$AA@  1010d358     LIBCMT:nlsdata.obj
 0002:0000a35c       ??_C@_03BMAOKBAD@Oct?$AA@  1010d35c     LIBCMT:nlsdata.obj
 0002:0000a360       ??_C@_03JPJOFNIA@Nov?$AA@  1010d360     LIBCMT:nlsdata.obj
 0002:0000a364       ??_C@_03MKABNOCG@Dec?$AA@  1010d364     LIBCMT:nlsdata.obj
 0002:0000a368       ??_C@_07CGJPFGJA@January?$AA@ 1010d368     LIBCMT:nlsdata.obj
 0002:0000a370       ??_C@_08GNJGEPFN@February?$AA@ 1010d370     LIBCMT:nlsdata.obj
 0002:0000a37c       ??_C@_05HPCKOFNC@March?$AA@ 1010d37c     LIBCMT:nlsdata.obj
 0002:0000a384       ??_C@_05DMJDNLEJ@April?$AA@ 1010d384     LIBCMT:nlsdata.obj
 0002:0000a38c       ??_C@_04CNLMGBGM@June?$AA@ 1010d38c     LIBCMT:nlsdata.obj
 0002:0000a394       ??_C@_04MIEPOIFP@July?$AA@ 1010d394     LIBCMT:nlsdata.obj
 0002:0000a39c       ??_C@_06LBBHFDDG@August?$AA@ 1010d39c     LIBCMT:nlsdata.obj
 0002:0000a3a4       ??_C@_09BHHEALKD@September?$AA@ 1010d3a4     LIBCMT:nlsdata.obj
 0002:0000a3b0       ??_C@_07JJNFCEND@October?$AA@ 1010d3b0     LIBCMT:nlsdata.obj
 0002:0000a3b8       ??_C@_08HCHEGEOA@November?$AA@ 1010d3b8     LIBCMT:nlsdata.obj
 0002:0000a3c4       ??_C@_08EDHMEBNP@December?$AA@ 1010d3c4     LIBCMT:nlsdata.obj
 0002:0000a3d0       ??_C@_02DEDBPAFC@AM?$AA@   1010d3d0     LIBCMT:nlsdata.obj
 0002:0000a3d4       ??_C@_02CJNFDJBF@PM?$AA@   1010d3d4     LIBCMT:nlsdata.obj
 0002:0000a3d8       ??_C@_08BPBNCDIB@MM?1dd?1yy?$AA@ 1010d3d8     LIBCMT:nlsdata.obj
 0002:0000a3e4       ??_C@_0BE@CKGJFCPC@dddd?0?5MMMM?5dd?0?5yyyy?$AA@ 1010d3e4     LIBCMT:nlsdata.obj
 0002:0000a3f8       ??_C@_08JCCMCCIL@HH?3mm?3ss?$AA@ 1010d3f8     LIBCMT:nlsdata.obj
 0002:0000a404       ??_C@_17MBGCMIPB@?$AAS?$AAu?$AAn?$AA?$AA@ 1010d404     LIBCMT:nlsdata.obj
 0002:0000a40c       ??_C@_17KBOMKBF@?$AAM?$AAo?$AAn?$AA?$AA@ 1010d40c     LIBCMT:nlsdata.obj
 0002:0000a414       ??_C@_17BMKGEGOJ@?$AAT?$AAu?$AAe?$AA?$AA@ 1010d414     LIBCMT:nlsdata.obj
 0002:0000a41c       ??_C@_17CJEDCEPE@?$AAW?$AAe?$AAd?$AA?$AA@ 1010d41c     LIBCMT:nlsdata.obj
 0002:0000a424       ??_C@_17PDPHAADD@?$AAT?$AAh?$AAu?$AA?$AA@ 1010d424     LIBCMT:nlsdata.obj
 0002:0000a42c       ??_C@_17HFOLPPLP@?$AAF?$AAr?$AAi?$AA?$AA@ 1010d42c     LIBCMT:nlsdata.obj
 0002:0000a434       ??_C@_17GGIBDPIH@?$AAS?$AAa?$AAt?$AA?$AA@ 1010d434     LIBCMT:nlsdata.obj
 0002:0000a43c       ??_C@_1O@IHNHDHPB@?$AAS?$AAu?$AAn?$AAd?$AAa?$AAy?$AA?$AA@ 1010d43c     LIBCMT:nlsdata.obj
 0002:0000a44c       ??_C@_1O@MMNBFLIA@?$AAM?$AAo?$AAn?$AAd?$AAa?$AAy?$AA?$AA@ 1010d44c     LIBCMT:nlsdata.obj
 0002:0000a45c       ??_C@_1BA@ENFBFFEK@?$AAT?$AAu?$AAe?$AAs?$AAd?$AAa?$AAy?$AA?$AA@ 1010d45c     LIBCMT:nlsdata.obj
 0002:0000a46c       ??_C@_1BE@EBOGMDOH@?$AAW?$AAe?$AAd?$AAn?$AAe?$AAs?$AAd?$AAa?$AAy?$AA?$AA@ 1010d46c     LIBCMT:nlsdata.obj
 0002:0000a480       ??_C@_1BC@HHMNLIHE@?$AAT?$AAh?$AAu?$AAr?$AAs?$AAd?$AAa?$AAy?$AA?$AA@ 1010d480     LIBCMT:nlsdata.obj
 0002:0000a494       ??_C@_1O@PDICJHAG@?$AAF?$AAr?$AAi?$AAd?$AAa?$AAy?$AA?$AA@ 1010d494     LIBCMT:nlsdata.obj
 0002:0000a4a4       ??_C@_1BC@ENMNNPAJ@?$AAS?$AAa?$AAt?$AAu?$AAr?$AAd?$AAa?$AAy?$AA?$AA@ 1010d4a4     LIBCMT:nlsdata.obj
 0002:0000a4b8       ??_C@_17DKNBKCHM@?$AAJ?$AAa?$AAn?$AA?$AA@ 1010d4b8     LIBCMT:nlsdata.obj
 0002:0000a4c0       ??_C@_17LMDJEKJN@?$AAF?$AAe?$AAb?$AA?$AA@ 1010d4c0     LIBCMT:nlsdata.obj
 0002:0000a4c8       ??_C@_17CKNLEDEC@?$AAM?$AAa?$AAr?$AA?$AA@ 1010d4c8     LIBCMT:nlsdata.obj
 0002:0000a4d0       ??_C@_17LFPOIHDD@?$AAA?$AAp?$AAr?$AA?$AA@ 1010d4d0     LIBCMT:nlsdata.obj
 0002:0000a4d8       ??_C@_17PNNKMEED@?$AAM?$AAa?$AAy?$AA?$AA@ 1010d4d8     LIBCMT:nlsdata.obj
 0002:0000a4e0       ??_C@_17KCJGOCPB@?$AAJ?$AAu?$AAn?$AA?$AA@ 1010d4e0     LIBCMT:nlsdata.obj
 0002:0000a4e8       ??_C@_17IJPCKHK@?$AAJ?$AAu?$AAl?$AA?$AA@ 1010d4e8     LIBCMT:nlsdata.obj
 0002:0000a4f0       ??_C@_17ICPELBCN@?$AAA?$AAu?$AAg?$AA?$AA@ 1010d4f0     LIBCMT:nlsdata.obj
 0002:0000a4f8       ??_C@_17HCHCOKMG@?$AAS?$AAe?$AAp?$AA?$AA@ 1010d4f8     LIBCMT:nlsdata.obj
 0002:0000a500       ??_C@_17FNLKOI@?$AAO?$AAc?$AAt?$AA?$AA@ 1010d500     LIBCMT:nlsdata.obj
 0002:0000a508       ??_C@_17BBDMLCIG@?$AAN?$AAo?$AAv?$AA?$AA@ 1010d508     LIBCMT:nlsdata.obj
 0002:0000a510       ??_C@_17EGKACKIF@?$AAD?$AAe?$AAc?$AA?$AA@ 1010d510     LIBCMT:nlsdata.obj
 0002:0000a518       ??_C@_1BA@EFMEIEBA@?$AAJ?$AAa?$AAn?$AAu?$AAa?$AAr?$AAy?$AA?$AA@ 1010d518     LIBCMT:nlsdata.obj
 0002:0000a528       ??_C@_1BC@JGDDFFAM@?$AAF?$AAe?$AAb?$AAr?$AAu?$AAa?$AAr?$AAy?$AA?$AA@ 1010d528     LIBCMT:nlsdata.obj
 0002:0000a53c       ??_C@_1M@IKEENEDF@?$AAM?$AAa?$AAr?$AAc?$AAh?$AA?$AA@ 1010d53c     LIBCMT:nlsdata.obj
 0002:0000a548       ??_C@_1M@GJNLMHFD@?$AAA?$AAp?$AAr?$AAi?$AAl?$AA?$AA@ 1010d548     LIBCMT:nlsdata.obj
 0002:0000a554       ??_C@_19EPFLPGAP@?$AAJ?$AAu?$AAn?$AAe?$AA?$AA@ 1010d554     LIBCMT:nlsdata.obj
 0002:0000a560       ??_C@_19BIFMLPCD@?$AAJ?$AAu?$AAl?$AAy?$AA?$AA@ 1010d560     LIBCMT:nlsdata.obj
 0002:0000a56c       ??_C@_1O@PAHLKOAC@?$AAA?$AAu?$AAg?$AAu?$AAs?$AAt?$AA?$AA@ 1010d56c     LIBCMT:nlsdata.obj
 0002:0000a57c       ??_C@_1BE@DKAAMBJL@?$AAS?$AAe?$AAp?$AAt?$AAe?$AAm?$AAb?$AAe?$AAr?$AA?$AA@ 1010d57c     LIBCMT:nlsdata.obj
 0002:0000a590       ??_C@_1BA@EPANDLNG@?$AAO?$AAc?$AAt?$AAo?$AAb?$AAe?$AAr?$AA?$AA@ 1010d590     LIBCMT:nlsdata.obj
 0002:0000a5a0       ??_C@_1BC@BGLIFPF@?$AAN?$AAo?$AAv?$AAe?$AAm?$AAb?$AAe?$AAr?$AA?$AA@ 1010d5a0     LIBCMT:nlsdata.obj
 0002:0000a5b4       ??_C@_1BC@FEMKIFH@?$AAD?$AAe?$AAc?$AAe?$AAm?$AAb?$AAe?$AAr?$AA?$AA@ 1010d5b4     LIBCMT:nlsdata.obj
 0002:0000a5c8       ??_C@_15ODEHAHHF@?$AAA?$AAM?$AA?$AA@ 1010d5c8     LIBCMT:nlsdata.obj
 0002:0000a5d0       ??_C@_15CLMNNGEL@?$AAP?$AAM?$AA?$AA@ 1010d5d0     LIBCMT:nlsdata.obj
 0002:0000a5d8       ??_C@_1BC@IEBCMHCM@?$AAM?$AAM?$AA?1?$AAd?$AAd?$AA?1?$AAy?$AAy?$AA?$AA@ 1010d5d8     LIBCMT:nlsdata.obj
 0002:0000a5ec       ??_C@_1CI@KNAKOEBC@?$AAd?$AAd?$AAd?$AAd?$AA?0?$AA?5?$AAM?$AAM?$AAM?$AAM?$AA?5?$AAd?$AAd?$AA?0?$AA?5?$AAy?$AAy?$AAy?$AAy?$AA?$AA@ 1010d5ec     LIBCMT:nlsdata.obj
 0002:0000a614       ??_C@_1BC@GDGBMEMK@?$AAH?$AAH?$AA?3?$AAm?$AAm?$AA?3?$AAs?$AAs?$AA?$AA@ 1010d614     LIBCMT:nlsdata.obj
 0002:0000a628       ??_C@_1M@BMHNFIME@?$AAe?$AAn?$AA?9?$AAU?$AAS?$AA?$AA@ 1010d628     LIBCMT:nlsdata.obj
 0002:0000a638       _LcidToLocaleNameTable     1010d638     LIBCMT:winapinls.obj
 0002:0000ad58       _LocaleNameToIndexTable    1010dd58     LIBCMT:winapinls.obj
 0002:0000b478       ??_C@_15EMKDOKLE@?$AAa?$AAr?$AA?$AA@ 1010e478     LIBCMT:winapinls.obj
 0002:0000b480       ??_C@_15KNPADPLH@?$AAb?$AAg?$AA?$AA@ 1010e480     LIBCMT:winapinls.obj
 0002:0000b488       ??_C@_15EDMHLDMO@?$AAc?$AAa?$AA?$AA@ 1010e488     LIBCMT:winapinls.obj
 0002:0000b490       ??_C@_1O@BPEAJADD@?$AAz?$AAh?$AA?9?$AAC?$AAH?$AAS?$AA?$AA@ 1010e490     LIBCMT:winapinls.obj
 0002:0000b4a0       ??_C@_15LJNHCMNK@?$AAc?$AAs?$AA?$AA@ 1010e4a0     LIBCMT:winapinls.obj
 0002:0000b4a8       ??_C@_15FOMCIDHG@?$AAd?$AAa?$AA?$AA@ 1010e4a8     LIBCMT:winapinls.obj
 0002:0000b4b0       ??_C@_15NBKABECB@?$AAd?$AAe?$AA?$AA@ 1010e4b0     LIBCMT:winapinls.obj
 0002:0000b4b8       ??_C@_15GHPEIIAO@?$AAe?$AAl?$AA?$AA@ 1010e4b8     LIBCMT:winapinls.obj
 0002:0000b4c0       ??_C@_15MNPNEAIF@?$AAe?$AAn?$AA?$AA@ 1010e4c0     LIBCMT:winapinls.obj
 0002:0000b4c8       ??_C@_15GPIOMPMH@?$AAe?$AAs?$AA?$AA@ 1010e4c8     LIBCMT:winapinls.obj
 0002:0000b4d0       ??_C@_15NGLOAKJC@?$AAf?$AAi?$AA?$AA@ 1010e4d0     LIBCMT:winapinls.obj
 0002:0000b4d8       ??_C@_15FBKGNKAM@?$AAf?$AAr?$AA?$AA@ 1010e4d8     LIBCMT:winapinls.obj
 0002:0000b4e0       ??_C@_15KGGCNEFK@?$AAh?$AAe?$AA?$AA@ 1010e4e0     LIBCMT:winapinls.obj
 0002:0000b4e8       ??_C@_15PGHLIDMF@?$AAh?$AAu?$AA?$AA@ 1010e4e8     LIBCMT:winapinls.obj
 0002:0000b4f0       ??_C@_15BIEMAPLM@?$AAi?$AAs?$AA?$AA@ 1010e4f0     LIBCMT:winapinls.obj
 0002:0000b4f8       ??_C@_15IFJLDHAF@?$AAi?$AAt?$AA?$AA@ 1010e4f8     LIBCMT:winapinls.obj
 0002:0000b500       ??_C@_15GEMIOCAG@?$AAj?$AAa?$AA?$AA@ 1010e500     LIBCMT:winapinls.obj
 0002:0000b508       ??_C@_15EPELEGJA@?$AAk?$AAo?$AA?$AA@ 1010e508     LIBCMT:winapinls.obj
 0002:0000b510       ??_C@_15NDDHIMN@?$AAn?$AAl?$AA?$AA@ 1010e510     LIBCMT:winapinls.obj
 0002:0000b518       ??_C@_15BPIGNHCD@?$AAn?$AAo?$AA?$AA@ 1010e518     LIBCMT:winapinls.obj
 0002:0000b520       ??_C@_15DEOPBLCG@?$AAp?$AAl?$AA?$AA@ 1010e520     LIBCMT:winapinls.obj
 0002:0000b528       ??_C@_15KBECGEFG@?$AAp?$AAt?$AA?$AA@ 1010e528     LIBCMT:winapinls.obj
 0002:0000b530       ??_C@_15GLJCBFMD@?$AAr?$AAo?$AA?$AA@ 1010e530     LIBCMT:winapinls.obj
 0002:0000b538       ??_C@_15FEDGKCDI@?$AAr?$AAu?$AA?$AA@ 1010e538     LIBCMT:winapinls.obj
 0002:0000b540       ??_C@_15GLKMLLHM@?$AAh?$AAr?$AA?$AA@ 1010e540     LIBCMT:winapinls.obj
 0002:0000b548       ??_C@_15CPKMFBDB@?$AAs?$AAk?$AA?$AA@ 1010e548     LIBCMT:winapinls.obj
 0002:0000b550       ??_C@_15BAAIOGMK@?$AAs?$AAq?$AA?$AA@ 1010e550     LIBCMT:winapinls.obj
 0002:0000b558       ??_C@_15INNPNOHD@?$AAs?$AAv?$AA?$AA@ 1010e558     LIBCMT:winapinls.obj
 0002:0000b560       ??_C@_15CABMMOGH@?$AAt?$AAh?$AA?$AA@ 1010e560     LIBCMT:winapinls.obj
 0002:0000b568       ??_C@_15BPLIHJJM@?$AAt?$AAr?$AA?$AA@ 1010e568     LIBCMT:winapinls.obj
 0002:0000b570       ??_C@_15NEOEKKDJ@?$AAu?$AAr?$AA?$AA@ 1010e570     LIBCMT:winapinls.obj
 0002:0000b578       ??_C@_15NFICGAJK@?$AAi?$AAd?$AA?$AA@ 1010e578     LIBCMT:winapinls.obj
 0002:0000b580       ??_C@_15PJPFLCCM@?$AAu?$AAk?$AA?$AA@ 1010e580     LIBCMT:winapinls.obj
 0002:0000b588       ??_C@_15HPJPHDM@?$AAb?$AAe?$AA?$AA@ 1010e588     LIBCMT:winapinls.obj
 0002:0000b590       ??_C@_15LCHLGJII@?$AAs?$AAl?$AA?$AA@ 1010e590     LIBCMT:winapinls.obj
 0002:0000b598       ??_C@_15PCFJPHHO@?$AAe?$AAt?$AA?$AA@ 1010e598     LIBCMT:winapinls.obj
 0002:0000b5a0       ??_C@_15HPFPGODN@?$AAl?$AAv?$AA?$AA@ 1010e5a0     LIBCMT:winapinls.obj
 0002:0000b5a8       ??_C@_15NFFGKGLG@?$AAl?$AAt?$AA?$AA@ 1010e5a8     LIBCMT:winapinls.obj
 0002:0000b5b0       ??_C@_15BDAKCCHN@?$AAf?$AAa?$AA?$AA@ 1010e5b0     LIBCMT:winapinls.obj
 0002:0000b5b8       ??_C@_15NFGIAIAJ@?$AAv?$AAi?$AA?$AA@ 1010e5b8     LIBCMT:winapinls.obj
 0002:0000b5c0       ??_C@_15LMKNDMHN@?$AAh?$AAy?$AA?$AA@ 1010e5c0     LIBCMT:winapinls.obj
 0002:0000b5c8       ??_C@_15IJBHMCFL@?$AAa?$AAz?$AA?$AA@ 1010e5c8     LIBCMT:winapinls.obj
 0002:0000b5d0       ??_C@_15EKOFJABL@?$AAe?$AAu?$AA?$AA@ 1010e5d0     LIBCMT:winapinls.obj
 0002:0000b5d8       ??_C@_15BGHADCNK@?$AAm?$AAk?$AA?$AA@ 1010e5d8     LIBCMT:winapinls.obj
 0002:0000b5e0       ??_C@_15JDNICKHM@?$AAa?$AAf?$AA?$AA@ 1010e5e0     LIBCMT:winapinls.obj
 0002:0000b5e8       ??_C@_15KPJEDBKD@?$AAk?$AAa?$AA?$AA@ 1010e5e8     LIBCMT:winapinls.obj
 0002:0000b5f0       ??_C@_15PDNFFFEO@?$AAf?$AAo?$AA?$AA@ 1010e5f0     LIBCMT:winapinls.obj
 0002:0000b5f8       ??_C@_15OMLEGLOC@?$AAh?$AAi?$AA?$AA@ 1010e5f8     LIBCMT:winapinls.obj
 0002:0000b600       ??_C@_15IDNNENKK@?$AAm?$AAs?$AA?$AA@ 1010e600     LIBCMT:winapinls.obj
 0002:0000b608       ??_C@_15MACJNBMH@?$AAk?$AAk?$AA?$AA@ 1010e608     LIBCMT:winapinls.obj
 0002:0000b610       ??_C@_15DKDJEOND@?$AAk?$AAy?$AA?$AA@ 1010e610     LIBCMT:winapinls.obj
 0002:0000b618       ??_C@_15DFGDLJBG@?$AAs?$AAw?$AA?$AA@ 1010e618     LIBCMT:winapinls.obj
 0002:0000b620       ??_C@_15BBFAICNG@?$AAu?$AAz?$AA?$AA@ 1010e620     LIBCMT:winapinls.obj
 0002:0000b628       ??_C@_15DKNDCGEA@?$AAt?$AAt?$AA?$AA@ 1010e628     LIBCMT:winapinls.obj
 0002:0000b630       ??_C@_15MGIFMDPL@?$AAp?$AAa?$AA?$AA@ 1010e630     LIBCMT:winapinls.obj
 0002:0000b638       ??_C@_15HCNDBBA@?$AAg?$AAu?$AA?$AA@ 1010e638     LIBCMT:winapinls.obj
 0002:0000b640       ??_C@_15FNBEIBON@?$AAt?$AAa?$AA?$AA@ 1010e640     LIBCMT:winapinls.obj
 0002:0000b648       ??_C@_15NCHGBGLK@?$AAt?$AAe?$AA?$AA@ 1010e648     LIBCMT:winapinls.obj
 0002:0000b650       ??_C@_15PHPHCBPF@?$AAk?$AAn?$AA?$AA@ 1010e650     LIBCMT:winapinls.obj
 0002:0000b658       ??_C@_15DLGBCKMP@?$AAm?$AAr?$AA?$AA@ 1010e658     LIBCMT:winapinls.obj
 0002:0000b660       ??_C@_15EABBLBFF@?$AAs?$AAa?$AA?$AA@ 1010e660     LIBCMT:winapinls.obj
 0002:0000b668       ??_C@_15CBKOMCOI@?$AAm?$AAn?$AA?$AA@ 1010e668     LIBCMT:winapinls.obj
 0002:0000b670       ??_C@_15CKDMCJAF@?$AAg?$AAl?$AA?$AA@ 1010e670     LIBCMT:winapinls.obj
 0002:0000b678       ??_C@_17CNJFBPG@?$AAk?$AAo?$AAk?$AA?$AA@ 1010e678     LIBCMT:winapinls.obj
 0002:0000b680       ??_C@_17FFBJICPL@?$AAs?$AAy?$AAr?$AA?$AA@ 1010e680     LIBCMT:winapinls.obj
 0002:0000b688       ??_C@_17KPNDCPAF@?$AAd?$AAi?$AAv?$AA?$AA@ 1010e688     LIBCMT:winapinls.obj
 0002:0000b690       ??_C@_11LOCGONAA@?$AA?$AA@ 1010e690     LIBCMT:winapinls.obj
 0002:0000b694       ??_C@_1M@OKAHONE@?$AAa?$AAr?$AA?9?$AAS?$AAA?$AA?$AA@ 1010e694     LIBCMT:winapinls.obj
 0002:0000b6a0       ??_C@_1M@FFFIGIGK@?$AAb?$AAg?$AA?9?$AAB?$AAG?$AA?$AA@ 1010e6a0     LIBCMT:winapinls.obj
 0002:0000b6ac       ??_C@_1M@BJNKEDC@?$AAc?$AAa?$AA?9?$AAE?$AAS?$AA?$AA@ 1010e6ac     LIBCMT:winapinls.obj
 0002:0000b6b8       ??_C@_1M@IJJHFJHA@?$AAc?$AAs?$AA?9?$AAC?$AAZ?$AA?$AA@ 1010e6b8     LIBCMT:winapinls.obj
 0002:0000b6c4       ??_C@_1M@CLPEOBGI@?$AAd?$AAa?$AA?9?$AAD?$AAK?$AA?$AA@ 1010e6c4     LIBCMT:winapinls.obj
 0002:0000b6d0       ??_C@_1M@MCMADGCB@?$AAd?$AAe?$AA?9?$AAD?$AAE?$AA?$AA@ 1010e6d0     LIBCMT:winapinls.obj
 0002:0000b6dc       ??_C@_1M@OOCKEMAM@?$AAe?$AAl?$AA?9?$AAG?$AAR?$AA?$AA@ 1010e6dc     LIBCMT:winapinls.obj
 0002:0000b6e8       ??_C@_1M@DDNJFGID@?$AAf?$AAi?$AA?9?$AAF?$AAI?$AA?$AA@ 1010e6e8     LIBCMT:winapinls.obj
 0002:0000b6f4       ??_C@_1M@GLIPPMAC@?$AAf?$AAr?$AA?9?$AAF?$AAR?$AA?$AA@ 1010e6f4     LIBCMT:winapinls.obj
 0002:0000b700       ??_C@_1M@GFMCHPE@?$AAh?$AAe?$AA?9?$AAI?$AAL?$AA?$AA@ 1010e700     LIBCMT:winapinls.obj
 0002:0000b70c       ??_C@_1M@MHLPGNKM@?$AAh?$AAu?$AA?9?$AAH?$AAU?$AA?$AA@ 1010e70c     LIBCMT:winapinls.obj
 0002:0000b718       ??_C@_1M@LPDDNNPN@?$AAi?$AAs?$AA?9?$AAI?$AAS?$AA?$AA@ 1010e718     LIBCMT:winapinls.obj
 0002:0000b724       ??_C@_1M@MADIPODN@?$AAi?$AAt?$AA?9?$AAI?$AAT?$AA?$AA@ 1010e724     LIBCMT:winapinls.obj
 0002:0000b730       ??_C@_1M@IHBJJGG@?$AAn?$AAl?$AA?9?$AAN?$AAL?$AA?$AA@ 1010e730     LIBCMT:winapinls.obj
 0002:0000b73c       ??_C@_1M@EANAGDL@?$AAn?$AAb?$AA?9?$AAN?$AAO?$AA?$AA@ 1010e73c     LIBCMT:winapinls.obj
 0002:0000b748       ??_C@_1M@NEIEMEGP@?$AAp?$AAl?$AA?9?$AAP?$AAL?$AA?$AA@ 1010e748     LIBCMT:winapinls.obj
 0002:0000b754       ??_C@_1M@BOCFIGEP@?$AAp?$AAt?$AA?9?$AAB?$AAR?$AA?$AA@ 1010e754     LIBCMT:winapinls.obj
 0002:0000b760       ??_C@_1M@IMPFOPBG@?$AAr?$AAo?$AA?9?$AAR?$AAO?$AA?$AA@ 1010e760     LIBCMT:winapinls.obj
 0002:0000b76c       ??_C@_1M@IDNNEJMM@?$AAr?$AAu?$AA?9?$AAR?$AAU?$AA?$AA@ 1010e76c     LIBCMT:winapinls.obj
 0002:0000b778       ??_C@_1M@LILEEOGM@?$AAh?$AAr?$AA?9?$AAH?$AAR?$AA?$AA@ 1010e778     LIBCMT:winapinls.obj
 0002:0000b784       ??_C@_1M@FKIFEHPB@?$AAs?$AAk?$AA?9?$AAS?$AAK?$AA?$AA@ 1010e784     LIBCMT:winapinls.obj
 0002:0000b790       ??_C@_1M@LJMAMNPJ@?$AAs?$AAq?$AA?9?$AAA?$AAL?$AA?$AA@ 1010e790     LIBCMT:winapinls.obj
 0002:0000b79c       ??_C@_1M@GIAKDKJK@?$AAs?$AAv?$AA?9?$AAS?$AAE?$AA?$AA@ 1010e79c     LIBCMT:winapinls.obj
 0002:0000b7a8       ??_C@_1M@MKJKIKCL@?$AAt?$AAh?$AA?9?$AAT?$AAH?$AA?$AA@ 1010e7a8     LIBCMT:winapinls.obj
 0002:0000b7b4       ??_C@_1M@MFLCCMPB@?$AAt?$AAr?$AA?9?$AAT?$AAR?$AA?$AA@ 1010e7b4     LIBCMT:winapinls.obj
 0002:0000b7c0       ??_C@_1M@OIJHDKJN@?$AAu?$AAr?$AA?9?$AAP?$AAK?$AA?$AA@ 1010e7c0     LIBCMT:winapinls.obj
 0002:0000b7cc       ??_C@_1M@LHIPCIEK@?$AAi?$AAd?$AA?9?$AAI?$AAD?$AA?$AA@ 1010e7cc     LIBCMT:winapinls.obj
 0002:0000b7d8       ??_C@_1M@MFMOBGI@?$AAu?$AAk?$AA?9?$AAU?$AAA?$AA?$AA@ 1010e7d8     LIBCMT:winapinls.obj
 0002:0000b7e4       ??_C@_1M@OBGLJIPL@?$AAb?$AAe?$AA?9?$AAB?$AAY?$AA?$AA@ 1010e7e4     LIBCMT:winapinls.obj
 0002:0000b7f0       ??_C@_1M@BCFAJEAD@?$AAs?$AAl?$AA?9?$AAS?$AAI?$AA?$AA@ 1010e7f0     LIBCMT:winapinls.obj
 0002:0000b7fc       ??_C@_1M@FKFFEDDN@?$AAe?$AAt?$AA?9?$AAE?$AAE?$AA?$AA@ 1010e7fc     LIBCMT:winapinls.obj
 0002:0000b808       ??_C@_1M@KGKKAACI@?$AAl?$AAv?$AA?9?$AAL?$AAV?$AA?$AA@ 1010e808     LIBCMT:winapinls.obj
 0002:0000b814       ??_C@_1M@IFGBIJO@?$AAl?$AAt?$AA?9?$AAL?$AAT?$AA?$AA@ 1010e814     LIBCMT:winapinls.obj
 0002:0000b820       ??_C@_1M@FGEAHEDM@?$AAf?$AAa?$AA?9?$AAI?$AAR?$AA?$AA@ 1010e820     LIBCMT:winapinls.obj
 0002:0000b82c       ??_C@_1M@KBMAIBFN@?$AAv?$AAi?$AA?9?$AAV?$AAN?$AA?$AA@ 1010e82c     LIBCMT:winapinls.obj
 0002:0000b838       ??_C@_1M@GPCBKDJK@?$AAh?$AAy?$AA?9?$AAA?$AAM?$AA?$AA@ 1010e838     LIBCMT:winapinls.obj
 0002:0000b844       ??_C@_1BG@BECMDDJB@?$AAa?$AAz?$AA?9?$AAA?$AAZ?$AA?9?$AAL?$AAa?$AAt?$AAn?$AA?$AA@ 1010e844     LIBCMT:winapinls.obj
 0002:0000b85c       ??_C@_1M@MAOFCAEA@?$AAe?$AAu?$AA?9?$AAE?$AAS?$AA?$AA@ 1010e85c     LIBCMT:winapinls.obj
 0002:0000b868       ??_C@_1M@IGHABKPI@?$AAm?$AAk?$AA?9?$AAM?$AAK?$AA?$AA@ 1010e868     LIBCMT:winapinls.obj
 0002:0000b874       ??_C@_1M@IAIGNEJG@?$AAt?$AAn?$AA?9?$AAZ?$AAA?$AA?$AA@ 1010e874     LIBCMT:winapinls.obj
 0002:0000b880       ??_C@_1M@IIJCOJFA@?$AAx?$AAh?$AA?9?$AAZ?$AAA?$AA?$AA@ 1010e880     LIBCMT:winapinls.obj
 0002:0000b88c       ??_C@_1M@LGPJHNJH@?$AAz?$AAu?$AA?9?$AAZ?$AAA?$AA?$AA@ 1010e88c     LIBCMT:winapinls.obj
 0002:0000b898       ??_C@_1M@HOKAOIO@?$AAa?$AAf?$AA?9?$AAZ?$AAA?$AA?$AA@ 1010e898     LIBCMT:winapinls.obj
 0002:0000b8a4       ??_C@_1M@DPCLHLIE@?$AAk?$AAa?$AA?9?$AAG?$AAE?$AA?$AA@ 1010e8a4     LIBCMT:winapinls.obj
 0002:0000b8b0       ??_C@_1M@BLKMHJBI@?$AAf?$AAo?$AA?9?$AAF?$AAO?$AA?$AA@ 1010e8b0     LIBCMT:winapinls.obj
 0002:0000b8bc       ??_C@_1M@LGGJAPPB@?$AAh?$AAi?$AA?9?$AAI?$AAN?$AA?$AA@ 1010e8bc     LIBCMT:winapinls.obj
 0002:0000b8c8       ??_C@_1M@FIKPIHFE@?$AAm?$AAt?$AA?9?$AAM?$AAT?$AA?$AA@ 1010e8c8     LIBCMT:winapinls.obj
 0002:0000b8d4       ??_C@_1M@HEGGPBFA@?$AAs?$AAe?$AA?9?$AAN?$AAO?$AA?$AA@ 1010e8d4     LIBCMT:winapinls.obj
 0002:0000b8e0       ??_C@_1M@EIBJEEPA@?$AAm?$AAs?$AA?9?$AAM?$AAY?$AA?$AA@ 1010e8e0     LIBCMT:winapinls.obj
 0002:0000b8ec       ??_C@_1M@FHLBGMPP@?$AAk?$AAk?$AA?9?$AAK?$AAZ?$AA?$AA@ 1010e8ec     LIBCMT:winapinls.obj
 0002:0000b8f8       ??_C@_1M@NGJJLCGI@?$AAk?$AAy?$AA?9?$AAK?$AAG?$AA?$AA@ 1010e8f8     LIBCMT:winapinls.obj
 0002:0000b904       ??_C@_1M@GIENNBFC@?$AAs?$AAw?$AA?9?$AAK?$AAE?$AA?$AA@ 1010e904     LIBCMT:winapinls.obj
 0002:0000b910       ??_C@_1BG@NDGMJIMJ@?$AAu?$AAz?$AA?9?$AAU?$AAZ?$AA?9?$AAL?$AAa?$AAt?$AAn?$AA?$AA@ 1010e910     LIBCMT:winapinls.obj
 0002:0000b928       ??_C@_1M@IDCCIHBC@?$AAt?$AAt?$AA?9?$AAR?$AAU?$AA?$AA@ 1010e928     LIBCMT:winapinls.obj
 0002:0000b934       ??_C@_1M@LOICPMOJ@?$AAb?$AAn?$AA?9?$AAI?$AAN?$AA?$AA@ 1010e934     LIBCMT:winapinls.obj
 0002:0000b940       ??_C@_1M@KPKKNEAH@?$AAp?$AAa?$AA?9?$AAI?$AAN?$AA?$AA@ 1010e940     LIBCMT:winapinls.obj
 0002:0000b94c       ??_C@_1M@PJGPPBOG@?$AAg?$AAu?$AA?9?$AAI?$AAN?$AA?$AA@ 1010e94c     LIBCMT:winapinls.obj
 0002:0000b958       ??_C@_1M@KMKMOPHI@?$AAt?$AAa?$AA?9?$AAI?$AAN?$AA?$AA@ 1010e958     LIBCMT:winapinls.obj
 0002:0000b964       ??_C@_1M@KFEHEPAC@?$AAt?$AAe?$AA?9?$AAI?$AAN?$AA?$AA@ 1010e964     LIBCMT:winapinls.obj
 0002:0000b970       ??_C@_1M@CDCLMGHI@?$AAk?$AAn?$AA?9?$AAI?$AAN?$AA?$AA@ 1010e970     LIBCMT:winapinls.obj
 0002:0000b97c       ??_C@_1M@MIODLDKF@?$AAm?$AAl?$AA?9?$AAI?$AAN?$AA?$AA@ 1010e97c     LIBCMT:winapinls.obj
 0002:0000b988       ??_C@_1M@PBIEACPO@?$AAm?$AAr?$AA?9?$AAI?$AAN?$AA?$AA@ 1010e988     LIBCMT:winapinls.obj
 0002:0000b994       ??_C@_1M@NIDEAGPH@?$AAs?$AAa?$AA?9?$AAI?$AAN?$AA?$AA@ 1010e994     LIBCMT:winapinls.obj
 0002:0000b9a0       ??_C@_1M@FHIHCBIO@?$AAm?$AAn?$AA?9?$AAM?$AAN?$AA?$AA@ 1010e9a0     LIBCMT:winapinls.obj
 0002:0000b9ac       ??_C@_1M@JAIJPENP@?$AAc?$AAy?$AA?9?$AAG?$AAB?$AA?$AA@ 1010e9ac     LIBCMT:winapinls.obj
 0002:0000b9b8       ??_C@_1M@PHGFBEPN@?$AAg?$AAl?$AA?9?$AAE?$AAS?$AA?$AA@ 1010e9b8     LIBCMT:winapinls.obj
 0002:0000b9c4       ??_C@_1O@KPIPDNCP@?$AAk?$AAo?$AAk?$AA?9?$AAI?$AAN?$AA?$AA@ 1010e9c4     LIBCMT:winapinls.obj
 0002:0000b9d4       ??_C@_1O@KNHJLDJA@?$AAs?$AAy?$AAr?$AA?9?$AAS?$AAY?$AA?$AA@ 1010e9d4     LIBCMT:winapinls.obj
 0002:0000b9e4       ??_C@_1O@MKEKBLAH@?$AAd?$AAi?$AAv?$AA?9?$AAM?$AAV?$AA?$AA@ 1010e9e4     LIBCMT:winapinls.obj
 0002:0000b9f4       ??_C@_1O@OHDCKDDF@?$AAq?$AAu?$AAz?$AA?9?$AAB?$AAO?$AA?$AA@ 1010e9f4     LIBCMT:winapinls.obj
 0002:0000ba04       ??_C@_1M@LEPJNLFD@?$AAn?$AAs?$AA?9?$AAZ?$AAA?$AA?$AA@ 1010ea04     LIBCMT:winapinls.obj
 0002:0000ba10       ??_C@_1M@OMLEIIJB@?$AAm?$AAi?$AA?9?$AAN?$AAZ?$AA?$AA@ 1010ea10     LIBCMT:winapinls.obj
 0002:0000ba1c       ??_C@_1M@PMPEAILG@?$AAa?$AAr?$AA?9?$AAI?$AAQ?$AA?$AA@ 1010ea1c     LIBCMT:winapinls.obj
 0002:0000ba28       ??_C@_1M@CNKPNOEE@?$AAd?$AAe?$AA?9?$AAC?$AAH?$AA?$AA@ 1010ea28     LIBCMT:winapinls.obj
 0002:0000ba34       ??_C@_1M@LKMGMLKO@?$AAe?$AAn?$AA?9?$AAG?$AAB?$AA?$AA@ 1010ea34     LIBCMT:winapinls.obj
 0002:0000ba40       ??_C@_1M@PGKJFFGL@?$AAe?$AAs?$AA?9?$AAM?$AAX?$AA?$AA@ 1010ea40     LIBCMT:winapinls.obj
 0002:0000ba4c       ??_C@_1M@DNNANBDC@?$AAf?$AAr?$AA?9?$AAB?$AAE?$AA?$AA@ 1010ea4c     LIBCMT:winapinls.obj
 0002:0000ba58       ??_C@_1M@HLGMDFHM@?$AAi?$AAt?$AA?9?$AAC?$AAH?$AA?$AA@ 1010ea58     LIBCMT:winapinls.obj
 0002:0000ba64       ??_C@_1M@CLLBGJH@?$AAn?$AAl?$AA?9?$AAB?$AAE?$AA?$AA@ 1010ea64     LIBCMT:winapinls.obj
 0002:0000ba70       ??_C@_1M@BODBOGLF@?$AAn?$AAn?$AA?9?$AAN?$AAO?$AA?$AA@ 1010ea70     LIBCMT:winapinls.obj
 0002:0000ba7c       ??_C@_1M@HFFAHKAD@?$AAp?$AAt?$AA?9?$AAP?$AAT?$AA?$AA@ 1010ea7c     LIBCMT:winapinls.obj
 0002:0000ba88       ??_C@_1BG@LNOAKHIE@?$AAs?$AAr?$AA?9?$AAS?$AAP?$AA?9?$AAL?$AAa?$AAt?$AAn?$AA?$AA@ 1010ea88     LIBCMT:winapinls.obj
 0002:0000baa0       ??_C@_1M@HBMHBGAK@?$AAs?$AAv?$AA?9?$AAF?$AAI?$AA?$AA@ 1010eaa0     LIBCMT:winapinls.obj
 0002:0000baac       ??_C@_1BG@DGCJGJBE@?$AAa?$AAz?$AA?9?$AAA?$AAZ?$AA?9?$AAC?$AAy?$AAr?$AAl?$AA?$AA@ 1010eaac     LIBCMT:winapinls.obj
 0002:0000bac4       ??_C@_1M@KEJDAAHB@?$AAs?$AAe?$AA?9?$AAS?$AAE?$AA?$AA@ 1010eac4     LIBCMT:winapinls.obj
 0002:0000bad0       ??_C@_1M@HEIBJJAD@?$AAm?$AAs?$AA?9?$AAB?$AAN?$AA?$AA@ 1010ead0     LIBCMT:winapinls.obj
 0002:0000badc       ??_C@_1BG@PBGJMCEM@?$AAu?$AAz?$AA?9?$AAU?$AAZ?$AA?9?$AAC?$AAy?$AAr?$AAl?$AA?$AA@ 1010eadc     LIBCMT:winapinls.obj
 0002:0000baf4       ??_C@_1O@LAOBCMDF@?$AAq?$AAu?$AAz?$AA?9?$AAE?$AAC?$AA?$AA@ 1010eaf4     LIBCMT:winapinls.obj
 0002:0000bb04       ??_C@_1M@POEEMAIO@?$AAa?$AAr?$AA?9?$AAE?$AAG?$AA?$AA@ 1010eb04     LIBCMT:winapinls.obj
 0002:0000bb10       ??_C@_1M@EFAKDEDL@?$AAz?$AAh?$AA?9?$AAH?$AAK?$AA?$AA@ 1010eb10     LIBCMT:winapinls.obj
 0002:0000bb1c       ??_C@_1M@HKKIJHGI@?$AAd?$AAe?$AA?9?$AAA?$AAT?$AA?$AA@ 1010eb1c     LIBCMT:winapinls.obj
 0002:0000bb28       ??_C@_1M@KBFBEHJF@?$AAe?$AAn?$AA?9?$AAA?$AAU?$AA?$AA@ 1010eb28     LIBCMT:winapinls.obj
 0002:0000bb34       ??_C@_1M@MNPLFAAH@?$AAe?$AAs?$AA?9?$AAE?$AAS?$AA?$AA@ 1010eb34     LIBCMT:winapinls.obj
 0002:0000bb40       ??_C@_1M@HJOOJFMA@?$AAf?$AAr?$AA?9?$AAC?$AAA?$AA?$AA@ 1010eb40     LIBCMT:winapinls.obj
 0002:0000bb4c       ??_C@_1BG@JPOFPNAB@?$AAs?$AAr?$AA?9?$AAS?$AAP?$AA?9?$AAC?$AAy?$AAr?$AAl?$AA?$AA@ 1010eb4c     LIBCMT:winapinls.obj
 0002:0000bb64       ??_C@_1M@LNFOCMOB@?$AAs?$AAe?$AA?9?$AAF?$AAI?$AA?$AA@ 1010eb64     LIBCMT:winapinls.obj
 0002:0000bb70       ??_C@_1O@MGJBOAMB@?$AAq?$AAu?$AAz?$AA?9?$AAP?$AAE?$AA?$AA@ 1010eb70     LIBCMT:winapinls.obj
 0002:0000bb80       ??_C@_1M@GJINLBOK@?$AAa?$AAr?$AA?9?$AAL?$AAY?$AA?$AA@ 1010eb80     LIBCMT:winapinls.obj
 0002:0000bb8c       ??_C@_1M@GGMNHJNL@?$AAz?$AAh?$AA?9?$AAS?$AAG?$AA?$AA@ 1010eb8c     LIBCMT:winapinls.obj
 0002:0000bb98       ??_C@_1M@HOIKODND@?$AAd?$AAe?$AA?9?$AAL?$AAU?$AA?$AA@ 1010eb98     LIBCMT:winapinls.obj
 0002:0000bba4       ??_C@_1M@DDOCCGFG@?$AAe?$AAn?$AA?9?$AAC?$AAA?$AA?$AA@ 1010eba4     LIBCMT:winapinls.obj
 0002:0000bbb0       ??_C@_1M@BNOEMJLF@?$AAe?$AAs?$AA?9?$AAG?$AAT?$AA?$AA@ 1010ebb0     LIBCMT:winapinls.obj
 0002:0000bbbc       ??_C@_1M@EOGNKEK@?$AAf?$AAr?$AA?9?$AAC?$AAH?$AA?$AA@ 1010ebbc     LIBCMT:winapinls.obj
 0002:0000bbc8       ??_C@_1M@FLIDJFHL@?$AAh?$AAr?$AA?9?$AAB?$AAA?$AA?$AA@ 1010ebc8     LIBCMT:winapinls.obj
 0002:0000bbd4       ??_C@_1O@FMCELNAJ@?$AAs?$AAm?$AAj?$AA?9?$AAN?$AAO?$AA?$AA@ 1010ebd4     LIBCMT:winapinls.obj
 0002:0000bbe4       ??_C@_1M@JHGLJMGJ@?$AAa?$AAr?$AA?9?$AAD?$AAZ?$AA?$AA@ 1010ebe4     LIBCMT:winapinls.obj
 0002:0000bbf0       ??_C@_1M@JKKFDCNP@?$AAz?$AAh?$AA?9?$AAM?$AAO?$AA?$AA@ 1010ebf0     LIBCMT:winapinls.obj
 0002:0000bbfc       ??_C@_1M@GEEFALPE@?$AAd?$AAe?$AA?9?$AAL?$AAI?$AA?$AA@ 1010ebfc     LIBCMT:winapinls.obj
 0002:0000bc08       ??_C@_1M@IGEOFBG@?$AAe?$AAn?$AA?9?$AAN?$AAZ?$AA?$AA@ 1010ec08     LIBCMT:winapinls.obj
 0002:0000bc14       ??_C@_1M@KDBONEHP@?$AAe?$AAs?$AA?9?$AAC?$AAR?$AA?$AA@ 1010ec14     LIBCMT:winapinls.obj
 0002:0000bc20       ??_C@_1M@FHMDOHNN@?$AAf?$AAr?$AA?9?$AAL?$AAU?$AA?$AA@ 1010ec20     LIBCMT:winapinls.obj
 0002:0000bc2c       ??_C@_1BG@NFKKMAFG@?$AAb?$AAs?$AA?9?$AAB?$AAA?$AA?9?$AAL?$AAa?$AAt?$AAn?$AA?$AA@ 1010ec2c     LIBCMT:winapinls.obj
 0002:0000bc44       ??_C@_1O@IMNBEMCI@?$AAs?$AAm?$AAj?$AA?9?$AAS?$AAE?$AA?$AA@ 1010ec44     LIBCMT:winapinls.obj
 0002:0000bc54       ??_C@_1M@DHHMBNDP@?$AAa?$AAr?$AA?9?$AAM?$AAA?$AA?$AA@ 1010ec54     LIBCMT:winapinls.obj
 0002:0000bc60       ??_C@_1M@BNBLJCGH@?$AAe?$AAn?$AA?9?$AAI?$AAE?$AA?$AA@ 1010ec60     LIBCMT:winapinls.obj
 0002:0000bc6c       ??_C@_1M@GEPAFMDL@?$AAe?$AAs?$AA?9?$AAP?$AAA?$AA?$AA@ 1010ec6c     LIBCMT:winapinls.obj
 0002:0000bc78       ??_C@_1M@OJONDMDL@?$AAf?$AAr?$AA?9?$AAM?$AAC?$AA?$AA@ 1010ec78     LIBCMT:winapinls.obj
 0002:0000bc84       ??_C@_1BG@OBCNFJB@?$AAs?$AAr?$AA?9?$AAB?$AAA?$AA?9?$AAL?$AAa?$AAt?$AAn?$AA?$AA@ 1010ec84     LIBCMT:winapinls.obj
 0002:0000bc9c       ??_C@_1O@KEMEEGPO@?$AAs?$AAm?$AAa?$AA?9?$AAN?$AAO?$AA?$AA@ 1010ec9c     LIBCMT:winapinls.obj
 0002:0000bcac       ??_C@_1M@ELMGFODK@?$AAa?$AAr?$AA?9?$AAT?$AAN?$AA?$AA@ 1010ecac     LIBCMT:winapinls.obj
 0002:0000bcb8       ??_C@_1M@BHDLHFAF@?$AAe?$AAn?$AA?9?$AAZ?$AAA?$AA?$AA@ 1010ecb8     LIBCMT:winapinls.obj
 0002:0000bcc4       ??_C@_1M@BMGIGLIF@?$AAe?$AAs?$AA?9?$AAD?$AAO?$AA?$AA@ 1010ecc4     LIBCMT:winapinls.obj
 0002:0000bcd0       ??_C@_1BG@CMBHIPBE@?$AAs?$AAr?$AA?9?$AAB?$AAA?$AA?9?$AAC?$AAy?$AAr?$AAl?$AA?$AA@ 1010ecd0     LIBCMT:winapinls.obj
 0002:0000bce8       ??_C@_1O@HEDBLHNP@?$AAs?$AAm?$AAa?$AA?9?$AAS?$AAE?$AA?$AA@ 1010ece8     LIBCMT:winapinls.obj
 0002:0000bcf8       ??_C@_1M@DAGCADIM@?$AAa?$AAr?$AA?9?$AAO?$AAM?$AA?$AA@ 1010ecf8     LIBCMT:winapinls.obj
 0002:0000bd04       ??_C@_1M@FODLMICG@?$AAe?$AAn?$AA?9?$AAJ?$AAM?$AA?$AA@ 1010ed04     LIBCMT:winapinls.obj
 0002:0000bd10       ??_C@_1M@DNMLCIHB@?$AAe?$AAs?$AA?9?$AAV?$AAE?$AA?$AA@ 1010ed10     LIBCMT:winapinls.obj
 0002:0000bd1c       ??_C@_1O@EOKHMKJK@?$AAs?$AAm?$AAs?$AA?9?$AAF?$AAI?$AA?$AA@ 1010ed1c     LIBCMT:winapinls.obj
 0002:0000bd2c       ??_C@_1M@CAFJMKOF@?$AAa?$AAr?$AA?9?$AAY?$AAE?$AA?$AA@ 1010ed2c     LIBCMT:winapinls.obj
 0002:0000bd38       ??_C@_1M@CBFHIJLI@?$AAe?$AAn?$AA?9?$AAC?$AAB?$AA?$AA@ 1010ed38     LIBCMT:winapinls.obj
 0002:0000bd44       ??_C@_1M@BGNFLDN@?$AAe?$AAs?$AA?9?$AAC?$AAO?$AA?$AA@ 1010ed44     LIBCMT:winapinls.obj
 0002:0000bd50       ??_C@_1O@JMPHMAMC@?$AAs?$AAm?$AAn?$AA?9?$AAF?$AAI?$AA?$AA@ 1010ed50     LIBCMT:winapinls.obj
 0002:0000bd60       ??_C@_1M@JLANABKE@?$AAa?$AAr?$AA?9?$AAS?$AAY?$AA?$AA@ 1010ed60     LIBCMT:winapinls.obj
 0002:0000bd6c       ??_C@_1M@HPKGCFGN@?$AAe?$AAn?$AA?9?$AAB?$AAZ?$AA?$AA@ 1010ed6c     LIBCMT:winapinls.obj
 0002:0000bd78       ??_C@_1M@OLJCMLGM@?$AAe?$AAs?$AA?9?$AAP?$AAE?$AA?$AA@ 1010ed78     LIBCMT:winapinls.obj
 0002:0000bd84       ??_C@_1M@MKKGFKLE@?$AAa?$AAr?$AA?9?$AAJ?$AAO?$AA?$AA@ 1010ed84     LIBCMT:winapinls.obj
 0002:0000bd90       ??_C@_1M@EKPGLDNI@?$AAe?$AAn?$AA?9?$AAT?$AAT?$AA?$AA@ 1010ed90     LIBCMT:winapinls.obj
 0002:0000bd9c       ??_C@_1M@OONGHFHE@?$AAe?$AAs?$AA?9?$AAA?$AAR?$AA?$AA@ 1010ed9c     LIBCMT:winapinls.obj
 0002:0000bda8       ??_C@_1M@OOJFGBHE@?$AAa?$AAr?$AA?9?$AAL?$AAB?$AA?$AA@ 1010eda8     LIBCMT:winapinls.obj
 0002:0000bdb4       ??_C@_1M@GCEJHNEG@?$AAe?$AAn?$AA?9?$AAZ?$AAW?$AA?$AA@ 1010edb4     LIBCMT:winapinls.obj
 0002:0000bdc0       ??_C@_1M@JNOCAHJI@?$AAe?$AAs?$AA?9?$AAE?$AAC?$AA?$AA@ 1010edc0     LIBCMT:winapinls.obj
 0002:0000bdcc       ??_C@_1M@JEFHPGGB@?$AAa?$AAr?$AA?9?$AAK?$AAW?$AA?$AA@ 1010edcc     LIBCMT:winapinls.obj
 0002:0000bdd8       ??_C@_1M@MLKIBJOJ@?$AAe?$AAn?$AA?9?$AAP?$AAH?$AA?$AA@ 1010edd8     LIBCMT:winapinls.obj
 0002:0000bde4       ??_C@_1M@BDNIPEND@?$AAe?$AAs?$AA?9?$AAC?$AAL?$AA?$AA@ 1010ede4     LIBCMT:winapinls.obj
 0002:0000bdf0       ??_C@_1M@MPNMEKBD@?$AAa?$AAr?$AA?9?$AAA?$AAE?$AA?$AA@ 1010edf0     LIBCMT:winapinls.obj
 0002:0000bdfc       ??_C@_1M@KBJALCPI@?$AAe?$AAs?$AA?9?$AAU?$AAY?$AA?$AA@ 1010edfc     LIBCMT:winapinls.obj
 0002:0000be08       ??_C@_1M@LLCCOAGA@?$AAa?$AAr?$AA?9?$AAB?$AAH?$AA?$AA@ 1010ee08     LIBCMT:winapinls.obj
 0002:0000be14       ??_C@_1M@PBFNCDEL@?$AAe?$AAs?$AA?9?$AAP?$AAY?$AA?$AA@ 1010ee14     LIBCMT:winapinls.obj
 0002:0000be20       ??_C@_1M@EDGINPNP@?$AAa?$AAr?$AA?9?$AAQ?$AAA?$AA?$AA@ 1010ee20     LIBCMT:winapinls.obj
 0002:0000be2c       ??_C@_1M@MKDBIIJI@?$AAe?$AAs?$AA?9?$AAB?$AAO?$AA?$AA@ 1010ee2c     LIBCMT:winapinls.obj
 0002:0000be38       ??_C@_1M@CPKKEBLD@?$AAe?$AAs?$AA?9?$AAS?$AAV?$AA?$AA@ 1010ee38     LIBCMT:winapinls.obj
 0002:0000be44       ??_C@_1M@NDBGMMJL@?$AAe?$AAs?$AA?9?$AAH?$AAN?$AA?$AA@ 1010ee44     LIBCMT:winapinls.obj
 0002:0000be50       ??_C@_1M@JIJIBHDP@?$AAe?$AAs?$AA?9?$AAN?$AAI?$AA?$AA@ 1010ee50     LIBCMT:winapinls.obj
 0002:0000be5c       ??_C@_1M@CGFMKEEK@?$AAe?$AAs?$AA?9?$AAP?$AAR?$AA?$AA@ 1010ee5c     LIBCMT:winapinls.obj
 0002:0000be68       ??_C@_1O@ICJHKIIK@?$AAz?$AAh?$AA?9?$AAC?$AAH?$AAT?$AA?$AA@ 1010ee68     LIBCMT:winapinls.obj
 0002:0000be78       ??_C@_15CLNEJCE@?$AAs?$AAr?$AA?$AA@ 1010ee78     LIBCMT:winapinls.obj
 0002:0000be80       ??_C@_1M@KAHEKEIG@?$AAa?$AAf?$AA?9?$AAz?$AAa?$AA?$AA@ 1010ee80     LIBCMT:winapinls.obj
 0002:0000be8c       ??_C@_1M@GIECOABL@?$AAa?$AAr?$AA?9?$AAa?$AAe?$AA?$AA@ 1010ee8c     LIBCMT:winapinls.obj
 0002:0000be98       ??_C@_1M@BMLMEKGI@?$AAa?$AAr?$AA?9?$AAb?$AAh?$AA?$AA@ 1010ee98     LIBCMT:winapinls.obj
 0002:0000bea4       ??_C@_1M@DAPFDGGB@?$AAa?$AAr?$AA?9?$AAd?$AAz?$AA?$AA@ 1010eea4     LIBCMT:winapinls.obj
 0002:0000beb0       ??_C@_1M@FJNKGKIG@?$AAa?$AAr?$AA?9?$AAe?$AAg?$AA?$AA@ 1010eeb0     LIBCMT:winapinls.obj
 0002:0000bebc       ??_C@_1M@FLGKKCLO@?$AAa?$AAr?$AA?9?$AAi?$AAq?$AA?$AA@ 1010eebc     LIBCMT:winapinls.obj
 0002:0000bec8       ??_C@_1M@GNDIPALM@?$AAa?$AAr?$AA?9?$AAj?$AAo?$AA?$AA@ 1010eec8     LIBCMT:winapinls.obj
 0002:0000bed4       ??_C@_1M@DDMJFMGJ@?$AAa?$AAr?$AA?9?$AAk?$AAw?$AA?$AA@ 1010eed4     LIBCMT:winapinls.obj
 0002:0000bee0       ??_C@_1M@EJALMLHM@?$AAa?$AAr?$AA?9?$AAl?$AAb?$AA?$AA@ 1010eee0     LIBCMT:winapinls.obj
 0002:0000beec       ??_C@_1M@MOBDBLOC@?$AAa?$AAr?$AA?9?$AAl?$AAy?$AA?$AA@ 1010eeec     LIBCMT:winapinls.obj
 0002:0000bef8       ??_C@_1M@JAOCLHDH@?$AAa?$AAr?$AA?9?$AAm?$AAa?$AA?$AA@ 1010eef8     LIBCMT:winapinls.obj
 0002:0000bf04       ??_C@_1M@JHPMKJIE@?$AAa?$AAr?$AA?9?$AAo?$AAm?$AA?$AA@ 1010ef04     LIBCMT:winapinls.obj
 0002:0000bf10       ??_C@_1M@OEPGHFNH@?$AAa?$AAr?$AA?9?$AAq?$AAa?$AA?$AA@ 1010ef10     LIBCMT:winapinls.obj
 0002:0000bf1c       ??_C@_1M@KJDONENM@?$AAa?$AAr?$AA?9?$AAs?$AAa?$AA?$AA@ 1010ef1c     LIBCMT:winapinls.obj
 0002:0000bf28       ??_C@_1M@DMJDKLKM@?$AAa?$AAr?$AA?9?$AAs?$AAy?$AA?$AA@ 1010ef28     LIBCMT:winapinls.obj
 0002:0000bf34       ??_C@_1M@OMFIPEDC@?$AAa?$AAr?$AA?9?$AAt?$AAn?$AA?$AA@ 1010ef34     LIBCMT:winapinls.obj
 0002:0000bf40       ??_C@_1M@IHMHGAON@?$AAa?$AAr?$AA?9?$AAy?$AAe?$AA?$AA@ 1010ef40     LIBCMT:winapinls.obj
 0002:0000bf4c       ??_C@_1BG@KDCPGJGB@?$AAa?$AAz?$AA?9?$AAa?$AAz?$AA?9?$AAc?$AAy?$AAr?$AAl?$AA?$AA@ 1010ef4c     LIBCMT:winapinls.obj
 0002:0000bf64       ??_C@_1BG@IBCKDDOE@?$AAa?$AAz?$AA?9?$AAa?$AAz?$AA?9?$AAl?$AAa?$AAt?$AAn?$AA?$AA@ 1010ef64     LIBCMT:winapinls.obj
 0002:0000bf7c       ??_C@_1M@EGPFDCPD@?$AAb?$AAe?$AA?9?$AAb?$AAy?$AA?$AA@ 1010ef7c     LIBCMT:winapinls.obj
 0002:0000bf88       ??_C@_1M@PCMGMCGC@?$AAb?$AAg?$AA?9?$AAb?$AAg?$AA?$AA@ 1010ef88     LIBCMT:winapinls.obj
 0002:0000bf94       ??_C@_1M@BJBMFGOB@?$AAb?$AAn?$AA?9?$AAi?$AAn?$AA?$AA@ 1010ef94     LIBCMT:winapinls.obj
 0002:0000bfa0       ??_C@_1BG@EAKMMACD@?$AAb?$AAs?$AA?9?$AAb?$AAa?$AA?9?$AAl?$AAa?$AAt?$AAn?$AA?$AA@ 1010efa0     LIBCMT:winapinls.obj
 0002:0000bfb8       ??_C@_1M@KGADAODK@?$AAc?$AAa?$AA?9?$AAe?$AAs?$AA?$AA@ 1010efb8     LIBCMT:winapinls.obj
 0002:0000bfc4       ??_C@_1M@COAJPDHI@?$AAc?$AAs?$AA?9?$AAc?$AAz?$AA?$AA@ 1010efc4     LIBCMT:winapinls.obj
 0002:0000bfd0       ??_C@_1M@DHBHFONH@?$AAc?$AAy?$AA?9?$AAg?$AAb?$AA?$AA@ 1010efd0     LIBCMT:winapinls.obj
 0002:0000bfdc       ??_C@_1M@IMGKELGA@?$AAd?$AAa?$AA?9?$AAd?$AAk?$AA?$AA@ 1010efdc     LIBCMT:winapinls.obj
 0002:0000bfe8       ??_C@_1M@NNDGDNGA@?$AAd?$AAe?$AA?9?$AAa?$AAt?$AA?$AA@ 1010efe8     LIBCMT:winapinls.obj
 0002:0000bff4       ??_C@_1M@IKDBHEEM@?$AAd?$AAe?$AA?9?$AAc?$AAh?$AA?$AA@ 1010eff4     LIBCMT:winapinls.obj
 0002:0000c000       ??_C@_1M@GFFOJMCJ@?$AAd?$AAe?$AA?9?$AAd?$AAe?$AA?$AA@ 1010f000     LIBCMT:winapinls.obj
 0002:0000c00c       ??_C@_1M@MDNLKBPM@?$AAd?$AAe?$AA?9?$AAl?$AAi?$AA?$AA@ 1010f00c     LIBCMT:winapinls.obj
 0002:0000c018       ??_C@_1M@NJBEEJNL@?$AAd?$AAe?$AA?9?$AAl?$AAu?$AA?$AA@ 1010f018     LIBCMT:winapinls.obj
 0002:0000c024       ??_C@_1O@GNNELBAP@?$AAd?$AAi?$AAv?$AA?9?$AAm?$AAv?$AA?$AA@ 1010f024     LIBCMT:winapinls.obj
 0002:0000c034       ??_C@_1M@EJLEOGAE@?$AAe?$AAl?$AA?9?$AAg?$AAr?$AA?$AA@ 1010f034     LIBCMT:winapinls.obj
 0002:0000c040       ??_C@_1M@GMPONJN@?$AAe?$AAn?$AA?9?$AAa?$AAu?$AA?$AA@ 1010f040     LIBCMT:winapinls.obj
 0002:0000c04c       ??_C@_1M@NIDIIPGF@?$AAe?$AAn?$AA?9?$AAb?$AAz?$AA?$AA@ 1010f04c     LIBCMT:winapinls.obj
 0002:0000c058       ??_C@_1M@JEHMIMFO@?$AAe?$AAn?$AA?9?$AAc?$AAa?$AA?$AA@ 1010f058     LIBCMT:winapinls.obj
 0002:0000c064       ??_C@_1M@IGMJCDLA@?$AAe?$AAn?$AA?9?$AAc?$AAb?$AA?$AA@ 1010f064     LIBCMT:winapinls.obj
 0002:0000c070       ??_C@_1M@BNFIGBKG@?$AAe?$AAn?$AA?9?$AAg?$AAb?$AA?$AA@ 1010f070     LIBCMT:winapinls.obj
 0002:0000c07c       ??_C@_1M@LKIFDIGP@?$AAe?$AAn?$AA?9?$AAi?$AAe?$AA?$AA@ 1010f07c     LIBCMT:winapinls.obj
 0002:0000c088       ??_C@_1M@PJKFGCCO@?$AAe?$AAn?$AA?9?$AAj?$AAm?$AA?$AA@ 1010f088     LIBCMT:winapinls.obj
 0002:0000c094       ??_C@_1M@KPPKEPBO@?$AAe?$AAn?$AA?9?$AAn?$AAz?$AA?$AA@ 1010f094     LIBCMT:winapinls.obj
 0002:0000c0a0       ??_C@_1M@GMDGLDOB@?$AAe?$AAn?$AA?9?$AAp?$AAh?$AA?$AA@ 1010f0a0     LIBCMT:winapinls.obj
 0002:0000c0ac       ??_C@_1M@ONGIBJNA@?$AAe?$AAn?$AA?9?$AAt?$AAt?$AA?$AA@ 1010f0ac     LIBCMT:winapinls.obj
 0002:0000c0b8       ??_C@_1M@LLODPCMM@?$AAe?$AAn?$AA?9?$AAu?$AAs?$AA?$AA@ 1010f0b8     LIBCMT:winapinls.obj
 0002:0000c0c4       ??_C@_1M@LAKFNPAN@?$AAe?$AAn?$AA?9?$AAz?$AAa?$AA?$AA@ 1010f0c4     LIBCMT:winapinls.obj
 0002:0000c0d0       ??_C@_1M@MFNHNHEO@?$AAe?$AAn?$AA?9?$AAz?$AAw?$AA?$AA@ 1010f0d0     LIBCMT:winapinls.obj
 0002:0000c0dc       ??_C@_1M@EJEINPHM@?$AAe?$AAs?$AA?9?$AAa?$AAr?$AA?$AA@ 1010f0dc     LIBCMT:winapinls.obj
 0002:0000c0e8       ??_C@_1M@GNKPCCJA@?$AAe?$AAs?$AA?9?$AAb?$AAo?$AA?$AA@ 1010f0e8     LIBCMT:winapinls.obj
 0002:0000c0f4       ??_C@_1M@LEEGFONL@?$AAe?$AAs?$AA?9?$AAc?$AAl?$AA?$AA@ 1010f0f4     LIBCMT:winapinls.obj
 0002:0000c100       ??_C@_1M@KGPDPBDF@?$AAe?$AAs?$AA?9?$AAc?$AAo?$AA?$AA@ 1010f100     LIBCMT:winapinls.obj
 0002:0000c10c       ??_C@_1M@EIAHOHH@?$AAe?$AAs?$AA?9?$AAc?$AAr?$AA?$AA@ 1010f10c     LIBCMT:winapinls.obj
 0002:0000c118       ??_C@_1M@LLPGMBIN@?$AAe?$AAs?$AA?9?$AAd?$AAo?$AA?$AA@ 1010f118     LIBCMT:winapinls.obj
 0002:0000c124       ??_C@_1M@DKHMKNJA@?$AAe?$AAs?$AA?9?$AAe?$AAc?$AA?$AA@ 1010f124     LIBCMT:winapinls.obj
 0002:0000c130       ??_C@_1M@GKGFPKAP@?$AAe?$AAs?$AA?9?$AAe?$AAs?$AA?$AA@ 1010f130     LIBCMT:winapinls.obj
 0002:0000c13c       ??_C@_1M@LKHKGDLN@?$AAe?$AAs?$AA?9?$AAg?$AAt?$AA?$AA@ 1010f13c     LIBCMT:winapinls.obj
 0002:0000c148       ??_C@_1M@HEIIGGJD@?$AAe?$AAs?$AA?9?$AAh?$AAn?$AA?$AA@ 1010f148     LIBCMT:winapinls.obj
 0002:0000c154       ??_C@_1M@FBDHPPGD@?$AAe?$AAs?$AA?9?$AAm?$AAx?$AA?$AA@ 1010f154     LIBCMT:winapinls.obj
 0002:0000c160       ??_C@_1M@DPAGLNDH@?$AAe?$AAs?$AA?9?$AAn?$AAi?$AA?$AA@ 1010f160     LIBCMT:winapinls.obj
 0002:0000c16c       ??_C@_1M@MDGOPGDD@?$AAe?$AAs?$AA?9?$AAp?$AAa?$AA?$AA@ 1010f16c     LIBCMT:winapinls.obj
 0002:0000c178       ??_C@_1M@EMAMGBGE@?$AAe?$AAs?$AA?9?$AAp?$AAe?$AA?$AA@ 1010f178     LIBCMT:winapinls.obj
 0002:0000c184       ??_C@_1M@IBMCAOEC@?$AAe?$AAs?$AA?9?$AAp?$AAr?$AA?$AA@ 1010f184     LIBCMT:winapinls.obj
 0002:0000c190       ??_C@_1M@FGMDIJED@?$AAe?$AAs?$AA?9?$AAp?$AAy?$AA?$AA@ 1010f190     LIBCMT:winapinls.obj
 0002:0000c19c       ??_C@_1M@IIDEOLLL@?$AAe?$AAs?$AA?9?$AAs?$AAv?$AA?$AA@ 1010f19c     LIBCMT:winapinls.obj
 0002:0000c1a8       ??_C@_1M@GAOBIPA@?$AAe?$AAs?$AA?9?$AAu?$AAy?$AA?$AA@ 1010f1a8     LIBCMT:winapinls.obj
 0002:0000c1b4       ??_C@_1M@JKFFICHJ@?$AAe?$AAs?$AA?9?$AAv?$AAe?$AA?$AA@ 1010f1b4     LIBCMT:winapinls.obj
 0002:0000c1c0       ??_C@_1M@PNMLOJDF@?$AAe?$AAt?$AA?9?$AAe?$AAe?$AA?$AA@ 1010f1c0     LIBCMT:winapinls.obj
 0002:0000c1cc       ??_C@_1M@GHHLIKEI@?$AAe?$AAu?$AA?9?$AAe?$AAs?$AA?$AA@ 1010f1cc     LIBCMT:winapinls.obj
 0002:0000c1d8       ??_C@_1M@PBNONODE@?$AAf?$AAa?$AA?9?$AAi?$AAr?$AA?$AA@ 1010f1d8     LIBCMT:winapinls.obj
 0002:0000c1e4       ??_C@_1M@JEEHPMIL@?$AAf?$AAi?$AA?9?$AAf?$AAi?$AA?$AA@ 1010f1e4     LIBCMT:winapinls.obj
 0002:0000c1f0       ??_C@_1M@LMDCNDBA@?$AAf?$AAo?$AA?9?$AAf?$AAo?$AA?$AA@ 1010f1f0     LIBCMT:winapinls.obj
 0002:0000c1fc       ??_C@_1M@JKEOHLDK@?$AAf?$AAr?$AA?9?$AAb?$AAe?$AA?$AA@ 1010f1fc     LIBCMT:winapinls.obj
 0002:0000c208       ??_C@_1M@NOHADPMI@?$AAf?$AAr?$AA?9?$AAc?$AAa?$AA?$AA@ 1010f208     LIBCMT:winapinls.obj
 0002:0000c214       ??_C@_1M@KDHIHAEC@?$AAf?$AAr?$AA?9?$AAc?$AAh?$AA?$AA@ 1010f214     LIBCMT:winapinls.obj
 0002:0000c220       ??_C@_1M@MMBBFGAK@?$AAf?$AAr?$AA?9?$AAf?$AAr?$AA?$AA@ 1010f220     LIBCMT:winapinls.obj
 0002:0000c22c       ??_C@_1M@PAFNENNF@?$AAf?$AAr?$AA?9?$AAl?$AAu?$AA?$AA@ 1010f22c     LIBCMT:winapinls.obj
 0002:0000c238       ??_C@_1M@EOHDJGDD@?$AAf?$AAr?$AA?9?$AAm?$AAc?$AA?$AA@ 1010f238     LIBCMT:winapinls.obj
 0002:0000c244       ??_C@_1M@FAPLLOPF@?$AAg?$AAl?$AA?9?$AAe?$AAs?$AA?$AA@ 1010f244     LIBCMT:winapinls.obj
 0002:0000c250       ??_C@_1M@FOPBFLOO@?$AAg?$AAu?$AA?9?$AAi?$AAn?$AA?$AA@ 1010f250     LIBCMT:winapinls.obj
 0002:0000c25c       ??_C@_1M@KBMCINPM@?$AAh?$AAe?$AA?9?$AAi?$AAl?$AA?$AA@ 1010f25c     LIBCMT:winapinls.obj
 0002:0000c268       ??_C@_1M@BBPHKFPJ@?$AAh?$AAi?$AA?9?$AAi?$AAn?$AA?$AA@ 1010f268     LIBCMT:winapinls.obj
 0002:0000c274       ??_C@_1M@PMBNDPHD@?$AAh?$AAr?$AA?9?$AAb?$AAa?$AA?$AA@ 1010f274     LIBCMT:winapinls.obj
 0002:0000c280       ??_C@_1M@BPCKOEGE@?$AAh?$AAr?$AA?9?$AAh?$AAr?$AA?$AA@ 1010f280     LIBCMT:winapinls.obj
 0002:0000c28c       ??_C@_1M@GACBMHKE@?$AAh?$AAu?$AA?9?$AAh?$AAu?$AA?$AA@ 1010f28c     LIBCMT:winapinls.obj
 0002:0000c298       ??_C@_1M@MILPAJJC@?$AAh?$AAy?$AA?9?$AAa?$AAm?$AA?$AA@ 1010f298     LIBCMT:winapinls.obj
 0002:0000c2a4       ??_C@_1M@BABBICEC@?$AAi?$AAd?$AA?9?$AAi?$AAd?$AA?$AA@ 1010f2a4     LIBCMT:winapinls.obj
 0002:0000c2b0       ??_C@_1M@BIKNHHPF@?$AAi?$AAs?$AA?9?$AAi?$AAs?$AA?$AA@ 1010f2b0     LIBCMT:winapinls.obj
 0002:0000c2bc       ??_C@_1M@NMPCJPHE@?$AAi?$AAt?$AA?9?$AAc?$AAh?$AA?$AA@ 1010f2bc     LIBCMT:winapinls.obj
 0002:0000c2c8       ??_C@_1M@GHKGFEDF@?$AAi?$AAt?$AA?9?$AAi?$AAt?$AA?$AA@ 1010f2c8     LIBCMT:winapinls.obj
 0002:0000c2d4       ??_C@_1M@NIEJCJJA@?$AAj?$AAa?$AA?9?$AAj?$AAp?$AA?$AA@ 1010f2d4     LIBCMT:winapinls.obj
 0002:0000c2e0       ??_C@_1M@JILFNBIM@?$AAk?$AAa?$AA?9?$AAg?$AAe?$AA?$AA@ 1010f2e0     LIBCMT:winapinls.obj
 0002:0000c2ec       ??_C@_1M@PACPMGPH@?$AAk?$AAk?$AA?9?$AAk?$AAz?$AA?$AA@ 1010f2ec     LIBCMT:winapinls.obj
 0002:0000c2f8       ??_C@_1M@IELFGMHA@?$AAk?$AAn?$AA?9?$AAi?$AAn?$AA?$AA@ 1010f2f8     LIBCMT:winapinls.obj
 0002:0000c304       ??_C@_1O@IBBJHCH@?$AAk?$AAo?$AAk?$AA?9?$AAi?$AAn?$AA?$AA@ 1010f304     LIBCMT:winapinls.obj
 0002:0000c314       ??_C@_1M@DMHAEOGC@?$AAk?$AAo?$AA?9?$AAk?$AAr?$AA?$AA@ 1010f314     LIBCMT:winapinls.obj
 0002:0000c320       ??_C@_1M@HBAHBIGA@?$AAk?$AAy?$AA?9?$AAk?$AAg?$AA?$AA@ 1010f320     LIBCMT:winapinls.obj
 0002:0000c32c       ??_C@_1M@KPMILCJG@?$AAl?$AAt?$AA?9?$AAl?$AAt?$AA?$AA@ 1010f32c     LIBCMT:winapinls.obj
 0002:0000c338       ??_C@_1M@BDEKKCA@?$AAl?$AAv?$AA?9?$AAl?$AAv?$AA?$AA@ 1010f338     LIBCMT:winapinls.obj
 0002:0000c344       ??_C@_1M@ELCKCCJJ@?$AAm?$AAi?$AA?9?$AAn?$AAz?$AA?$AA@ 1010f344     LIBCMT:winapinls.obj
 0002:0000c350       ??_C@_1M@CBOOLAPA@?$AAm?$AAk?$AA?9?$AAm?$AAk?$AA?$AA@ 1010f350     LIBCMT:winapinls.obj
 0002:0000c35c       ??_C@_1M@GPHNBJKN@?$AAm?$AAl?$AA?9?$AAi?$AAn?$AA?$AA@ 1010f35c     LIBCMT:winapinls.obj
 0002:0000c368       ??_C@_1M@PABJILIG@?$AAm?$AAn?$AA?9?$AAm?$AAn?$AA?$AA@ 1010f368     LIBCMT:winapinls.obj
 0002:0000c374       ??_C@_1M@FGBKKIPG@?$AAm?$AAr?$AA?9?$AAi?$AAn?$AA?$AA@ 1010f374     LIBCMT:winapinls.obj
 0002:0000c380       ??_C@_1M@NDBPDDAL@?$AAm?$AAs?$AA?9?$AAb?$AAn?$AA?$AA@ 1010f380     LIBCMT:winapinls.obj
 0002:0000c38c       ??_C@_1M@OPIHOOPI@?$AAm?$AAs?$AA?9?$AAm?$AAy?$AA?$AA@ 1010f38c     LIBCMT:winapinls.obj
 0002:0000c398       ??_C@_1M@PPDBCNFM@?$AAm?$AAt?$AA?9?$AAm?$AAt?$AA?$AA@ 1010f398     LIBCMT:winapinls.obj
 0002:0000c3a4       ??_C@_1M@KDJDKMDD@?$AAn?$AAb?$AA?9?$AAn?$AAo?$AA?$AA@ 1010f3a4     LIBCMT:winapinls.obj
 0002:0000c3b0       ??_C@_1M@KFCFLMJP@?$AAn?$AAl?$AA?9?$AAb?$AAe?$AA?$AA@ 1010f3b0     LIBCMT:winapinls.obj
 0002:0000c3bc       ??_C@_1M@KPOPDDGO@?$AAn?$AAl?$AA?9?$AAn?$AAl?$AA?$AA@ 1010f3bc     LIBCMT:winapinls.obj
 0002:0000c3c8       ??_C@_1M@LJKPEMLN@?$AAn?$AAn?$AA?9?$AAn?$AAo?$AA?$AA@ 1010f3c8     LIBCMT:winapinls.obj
 0002:0000c3d4       ??_C@_1M@BDGHHBFL@?$AAn?$AAs?$AA?9?$AAz?$AAa?$AA?$AA@ 1010f3d4     LIBCMT:winapinls.obj
 0002:0000c3e0       ??_C@_1M@IDEHOAP@?$AAp?$AAa?$AA?9?$AAi?$AAn?$AA?$AA@ 1010f3e0     LIBCMT:winapinls.obj
 0002:0000c3ec       ??_C@_1M@HDBKGOGH@?$AAp?$AAl?$AA?9?$AAp?$AAl?$AA?$AA@ 1010f3ec     LIBCMT:winapinls.obj
 0002:0000c3f8       ??_C@_1M@LJLLCMEH@?$AAp?$AAt?$AA?9?$AAb?$AAr?$AA?$AA@ 1010f3f8     LIBCMT:winapinls.obj
 0002:0000c404       ??_C@_1M@NCMONAAL@?$AAp?$AAt?$AA?9?$AAp?$AAt?$AA?$AA@ 1010f404     LIBCMT:winapinls.obj
 0002:0000c410       ??_C@_1O@EAKMAJDN@?$AAq?$AAu?$AAz?$AA?9?$AAb?$AAo?$AA?$AA@ 1010f410     LIBCMT:winapinls.obj
 0002:0000c420       ??_C@_1O@BHHPIGDN@?$AAq?$AAu?$AAz?$AA?9?$AAe?$AAc?$AA?$AA@ 1010f420     LIBCMT:winapinls.obj
 0002:0000c430       ??_C@_1O@GBAPEKMJ@?$AAq?$AAu?$AAz?$AA?9?$AAp?$AAe?$AA?$AA@ 1010f430     LIBCMT:winapinls.obj
 0002:0000c440       ??_C@_1M@CLGLEFBO@?$AAr?$AAo?$AA?9?$AAr?$AAo?$AA?$AA@ 1010f440     LIBCMT:winapinls.obj
 0002:0000c44c       ??_C@_1M@CEEDODME@?$AAr?$AAu?$AA?9?$AAr?$AAu?$AA?$AA@ 1010f44c     LIBCMT:winapinls.obj
 0002:0000c458       ??_C@_1M@HPKKKMPP@?$AAs?$AAa?$AA?9?$AAi?$AAn?$AA?$AA@ 1010f458     LIBCMT:winapinls.obj
 0002:0000c464       ??_C@_1M@BKMAIGOJ@?$AAs?$AAe?$AA?9?$AAf?$AAi?$AA?$AA@ 1010f464     LIBCMT:winapinls.obj
 0002:0000c470       ??_C@_1M@NDPIFLFI@?$AAs?$AAe?$AA?9?$AAn?$AAo?$AA?$AA@ 1010f470     LIBCMT:winapinls.obj
 0002:0000c47c       ??_C@_1M@DANKKHJ@?$AAs?$AAe?$AA?9?$AAs?$AAe?$AA?$AA@ 1010f47c     LIBCMT:winapinls.obj
 0002:0000c488       ??_C@_1M@PNBLONPJ@?$AAs?$AAk?$AA?9?$AAs?$AAk?$AA?$AA@ 1010f488     LIBCMT:winapinls.obj
 0002:0000c494       ??_C@_1M@LFMODOAL@?$AAs?$AAl?$AA?9?$AAs?$AAi?$AA?$AA@ 1010f494     LIBCMT:winapinls.obj
 0002:0000c4a0       ??_C@_1O@DFKOMPG@?$AAs?$AAm?$AAa?$AA?9?$AAn?$AAo?$AA?$AA@ 1010f4a0     LIBCMT:winapinls.obj
 0002:0000c4b0       ??_C@_1O@NDKPBNNH@?$AAs?$AAm?$AAa?$AA?9?$AAs?$AAe?$AA?$AA@ 1010f4b0     LIBCMT:winapinls.obj
 0002:0000c4c0       ??_C@_1O@PLLKBHAB@?$AAs?$AAm?$AAj?$AA?9?$AAn?$AAo?$AA?$AA@ 1010f4c0     LIBCMT:winapinls.obj
 0002:0000c4d0       ??_C@_1O@CLEPOGCA@?$AAs?$AAm?$AAj?$AA?9?$AAs?$AAe?$AA?$AA@ 1010f4d0     LIBCMT:winapinls.obj
 0002:0000c4e0       ??_C@_1O@DLGJGKMK@?$AAs?$AAm?$AAn?$AA?9?$AAf?$AAi?$AA?$AA@ 1010f4e0     LIBCMT:winapinls.obj
 0002:0000c4f0       ??_C@_1O@OJDJGAJC@?$AAs?$AAm?$AAs?$AA?9?$AAf?$AAi?$AA?$AA@ 1010f4f0     LIBCMT:winapinls.obj
 0002:0000c500       ??_C@_1M@BOFOGHPB@?$AAs?$AAq?$AA?9?$AAa?$AAl?$AA?$AA@ 1010f500     LIBCMT:winapinls.obj
 0002:0000c50c       ??_C@_1BG@LJBBIPGB@?$AAs?$AAr?$AA?9?$AAb?$AAa?$AA?9?$AAc?$AAy?$AAr?$AAl?$AA?$AA@ 1010f50c     LIBCMT:winapinls.obj
 0002:0000c524       ??_C@_1BG@JLBENFOE@?$AAs?$AAr?$AA?9?$AAb?$AAa?$AA?9?$AAl?$AAa?$AAt?$AAn?$AA?$AA@ 1010f524     LIBCMT:winapinls.obj
 0002:0000c53c       ??_C@_1BG@KODPNHE@?$AAs?$AAr?$AA?9?$AAs?$AAp?$AA?9?$AAc?$AAy?$AAr?$AAl?$AA?$AA@ 1010f53c     LIBCMT:winapinls.obj
 0002:0000c554       ??_C@_1BG@CIOGKHPB@?$AAs?$AAr?$AA?9?$AAs?$AAp?$AA?9?$AAl?$AAa?$AAt?$AAn?$AA?$AA@ 1010f554     LIBCMT:winapinls.obj
 0002:0000c56c       ??_C@_1M@NGFJLMAC@?$AAs?$AAv?$AA?9?$AAf?$AAi?$AA?$AA@ 1010f56c     LIBCMT:winapinls.obj
 0002:0000c578       ??_C@_1M@MPJEJAJC@?$AAs?$AAv?$AA?9?$AAs?$AAe?$AA?$AA@ 1010f578     LIBCMT:winapinls.obj
 0002:0000c584       ??_C@_1M@MPNDHLFK@?$AAs?$AAw?$AA?9?$AAk?$AAe?$AA?$AA@ 1010f584     LIBCMT:winapinls.obj
 0002:0000c590       ??_C@_1O@KOHBJJI@?$AAs?$AAy?$AAr?$AA?9?$AAs?$AAy?$AA?$AA@ 1010f590     LIBCMT:winapinls.obj
 0002:0000c5a0       ??_C@_1M@LDCEFHA@?$AAt?$AAa?$AA?9?$AAi?$AAn?$AA?$AA@ 1010f5a0     LIBCMT:winapinls.obj
 0002:0000c5ac       ??_C@_1M@CNJOFAK@?$AAt?$AAe?$AA?9?$AAi?$AAn?$AA?$AA@ 1010f5ac     LIBCMT:winapinls.obj
 0002:0000c5b8       ??_C@_1M@GNAECACD@?$AAt?$AAh?$AA?9?$AAt?$AAh?$AA?$AA@ 1010f5b8     LIBCMT:winapinls.obj
 0002:0000c5c4       ??_C@_1M@CHBIHOJO@?$AAt?$AAn?$AA?9?$AAz?$AAa?$AA?$AA@ 1010f5c4     LIBCMT:winapinls.obj
 0002:0000c5d0       ??_C@_1M@GCCMIGPJ@?$AAt?$AAr?$AA?9?$AAt?$AAr?$AA?$AA@ 1010f5d0     LIBCMT:winapinls.obj
 0002:0000c5dc       ??_C@_1M@CELMCNBK@?$AAt?$AAt?$AA?9?$AAr?$AAu?$AA?$AA@ 1010f5dc     LIBCMT:winapinls.obj
 0002:0000c5e8       ??_C@_1M@KLMCELGA@?$AAu?$AAk?$AA?9?$AAu?$AAa?$AA?$AA@ 1010f5e8     LIBCMT:winapinls.obj
 0002:0000c5f4       ??_C@_1M@EPAJJAJF@?$AAu?$AAr?$AA?9?$AAp?$AAk?$AA?$AA@ 1010f5f4     LIBCMT:winapinls.obj
 0002:0000c600       ??_C@_1BG@GEGPMCDJ@?$AAu?$AAz?$AA?9?$AAu?$AAz?$AA?9?$AAc?$AAy?$AAr?$AAl?$AA?$AA@ 1010f600     LIBCMT:winapinls.obj
 0002:0000c618       ??_C@_1BG@EGGKJILM@?$AAu?$AAz?$AA?9?$AAu?$AAz?$AA?9?$AAl?$AAa?$AAt?$AAn?$AA?$AA@ 1010f618     LIBCMT:winapinls.obj
 0002:0000c630       ??_C@_1M@GFOCLFF@?$AAv?$AAi?$AA?9?$AAv?$AAn?$AA?$AA@ 1010f630     LIBCMT:winapinls.obj
 0002:0000c63c       ??_C@_1M@CPAMEDFI@?$AAx?$AAh?$AA?9?$AAz?$AAa?$AA?$AA@ 1010f63c     LIBCMT:winapinls.obj
 0002:0000c648       ??_C@_1O@EBKIFIGN@?$AAz?$AAh?$AA?9?$AAc?$AAh?$AAs?$AA?$AA@ 1010f648     LIBCMT:winapinls.obj
 0002:0000c658       ??_C@_1O@NMHPGANE@?$AAz?$AAh?$AA?9?$AAc?$AAh?$AAt?$AA?$AA@ 1010f658     LIBCMT:winapinls.obj
 0002:0000c668       ??_C@_1M@LPINJOMC@?$AAz?$AAh?$AA?9?$AAc?$AAn?$AA?$AA@ 1010f668     LIBCMT:winapinls.obj
 0002:0000c674       ??_C@_1M@OCJEJODD@?$AAz?$AAh?$AA?9?$AAh?$AAk?$AA?$AA@ 1010f674     LIBCMT:winapinls.obj
 0002:0000c680       ??_C@_1M@DNDLJINH@?$AAz?$AAh?$AA?9?$AAm?$AAo?$AA?$AA@ 1010f680     LIBCMT:winapinls.obj
 0002:0000c68c       ??_C@_1M@MBFDNDND@?$AAz?$AAh?$AA?9?$AAs?$AAg?$AA?$AA@ 1010f68c     LIBCMT:winapinls.obj
 0002:0000c698       ??_C@_1M@IMEPLEPE@?$AAz?$AAh?$AA?9?$AAt?$AAw?$AA?$AA@ 1010f698     LIBCMT:winapinls.obj
 0002:0000c6a4       ??_C@_1M@BBGHNHJP@?$AAz?$AAu?$AA?9?$AAz?$AAa?$AA?$AA@ 1010f6a4     LIBCMT:winapinls.obj
 0002:0000c6b0       ___lookuptable_s           1010f6b0     LIBCMT:outputs.obj
 0002:0000c710       __indefinite               1010f710     LIBCMT:87disp.obj
 0002:0000c71a       __piby2                    1010f71a     LIBCMT:87disp.obj
 0002:0000c748       __DEFAULT_CW_in_mem        1010f748     LIBCMT:common.obj
 0002:0000c74a       __pi_by_2_to_61            1010f74a     LIBCMT:common.obj
 0002:0000c914       ??_C@_08EHJDFFNH@__based?$CI?$AA@ 1010f914     LIBCMT:undname.obj
 0002:0000c920       ??_C@_07KOLFKCDI@__cdecl?$AA@ 1010f920     LIBCMT:undname.obj
 0002:0000c928       ??_C@_08GHMPAG@__pascal?$AA@ 1010f928     LIBCMT:undname.obj
 0002:0000c934       ??_C@_09IFJBGAPI@__stdcall?$AA@ 1010f934     LIBCMT:undname.obj
 0002:0000c940       ??_C@_0L@NPHFGOKO@__thiscall?$AA@ 1010f940     LIBCMT:undname.obj
 0002:0000c94c       ??_C@_0L@JMKHOMEK@__fastcall?$AA@ 1010f94c     LIBCMT:undname.obj
 0002:0000c958       ??_C@_0N@BCKKPABJ@__vectorcall?$AA@ 1010f958     LIBCMT:undname.obj
 0002:0000c968       ??_C@_09HIJEGCPM@__clrcall?$AA@ 1010f968     LIBCMT:undname.obj
 0002:0000c974       ??_C@_06GHPCKEAG@__eabi?$AA@ 1010f974     LIBCMT:undname.obj
 0002:0000c97c       ??_C@_07JOMMBBKO@__ptr64?$AA@ 1010f97c     LIBCMT:undname.obj
 0002:0000c984       ??_C@_0L@PILCLIHE@__restrict?$AA@ 1010f984     LIBCMT:undname.obj
 0002:0000c990       ??_C@_0M@GFIIJFMG@__unaligned?$AA@ 1010f990     LIBCMT:undname.obj
 0002:0000c99c       ??_C@_09DHDLOLLB@restrict?$CI?$AA@ 1010f99c     LIBCMT:undname.obj
 0002:0000c9a8       ??_C@_04NIHEBCM@?5new?$AA@ 1010f9a8     LIBCMT:undname.obj
 0002:0000c9b0       ??_C@_07FPCDHGMM@?5delete?$AA@ 1010f9b0     LIBCMT:undname.obj
 0002:0000c9b8       ??_C@_01NEMOKFLO@?$DN?$AA@ 1010f9b8     LIBCMT:undname.obj
 0002:0000c9bc       ??_C@_02GPIOPFAK@?$DO?$DO?$AA@ 1010f9bc     LIBCMT:undname.obj
 0002:0000c9c0       ??_C@_02FODMEDOG@?$DM?$DM?$AA@ 1010f9c0     LIBCMT:undname.obj
 0002:0000c9c4       ??_C@_01DCLJPIOD@?$CB?$AA@ 1010f9c4     LIBCMT:undname.obj
 0002:0000c9c8       ??_C@_02EGOFBIJA@?$DN?$DN?$AA@ 1010f9c8     LIBCMT:undname.obj
 0002:0000c9cc       ??_C@_02FDNJECIE@?$CB?$DN?$AA@ 1010f9cc     LIBCMT:undname.obj
 0002:0000c9d0       ??_C@_02GPECMEKF@?$FL?$FN?$AA@ 1010f9d0     LIBCMT:undname.obj
 0002:0000c9d4       ??_C@_08LHJFAFGD@operator?$AA@ 1010f9d4     LIBCMT:undname.obj
 0002:0000c9e0       ??_C@_02HBOOOICD@?9?$DO?$AA@ 1010f9e0     LIBCMT:undname.obj
 0002:0000c9e4       ??_C@_01NBENCBCI@?$CK?$AA@ 1010f9e4     LIBCMT:undname.obj
 0002:0000c9e8       ??_C@_02ECNGHCIF@?$CL?$CL?$AA@ 1010f9e8     LIBCMT:undname.obj
 0002:0000c9ec       ??_C@_02BAABKJLB@?9?9?$AA@ 1010f9ec     LIBCMT:undname.obj
 0002:0000c9f0       ??_C@_01JOAMLHOP@?9?$AA@   1010f9f0     LIBCMT:undname.obj
 0002:0000c9f4       ??_C@_01MIFGBAGJ@?$CL?$AA@ 1010f9f4     LIBCMT:undname.obj
 0002:0000c9f8       ??_C@_01HNPIGOCE@?$CG?$AA@ 1010f9f8     LIBCMT:undname.obj
 0002:0000c9fc       ??_C@_03MNHNFDLC@?9?$DO?$CK?$AA@ 1010f9fc     LIBCMT:undname.obj
 0002:0000ca00       ??_C@_01KMDKNFGN@?1?$AA@   1010fa00     LIBCMT:undname.obj
 0002:0000ca04       ??_C@_01FGNFDNOH@?$CF?$AA@ 1010fa04     LIBCMT:undname.obj
 0002:0000ca08       ??_C@_01MNNFJEPP@?$DM?$AA@ 1010fa08     LIBCMT:undname.obj
 0002:0000ca0c       ??_C@_02EHCHHCKH@?$DM?$DN?$AA@ 1010fa0c     LIBCMT:undname.obj
 0002:0000ca10       ??_C@_01PPODPGHN@?$DO?$AA@ 1010fa10     LIBCMT:undname.obj
 0002:0000ca14       ??_C@_02EEKDKGMJ@?$DO?$DN?$AA@ 1010fa14     LIBCMT:undname.obj
 0002:0000ca18       ??_C@_01IHBHIGKO@?0?$AA@   1010fa18     LIBCMT:undname.obj
 0002:0000ca1c       ??_C@_02HCKGKOFO@?$CI?$CJ?$AA@ 1010fa1c     LIBCMT:undname.obj
 0002:0000ca20       ??_C@_01PJKLJHI@?$HO?$AA@  1010fa20     LIBCMT:undname.obj
 0002:0000ca24       ??_C@_01JKBOJNNK@?$FO?$AA@ 1010fa24     LIBCMT:undname.obj
 0002:0000ca28       ??_C@_02PPKAJPJL@?$CG?$CG?$AA@ 1010fa28     LIBCMT:undname.obj
 0002:0000ca2c       ??_C@_02NONPIBCD@?$HM?$HM?$AA@ 1010fa2c     LIBCMT:undname.obj
 0002:0000ca30       ??_C@_02FPIMKNGF@?$CK?$DN?$AA@ 1010fa30     LIBCMT:undname.obj
 0002:0000ca34       ??_C@_02FOEOMHFC@?$CL?$DN?$AA@ 1010fa34     LIBCMT:undname.obj
 0002:0000ca38       ??_C@_02FKMDLLOA@?9?$DN?$AA@ 1010fa38     LIBCMT:undname.obj
 0002:0000ca3c       ??_C@_02FJEHGPIO@?1?$DN?$AA@ 1010fa3c     LIBCMT:undname.obj
 0002:0000ca40       ??_C@_02FENAOKFI@?$CF?$DN?$AA@ 1010fa40     LIBCMT:undname.obj
 0002:0000ca44       ??_C@_03IKFCCPFF@?$DO?$DO?$DN?$AA@ 1010fa44     LIBCMT:undname.obj
 0002:0000ca48       ??_C@_03CDNPDDLA@?$DM?$DM?$DN?$AA@ 1010fa48     LIBCMT:undname.obj
 0002:0000ca4c       ??_C@_02FGJGFEAB@?$CG?$DN?$AA@ 1010fa4c     LIBCMT:undname.obj
 0002:0000ca50       ??_C@_02DHLNPPGH@?$HM?$DN?$AA@ 1010fa50     LIBCMT:undname.obj
 0002:0000ca54       ??_C@_02MHEGNOJ@?$FO?$DN?$AA@ 1010fa54     LIBCMT:undname.obj
 0002:0000ca58       ??_C@_09IFPLHPGF@?$GAvftable?8?$AA@ 1010fa58     LIBCMT:undname.obj
 0002:0000ca64       ??_C@_09BLBHBJP@?$GAvbtable?8?$AA@ 1010fa64     LIBCMT:undname.obj
 0002:0000ca70       ??_C@_07FEEIOKP@?$GAvcall?8?$AA@ 1010fa70     LIBCMT:undname.obj
 0002:0000ca78       ??_C@_08LLFFHHDJ@?$GAtypeof?8?$AA@ 1010fa78     LIBCMT:undname.obj
 0002:0000ca84       ??_C@_0BF@KDPPACIK@?$GAlocal?5static?5guard?8?$AA@ 1010fa84     LIBCMT:undname.obj
 0002:0000ca9c       ??_C@_08OBABFOLI@?$GAstring?8?$AA@ 1010fa9c     LIBCMT:undname.obj
 0002:0000caa8       ??_C@_0BD@JDLKDPAB@?$GAvbase?5destructor?8?$AA@ 1010faa8     LIBCMT:undname.obj
 0002:0000cabc       ??_C@_0BN@DEGPLNFK@?$GAvector?5deleting?5destructor?8?$AA@ 1010fabc     LIBCMT:undname.obj
 0002:0000cadc       ??_C@_0BO@OBMKPJIG@?$GAdefault?5constructor?5closure?8?$AA@ 1010fadc     LIBCMT:undname.obj
 0002:0000cafc       ??_C@_0BN@IMDCHIKM@?$GAscalar?5deleting?5destructor?8?$AA@ 1010fafc     LIBCMT:undname.obj
 0002:0000cb1c       ??_C@_0BO@PFGOCPJJ@?$GAvector?5constructor?5iterator?8?$AA@ 1010fb1c     LIBCMT:undname.obj
 0002:0000cb3c       ??_C@_0BN@LFPFMEDL@?$GAvector?5destructor?5iterator?8?$AA@ 1010fb3c     LIBCMT:undname.obj
 0002:0000cb5c       ??_C@_0CE@IKBNEHA@?$GAvector?5vbase?5constructor?5iterat@ 1010fb5c     LIBCMT:undname.obj
 0002:0000cb80       ??_C@_0BL@NILFHHPC@?$GAvirtual?5displacement?5map?8?$AA@ 1010fb80     LIBCMT:undname.obj
 0002:0000cb9c       ??_C@_0CB@JONCMFFK@?$GAeh?5vector?5constructor?5iterator?8@ 1010fb9c     LIBCMT:undname.obj
 0002:0000cbc0       ??_C@_0CA@GCEOPDGL@?$GAeh?5vector?5destructor?5iterator?8?$AA@ 1010fbc0     LIBCMT:undname.obj
 0002:0000cbe0       ??_C@_0CH@OOJPLCPH@?$GAeh?5vector?5vbase?5constructor?5ite@ 1010fbe0     LIBCMT:undname.obj
 0002:0000cc08       ??_C@_0BL@LLKPOHJI@?$GAcopy?5constructor?5closure?8?$AA@ 1010fc08     LIBCMT:undname.obj
 0002:0000cc24       ??_C@_0BA@KBCDOMBN@?$GAudt?5returning?8?$AA@ 1010fc24     LIBCMT:undname.obj
 0002:0000cc34       ??_C@_03KLGMFNMG@?$GAEH?$AA@ 1010fc34     LIBCMT:undname.obj
 0002:0000cc38       ??_C@_05KHLCHHI@?$GARTTI?$AA@ 1010fc38     LIBCMT:undname.obj
 0002:0000cc40       ??_C@_0BA@KKLDJDLB@?$GAlocal?5vftable?8?$AA@ 1010fc40     LIBCMT:undname.obj
 0002:0000cc50       ??_C@_0CE@IIHCMGGL@?$GAlocal?5vftable?5constructor?5closu@ 1010fc50     LIBCMT:undname.obj
 0002:0000cc74       ??_C@_06FHBGPFGH@?5new?$FL?$FN?$AA@ 1010fc74     LIBCMT:undname.obj
 0002:0000cc7c       ??_C@_09LBNFPBCA@?5delete?$FL?$FN?$AA@ 1010fc7c     LIBCMT:undname.obj
 0002:0000cc88       ??_C@_0P@HJKNJFNN@?$GAomni?5callsig?8?$AA@ 1010fc88     LIBCMT:undname.obj
 0002:0000cc98       ??_C@_0BL@CNOONJFP@?$GAplacement?5delete?5closure?8?$AA@ 1010fc98     LIBCMT:undname.obj
 0002:0000ccb4       ??_C@_0BN@CKNJLHMB@?$GAplacement?5delete?$FL?$FN?5closure?8?$AA@ 1010fcb4     LIBCMT:undname.obj
 0002:0000ccd4       ??_C@_0CG@CFDHKGGD@?$GAmanaged?5vector?5constructor?5iter@ 1010fcd4     LIBCMT:undname.obj
 0002:0000ccfc       ??_C@_0CF@IMGKMJNO@?$GAmanaged?5vector?5destructor?5itera@ 1010fcfc     LIBCMT:undname.obj
 0002:0000cd24       ??_C@_0CG@HLDDJMAG@?$GAeh?5vector?5copy?5constructor?5iter@ 1010fd24     LIBCMT:undname.obj
 0002:0000cd4c       ??_C@_0CM@FCBBDIGB@?$GAeh?5vector?5vbase?5copy?5constructo@ 1010fd4c     LIBCMT:undname.obj
 0002:0000cd78       ??_C@_0BL@CLIPGLGB@?$GAdynamic?5initializer?5for?5?8?$AA@ 1010fd78     LIBCMT:undname.obj
 0002:0000cd94       ??_C@_0CB@PDBIFEP@?$GAdynamic?5atexit?5destructor?5for?5?8@ 1010fd94     LIBCMT:undname.obj
 0002:0000cdb8       ??_C@_0CD@CGAJBKEJ@?$GAvector?5copy?5constructor?5iterato@ 1010fdb8     LIBCMT:undname.obj
 0002:0000cddc       ??_C@_0CJ@GJELGAMM@?$GAvector?5vbase?5copy?5constructor?5i@ 1010fddc     LIBCMT:undname.obj
 0002:0000ce08       ??_C@_0CL@FGIJHLCE@?$GAmanaged?5vector?5copy?5constructor@ 1010fe08     LIBCMT:undname.obj
 0002:0000ce34       ??_C@_0BM@PMGGMLDN@?$GAlocal?5static?5thread?5guard?8?$AA@ 1010fe34     LIBCMT:undname.obj
 0002:0000ce50       ??_C@_0BC@DAFEJGAK@?5Type?5Descriptor?8?$AA@ 1010fe50     LIBCMT:undname.obj
 0002:0000ce64       ??_C@_0BM@LDKODKLH@?5Base?5Class?5Descriptor?5at?5?$CI?$AA@ 1010fe64     LIBCMT:undname.obj
 0002:0000ce80       ??_C@_0BD@LGICGFMM@?5Base?5Class?5Array?8?$AA@ 1010fe80     LIBCMT:undname.obj
 0002:0000ce94       ??_C@_0BN@MECKDCOJ@?5Class?5Hierarchy?5Descriptor?8?$AA@ 1010fe94     LIBCMT:undname.obj
 0002:0000ceb4       ??_C@_0BK@CFCOFLF@?5Complete?5Object?5Locator?8?$AA@ 1010feb4     LIBCMT:undname.obj
 0002:0000ced0       ??_C@_04HEJADOOB@CV?3?5?$AA@ 1010fed0     LIBCMT:undname.obj
 0002:0000ced8       ??_C@_02MOLJINC@?3?3?$AA@  1010fed8     LIBCMT:undname.obj
 0002:0000cedc       ??_C@_0BE@JAEOCHPE@template?9parameter?9?$AA@ 1010fedc     LIBCMT:undname.obj
 0002:0000cef0       ??_C@_0O@KHGCOMHP@generic?9type?9?$AA@ 1010fef0     LIBCMT:undname.obj
 0002:0000cf00       ??_C@_01NLNLIGKH@?$GA?$AA@ 1010ff00     LIBCMT:undname.obj
 0002:0000cf04       ??_C@_01GEODFPGF@?8?$AA@   1010ff04     LIBCMT:undname.obj
 0002:0000cf08       ??_C@_0BG@JNJLAMPM@?$GAanonymous?5namespace?8?$AA@ 1010ff08     LIBCMT:undname.obj
 0002:0000cf20       ??_C@_02OHHJMEON@?8?8?$AA@ 1010ff20     LIBCMT:undname.obj
 0002:0000cf24       ??_C@_0BN@IBLMMFAP@?$GAnon?9type?9template?9parameter?$AA@ 1010ff24     LIBCMT:undname.obj
 0002:0000cf44       ??_C@_04GKJNKENE@void?$AA@ 1010ff44     LIBCMT:undname.obj
 0002:0000cf4c       ??_C@_0BE@EODMJLIF@?$GAtemplate?9parameter?$AA@ 1010ff4c     LIBCMT:undname.obj
 0002:0000cf60       ??_C@_03KHICJKCI@?4?4?4?$AA@ 1010ff60     LIBCMT:undname.obj
 0002:0000cf64       ??_C@_04HIBGFPH@NULL?$AA@  1010ff64     LIBCMT:undname.obj
 0002:0000cf6c       ??_C@_03OPGICMGF@?$HN?8?5?$AA@ 1010ff6c     LIBCMT:undname.obj
 0002:0000cf70       ??_C@_02IGFCGPIL@?$HN?8?$AA@ 1010ff70     LIBCMT:undname.obj
 0002:0000cf74       ??_C@_01CLKCMJKC@?5?$AA@   1010ff74     LIBCMT:undname.obj
 0002:0000cf78       ??_C@_0N@CBHHHENL@?$GAvtordispex?$HL?$AA@ 1010ff78     LIBCMT:undname.obj
 0002:0000cf88       ??_C@_0L@GHPFDFH@?$GAvtordisp?$HL?$AA@ 1010ff88     LIBCMT:undname.obj
 0002:0000cf94       ??_C@_0L@HNGCOGAE@?$GAadjustor?$HL?$AA@ 1010ff94     LIBCMT:undname.obj
 0002:0000cfa0       ??_C@_0CB@KJDOOODE@?$GAlocal?5static?5destructor?5helper?8@ 1010ffa0     LIBCMT:undname.obj
 0002:0000cfc4       ??_C@_0DB@ILEFOCIJ@?$GAtemplate?5static?5data?5member?5con@ 1010ffc4     LIBCMT:undname.obj
 0002:0000cff8       ??_C@_0DA@HGFJFBBE@?$GAtemplate?5static?5data?5member?5des@ 1010fff8     LIBCMT:undname.obj
 0002:0000d028       ??_C@_07PGOEDBHP@static?5?$AA@ 10110028     LIBCMT:undname.obj
 0002:0000d030       ??_C@_08NIEOINHE@virtual?5?$AA@ 10110030     LIBCMT:undname.obj
 0002:0000d03c       ??_C@_09LAPHOOG@private?3?5?$AA@ 1011003c     LIBCMT:undname.obj
 0002:0000d048       ??_C@_0M@GAIFPFIP@protected?3?5?$AA@ 10110048     LIBCMT:undname.obj
 0002:0000d054       ??_C@_08GPDDCMKI@public?3?5?$AA@ 10110054     LIBCMT:undname.obj
 0002:0000d060       ??_C@_08KJLFOPNE@?$FLthunk?$FN?3?$AA@ 10110060     LIBCMT:undname.obj
 0002:0000d06c       ??_C@_0M@DHNBOJMP@extern?5?$CCC?$CC?5?$AA@ 1011006c     LIBCMT:undname.obj
 0002:0000d078       ??_C@_02KCKGHPCA@?$CJ?5?$AA@ 10110078     LIBCMT:undname.obj
 0002:0000d07c       ??_C@_05CIHEBHNO@char?5?$AA@ 1011007c     LIBCMT:undname.obj
 0002:0000d084       ??_C@_06EHJMALKF@short?5?$AA@ 10110084     LIBCMT:undname.obj
 0002:0000d08c       ??_C@_04LAHKHJMA@int?5?$AA@ 1011008c     LIBCMT:undname.obj
 0002:0000d094       ??_C@_05CJIMAING@long?5?$AA@ 10110094     LIBCMT:undname.obj
 0002:0000d09c       ??_C@_09EBBEKKIH@unsigned?5?$AA@ 1011009c     LIBCMT:undname.obj
 0002:0000d0a8       ??_C@_05BEFAKPML@void?5?$AA@ 101100a8     LIBCMT:undname.obj
 0002:0000d0b0       ??_C@_08PABEKFH@volatile?$AA@ 101100b0     LIBCMT:undname.obj
 0002:0000d0bc       ??_C@_0P@GCOCNKDM@std?3?3nullptr_t?$AA@ 101100bc     LIBCMT:undname.obj
 0002:0000d0cc       ??_C@_0L@EGPHHEKN@?$DMellipsis?$DO?$AA@ 101100cc     LIBCMT:undname.obj
 0002:0000d0d8       ??_C@_04EENFHACM@?0?4?4?4?$AA@ 101100d8     LIBCMT:undname.obj
 0002:0000d0e0       ??_C@_0M@ELJOJFFH@?0?$DMellipsis?$DO?$AA@ 101100e0     LIBCMT:undname.obj
 0002:0000d0ec       ??_C@_07HDJPLPEK@?5throw?$CI?$AA@ 101100ec     LIBCMT:undname.obj
 0002:0000d0f4       ??_C@_03PBJBJNON@cpu?$AA@  101100f4     LIBCMT:undname.obj
 0002:0000d0f8       ??_C@_03DCBBJBAA@amp?$AA@  101100f8     LIBCMT:undname.obj
 0002:0000d0fc       ??_C@_02KEGNLNML@?0?5?$AA@ 101100fc     LIBCMT:undname.obj
 0002:0000d100       ??_C@_04ENMBGAPA@char?$AA@ 10110100     LIBCMT:undname.obj
 0002:0000d108       ??_C@_05BFKKPKCG@short?$AA@ 10110108     LIBCMT:undname.obj
 0002:0000d110       ??_C@_03JBIPMCLC@int?$AA@  10110110     LIBCMT:undname.obj
 0002:0000d114       ??_C@_04GOKPGOLB@long?$AA@ 10110114     LIBCMT:undname.obj
 0002:0000d11c       ??_C@_04DDKJGDCM@bool?$AA@ 1011011c     LIBCMT:undname.obj
 0002:0000d124       ??_C@_06EBGKOKIG@__int8?$AA@ 10110124     LIBCMT:undname.obj
 0002:0000d12c       ??_C@_07ICFHOGAF@__int16?$AA@ 1011012c     LIBCMT:undname.obj
 0002:0000d134       ??_C@_07OFLPPHGP@__int32?$AA@ 10110134     LIBCMT:undname.obj
 0002:0000d13c       ??_C@_07LFCOJCAC@__int64?$AA@ 1011013c     LIBCMT:undname.obj
 0002:0000d144       ??_C@_08GAHOLHEO@__int128?$AA@ 10110144     LIBCMT:undname.obj
 0002:0000d150       ??_C@_09EEKGDCPH@?$DMunknown?$DO?$AA@ 10110150     LIBCMT:undname.obj
 0002:0000d15c       ??_C@_07CLGGIAMF@wchar_t?$AA@ 1011015c     LIBCMT:undname.obj
 0002:0000d164       ??_C@_06GCICPBLB@__w64?5?$AA@ 10110164     LIBCMT:undname.obj
 0002:0000d16c       ??_C@_07NFANNNEC@UNKNOWN?$AA@ 1011016c     LIBCMT:undname.obj
 0002:0000d174       ??_C@_07EDHNAJHC@signed?5?$AA@ 10110174     LIBCMT:undname.obj
 0002:0000d17c       ??_C@_05BNCCCJPP@const?$AA@ 1011017c     LIBCMT:undname.obj
 0002:0000d184       ??_C@_09EFNPDFFP@?5volatile?$AA@ 10110184     LIBCMT:undname.obj
 0002:0000d190       ??_C@_0P@GCIFDJCJ@?$GAunknown?5ecsu?8?$AA@ 10110190     LIBCMT:undname.obj
 0002:0000d1a0       ??_C@_06MOJHIBMG@union?5?$AA@ 101101a0     LIBCMT:undname.obj
 0002:0000d1a8       ??_C@_07DIBCDNGL@struct?5?$AA@ 101101a8     LIBCMT:undname.obj
 0002:0000d1b0       ??_C@_06LJBABKPM@class?5?$AA@ 101101b0     LIBCMT:undname.obj
 0002:0000d1b8       ??_C@_08KOFANOFK@coclass?5?$AA@ 101101b8     LIBCMT:undname.obj
 0002:0000d1c4       ??_C@_0N@DLIEFKNA@cointerface?5?$AA@ 101101c4     LIBCMT:undname.obj
 0002:0000d1d4       ??_C@_05LJGMCFOG@enum?5?$AA@ 101101d4     LIBCMT:undname.obj
 0002:0000d1dc       ??_C@_09GAIEOBLP@volatile?5?$AA@ 101101dc     LIBCMT:undname.obj
 0002:0000d1e8       ??_C@_06LIJLOJAG@const?5?$AA@ 101101e8     LIBCMT:undname.obj
 0002:0000d1f0       ??_C@_0M@EALIELKG@cli?3?3array?$DM?$AA@ 101101f0     LIBCMT:undname.obj
 0002:0000d1fc       ??_C@_0O@GKABPPIF@cli?3?3pin_ptr?$DM?$AA@ 101101fc     LIBCMT:undname.obj
 0002:0000d20c       ??_C@_02GOGNNPBN@?$CJ?$FL?$AA@ 1011020c     LIBCMT:undname.obj
 0002:0000d210       ??_C@_06EEGAIFAK@?$HLflat?$HN?$AA@ 10110210     LIBCMT:undname.obj
 0002:0000d218       ??_C@_05JIBOFOHK@?$HLfor?5?$AA@ 10110218     LIBCMT:undname.obj
 0002:0000d220       ??_C@_02MDINNEEG@s?5?$AA@  10110220     LIBCMT:undname.obj
 0002:0000d228       ??_7DNameNode@@6B@         10110228     LIBCMT:undname.obj
 0002:0000d238       ??_7charNode@@6B@          10110238     LIBCMT:undname.obj
 0002:0000d248       ??_7pcharNode@@6B@         10110248     LIBCMT:undname.obj
 0002:0000d258       ??_7pDNameNode@@6B@        10110258     LIBCMT:undname.obj
 0002:0000d268       ??_7DNameStatusNode@@6B@   10110268     LIBCMT:undname.obj
 0002:0000d278       ??_7pairNode@@6B@          10110278     LIBCMT:undname.obj
 0002:0000d284       ??_C@_04OKOHEJBO@?5?$DP?$DP?5?$AA@ 10110284     LIBCMT:undname.obj
 0002:0000d290       ___lc_category             10110290     LIBCMT:wsetloca.obj
 0002:0000d2d8       ??_C@_1O@GIFLHMA@?$AAL?$AAC?$AA_?$AAA?$AAL?$AAL?$AA?$AA@ 101102d8     LIBCMT:wsetloca.obj
 0002:0000d2e8       ??_C@_1BG@PPOMIBNJ@?$AAL?$AAC?$AA_?$AAC?$AAO?$AAL?$AAL?$AAA?$AAT?$AAE?$AA?$AA@ 101102e8     LIBCMT:wsetloca.obj
 0002:0000d300       ??_C@_1BC@FFJGAPJM@?$AAL?$AAC?$AA_?$AAC?$AAT?$AAY?$AAP?$AAE?$AA?$AA@ 10110300     LIBCMT:wsetloca.obj
 0002:0000d314       ??_C@_1BI@PCKFNJFB@?$AAL?$AAC?$AA_?$AAM?$AAO?$AAN?$AAE?$AAT?$AAA?$AAR?$AAY?$AA?$AA@ 10110314     LIBCMT:wsetloca.obj
 0002:0000d32c       ??_C@_1BG@ENIEDKID@?$AAL?$AAC?$AA_?$AAN?$AAU?$AAM?$AAE?$AAR?$AAI?$AAC?$AA?$AA@ 1011032c     LIBCMT:wsetloca.obj
 0002:0000d344       ??_C@_1BA@HAAOMIIG@?$AAL?$AAC?$AA_?$AAT?$AAI?$AAM?$AAE?$AA?$AA@ 10110344     LIBCMT:wsetloca.obj
 0002:0000d3d8       ??_C@_15NBPDDFIP@?$AA?$DN?$AA?$DL?$AA?$AA@ 101103d8     LIBCMT:wsetloca.obj
 0002:0000d3e0       ??_C@_13PJJBFPED@?$AA?$DL?$AA?$AA@ 101103e0     LIBCMT:wsetloca.obj
 0002:0000d3e4       ??_C@_13NMPKAAJP@?$AA?$DN?$AA?$AA@ 101103e4     LIBCMT:wsetloca.obj
 0002:0000d3e8       ??_C@_13FHBKNHDA@?$AAC?$AA?$AA@ 101103e8     LIBCMT:wsetloca.obj
 0002:0000d3ec       ??_C@_17MBJJLFDM@?$AA_?$AA?4?$AA?0?$AA?$AA@ 101103ec     LIBCMT:wsetloca.obj
 0002:0000d3f4       ??_C@_13ENNFDPBH@?$AA_?$AA?$AA@ 101103f4     LIBCMT:wsetloca.obj
 0002:0000d3f8       ??_C@_13JOFGPIOO@?$AA?4?$AA?$AA@ 101103f8     LIBCMT:wsetloca.obj
 0002:0000d3fc       ??_C@_06PGGFOGJG@1?$CDSNAN?$AA@ 101103fc     LIBCMT:x10fout.obj
 0002:0000d404       ??_C@_05PHHOCPM@1?$CDIND?$AA@ 10110404     LIBCMT:x10fout.obj
 0002:0000d40c       ??_C@_05DNEBIAHO@1?$CDINF?$AA@ 1011040c     LIBCMT:x10fout.obj
 0002:0000d414       ??_C@_06IMKFLFPG@1?$CDQNAN?$AA@ 10110414     LIBCMT:x10fout.obj
 0002:0000d420       ___newctype                10110420     LIBCMT:ctype.obj
 0002:0000d720       __wctype                   10110720     LIBCMT:ctype.obj
 0002:0000d928       ___newclmap                10110928     LIBCMT:ctype.obj
 0002:0000daa8       ___newcumap                10110aa8     LIBCMT:ctype.obj
 0002:0000dc28       ??_C@_0M@HHGEPIBF@CreateFile2?$AA@ 10110c28     LIBCMT:wopen.obj
 0002:0000dc34       ??_C@_1BA@BALFACEM@?$AAC?$AAO?$AAN?$AAO?$AAU?$AAT?$AA$?$AA?$AA@ 10110c34     LIBCMT:initcon.obj
 0002:0000dc48       ___rg_language             10110c48     LIBCMT:getqloc.obj
 0002:0000df54       ??_C@_1BC@LLOKLNP@?$AAa?$AAm?$AAe?$AAr?$AAi?$AAc?$AAa?$AAn?$AA?$AA@ 10110f54     LIBCMT:getqloc.obj
 0002:0000df68       ??_C@_1CC@HEIGCDGG@?$AAa?$AAm?$AAe?$AAr?$AAi?$AAc?$AAa?$AAn?$AA?5?$AAe?$AAn?$AAg?$AAl?$AAi?$AAs?$AAh?$AA?$AA@ 10110f68     LIBCMT:getqloc.obj
 0002:0000df8c       ??_C@_1CC@IHCNOMIN@?$AAa?$AAm?$AAe?$AAr?$AAi?$AAc?$AAa?$AAn?$AA?9?$AAe?$AAn?$AAg?$AAl?$AAi?$AAs?$AAh?$AA?$AA@ 10110f8c     LIBCMT:getqloc.obj
 0002:0000dfb0       ??_C@_1BG@GKAGPCGG@?$AAa?$AAu?$AAs?$AAt?$AAr?$AAa?$AAl?$AAi?$AAa?$AAn?$AA?$AA@ 10110fb0     LIBCMT:getqloc.obj
 0002:0000dfc8       ??_C@_1BA@GMENCENF@?$AAb?$AAe?$AAl?$AAg?$AAi?$AAa?$AAn?$AA?$AA@ 10110fc8     LIBCMT:getqloc.obj
 0002:0000dfd8       ??_C@_1BC@PJMIIAAN@?$AAc?$AAa?$AAn?$AAa?$AAd?$AAi?$AAa?$AAn?$AA?$AA@ 10110fd8     LIBCMT:getqloc.obj
 0002:0000dfec       ??_C@_17NOIMNFBF@?$AAc?$AAh?$AAh?$AA?$AA@ 10110fec     LIBCMT:getqloc.obj
 0002:0000dff4       ??_C@_17GGDALCHA@?$AAc?$AAh?$AAi?$AA?$AA@ 10110ff4     LIBCMT:getqloc.obj
 0002:0000dffc       ??_C@_1BA@NPNJKIBL@?$AAc?$AAh?$AAi?$AAn?$AAe?$AAs?$AAe?$AA?$AA@ 10110ffc     LIBCMT:getqloc.obj
 0002:0000e00c       ??_C@_1CC@DINBAMMJ@?$AAc?$AAh?$AAi?$AAn?$AAe?$AAs?$AAe?$AA?9?$AAh?$AAo?$AAn?$AAg?$AAk?$AAo?$AAn?$AAg?$AA?$AA@ 1011100c     LIBCMT:getqloc.obj
 0002:0000e030       ??_C@_1CG@IOBJPACO@?$AAc?$AAh?$AAi?$AAn?$AAe?$AAs?$AAe?$AA?9?$AAs?$AAi?$AAm?$AAp?$AAl?$AAi?$AAf?$AAi?$AAe?$AAd?$AA?$AA@ 10111030     LIBCMT:getqloc.obj
 0002:0000e058       ??_C@_1CE@GAJNDCKG@?$AAc?$AAh?$AAi?$AAn?$AAe?$AAs?$AAe?$AA?9?$AAs?$AAi?$AAn?$AAg?$AAa?$AAp?$AAo?$AAr?$AAe?$AA?$AA@ 10111058     LIBCMT:getqloc.obj
 0002:0000e07c       ??_C@_1CI@PAJPIOOD@?$AAc?$AAh?$AAi?$AAn?$AAe?$AAs?$AAe?$AA?9?$AAt?$AAr?$AAa?$AAd?$AAi?$AAt?$AAi?$AAo?$AAn?$AAa?$AAl?$AA?$AA@ 1011107c     LIBCMT:getqloc.obj
 0002:0000e0a4       ??_C@_1BM@NILJBMMD@?$AAd?$AAu?$AAt?$AAc?$AAh?$AA?9?$AAb?$AAe?$AAl?$AAg?$AAi?$AAa?$AAn?$AA?$AA@ 101110a4     LIBCMT:getqloc.obj
 0002:0000e0c0       ??_C@_1CC@OOJPJNEJ@?$AAe?$AAn?$AAg?$AAl?$AAi?$AAs?$AAh?$AA?9?$AAa?$AAm?$AAe?$AAr?$AAi?$AAc?$AAa?$AAn?$AA?$AA@ 101110c0     LIBCMT:getqloc.obj
 0002:0000e0e4       ??_C@_1BI@IOLFEEM@?$AAe?$AAn?$AAg?$AAl?$AAi?$AAs?$AAh?$AA?9?$AAa?$AAu?$AAs?$AA?$AA@ 101110e4     LIBCMT:getqloc.obj
 0002:0000e0fc       ??_C@_1BO@HFFNLENJ@?$AAe?$AAn?$AAg?$AAl?$AAi?$AAs?$AAh?$AA?9?$AAb?$AAe?$AAl?$AAi?$AAz?$AAe?$AA?$AA@ 101110fc     LIBCMT:getqloc.obj
 0002:0000e11c       ??_C@_1BI@HAPKJMPO@?$AAe?$AAn?$AAg?$AAl?$AAi?$AAs?$AAh?$AA?9?$AAc?$AAa?$AAn?$AA?$AA@ 1011111c     LIBCMT:getqloc.obj
 0002:0000e134       ??_C@_1CE@HLNDMIOJ@?$AAe?$AAn?$AAg?$AAl?$AAi?$AAs?$AAh?$AA?9?$AAc?$AAa?$AAr?$AAi?$AAb?$AAb?$AAe?$AAa?$AAn?$AA?$AA@ 10111134     LIBCMT:getqloc.obj
 0002:0000e158       ??_C@_1BI@LDHJHHAC@?$AAe?$AAn?$AAg?$AAl?$AAi?$AAs?$AAh?$AA?9?$AAi?$AAr?$AAe?$AA?$AA@ 10111158     LIBCMT:getqloc.obj
 0002:0000e170       ??_C@_1CA@NJMMCFOC@?$AAe?$AAn?$AAg?$AAl?$AAi?$AAs?$AAh?$AA?9?$AAj?$AAa?$AAm?$AAa?$AAi?$AAc?$AAa?$AA?$AA@ 10111170     LIBCMT:getqloc.obj
 0002:0000e190       ??_C@_1BG@BHJEBBGG@?$AAe?$AAn?$AAg?$AAl?$AAi?$AAs?$AAh?$AA?9?$AAn?$AAz?$AA?$AA@ 10111190     LIBCMT:getqloc.obj
 0002:0000e1a8       ??_C@_1CK@FGOEJJCO@?$AAe?$AAn?$AAg?$AAl?$AAi?$AAs?$AAh?$AA?9?$AAs?$AAo?$AAu?$AAt?$AAh?$AA?5?$AAa?$AAf?$AAr?$AAi?$AAc?$AAa?$AA?$AA@ 101111a8     LIBCMT:getqloc.obj
 0002:0000e1d4       ??_C@_1DE@PDBJPCJ@?$AAe?$AAn?$AAg?$AAl?$AAi?$AAs?$AAh?$AA?9?$AAt?$AAr?$AAi?$AAn?$AAi?$AAd?$AAa?$AAd?$AA?5?$AAy?$AA?5?$AAt?$AAo?$AAb?$AAa?$AAg?$AAo?$AA?$AA@ 101111d4     LIBCMT:getqloc.obj
 0002:0000e208       ??_C@_1BG@JGCANDME@?$AAe?$AAn?$AAg?$AAl?$AAi?$AAs?$AAh?$AA?9?$AAu?$AAk?$AA?$AA@ 10111208     LIBCMT:getqloc.obj
 0002:0000e220       ??_C@_1BG@DINKMLE@?$AAe?$AAn?$AAg?$AAl?$AAi?$AAs?$AAh?$AA?9?$AAu?$AAs?$AA?$AA@ 10111220     LIBCMT:getqloc.obj
 0002:0000e238       ??_C@_1BI@NMFDBHJE@?$AAe?$AAn?$AAg?$AAl?$AAi?$AAs?$AAh?$AA?9?$AAu?$AAs?$AAa?$AA?$AA@ 10111238     LIBCMT:getqloc.obj
 0002:0000e250       ??_C@_1BO@OIHKJKII@?$AAf?$AAr?$AAe?$AAn?$AAc?$AAh?$AA?9?$AAb?$AAe?$AAl?$AAg?$AAi?$AAa?$AAn?$AA?$AA@ 10111250     LIBCMT:getqloc.obj
 0002:0000e270       ??_C@_1CA@NKAELJKI@?$AAf?$AAr?$AAe?$AAn?$AAc?$AAh?$AA?9?$AAc?$AAa?$AAn?$AAa?$AAd?$AAi?$AAa?$AAn?$AA?$AA@ 10111270     LIBCMT:getqloc.obj
 0002:0000e290       ??_C@_1CE@MGKCNLGN@?$AAf?$AAr?$AAe?$AAn?$AAc?$AAh?$AA?9?$AAl?$AAu?$AAx?$AAe?$AAm?$AAb?$AAo?$AAu?$AAr?$AAg?$AA?$AA@ 10111290     LIBCMT:getqloc.obj
 0002:0000e2b4       ??_C@_1BK@CEGEAILM@?$AAf?$AAr?$AAe?$AAn?$AAc?$AAh?$AA?9?$AAs?$AAw?$AAi?$AAs?$AAs?$AA?$AA@ 101112b4     LIBCMT:getqloc.obj
 0002:0000e2d0       ??_C@_1CA@PAFKEOCC@?$AAg?$AAe?$AAr?$AAm?$AAa?$AAn?$AA?9?$AAa?$AAu?$AAs?$AAt?$AAr?$AAi?$AAa?$AAn?$AA?$AA@ 101112d0     LIBCMT:getqloc.obj
 0002:0000e2f0       ??_C@_1CI@HCFHGOFD@?$AAg?$AAe?$AAr?$AAm?$AAa?$AAn?$AA?9?$AAl?$AAi?$AAc?$AAh?$AAt?$AAe?$AAn?$AAs?$AAt?$AAe?$AAi?$AAn?$AA?$AA@ 101112f0     LIBCMT:getqloc.obj
 0002:0000e318       ??_C@_1CE@FEDDNPDG@?$AAg?$AAe?$AAr?$AAm?$AAa?$AAn?$AA?9?$AAl?$AAu?$AAx?$AAe?$AAm?$AAb?$AAo?$AAu?$AAr?$AAg?$AA?$AA@ 10111318     LIBCMT:getqloc.obj
 0002:0000e33c       ??_C@_1BK@LIMINNMN@?$AAg?$AAe?$AAr?$AAm?$AAa?$AAn?$AA?9?$AAs?$AAw?$AAi?$AAs?$AAs?$AA?$AA@ 1011133c     LIBCMT:getqloc.obj
 0002:0000e358       ??_C@_1BM@LGMDBEPD@?$AAi?$AAr?$AAi?$AAs?$AAh?$AA?9?$AAe?$AAn?$AAg?$AAl?$AAi?$AAs?$AAh?$AA?$AA@ 10111358     LIBCMT:getqloc.obj
 0002:0000e374       ??_C@_1BM@NNCFBAEE@?$AAi?$AAt?$AAa?$AAl?$AAi?$AAa?$AAn?$AA?9?$AAs?$AAw?$AAi?$AAs?$AAs?$AA?$AA@ 10111374     LIBCMT:getqloc.obj
 0002:0000e390       ??_C@_1BE@FEDJNPIB@?$AAn?$AAo?$AAr?$AAw?$AAe?$AAg?$AAi?$AAa?$AAn?$AA?$AA@ 10111390     LIBCMT:getqloc.obj
 0002:0000e3a4       ??_C@_1CC@CILKDEIE@?$AAn?$AAo?$AAr?$AAw?$AAe?$AAg?$AAi?$AAa?$AAn?$AA?9?$AAb?$AAo?$AAk?$AAm?$AAa?$AAl?$AA?$AA@ 101113a4     LIBCMT:getqloc.obj
 0002:0000e3c8       ??_C@_1CE@DHMMHEPL@?$AAn?$AAo?$AAr?$AAw?$AAe?$AAg?$AAi?$AAa?$AAn?$AA?9?$AAn?$AAy?$AAn?$AAo?$AAr?$AAs?$AAk?$AA?$AA@ 101113c8     LIBCMT:getqloc.obj
 0002:0000e3ec       ??_C@_1CK@OPNMHECD@?$AAp?$AAo?$AAr?$AAt?$AAu?$AAg?$AAu?$AAe?$AAs?$AAe?$AA?9?$AAb?$AAr?$AAa?$AAz?$AAi?$AAl?$AAi?$AAa?$AAn?$AA?$AA@ 101113ec     LIBCMT:getqloc.obj
 0002:0000e418       ??_C@_1CE@KEEHCDB@?$AAs?$AAp?$AAa?$AAn?$AAi?$AAs?$AAh?$AA?9?$AAa?$AAr?$AAg?$AAe?$AAn?$AAt?$AAi?$AAn?$AAa?$AA?$AA@ 10111418     LIBCMT:getqloc.obj
 0002:0000e43c       ??_C@_1CA@GIAOLHJD@?$AAs?$AAp?$AAa?$AAn?$AAi?$AAs?$AAh?$AA?9?$AAb?$AAo?$AAl?$AAi?$AAv?$AAi?$AAa?$AA?$AA@ 1011143c     LIBCMT:getqloc.obj
 0002:0000e45c       ??_C@_1BM@OJNDFNPD@?$AAs?$AAp?$AAa?$AAn?$AAi?$AAs?$AAh?$AA?9?$AAc?$AAh?$AAi?$AAl?$AAe?$AA?$AA@ 1011145c     LIBCMT:getqloc.obj
 0002:0000e478       ??_C@_1CC@OCOLPALL@?$AAs?$AAp?$AAa?$AAn?$AAi?$AAs?$AAh?$AA?9?$AAc?$AAo?$AAl?$AAo?$AAm?$AAb?$AAi?$AAa?$AA?$AA@ 10111478     LIBCMT:getqloc.obj
 0002:0000e49c       ??_C@_1CG@BPOFMKBB@?$AAs?$AAp?$AAa?$AAn?$AAi?$AAs?$AAh?$AA?9?$AAc?$AAo?$AAs?$AAt?$AAa?$AA?5?$AAr?$AAi?$AAc?$AAa?$AA?$AA@ 1011149c     LIBCMT:getqloc.obj
 0002:0000e4c4       ??_C@_1DG@IGOBAPBB@?$AAs?$AAp?$AAa?$AAn?$AAi?$AAs?$AAh?$AA?9?$AAd?$AAo?$AAm?$AAi?$AAn?$AAi?$AAc?$AAa?$AAn?$AA?5?$AAr?$AAe?$AAp?$AAu?$AAb?$AAl?$AAi?$AAc?$AA?$AA@ 101114c4     LIBCMT:getqloc.obj
 0002:0000e4fc       ??_C@_1CA@JHAPGEGI@?$AAs?$AAp?$AAa?$AAn?$AAi?$AAs?$AAh?$AA?9?$AAe?$AAc?$AAu?$AAa?$AAd?$AAo?$AAr?$AA?$AA@ 101114fc     LIBCMT:getqloc.obj
 0002:0000e51c       ??_C@_1CI@LAPALJPP@?$AAs?$AAp?$AAa?$AAn?$AAi?$AAs?$AAh?$AA?9?$AAe?$AAl?$AA?5?$AAs?$AAa?$AAl?$AAv?$AAa?$AAd?$AAo?$AAr?$AA?$AA@ 1011151c     LIBCMT:getqloc.obj
 0002:0000e544       ??_C@_1CE@PDGBOFOM@?$AAs?$AAp?$AAa?$AAn?$AAi?$AAs?$AAh?$AA?9?$AAg?$AAu?$AAa?$AAt?$AAe?$AAm?$AAa?$AAl?$AAa?$AA?$AA@ 10111544     LIBCMT:getqloc.obj
 0002:0000e568       ??_C@_1CC@NBEBAODI@?$AAs?$AAp?$AAa?$AAn?$AAi?$AAs?$AAh?$AA?9?$AAh?$AAo?$AAn?$AAd?$AAu?$AAr?$AAa?$AAs?$AA?$AA@ 10111568     LIBCMT:getqloc.obj
 0002:0000e58c       ??_C@_1CA@LLKGHBMF@?$AAs?$AAp?$AAa?$AAn?$AAi?$AAs?$AAh?$AA?9?$AAm?$AAe?$AAx?$AAi?$AAc?$AAa?$AAn?$AA?$AA@ 1011158c     LIBCMT:getqloc.obj
 0002:0000e5ac       ??_C@_1BO@LKNDOIGD@?$AAs?$AAp?$AAa?$AAn?$AAi?$AAs?$AAh?$AA?9?$AAm?$AAo?$AAd?$AAe?$AAr?$AAn?$AA?$AA@ 101115ac     LIBCMT:getqloc.obj
 0002:0000e5cc       ??_C@_1CE@NMDMOEEB@?$AAs?$AAp?$AAa?$AAn?$AAi?$AAs?$AAh?$AA?9?$AAn?$AAi?$AAc?$AAa?$AAr?$AAa?$AAg?$AAu?$AAa?$AA?$AA@ 101115cc     LIBCMT:getqloc.obj
 0002:0000e5f0       ??_C@_1BO@LLCBEJGB@?$AAs?$AAp?$AAa?$AAn?$AAi?$AAs?$AAh?$AA?9?$AAp?$AAa?$AAn?$AAa?$AAm?$AAa?$AA?$AA@ 101115f0     LIBCMT:getqloc.obj
 0002:0000e610       ??_C@_1CC@FKPGGIHO@?$AAs?$AAp?$AAa?$AAn?$AAi?$AAs?$AAh?$AA?9?$AAp?$AAa?$AAr?$AAa?$AAg?$AAu?$AAa?$AAy?$AA?$AA@ 10111610     LIBCMT:getqloc.obj
 0002:0000e634       ??_C@_1BK@CDEIHOOP@?$AAs?$AAp?$AAa?$AAn?$AAi?$AAs?$AAh?$AA?9?$AAp?$AAe?$AAr?$AAu?$AA?$AA@ 10111634     LIBCMT:getqloc.obj
 0002:0000e650       ??_C@_1CI@GAHAKKGP@?$AAs?$AAp?$AAa?$AAn?$AAi?$AAs?$AAh?$AA?9?$AAp?$AAu?$AAe?$AAr?$AAt?$AAo?$AA?5?$AAr?$AAi?$AAc?$AAo?$AA?$AA@ 10111650     LIBCMT:getqloc.obj
 0002:0000e678       ??_C@_1CA@NKJBCAGP@?$AAs?$AAp?$AAa?$AAn?$AAi?$AAs?$AAh?$AA?9?$AAu?$AAr?$AAu?$AAg?$AAu?$AAa?$AAy?$AA?$AA@ 10111678     LIBCMT:getqloc.obj
 0002:0000e698       ??_C@_1CE@ODILCONM@?$AAs?$AAp?$AAa?$AAn?$AAi?$AAs?$AAh?$AA?9?$AAv?$AAe?$AAn?$AAe?$AAz?$AAu?$AAe?$AAl?$AAa?$AA?$AA@ 10111698     LIBCMT:getqloc.obj
 0002:0000e6bc       ??_C@_1CA@OBNMCGFO@?$AAs?$AAw?$AAe?$AAd?$AAi?$AAs?$AAh?$AA?9?$AAf?$AAi?$AAn?$AAl?$AAa?$AAn?$AAd?$AA?$AA@ 101116bc     LIBCMT:getqloc.obj
 0002:0000e6dc       ??_C@_1M@PIPDDPPI@?$AAs?$AAw?$AAi?$AAs?$AAs?$AA?$AA@ 101116dc     LIBCMT:getqloc.obj
 0002:0000e6e8       ??_C@_15GMFIMNFM@?$AAu?$AAs?$AA?$AA@ 101116e8     LIBCMT:getqloc.obj
 0002:0000e6f0       ??_C@_17HAEBFAGL@?$AAu?$AAs?$AAa?$AA?$AA@ 101116f0     LIBCMT:getqloc.obj
 0002:0000e6f8       ___rg_country              101116f8     LIBCMT:getqloc.obj
 0002:0000e80c       ??_C@_1BA@DPFJEPHB@?$AAa?$AAm?$AAe?$AAr?$AAi?$AAc?$AAa?$AA?$AA@ 1011180c     LIBCMT:getqloc.obj
 0002:0000e81c       ??_C@_1BA@ELOGGFK@?$AAb?$AAr?$AAi?$AAt?$AAa?$AAi?$AAn?$AA?$AA@ 1011181c     LIBCMT:getqloc.obj
 0002:0000e82c       ??_C@_1M@GHBGIGDA@?$AAc?$AAh?$AAi?$AAn?$AAa?$AA?$AA@ 1011182c     LIBCMT:getqloc.obj
 0002:0000e838       ??_C@_1M@NCHEJOPO@?$AAc?$AAz?$AAe?$AAc?$AAh?$AA?$AA@ 10111838     LIBCMT:getqloc.obj
 0002:0000e844       ??_C@_1BA@BKPAPBLA@?$AAe?$AAn?$AAg?$AAl?$AAa?$AAn?$AAd?$AA?$AA@ 10111844     LIBCMT:getqloc.obj
 0002:0000e854       ??_C@_1BM@HKBCKIPC@?$AAg?$AAr?$AAe?$AAa?$AAt?$AA?5?$AAb?$AAr?$AAi?$AAt?$AAa?$AAi?$AAn?$AA?$AA@ 10111854     LIBCMT:getqloc.obj
 0002:0000e870       ??_C@_1BA@PPCHPGJB@?$AAh?$AAo?$AAl?$AAl?$AAa?$AAn?$AAd?$AA?$AA@ 10111870     LIBCMT:getqloc.obj
 0002:0000e880       ??_C@_1BE@JBMPEGDG@?$AAh?$AAo?$AAn?$AAg?$AA?9?$AAk?$AAo?$AAn?$AAg?$AA?$AA@ 10111880     LIBCMT:getqloc.obj
 0002:0000e894       ??_C@_1BI@KOELBBPJ@?$AAn?$AAe?$AAw?$AA?9?$AAz?$AAe?$AAa?$AAl?$AAa?$AAn?$AAd?$AA?$AA@ 10111894     LIBCMT:getqloc.obj
 0002:0000e8ac       ??_C@_15HIEBHAIO@?$AAn?$AAz?$AA?$AA@ 101118ac     LIBCMT:getqloc.obj
 0002:0000e8b4       ??_C@_1BC@CHBCPFPI@?$AAp?$AAr?$AA?5?$AAc?$AAh?$AAi?$AAn?$AAa?$AA?$AA@ 101118b4     LIBCMT:getqloc.obj
 0002:0000e8c8       ??_C@_1BC@JAOIIFKD@?$AAp?$AAr?$AA?9?$AAc?$AAh?$AAi?$AAn?$AAa?$AA?$AA@ 101118c8     LIBCMT:getqloc.obj
 0002:0000e8dc       ??_C@_1BI@BEHPPHKC@?$AAp?$AAu?$AAe?$AAr?$AAt?$AAo?$AA?9?$AAr?$AAi?$AAc?$AAo?$AA?$AA@ 101118dc     LIBCMT:getqloc.obj
 0002:0000e8f4       ??_C@_1O@PAEOFKDI@?$AAs?$AAl?$AAo?$AAv?$AAa?$AAk?$AA?$AA@ 101118f4     LIBCMT:getqloc.obj
 0002:0000e904       ??_C@_1BK@FIHMCKAM@?$AAs?$AAo?$AAu?$AAt?$AAh?$AA?5?$AAa?$AAf?$AAr?$AAi?$AAc?$AAa?$AA?$AA@ 10111904     LIBCMT:getqloc.obj
 0002:0000e920       ??_C@_1BI@NAEOODKB@?$AAs?$AAo?$AAu?$AAt?$AAh?$AA?5?$AAk?$AAo?$AAr?$AAe?$AAa?$AA?$AA@ 10111920     LIBCMT:getqloc.obj
 0002:0000e938       ??_C@_1BK@FBDGGIFF@?$AAs?$AAo?$AAu?$AAt?$AAh?$AA?9?$AAa?$AAf?$AAr?$AAi?$AAc?$AAa?$AA?$AA@ 10111938     LIBCMT:getqloc.obj
 0002:0000e954       ??_C@_1BI@GHLEJDPK@?$AAs?$AAo?$AAu?$AAt?$AAh?$AA?9?$AAk?$AAo?$AAr?$AAe?$AAa?$AA?$AA@ 10111954     LIBCMT:getqloc.obj
 0002:0000e96c       ??_C@_1CE@PLHLOMJF@?$AAt?$AAr?$AAi?$AAn?$AAi?$AAd?$AAa?$AAd?$AA?5?$AA?$CG?$AA?5?$AAt?$AAo?$AAb?$AAa?$AAg?$AAo?$AA?$AA@ 1011196c     LIBCMT:getqloc.obj
 0002:0000e990       ??_C@_1BO@MODIMHHI@?$AAu?$AAn?$AAi?$AAt?$AAe?$AAd?$AA?9?$AAk?$AAi?$AAn?$AAg?$AAd?$AAo?$AAm?$AA?$AA@ 10111990     LIBCMT:getqloc.obj
 0002:0000e9b0       ??_C@_1BM@FFHJONBJ@?$AAu?$AAn?$AAi?$AAt?$AAe?$AAd?$AA?9?$AAs?$AAt?$AAa?$AAt?$AAe?$AAs?$AA?$AA@ 101119b0     LIBCMT:getqloc.obj
 0002:0000e9cc       ___rg_language_count       101119cc     LIBCMT:getqloc.obj
 0002:0000e9d0       ___rg_country_count        101119d0     LIBCMT:getqloc.obj
 0002:0000e9d4       ??_C@_17DNCLJFIF@?$AAA?$AAC?$AAP?$AA?$AA@ 101119d4     LIBCMT:getqloc.obj
 0002:0000e9dc       ??_C@_17CIKBIHLH@?$AAO?$AAC?$AAP?$AA?$AA@ 101119dc     LIBCMT:getqloc.obj
 0002:0000e9e4       ___rglangidNotDefault      101119e4     LIBCMT:getqloc_downlevel.obj
 0002:0000e9f8       __real@00000000            101119f8     LIBCMT:wcstoq.obj
 0002:0000e9fc       ?has_quiet_NaN@_Num_float_base@std@@2_NB 101119fc     libcpmt:xthrow.obj
 0002:0000e9fd       ?has_signaling_NaN@_Num_float_base@std@@2_NB 101119fd     libcpmt:xthrow.obj
 0002:0000e9fe       ?is_bounded@_Num_float_base@std@@2_NB 101119fe     libcpmt:xthrow.obj
 0002:0000ea00       ??_C@_1M@KLMEPMCM@?$AAa?$AAl?$AAn?$AAu?$AAm?$AA?$AA@ 10111a00     libcpmt:xthrow.obj
 0002:0000ea0c       ??_C@_1M@DHGLHBMI@?$AAa?$AAl?$AAp?$AAh?$AAa?$AA?$AA@ 10111a0c     libcpmt:xthrow.obj
 0002:0000ea18       ?is_exact@_Num_float_base@std@@2_NB 10111a18     libcpmt:xthrow.obj
 0002:0000ea1c       ??_C@_1M@EJAAJBPE@?$AAb?$AAl?$AAa?$AAn?$AAk?$AA?$AA@ 10111a1c     libcpmt:xthrow.obj
 0002:0000ea28       ??_C@_1M@LMIMILA@?$AAc?$AAn?$AAt?$AAr?$AAl?$AA?$AA@ 10111a28     libcpmt:xthrow.obj
 0002:0000ea34       ??_C@_13GKPPEALH@?$AAd?$AA?$AA@ 10111a34     libcpmt:xthrow.obj
 0002:0000ea38       ?is_iec559@_Num_float_base@std@@2_NB 10111a38     libcpmt:xthrow.obj
 0002:0000ea3c       ??_C@_1M@JDAEIBKG@?$AAd?$AAi?$AAg?$AAi?$AAt?$AA?$AA@ 10111a3c     libcpmt:xthrow.obj
 0002:0000ea48       ??_C@_1M@MDKNJLLK@?$AAg?$AAr?$AAa?$AAp?$AAh?$AA?$AA@ 10111a48     libcpmt:xthrow.obj
 0002:0000ea54       ??_C@_1M@LGAECJJD@?$AAl?$AAo?$AAw?$AAe?$AAr?$AA?$AA@ 10111a54     libcpmt:xthrow.obj
 0002:0000ea60       ?is_integer@_Num_float_base@std@@2_NB 10111a60     libcpmt:xthrow.obj
 0002:0000ea64       ??_C@_1M@ELNLAPLA@?$AAp?$AAr?$AAi?$AAn?$AAt?$AA?$AA@ 10111a64     libcpmt:xthrow.obj
 0002:0000ea70       ??_C@_1M@BPFMAOAO@?$AAp?$AAu?$AAn?$AAc?$AAt?$AA?$AA@ 10111a70     libcpmt:xthrow.obj
 0002:0000ea7c       ??_C@_1M@LPGODFOM@?$AAs?$AAp?$AAa?$AAc?$AAe?$AA?$AA@ 10111a7c     libcpmt:xthrow.obj
 0002:0000ea88       ?is_modulo@_Num_float_base@std@@2_NB 10111a88     libcpmt:xthrow.obj
 0002:0000ea8c       ??_C@_13KHDBCPJB@?$AAs?$AA?$AA@ 10111a8c     libcpmt:xthrow.obj
 0002:0000ea90       ??_C@_1M@PLNFCNIC@?$AAu?$AAp?$AAp?$AAe?$AAr?$AA?$AA@ 10111a90     libcpmt:xthrow.obj
 0002:0000ea9c       ??_C@_13CIFDLIMG@?$AAw?$AA?$AA@ 10111a9c     libcpmt:xthrow.obj
 0002:0000eaa0       ?is_signed@_Num_float_base@std@@2_NB 10111aa0     libcpmt:xthrow.obj
 0002:0000eaa4       ??_C@_1O@OAFMJDHN@?$AAx?$AAd?$AAi?$AAg?$AAi?$AAt?$AA?$AA@ 10111aa4     libcpmt:xthrow.obj
 0002:0000eab2       ?is_specialized@_Num_float_base@std@@2_NB 10111ab2     libcpmt:xthrow.obj
 0002:0000eab3       ?tinyness_before@_Num_float_base@std@@2_NB 10111ab3     libcpmt:xthrow.obj
 0002:0000eab4       ?traps@_Num_float_base@std@@2_NB 10111ab4     libcpmt:xthrow.obj
 0002:0000eab8       ?round_style@_Num_float_base@std@@2W4float_round_style@2@B 10111ab8     libcpmt:xthrow.obj
 0002:0000eabc       ?radix@_Num_float_base@std@@2HB 10111abc     libcpmt:xthrow.obj
 0002:0000eac0       ?is_signed@?$numeric_limits@D@std@@2_NB 10111ac0     libcpmt:xthrow.obj
 0002:0000eac4       ?digits@?$numeric_limits@D@std@@2HB 10111ac4     libcpmt:xthrow.obj
 0002:0000eac8       ?digits10@?$numeric_limits@D@std@@2HB 10111ac8     libcpmt:xthrow.obj
 0002:0000eacc       ?is_signed@?$numeric_limits@_W@std@@2_NB 10111acc     libcpmt:xthrow.obj
 0002:0000ead0       ?digits@?$numeric_limits@_W@std@@2HB 10111ad0     libcpmt:xthrow.obj
 0002:0000ead4       ?digits10@?$numeric_limits@_W@std@@2HB 10111ad4     libcpmt:xthrow.obj
 0002:0000ead8       ?is_modulo@?$numeric_limits@_N@std@@2_NB 10111ad8     libcpmt:xthrow.obj
 0002:0000ead9       ?is_signed@?$numeric_limits@_N@std@@2_NB 10111ad9     libcpmt:xthrow.obj
 0002:0000eadc       ?digits@?$numeric_limits@_N@std@@2HB 10111adc     libcpmt:xthrow.obj
 0002:0000eae0       ?digits10@?$numeric_limits@_N@std@@2HB 10111ae0     libcpmt:xthrow.obj
 0002:0000eae4       ?_VBITS@?$vector@_NV?$allocator@_N@std@@@std@@2HB 10111ae4     libcpmt:xthrow.obj
 0002:0000eae8       ?is_signed@?$numeric_limits@C@std@@2_NB 10111ae8     libcpmt:xthrow.obj
 0002:0000eaec       ?digits@?$numeric_limits@C@std@@2HB 10111aec     libcpmt:xthrow.obj
 0002:0000eaf0       ?digits10@?$numeric_limits@C@std@@2HB 10111af0     libcpmt:xthrow.obj
 0002:0000eaf4       ?is_signed@?$numeric_limits@E@std@@2_NB 10111af4     libcpmt:xthrow.obj
 0002:0000eaf8       ?digits@?$numeric_limits@E@std@@2HB 10111af8     libcpmt:xthrow.obj
 0002:0000eafc       ?digits10@?$numeric_limits@E@std@@2HB 10111afc     libcpmt:xthrow.obj
 0002:0000eb00       ?skipws@?$_Iosb@H@std@@2W4_Fmtflags@12@B 10111b00     libcpmt:xthrow.obj
 0002:0000eb04       ?unitbuf@?$_Iosb@H@std@@2W4_Fmtflags@12@B 10111b04     libcpmt:xthrow.obj
 0002:0000eb08       ?uppercase@?$_Iosb@H@std@@2W4_Fmtflags@12@B 10111b08     libcpmt:xthrow.obj
 0002:0000eb0c       ?showbase@?$_Iosb@H@std@@2W4_Fmtflags@12@B 10111b0c     libcpmt:xthrow.obj
 0002:0000eb10       ?showpoint@?$_Iosb@H@std@@2W4_Fmtflags@12@B 10111b10     libcpmt:xthrow.obj
 0002:0000eb14       ?showpos@?$_Iosb@H@std@@2W4_Fmtflags@12@B 10111b14     libcpmt:xthrow.obj
 0002:0000eb18       ?left@?$_Iosb@H@std@@2W4_Fmtflags@12@B 10111b18     libcpmt:xthrow.obj
 0002:0000eb1c       ?right@?$_Iosb@H@std@@2W4_Fmtflags@12@B 10111b1c     libcpmt:xthrow.obj
 0002:0000eb20       ?internal@?$_Iosb@H@std@@2W4_Fmtflags@12@B 10111b20     libcpmt:xthrow.obj
 0002:0000eb24       ?is_signed@?$numeric_limits@F@std@@2_NB 10111b24     libcpmt:xthrow.obj
 0002:0000eb28       ?dec@?$_Iosb@H@std@@2W4_Fmtflags@12@B 10111b28     libcpmt:xthrow.obj
 0002:0000eb2c       ?digits@?$numeric_limits@F@std@@2HB 10111b2c     libcpmt:xthrow.obj
 0002:0000eb30       ?oct@?$_Iosb@H@std@@2W4_Fmtflags@12@B 10111b30     libcpmt:xthrow.obj
 0002:0000eb34       ?digits10@?$numeric_limits@F@std@@2HB 10111b34     libcpmt:xthrow.obj
 0002:0000eb38       ?hex@?$_Iosb@H@std@@2W4_Fmtflags@12@B 10111b38     libcpmt:xthrow.obj
 0002:0000eb3c       ?scientific@?$_Iosb@H@std@@2W4_Fmtflags@12@B 10111b3c     libcpmt:xthrow.obj
 0002:0000eb40       ?fixed@?$_Iosb@H@std@@2W4_Fmtflags@12@B 10111b40     libcpmt:xthrow.obj
 0002:0000eb44       ?hexfloat@?$_Iosb@H@std@@2W4_Fmtflags@12@B 10111b44     libcpmt:xthrow.obj
 0002:0000eb48       ?boolalpha@?$_Iosb@H@std@@2W4_Fmtflags@12@B 10111b48     libcpmt:xthrow.obj
 0002:0000eb4c       ?_Stdio@?$_Iosb@H@std@@2W4_Fmtflags@12@B 10111b4c     libcpmt:xthrow.obj
 0002:0000eb50       ?adjustfield@?$_Iosb@H@std@@2W4_Fmtflags@12@B 10111b50     libcpmt:xthrow.obj
 0002:0000eb54       ?basefield@?$_Iosb@H@std@@2W4_Fmtflags@12@B 10111b54     libcpmt:xthrow.obj
 0002:0000eb58       ?floatfield@?$_Iosb@H@std@@2W4_Fmtflags@12@B 10111b58     libcpmt:xthrow.obj
 0002:0000eb5c       ?goodbit@?$_Iosb@H@std@@2W4_Iostate@12@B 10111b5c     libcpmt:xthrow.obj
 0002:0000eb60       ?is_signed@?$numeric_limits@G@std@@2_NB 10111b60     libcpmt:xthrow.obj
 0002:0000eb64       ?eofbit@?$_Iosb@H@std@@2W4_Iostate@12@B 10111b64     libcpmt:xthrow.obj
 0002:0000eb68       ?digits@?$numeric_limits@G@std@@2HB 10111b68     libcpmt:xthrow.obj
 0002:0000eb6c       ?failbit@?$_Iosb@H@std@@2W4_Iostate@12@B 10111b6c     libcpmt:xthrow.obj
 0002:0000eb70       ?digits10@?$numeric_limits@G@std@@2HB 10111b70     libcpmt:xthrow.obj
 0002:0000eb74       ?badbit@?$_Iosb@H@std@@2W4_Iostate@12@B 10111b74     libcpmt:xthrow.obj
 0002:0000eb78       ?_Hardfail@?$_Iosb@H@std@@2W4_Iostate@12@B 10111b78     libcpmt:xthrow.obj
 0002:0000eb7c       ?in@?$_Iosb@H@std@@2W4_Openmode@12@B 10111b7c     libcpmt:xthrow.obj
 0002:0000eb80       ?out@?$_Iosb@H@std@@2W4_Openmode@12@B 10111b80     libcpmt:xthrow.obj
 0002:0000eb84       ?ate@?$_Iosb@H@std@@2W4_Openmode@12@B 10111b84     libcpmt:xthrow.obj
 0002:0000eb88       ?app@?$_Iosb@H@std@@2W4_Openmode@12@B 10111b88     libcpmt:xthrow.obj
 0002:0000eb8c       ?trunc@?$_Iosb@H@std@@2W4_Openmode@12@B 10111b8c     libcpmt:xthrow.obj
 0002:0000eb90       ?_Nocreate@?$_Iosb@H@std@@2W4_Openmode@12@B 10111b90     libcpmt:xthrow.obj
 0002:0000eb94       ?_Noreplace@?$_Iosb@H@std@@2W4_Openmode@12@B 10111b94     libcpmt:xthrow.obj
 0002:0000eb98       ?binary@?$_Iosb@H@std@@2W4_Openmode@12@B 10111b98     libcpmt:xthrow.obj
 0002:0000eb9c       ?is_signed@?$numeric_limits@H@std@@2_NB 10111b9c     libcpmt:xthrow.obj
 0002:0000eba0       ?beg@?$_Iosb@H@std@@2W4_Seekdir@12@B 10111ba0     libcpmt:xthrow.obj
 0002:0000eba4       ?digits@?$numeric_limits@H@std@@2HB 10111ba4     libcpmt:xthrow.obj
 0002:0000eba8       ?cur@?$_Iosb@H@std@@2W4_Seekdir@12@B 10111ba8     libcpmt:xthrow.obj
 0002:0000ebac       ?digits10@?$numeric_limits@H@std@@2HB 10111bac     libcpmt:xthrow.obj
 0002:0000ebb0       ?end@?$_Iosb@H@std@@2W4_Seekdir@12@B 10111bb0     libcpmt:xthrow.obj
 0002:0000ebb4       ?is_signed@?$numeric_limits@I@std@@2_NB 10111bb4     libcpmt:xthrow.obj
 0002:0000ebb8       ?digits@?$numeric_limits@I@std@@2HB 10111bb8     libcpmt:xthrow.obj
 0002:0000ebbc       ?digits10@?$numeric_limits@I@std@@2HB 10111bbc     libcpmt:xthrow.obj
 0002:0000ebc0       ?value@?$integral_constant@H$0A@@std@@2HB 10111bc0     libcpmt:xthrow.obj
 0002:0000ebc4       ?is_signed@?$numeric_limits@J@std@@2_NB 10111bc4     libcpmt:xthrow.obj
 0002:0000ebc8       ?digits@?$numeric_limits@J@std@@2HB 10111bc8     libcpmt:xthrow.obj
 0002:0000ebcc       ?digits10@?$numeric_limits@J@std@@2HB 10111bcc     libcpmt:xthrow.obj
 0002:0000ebd0       ?is_signed@?$numeric_limits@K@std@@2_NB 10111bd0     libcpmt:xthrow.obj
 0002:0000ebd4       ?digits@?$numeric_limits@K@std@@2HB 10111bd4     libcpmt:xthrow.obj
 0002:0000ebd8       ?digits10@?$numeric_limits@K@std@@2HB 10111bd8     libcpmt:xthrow.obj
 0002:0000ebdc       ?is_signed@?$numeric_limits@_J@std@@2_NB 10111bdc     libcpmt:xthrow.obj
 0002:0000ebe0       ?digits@?$numeric_limits@_J@std@@2HB 10111be0     libcpmt:xthrow.obj
 0002:0000ebe4       ?digits10@?$numeric_limits@_J@std@@2HB 10111be4     libcpmt:xthrow.obj
 0002:0000ebe8       ?is_signed@?$numeric_limits@_K@std@@2_NB 10111be8     libcpmt:xthrow.obj
 0002:0000ebec       ?digits@?$numeric_limits@_K@std@@2HB 10111bec     libcpmt:xthrow.obj
 0002:0000ebf0       ?digits10@?$numeric_limits@_K@std@@2HB 10111bf0     libcpmt:xthrow.obj
 0002:0000ebf4       ?collate@?$_Locbase@H@std@@2HB 10111bf4     libcpmt:xthrow.obj
 0002:0000ebf8       ?ctype@?$_Locbase@H@std@@2HB 10111bf8     libcpmt:xthrow.obj
 0002:0000ebfc       ?monetary@?$_Locbase@H@std@@2HB 10111bfc     libcpmt:xthrow.obj
 0002:0000ec00       ?numeric@?$_Locbase@H@std@@2HB 10111c00     libcpmt:xthrow.obj
 0002:0000ec04       ?time@?$_Locbase@H@std@@2HB 10111c04     libcpmt:xthrow.obj
 0002:0000ec08       ?messages@?$_Locbase@H@std@@2HB 10111c08     libcpmt:xthrow.obj
 0002:0000ec0c       ?all@?$_Locbase@H@std@@2HB 10111c0c     libcpmt:xthrow.obj
 0002:0000ec10       ?none@?$_Locbase@H@std@@2HB 10111c10     libcpmt:xthrow.obj
 0002:0000ec14       ?digits@?$numeric_limits@M@std@@2HB 10111c14     libcpmt:xthrow.obj
 0002:0000ec18       ?digits10@?$numeric_limits@M@std@@2HB 10111c18     libcpmt:xthrow.obj
 0002:0000ec1c       ?max_digits10@?$numeric_limits@M@std@@2HB 10111c1c     libcpmt:xthrow.obj
 0002:0000ec20       ?max_exponent@?$numeric_limits@M@std@@2HB 10111c20     libcpmt:xthrow.obj
 0002:0000ec24       ?max_exponent10@?$numeric_limits@M@std@@2HB 10111c24     libcpmt:xthrow.obj
 0002:0000ec28       ?min_exponent@?$numeric_limits@M@std@@2HB 10111c28     libcpmt:xthrow.obj
 0002:0000ec2c       ?min_exponent10@?$numeric_limits@M@std@@2HB 10111c2c     libcpmt:xthrow.obj
 0002:0000ec30       ?digits@?$numeric_limits@N@std@@2HB 10111c30     libcpmt:xthrow.obj
 0002:0000ec34       ?digits10@?$numeric_limits@N@std@@2HB 10111c34     libcpmt:xthrow.obj
 0002:0000ec38       ?max_digits10@?$numeric_limits@N@std@@2HB 10111c38     libcpmt:xthrow.obj
 0002:0000ec3c       ?max_exponent@?$numeric_limits@N@std@@2HB 10111c3c     libcpmt:xthrow.obj
 0002:0000ec40       ?max_exponent10@?$numeric_limits@N@std@@2HB 10111c40     libcpmt:xthrow.obj
 0002:0000ec44       ?min_exponent@?$numeric_limits@N@std@@2HB 10111c44     libcpmt:xthrow.obj
 0002:0000ec48       ?min_exponent10@?$numeric_limits@N@std@@2HB 10111c48     libcpmt:xthrow.obj
 0002:0000ec4c       ?digits@?$numeric_limits@O@std@@2HB 10111c4c     libcpmt:xthrow.obj
 0002:0000ec50       ?digits10@?$numeric_limits@O@std@@2HB 10111c50     libcpmt:xthrow.obj
 0002:0000ec54       ?max_digits10@?$numeric_limits@O@std@@2HB 10111c54     libcpmt:xthrow.obj
 0002:0000ec58       ?max_exponent@?$numeric_limits@O@std@@2HB 10111c58     libcpmt:xthrow.obj
 0002:0000ec5c       ?max_exponent10@?$numeric_limits@O@std@@2HB 10111c5c     libcpmt:xthrow.obj
 0002:0000ec60       ?min_exponent@?$numeric_limits@O@std@@2HB 10111c60     libcpmt:xthrow.obj
 0002:0000ec64       ?min_exponent10@?$numeric_limits@O@std@@2HB 10111c64     libcpmt:xthrow.obj
 0002:0000ec68       ?table_size@?$ctype@D@std@@2IB 10111c68     libcpmt:xthrow.obj
 0002:0000ec6c       ?value@?$integral_constant@I$07@std@@2IB 10111c6c     libcpmt:xthrow.obj
 0002:0000ec70       ?value@?$integral_constant@I$03@std@@2IB 10111c70     libcpmt:xthrow.obj
 0002:0000ec74       ?value@?$integral_constant@I$01@std@@2IB 10111c74     libcpmt:xthrow.obj
 0002:0000ec78       ?value@?$integral_constant@I$00@std@@2IB 10111c78     libcpmt:xthrow.obj
 0002:0000ec7c       ?value@?$_Maximum@$S@std@@2IB 10111c7c     libcpmt:xthrow.obj
 0002:0000ec80       ?_Names@?$_Regex_traits@D@std@@0QBU?$_Cl_names@D@2@B 10111c80     libcpmt:xthrow.obj
 0002:0000ed40       ?has_denorm@_Num_base@std@@2W4float_denorm_style@2@B 10111d40     libcpmt:xthrow.obj
 0002:0000ed44       ?has_denorm_loss@_Num_base@std@@2_NB 10111d44     libcpmt:xthrow.obj
 0002:0000ed45       ?has_infinity@_Num_base@std@@2_NB 10111d45     libcpmt:xthrow.obj
 0002:0000ed46       ?has_quiet_NaN@_Num_base@std@@2_NB 10111d46     libcpmt:xthrow.obj
 0002:0000ed47       ?has_signaling_NaN@_Num_base@std@@2_NB 10111d47     libcpmt:xthrow.obj
 0002:0000ed48       ?is_bounded@_Num_base@std@@2_NB 10111d48     libcpmt:xthrow.obj
 0002:0000ed49       ?is_exact@_Num_base@std@@2_NB 10111d49     libcpmt:xthrow.obj
 0002:0000ed4a       ?is_iec559@_Num_base@std@@2_NB 10111d4a     libcpmt:xthrow.obj
 0002:0000ed4b       ?is_integer@_Num_base@std@@2_NB 10111d4b     libcpmt:xthrow.obj
 0002:0000ed4c       ?is_modulo@_Num_base@std@@2_NB 10111d4c     libcpmt:xthrow.obj
 0002:0000ed4d       ?is_signed@_Num_base@std@@2_NB 10111d4d     libcpmt:xthrow.obj
 0002:0000ed50       ??_C@_05IIMHCHIO@alnum?$AA@ 10111d50     libcpmt:xthrow.obj
 0002:0000ed58       ??_C@_05IAEKHIAN@alpha?$AA@ 10111d58     libcpmt:xthrow.obj
 0002:0000ed60       ??_C@_05BABJKOGB@blank?$AA@ 10111d60     libcpmt:xthrow.obj
 0002:0000ed68       ?value@?$integral_constant@I$0A@@std@@2IB 10111d68     libcpmt:xthrow.obj
 0002:0000ed6c       ?is_specialized@_Num_base@std@@2_NB 10111d6c     libcpmt:xthrow.obj
 0002:0000ed70       ??_C@_05JMDPEFNK@cntrl?$AA@ 10111d70     libcpmt:xthrow.obj
 0002:0000ed78       ??_C@_01LPLHEDKD@d?$AA@    10111d78     libcpmt:xthrow.obj
 0002:0000ed7c       ??_C@_05ODNOIFML@digit?$AA@ 10111d7c     libcpmt:xthrow.obj
 0002:0000ed82       ?tinyness_before@_Num_base@std@@2_NB 10111d82     libcpmt:xthrow.obj
 0002:0000ed84       ??_C@_05KCJBMLII@graph?$AA@ 10111d84     libcpmt:xthrow.obj
 0002:0000ed8c       ??_C@_05IPJEPLHL@lower?$AA@ 10111d8c     libcpmt:xthrow.obj
 0002:0000ed94       ??_C@_05IJDJACGD@print?$AA@ 10111d94     libcpmt:xthrow.obj
 0002:0000ed9a       ?traps@_Num_base@std@@2_NB 10111d9a     libcpmt:xthrow.obj
 0002:0000ed9c       ??_C@_05KOBGHFJJ@punct?$AA@ 10111d9c     libcpmt:xthrow.obj
 0002:0000eda4       ??_C@_05OLNILLAB@space?$AA@ 10111da4     libcpmt:xthrow.obj
 0002:0000edac       ??_C@_01LKDEMHDF@s?$AA@    10111dac     libcpmt:xthrow.obj
 0002:0000edb0       ?round_style@_Num_base@std@@2W4float_round_style@2@B 10111db0     libcpmt:xthrow.obj
 0002:0000edb4       ??_C@_05NECKJAMC@upper?$AA@ 10111db4     libcpmt:xthrow.obj
 0002:0000edbc       ??_C@_01NOFIACDB@w?$AA@    10111dbc     libcpmt:xthrow.obj
 0002:0000edc0       ??_C@_06BAPHGFFK@xdigit?$AA@ 10111dc0     libcpmt:xthrow.obj
 0002:0000edc8       ?digits@_Num_base@std@@2HB 10111dc8     libcpmt:xthrow.obj
 0002:0000edcc       ?digits10@_Num_base@std@@2HB 10111dcc     libcpmt:xthrow.obj
 0002:0000edd0       ?max_digits10@_Num_base@std@@2HB 10111dd0     libcpmt:xthrow.obj
 0002:0000edd4       ?max_exponent@_Num_base@std@@2HB 10111dd4     libcpmt:xthrow.obj
 0002:0000edd8       ?max_exponent10@_Num_base@std@@2HB 10111dd8     libcpmt:xthrow.obj
 0002:0000eddc       ?min_exponent@_Num_base@std@@2HB 10111ddc     libcpmt:xthrow.obj
 0002:0000ede0       ?min_exponent10@_Num_base@std@@2HB 10111de0     libcpmt:xthrow.obj
 0002:0000ede4       ?radix@_Num_base@std@@2HB  10111de4     libcpmt:xthrow.obj
 0002:0000ede8       ?is_bounded@_Num_int_base@std@@2_NB 10111de8     libcpmt:xthrow.obj
 0002:0000ede9       ?is_exact@_Num_int_base@std@@2_NB 10111de9     libcpmt:xthrow.obj
 0002:0000edea       ?is_integer@_Num_int_base@std@@2_NB 10111dea     libcpmt:xthrow.obj
 0002:0000edeb       ?is_modulo@_Num_int_base@std@@2_NB 10111deb     libcpmt:xthrow.obj
 0002:0000edf0       ?_Names@?$_Regex_traits@_W@std@@0QBU?$_Cl_names@_W@2@B 10111df0     libcpmt:xthrow.obj
 0002:0000eeb0       ?is_specialized@_Num_int_base@std@@2_NB 10111eb0     libcpmt:xthrow.obj
 0002:0000eeb4       ?radix@_Num_int_base@std@@2HB 10111eb4     libcpmt:xthrow.obj
 0002:0000eeb8       ?has_denorm@_Num_float_base@std@@2W4float_denorm_style@2@B 10111eb8     libcpmt:xthrow.obj
 0002:0000eebc       ?has_denorm_loss@_Num_float_base@std@@2_NB 10111ebc     libcpmt:xthrow.obj
 0002:0000eebd       ?has_infinity@_Num_float_base@std@@2_NB 10111ebd     libcpmt:xthrow.obj
 0002:0000eec4       ??_7length_error@std@@6B@  10111ec4     libcpmt:xthrow.obj
 0002:0000eed0       ??_7out_of_range@std@@6B@  10111ed0     libcpmt:xthrow.obj
 0002:0000eedc       ??_7overflow_error@std@@6B@ 10111edc     libcpmt:xthrow.obj
 0002:0000eee8       ??_7bad_function_call@std@@6B@ 10111ee8     libcpmt:xthrow.obj
 0002:0000eef0       ??_C@_0BC@DPJNKNAF@bad?5function?5call?$AA@ 10111ef0     libcpmt:xthrow.obj
 0002:0000ef08       ??_7regex_error@std@@6B@   10111f08     libcpmt:xthrow.obj
 0002:0000ef10       ??_C@_0FI@CMNGHIFF@regex_error?$CIerror_collate?$CJ?3?5The?5@ 10111f10     libcpmt:xthrow.obj
 0002:0000ef68       ??_C@_0FE@LJMHKIOC@regex_error?$CIerror_ctype?$CJ?3?5The?5ex@ 10111f68     libcpmt:xthrow.obj
 0002:0000efc0       ??_C@_0GI@HEGGMMDL@regex_error?$CIerror_escape?$CJ?3?5The?5e@ 10111fc0     libcpmt:xthrow.obj
 0002:0000f028       ??_C@_0FA@HFMLPGNN@regex_error?$CIerror_backref?$CJ?3?5The?5@ 10112028     libcpmt:xthrow.obj
 0002:0000f078       ??_C@_0EH@LGEANNAL@regex_error?$CIerror_brack?$CJ?3?5The?5ex@ 10112078     libcpmt:xthrow.obj
 0002:0000f0c0       ??_C@_0EH@CAGOJGLE@regex_error?$CIerror_paren?$CJ?3?5The?5ex@ 101120c0     libcpmt:xthrow.obj
 0002:0000f108       ??_C@_0EH@DICJJKLO@regex_error?$CIerror_brace?$CJ?3?5The?5ex@ 10112108     libcpmt:xthrow.obj
 0002:0000f150       ??_C@_0FM@BLDIHIBB@regex_error?$CIerror_badbrace?$CJ?3?5The@ 10112150     libcpmt:xthrow.obj
 0002:0000f1b0       ??_C@_0HA@ICNJLCMC@regex_error?$CIerror_range?$CJ?3?5The?5ex@ 101121b0     libcpmt:xthrow.obj
 0002:0000f220       ??_C@_0GP@PICOBCHA@regex_error?$CIerror_space?$CJ?3?5There?5@ 10112220     libcpmt:xthrow.obj
 0002:0000f290       ??_C@_0FK@LCHHHEOA@regex_error?$CIerror_badrepeat?$CJ?3?5On@ 10112290     libcpmt:xthrow.obj
 0002:0000f2f0       ??_C@_0HL@NEKOFBJA@regex_error?$CIerror_complexity?$CJ?3?5T@ 101122f0     libcpmt:xthrow.obj
 0002:0000f370       ??_C@_0JC@HCDLJLGO@regex_error?$CIerror_stack?$CJ?3?5There?5@ 10112370     libcpmt:xthrow.obj
 0002:0000f404       ??_C@_0BJ@CHBLKGNM@regex_error?$CIerror_parse?$CJ?$AA@ 10112404     libcpmt:xthrow.obj
 0002:0000f420       ??_C@_0BK@DFJCACNI@regex_error?$CIerror_syntax?$CJ?$AA@ 10112420     libcpmt:xthrow.obj
 0002:0000f43c       ??_C@_0M@KGKAAGCA@regex_error?$AA@ 1011243c     libcpmt:xthrow.obj
 0002:0000f448       ??_C@_0BG@DHPCNBJB@address?5not?5available?$AA@ 10112448     libcpmt:syserror.obj
 0002:0000f460       ??_C@_0BC@DFIBIBIL@already?5connected?$AA@ 10112460     libcpmt:syserror.obj
 0002:0000f474       ??_C@_0BH@CAKOHOMI@argument?5list?5too?5long?$AA@ 10112474     libcpmt:syserror.obj
 0002:0000f48c       ??_C@_0BH@CGIMPKIM@argument?5out?5of?5domain?$AA@ 1011248c     libcpmt:syserror.obj
 0002:0000f4a4       ??_C@_0M@KGHGGJGL@bad?5address?$AA@ 101124a4     libcpmt:syserror.obj
 0002:0000f4b0       ??_C@_0BE@MPJPGCEO@bad?5file?5descriptor?$AA@ 101124b0     libcpmt:syserror.obj
 0002:0000f4c4       ??_C@_0M@PMMIEFCP@bad?5message?$AA@ 101124c4     libcpmt:syserror.obj
 0002:0000f4d0       ??_C@_0M@KPHOFDBE@broken?5pipe?$AA@ 101124d0     libcpmt:syserror.obj
 0002:0000f4dc       ??_C@_0BD@MGNDDEGM@connection?5aborted?$AA@ 101124dc     libcpmt:syserror.obj
 0002:0000f4f0       ??_C@_0BP@KAIHPOGN@connection?5already?5in?5progress?$AA@ 101124f0     libcpmt:syserror.obj
 0002:0000f510       ??_C@_0BD@PJLIIJEL@connection?5refused?$AA@ 10112510     libcpmt:syserror.obj
 0002:0000f524       ??_C@_0BB@IECNJNOI@connection?5reset?$AA@ 10112524     libcpmt:syserror.obj
 0002:0000f538       ??_C@_0BN@KDMIFEIP@destination?5address?5required?$AA@ 10112538     libcpmt:syserror.obj
 0002:0000f558       ??_C@_0BI@BNCLIGPB@executable?5format?5error?$AA@ 10112558     libcpmt:syserror.obj
 0002:0000f570       ??_C@_0P@DNAJLBJK@file?5too?5large?$AA@ 10112570     libcpmt:syserror.obj
 0002:0000f580       ??_C@_0BB@DHFDFGDM@host?5unreachable?$AA@ 10112580     libcpmt:syserror.obj
 0002:0000f594       ??_C@_0BD@JPHBMONG@identifier?5removed?$AA@ 10112594     libcpmt:syserror.obj
 0002:0000f5a8       ??_C@_0BG@CDNPAGJK@illegal?5byte?5sequence?$AA@ 101125a8     libcpmt:syserror.obj
 0002:0000f5c0       ??_C@_0CD@BNPLBMNA@inappropriate?5io?5control?5operati@ 101125c0     libcpmt:syserror.obj
 0002:0000f5e4       ??_C@_0N@OHAFKDEK@invalid?5seek?$AA@ 101125e4     libcpmt:syserror.obj
 0002:0000f5f4       ??_C@_0P@FLLDBIDK@is?5a?5directory?$AA@ 101125f4     libcpmt:syserror.obj
 0002:0000f604       ??_C@_0N@IFLPBIOP@message?5size?$AA@ 10112604     libcpmt:syserror.obj
 0002:0000f614       ??_C@_0N@KIIEAAIO@network?5down?$AA@ 10112614     libcpmt:syserror.obj
 0002:0000f624       ??_C@_0O@FNPDBHEE@network?5reset?$AA@ 10112624     libcpmt:syserror.obj
 0002:0000f634       ??_C@_0BE@IFNCKGE@network?5unreachable?$AA@ 10112634     libcpmt:syserror.obj
 0002:0000f648       ??_C@_0BA@PFFCAOFK@no?5buffer?5space?$AA@ 10112648     libcpmt:syserror.obj
 0002:0000f658       ??_C@_0BB@IEPBLJHK@no?5child?5process?$AA@ 10112658     libcpmt:syserror.obj
 0002:0000f66c       ??_C@_07PLECNNKG@no?5link?$AA@ 1011266c     libcpmt:syserror.obj
 0002:0000f674       ??_C@_0BF@PBGGPKKE@no?5message?5available?$AA@ 10112674     libcpmt:syserror.obj
 0002:0000f68c       ??_C@_0L@EDOLMPAK@no?5message?$AA@ 1011268c     libcpmt:syserror.obj
 0002:0000f698       ??_C@_0BD@EAMBFIDF@no?5protocol?5option?$AA@ 10112698     libcpmt:syserror.obj
 0002:0000f6ac       ??_C@_0BE@MKFDAFMP@no?5stream?5resources?$AA@ 101126ac     libcpmt:syserror.obj
 0002:0000f6c0       ??_C@_0BK@IMCPHCBI@no?5such?5device?5or?5address?$AA@ 101126c0     libcpmt:syserror.obj
 0002:0000f6dc       ??_C@_0BA@ENLPPKBN@no?5such?5process?$AA@ 101126dc     libcpmt:syserror.obj
 0002:0000f6ec       ??_C@_0BA@DOCPFFJG@not?5a?5directory?$AA@ 101126ec     libcpmt:syserror.obj
 0002:0000f6fc       ??_C@_0N@POEIPGGF@not?5a?5socket?$AA@ 101126fc     libcpmt:syserror.obj
 0002:0000f70c       ??_C@_0N@LGAPMMPI@not?5a?5stream?$AA@ 1011270c     libcpmt:syserror.obj
 0002:0000f71c       ??_C@_0O@GLMIBBEG@not?5connected?$AA@ 1011271c     libcpmt:syserror.obj
 0002:0000f72c       ??_C@_0O@NHEDABJP@not?5supported?$AA@ 1011272c     libcpmt:syserror.obj
 0002:0000f73c       ??_C@_0BG@KDKHOPCO@operation?5in?5progress?$AA@ 1011273c     libcpmt:syserror.obj
 0002:0000f754       ??_C@_0BI@OHIEJAAB@operation?5not?5permitted?$AA@ 10112754     libcpmt:syserror.obj
 0002:0000f76c       ??_C@_0BI@LNEGIFLN@operation?5not?5supported?$AA@ 1011276c     libcpmt:syserror.obj
 0002:0000f784       ??_C@_0BG@OEMDKMEE@operation?5would?5block?$AA@ 10112784     libcpmt:syserror.obj
 0002:0000f79c       ??_C@_0L@BLPOFLNJ@owner?5dead?$AA@ 1011279c     libcpmt:syserror.obj
 0002:0000f7a8       ??_C@_0P@FNPOCJBE@protocol?5error?$AA@ 101127a8     libcpmt:syserror.obj
 0002:0000f7b8       ??_C@_0BH@JPPPLHJB@protocol?5not?5supported?$AA@ 101127b8     libcpmt:syserror.obj
 0002:0000f7d0       ??_C@_0BG@EICBIHDP@read?5only?5file?5system?$AA@ 101127d0     libcpmt:syserror.obj
 0002:0000f7e8       ??_C@_0BO@BJBOMOEJ@resource?5deadlock?5would?5occur?$AA@ 101127e8     libcpmt:syserror.obj
 0002:0000f808       ??_C@_0BE@GOIPJJHG@result?5out?5of?5range?$AA@ 10112808     libcpmt:syserror.obj
 0002:0000f81c       ??_C@_0BG@MPLKFPAE@state?5not?5recoverable?$AA@ 1011281c     libcpmt:syserror.obj
 0002:0000f834       ??_C@_0P@DIIFGFCG@stream?5timeout?$AA@ 10112834     libcpmt:syserror.obj
 0002:0000f844       ??_C@_0P@IPFDMIFL@text?5file?5busy?$AA@ 10112844     libcpmt:syserror.obj
 0002:0000f854       ??_C@_09KJPPMAOI@timed?5out?$AA@ 10112854     libcpmt:syserror.obj
 0002:0000f860       ??_C@_0BO@HACHBEKI@too?5many?5files?5open?5in?5system?$AA@ 10112860     libcpmt:syserror.obj
 0002:0000f880       ??_C@_0P@HCOMKFCC@too?5many?5links?$AA@ 10112880     libcpmt:syserror.obj
 0002:0000f890       ??_C@_0BO@EFGOJEF@too?5many?5symbolic?5link?5levels?$AA@ 10112890     libcpmt:syserror.obj
 0002:0000f8b0       ??_C@_0BA@KGKGOOJA@value?5too?5large?$AA@ 101128b0     libcpmt:syserror.obj
 0002:0000f8c0       ??_C@_0BE@MIEJDDNH@wrong?5protocol?5type?$AA@ 101128c0     libcpmt:syserror.obj
 0002:0000fda8       ??_C@_0BC@CIJDGCDI@permission?5denied?$AA@ 10112da8     libcpmt:syserror.obj
 0002:0000fdbc       ??_C@_0M@MIDIAGJP@file?5exists?$AA@ 10112dbc     libcpmt:syserror.obj
 0002:0000fdc8       ??_C@_0P@FDINDDOK@no?5such?5device?$AA@ 10112dc8     libcpmt:syserror.obj
 0002:0000fdd8       ??_C@_0BC@EJHOMAAK@filename?5too?5long?$AA@ 10112dd8     libcpmt:syserror.obj
 0002:0000fdec       ??_C@_0BI@NGCEHDD@device?5or?5resource?5busy?$AA@ 10112dec     libcpmt:syserror.obj
 0002:0000fe04       ??_C@_08GLNPIFBN@io?5error?$AA@ 10112e04     libcpmt:syserror.obj
 0002:0000fe10       ??_C@_0BE@JIDOCPHM@directory?5not?5empty?$AA@ 10112e10     libcpmt:syserror.obj
 0002:0000fe24       ??_C@_0BB@FCMFBGOM@invalid?5argument?$AA@ 10112e24     libcpmt:syserror.obj
 0002:0000fe38       ??_C@_0BD@IJDJKDEA@no?5space?5on?5device?$AA@ 10112e38     libcpmt:syserror.obj
 0002:0000fe4c       ??_C@_0BK@NDOCBPGE@no?5such?5file?5or?5directory?$AA@ 10112e4c     libcpmt:syserror.obj
 0002:0000fe68       ??_C@_0BH@KEFGLDAF@function?5not?5supported?$AA@ 10112e68     libcpmt:syserror.obj
 0002:0000fe80       ??_C@_0BC@NJECKMKE@no?5lock?5available?$AA@ 10112e80     libcpmt:syserror.obj
 0002:0000fe94       ??_C@_0BC@ENOOLCNF@not?5enough?5memory?$AA@ 10112e94     libcpmt:syserror.obj
 0002:0000fea8       ??_C@_0BP@LKNGHENJ@resource?5unavailable?5try?5again?$AA@ 10112ea8     libcpmt:syserror.obj
 0002:0000fec8       ??_C@_0BC@PPHBOELF@cross?5device?5link?$AA@ 10112ec8     libcpmt:syserror.obj
 0002:0000fedc       ??_C@_0BD@MOLBPMEA@operation?5canceled?$AA@ 10112edc     libcpmt:syserror.obj
 0002:0000fef0       ??_C@_0BE@GHAFMPAH@too?5many?5files?5open?$AA@ 10112ef0     libcpmt:syserror.obj
 0002:0000ff04       ??_C@_0BC@FNODOBAE@permission_denied?$AA@ 10112f04     libcpmt:syserror.obj
 0002:0000ff18       ??_C@_0P@LNDJPBFK@address_in_use?$AA@ 10112f18     libcpmt:syserror.obj
 0002:0000ff28       ??_C@_0BG@IPMGOJF@address_not_available?$AA@ 10112f28     libcpmt:syserror.obj
 0002:0000ff40       ??_C@_0BN@LCBDHODA@address_family_not_supported?$AA@ 10112f40     libcpmt:syserror.obj
 0002:0000ff60       ??_C@_0BP@FOJJHMCC@connection_already_in_progress?$AA@ 10112f60     libcpmt:syserror.obj
 0002:0000ff80       ??_C@_0BE@DLHHIBGN@bad_file_descriptor?$AA@ 10112f80     libcpmt:syserror.obj
 0002:0000ff94       ??_C@_0BD@OJMJDIGI@connection_aborted?$AA@ 10112f94     libcpmt:syserror.obj
 0002:0000ffa8       ??_C@_0BD@NGKCIFEP@connection_refused?$AA@ 10112fa8     libcpmt:syserror.obj
 0002:0000ffbc       ??_C@_0BB@JOANDNCK@connection_reset?$AA@ 10112fbc     libcpmt:syserror.obj
 0002:0000ffd0       ??_C@_0BN@JLJNLKLK@destination_address_required?$AA@ 10112fd0     libcpmt:syserror.obj
 0002:0000fff0       ??_C@_0M@IJGMGFGP@bad_address?$AA@ 10112ff0     libcpmt:syserror.obj
 0002:0000fffc       ??_C@_0BB@KKNHPPIN@host_unreachable?$AA@ 10112ffc     libcpmt:syserror.obj
 0002:00010010       ??_C@_0BG@DJGBJIIK@operation_in_progress?$AA@ 10113010     libcpmt:syserror.obj
 0002:00010028       ??_C@_0M@EGEKIIMP@interrupted?$AA@ 10113028     libcpmt:syserror.obj
 0002:00010034       ??_C@_0BB@FFIHMIPJ@invalid_argument?$AA@ 10113034     libcpmt:syserror.obj
 0002:00010048       ??_C@_0BC@FIFLCHLO@already_connected?$AA@ 10113048     libcpmt:syserror.obj
 0002:0001005c       ??_C@_0BE@GJJJJDDA@too_many_files_open?$AA@ 1011305c     libcpmt:syserror.obj
 0002:00010070       ??_C@_0N@HPMLKHPL@message_size?$AA@ 10113070     libcpmt:syserror.obj
 0002:00010080       ??_C@_0BC@LEEIKBAL@filename_too_long?$AA@ 10113080     libcpmt:syserror.obj
 0002:00010094       ??_C@_0N@FCPALPJK@network_down?$AA@ 10113094     libcpmt:syserror.obj
 0002:000100a4       ??_C@_0O@EHNDLHIG@network_reset?$AA@ 101130a4     libcpmt:syserror.obj
 0002:000100b4       ??_C@_0BE@JFNJIDNF@network_unreachable?$AA@ 101130b4     libcpmt:syserror.obj
 0002:000100c8       ??_C@_0BA@FDIJKJCL@no_buffer_space?$AA@ 101130c8     libcpmt:syserror.obj
 0002:000100d8       ??_C@_0BD@JHIHCGKP@no_protocol_option?$AA@ 101130d8     libcpmt:syserror.obj
 0002:000100ec       ??_C@_0O@GBCLHHD@not_connected?$AA@ 101130ec     libcpmt:syserror.obj
 0002:000100fc       ??_C@_0N@IMHKKLEM@not_a_socket?$AA@ 101130fc     libcpmt:syserror.obj
 0002:0001010c       ??_C@_0BI@ICEIDKLJ@operation_not_supported?$AA@ 1011310c     libcpmt:syserror.obj
 0002:00010124       ??_C@_0BH@KAPBAIJF@protocol_not_supported?$AA@ 10113124     libcpmt:syserror.obj
 0002:0001013c       ??_C@_0BE@GAOJJFPC@wrong_protocol_type?$AA@ 1011313c     libcpmt:syserror.obj
 0002:00010150       ??_C@_09NCHNLHPG@timed_out?$AA@ 10113150     libcpmt:syserror.obj
 0002:0001015c       ??_C@_0BG@GDGHKFDH@operation_would_block?$AA@ 1011315c     libcpmt:syserror.obj
 0002:00010174       ??_C@_0BN@LKKBCCDB@address?5family?5not?5supported?$AA@ 10113174     libcpmt:syserror.obj
 0002:00010194       ??_C@_0P@LDMLAFHI@address?5in?5use?$AA@ 10113194     libcpmt:syserror.obj
 0002:000101a8       ??_7_Locimp@locale@std@@6B@ 101131a8     libcpmt:locale0.obj
 0002:000101b4       ??_C@_01GFHCPBMG@C?$AA@    101131b4     libcpmt:locale0.obj
 0002:000101b8       ?_BADOFF@std@@3_JB         101131b8     libcpmt:ios.obj
 0002:000101fc       ??_C@_01MCMALHOG@a?$AA@    101131fc     libcpmt:fiopen.obj
 0002:00010200       ??_C@_02JDPG@rb?$AA@       10113200     libcpmt:fiopen.obj
 0002:00010204       ??_C@_02GMLFBBN@wb?$AA@    10113204     libcpmt:fiopen.obj
 0002:00010208       ??_C@_02BOGAIONP@ab?$AA@   10113208     libcpmt:fiopen.obj
 0002:0001020c       ??_C@_02CBLLGHLK@r?$CL?$AA@ 1011320c     libcpmt:fiopen.obj
 0002:00010210       ??_C@_02CHHAKFFB@w?$CL?$AA@ 10113210     libcpmt:fiopen.obj
 0002:00010214       ??_C@_02DPNLHKJD@a?$CL?$AA@ 10113214     libcpmt:fiopen.obj
 0002:00010218       ??_C@_03HMFOOINA@r?$CLb?$AA@ 10113218     libcpmt:fiopen.obj
 0002:0001021c       ??_C@_03DOPCBAKB@a?$CLb?$AA@ 1011321c     libcpmt:fiopen.obj
 0002:0001025c       ??_C@_13BPINEIPE@?$AAr?$AA?$AA@ 1011325c     libcpmt:fiopen.obj
 0002:00010260       ??_C@_13FNCBLAIF@?$AAa?$AA?$AA@ 10113260     libcpmt:fiopen.obj
 0002:00010264       ??_C@_15JJPIMNBO@?$AAr?$AAb?$AA?$AA@ 10113264     libcpmt:fiopen.obj
 0002:0001026c       ??_C@_15MJDFFMKN@?$AAw?$AAb?$AA?$AA@ 1011326c     libcpmt:fiopen.obj
 0002:00010274       ??_C@_15BMLKLNCL@?$AAa?$AAb?$AA?$AA@ 10113274     libcpmt:fiopen.obj
 0002:0001027c       ??_C@_15HPOENKKJ@?$AAr?$AA?$CL?$AA?$AA@ 1011327c     libcpmt:fiopen.obj
 0002:00010284       ??_C@_15CPCJELBK@?$AAw?$AA?$CL?$AA?$AA@ 10113284     libcpmt:fiopen.obj
 0002:0001028c       ??_C@_15PKKGKKJM@?$AAa?$AA?$CL?$AA?$AA@ 1011328c     libcpmt:fiopen.obj
 0002:00010294       ??_C@_17IIOMHMAG@?$AAr?$AA?$CL?$AAb?$AA?$AA@ 10113294     libcpmt:fiopen.obj
 0002:0001029c       ??_C@_17MAAMHCGC@?$AAw?$AA?$CL?$AAb?$AA?$AA@ 1011329c     libcpmt:fiopen.obj
 0002:000102a4       ??_C@_17HKNIEKMO@?$AAa?$AA?$CL?$AAb?$AA?$AA@ 101132a4     libcpmt:fiopen.obj
 0002:000102ac       ?valid@?1???$_Xfiopen@D@std@@YAPAU_iobuf@@PBDHH@Z@4QBHB 101132ac     libcpmt:fiopen.obj
 0002:000102e8       ?valid@?1???$_Xfiopen@_W@std@@YAPAU_iobuf@@PB_WHH@Z@4QBHB 101132e8     libcpmt:fiopen.obj
 0002:00010324       ??_C@_05LAPONLG@false?$AA@ 10113324     libcpmt:locale.obj
 0002:0001032c       ??_C@_04LOAJBDKD@true?$AA@ 1011332c     libcpmt:locale.obj
 0002:00010338       ??_7?$num_get@DV?$istreambuf_iterator@DU?$char_traits@D@std@@@std@@@std@@6B@ 10113338     libcpmt:locale.obj
 0002:00010374       ??_7?$num_put@DV?$ostreambuf_iterator@DU?$char_traits@D@std@@@std@@@std@@6B@ 10113374     libcpmt:locale.obj
 0002:000103a4       ??_7?$numpunct@D@std@@6B@  101133a4     libcpmt:locale.obj
 0002:000103c4       ??_C@_02EAOCLKAK@ld?$AA@   101133c4     libcpmt:locale.obj
 0002:000103c8       ??_C@_02BDDLJJBK@lu?$AA@   101133c8     libcpmt:locale.obj
 0002:000103cc       ??_C@_02HIKPPMOK@Ld?$AA@   101133cc     libcpmt:locale.obj
 0002:000103d0       ??_C@_02CLHGNPPK@Lu?$AA@   101133d0     libcpmt:locale.obj
 0002:000103d4       ??_C@_02BBAHNLBA@?$CFp?$AA@ 101133d4     libcpmt:locale.obj
 0002:000103d8       ?_Src@?1??_Getifld@?$num_get@DV?$istreambuf_iterator@DU?$char_traits@D@std@@@std@@@std@@ABAHPADAAV?$istreambuf_iterator@DU?$char_traits@D@std@@@3@1HABVlocale@3@@Z@4QBDB 101133d8     libcpmt:locale.obj
 0002:000103f4       ?_Src@?3??_Getffld@?$num_get@DV?$istreambuf_iterator@DU?$char_traits@D@std@@@std@@@std@@ABAHPADAAV?$istreambuf_iterator@DU?$char_traits@D@std@@@3@1AAVios_base@3@PAH@Z@4QBDB 101133f4     libcpmt:locale.obj
 0002:00010404       ??_C@_02MDKMJEGG@eE?$AA@   10113404     libcpmt:locale.obj
 0002:00010408       ??_C@_02OOPEBDOJ@pP?$AA@   10113408     libcpmt:locale.obj
 0002:0001040c       ?_Src@?1??_Getffldx@?$num_get@DV?$istreambuf_iterator@DU?$char_traits@D@std@@@std@@@std@@ABAHPADAAV?$istreambuf_iterator@DU?$char_traits@D@std@@@3@1AAVios_base@3@PAH@Z@4QBDB 1011340c     libcpmt:locale.obj
 0002:00010430       __real@38aa95a5b7f87a0f    10113430     libcpmt:locale.obj
 0002:00010438       __real@4202a05f20000000    10113438     libcpmt:locale.obj
 0002:00010440       __real@4733426172c74d82    10113440     libcpmt:locale.obj
 0002:00010448       ??_C@_0FG@EOHGAEB@?3Sun?3Sunday?3Mon?3Monday?3Tue?3Tuesd@ 10113448     libcpmt:wlocale.obj
 0002:000104a0       ??_C@_0IH@HPGJLCCK@?3Jan?3January?3Feb?3February?3Mar?3Ma@ 101134a0     libcpmt:wlocale.obj
 0002:00010528       ??_C@_1KM@LPDIELBN@?$AA?3?$AAS?$AAu?$AAn?$AA?3?$AAS?$AAu?$AAn?$AAd?$AAa?$AAy?$AA?3?$AAM?$AAo?$AAn?$AA?3?$AAM?$AAo?$AAn?$AAd?$AAa?$AAy?$AA?3?$AAT?$AAu?$AAe?$AA?3?$AAT?$AAu?$AAe?$AAs?$AAd@ 10113528     libcpmt:wlocale.obj
 0002:000105d8       ??_C@_1BAO@JIKOGLKA@?$AA?3?$AAJ?$AAa?$AAn?$AA?3?$AAJ?$AAa?$AAn?$AAu?$AAa?$AAr?$AAy?$AA?3?$AAF?$AAe?$AAb?$AA?3?$AAF?$AAe?$AAb?$AAr?$AAu?$AAa?$AAr?$AAy?$AA?3?$AAM?$AAa?$AAr?$AA?3?$AAM?$AAa@ 101135d8     libcpmt:wlocale.obj
 0002:000106ec       ??_7?$codecvt@_WDH@std@@6B@ 101136ec     libcpmt:wlocale.obj
 0002:00010718       ??_7?$codecvt@GDH@std@@6B@ 10113718     libcpmt:wlocale.obj
 0002:00010744       ??_7?$ctype@_W@std@@6B@    10113744     libcpmt:wlocale.obj
 0002:00010784       ??_7?$ctype@G@std@@6B@     10113784     libcpmt:wlocale.obj
 0002:000107c4       ??_7messages_base@std@@6B@ 101137c4     libcpmt:wlocale.obj
 0002:000107d4       ??_7money_base@std@@6B@    101137d4     libcpmt:wlocale.obj
 0002:000107e4       ??_7time_base@std@@6B@     101137e4     libcpmt:wlocale.obj
 0002:000107f4       ??_7?$time_put@_WV?$ostreambuf_iterator@_WU?$char_traits@_W@std@@@std@@@std@@6B@ 101137f4     libcpmt:wlocale.obj
 0002:00010808       ??_7?$num_get@_WV?$istreambuf_iterator@_WU?$char_traits@_W@std@@@std@@@std@@6B@ 10113808     libcpmt:wlocale.obj
 0002:00010844       ??_7?$num_put@_WV?$ostreambuf_iterator@_WU?$char_traits@_W@std@@@std@@@std@@6B@ 10113844     libcpmt:wlocale.obj
 0002:00010874       ??_7?$numpunct@_W@std@@6B@ 10113874     libcpmt:wlocale.obj
 0002:00010898       ??_7?$collate@_W@std@@6B@  10113898     libcpmt:wlocale.obj
 0002:000108b4       ??_7?$messages@_W@std@@6B@ 101138b4     libcpmt:wlocale.obj
 0002:000108d0       ??_7?$money_get@_WV?$istreambuf_iterator@_WU?$char_traits@_W@std@@@std@@@std@@6B@ 101138d0     libcpmt:wlocale.obj
 0002:000108e8       ??_7?$money_put@_WV?$ostreambuf_iterator@_WU?$char_traits@_W@std@@@std@@@std@@6B@ 101138e8     libcpmt:wlocale.obj
 0002:00010900       ??_7?$_Mpunct@_W@std@@6B@  10113900     libcpmt:wlocale.obj
 0002:00010934       ??_7?$moneypunct@_W$0A@@std@@6B@ 10113934     libcpmt:wlocale.obj
 0002:00010968       ??_7?$moneypunct@_W$00@std@@6B@ 10113968     libcpmt:wlocale.obj
 0002:0001099c       ??_7?$time_get@_WV?$istreambuf_iterator@_WU?$char_traits@_W@std@@@std@@@std@@6B@ 1011399c     libcpmt:wlocale.obj
 0002:000109c8       ??_7?$num_get@GV?$istreambuf_iterator@GU?$char_traits@G@std@@@std@@@std@@6B@ 101139c8     libcpmt:wlocale.obj
 0002:00010a04       ??_7?$num_put@GV?$ostreambuf_iterator@GU?$char_traits@G@std@@@std@@@std@@6B@ 10113a04     libcpmt:wlocale.obj
 0002:00010a34       ??_7?$numpunct@G@std@@6B@  10113a34     libcpmt:wlocale.obj
 0002:00010a58       ??_7?$collate@G@std@@6B@   10113a58     libcpmt:wlocale.obj
 0002:00010a74       ??_7?$messages@G@std@@6B@  10113a74     libcpmt:wlocale.obj
 0002:00010a90       ??_7?$money_get@GV?$istreambuf_iterator@GU?$char_traits@G@std@@@std@@@std@@6B@ 10113a90     libcpmt:wlocale.obj
 0002:00010aa8       ??_7?$money_put@GV?$ostreambuf_iterator@GU?$char_traits@G@std@@@std@@@std@@6B@ 10113aa8     libcpmt:wlocale.obj
 0002:00010ac0       ??_7?$_Mpunct@G@std@@6B@   10113ac0     libcpmt:wlocale.obj
 0002:00010af4       ??_7?$moneypunct@G$0A@@std@@6B@ 10113af4     libcpmt:wlocale.obj
 0002:00010b28       ??_7?$moneypunct@G$00@std@@6B@ 10113b28     libcpmt:wlocale.obj
 0002:00010b5c       ??_7?$time_get@GV?$istreambuf_iterator@GU?$char_traits@G@std@@@std@@@std@@6B@ 10113b5c     libcpmt:wlocale.obj
 0002:00010b88       ??_7?$time_put@GV?$ostreambuf_iterator@GU?$char_traits@G@std@@@std@@@std@@6B@ 10113b88     libcpmt:wlocale.obj
 0002:00010b98       ??_C@_19OKANBMPJ@?$AA?$CB?$AA?$CF?$AAx?$AA?$AA?$AA?$AA@ 10113b98     libcpmt:wlocale.obj
 0002:00010ba4       ??_C@_05NNKBBLJI@?$CF?40Lf?$AA@ 10113ba4     libcpmt:wlocale.obj
 0002:00010bac       ?_Src@?1??do_put@?$money_put@_WV?$ostreambuf_iterator@_WU?$char_traits@_W@std@@@std@@@std@@MBE?AV?$ostreambuf_iterator@_WU?$char_traits@_W@std@@@3@V43@_NAAVios_base@3@_WABV?$basic_string@_WU?$char_traits@_W@std@@V?$allocator@_W@2@@3@@Z@4QBDB 10113bac     libcpmt:wlocale.obj
 0002:00010bb8       ??_C@_0BG@ELKJEKEA@?$CFb?5?$CFd?5?$CFH?5?3?5?$CFM?5?3?5?$CFS?5?$CFY?$AA@ 10113bb8     libcpmt:wlocale.obj
 0002:00010bd0       ??_C@_0N@LIAHCJPJ@?$CFm?5?1?5?$CFd?5?1?5?$CFy?$AA@ 10113bd0     libcpmt:wlocale.obj
 0002:00010be0       ??_C@_0N@LPFKKEBD@?3AM?3am?3PM?3pm?$AA@ 10113be0     libcpmt:wlocale.obj
 0002:00010bf0       ??_C@_0BA@HGEPHOKI@?$CFI?5?3?5?$CFM?5?3?5?$CFS?5?$CFp?$AA@ 10113bf0     libcpmt:wlocale.obj
 0002:00010c00       ??_C@_07GLPBMING@?$CFH?5?3?5?$CFM?$AA@ 10113c00     libcpmt:wlocale.obj
 0002:00010c08       ??_C@_0M@LMMIDGCH@?$CFH?5?3?5?$CFM?5?3?5S?$AA@ 10113c08     libcpmt:wlocale.obj
 0002:00010c14       ??_C@_0N@LADGFGLL@?$CFd?5?1?5?$CFm?5?1?5?$CFy?$AA@ 10113c14     libcpmt:wlocale.obj
 0002:00010c24       ?_Src@?1??do_put@?$money_put@GV?$ostreambuf_iterator@GU?$char_traits@G@std@@@std@@@std@@MBE?AV?$ostreambuf_iterator@GU?$char_traits@G@std@@@3@V43@_NAAVios_base@3@GABV?$basic_string@GU?$char_traits@G@std@@V?$allocator@G@2@@3@@Z@4QBDB 10113c24     libcpmt:wlocale.obj
 0002:00010c30       ?_Src@?1??_Getifld@?$num_get@_WV?$istreambuf_iterator@_WU?$char_traits@_W@std@@@std@@@std@@ABAHPADAAV?$istreambuf_iterator@_WU?$char_traits@_W@std@@@3@1HABVlocale@3@@Z@4QBDB 10113c30     libcpmt:wlocale.obj
 0002:00010c4c       ?_Src@?3??_Getffld@?$num_get@_WV?$istreambuf_iterator@_WU?$char_traits@_W@std@@@std@@@std@@ABAHPADAAV?$istreambuf_iterator@_WU?$char_traits@_W@std@@@3@1AAVios_base@3@PAH@Z@4QBDB 10113c4c     libcpmt:wlocale.obj
 0002:00010c5c       ?_Src@?4??_Getmfld@?$money_get@_WV?$istreambuf_iterator@_WU?$char_traits@_W@std@@@std@@@std@@ABE?AV?$basic_string@DU?$char_traits@D@std@@V?$allocator@D@2@@3@AAV?$istreambuf_iterator@_WU?$char_traits@_W@std@@@3@0_NAAVios_base@3@PA_W@Z@4QBDB 10113c5c     libcpmt:wlocale.obj
 0002:00010c68       ?_Src@?1??_Getifld@?$num_get@GV?$istreambuf_iterator@GU?$char_traits@G@std@@@std@@@std@@ABAHPADAAV?$istreambuf_iterator@GU?$char_traits@G@std@@@3@1HABVlocale@3@@Z@4QBDB 10113c68     libcpmt:wlocale.obj
 0002:00010c84       ?_Src@?3??_Getffld@?$num_get@GV?$istreambuf_iterator@GU?$char_traits@G@std@@@std@@@std@@ABAHPADAAV?$istreambuf_iterator@GU?$char_traits@G@std@@@3@1AAVios_base@3@PAH@Z@4QBDB 10113c84     libcpmt:wlocale.obj
 0002:00010c94       ?_Src@?4??_Getmfld@?$money_get@GV?$istreambuf_iterator@GU?$char_traits@G@std@@@std@@@std@@ABE?AV?$basic_string@DU?$char_traits@D@std@@V?$allocator@D@2@@3@AAV?$istreambuf_iterator@GU?$char_traits@G@std@@@3@0_NAAVios_base@3@PAG@Z@4QBDB 10113c94     libcpmt:wlocale.obj
 0002:00010ca0       ?_Src@?1??_Getffldx@?$num_get@_WV?$istreambuf_iterator@_WU?$char_traits@_W@std@@@std@@@std@@ABAHPADAAV?$istreambuf_iterator@_WU?$char_traits@_W@std@@@3@1AAVios_base@3@PAH@Z@4QBDB 10113ca0     libcpmt:wlocale.obj
 0002:00010cc0       ??_C@_04FJCIEOIB@$?$CLxv?$AA@ 10113cc0     libcpmt:wlocale.obj
 0002:00010cc8       ??_C@_1BK@MHIKGOKE@?$AA?3?$AAA?$AAM?$AA?3?$AAa?$AAm?$AA?3?$AAP?$AAM?$AA?3?$AAp?$AAm?$AA?$AA@ 10113cc8     libcpmt:wlocale.obj
 0002:00010ce4       ?_Src@?1??_Getffldx@?$num_get@GV?$istreambuf_iterator@GU?$char_traits@G@std@@@std@@@std@@ABAHPADAAV?$istreambuf_iterator@GU?$char_traits@G@std@@@3@1AAVios_base@3@PAH@Z@4QBDB 10113ce4     libcpmt:wlocale.obj
 0002:00010d04       ??_C@_13IMODFHAA@?$AA?9?$AA?$AA@ 10113d04     libcpmt:wlocale.obj
 0002:00010d08       ??_C@_0HJ@PJOMAIHM@?$CLv$x?$CLv$xv$?$CLxv?$CL$xv$?$CLx?$CL$vx?$CL$vx$v?$CLx@ 10113d08     libcpmt:wlocale.obj
 0002:00010d88       ??_7?$collate@D@std@@6B@   10113d88     libcpmt:xlocale.obj
 0002:00010da4       ??_7?$messages@D@std@@6B@  10113da4     libcpmt:xlocale.obj
 0002:00010dc0       ??_7?$money_get@DV?$istreambuf_iterator@DU?$char_traits@D@std@@@std@@@std@@6B@ 10113dc0     libcpmt:xlocale.obj
 0002:00010dd8       ??_7?$money_put@DV?$ostreambuf_iterator@DU?$char_traits@D@std@@@std@@@std@@6B@ 10113dd8     libcpmt:xlocale.obj
 0002:00010df0       ??_7?$_Mpunct@D@std@@6B@   10113df0     libcpmt:xlocale.obj
 0002:00010e24       ??_7?$moneypunct@D$0A@@std@@6B@ 10113e24     libcpmt:xlocale.obj
 0002:00010e58       ??_7?$moneypunct@D$00@std@@6B@ 10113e58     libcpmt:xlocale.obj
 0002:00010e8c       ??_7?$time_get@DV?$istreambuf_iterator@DU?$char_traits@D@std@@@std@@@std@@6B@ 10113e8c     libcpmt:xlocale.obj
 0002:00010eb8       ??_7?$time_put@DV?$ostreambuf_iterator@DU?$char_traits@D@std@@@std@@@std@@6B@ 10113eb8     libcpmt:xlocale.obj
 0002:00010ec8       ?_Src@?1??do_put@?$money_put@DV?$ostreambuf_iterator@DU?$char_traits@D@std@@@std@@@std@@MBE?AV?$ostreambuf_iterator@DU?$char_traits@D@std@@@3@V43@_NAAVios_base@3@DABV?$basic_string@DU?$char_traits@D@std@@V?$allocator@D@2@@3@@Z@4QBDB 10113ec8     libcpmt:xlocale.obj
 0002:00010ed4       ??_C@_04IHCGILC@?$CB?$CFx?$AA?$AA@ 10113ed4     libcpmt:xlocale.obj
 0002:00010edc       ?_Src@?4??_Getmfld@?$money_get@DV?$istreambuf_iterator@DU?$char_traits@D@std@@@std@@@std@@ABE?AV?$basic_string@DU?$char_traits@D@std@@V?$allocator@D@2@@3@AAV?$istreambuf_iterator@DU?$char_traits@D@std@@@3@0_NAAVios_base@3@PAD@Z@4QBDB 10113edc     libcpmt:xlocale.obj
 0002:00010ee8       __real@4d800000            10113ee8     libcpmt:xstof.obj
 0002:00010eec       __real@4e6e6b28            10113eec     libcpmt:xstof.obj
 0002:00010ef0       __real@41b0000000000000    10113ef0     libcpmt:xstod.obj
 0002:00010fc8       __real@3f800000            10113fc8     libcpmt:xfprec.obj
 0002:00010fcc       __real@3fc00000            10113fcc     libcpmt:xfprec.obj
 0002:00010fd0       __real@461c4000            10113fd0     libcpmt:xfprec.obj
 0002:00010fd4       __real@bf000000            10113fd4     libcpmt:xfprec.obj
 0002:00010fd8       __real@bf800000            10113fd8     libcpmt:xfprec.obj
 0002:00010fe8       __real@41200000            10113fe8     libcpmt:xfdtento.obj
 0002:00010ff0       __real@3ff8000000000000    10113ff0     libcpmt:xprec.obj
 0002:00010ff8       __real@bfe0000000000000    10113ff8     libcpmt:xprec.obj
 0002:00028bc0       ??_C@_0BH@DPNNDOEK@invalid?5stoul?5argument?$AA@ 1012bbc0     libsg_MSVC120_vc:sg_common.obj
 0002:00028bd8       ??_C@_0BM@MOLGGFGJ@stoul?5argument?5out?5of?5range?$AA@ 1012bbd8     libsg_MSVC120_vc:sg_common.obj
 0002:00028bf4       ??_C@_05LLAMLEHD@?$CFI64d?$AA@ 1012bbf4     libsg_MSVC120_vc:sg_common.obj
 0002:00028bfc       ??_C@_0CG@HGCDJNPD@?$CFs?5ID?$CFi?3?5Invalid?5PCI?5bus?5argumen@ 1012bbfc     libsg_MSVC120_vc:sg_common.obj
 0002:00028c24       ??_C@_0CO@FBMLOABH@?$CFs?5ID?$CFi?3?5Not?5found?5at?5bus?5?$CFi?0?5sl@ 1012bc24     libsg_MSVC120_vc:sg_common.obj
 0002:00028c54       ??_C@_0BJ@EIMDIBO@?$CFs?3?5No?5such?5module?5found?$AA@ 1012bc54     libsg_MSVC120_vc:sg_common.obj
 0002:00028c70       ??_C@_0JM@PEIHKLM@?$CFs?5ID?$CFi?3?5Only?5?$CFi?5modules?5found?4?5@ 1012bc70     libsg_MSVC120_vc:sg_common.obj
 0002:00028d0c       ??_C@_0BH@OIBECGCO@?$CFs?5ID?$CFi?3?5Unknown?5error?$AA@ 1012bd0c     libsg_MSVC120_vc:sg_common.obj
 0002:00028d24       ??_C@_01KICIPPFI@?2?$AA@   1012bd24     libsg_MSVC120_vc:sg_common.obj
 0002:00028d28       ??_C@_0M@KJDBOOKF@?$CFc?3?1private?$AA@ 1012bd28     libsg_MSVC120_vc:sg_common.obj
 0002:00028d34       ??_C@_03CGGPNEOP@?$CFc?3?$AA@ 1012bd34     libsg_MSVC120_vc:sg_common.obj
 0002:00028d38       ??_C@_0BL@JFNNPFLJ@C?3?2authentication_info?4txt?$AA@ 1012bd38     libsg_MSVC120_vc:sg_common.obj
 0002:00028d54       ??_C@_0BK@HJFGAJJP@?$CF02X?$CF02X?$CF02X?$CF02X?$CF02X?$CF02X?6?$AA@ 1012bd54     libsg_MSVC120_vc:sg_common.obj
 0002:00028d70       ??_C@_0DG@IJKDDMBP@WARNING?3?5Failed?5to?5authenticate?5@ 1012bd70     libsg_MSVC120_vc:sg_common.obj
 0002:00028da8       ??_C@_0II@EEMDOLCB@Please?5execute?5?$CCspeedgoat?4getTar@ 1012bda8     libsg_MSVC120_vc:sg_common.obj
 0002:00028e30       ??_C@_0CL@HEHPFKND@Could?5not?5authenticate?5this?5targ@ 1012be30     libsg_MSVC120_vc:sg_common.obj
 0002:00028e5c       ??_C@_0L@OEBJDFEB@C?3?2sn?$CK?4txt?$AA@ 1012be5c     libsg_MSVC120_vc:sg_common.obj
 0002:00028e68       ??_C@_03GIOIKFCO@C?3?2?$AA@ 1012be68     libsg_MSVC120_vc:sg_common.obj
 0002:00028e6c       ??_C@_0M@MKPBBFKF@Content?5of?5?$AA@ 1012be6c     libsg_MSVC120_vc:sg_common.obj
 0002:00028e78       ??_C@_0BI@HCPPCGN@Found?5matching?5hash?5in?5?$AA@ 1012be78     libsg_MSVC120_vc:sg_common.obj
 0002:00028e90       ??_C@_0BF@HGDMHCNA@Removing?5left?5over?3?5?$AA@ 1012be90     libsg_MSVC120_vc:sg_common.obj
 0002:00028ea8       ??_C@_0BP@IMFDMJDB@Hash?5did?5not?5match?0?5removing?3?5?$AA@ 1012bea8     libsg_MSVC120_vc:sg_common.obj
 0002:00028ec8       ??_C@_0DO@IJECAAME@No?5valid?5sn?$CK?4txt?5files?5found?0?5st@ 1012bec8     libsg_MSVC120_vc:sg_common.obj
 0002:00028f08       ??_C@_09NINLLEJH@?0?5hash?5?$DN?5?$AA@ 1012bf08     libsg_MSVC120_vc:sg_common.obj
 0002:00028f14       ??_C@_0BK@GAJLKPLN@Found?5hash?5in?5list?5under?5?$AA@ 1012bf14     libsg_MSVC120_vc:sg_common.obj
 0002:00028f30       ??_C@_05HCKGID@C?3?2sn?$AA@ 1012bf30     libsg_MSVC120_vc:sg_common.obj
 0002:00028f38       ??_C@_04LCMACLFG@?4txt?$AA@ 1012bf38     libsg_MSVC120_vc:sg_common.obj
 0002:00028f40       ??_C@_0L@IMMGEBDC@?0?5content?3?$AA@ 1012bf40     libsg_MSVC120_vc:sg_common.obj
 0002:00028f4c       ??_C@_0BE@PBJICLEC@Creating?5new?5file?3?5?$AA@ 1012bf4c     libsg_MSVC120_vc:sg_common.obj
 0002:00028f60       ??_C@_0EH@LGNMCHLI@Nothing?5found?5in?5serial?5list?0?5st@ 1012bf60     libsg_MSVC120_vc:sg_common.obj
 0002:00028fa8       ??_C@_0CD@CAPDBBG@Found?5hash?5in?5internal?5list?5unde@ 1012bfa8     libsg_MSVC120_vc:sg_common.obj
 0002:00028fcc       ??_C@_06MAIOHANC@C?3?2sni?$AA@ 1012bfcc     libsg_MSVC120_vc:sg_common.obj
 0002:00028fd8       ??_C@_0EJ@BGCHNLAM@Nothing?5found?5in?5internal?5list?0?5@ 1012bfd8     libsg_MSVC120_vc:sg_common.obj
 0002:00029024       ??_C@_0CD@PFIBLOKA@Found?5hash?5in?5supplier?5list?5unde@ 1012c024     libsg_MSVC120_vc:sg_common.obj
 0002:00029048       ??_C@_06HAKDIKAJ@C?3?2sns?$AA@ 1012c048     libsg_MSVC120_vc:sg_common.obj
 0002:00029050       ??_C@_0CC@NPPIBBIO@Hash?5was?5not?5found?5in?5serial?5lis@ 1012c050     libsg_MSVC120_vc:sg_common.obj
 0002:00029074       ??_C@_0CA@OAHLAOAI@Created?5authentication_info?4txt?$AA@ 1012c074     libsg_MSVC120_vc:sg_common.obj
 0002:00029098       __real@4000000000000000    1012c098     libsg_MSVC120_vc:sg_common.obj
 0002:000290a0       __xmm@80000000000000008000000000000000 1012c0a0     libsg_MSVC120_vc:sg_common.obj
 0002:000290b0       ??_C@_0BG@HGEDEDEC@invalid?5stoi?5argument?$AA@ 1012c0b0     libsg_MSVC120_vc:sg_target.obj
 0002:000290c8       ??_C@_0BL@MFFNMGGC@stoi?5argument?5out?5of?5range?$AA@ 1012c0c8     libsg_MSVC120_vc:sg_target.obj
 0002:000290e4       ??_C@_09PCFJFKEK@NICGetMac?$AA@ 1012c0e4     libsg_MSVC120_vc:sg_target.obj
 0002:000290f0       ??_C@_01LFCBOECM@?4?$AA@   1012c0f0     libsg_MSVC120_vc:sg_target.obj
 0002:000290f4       ??_C@_1M@PBPMMENC@?$AAa?$AAm?$AA?1?$AAp?$AAm?$AA?$AA@ 1012c0f4     LIBCMT:wcsftime.obj
 0002:00029100       ??_C@_17BLFJJHMM@?$AAa?$AA?1?$AAp?$AA?$AA@ 1012c100     LIBCMT:wcsftime.obj
 0002:0002ca88       ??_C@_02CLFPBFFP@TZ?$AA@   1012fa88     LIBCMT:tzset.obj
 0002:0002ca8c       ___dnames                  1012fa8c     LIBCMT:timeset.obj
 0002:0002caa4       ___mnames                  1012faa4     LIBCMT:timeset.obj
 0002:00030410       __infinity                 10133410     LIBCMT:87tran.obj
 0002:0003041a       __minfinity                1013341a     LIBCMT:87tran.obj
 0002:00030424       __logemax                  10133424     LIBCMT:87tran.obj
 0002:0003044a       __OP_EXPjmptab             1013344a     LIBCMT:87tran.obj
 0002:00030470       __real@3f538bcdfefbf402    10133470     xpcruntime:xpcPCFunctions.obj
 0002:00030478       __real@40112e0be826d695    10133478     xpcruntime:xpcPCFunctions.obj
 0002:00030480       __real@40f0000000000000    10133480     xpcruntime:xpcPCFunctions.obj
 0002:00030488       __load_config_used         10133488     LIBCMT:loadcfg.obj
 0002:0003951c       ??_R4error_category@std@@6B@ 1013c51c     IO61X_Library_MSVC120_vc:IO61X_iConcurrentExecution.obj
 0002:00039530       ??_R3error_category@std@@8 1013c530     IO61X_Library_MSVC120_vc:IO61X_iConcurrentExecution.obj
 0002:00039540       ??_R2error_category@std@@8 1013c540     IO61X_Library_MSVC120_vc:IO61X_iConcurrentExecution.obj
 0002:00039548       ??_R1A@?0A@EA@error_category@std@@8 1013c548     IO61X_Library_MSVC120_vc:IO61X_iConcurrentExecution.obj
 0002:00039564       ??_R4_Generic_error_category@std@@6B@ 1013c564     IO61X_Library_MSVC120_vc:IO61X_iConcurrentExecution.obj
 0002:00039578       ??_R3_Generic_error_category@std@@8 1013c578     IO61X_Library_MSVC120_vc:IO61X_iConcurrentExecution.obj
 0002:00039588       ??_R2_Generic_error_category@std@@8 1013c588     IO61X_Library_MSVC120_vc:IO61X_iConcurrentExecution.obj
 0002:00039594       ??_R1A@?0A@EA@_Generic_error_category@std@@8 1013c594     IO61X_Library_MSVC120_vc:IO61X_iConcurrentExecution.obj
 0002:000395b0       ??_R4_Iostream_error_category@std@@6B@ 1013c5b0     IO61X_Library_MSVC120_vc:IO61X_iConcurrentExecution.obj
 0002:000395c4       ??_R3_Iostream_error_category@std@@8 1013c5c4     IO61X_Library_MSVC120_vc:IO61X_iConcurrentExecution.obj
 0002:000395d4       ??_R2_Iostream_error_category@std@@8 1013c5d4     IO61X_Library_MSVC120_vc:IO61X_iConcurrentExecution.obj
 0002:000395e4       ??_R1A@?0A@EA@_Iostream_error_category@std@@8 1013c5e4     IO61X_Library_MSVC120_vc:IO61X_iConcurrentExecution.obj
 0002:00039600       ??_R4_System_error_category@std@@6B@ 1013c600     IO61X_Library_MSVC120_vc:IO61X_iConcurrentExecution.obj
 0002:00039614       ??_R3_System_error_category@std@@8 1013c614     IO61X_Library_MSVC120_vc:IO61X_iConcurrentExecution.obj
 0002:00039624       ??_R2_System_error_category@std@@8 1013c624     IO61X_Library_MSVC120_vc:IO61X_iConcurrentExecution.obj
 0002:00039634       ??_R1A@?0A@EA@_System_error_category@std@@8 1013c634     IO61X_Library_MSVC120_vc:IO61X_iConcurrentExecution.obj
 0002:00039650       ??_R1A@?0A@EA@exception@std@@8 1013c650     IO61X_Library_MSVC120_vc:IO61X_DriverObject.obj
 0002:0003966c       ??_R3exception@std@@8      1013c66c     IO61X_Library_MSVC120_vc:IO61X_DriverObject.obj
 0002:0003967c       ??_R2exception@std@@8      1013c67c     IO61X_Library_MSVC120_vc:IO61X_DriverObject.obj
 0002:00039684       ??_R4ios_base@std@@6B@     1013c684     IO61X_Library_MSVC120_vc:IO61X_DriverObject.obj
 0002:00039698       ??_R3ios_base@std@@8       1013c698     IO61X_Library_MSVC120_vc:IO61X_DriverObject.obj
 0002:000396a8       ??_R2ios_base@std@@8       1013c6a8     IO61X_Library_MSVC120_vc:IO61X_DriverObject.obj
 0002:000396b4       ??_R1A@?0A@EA@ios_base@std@@8 1013c6b4     IO61X_Library_MSVC120_vc:IO61X_DriverObject.obj
 0002:000396d0       ??_R17?0A@EA@?$_Iosb@H@std@@8 1013c6d0     IO61X_Library_MSVC120_vc:IO61X_DriverObject.obj
 0002:000396ec       ??_R3?$_Iosb@H@std@@8      1013c6ec     IO61X_Library_MSVC120_vc:IO61X_DriverObject.obj
 0002:000396fc       ??_R2?$_Iosb@H@std@@8      1013c6fc     IO61X_Library_MSVC120_vc:IO61X_DriverObject.obj
 0002:00039704       ??_R1A@?0A@EA@?$_Iosb@H@std@@8 1013c704     IO61X_Library_MSVC120_vc:IO61X_DriverObject.obj
 0002:00039720       ??_R4?$basic_ios@DU?$char_traits@D@std@@@std@@6B@ 1013c720     IO61X_Library_MSVC120_vc:IO61X_DriverObject.obj
 0002:00039734       ??_R3?$basic_ios@DU?$char_traits@D@std@@@std@@8 1013c734     IO61X_Library_MSVC120_vc:IO61X_DriverObject.obj
 0002:00039744       ??_R2?$basic_ios@DU?$char_traits@D@std@@@std@@8 1013c744     IO61X_Library_MSVC120_vc:IO61X_DriverObject.obj
 0002:00039754       ??_R1A@?0A@EA@?$basic_ios@DU?$char_traits@D@std@@@std@@8 1013c754     IO61X_Library_MSVC120_vc:IO61X_DriverObject.obj
 0002:00039770       ??_R4?$basic_streambuf@DU?$char_traits@D@std@@@std@@6B@ 1013c770     IO61X_Library_MSVC120_vc:IO61X_DriverObject.obj
 0002:00039784       ??_R3?$basic_streambuf@DU?$char_traits@D@std@@@std@@8 1013c784     IO61X_Library_MSVC120_vc:IO61X_DriverObject.obj
 0002:00039794       ??_R2?$basic_streambuf@DU?$char_traits@D@std@@@std@@8 1013c794     IO61X_Library_MSVC120_vc:IO61X_DriverObject.obj
 0002:0003979c       ??_R1A@?0A@EA@?$basic_streambuf@DU?$char_traits@D@std@@@std@@8 1013c79c     IO61X_Library_MSVC120_vc:IO61X_DriverObject.obj
 0002:000397b8       ??_R1A@A@3FA@?$basic_ios@DU?$char_traits@D@std@@@std@@8 1013c7b8     IO61X_Library_MSVC120_vc:IO61X_DriverObject.obj
 0002:000397d4       ??_R1A@A@3EA@ios_base@std@@8 1013c7d4     IO61X_Library_MSVC120_vc:IO61X_DriverObject.obj
 0002:000397f0       ??_R17A@3EA@?$_Iosb@H@std@@8 1013c7f0     IO61X_Library_MSVC120_vc:IO61X_DriverObject.obj
 0002:0003980c       ??_R4?$basic_ostream@DU?$char_traits@D@std@@@std@@6B@ 1013c80c     IO61X_Library_MSVC120_vc:IO61X_DriverObject.obj
 0002:00039820       ??_R3?$basic_ostream@DU?$char_traits@D@std@@@std@@8 1013c820     IO61X_Library_MSVC120_vc:IO61X_DriverObject.obj
 0002:00039830       ??_R2?$basic_ostream@DU?$char_traits@D@std@@@std@@8 1013c830     IO61X_Library_MSVC120_vc:IO61X_DriverObject.obj
 0002:00039844       ??_R1A@?0A@EA@?$basic_ostream@DU?$char_traits@D@std@@@std@@8 1013c844     IO61X_Library_MSVC120_vc:IO61X_DriverObject.obj
 0002:00039860       ??_R4?$basic_filebuf@DU?$char_traits@D@std@@@std@@6B@ 1013c860     IO61X_Library_MSVC120_vc:IO61X_DriverObject.obj
 0002:00039874       ??_R3?$basic_filebuf@DU?$char_traits@D@std@@@std@@8 1013c874     IO61X_Library_MSVC120_vc:IO61X_DriverObject.obj
 0002:00039884       ??_R2?$basic_filebuf@DU?$char_traits@D@std@@@std@@8 1013c884     IO61X_Library_MSVC120_vc:IO61X_DriverObject.obj
 0002:00039890       ??_R1A@?0A@EA@?$basic_filebuf@DU?$char_traits@D@std@@@std@@8 1013c890     IO61X_Library_MSVC120_vc:IO61X_DriverObject.obj
 0002:000398ac       ??_R4?$basic_ofstream@DU?$char_traits@D@std@@@std@@6B@ 1013c8ac     IO61X_Library_MSVC120_vc:IO61X_DriverObject.obj
 0002:000398c0       ??_R3?$basic_ofstream@DU?$char_traits@D@std@@@std@@8 1013c8c0     IO61X_Library_MSVC120_vc:IO61X_DriverObject.obj
 0002:000398d0       ??_R2?$basic_ofstream@DU?$char_traits@D@std@@@std@@8 1013c8d0     IO61X_Library_MSVC120_vc:IO61X_DriverObject.obj
 0002:000398e8       ??_R1A@?0A@EA@?$basic_ofstream@DU?$char_traits@D@std@@@std@@8 1013c8e8     IO61X_Library_MSVC120_vc:IO61X_DriverObject.obj
 0002:00039904       ??_R4logic_error@std@@6B@  1013c904     IO61X_Library_MSVC120_vc:IO61X_DriverObject.obj
 0002:00039918       ??_R3logic_error@std@@8    1013c918     IO61X_Library_MSVC120_vc:IO61X_DriverObject.obj
 0002:00039928       ??_R2logic_error@std@@8    1013c928     IO61X_Library_MSVC120_vc:IO61X_DriverObject.obj
 0002:00039934       ??_R1A@?0A@EA@logic_error@std@@8 1013c934     IO61X_Library_MSVC120_vc:IO61X_DriverObject.obj
 0002:00039950       ??_R4invalid_argument@std@@6B@ 1013c950     IO61X_Library_MSVC120_vc:IO61X_DriverObject.obj
 0002:00039964       ??_R3invalid_argument@std@@8 1013c964     IO61X_Library_MSVC120_vc:IO61X_DriverObject.obj
 0002:00039974       ??_R2invalid_argument@std@@8 1013c974     IO61X_Library_MSVC120_vc:IO61X_DriverObject.obj
 0002:00039984       ??_R1A@?0A@EA@invalid_argument@std@@8 1013c984     IO61X_Library_MSVC120_vc:IO61X_DriverObject.obj
 0002:000399a0       ??_R4runtime_error@std@@6B@ 1013c9a0     IO61X_Library_MSVC120_vc:IO61X_DriverObject.obj
 0002:000399b4       ??_R3runtime_error@std@@8  1013c9b4     IO61X_Library_MSVC120_vc:IO61X_DriverObject.obj
 0002:000399c4       ??_R2runtime_error@std@@8  1013c9c4     IO61X_Library_MSVC120_vc:IO61X_DriverObject.obj
 0002:000399d0       ??_R1A@?0A@EA@runtime_error@std@@8 1013c9d0     IO61X_Library_MSVC120_vc:IO61X_DriverObject.obj
 0002:000399ec       ??_R4_Facet_base@std@@6B@  1013c9ec     IO61X_Library_MSVC120_vc:IO61X_DriverObject.obj
 0002:00039a00       ??_R3_Facet_base@std@@8    1013ca00     IO61X_Library_MSVC120_vc:IO61X_DriverObject.obj
 0002:00039a10       ??_R2_Facet_base@std@@8    1013ca10     IO61X_Library_MSVC120_vc:IO61X_DriverObject.obj
 0002:00039a18       ??_R1A@?0A@EA@_Facet_base@std@@8 1013ca18     IO61X_Library_MSVC120_vc:IO61X_DriverObject.obj
 0002:00039a34       ??_R1A@?0A@EA@facet@locale@std@@8 1013ca34     IO61X_Library_MSVC120_vc:IO61X_DriverObject.obj
 0002:00039a50       ??_R3facet@locale@std@@8   1013ca50     IO61X_Library_MSVC120_vc:IO61X_DriverObject.obj
 0002:00039a60       ??_R2facet@locale@std@@8   1013ca60     IO61X_Library_MSVC120_vc:IO61X_DriverObject.obj
 0002:00039a6c       ??_R4facet@locale@std@@6B@ 1013ca6c     IO61X_Library_MSVC120_vc:IO61X_DriverObject.obj
 0002:00039a80       ??_R4codecvt_base@std@@6B@ 1013ca80     IO61X_Library_MSVC120_vc:IO61X_DriverObject.obj
 0002:00039a94       ??_R3codecvt_base@std@@8   1013ca94     IO61X_Library_MSVC120_vc:IO61X_DriverObject.obj
 0002:00039aa4       ??_R2codecvt_base@std@@8   1013caa4     IO61X_Library_MSVC120_vc:IO61X_DriverObject.obj
 0002:00039ab4       ??_R1A@?0A@EA@codecvt_base@std@@8 1013cab4     IO61X_Library_MSVC120_vc:IO61X_DriverObject.obj
 0002:00039ad0       ??_R4ctype_base@std@@6B@   1013cad0     IO61X_Library_MSVC120_vc:IO61X_DriverObject.obj
 0002:00039ae4       ??_R3ctype_base@std@@8     1013cae4     IO61X_Library_MSVC120_vc:IO61X_DriverObject.obj
 0002:00039af4       ??_R2ctype_base@std@@8     1013caf4     IO61X_Library_MSVC120_vc:IO61X_DriverObject.obj
 0002:00039b04       ??_R1A@?0A@EA@ctype_base@std@@8 1013cb04     IO61X_Library_MSVC120_vc:IO61X_DriverObject.obj
 0002:00039b20       ??_R4?$ctype@D@std@@6B@    1013cb20     IO61X_Library_MSVC120_vc:IO61X_DriverObject.obj
 0002:00039b34       ??_R3?$ctype@D@std@@8      1013cb34     IO61X_Library_MSVC120_vc:IO61X_DriverObject.obj
 0002:00039b44       ??_R2?$ctype@D@std@@8      1013cb44     IO61X_Library_MSVC120_vc:IO61X_DriverObject.obj
 0002:00039b58       ??_R1A@?0A@EA@?$ctype@D@std@@8 1013cb58     IO61X_Library_MSVC120_vc:IO61X_DriverObject.obj
 0002:00039b74       ??_R4_System_error@std@@6B@ 1013cb74     IO61X_Library_MSVC120_vc:IO61X_DriverObject.obj
 0002:00039b88       ??_R3_System_error@std@@8  1013cb88     IO61X_Library_MSVC120_vc:IO61X_DriverObject.obj
 0002:00039b98       ??_R2_System_error@std@@8  1013cb98     IO61X_Library_MSVC120_vc:IO61X_DriverObject.obj
 0002:00039ba8       ??_R1A@?0A@EA@_System_error@std@@8 1013cba8     IO61X_Library_MSVC120_vc:IO61X_DriverObject.obj
 0002:00039bc4       ??_R4system_error@std@@6B@ 1013cbc4     IO61X_Library_MSVC120_vc:IO61X_DriverObject.obj
 0002:00039bd8       ??_R3system_error@std@@8   1013cbd8     IO61X_Library_MSVC120_vc:IO61X_DriverObject.obj
 0002:00039be8       ??_R2system_error@std@@8   1013cbe8     IO61X_Library_MSVC120_vc:IO61X_DriverObject.obj
 0002:00039bfc       ??_R1A@?0A@EA@system_error@std@@8 1013cbfc     IO61X_Library_MSVC120_vc:IO61X_DriverObject.obj
 0002:00039c18       ??_R4failure@ios_base@std@@6B@ 1013cc18     IO61X_Library_MSVC120_vc:IO61X_DriverObject.obj
 0002:00039c2c       ??_R3failure@ios_base@std@@8 1013cc2c     IO61X_Library_MSVC120_vc:IO61X_DriverObject.obj
 0002:00039c3c       ??_R2failure@ios_base@std@@8 1013cc3c     IO61X_Library_MSVC120_vc:IO61X_DriverObject.obj
 0002:00039c54       ??_R1A@?0A@EA@failure@ios_base@std@@8 1013cc54     IO61X_Library_MSVC120_vc:IO61X_DriverObject.obj
 0002:00039c70       ??_R4?$codecvt@DDH@std@@6B@ 1013cc70     IO61X_Library_MSVC120_vc:IO61X_DriverObject.obj
 0002:00039c84       ??_R3?$codecvt@DDH@std@@8  1013cc84     IO61X_Library_MSVC120_vc:IO61X_DriverObject.obj
 0002:00039c94       ??_R2?$codecvt@DDH@std@@8  1013cc94     IO61X_Library_MSVC120_vc:IO61X_DriverObject.obj
 0002:00039ca8       ??_R1A@?0A@EA@?$codecvt@DDH@std@@8 1013cca8     IO61X_Library_MSVC120_vc:IO61X_DriverObject.obj
 0002:00039cc4       ??_R4IO61X_Port@@6B@       1013ccc4     IO61X_Library_MSVC120_vc:IO61X_Port.obj
 0002:00039cd8       ??_R3IO61X_Port@@8         1013ccd8     IO61X_Library_MSVC120_vc:IO61X_Port.obj
 0002:00039ce8       ??_R2IO61X_Port@@8         1013cce8     IO61X_Library_MSVC120_vc:IO61X_Port.obj
 0002:00039cf0       ??_R1A@?0A@EA@IO61X_Port@@8 1013ccf0     IO61X_Library_MSVC120_vc:IO61X_Port.obj
 0002:00039d0c       ??_R4IO61X_CanPort@@6B@    1013cd0c     IO61X_Library_MSVC120_vc:IO61X_CanPort.obj
 0002:00039d20       ??_R3IO61X_CanPort@@8      1013cd20     IO61X_Library_MSVC120_vc:IO61X_CanPort.obj
 0002:00039d30       ??_R2IO61X_CanPort@@8      1013cd30     IO61X_Library_MSVC120_vc:IO61X_CanPort.obj
 0002:00039d3c       ??_R1A@?0A@EA@IO61X_CanPort@@8 1013cd3c     IO61X_Library_MSVC120_vc:IO61X_CanPort.obj
 0002:00039d58       ??_R4IO61X_CanFdPort@@6B@  1013cd58     IO61X_Library_MSVC120_vc:IO61X_CanFdPort.obj
 0002:00039d6c       ??_R3IO61X_CanFdPort@@8    1013cd6c     IO61X_Library_MSVC120_vc:IO61X_CanFdPort.obj
 0002:00039d7c       ??_R2IO61X_CanFdPort@@8    1013cd7c     IO61X_Library_MSVC120_vc:IO61X_CanFdPort.obj
 0002:00039d88       ??_R1A@?0A@EA@IO61X_CanFdPort@@8 1013cd88     IO61X_Library_MSVC120_vc:IO61X_CanFdPort.obj
 0002:00039da4       ??_R4IO61X_LinPort@@6B@    1013cda4     IO61X_Library_MSVC120_vc:IO61X_LinPort.obj
 0002:00039db8       ??_R3IO61X_LinPort@@8      1013cdb8     IO61X_Library_MSVC120_vc:IO61X_LinPort.obj
 0002:00039dc8       ??_R2IO61X_LinPort@@8      1013cdc8     IO61X_Library_MSVC120_vc:IO61X_LinPort.obj
 0002:00039dd4       ??_R1A@?0A@EA@IO61X_LinPort@@8 1013cdd4     IO61X_Library_MSVC120_vc:IO61X_LinPort.obj
 0002:00039df0       ??_R4bad_alloc@std@@6B@    1013cdf0     LIBCMT:new.obj
 0002:00039e04       ??_R3bad_alloc@std@@8      1013ce04     LIBCMT:new.obj
 0002:00039e14       ??_R2bad_alloc@std@@8      1013ce14     LIBCMT:new.obj
 0002:00039e20       ??_R1A@?0A@EA@bad_alloc@std@@8 1013ce20     LIBCMT:new.obj
 0002:00039e3c       ??_R4type_info@@6B@        1013ce3c     LIBCMT:typinfo.obj
 0002:00039e50       ??_R3type_info@@8          1013ce50     LIBCMT:typinfo.obj
 0002:00039e60       ??_R2type_info@@8          1013ce60     LIBCMT:typinfo.obj
 0002:00039e68       ??_R1A@?0A@EA@type_info@@8 1013ce68     LIBCMT:typinfo.obj
 0002:00039e84       ??_R4exception@std@@6B@    1013ce84     LIBCMT:stdexcpt.obj
 0002:00039e98       ??_R4bad_cast@std@@6B@     1013ce98     LIBCMT:stdexcpt.obj
 0002:00039eac       ??_R3bad_cast@std@@8       1013ceac     LIBCMT:stdexcpt.obj
 0002:00039ebc       ??_R2bad_cast@std@@8       1013cebc     LIBCMT:stdexcpt.obj
 0002:00039ec8       ??_R1A@?0A@EA@bad_cast@std@@8 1013cec8     LIBCMT:stdexcpt.obj
 0002:00039ee4       ??_R4bad_typeid@std@@6B@   1013cee4     LIBCMT:stdexcpt.obj
 0002:00039ef8       ??_R3bad_typeid@std@@8     1013cef8     LIBCMT:stdexcpt.obj
 0002:00039f08       ??_R2bad_typeid@std@@8     1013cf08     LIBCMT:stdexcpt.obj
 0002:00039f14       ??_R1A@?0A@EA@bad_typeid@std@@8 1013cf14     LIBCMT:stdexcpt.obj
 0002:00039f30       ??_R4__non_rtti_object@std@@6B@ 1013cf30     LIBCMT:stdexcpt.obj
 0002:00039f44       ??_R3__non_rtti_object@std@@8 1013cf44     LIBCMT:stdexcpt.obj
 0002:00039f54       ??_R2__non_rtti_object@std@@8 1013cf54     LIBCMT:stdexcpt.obj
 0002:00039f64       ??_R1A@?0A@EA@__non_rtti_object@std@@8 1013cf64     LIBCMT:stdexcpt.obj
 0002:00039f80       ??_R4bad_exception@std@@6B@ 1013cf80     LIBCMT:frame.obj
 0002:00039f94       ??_R3bad_exception@std@@8  1013cf94     LIBCMT:frame.obj
 0002:00039fa4       ??_R2bad_exception@std@@8  1013cfa4     LIBCMT:frame.obj
 0002:00039fb0       ??_R1A@?0A@EA@bad_exception@std@@8 1013cfb0     LIBCMT:frame.obj
 0002:00039fcc       ??_R4DNameNode@@6B@        1013cfcc     LIBCMT:undname.obj
 0002:00039fe0       ??_R3DNameNode@@8          1013cfe0     LIBCMT:undname.obj
 0002:00039ff0       ??_R2DNameNode@@8          1013cff0     LIBCMT:undname.obj
 0002:00039ff8       ??_R1A@?0A@EA@DNameNode@@8 1013cff8     LIBCMT:undname.obj
 0002:0003a014       ??_R4charNode@@6B@         1013d014     LIBCMT:undname.obj
 0002:0003a028       ??_R3charNode@@8           1013d028     LIBCMT:undname.obj
 0002:0003a038       ??_R2charNode@@8           1013d038     LIBCMT:undname.obj
 0002:0003a044       ??_R1A@?0A@EA@charNode@@8  1013d044     LIBCMT:undname.obj
 0002:0003a060       ??_R4pcharNode@@6B@        1013d060     LIBCMT:undname.obj
 0002:0003a074       ??_R3pcharNode@@8          1013d074     LIBCMT:undname.obj
 0002:0003a084       ??_R2pcharNode@@8          1013d084     LIBCMT:undname.obj
 0002:0003a090       ??_R1A@?0A@EA@pcharNode@@8 1013d090     LIBCMT:undname.obj
 0002:0003a0ac       ??_R4pDNameNode@@6B@       1013d0ac     LIBCMT:undname.obj
 0002:0003a0c0       ??_R3pDNameNode@@8         1013d0c0     LIBCMT:undname.obj
 0002:0003a0d0       ??_R2pDNameNode@@8         1013d0d0     LIBCMT:undname.obj
 0002:0003a0dc       ??_R1A@?0A@EA@pDNameNode@@8 1013d0dc     LIBCMT:undname.obj
 0002:0003a0f8       ??_R4DNameStatusNode@@6B@  1013d0f8     LIBCMT:undname.obj
 0002:0003a10c       ??_R3DNameStatusNode@@8    1013d10c     LIBCMT:undname.obj
 0002:0003a11c       ??_R2DNameStatusNode@@8    1013d11c     LIBCMT:undname.obj
 0002:0003a128       ??_R1A@?0A@EA@DNameStatusNode@@8 1013d128     LIBCMT:undname.obj
 0002:0003a144       ??_R4pairNode@@6B@         1013d144     LIBCMT:undname.obj
 0002:0003a158       ??_R3pairNode@@8           1013d158     LIBCMT:undname.obj
 0002:0003a168       ??_R2pairNode@@8           1013d168     LIBCMT:undname.obj
 0002:0003a174       ??_R1A@?0A@EA@pairNode@@8  1013d174     LIBCMT:undname.obj
 0002:0003a190       ??_R4length_error@std@@6B@ 1013d190     libcpmt:xthrow.obj
 0002:0003a1a4       ??_R3length_error@std@@8   1013d1a4     libcpmt:xthrow.obj
 0002:0003a1b4       ??_R2length_error@std@@8   1013d1b4     libcpmt:xthrow.obj
 0002:0003a1c4       ??_R1A@?0A@EA@length_error@std@@8 1013d1c4     libcpmt:xthrow.obj
 0002:0003a1e0       ??_R4out_of_range@std@@6B@ 1013d1e0     libcpmt:xthrow.obj
 0002:0003a1f4       ??_R3out_of_range@std@@8   1013d1f4     libcpmt:xthrow.obj
 0002:0003a204       ??_R2out_of_range@std@@8   1013d204     libcpmt:xthrow.obj
 0002:0003a214       ??_R1A@?0A@EA@out_of_range@std@@8 1013d214     libcpmt:xthrow.obj
 0002:0003a230       ??_R4overflow_error@std@@6B@ 1013d230     libcpmt:xthrow.obj
 0002:0003a244       ??_R3overflow_error@std@@8 1013d244     libcpmt:xthrow.obj
 0002:0003a254       ??_R2overflow_error@std@@8 1013d254     libcpmt:xthrow.obj
 0002:0003a264       ??_R1A@?0A@EA@overflow_error@std@@8 1013d264     libcpmt:xthrow.obj
 0002:0003a280       ??_R4bad_function_call@std@@6B@ 1013d280     libcpmt:xthrow.obj
 0002:0003a294       ??_R3bad_function_call@std@@8 1013d294     libcpmt:xthrow.obj
 0002:0003a2a4       ??_R2bad_function_call@std@@8 1013d2a4     libcpmt:xthrow.obj
 0002:0003a2b0       ??_R1A@?0A@EA@bad_function_call@std@@8 1013d2b0     libcpmt:xthrow.obj
 0002:0003a2cc       ??_R4regex_error@std@@6B@  1013d2cc     libcpmt:xthrow.obj
 0002:0003a2e0       ??_R3regex_error@std@@8    1013d2e0     libcpmt:xthrow.obj
 0002:0003a2f0       ??_R2regex_error@std@@8    1013d2f0     libcpmt:xthrow.obj
 0002:0003a300       ??_R1A@?0A@EA@regex_error@std@@8 1013d300     libcpmt:xthrow.obj
 0002:0003a31c       ??_R4_Locimp@locale@std@@6B@ 1013d31c     libcpmt:locale0.obj
 0002:0003a330       ??_R3_Locimp@locale@std@@8 1013d330     libcpmt:locale0.obj
 0002:0003a340       ??_R2_Locimp@locale@std@@8 1013d340     libcpmt:locale0.obj
 0002:0003a350       ??_R1A@?0A@EA@_Locimp@locale@std@@8 1013d350     libcpmt:locale0.obj
 0002:0003a36c       ??_R4?$num_get@DV?$istreambuf_iterator@DU?$char_traits@D@std@@@std@@@std@@6B@ 1013d36c     libcpmt:locale.obj
 0002:0003a380       ??_R3?$num_get@DV?$istreambuf_iterator@DU?$char_traits@D@std@@@std@@@std@@8 1013d380     libcpmt:locale.obj
 0002:0003a390       ??_R2?$num_get@DV?$istreambuf_iterator@DU?$char_traits@D@std@@@std@@@std@@8 1013d390     libcpmt:locale.obj
 0002:0003a3a0       ??_R1A@?0A@EA@?$num_get@DV?$istreambuf_iterator@DU?$char_traits@D@std@@@std@@@std@@8 1013d3a0     libcpmt:locale.obj
 0002:0003a3bc       ??_R4?$num_put@DV?$ostreambuf_iterator@DU?$char_traits@D@std@@@std@@@std@@6B@ 1013d3bc     libcpmt:locale.obj
 0002:0003a3d0       ??_R3?$num_put@DV?$ostreambuf_iterator@DU?$char_traits@D@std@@@std@@@std@@8 1013d3d0     libcpmt:locale.obj
 0002:0003a3e0       ??_R2?$num_put@DV?$ostreambuf_iterator@DU?$char_traits@D@std@@@std@@@std@@8 1013d3e0     libcpmt:locale.obj
 0002:0003a3f0       ??_R1A@?0A@EA@?$num_put@DV?$ostreambuf_iterator@DU?$char_traits@D@std@@@std@@@std@@8 1013d3f0     libcpmt:locale.obj
 0002:0003a40c       ??_R4?$numpunct@D@std@@6B@ 1013d40c     libcpmt:locale.obj
 0002:0003a420       ??_R3?$numpunct@D@std@@8   1013d420     libcpmt:locale.obj
 0002:0003a430       ??_R2?$numpunct@D@std@@8   1013d430     libcpmt:locale.obj
 0002:0003a440       ??_R1A@?0A@EA@?$numpunct@D@std@@8 1013d440     libcpmt:locale.obj
 0002:0003a45c       ??_R4?$codecvt@_WDH@std@@6B@ 1013d45c     libcpmt:wlocale.obj
 0002:0003a470       ??_R3?$codecvt@_WDH@std@@8 1013d470     libcpmt:wlocale.obj
 0002:0003a480       ??_R2?$codecvt@_WDH@std@@8 1013d480     libcpmt:wlocale.obj
 0002:0003a494       ??_R1A@?0A@EA@?$codecvt@_WDH@std@@8 1013d494     libcpmt:wlocale.obj
 0002:0003a4b0       ??_R4?$codecvt@GDH@std@@6B@ 1013d4b0     libcpmt:wlocale.obj
 0002:0003a4c4       ??_R3?$codecvt@GDH@std@@8  1013d4c4     libcpmt:wlocale.obj
 0002:0003a4d4       ??_R2?$codecvt@GDH@std@@8  1013d4d4     libcpmt:wlocale.obj
 0002:0003a4e8       ??_R1A@?0A@EA@?$codecvt@GDH@std@@8 1013d4e8     libcpmt:wlocale.obj
 0002:0003a504       ??_R4?$ctype@_W@std@@6B@   1013d504     libcpmt:wlocale.obj
 0002:0003a518       ??_R3?$ctype@_W@std@@8     1013d518     libcpmt:wlocale.obj
 0002:0003a528       ??_R2?$ctype@_W@std@@8     1013d528     libcpmt:wlocale.obj
 0002:0003a53c       ??_R1A@?0A@EA@?$ctype@_W@std@@8 1013d53c     libcpmt:wlocale.obj
 0002:0003a558       ??_R4?$ctype@G@std@@6B@    1013d558     libcpmt:wlocale.obj
 0002:0003a56c       ??_R3?$ctype@G@std@@8      1013d56c     libcpmt:wlocale.obj
 0002:0003a57c       ??_R2?$ctype@G@std@@8      1013d57c     libcpmt:wlocale.obj
 0002:0003a590       ??_R1A@?0A@EA@?$ctype@G@std@@8 1013d590     libcpmt:wlocale.obj
 0002:0003a5ac       ??_R4?$num_get@_WV?$istreambuf_iterator@_WU?$char_traits@_W@std@@@std@@@std@@6B@ 1013d5ac     libcpmt:wlocale.obj
 0002:0003a5c0       ??_R3?$num_get@_WV?$istreambuf_iterator@_WU?$char_traits@_W@std@@@std@@@std@@8 1013d5c0     libcpmt:wlocale.obj
 0002:0003a5d0       ??_R2?$num_get@_WV?$istreambuf_iterator@_WU?$char_traits@_W@std@@@std@@@std@@8 1013d5d0     libcpmt:wlocale.obj
 0002:0003a5e0       ??_R1A@?0A@EA@?$num_get@_WV?$istreambuf_iterator@_WU?$char_traits@_W@std@@@std@@@std@@8 1013d5e0     libcpmt:wlocale.obj
 0002:0003a5fc       ??_R4?$num_get@GV?$istreambuf_iterator@GU?$char_traits@G@std@@@std@@@std@@6B@ 1013d5fc     libcpmt:wlocale.obj
 0002:0003a610       ??_R3?$num_get@GV?$istreambuf_iterator@GU?$char_traits@G@std@@@std@@@std@@8 1013d610     libcpmt:wlocale.obj
 0002:0003a620       ??_R2?$num_get@GV?$istreambuf_iterator@GU?$char_traits@G@std@@@std@@@std@@8 1013d620     libcpmt:wlocale.obj
 0002:0003a630       ??_R1A@?0A@EA@?$num_get@GV?$istreambuf_iterator@GU?$char_traits@G@std@@@std@@@std@@8 1013d630     libcpmt:wlocale.obj
 0002:0003a64c       ??_R4?$numpunct@_W@std@@6B@ 1013d64c     libcpmt:wlocale.obj
 0002:0003a660       ??_R3?$numpunct@_W@std@@8  1013d660     libcpmt:wlocale.obj
 0002:0003a670       ??_R2?$numpunct@_W@std@@8  1013d670     libcpmt:wlocale.obj
 0002:0003a680       ??_R1A@?0A@EA@?$numpunct@_W@std@@8 1013d680     libcpmt:wlocale.obj
 0002:0003a69c       ??_R4messages_base@std@@6B@ 1013d69c     libcpmt:wlocale.obj
 0002:0003a6b0       ??_R3messages_base@std@@8  1013d6b0     libcpmt:wlocale.obj
 0002:0003a6c0       ??_R2messages_base@std@@8  1013d6c0     libcpmt:wlocale.obj
 0002:0003a6d0       ??_R1A@?0A@EA@messages_base@std@@8 1013d6d0     libcpmt:wlocale.obj
 0002:0003a6ec       ??_R4money_base@std@@6B@   1013d6ec     libcpmt:wlocale.obj
 0002:0003a700       ??_R3money_base@std@@8     1013d700     libcpmt:wlocale.obj
 0002:0003a710       ??_R2money_base@std@@8     1013d710     libcpmt:wlocale.obj
 0002:0003a720       ??_R1A@?0A@EA@money_base@std@@8 1013d720     libcpmt:wlocale.obj
 0002:0003a73c       ??_R4time_base@std@@6B@    1013d73c     libcpmt:wlocale.obj
 0002:0003a750       ??_R3time_base@std@@8      1013d750     libcpmt:wlocale.obj
 0002:0003a760       ??_R2time_base@std@@8      1013d760     libcpmt:wlocale.obj
 0002:0003a770       ??_R1A@?0A@EA@time_base@std@@8 1013d770     libcpmt:wlocale.obj
 0002:0003a78c       ??_R4?$num_put@_WV?$ostreambuf_iterator@_WU?$char_traits@_W@std@@@std@@@std@@6B@ 1013d78c     libcpmt:wlocale.obj
 0002:0003a7a0       ??_R3?$num_put@_WV?$ostreambuf_iterator@_WU?$char_traits@_W@std@@@std@@@std@@8 1013d7a0     libcpmt:wlocale.obj
 0002:0003a7b0       ??_R2?$num_put@_WV?$ostreambuf_iterator@_WU?$char_traits@_W@std@@@std@@@std@@8 1013d7b0     libcpmt:wlocale.obj
 0002:0003a7c0       ??_R1A@?0A@EA@?$num_put@_WV?$ostreambuf_iterator@_WU?$char_traits@_W@std@@@std@@@std@@8 1013d7c0     libcpmt:wlocale.obj
 0002:0003a7dc       ??_R4?$collate@_W@std@@6B@ 1013d7dc     libcpmt:wlocale.obj
 0002:0003a7f0       ??_R3?$collate@_W@std@@8   1013d7f0     libcpmt:wlocale.obj
 0002:0003a800       ??_R2?$collate@_W@std@@8   1013d800     libcpmt:wlocale.obj
 0002:0003a810       ??_R1A@?0A@EA@?$collate@_W@std@@8 1013d810     libcpmt:wlocale.obj
 0002:0003a82c       ??_R4?$messages@_W@std@@6B@ 1013d82c     libcpmt:wlocale.obj
 0002:0003a840       ??_R3?$messages@_W@std@@8  1013d840     libcpmt:wlocale.obj
 0002:0003a850       ??_R2?$messages@_W@std@@8  1013d850     libcpmt:wlocale.obj
 0002:0003a864       ??_R1A@?0A@EA@?$messages@_W@std@@8 1013d864     libcpmt:wlocale.obj
 0002:0003a880       ??_R4?$money_get@_WV?$istreambuf_iterator@_WU?$char_traits@_W@std@@@std@@@std@@6B@ 1013d880     libcpmt:wlocale.obj
 0002:0003a894       ??_R3?$money_get@_WV?$istreambuf_iterator@_WU?$char_traits@_W@std@@@std@@@std@@8 1013d894     libcpmt:wlocale.obj
 0002:0003a8a4       ??_R2?$money_get@_WV?$istreambuf_iterator@_WU?$char_traits@_W@std@@@std@@@std@@8 1013d8a4     libcpmt:wlocale.obj
 0002:0003a8b4       ??_R1A@?0A@EA@?$money_get@_WV?$istreambuf_iterator@_WU?$char_traits@_W@std@@@std@@@std@@8 1013d8b4     libcpmt:wlocale.obj
 0002:0003a8d0       ??_R4?$money_put@_WV?$ostreambuf_iterator@_WU?$char_traits@_W@std@@@std@@@std@@6B@ 1013d8d0     libcpmt:wlocale.obj
 0002:0003a8e4       ??_R3?$money_put@_WV?$ostreambuf_iterator@_WU?$char_traits@_W@std@@@std@@@std@@8 1013d8e4     libcpmt:wlocale.obj
 0002:0003a8f4       ??_R2?$money_put@_WV?$ostreambuf_iterator@_WU?$char_traits@_W@std@@@std@@@std@@8 1013d8f4     libcpmt:wlocale.obj
 0002:0003a904       ??_R1A@?0A@EA@?$money_put@_WV?$ostreambuf_iterator@_WU?$char_traits@_W@std@@@std@@@std@@8 1013d904     libcpmt:wlocale.obj
 0002:0003a920       ??_R4?$moneypunct@_W$0A@@std@@6B@ 1013d920     libcpmt:wlocale.obj
 0002:0003a934       ??_R3?$moneypunct@_W$0A@@std@@8 1013d934     libcpmt:wlocale.obj
 0002:0003a944       ??_R2?$moneypunct@_W$0A@@std@@8 1013d944     libcpmt:wlocale.obj
 0002:0003a95c       ??_R1A@?0A@EA@?$moneypunct@_W$0A@@std@@8 1013d95c     libcpmt:wlocale.obj
 0002:0003a978       ??_R1A@?0A@EA@?$_Mpunct@_W@std@@8 1013d978     libcpmt:wlocale.obj
 0002:0003a994       ??_R3?$_Mpunct@_W@std@@8   1013d994     libcpmt:wlocale.obj
 0002:0003a9a4       ??_R2?$_Mpunct@_W@std@@8   1013d9a4     libcpmt:wlocale.obj
 0002:0003a9b8       ??_R4?$moneypunct@_W$00@std@@6B@ 1013d9b8     libcpmt:wlocale.obj
 0002:0003a9cc       ??_R3?$moneypunct@_W$00@std@@8 1013d9cc     libcpmt:wlocale.obj
 0002:0003a9dc       ??_R2?$moneypunct@_W$00@std@@8 1013d9dc     libcpmt:wlocale.obj
 0002:0003a9f4       ??_R1A@?0A@EA@?$moneypunct@_W$00@std@@8 1013d9f4     libcpmt:wlocale.obj
 0002:0003aa10       ??_R4?$time_get@_WV?$istreambuf_iterator@_WU?$char_traits@_W@std@@@std@@@std@@6B@ 1013da10     libcpmt:wlocale.obj
 0002:0003aa24       ??_R3?$time_get@_WV?$istreambuf_iterator@_WU?$char_traits@_W@std@@@std@@@std@@8 1013da24     libcpmt:wlocale.obj
 0002:0003aa34       ??_R2?$time_get@_WV?$istreambuf_iterator@_WU?$char_traits@_W@std@@@std@@@std@@8 1013da34     libcpmt:wlocale.obj
 0002:0003aa48       ??_R1A@?0A@EA@?$time_get@_WV?$istreambuf_iterator@_WU?$char_traits@_W@std@@@std@@@std@@8 1013da48     libcpmt:wlocale.obj
 0002:0003aa64       ??_R4?$time_put@_WV?$ostreambuf_iterator@_WU?$char_traits@_W@std@@@std@@@std@@6B@ 1013da64     libcpmt:wlocale.obj
 0002:0003aa78       ??_R3?$time_put@_WV?$ostreambuf_iterator@_WU?$char_traits@_W@std@@@std@@@std@@8 1013da78     libcpmt:wlocale.obj
 0002:0003aa88       ??_R2?$time_put@_WV?$ostreambuf_iterator@_WU?$char_traits@_W@std@@@std@@@std@@8 1013da88     libcpmt:wlocale.obj
 0002:0003aa98       ??_R1A@?0A@EA@?$time_put@_WV?$ostreambuf_iterator@_WU?$char_traits@_W@std@@@std@@@std@@8 1013da98     libcpmt:wlocale.obj
 0002:0003aab4       ??_R4?$_Mpunct@_W@std@@6B@ 1013dab4     libcpmt:wlocale.obj
 0002:0003aac8       ??_R4?$num_put@GV?$ostreambuf_iterator@GU?$char_traits@G@std@@@std@@@std@@6B@ 1013dac8     libcpmt:wlocale.obj
 0002:0003aadc       ??_R3?$num_put@GV?$ostreambuf_iterator@GU?$char_traits@G@std@@@std@@@std@@8 1013dadc     libcpmt:wlocale.obj
 0002:0003aaec       ??_R2?$num_put@GV?$ostreambuf_iterator@GU?$char_traits@G@std@@@std@@@std@@8 1013daec     libcpmt:wlocale.obj
 0002:0003aafc       ??_R1A@?0A@EA@?$num_put@GV?$ostreambuf_iterator@GU?$char_traits@G@std@@@std@@@std@@8 1013dafc     libcpmt:wlocale.obj
 0002:0003ab18       ??_R4?$numpunct@G@std@@6B@ 1013db18     libcpmt:wlocale.obj
 0002:0003ab2c       ??_R3?$numpunct@G@std@@8   1013db2c     libcpmt:wlocale.obj
 0002:0003ab3c       ??_R2?$numpunct@G@std@@8   1013db3c     libcpmt:wlocale.obj
 0002:0003ab4c       ??_R1A@?0A@EA@?$numpunct@G@std@@8 1013db4c     libcpmt:wlocale.obj
 0002:0003ab68       ??_R4?$collate@G@std@@6B@  1013db68     libcpmt:wlocale.obj
 0002:0003ab7c       ??_R3?$collate@G@std@@8    1013db7c     libcpmt:wlocale.obj
 0002:0003ab8c       ??_R2?$collate@G@std@@8    1013db8c     libcpmt:wlocale.obj
 0002:0003ab9c       ??_R1A@?0A@EA@?$collate@G@std@@8 1013db9c     libcpmt:wlocale.obj
 0002:0003abb8       ??_R4?$messages@G@std@@6B@ 1013dbb8     libcpmt:wlocale.obj
 0002:0003abcc       ??_R3?$messages@G@std@@8   1013dbcc     libcpmt:wlocale.obj
 0002:0003abdc       ??_R2?$messages@G@std@@8   1013dbdc     libcpmt:wlocale.obj
 0002:0003abf0       ??_R1A@?0A@EA@?$messages@G@std@@8 1013dbf0     libcpmt:wlocale.obj
 0002:0003ac0c       ??_R4?$money_get@GV?$istreambuf_iterator@GU?$char_traits@G@std@@@std@@@std@@6B@ 1013dc0c     libcpmt:wlocale.obj
 0002:0003ac20       ??_R3?$money_get@GV?$istreambuf_iterator@GU?$char_traits@G@std@@@std@@@std@@8 1013dc20     libcpmt:wlocale.obj
 0002:0003ac30       ??_R2?$money_get@GV?$istreambuf_iterator@GU?$char_traits@G@std@@@std@@@std@@8 1013dc30     libcpmt:wlocale.obj
 0002:0003ac40       ??_R1A@?0A@EA@?$money_get@GV?$istreambuf_iterator@GU?$char_traits@G@std@@@std@@@std@@8 1013dc40     libcpmt:wlocale.obj
 0002:0003ac5c       ??_R4?$money_put@GV?$ostreambuf_iterator@GU?$char_traits@G@std@@@std@@@std@@6B@ 1013dc5c     libcpmt:wlocale.obj
 0002:0003ac70       ??_R3?$money_put@GV?$ostreambuf_iterator@GU?$char_traits@G@std@@@std@@@std@@8 1013dc70     libcpmt:wlocale.obj
 0002:0003ac80       ??_R2?$money_put@GV?$ostreambuf_iterator@GU?$char_traits@G@std@@@std@@@std@@8 1013dc80     libcpmt:wlocale.obj
 0002:0003ac90       ??_R1A@?0A@EA@?$money_put@GV?$ostreambuf_iterator@GU?$char_traits@G@std@@@std@@@std@@8 1013dc90     libcpmt:wlocale.obj
 0002:0003acac       ??_R4?$moneypunct@G$0A@@std@@6B@ 1013dcac     libcpmt:wlocale.obj
 0002:0003acc0       ??_R3?$moneypunct@G$0A@@std@@8 1013dcc0     libcpmt:wlocale.obj
 0002:0003acd0       ??_R2?$moneypunct@G$0A@@std@@8 1013dcd0     libcpmt:wlocale.obj
 0002:0003ace8       ??_R1A@?0A@EA@?$moneypunct@G$0A@@std@@8 1013dce8     libcpmt:wlocale.obj
 0002:0003ad04       ??_R1A@?0A@EA@?$_Mpunct@G@std@@8 1013dd04     libcpmt:wlocale.obj
 0002:0003ad20       ??_R3?$_Mpunct@G@std@@8    1013dd20     libcpmt:wlocale.obj
 0002:0003ad30       ??_R2?$_Mpunct@G@std@@8    1013dd30     libcpmt:wlocale.obj
 0002:0003ad44       ??_R4?$moneypunct@G$00@std@@6B@ 1013dd44     libcpmt:wlocale.obj
 0002:0003ad58       ??_R3?$moneypunct@G$00@std@@8 1013dd58     libcpmt:wlocale.obj
 0002:0003ad68       ??_R2?$moneypunct@G$00@std@@8 1013dd68     libcpmt:wlocale.obj
 0002:0003ad80       ??_R1A@?0A@EA@?$moneypunct@G$00@std@@8 1013dd80     libcpmt:wlocale.obj
 0002:0003ad9c       ??_R4?$time_get@GV?$istreambuf_iterator@GU?$char_traits@G@std@@@std@@@std@@6B@ 1013dd9c     libcpmt:wlocale.obj
 0002:0003adb0       ??_R3?$time_get@GV?$istreambuf_iterator@GU?$char_traits@G@std@@@std@@@std@@8 1013ddb0     libcpmt:wlocale.obj
 0002:0003adc0       ??_R2?$time_get@GV?$istreambuf_iterator@GU?$char_traits@G@std@@@std@@@std@@8 1013ddc0     libcpmt:wlocale.obj
 0002:0003add4       ??_R1A@?0A@EA@?$time_get@GV?$istreambuf_iterator@GU?$char_traits@G@std@@@std@@@std@@8 1013ddd4     libcpmt:wlocale.obj
 0002:0003adf0       ??_R4?$time_put@GV?$ostreambuf_iterator@GU?$char_traits@G@std@@@std@@@std@@6B@ 1013ddf0     libcpmt:wlocale.obj
 0002:0003ae04       ??_R3?$time_put@GV?$ostreambuf_iterator@GU?$char_traits@G@std@@@std@@@std@@8 1013de04     libcpmt:wlocale.obj
 0002:0003ae14       ??_R2?$time_put@GV?$ostreambuf_iterator@GU?$char_traits@G@std@@@std@@@std@@8 1013de14     libcpmt:wlocale.obj
 0002:0003ae24       ??_R1A@?0A@EA@?$time_put@GV?$ostreambuf_iterator@GU?$char_traits@G@std@@@std@@@std@@8 1013de24     libcpmt:wlocale.obj
 0002:0003ae40       ??_R4?$_Mpunct@G@std@@6B@  1013de40     libcpmt:wlocale.obj
 0002:0003ae54       ??_R4?$collate@D@std@@6B@  1013de54     libcpmt:xlocale.obj
 0002:0003ae68       ??_R3?$collate@D@std@@8    1013de68     libcpmt:xlocale.obj
 0002:0003ae78       ??_R2?$collate@D@std@@8    1013de78     libcpmt:xlocale.obj
 0002:0003ae88       ??_R1A@?0A@EA@?$collate@D@std@@8 1013de88     libcpmt:xlocale.obj
 0002:0003aea4       ??_R4?$messages@D@std@@6B@ 1013dea4     libcpmt:xlocale.obj
 0002:0003aeb8       ??_R3?$messages@D@std@@8   1013deb8     libcpmt:xlocale.obj
 0002:0003aec8       ??_R2?$messages@D@std@@8   1013dec8     libcpmt:xlocale.obj
 0002:0003aedc       ??_R1A@?0A@EA@?$messages@D@std@@8 1013dedc     libcpmt:xlocale.obj
 0002:0003aef8       ??_R4?$money_get@DV?$istreambuf_iterator@DU?$char_traits@D@std@@@std@@@std@@6B@ 1013def8     libcpmt:xlocale.obj
 0002:0003af0c       ??_R3?$money_get@DV?$istreambuf_iterator@DU?$char_traits@D@std@@@std@@@std@@8 1013df0c     libcpmt:xlocale.obj
 0002:0003af1c       ??_R2?$money_get@DV?$istreambuf_iterator@DU?$char_traits@D@std@@@std@@@std@@8 1013df1c     libcpmt:xlocale.obj
 0002:0003af2c       ??_R1A@?0A@EA@?$money_get@DV?$istreambuf_iterator@DU?$char_traits@D@std@@@std@@@std@@8 1013df2c     libcpmt:xlocale.obj
 0002:0003af48       ??_R4?$money_put@DV?$ostreambuf_iterator@DU?$char_traits@D@std@@@std@@@std@@6B@ 1013df48     libcpmt:xlocale.obj
 0002:0003af5c       ??_R3?$money_put@DV?$ostreambuf_iterator@DU?$char_traits@D@std@@@std@@@std@@8 1013df5c     libcpmt:xlocale.obj
 0002:0003af6c       ??_R2?$money_put@DV?$ostreambuf_iterator@DU?$char_traits@D@std@@@std@@@std@@8 1013df6c     libcpmt:xlocale.obj
 0002:0003af7c       ??_R1A@?0A@EA@?$money_put@DV?$ostreambuf_iterator@DU?$char_traits@D@std@@@std@@@std@@8 1013df7c     libcpmt:xlocale.obj
 0002:0003af98       ??_R4?$moneypunct@D$0A@@std@@6B@ 1013df98     libcpmt:xlocale.obj
 0002:0003afac       ??_R3?$moneypunct@D$0A@@std@@8 1013dfac     libcpmt:xlocale.obj
 0002:0003afbc       ??_R2?$moneypunct@D$0A@@std@@8 1013dfbc     libcpmt:xlocale.obj
 0002:0003afd4       ??_R1A@?0A@EA@?$moneypunct@D$0A@@std@@8 1013dfd4     libcpmt:xlocale.obj
 0002:0003aff0       ??_R1A@?0A@EA@?$_Mpunct@D@std@@8 1013dff0     libcpmt:xlocale.obj
 0002:0003b00c       ??_R3?$_Mpunct@D@std@@8    1013e00c     libcpmt:xlocale.obj
 0002:0003b01c       ??_R2?$_Mpunct@D@std@@8    1013e01c     libcpmt:xlocale.obj
 0002:0003b030       ??_R4?$moneypunct@D$00@std@@6B@ 1013e030     libcpmt:xlocale.obj
 0002:0003b044       ??_R3?$moneypunct@D$00@std@@8 1013e044     libcpmt:xlocale.obj
 0002:0003b054       ??_R2?$moneypunct@D$00@std@@8 1013e054     libcpmt:xlocale.obj
 0002:0003b06c       ??_R1A@?0A@EA@?$moneypunct@D$00@std@@8 1013e06c     libcpmt:xlocale.obj
 0002:0003b088       ??_R4?$time_get@DV?$istreambuf_iterator@DU?$char_traits@D@std@@@std@@@std@@6B@ 1013e088     libcpmt:xlocale.obj
 0002:0003b09c       ??_R3?$time_get@DV?$istreambuf_iterator@DU?$char_traits@D@std@@@std@@@std@@8 1013e09c     libcpmt:xlocale.obj
 0002:0003b0ac       ??_R2?$time_get@DV?$istreambuf_iterator@DU?$char_traits@D@std@@@std@@@std@@8 1013e0ac     libcpmt:xlocale.obj
 0002:0003b0c0       ??_R1A@?0A@EA@?$time_get@DV?$istreambuf_iterator@DU?$char_traits@D@std@@@std@@@std@@8 1013e0c0     libcpmt:xlocale.obj
 0002:0003b0dc       ??_R4?$time_put@DV?$ostreambuf_iterator@DU?$char_traits@D@std@@@std@@@std@@6B@ 1013e0dc     libcpmt:xlocale.obj
 0002:0003b0f0       ??_R3?$time_put@DV?$ostreambuf_iterator@DU?$char_traits@D@std@@@std@@@std@@8 1013e0f0     libcpmt:xlocale.obj
 0002:0003b100       ??_R2?$time_put@DV?$ostreambuf_iterator@DU?$char_traits@D@std@@@std@@@std@@8 1013e100     libcpmt:xlocale.obj
 0002:0003b110       ??_R1A@?0A@EA@?$time_put@DV?$ostreambuf_iterator@DU?$char_traits@D@std@@@std@@@std@@8 1013e110     libcpmt:xlocale.obj
 0002:0003b12c       ??_R4?$_Mpunct@D@std@@6B@  1013e12c     libcpmt:xlocale.obj
 0002:0003b7e0       ___safe_se_handler_table   1013e7e0     <linker-defined>
 0002:0003bda0       ___rtc_iaa                 1013eda0     LIBCMT:initsect.obj
 0002:0003bea4       ___rtc_izz                 1013eea4     LIBCMT:initsect.obj
 0002:0003bfa8       ___rtc_taa                 1013efa8     LIBCMT:initsect.obj
 0002:0003c0ac       ___rtc_tzz                 1013f0ac     LIBCMT:initsect.obj
 0002:0003c768       __TI2?AVruntime_error@std@@ 1013f768     IO61X_Library_MSVC120_vc:IO61X_DriverObject.obj
 0002:0003c778       __CTA2?AVruntime_error@std@@ 1013f778     IO61X_Library_MSVC120_vc:IO61X_DriverObject.obj
 0002:0003c784       __CT??_R0?AVruntime_error@std@@@8??0runtime_error@std@@QAE@ABV01@@Z12 1013f784     IO61X_Library_MSVC120_vc:IO61X_DriverObject.obj
 0002:0003c7a0       __CT??_R0?AVexception@std@@@8??0exception@std@@QAE@ABV01@@Z12 1013f7a0     IO61X_Library_MSVC120_vc:IO61X_DriverObject.obj
 0002:0003c7bc       __TI5?AVfailure@ios_base@std@@ 1013f7bc     IO61X_Library_MSVC120_vc:IO61X_DriverObject.obj
 0002:0003c7cc       __CTA5?AVfailure@ios_base@std@@ 1013f7cc     IO61X_Library_MSVC120_vc:IO61X_DriverObject.obj
 0002:0003c7e4       __CT??_R0?AVfailure@ios_base@std@@@8??0failure@ios_base@std@@QAE@ABV012@@Z20 1013f7e4     IO61X_Library_MSVC120_vc:IO61X_DriverObject.obj
 0002:0003c800       __CT??_R0?AVsystem_error@std@@@8??0system_error@std@@QAE@ABV01@@Z20 1013f800     IO61X_Library_MSVC120_vc:IO61X_DriverObject.obj
 0002:0003c81c       __CT??_R0?AV_System_error@std@@@8??0_System_error@std@@QAE@ABV01@@Z20 1013f81c     IO61X_Library_MSVC120_vc:IO61X_DriverObject.obj
 0002:0003c838       __TI3?AVinvalid_argument@std@@ 1013f838     IO61X_Library_MSVC120_vc:IO61X_DriverObject.obj
 0002:0003c848       __CTA3?AVinvalid_argument@std@@ 1013f848     IO61X_Library_MSVC120_vc:IO61X_DriverObject.obj
 0002:0003c858       __CT??_R0?AVinvalid_argument@std@@@8??0invalid_argument@std@@QAE@ABV01@@Z12 1013f858     IO61X_Library_MSVC120_vc:IO61X_DriverObject.obj
 0002:0003c874       __CT??_R0?AVlogic_error@std@@@8??0logic_error@std@@QAE@ABV01@@Z12 1013f874     IO61X_Library_MSVC120_vc:IO61X_DriverObject.obj
 0002:0003c890       __TI2?AVbad_cast@std@@     1013f890     IO61X_Library_MSVC120_vc:IO61X_DriverObject.obj
 0002:0003c8a0       __CTA2?AVbad_cast@std@@    1013f8a0     IO61X_Library_MSVC120_vc:IO61X_DriverObject.obj
 0002:0003c8ac       __CT??_R0?AVbad_cast@std@@@8??0bad_cast@std@@QAE@ABV01@@Z12 1013f8ac     IO61X_Library_MSVC120_vc:IO61X_DriverObject.obj
 0002:0003cf74       __TI2?AVbad_alloc@std@@    1013ff74     LIBCMT:new.obj
 0002:0003cf84       __CTA2?AVbad_alloc@std@@   1013ff84     LIBCMT:new.obj
 0002:0003cf90       __CT??_R0?AVbad_alloc@std@@@8??0bad_alloc@std@@QAE@ABV01@@Z12 1013ff90     LIBCMT:new.obj
 0002:0003d4cc       __TI2?AVbad_exception@std@@ 101404cc     LIBCMT:frame.obj
 0002:0003d4dc       __CTA2?AVbad_exception@std@@ 101404dc     LIBCMT:frame.obj
 0002:0003d4e8       __CT??_R0?AVbad_exception@std@@@8??0bad_exception@std@@QAE@ABV01@@Z12 101404e8     LIBCMT:frame.obj
 0002:0003d894       __TI3?AVlength_error@std@@ 10140894     libcpmt:xthrow.obj
 0002:0003d8a4       __CTA3?AVlength_error@std@@ 101408a4     libcpmt:xthrow.obj
 0002:0003d8b4       __CT??_R0?AVlength_error@std@@@8??0length_error@std@@QAE@ABV01@@Z12 101408b4     libcpmt:xthrow.obj
 0002:0003d8d0       __TI3?AVout_of_range@std@@ 101408d0     libcpmt:xthrow.obj
 0002:0003d8e0       __CTA3?AVout_of_range@std@@ 101408e0     libcpmt:xthrow.obj
 0002:0003d8f0       __CT??_R0?AVout_of_range@std@@@8??0out_of_range@std@@QAE@ABV01@@Z12 101408f0     libcpmt:xthrow.obj
 0002:0003d90c       __TI3?AVoverflow_error@std@@ 1014090c     libcpmt:xthrow.obj
 0002:0003d91c       __CTA3?AVoverflow_error@std@@ 1014091c     libcpmt:xthrow.obj
 0002:0003d92c       __CT??_R0?AVoverflow_error@std@@@8??0overflow_error@std@@QAE@ABV01@@Z12 1014092c     libcpmt:xthrow.obj
 0002:0003d948       __TI2?AVbad_function_call@std@@ 10140948     libcpmt:xthrow.obj
 0002:0003d958       __CTA2?AVbad_function_call@std@@ 10140958     libcpmt:xthrow.obj
 0002:0003d964       __CT??_R0?AVbad_function_call@std@@@8??0bad_function_call@std@@QAE@ABV01@@Z12 10140964     libcpmt:xthrow.obj
 0002:0003d980       __TI3?AVregex_error@std@@  10140980     libcpmt:xthrow.obj
 0002:0003d990       __CTA3?AVregex_error@std@@ 10140990     libcpmt:xthrow.obj
 0002:0003d9a0       __CT??_R0?AVregex_error@std@@@8??0regex_error@std@@QAE@ABV01@@Z16 101409a0     libcpmt:xthrow.obj
 0003:00000000       _pci20041digout            10145000     xpctarget.obj
 0003:00000004       _nipcdio24cnfg             10145004     xpctarget.obj
 0003:00000008       _rtddm6604cnfg             10145008     xpctarget.obj
 0003:00000408       _CANTest_P                 10145408     CANTest_data.obj
 0003:00000a28       _DefaultCOMIOBase          10145a28     xpcruntime:xpcimports.obj
 0003:00000a38       _DefaultCOMIRQ             10145a38     xpcruntime:xpcimports.obj
 0003:00000a48       ?_Generic_object@?$_Error_objects@H@std@@2V_Generic_error_category@2@A 10145a48     IO61X_Library_MSVC120_vc:IO61X_iConcurrentExecution.obj
 0003:00000a4c       ?_Iostream_object@?$_Error_objects@H@std@@2V_Iostream_error_category@2@A 10145a4c     IO61X_Library_MSVC120_vc:IO61X_iConcurrentExecution.obj
 0003:00000a50       ?_System_object@?$_Error_objects@H@std@@2V_System_error_category@2@A 10145a50     IO61X_Library_MSVC120_vc:IO61X_iConcurrentExecution.obj
 0003:00000a54       __fltused                  10145a54     LIBCMT:fpinit.obj
 0003:00000a58       __ldused                   10145a58     LIBCMT:fpinit.obj
 0003:00000a60       __iob                      10145a60     LIBCMT:_file.obj
 0003:00000ce0       ___isa_enabled             10145ce0     LIBCMT:cpu_disp.obj
 0003:00000ce4       ___security_cookie         10145ce4     LIBCMT:gs_cookie.obj
 0003:00000ce8       ___security_cookie_complement 10145ce8     LIBCMT:gs_cookie.obj
 0003:00000ec0       __cfltcvt_tab              10145ec0     LIBCMT:cmiscdat.obj
 0003:00001100       __mbctype                  10146100     LIBCMT:mbctype.obj
 0003:00001208       __mbcasemap                10146208     LIBCMT:mbctype.obj
 0003:00001308       ___initialmbcinfo          10146308     LIBCMT:mbctype.obj
 0003:0000152c       ___ptmbcinfo               1014652c     LIBCMT:mbctype.obj
 0003:00001620       ___nullstring              10146620     LIBCMT:output.obj
 0003:00001624       ___wnullstring             10146624     LIBCMT:output.obj
 0003:00001628       ___badioinfo               10146628     LIBCMT:ioinit.obj
 0003:00001668       __lookuptrailbytes         10146668     LIBCMT:read.obj
 0003:00001768       __d_inf                    10146768     LIBCMT:util.obj
 0003:00001770       __d_ind                    10146770     LIBCMT:util.obj
 0003:00001778       __d_max                    10146778     LIBCMT:util.obj
 0003:00001780       __d_min                    10146780     LIBCMT:util.obj
 0003:00001788       __d_mzero                  10146788     LIBCMT:util.obj
 0003:000017ac       ___abort_behavior          101467ac     LIBCMT:abort.obj
 0003:000017b0       ___flsindex                101467b0     LIBCMT:tidtable.obj
 0003:000017e0       ___mb_cur_max              101467e0     LIBCMT:nlsdata.obj
 0003:000017e4       ___wclocalestr             101467e4     LIBCMT:nlsdata.obj
 0003:000017e8       ___lc_time_c               101467e8     LIBCMT:nlsdata.obj
 0003:0000194c       ___ptlocinfo               1014694c     LIBCMT:nlsdata.obj
 0003:00001950       ___initiallocinfo          10146950     LIBCMT:nlsdata.obj
 0003:00001a08       ___initiallocalestructinfo 10146a08     LIBCMT:nlsdata.obj
 0003:00001a10       ___globallocalestatus      10146a10     LIBCMT:glstatus.obj
 0003:00001a14       __matherr_flag             10146a14     LIBCMT:matherr.obj
 0003:00001a20       __NLG_Destination          10146a20     LIBCMT:exsup.obj
 0003:00001a30       ___lconv                   10146a30     LIBCMT:lconv.obj
 0003:00001a34       ___lconv_static_decimal    10146a34     LIBCMT:lconv.obj
 0003:00001a38       ___lconv_c                 10146a38     LIBCMT:lconv.obj
 0003:00001a88       ___lconv_static_W_decimal  10146a88     LIBCMT:lconv.obj
 0003:00001ac0       __pctype                   10146ac0     LIBCMT:ctype.obj
 0003:00001ac4       __pwctype                  10146ac4     LIBCMT:ctype.obj
 0003:00001ad0       __confh                    10146ad0     LIBCMT:initcon.obj
 0003:00001ad8       __pow10pos                 10146ad8     LIBCMT:constpow.obj
 0003:00001c38       __pow10neg                 10146c38     LIBCMT:constpow.obj
 0003:00001da0       __HUGE                     10146da0     LIBCMT:huge.obj
 0003:00001dac       ?_Sync@ios_base@std@@0_NA  10146dac     libcpmt:ios.obj
 0003:00001db8       ?_PJP_CPP_Copyright@@3PADA 10146db8     libcpmt:iosptrs.obj
 0003:00001e18       __FDenorm                  10146e18     libcpmt:xfvalues.obj
 0003:00001e28       __FInf                     10146e28     libcpmt:xfvalues.obj
 0003:00001e38       __FNan                     10146e38     libcpmt:xfvalues.obj
 0003:00001e48       __FSnan                    10146e48     libcpmt:xfvalues.obj
 0003:00001e58       __FEps                     10146e58     libcpmt:xfvalues.obj
 0003:00001e68       __FRteps                   10146e68     libcpmt:xfvalues.obj
 0003:00001e78       __FXbig                    10146e78     libcpmt:xfvalues.obj
 0003:00001e80       __Denorm                   10146e80     libcpmt:xvalues.obj
 0003:00001e90       __Hugeval                  10146e90     libcpmt:xvalues.obj
 0003:00001ea0       __Inf                      10146ea0     libcpmt:xvalues.obj
 0003:00001eb0       __Nan                      10146eb0     libcpmt:xvalues.obj
 0003:00001ec0       __Snan                     10146ec0     libcpmt:xvalues.obj
 0003:00001ed0       __Eps                      10146ed0     libcpmt:xvalues.obj
 0003:00001ee0       __Rteps                    10146ee0     libcpmt:xvalues.obj
 0003:00001ef0       __Xbig                     10146ef0     libcpmt:xvalues.obj
 0003:00001ef8       __LDenorm                  10146ef8     libcpmt:xlvalues.obj
 0003:00001f08       __LInf                     10146f08     libcpmt:xlvalues.obj
 0003:00001f18       __LNan                     10146f18     libcpmt:xlvalues.obj
 0003:00001f28       __LSnan                    10146f28     libcpmt:xlvalues.obj
 0003:00001f38       __LEps                     10146f38     libcpmt:xlvalues.obj
 0003:00001f48       __LRteps                   10146f48     libcpmt:xlvalues.obj
 0003:00001f58       __LXbig                    10146f58     libcpmt:xlvalues.obj
 0003:00001f88       __timezone                 10146f88     LIBCMT:timeset.obj
 0003:00001f8c       __daylight                 10146f8c     LIBCMT:timeset.obj
 0003:00001f90       __dstbias                  10146f90     LIBCMT:timeset.obj
 0003:00002018       __tzname                   10147018     LIBCMT:timeset.obj
 0003:00002020       __half                     10147020     LIBCMT:pow.obj
 0003:0000202c       __days                     1014702c     LIBCMT:days.obj
 0003:00002060       __lpdays                   10147060     LIBCMT:days.obj
 0003:00002628       ??_R0?AVexception@std@@@8  10147628     IO61X_Library_MSVC120_vc:IO61X_iConcurrentExecution.obj
 0003:00002644       ??_R0?AVerror_category@std@@@8 10147644     IO61X_Library_MSVC120_vc:IO61X_iConcurrentExecution.obj
 0003:00002668       ??_R0?AV_Generic_error_category@std@@@8 10147668     IO61X_Library_MSVC120_vc:IO61X_iConcurrentExecution.obj
 0003:00002694       ??_R0?AV_Iostream_error_category@std@@@8 10147694     IO61X_Library_MSVC120_vc:IO61X_iConcurrentExecution.obj
 0003:000026c0       ??_R0?AV_System_error_category@std@@@8 101476c0     IO61X_Library_MSVC120_vc:IO61X_iConcurrentExecution.obj
 0003:000026ec       ??_R0?AVruntime_error@std@@@8 101476ec     IO61X_Library_MSVC120_vc:IO61X_DriverObject.obj
 0003:0000270c       ??_R0?AVfailure@ios_base@std@@@8 1014770c     IO61X_Library_MSVC120_vc:IO61X_DriverObject.obj
 0003:00002730       ??_R0?AVsystem_error@std@@@8 10147730     IO61X_Library_MSVC120_vc:IO61X_DriverObject.obj
 0003:00002750       ??_R0?AV_System_error@std@@@8 10147750     IO61X_Library_MSVC120_vc:IO61X_DriverObject.obj
 0003:00002770       ??_R0?AVinvalid_argument@std@@@8 10147770     IO61X_Library_MSVC120_vc:IO61X_DriverObject.obj
 0003:00002794       ??_R0?AVlogic_error@std@@@8 10147794     IO61X_Library_MSVC120_vc:IO61X_DriverObject.obj
 0003:000027b4       ??_R0?AVbad_cast@std@@@8   101477b4     IO61X_Library_MSVC120_vc:IO61X_DriverObject.obj
 0003:000027d0       ??_R0?AVios_base@std@@@8   101477d0     IO61X_Library_MSVC120_vc:IO61X_DriverObject.obj
 0003:000027ec       ??_R0?AV?$_Iosb@H@std@@@8  101477ec     IO61X_Library_MSVC120_vc:IO61X_DriverObject.obj
 0003:00002808       ??_R0?AV?$basic_ios@DU?$char_traits@D@std@@@std@@@8 10147808     IO61X_Library_MSVC120_vc:IO61X_DriverObject.obj
 0003:00002840       ??_R0?AV?$basic_streambuf@DU?$char_traits@D@std@@@std@@@8 10147840     IO61X_Library_MSVC120_vc:IO61X_DriverObject.obj
 0003:0000287c       ??_R0?AV?$basic_ostream@DU?$char_traits@D@std@@@std@@@8 1014787c     IO61X_Library_MSVC120_vc:IO61X_DriverObject.obj
 0003:000028b8       ??_R0?AV?$basic_filebuf@DU?$char_traits@D@std@@@std@@@8 101478b8     IO61X_Library_MSVC120_vc:IO61X_DriverObject.obj
 0003:000028f4       ??_R0?AV?$basic_ofstream@DU?$char_traits@D@std@@@std@@@8 101478f4     IO61X_Library_MSVC120_vc:IO61X_DriverObject.obj
 0003:00002930       ??_R0?AV_Facet_base@std@@@8 10147930     IO61X_Library_MSVC120_vc:IO61X_DriverObject.obj
 0003:00002950       ??_R0?AVfacet@locale@std@@@8 10147950     IO61X_Library_MSVC120_vc:IO61X_DriverObject.obj
 0003:00002970       ??_R0?AVcodecvt_base@std@@@8 10147970     IO61X_Library_MSVC120_vc:IO61X_DriverObject.obj
 0003:00002990       ??_R0?AUctype_base@std@@@8 10147990     IO61X_Library_MSVC120_vc:IO61X_DriverObject.obj
 0003:000029b0       ??_R0?AV?$ctype@D@std@@@8  101479b0     IO61X_Library_MSVC120_vc:IO61X_DriverObject.obj
 0003:000029cc       ??_R0?AV?$codecvt@DDH@std@@@8 101479cc     IO61X_Library_MSVC120_vc:IO61X_DriverObject.obj
 0003:000029ec       ??_R0?AVIO61X_Port@@@8     101479ec     IO61X_Library_MSVC120_vc:IO61X_Port.obj
 0003:00002a08       ??_R0?AVIO61X_CanPort@@@8  10147a08     IO61X_Library_MSVC120_vc:IO61X_CanPort.obj
 0003:00002a24       ??_R0?AVIO61X_CanFdPort@@@8 10147a24     IO61X_Library_MSVC120_vc:IO61X_CanFdPort.obj
 0003:00002a44       ??_R0?AVIO61X_LinPort@@@8  10147a44     IO61X_Library_MSVC120_vc:IO61X_LinPort.obj
 0003:00002a60       ??_R0?AVbad_alloc@std@@@8  10147a60     LIBCMT:new.obj
 0003:00002a7c       ??_R0?AVtype_info@@@8      10147a7c     LIBCMT:typinfo.obj
 0003:00002a94       ??_R0?AVbad_typeid@std@@@8 10147a94     LIBCMT:stdexcpt.obj
 0003:00002ab4       ??_R0?AV__non_rtti_object@std@@@8 10147ab4     LIBCMT:stdexcpt.obj
 0003:00002ad8       ??_R0?AVbad_exception@std@@@8 10147ad8     LIBCMT:frame.obj
 0003:00002af8       ??_R0?AVDNameNode@@@8      10147af8     LIBCMT:undname.obj
 0003:00002b10       ??_R0?AVcharNode@@@8       10147b10     LIBCMT:undname.obj
 0003:00002b28       ??_R0?AVpcharNode@@@8      10147b28     LIBCMT:undname.obj
 0003:00002b40       ??_R0?AVpDNameNode@@@8     10147b40     LIBCMT:undname.obj
 0003:00002b5c       ??_R0?AVDNameStatusNode@@@8 10147b5c     LIBCMT:undname.obj
 0003:00002b7c       ??_R0?AVpairNode@@@8       10147b7c     LIBCMT:undname.obj
 0003:00002b94       ??_R0?AVlength_error@std@@@8 10147b94     libcpmt:xthrow.obj
 0003:00002bb4       ??_R0?AVout_of_range@std@@@8 10147bb4     libcpmt:xthrow.obj
 0003:00002bd4       ??_R0?AVoverflow_error@std@@@8 10147bd4     libcpmt:xthrow.obj
 0003:00002bf8       ??_R0?AVbad_function_call@std@@@8 10147bf8     libcpmt:xthrow.obj
 0003:00002c1c       ??_R0?AVregex_error@std@@@8 10147c1c     libcpmt:xthrow.obj
 0003:00002c3c       ??_R0?AV_Locimp@locale@std@@@8 10147c3c     libcpmt:locale0.obj
 0003:00002c60       ??_R0?AV?$num_get@DV?$istreambuf_iterator@DU?$char_traits@D@std@@@std@@@std@@@8 10147c60     libcpmt:locale.obj
 0003:00002cb8       ??_R0?AV?$num_put@DV?$ostreambuf_iterator@DU?$char_traits@D@std@@@std@@@std@@@8 10147cb8     libcpmt:locale.obj
 0003:00002d0c       ??_R0?AV?$numpunct@D@std@@@8 10147d0c     libcpmt:locale.obj
 0003:00002d2c       ??_R0?AV?$codecvt@_WDH@std@@@8 10147d2c     libcpmt:wlocale.obj
 0003:00002d50       ??_R0?AV?$codecvt@GDH@std@@@8 10147d50     libcpmt:wlocale.obj
 0003:00002d70       ??_R0?AV?$ctype@_W@std@@@8 10147d70     libcpmt:wlocale.obj
 0003:00002d90       ??_R0?AV?$ctype@G@std@@@8  10147d90     libcpmt:wlocale.obj
 0003:00002db0       ??_R0?AV?$num_get@_WV?$istreambuf_iterator@_WU?$char_traits@_W@std@@@std@@@std@@@8 10147db0     libcpmt:wlocale.obj
 0003:00002e08       ??_R0?AV?$num_get@GV?$istreambuf_iterator@GU?$char_traits@G@std@@@std@@@std@@@8 10147e08     libcpmt:wlocale.obj
 0003:00002e5c       ??_R0?AV?$numpunct@_W@std@@@8 10147e5c     libcpmt:wlocale.obj
 0003:00002e7c       ??_R0?AUmessages_base@std@@@8 10147e7c     libcpmt:wlocale.obj
 0003:00002e9c       ??_R0?AUmoney_base@std@@@8 10147e9c     libcpmt:wlocale.obj
 0003:00002ebc       ??_R0?AUtime_base@std@@@8  10147ebc     libcpmt:wlocale.obj
 0003:00002ed8       ??_R0?AV?$num_put@_WV?$ostreambuf_iterator@_WU?$char_traits@_W@std@@@std@@@std@@@8 10147ed8     libcpmt:wlocale.obj
 0003:00002f30       ??_R0?AV?$collate@_W@std@@@8 10147f30     libcpmt:wlocale.obj
 0003:00002f50       ??_R0?AV?$messages@_W@std@@@8 10147f50     libcpmt:wlocale.obj
 0003:00002f70       ??_R0?AV?$money_get@_WV?$istreambuf_iterator@_WU?$char_traits@_W@std@@@std@@@std@@@8 10147f70     libcpmt:wlocale.obj
 0003:00002fc8       ??_R0?AV?$money_put@_WV?$ostreambuf_iterator@_WU?$char_traits@_W@std@@@std@@@std@@@8 10147fc8     libcpmt:wlocale.obj
 0003:00003020       ??_R0?AV?$moneypunct@_W$0A@@std@@@8 10148020     libcpmt:wlocale.obj
 0003:00003048       ??_R0?AV?$_Mpunct@_W@std@@@8 10148048     libcpmt:wlocale.obj
 0003:00003068       ??_R0?AV?$moneypunct@_W$00@std@@@8 10148068     libcpmt:wlocale.obj
 0003:00003090       ??_R0?AV?$time_get@_WV?$istreambuf_iterator@_WU?$char_traits@_W@std@@@std@@@std@@@8 10148090     libcpmt:wlocale.obj
 0003:000030e8       ??_R0?AV?$time_put@_WV?$ostreambuf_iterator@_WU?$char_traits@_W@std@@@std@@@std@@@8 101480e8     libcpmt:wlocale.obj
 0003:00003140       ??_R0?AV?$num_put@GV?$ostreambuf_iterator@GU?$char_traits@G@std@@@std@@@std@@@8 10148140     libcpmt:wlocale.obj
 0003:00003194       ??_R0?AV?$numpunct@G@std@@@8 10148194     libcpmt:wlocale.obj
 0003:000031b4       ??_R0?AV?$collate@G@std@@@8 101481b4     libcpmt:wlocale.obj
 0003:000031d4       ??_R0?AV?$messages@G@std@@@8 101481d4     libcpmt:wlocale.obj
 0003:000031f8       ??_R0?AV?$money_get@GV?$istreambuf_iterator@GU?$char_traits@G@std@@@std@@@std@@@8 101481f8     libcpmt:wlocale.obj
 0003:00003250       ??_R0?AV?$money_put@GV?$ostreambuf_iterator@GU?$char_traits@G@std@@@std@@@std@@@8 10148250     libcpmt:wlocale.obj
 0003:000032a4       ??_R0?AV?$moneypunct@G$0A@@std@@@8 101482a4     libcpmt:wlocale.obj
 0003:000032cc       ??_R0?AV?$_Mpunct@G@std@@@8 101482cc     libcpmt:wlocale.obj
 0003:000032ec       ??_R0?AV?$moneypunct@G$00@std@@@8 101482ec     libcpmt:wlocale.obj
 0003:00003310       ??_R0?AV?$time_get@GV?$istreambuf_iterator@GU?$char_traits@G@std@@@std@@@std@@@8 10148310     libcpmt:wlocale.obj
 0003:00003368       ??_R0?AV?$time_put@GV?$ostreambuf_iterator@GU?$char_traits@G@std@@@std@@@std@@@8 10148368     libcpmt:wlocale.obj
 0003:000033bc       ??_R0?AV?$collate@D@std@@@8 101483bc     libcpmt:xlocale.obj
 0003:000033dc       ??_R0?AV?$messages@D@std@@@8 101483dc     libcpmt:xlocale.obj
 0003:00003400       ??_R0?AV?$money_get@DV?$istreambuf_iterator@DU?$char_traits@D@std@@@std@@@std@@@8 10148400     libcpmt:xlocale.obj
 0003:00003458       ??_R0?AV?$money_put@DV?$ostreambuf_iterator@DU?$char_traits@D@std@@@std@@@std@@@8 10148458     libcpmt:xlocale.obj
 0003:000034ac       ??_R0?AV?$moneypunct@D$0A@@std@@@8 101484ac     libcpmt:xlocale.obj
 0003:000034d4       ??_R0?AV?$_Mpunct@D@std@@@8 101484d4     libcpmt:xlocale.obj
 0003:000034f4       ??_R0?AV?$moneypunct@D$00@std@@@8 101484f4     libcpmt:xlocale.obj
 0003:00003518       ??_R0?AV?$time_get@DV?$istreambuf_iterator@DU?$char_traits@D@std@@@std@@@std@@@8 10148518     libcpmt:xlocale.obj
 0003:00003570       ??_R0?AV?$time_put@DV?$ostreambuf_iterator@DU?$char_traits@D@std@@@std@@@std@@@8 10148570     libcpmt:xlocale.obj
 0003:00003a00       _pci20098PortA             10148a00     xpctarget.obj
 0003:00003a04       _pci20098PortB             10148a04     xpctarget.obj
 0003:00003a08       _siepowercan_firmware_initialized 10148a08     xpctarget.obj
 0003:00003a0c       _siepowercan_port1_configured 10148a0c     xpctarget.obj
 0003:00003a10       _siepowercan_port2_configured 10148a10     xpctarget.obj
 0003:00003a14       _CANAC2_FIRMWARE_LOADED    10148a14     xpctarget.obj
 0003:00003a18       _rs232ports                10148a18     xpctarget.obj
 0003:00003a28       _NI_AT_MIO_16F_5_commreg2  10148a28     xpctarget.obj
 0003:00003a2c       _RTD_DM6430_init           10148a2c     xpctarget.obj
 0003:00003a30       _RTD_DM6420_init           10148a30     xpctarget.obj
 0003:00003a34       _CANAC2_FIRMWARE_LOADED_mb1 10148a34     xpctarget.obj
 0003:00003a38       _CANAC2_FIRMWARE_LOADED_mb2 10148a38     xpctarget.obj
 0003:00003a3c       _CANAC2_FIRMWARE_LOADED_mb3 10148a3c     xpctarget.obj
 0003:00003a40       _xmlsize                   10148a40     xpctarget.obj
 0003:00003a64       ___isa_available_default   10148a64     rt_logging.obj
 0003:00003af4       _mxi                       10148af4     CANTest_xcp.obj
 0003:00003ed8       ?g_IO61X@@3VIO61X_DriverObject@@A 10148ed8     IO61X_Library_MSVC120_vc:IO61X_iConcurrentExecution.obj
 0003:00003f34       ?g_log@@3VIO61X_Logger@@A  10148f34     IO61X_Library_MSVC120_vc:IO61X_iConcurrentExecution.obj
 0003:00003f60       ?id@?$codecvt@DDH@std@@2V0locale@2@A 10148f60     IO61X_Library_MSVC120_vc:IO61X_DriverObject.obj
 0003:00003f64       ?_Stinit@?1??_Init@?$basic_filebuf@DU?$char_traits@D@std@@@std@@IAEXPAU_iobuf@@W4_Initfl@23@@Z@4HA 10148f64     IO61X_Library_MSVC120_vc:IO61X_DriverObject.obj
 0003:00003f68       ?_Psave@?$_Facetptr@V?$ctype@D@std@@@std@@2PBVfacet@locale@2@B 10148f68     IO61X_Library_MSVC120_vc:IO61X_DriverObject.obj
 0003:00003f6c       ?_Psave@?$_Facetptr@V?$codecvt@DDH@std@@@std@@2PBVfacet@locale@2@B 10148f6c     IO61X_Library_MSVC120_vc:IO61X_DriverObject.obj
 0003:00003f78       ?_Guard@?4??_Atomic_thread_fence@std@@YAXW4memory_order@2@@Z@4KA 10148f78     IO61X_Library_MSVC120_vc:IO61X_ModuleManager.obj
 0003:00003fc8       ___fastflag                10148fc8     LIBCMT:fpinit.obj
 0003:000042f0       __C_Exit_Done              101492f0     LIBCMT:crt0dat.obj
 0003:000042f4       ___argc                    101492f4     LIBCMT:crt0dat.obj
 0003:000042f8       ___argv                    101492f8     LIBCMT:crt0dat.obj
 0003:000042fc       ___wargv                   101492fc     LIBCMT:crt0dat.obj
 0003:00004300       __environ                  10149300     LIBCMT:crt0dat.obj
 0003:00004304       __wenviron                 10149304     LIBCMT:crt0dat.obj
 0003:00004308       __pgmptr                   10149308     LIBCMT:crt0dat.obj
 0003:0000430c       __wpgmptr                  1014930c     LIBCMT:crt0dat.obj
 0003:00004310       __umaskval                 10149310     LIBCMT:crt0dat.obj
 0003:00004314       __exitflag                 10149314     LIBCMT:crt0dat.obj
 0003:00004318       __C_Termination_Done       10149318     LIBCMT:crt0dat.obj
 0003:0000431c       ___winitenv                1014931c     LIBCMT:crt0dat.obj
 0003:00004320       ___initenv                 10149320     LIBCMT:crt0dat.obj
 0003:00004324       __cflush                   10149324     LIBCMT:_file.obj
 0003:0000432c       ___isa_available           1014932c     LIBCMT:cpu_disp.obj
 0003:00004330       ___favor                   10149330     LIBCMT:cpu_disp.obj
 0003:00004338       __aenvptr                  10149338     LIBCMT:dllcrt0.obj
 0003:0000433c       __wenvptr                  1014933c     LIBCMT:dllcrt0.obj
 0003:00004340       ?_pnhHeap@@3P6AHI@ZA       10149340     LIBCMT:handler.obj
 0003:00004348       ___app_type                10149348     LIBCMT:crt0msg.obj
 0003:00004978       __newmode                  10149978     LIBCMT:_newmode.obj
 0003:0000497c       __crtheap                  1014997c     LIBCMT:heapinit.obj
 0003:00004980       ___pInvalidArgHandler      10149980     LIBCMT:invarg.obj
 0003:00004ad8       __maxwait                  10149ad8     LIBCMT:crtheap.obj
 0003:00004adc       ?__pInconsistency@@3P6AXXZA 10149adc     LIBCMT:hooks.obj
 0003:00004ae0       ___pPurecall               10149ae0     LIBCMT:inithelp.obj
 0003:00004afc       ___mbcodepage              10149afc     LIBCMT:mbctype.obj
 0003:00004b00       ___ismbcodepage            10149b00     LIBCMT:mbctype.obj
 0003:00004b04       ___mbulinfo                10149b04     LIBCMT:mbctype.obj
 0003:00004b10       ___mblocalename            10149b10     LIBCMT:mbctype.obj
 0003:00004b18       __stdbuf                   10149b18     LIBCMT:_sftbuf.obj
 0003:00004b20       ___pioinfo                 10149b20     LIBCMT:ioinit.obj
 0003:00004c20       ___error_mode              10149c20     LIBCMT:errmode.obj
 0003:00004d40       ?g_OutOfMemoryExceptionCallback@@3P6GPAXXZA 10149d40     LIBCMT:frame.obj
 0003:00004d50       __outputformat             10149d50     LIBCMT:outputformat.obj
 0003:00004d58       __commode                  10149d58     LIBCMT:ncommode.obj
 0003:00004d5c       ?pArgList@UnDecorator@@0PAVReplicator@@A 10149d5c     LIBCMT:undname.obj
 0003:00004d60       ?pZNameList@UnDecorator@@0PAVReplicator@@A 10149d60     LIBCMT:undname.obj
 0003:00004d64       ?pTemplateArgList@UnDecorator@@0PAVReplicator@@A 10149d64     LIBCMT:undname.obj
 0003:00004d68       ?gName@UnDecorator@@0PBDB  10149d68     LIBCMT:undname.obj
 0003:00004d6c       ?name@UnDecorator@@0PBDB   10149d6c     LIBCMT:undname.obj
 0003:00004d70       ?outputString@UnDecorator@@0PADA 10149d70     LIBCMT:undname.obj
 0003:00004d74       ?maxStringLength@UnDecorator@@0HA 10149d74     LIBCMT:undname.obj
 0003:00004d78       ?disableFlags@UnDecorator@@0KA 10149d78     LIBCMT:undname.obj
 0003:00004d7c       ?fExplicitTemplateParams@UnDecorator@@0_NA 10149d7c     LIBCMT:undname.obj
 0003:00004d7d       ?fGetTemplateArgumentList@UnDecorator@@0_NA 10149d7d     LIBCMT:undname.obj
 0003:00004d80       ?m_pGetParameter@UnDecorator@@0P6APADJ@ZA 10149d80     LIBCMT:undname.obj
 0003:00004d98       ?nodes@?1??make@DNameStatusNode@@SAPAV2@W4DNameStatus@@@Z@4PAV2@A 10149d98     LIBCMT:undname.obj
 0003:00004dc8       ??_B?1??make@DNameStatusNode@@SAPAV1@W4DNameStatus@@@Z@51 10149dc8     LIBCMT:undname.obj
 0003:00004dcc       ___lconv_static_null       10149dcc     LIBCMT:lconv.obj
 0003:00004dd0       ___lconv_static_W_null     10149dd0     LIBCMT:lconv.obj
 0003:00004dd4       ___locale_changed          10149dd4     LIBCMT:wsetloca.obj
 0003:00004dd8       __fmode                    10149dd8     LIBCMT:txtmode.obj
 0003:00004de0       ?id@?$num_put@DV?$back_insert_iterator@V?$basic_string@DU?$char_traits@D@std@@V?$allocator@D@2@@std@@@std@@@std@@2V0locale@2@A 10149de0     libcpmt:xthrow.obj
 0003:00004de4       ?id@?$num_put@_WV?$back_insert_iterator@V?$basic_string@_WU?$char_traits@_W@std@@V?$allocator@_W@2@@std@@@std@@@std@@2V0locale@2@A 10149de4     libcpmt:xthrow.obj
 0003:00004de8       ?id@?$numpunct@D@std@@2V0locale@2@A 10149de8     libcpmt:xthrow.obj
 0003:00004dec       ?id@?$numpunct@_W@std@@2V0locale@2@A 10149dec     libcpmt:xthrow.obj
 0003:00004e60       ?_Id_cnt@id@locale@std@@0HA 10149e60     libcpmt:locale0.obj
 0003:00004e68       ?_Clocptr@_Locimp@locale@std@@0PAV123@A 10149e68     libcpmt:locale0.obj
 0003:00004e70       ?id@?$ctype@D@std@@2V0locale@2@A 10149e70     libcpmt:locale0.obj
 0003:00004e74       ?id@?$codecvt@GDH@std@@2V0locale@2@A 10149e74     libcpmt:locale0.obj
 0003:00004e7c       ?id@?$ctype@_W@std@@2V0locale@2@A 10149e7c     libcpmt:locale0.obj
 0003:00004e80       ?id@?$codecvt@_WDH@std@@2V0locale@2@A 10149e80     libcpmt:locale0.obj
 0003:00004e88       ?id@?$ctype@G@std@@2V0locale@2@A 10149e88     libcpmt:locale0.obj
 0003:00004e90       ?_Index@ios_base@std@@0HA  10149e90     libcpmt:ios.obj
 0003:00004ecc       ?_Ptr_cin@std@@3PAV?$basic_istream@DU?$char_traits@D@std@@@1@A 10149ecc     libcpmt:iosptrs.obj
 0003:00004ed0       ?_Ptr_cout@std@@3PAV?$basic_ostream@DU?$char_traits@D@std@@@1@A 10149ed0     libcpmt:iosptrs.obj
 0003:00004ed4       ?_Ptr_cerr@std@@3PAV?$basic_ostream@DU?$char_traits@D@std@@@1@A 10149ed4     libcpmt:iosptrs.obj
 0003:00004ed8       ?_Ptr_clog@std@@3PAV?$basic_ostream@DU?$char_traits@D@std@@@1@A 10149ed8     libcpmt:iosptrs.obj
 0003:00004edc       ?_Ptr_wcin@std@@3PAV?$basic_istream@_WU?$char_traits@_W@std@@@1@A 10149edc     libcpmt:iosptrs.obj
 0003:00004ee0       ?_Ptr_wcout@std@@3PAV?$basic_ostream@_WU?$char_traits@_W@std@@@1@A 10149ee0     libcpmt:iosptrs.obj
 0003:00004ee4       ?_Ptr_wcerr@std@@3PAV?$basic_ostream@_WU?$char_traits@_W@std@@@1@A 10149ee4     libcpmt:iosptrs.obj
 0003:00004ee8       ?_Ptr_wclog@std@@3PAV?$basic_ostream@_WU?$char_traits@_W@std@@@1@A 10149ee8     libcpmt:iosptrs.obj
 0003:00004f1c       ?id@?$num_get@DV?$istreambuf_iterator@DU?$char_traits@D@std@@@std@@@std@@2V0locale@2@A 10149f1c     libcpmt:locale.obj
 0003:00004f20       ?id@?$num_put@DV?$ostreambuf_iterator@DU?$char_traits@D@std@@@std@@@std@@2V0locale@2@A 10149f20     libcpmt:locale.obj
 0003:00004f24       ?_Psave@?$_Facetptr@V?$num_get@DV?$istreambuf_iterator@DU?$char_traits@D@std@@@std@@@std@@@std@@2PBVfacet@locale@2@B 10149f24     libcpmt:locale.obj
 0003:00004f28       ?_Psave@?$_Facetptr@V?$num_put@DV?$ostreambuf_iterator@DU?$char_traits@D@std@@@std@@@std@@@std@@2PBVfacet@locale@2@B 10149f28     libcpmt:locale.obj
 0003:00004f2c       ?_Psave@?$_Facetptr@V?$numpunct@D@std@@@std@@2PBVfacet@locale@2@B 10149f2c     libcpmt:locale.obj
 0003:00004f34       ?id@?$time_put@_WV?$ostreambuf_iterator@_WU?$char_traits@_W@std@@@std@@@std@@2V0locale@2@A 10149f34     libcpmt:wlocale.obj
 0003:00004f38       ?id@?$num_get@_WV?$istreambuf_iterator@_WU?$char_traits@_W@std@@@std@@@std@@2V0locale@2@A 10149f38     libcpmt:wlocale.obj
 0003:00004f3c       ?id@?$num_put@_WV?$ostreambuf_iterator@_WU?$char_traits@_W@std@@@std@@@std@@2V0locale@2@A 10149f3c     libcpmt:wlocale.obj
 0003:00004f40       ?id@?$collate@_W@std@@2V0locale@2@A 10149f40     libcpmt:wlocale.obj
 0003:00004f44       ?id@?$messages@_W@std@@2V0locale@2@A 10149f44     libcpmt:wlocale.obj
 0003:00004f48       ?id@?$money_get@_WV?$istreambuf_iterator@_WU?$char_traits@_W@std@@@std@@@std@@2V0locale@2@A 10149f48     libcpmt:wlocale.obj
 0003:00004f4c       ?id@?$money_put@_WV?$ostreambuf_iterator@_WU?$char_traits@_W@std@@@std@@@std@@2V0locale@2@A 10149f4c     libcpmt:wlocale.obj
 0003:00004f50       ?id@?$moneypunct@_W$0A@@std@@2V0locale@2@A 10149f50     libcpmt:wlocale.obj
 0003:00004f54       ?id@?$moneypunct@_W$00@std@@2V0locale@2@A 10149f54     libcpmt:wlocale.obj
 0003:00004f58       ?id@?$time_get@_WV?$istreambuf_iterator@_WU?$char_traits@_W@std@@@std@@@std@@2V0locale@2@A 10149f58     libcpmt:wlocale.obj
 0003:00004f5c       ?id@?$num_get@GV?$istreambuf_iterator@GU?$char_traits@G@std@@@std@@@std@@2V0locale@2@A 10149f5c     libcpmt:wlocale.obj
 0003:00004f60       ?id@?$num_put@GV?$ostreambuf_iterator@GU?$char_traits@G@std@@@std@@@std@@2V0locale@2@A 10149f60     libcpmt:wlocale.obj
 0003:00004f64       ?id@?$numpunct@G@std@@2V0locale@2@A 10149f64     libcpmt:wlocale.obj
 0003:00004f68       ?id@?$collate@G@std@@2V0locale@2@A 10149f68     libcpmt:wlocale.obj
 0003:00004f6c       ?id@?$messages@G@std@@2V0locale@2@A 10149f6c     libcpmt:wlocale.obj
 0003:00004f70       ?id@?$money_get@GV?$istreambuf_iterator@GU?$char_traits@G@std@@@std@@@std@@2V0locale@2@A 10149f70     libcpmt:wlocale.obj
 0003:00004f74       ?id@?$money_put@GV?$ostreambuf_iterator@GU?$char_traits@G@std@@@std@@@std@@2V0locale@2@A 10149f74     libcpmt:wlocale.obj
 0003:00004f78       ?id@?$moneypunct@G$0A@@std@@2V0locale@2@A 10149f78     libcpmt:wlocale.obj
 0003:00004f7c       ?id@?$moneypunct@G$00@std@@2V0locale@2@A 10149f7c     libcpmt:wlocale.obj
 0003:00004f80       ?id@?$time_get@GV?$istreambuf_iterator@GU?$char_traits@G@std@@@std@@@std@@2V0locale@2@A 10149f80     libcpmt:wlocale.obj
 0003:00004f84       ?id@?$time_put@GV?$ostreambuf_iterator@GU?$char_traits@G@std@@@std@@@std@@2V0locale@2@A 10149f84     libcpmt:wlocale.obj
 0003:00004f88       ?_Psave@?$_Facetptr@V?$ctype@_W@std@@@std@@2PBVfacet@locale@2@B 10149f88     libcpmt:wlocale.obj
 0003:00004f8c       ?_Psave@?$_Facetptr@V?$ctype@G@std@@@std@@2PBVfacet@locale@2@B 10149f8c     libcpmt:wlocale.obj
 0003:00004f90       ?_Psave@?$_Facetptr@V?$num_get@_WV?$istreambuf_iterator@_WU?$char_traits@_W@std@@@std@@@std@@@std@@2PBVfacet@locale@2@B 10149f90     libcpmt:wlocale.obj
 0003:00004f94       ?_Psave@?$_Facetptr@V?$num_put@_WV?$ostreambuf_iterator@_WU?$char_traits@_W@std@@@std@@@std@@@std@@2PBVfacet@locale@2@B 10149f94     libcpmt:wlocale.obj
 0003:00004f98       ?_Psave@?$_Facetptr@V?$numpunct@_W@std@@@std@@2PBVfacet@locale@2@B 10149f98     libcpmt:wlocale.obj
 0003:00004f9c       ?_Psave@?$_Facetptr@V?$collate@_W@std@@@std@@2PBVfacet@locale@2@B 10149f9c     libcpmt:wlocale.obj
 0003:00004fa0       ?_Psave@?$_Facetptr@V?$messages@_W@std@@@std@@2PBVfacet@locale@2@B 10149fa0     libcpmt:wlocale.obj
 0003:00004fa4       ?_Psave@?$_Facetptr@V?$money_get@_WV?$istreambuf_iterator@_WU?$char_traits@_W@std@@@std@@@std@@@std@@2PBVfacet@locale@2@B 10149fa4     libcpmt:wlocale.obj
 0003:00004fa8       ?_Psave@?$_Facetptr@V?$money_put@_WV?$ostreambuf_iterator@_WU?$char_traits@_W@std@@@std@@@std@@@std@@2PBVfacet@locale@2@B 10149fa8     libcpmt:wlocale.obj
 0003:00004fac       ?_Psave@?$_Facetptr@V?$moneypunct@_W$0A@@std@@@std@@2PBVfacet@locale@2@B 10149fac     libcpmt:wlocale.obj
 0003:00004fb0       ?_Psave@?$_Facetptr@V?$moneypunct@_W$00@std@@@std@@2PBVfacet@locale@2@B 10149fb0     libcpmt:wlocale.obj
 0003:00004fb4       ?_Psave@?$_Facetptr@V?$time_get@_WV?$istreambuf_iterator@_WU?$char_traits@_W@std@@@std@@@std@@@std@@2PBVfacet@locale@2@B 10149fb4     libcpmt:wlocale.obj
 0003:00004fb8       ?_Psave@?$_Facetptr@V?$time_put@_WV?$ostreambuf_iterator@_WU?$char_traits@_W@std@@@std@@@std@@@std@@2PBVfacet@locale@2@B 10149fb8     libcpmt:wlocale.obj
 0003:00004fbc       ?_Psave@?$_Facetptr@V?$codecvt@_WDH@std@@@std@@2PBVfacet@locale@2@B 10149fbc     libcpmt:wlocale.obj
 0003:00004fc0       ?_Psave@?$_Facetptr@V?$num_get@GV?$istreambuf_iterator@GU?$char_traits@G@std@@@std@@@std@@@std@@2PBVfacet@locale@2@B 10149fc0     libcpmt:wlocale.obj
 0003:00004fc4       ?_Psave@?$_Facetptr@V?$num_put@GV?$ostreambuf_iterator@GU?$char_traits@G@std@@@std@@@std@@@std@@2PBVfacet@locale@2@B 10149fc4     libcpmt:wlocale.obj
 0003:00004fc8       ?_Psave@?$_Facetptr@V?$numpunct@G@std@@@std@@2PBVfacet@locale@2@B 10149fc8     libcpmt:wlocale.obj
 0003:00004fcc       ?_Psave@?$_Facetptr@V?$collate@G@std@@@std@@2PBVfacet@locale@2@B 10149fcc     libcpmt:wlocale.obj
 0003:00004fd0       ?_Psave@?$_Facetptr@V?$messages@G@std@@@std@@2PBVfacet@locale@2@B 10149fd0     libcpmt:wlocale.obj
 0003:00004fd4       ?_Psave@?$_Facetptr@V?$money_get@GV?$istreambuf_iterator@GU?$char_traits@G@std@@@std@@@std@@@std@@2PBVfacet@locale@2@B 10149fd4     libcpmt:wlocale.obj
 0003:00004fd8       ?_Psave@?$_Facetptr@V?$money_put@GV?$ostreambuf_iterator@GU?$char_traits@G@std@@@std@@@std@@@std@@2PBVfacet@locale@2@B 10149fd8     libcpmt:wlocale.obj
 0003:00004fdc       ?_Psave@?$_Facetptr@V?$moneypunct@G$0A@@std@@@std@@2PBVfacet@locale@2@B 10149fdc     libcpmt:wlocale.obj
 0003:00004fe0       ?_Psave@?$_Facetptr@V?$moneypunct@G$00@std@@@std@@2PBVfacet@locale@2@B 10149fe0     libcpmt:wlocale.obj
 0003:00004fe4       ?_Psave@?$_Facetptr@V?$time_get@GV?$istreambuf_iterator@GU?$char_traits@G@std@@@std@@@std@@@std@@2PBVfacet@locale@2@B 10149fe4     libcpmt:wlocale.obj
 0003:00004fe8       ?_Psave@?$_Facetptr@V?$time_put@GV?$ostreambuf_iterator@GU?$char_traits@G@std@@@std@@@std@@@std@@2PBVfacet@locale@2@B 10149fe8     libcpmt:wlocale.obj
 0003:00004fec       ?_Psave@?$_Facetptr@V?$codecvt@GDH@std@@@std@@2PBVfacet@locale@2@B 10149fec     libcpmt:wlocale.obj
 0003:00004ff4       ?id@?$collate@D@std@@2V0locale@2@A 10149ff4     libcpmt:xlocale.obj
 0003:00004ff8       ?id@?$messages@D@std@@2V0locale@2@A 10149ff8     libcpmt:xlocale.obj
 0003:00004ffc       ?id@?$money_get@DV?$istreambuf_iterator@DU?$char_traits@D@std@@@std@@@std@@2V0locale@2@A 10149ffc     libcpmt:xlocale.obj
 0003:00005000       ?id@?$money_put@DV?$ostreambuf_iterator@DU?$char_traits@D@std@@@std@@@std@@2V0locale@2@A 1014a000     libcpmt:xlocale.obj
 0003:00005004       ?id@?$moneypunct@D$0A@@std@@2V0locale@2@A 1014a004     libcpmt:xlocale.obj
 0003:00005008       ?id@?$moneypunct@D$00@std@@2V0locale@2@A 1014a008     libcpmt:xlocale.obj
 0003:0000500c       ?id@?$time_get@DV?$istreambuf_iterator@DU?$char_traits@D@std@@@std@@@std@@2V0locale@2@A 1014a00c     libcpmt:xlocale.obj
 0003:00005010       ?id@?$time_put@DV?$ostreambuf_iterator@DU?$char_traits@D@std@@@std@@@std@@2V0locale@2@A 1014a010     libcpmt:xlocale.obj
 0003:00005014       ?_Psave@?$_Facetptr@V?$collate@D@std@@@std@@2PBVfacet@locale@2@B 1014a014     libcpmt:xlocale.obj
 0003:00005018       ?_Psave@?$_Facetptr@V?$messages@D@std@@@std@@2PBVfacet@locale@2@B 1014a018     libcpmt:xlocale.obj
 0003:0000501c       ?_Psave@?$_Facetptr@V?$money_get@DV?$istreambuf_iterator@DU?$char_traits@D@std@@@std@@@std@@@std@@2PBVfacet@locale@2@B 1014a01c     libcpmt:xlocale.obj
 0003:00005020       ?_Psave@?$_Facetptr@V?$money_put@DV?$ostreambuf_iterator@DU?$char_traits@D@std@@@std@@@std@@@std@@2PBVfacet@locale@2@B 1014a020     libcpmt:xlocale.obj
 0003:00005024       ?_Psave@?$_Facetptr@V?$moneypunct@D$0A@@std@@@std@@2PBVfacet@locale@2@B 1014a024     libcpmt:xlocale.obj
 0003:00005028       ?_Psave@?$_Facetptr@V?$moneypunct@D$00@std@@@std@@2PBVfacet@locale@2@B 1014a028     libcpmt:xlocale.obj
 0003:0000502c       ?_Psave@?$_Facetptr@V?$time_get@DV?$istreambuf_iterator@DU?$char_traits@D@std@@@std@@@std@@@std@@2PBVfacet@locale@2@B 1014a02c     libcpmt:xlocale.obj
 0003:00005030       ?_Psave@?$_Facetptr@V?$time_put@DV?$ostreambuf_iterator@DU?$char_traits@D@std@@@std@@@std@@@std@@2PBVfacet@locale@2@B 1014a030     libcpmt:xlocale.obj
 0003:00005038       __FZero                    1014a038     libcpmt:xfvalues.obj
 0003:00005040       __Zero                     1014a040     libcpmt:xvalues.obj
 0003:00005048       __LZero                    1014a048     libcpmt:xlvalues.obj
 0003:00005050       _g_targetAuthenticationResult 1014a050     libsg_MSVC120_vc:sg_common.obj
 0003:00005058       _pSgErrorStr               1014a058     libsg_MSVC120_vc:sg_common.obj
 0003:00005254       _myNICGetMac               1014a254     libsg_MSVC120_vc:sg_target.obj
 0003:00005380       ?cout@std@@3V?$basic_ostream@DU?$char_traits@D@std@@@1@A 1014a380     libcpmt:cout.obj
 0003:000053d0       _rtNaNF                    1014a3d0     <common>
 0003:000053e4       _rtMinusInfF               1014a3e4     <common>
 0003:000053e8       _rtInfF                    1014a3e8     <common>
 0003:000053f0       _rtNaN                     1014a3f0     <common>
 0003:000053f8       _rtMinusInf                1014a3f8     <common>
 0003:00005400       _rtInf                     1014a400     <common>
 0003:00005420       _slrtTETViaXCP             1014a420     <common>
 0003:00005460       _CANTest_M_                1014a460     <common>
 0003:00006940       _CANTest_DW                1014b940     <common>
 0003:000069c0       _CANTest_B                 1014b9c0     <common>
 0003:00006aa0       _CANAC2_2_receiveindex_mb3 1014baa0     <common>
 0003:00009b74       _CANAC2_2_receivemaxindex_mb3 1014eb74     <common>
 0003:00009b80       _CANAC2_2_sendindex_mb3    1014eb80     <common>
 0003:00009ea0       _CANAC2_2_sendmaxindex_mb3 1014eea0     <common>
 0003:00009ec0       _CANAC2_1_receiveindex_mb3 1014eec0     <common>
 0003:0000a1e0       _CANAC2_1_receivemaxindex_mb3 1014f1e0     <common>
 0003:0000a200       _CANAC2_1_sendindex_mb3    1014f200     <common>
 0003:0000a520       _CANAC2_1_sendmaxindex_mb3 1014f520     <common>
 0003:0000a540       _CANAC2_2_receive_mb3      1014f540     <common>
 0003:0000a860       _CANAC2_2_send_mb3         1014f860     <common>
 0003:0000ab80       _CANAC2_1_receive_mb3      1014fb80     <common>
 0003:0000aea0       _CANAC2_1_send_mb3         1014fea0     <common>
 0003:0000b1c0       _CANAC2_2_receiveindex_mb2 101501c0     <common>
 0003:0000b4e0       _CANAC2_2_receivemaxindex_mb2 101504e0     <common>
 0003:0000b500       _CANAC2_2_sendindex_mb2    10150500     <common>
 0003:0000b820       _CANAC2_2_sendmaxindex_mb2 10150820     <common>
 0003:0000b840       _CANAC2_1_receiveindex_mb2 10150840     <common>
 0003:0000bb60       _CANAC2_1_receivemaxindex_mb2 10150b60     <common>
 0003:0000bb80       _CANAC2_1_sendindex_mb2    10150b80     <common>
 0003:0000bea0       _CANAC2_1_sendmaxindex_mb2 10150ea0     <common>
 0003:0000bec0       _CANAC2_2_receive_mb2      10150ec0     <common>
 0003:0000c1e0       _CANAC2_2_send_mb2         101511e0     <common>
 0003:0000c500       _CANAC2_1_receive_mb2      10151500     <common>
 0003:0000c820       _CANAC2_1_send_mb2         10151820     <common>
 0003:0000cb40       _CANAC2_2_receiveindex_mb1 10151b40     <common>
 0003:0000ce60       _CANAC2_2_receivemaxindex_mb1 10151e60     <common>
 0003:0000ce80       _CANAC2_2_sendindex_mb1    10151e80     <common>
 0003:0000d1a0       _CANAC2_2_sendmaxindex_mb1 101521a0     <common>
 0003:0000d1c0       _CANAC2_1_receiveindex_mb1 101521c0     <common>
 0003:0000d4e0       _CANAC2_1_receivemaxindex_mb1 101524e0     <common>
 0003:0000d500       _CANAC2_1_sendindex_mb1    10152500     <common>
 0003:0000d820       _CANAC2_1_sendmaxindex_mb1 10152820     <common>
 0003:0000d840       _CANAC2_2_receive_mb1      10152840     <common>
 0003:0000db60       _CANAC2_2_send_mb1         10152b60     <common>
 0003:0000de80       _CANAC2_1_receive_mb1      10152e80     <common>
 0003:0000e1a0       _CANAC2_1_send_mb1         101531a0     <common>
 0003:0000e4c0       _CANAC2_2_receiveindex     101534c0     <common>
 0003:0000e7e0       _CANAC2_2_receivemaxindex  101537e0     <common>
 0003:0000e800       _CANAC2_2_sendindex        10153800     <common>
 0003:0000eb20       _CANAC2_2_sendmaxindex     10153b20     <common>
 0003:0000eb40       _CANAC2_1_receiveindex     10153b40     <common>
 0003:0000ee60       _CANAC2_1_receivemaxindex  10153e60     <common>
 0003:0000ee80       _CANAC2_1_sendindex        10153e80     <common>
 0003:0000f1a0       _CANAC2_1_sendmaxindex     101541a0     <common>
 0003:0000f1c0       _CANAC2_2_receive          101541c0     <common>
 0003:0000f4e0       _CANAC2_2_send             101544e0     <common>
 0003:0000f800       _CANAC2_1_receive          10154800     <common>
 0003:0000fb20       _CANAC2_1_send             10154b20     <common>
 0003:0000fe40       _siepowercan_can_object_buffer_port2 10154e40     <common>
 0003:00013e60       _siepowercan_can_object_buffer_port1 10158e60     <common>
 0003:00017e60       _xpceFSScopeSet            1015ce60     <common>
 0003:00017ed8       _rl32eSetScope             1015ced8     <common>
 0003:00017edc       _rl32eAddSignal            1015cedc     <common>
 0003:00017ee0       _rl32eGetSignalNo          1015cee0     <common>
 0003:00017ee4       _rl32eDefScope             1015cee4     <common>
 0003:00017ee8       _rl32eScopeExists          1015cee8     <common>
 0003:00017eec       _TBGiveSpinFast            1015ceec     <common>
 0003:00017ef0       _TBTakeSpinFast            1015cef0     <common>
 0003:00017ef4       _TBDeleteSpin              1015cef4     <common>
 0003:00017ef8       _TBCreateSpin              1015cef8     <common>
 0003:00017efc       _xpceGetParamDims          1015cefc     <common>
 0003:00017f00       _xpceGetParameter          1015cf00     <common>
 0003:00017f04       _xpceSetParameter          1015cf04     <common>
 0003:00017f08       _xpceGetSignalValue        1015cf08     <common>
 0003:00017f0c       _xpceAssignPCIInterrupt    1015cf0c     <common>
 0003:00017f10       _rl32eGetPCIInfoAtSlot     1015cf10     <common>
 0003:00017f14       _rl32eGetPCIInfo           1015cf14     <common>
 0003:00017f18       _rl32eShowPCIInfo          1015cf18     <common>
 0003:00017f1c       _rl32eShowPCIDev           1015cf1c     <common>
 0003:00017f20       _xpceGetTET                1015cf20     <common>
 0003:00017f24       _xpceaddEvent              1015cf24     <common>
 0003:00017f28       _xpceDeRegisterISR         1015cf28     <common>
 0003:00017f2c       _xpceRegisterISR           1015cf2c     <common>
 0003:00017f30       _xpcIsModelInit            1015cf30     <common>
 0003:00017f34       _xpcGetElapsedTime         1015cf34     <common>
 0003:00017f38       _xpcBusyWait               1015cf38     <common>
 0003:00017f3c       _xpcFreePhysicalMemory     1015cf3c     <common>
 0003:00017f40       _xpcAllocPhysicalMemory    1015cf40     <common>
 0003:00017f44       _xpcReserveMemoryRegion    1015cf44     <common>
 0003:00017f48       _xpcOutpB                  1015cf48     <common>
 0003:00017f4c       _xpcOutpW                  1015cf4c     <common>
 0003:00017f50       _xpcOutpDW                 1015cf50     <common>
 0003:00017f54       _xpcInpB                   1015cf54     <common>
 0003:00017f58       _xpcInpW                   1015cf58     <common>
 0003:00017f5c       _xpcInpDW                  1015cf5c     <common>
 0003:00017f60       _waitForDFTask             1015cf60     <common>
 0003:00017f64       _triggerDFTask             1015cf64     <common>
 0003:00017f68       _deregisterDFTask          1015cf68     <common>
 0003:00017f6c       _registerDFTask            1015cf6c     <common>
 0003:00017f70       _UDPCloseReceive           1015cf70     <common>
 0003:00017f74       _UDPCloseSend              1015cf74     <common>
 0003:00017f78       _UDPAddMulticastMembership 1015cf78     <common>
 0003:00017f7c       _UDPOpenReceive            1015cf7c     <common>
 0003:00017f80       _UDPOpenSend               1015cf80     <common>
 0003:00017f84       _ResetClientSocket         1015cf84     <common>
 0003:00017f88       _CloseClientSocket         1015cf88     <common>
 0003:00017f8c       _ConnectClientSocket       1015cf8c     <common>
 0003:00017f90       _BindClientSocket          1015cf90     <common>
 0003:00017f94       _CreateClientSocket        1015cf94     <common>
 0003:00017f98       _ResetServerSocket         1015cf98     <common>
 0003:00017f9c       _CloseServerSocket         1015cf9c     <common>
 0003:00017fa0       _ConnectServerSocket       1015cfa0     <common>
 0003:00017fa4       _OpenServerListen          1015cfa4     <common>
 0003:00017fa8       _CreateServerSocket        1015cfa8     <common>
 0003:00017fac       _SocketReceive             1015cfac     <common>
 0003:00017fb0       _SocketSend                1015cfb0     <common>
 0003:00017fb4       _GetSocketState            1015cfb4     <common>
 0003:00017fb8       _GetSocket                 1015cfb8     <common>
 0003:00017fbc       _socket                    1015cfbc     <common>
 0003:00017fc0       _inet_addr                 1015cfc0     <common>
 0003:00017fc4       _sendto                    1015cfc4     <common>
 0003:00017fc8       _recvfrom                  1015cfc8     <common>
 0003:00017fcc       _listen                    1015cfcc     <common>
 0003:00017fd0       _ioctlsocket               1015cfd0     <common>
 0003:00017fd4       _connect                   1015cfd4     <common>
 0003:00017fd8       _closesocket               1015cfd8     <common>
 0003:00017fdc       _setsockopt                1015cfdc     <common>
 0003:00017fe0       _bind                      1015cfe0     <common>
 0003:00017fe4       _accept                    1015cfe4     <common>
 0003:00017fe8       _GetHostTarIPAdd           1015cfe8     <common>
 0003:00017fec       _GetDCUUsage               1015cfec     <common>
 0003:00017ff0       _DeleteRoute               1015cff0     <common>
 0003:00017ff4       _AddMulticastRoute         1015cff4     <common>
 0003:00017ff8       _AddGatewayRoute           1015cff8     <common>
 0003:00017ffc       _SetIP                     1015cffc     <common>
 0003:00018000       _CloseInterface            1015d000     <common>
 0003:00018004       _OpenInterface             1015d004     <common>
 0003:00018008       _SetIPTASKPriority         1015d008     <common>
 0003:0001800c       _releaseNIC                1015d00c     <common>
 0003:00018010       _NICGetIface               1015d010     <common>
 0003:00018014       _NICSetIface               1015d014     <common>
 0003:00018018       _registerNIC               1015d018     <common>
 0003:0001801c       _slrtWarning               1015d01c     <common>
 0003:00018020       _slrtGetCPUTCelsius        1015d020     <common>
 0003:00018024       _geterrorstring            1015d024     <common>
 0003:00018028       _getlasterror              1015d028     <common>
 0003:0001802c       _slrtGetProfilerState      1015d02c     <common>
 0003:00018030       _slrtStopProfiler          1015d030     <common>
 0003:00018034       _slrtStartProfiler         1015d034     <common>
 0003:00018038       _slrtLogEvent              1015d038     <common>
 0003:0001803c       _slrtGetDefaultDrive       1015d03c     <common>
 0003:00018040       _slrtfsFread               1015d040     <common>
 0003:00018044       _slrtfsGetFileStatus       1015d044     <common>
 0003:00018048       _slrtfsOpenFileAsync       1015d048     <common>
 0003:0001804c       _slrtfsCloseFileAsync      1015d04c     <common>
 0003:00018050       _slrtfsGetFileErrorMessage 1015d050     <common>
 0003:00018054       _slrtfsGetFileError        1015d054     <common>
 0003:00018058       _slrtfsWriteToFile         1015d058     <common>
 0003:0001805c       _slrtfsCloseFile           1015d05c     <common>
 0003:00018060       _slrtfsOpenFile            1015d060     <common>
 0003:00018064       _slrtGetSgCRBSpace         1015d064     <common>
 0003:00018068       _slrtGetCRBScratchSpace    1015d068     <common>
 0003:0001806c       _slrteSetupMSI             1015d06c     <common>
 0003:00018070       _slTestRegAssessment       1015d070     <common>
 0003:00018074       _slTestTerminate           1015d074     <common>
 0003:00018078       _slTestEvalOnFail          1015d078     <common>
 0003:0001807c       _slTestLogAssessments      1015d07c     <common>
 0003:00018080       _slTestInitialize          1015d080     <common>
 0003:00018084       _unRegisterPTPTimeRead     1015d084     <common>
 0003:00018088       _registerPTPTimeRead       1015d088     <common>
 0003:0001808c       _slrteGetCurrentStepSize   1015d08c     <common>
 0003:00018090       _slrteSetStepSizeDelta     1015d090     <common>
 0003:00018094       _slrtLogSignal             1015d094     <common>
 0003:00018098       _slrtRegisterSignal        1015d098     <common>
 0003:0001809c       _xpceDAQUpdateTimeStamp    1015d09c     <common>
 0003:000180a0       _xpceDAQPostEvent          1015d0a0     <common>
 0003:000180a4       _StreamVideo               1015d0a4     <common>
 0003:000180a8       _StopVideoDisplay          1015d0a8     <common>
 0003:000180ac       _StartVideoDisplay         1015d0ac     <common>
 0003:000180b0       _DestroyVideoDisplay       1015d0b0     <common>
 0003:000180b4       _CreateVideoDisplay        1015d0b4     <common>
 0003:000180b8       _ConvertUImage             1015d0b8     <common>
 0003:000180bc       _StopVideo                 1015d0bc     <common>
 0003:000180c0       _ReadFrameBuffer           1015d0c0     <common>
 0003:000180c4       _StartVideo                1015d0c4     <common>
 0003:000180c8       _GetVideoConfigs           1015d0c8     <common>
 0003:000180cc       _FindUsbVideoDevice        1015d0cc     <common>
 0003:000180d0       _xpceDeleteSemaphore       1015d0d0     <common>
 0003:000180d4       _xpceSignalSemaphore       1015d0d4     <common>
 0003:000180d8       _xpceWaitSemaphore         1015d0d8     <common>
 0003:000180dc       _xpceCreateSemaphore       1015d0dc     <common>
 0003:000180e0       _xpceScopeAcqOK            1015d0e0     <common>
 0003:000180e4       _rl32eRestartAcquisition   1015d0e4     <common>
 0003:000180e8       _rl32eSetTargetScopeSigFt  1015d0e8     <common>
 0003:000180ec       _rl32eSetTargetScope       1015d0ec     <common>
 0003:000180f0       ___unguarded_readlc_active 1015d0f0     <common>
 0003:00018100       ___setlc_active            1015d100     <common>
 0003:00018104       ___use_sse2_mathfcns       1015d104     <common>
 0003:00018110       __pmatherr                 1015d110     <common>
 0003:0001811c       __nhandle                  1015d11c     <common>
 0003:00018140       _encodedKERNEL32Functions  1015d140     <common>
 0003:000181e8       __debugger_hook_dummy      1015d1e8     <common>
 0003:000181f4       __acmdln                   1015d1f4     <common>
 0003:00018200       __bufin                    1015d200     <common>
 0003:0001953c       ___piob                    1015e53c     <common>
 0003:00019540       __nstream                  1015e540     <common>
 0003:00019544       ___dyn_tls_init_callback   1015e544     <common>
 0003:00019554       ___onexitend               1015e554     <common>
 0003:00019558       ___onexitbegin             1015e558     <common>
 0003:0001955c       ___mbctype_initialized     1015e55c     <common>
 0003:00019560       ___env_initialized         1015e560     <common>
 0004:00000000       __imp__GetModuleHandleA@4  1015f000     kernel32:KERNEL32.dll
 0004:00000004       __imp__GetProcAddress@8    1015f004     kernel32:KERNEL32.dll
 0004:00000008       __imp__WaitForSingleObject@8 1015f008     kernel32:KERNEL32.dll
 0004:0000000c       __imp__HeapAlloc@12        1015f00c     kernel32:KERNEL32.dll
 0004:00000010       __imp__GetLastError@0      1015f010     kernel32:KERNEL32.dll
 0004:00000014       __imp__HeapFree@12         1015f014     kernel32:KERNEL32.dll
 0004:00000018       __imp__IsDebuggerPresent@0 1015f018     kernel32:KERNEL32.dll
 0004:0000001c       __imp__IsProcessorFeaturePresent@4 1015f01c     kernel32:KERNEL32.dll
 0004:00000020       __imp__EncodePointer@4     1015f020     kernel32:KERNEL32.dll
 0004:00000024       __imp__DecodePointer@4     1015f024     kernel32:KERNEL32.dll
 0004:00000028       __imp__ExitProcess@4       1015f028     kernel32:KERNEL32.dll
 0004:0000002c       __imp__GetModuleHandleExW@12 1015f02c     kernel32:KERNEL32.dll
 0004:00000030       __imp__AreFileApisANSI@0   1015f030     kernel32:KERNEL32.dll
 0004:00000034       __imp__MultiByteToWideChar@24 1015f034     kernel32:KERNEL32.dll
 0004:00000038       __imp__WideCharToMultiByte@32 1015f038     kernel32:KERNEL32.dll
 0004:0000003c       __imp__HeapReAlloc@16      1015f03c     kernel32:KERNEL32.dll
 0004:00000040       __imp__EnterCriticalSection@4 1015f040     kernel32:KERNEL32.dll
 0004:00000044       __imp__LeaveCriticalSection@4 1015f044     kernel32:KERNEL32.dll
 0004:00000048       __imp__GetStdHandle@4      1015f048     kernel32:KERNEL32.dll
 0004:0000004c       __imp__GetFileType@4       1015f04c     kernel32:KERNEL32.dll
 0004:00000050       __imp__GetModuleFileNameW@12 1015f050     kernel32:KERNEL32.dll
 0004:00000054       __imp__WriteConsoleW@20    1015f054     kernel32:KERNEL32.dll
 0004:00000058       __imp__GetCommandLineA@0   1015f058     kernel32:KERNEL32.dll
 0004:0000005c       __imp__GetCurrentThreadId@0 1015f05c     kernel32:KERNEL32.dll
 0004:00000060       __imp__RaiseException@16   1015f060     kernel32:KERNEL32.dll
 0004:00000064       __imp__RtlUnwind@16        1015f064     kernel32:KERNEL32.dll
 0004:00000068       __imp__WriteFile@20        1015f068     kernel32:KERNEL32.dll
 0004:0000006c       __imp__GetProcessHeap@0    1015f06c     kernel32:KERNEL32.dll
 0004:00000070       __imp__UnhandledExceptionFilter@4 1015f070     kernel32:KERNEL32.dll
 0004:00000074       __imp__SetUnhandledExceptionFilter@4 1015f074     kernel32:KERNEL32.dll
 0004:00000078       __imp__SetLastError@4      1015f078     kernel32:KERNEL32.dll
 0004:0000007c       __imp__InitializeCriticalSectionAndSpinCount@8 1015f07c     kernel32:KERNEL32.dll
 0004:00000080       __imp__CreateEventW@16     1015f080     kernel32:KERNEL32.dll
 0004:00000084       __imp__Sleep@4             1015f084     kernel32:KERNEL32.dll
 0004:00000088       __imp__GetCurrentProcess@0 1015f088     kernel32:KERNEL32.dll
 0004:0000008c       __imp__TerminateProcess@8  1015f08c     kernel32:KERNEL32.dll
 0004:00000090       __imp__TlsAlloc@0          1015f090     kernel32:KERNEL32.dll
 0004:00000094       __imp__TlsGetValue@4       1015f094     kernel32:KERNEL32.dll
 0004:00000098       __imp__TlsSetValue@8       1015f098     kernel32:KERNEL32.dll
 0004:0000009c       __imp__TlsFree@4           1015f09c     kernel32:KERNEL32.dll
 0004:000000a0       __imp__GetStartupInfoW@4   1015f0a0     kernel32:KERNEL32.dll
 0004:000000a4       __imp__GetTickCount@0      1015f0a4     kernel32:KERNEL32.dll
 0004:000000a8       __imp__GetModuleHandleW@4  1015f0a8     kernel32:KERNEL32.dll
 0004:000000ac       __imp__CreateSemaphoreW@16 1015f0ac     kernel32:KERNEL32.dll
 0004:000000b0       __imp__DeleteCriticalSection@4 1015f0b0     kernel32:KERNEL32.dll
 0004:000000b4       __imp__FatalAppExitA@8     1015f0b4     kernel32:KERNEL32.dll
 0004:000000b8       __imp__SetConsoleCtrlHandler@8 1015f0b8     kernel32:KERNEL32.dll
 0004:000000bc       __imp__FreeLibrary@4       1015f0bc     kernel32:KERNEL32.dll
 0004:000000c0       __imp__LoadLibraryExW@12   1015f0c0     kernel32:KERNEL32.dll
 0004:000000c4       __imp__IsValidCodePage@4   1015f0c4     kernel32:KERNEL32.dll
 0004:000000c8       __imp__GetACP@0            1015f0c8     kernel32:KERNEL32.dll
 0004:000000cc       __imp__GetOEMCP@0          1015f0cc     kernel32:KERNEL32.dll
 0004:000000d0       __imp__GetCPInfo@8         1015f0d0     kernel32:KERNEL32.dll
 0004:000000d4       __imp__CloseHandle@4       1015f0d4     kernel32:KERNEL32.dll
 0004:000000d8       __imp__ReadFile@20         1015f0d8     kernel32:KERNEL32.dll
 0004:000000dc       __imp__GetConsoleMode@8    1015f0dc     kernel32:KERNEL32.dll
 0004:000000e0       __imp__ReadConsoleW@20     1015f0e0     kernel32:KERNEL32.dll
 0004:000000e4       __imp__GetConsoleCP@0      1015f0e4     kernel32:KERNEL32.dll
 0004:000000e8       __imp__DeleteFileW@4       1015f0e8     kernel32:KERNEL32.dll
 0004:000000ec       __imp__SetFilePointerEx@20 1015f0ec     kernel32:KERNEL32.dll
 0004:000000f0       __imp__OutputDebugStringW@4 1015f0f0     kernel32:KERNEL32.dll
 0004:000000f4       __imp__GetCurrentThread@0  1015f0f4     kernel32:KERNEL32.dll
 0004:000000f8       __imp__GetModuleFileNameA@12 1015f0f8     kernel32:KERNEL32.dll
 0004:000000fc       __imp__QueryPerformanceCounter@4 1015f0fc     kernel32:KERNEL32.dll
 0004:00000100       __imp__GetCurrentProcessId@0 1015f100     kernel32:KERNEL32.dll
 0004:00000104       __imp__GetSystemTimeAsFileTime@4 1015f104     kernel32:KERNEL32.dll
 0004:00000108       __imp__GetEnvironmentStringsW@0 1015f108     kernel32:KERNEL32.dll
 0004:0000010c       __imp__FreeEnvironmentStringsW@4 1015f10c     kernel32:KERNEL32.dll
 0004:00000110       __imp__HeapSize@12         1015f110     kernel32:KERNEL32.dll
 0004:00000114       __imp__FlushFileBuffers@4  1015f114     kernel32:KERNEL32.dll
 0004:00000118       __imp__GetDateFormatW@24   1015f118     kernel32:KERNEL32.dll
 0004:0000011c       __imp__GetTimeFormatW@24   1015f11c     kernel32:KERNEL32.dll
 0004:00000120       __imp__CompareStringW@24   1015f120     kernel32:KERNEL32.dll
 0004:00000124       __imp__LCMapStringW@24     1015f124     kernel32:KERNEL32.dll
 0004:00000128       __imp__GetLocaleInfoW@16   1015f128     kernel32:KERNEL32.dll
 0004:0000012c       __imp__IsValidLocale@8     1015f12c     kernel32:KERNEL32.dll
 0004:00000130       __imp__GetUserDefaultLCID@0 1015f130     kernel32:KERNEL32.dll
 0004:00000134       __imp__EnumSystemLocalesW@8 1015f134     kernel32:KERNEL32.dll
 0004:00000138       __imp__GetStringTypeW@16   1015f138     kernel32:KERNEL32.dll
 0004:0000013c       __imp__SetStdHandle@8      1015f13c     kernel32:KERNEL32.dll
 0004:00000140       __imp__CreateFileW@28      1015f140     kernel32:KERNEL32.dll
 0004:00000144       __imp__SetEndOfFile@4      1015f144     kernel32:KERNEL32.dll
 0004:00000148       __imp__FindFirstFileA@8    1015f148     kernel32:KERNEL32.dll
 0004:0000014c       __imp__FindNextFileA@8     1015f14c     kernel32:KERNEL32.dll
 0004:00000150       __imp__ReleaseSemaphore@12 1015f150     kernel32:KERNEL32.dll
 0004:00000154       __imp__ReleaseMutex@4      1015f154     kernel32:KERNEL32.dll
 0004:00000158       __imp__CreateMutexA@12     1015f158     kernel32:KERNEL32.dll
 0004:0000015c       __imp__CreateThread@24     1015f15c     kernel32:KERNEL32.dll
 0004:00000160       __imp__TerminateThread@8   1015f160     kernel32:KERNEL32.dll
 0004:00000164       __imp__CreateSemaphoreA@16 1015f164     kernel32:KERNEL32.dll
 0004:00000168       __imp__GetTimeZoneInformation@4 1015f168     kernel32:KERNEL32.dll
 0004:0000016c       __imp__GetFileAttributesExW@12 1015f16c     kernel32:KERNEL32.dll
 0004:00000170       __imp__SetEnvironmentVariableA@8 1015f170     kernel32:KERNEL32.dll
 0004:00000174       \177KERNEL32_NULL_THUNK_DATA 1015f174     kernel32:KERNEL32.dll
 0004:000001e8       __IMPORT_DESCRIPTOR_KERNEL32 1015f1e8     kernel32:KERNEL32.dll
 0004:000001fc       __NULL_IMPORT_DESCRIPTOR   1015f1fc     kernel32:KERNEL32.dll

 entry point at        0001:0007ad1f

